 RILGOBI

 Timestamp is 548ff4da (Tue Dec 16 17:01:14 2014)

 Preferred load address is 00100000

 Start         Length     Name                   Class
 0001:00000000 0003f49cH .text                   CODE
 0001:0003f49c 0000007cH .text$yc                CODE
 0001:0003f518 00000060H .text$yd                CODE
 0002:00000000 000233ecH .rdata                  DATA
 0002:000233ec 0000016cH .rdata$r                DATA
 0002:00023558 0000018cH .xdata                  DATA
 0002:000236e4 000000e8H .xdata$x                DATA
 0002:000237cc 00000078H .idata$2                DATA
 0002:00023844 00000014H .idata$3                DATA
 0002:00023858 0000039cH .idata$4                DATA
 0002:00023bf4 00000fb2H .idata$6                DATA
 0002:00024bb0 00000103H .edata                  DATA
 0003:00000000 0000039cH .idata$5                DATA
 0003:0000039c 00000004H .CRT$XCA                DATA
 0003:000003a0 00000004H .CRT$XCAA               DATA
 0003:000003a4 0000000cH .CRT$XCU                DATA
 0003:000003b0 00000004H .CRT$XCZ                DATA
 0003:000003b4 00000004H .CRT$XIA                DATA
 0003:000003b8 00000004H .CRT$XIZ                DATA
 0003:000003bc 00000004H .CRT$XPA                DATA
 0003:000003c0 00000004H .CRT$XPZ                DATA
 0003:000003c4 00000004H .CRT$XTA                DATA
 0003:000003c8 00000004H .CRT$XTZ                DATA
 0003:000003d0 00009720H .data                   DATA
 0003:00009af0 000001a0H .bss                    DATA
 0004:00000000 00001bb8H .pdata                  DATA
 0005:00000000 000000a0H .rsrc$01                DATA
 0005:000000a0 000003f8H .rsrc$02                DATA

  Address         Publics by Value              Rva+Base       Lib:Object

 0000:00000000       ___safe_se_handler_count   00000000     <absolute>
 0000:00000000       ___safe_se_handler_table   00000000     <absolute>
 0001:00000000       ??1SYNCBLOCK_Implementation@@QAA@XZ 00101000 f i atcmd.obj
 0001:00000008       ??1bad_alloc@std@@UAA@XZ   00101008 f i atcmd.obj
 0001:0000001c       ??_Gbad_alloc@std@@UAAPAXI@Z 0010101c f i atcmd.obj
 0001:0000001c       ??_Ebad_alloc@std@@UAAPAXI@Z 0010101c f i atcmd.obj
 0001:0000004c       ?GetDevice@CRilInstanceHandle@@QBAPAVCRilHandle@@XZ 0010104c f i atcmd.obj
 0001:000000e4       ?GetCmdList@CRilInstanceHandle@@QBAPAV?$CDblList@VCCommand@@@@XZ 001010e4 f i atcmd.obj
 0001:00000144       ?ReadThreadProc@@YAKPAX@Z  00101144 f   atcmd.obj
 0001:00000264       ?_Inside@?$basic_string@DU?$char_traits@D@std@@V?$allocator@D@2@@std@@IAA_NPBD@Z 00101264 f i atcmd.obj
 0001:000002a4       ?Add@?$CDblList@VCCommand@@@@QAAHQAVCCommand@@@Z 001012a4 f i atcmd.obj
 0001:000002f4       ?Remove@?$CDblList@VCCommand@@@@QAAHQBVCCommand@@@Z 001012f4 f i atcmd.obj
 0001:00000368       ??$_Allocate@D@std@@YAPADIPAD@Z 00101368 f i atcmd.obj
 0001:000003d4       ??0bad_alloc@std@@QAA@ABV01@@Z 001013d4 f i atcmd.obj
 0001:000003f4       ??D?$_Deque_const_iterator@PAVCCommand@@V?$allocator@PAVCCommand@@@std@@$00@std@@QBAABQAVCCommand@@XZ 001013f4 f i atcmd.obj
 0001:00000450       ??$_Allocate@PAVCCommand@@@std@@YAPAPAVCCommand@@IPAPAV1@@Z 00101450 f i atcmd.obj
 0001:000004bc       ??$_Allocate@PAPAVCCommand@@@std@@YAPAPAPAVCCommand@@IPAPAPAV1@@Z 001014bc f i atcmd.obj
 0001:00000528       ??0?$_Deque_const_iterator@PAVCCommand@@V?$allocator@PAVCCommand@@@std@@$00@std@@QAA@IPBU_Container_base@1@@Z 00101528 f i atcmd.obj
 0001:00000574       ?_Tidy@?$basic_string@DU?$char_traits@D@std@@V?$allocator@D@2@@std@@IAAX_NI@Z 00101574 f i atcmd.obj
 0001:000005d4       ?erase@?$basic_string@DU?$char_traits@D@std@@V?$allocator@D@2@@std@@QAAAAV12@II@Z 001015d4 f i atcmd.obj
 0001:00000670       ?_Copy@?$basic_string@DU?$char_traits@D@std@@V?$allocator@D@2@@std@@IAAXII@Z 00101670 f i atcmd.obj
 0001:000007b8       ?pop_front@?$deque@PAVCCommand@@V?$allocator@PAVCCommand@@@std@@@std@@QAAXXZ 001017b8 f i atcmd.obj
 0001:00000800       ??1?$basic_string@DU?$char_traits@D@std@@V?$allocator@D@2@@std@@QAA@XZ 00101800 f i atcmd.obj
 0001:0000080c       ?_Grow@?$basic_string@DU?$char_traits@D@std@@V?$allocator@D@2@@std@@IAA_NI_N@Z 0010180c f i atcmd.obj
 0001:000008b0       ?what@logic_error@std@@UBAPBDXZ 001018b0 f i atcmd.obj
 0001:000008c8       ??_Glogic_error@std@@UAAPAXI@Z 001018c8 f i atcmd.obj
 0001:000008c8       ??_Elogic_error@std@@UAAPAXI@Z 001018c8 f i atcmd.obj
 0001:00000908       ?assign@?$basic_string@DU?$char_traits@D@std@@V?$allocator@D@2@@std@@QAAAAV12@ABV12@II@Z 00101908 f i atcmd.obj
 0001:000009cc       ?assign@?$basic_string@DU?$char_traits@D@std@@V?$allocator@D@2@@std@@QAAAAV12@PBDI@Z 001019cc f i atcmd.obj
 0001:00000a74       ??0logic_error@std@@QAA@ABV?$basic_string@DU?$char_traits@D@std@@V?$allocator@D@2@@1@@Z 00101a74 f i atcmd.obj
 0001:00000aec       ??1length_error@std@@UAA@XZ 00101aec f i atcmd.obj
 0001:00000b18       ??_Glength_error@std@@UAAPAXI@Z 00101b18 f i atcmd.obj
 0001:00000b18       ??_Elength_error@std@@UAAPAXI@Z 00101b18 f i atcmd.obj
 0001:00000b58       ??0?$basic_string@DU?$char_traits@D@std@@V?$allocator@D@2@@std@@QAA@PBD@Z 00101b58 f i atcmd.obj
 0001:00000b90       ?Pop_Front@?$CThreadSafeQueue@PAVCCommand@@@@QAAPAVCCommand@@XZ 00101b90 f i atcmd.obj
 0001:00000c28       ?_Xlen@?$deque@PAVCCommand@@V?$allocator@PAVCCommand@@@std@@@std@@KAXXZ 00101c28 f i atcmd.obj
 0001:00000c9c       ??0logic_error@std@@QAA@ABV01@@Z 00101c9c f i atcmd.obj
 0001:00000d14       ??0length_error@std@@QAA@ABV01@@Z 00101d14 f i atcmd.obj
 0001:00000d34       ?CommandThread@CRilHandle@@QAAKXZ 00101d34 f   atcmd.obj
 0001:00000eec       ?_Growmap@?$deque@PAVCCommand@@V?$allocator@PAVCCommand@@@std@@@std@@IAAXI@Z 00101eec f i atcmd.obj
 0001:00001078       ?CmdThreadProc@@YAKPAX@Z   00102078 f   atcmd.obj
 0001:00001150       ?push_back@?$deque@PAVCCommand@@V?$allocator@PAVCCommand@@@std@@@std@@QAAXABQAVCCommand@@@Z 00102150 f i atcmd.obj
 0001:000011f0       ?Push_Back@?$CThreadSafeQueue@PAVCCommand@@@@QAAXABQAVCCommand@@@Z 001021f0 f i atcmd.obj
 0001:0000123c       ?QueueCmdWithTimeout@@YAHQAVCRilInstanceHandle@@KW4APIID@@PAXAAJKK@Z 0010223c f   atcmd.obj
 0001:000015b4       ?QueueCmd@@YAHQAVCRilInstanceHandle@@KW4APIID@@PAXAAJK@Z 001025b4 f   atcmd.obj
 0001:000015e0       ?GetRadioHandle@CRilHandle@@QAAPAVCRadio@@XZ 001025e0 f i callctrl.obj
 0001:00001630       ?Wait4ATConnectThreadProc@@YAKPAX@Z 00102630 f   callctrl.obj
 0001:00001640       ?ConvertToRILDisconnectCode@@YAKW4SWI_TYPE_EndReason@@@Z 00102640 f   callctrl.obj
 0001:000016d0       ?RILDrv_Answer@@YAJK@Z     001026d0 f   callctrl.obj
 0001:00001730       ?RILDrv_DataDormant@@YAJK@Z 00102730 f   callctrl.obj
 0001:00001798       ?RILDrv_SendDTMF@@YAJKPBDK@Z 00102798 f   callctrl.obj
 0001:00001984       ?RILDrv_GetCallList@@YAJK@Z 00102984 f   callctrl.obj
 0001:00001a2c       ?RILDrv_ManageCalls@@YAJKKK@Z 00102a2c f   callctrl.obj
 0001:00001b28       ?RILDrv_GetLineStatus@@YAJK@Z 00102b28 f   callctrl.obj
 0001:00001bc8       ?RILDrv_GetCurrentPrivacyStatus@@YAJK@Z 00102bc8 f   callctrl.obj
 0001:00001c28       ?RILDrv_SendAKey@@YAJKPBD@Z 00102c28 f   callctrl.obj
 0001:00001d20       ?RILDrv_SendFlash@@YAJKPAUriladdress_tag@@@Z 00102d20 f   callctrl.obj
 0001:00001ed0       ?FillCallInfoStruct@@YAXPAUrilcallinfo_tag@@KKKPAGK@Z 00102ed0 f   callctrl.obj
 0001:00001fc0       ?GetLineStatus@CRadio@@QAAJPAVCResponse@@@Z 00102fc0 f   callctrl.obj
 0001:00002114       ?ReadCurrentPrivacyStatus@CRadio@@QAAJXZ 00103114 f   callctrl.obj
 0001:0000215c       ?GetCurrentPrivacyStatus@CRadio@@QAAJPAVCResponse@@@Z 0010315c f   callctrl.obj
 0001:000021c4       ?SendAKey@CRadio@@QAAJPAVCResponse@@PAX@Z 001031c4 f   callctrl.obj
 0001:00002298       ?SetCurrentAddressId@CRadio@@QAAJPAVCResponse@@PAX@Z 00103298 f   callctrl.obj
 0001:0000245c       ?GetCurrentAddressId@CRadio@@QAAJPAVCResponse@@@Z 0010345c f   callctrl.obj
 0001:000024fc       ?RILDrv_SetBearerServiceOptions@@YAJKPBUrilbearersvcinfo_tag@@@Z 001034fc f   callctrl.obj
 0001:000025cc       ?SetBearerServiceInfo@CRadio@@QAAJPAVCResponse@@PAX@Z 001035cc f   callctrl.obj
 0001:00002610       ?FillRemotePartyInfo@@YAXPAUrilremotepartyinfo_tag@@PBUriladdress_tag@@@Z 00103610 f   callctrl.obj
 0001:00002734       ?BroadcastRemotePartyInfo@CRadio@@QAAXKPBUriladdress_tag@@@Z 00103734 f   callctrl.obj
 0001:00002798       ?LookupCallIdByCallStatus@CRadio@@QAAHKAAK@Z 00103798 f   callctrl.obj
 0001:00002800       ?CallExists@CRadio@@QAAKK@Z 00103800 f   callctrl.obj
 0001:00002898       ?GetNumOfActiveCalls@CRadio@@QAAIXZ 00103898 f   callctrl.obj
 0001:000028d0       ?GetNumOfActiveVoiceCalls@CRadio@@QAAIXZ 001038d0 f   callctrl.obj
 0001:00002908       ?PacketDataCallOnEVDOsystem@CRadio@@QAAHXZ 00103908 f   callctrl.obj
 0001:00002920       ?LookupCallIDByQmiID@CRadio@@QAAHEAAK@Z 00103920 f   callctrl.obj
 0001:00002978       ?SetMultiParty@CRadio@@QAAHKK@Z 00103978 f   callctrl.obj
 0001:00002a00       ?UpdateLineStatus@CRadio@@QAAXXZ 00103a00 f   callctrl.obj
 0001:00002b74       ?GetCallInfo@CRadio@@QAAPBUrilcallinfo_tag@@K@Z 00103b74 f   callctrl.obj
 0001:00002bc0       ?CloseDataPort@CRadio@@QAAHH@Z 00103bc0 f   callctrl.obj
 0001:00002c64       ?HandleSWI_NOTIFY_OTASPState@CRadio@@QAAXPAUSwiNotifyVariant@@@Z 00103c64 f   callctrl.obj
 0001:00002dc8       ?HandleSWI_NOTIFY_USSD@CRadio@@QAAXPAUSwiNotifyVariant@@@Z 00103dc8 f   callctrl.obj
 0001:00003030       ?BroadcastCallStateChangedNotification@CRadio@@QAAXXZ 00104030 f   callctrl.obj
 0001:0000314c       ?PacketDataStatusNotification@CRadio@@QAAXW4SWI_TYPE_CDMA_CallState@@@Z 0010414c f   callctrl.obj
 0001:000031f8       ??E?$_Const_iterator@$00@?$list@UtagEMERGENCY_NUM_INFO@@V?$allocator@UtagEMERGENCY_NUM_INFO@@@std@@@std@@QAAAAV012@XZ 001041f8 f i callctrl.obj
 0001:00003234       ??8?$_Const_iterator@$00@?$list@UtagEMERGENCY_NUM_INFO@@V?$allocator@UtagEMERGENCY_NUM_INFO@@@std@@@std@@QBA_NABV012@@Z 00104234 f i callctrl.obj
 0001:0000327c       ?RILDrv_Hangup@@YAJK@Z     0010427c f   callctrl.obj
 0001:0000330c       ?Answer@CRadio@@QAAJPAVCResponse@@@Z 0010430c f   callctrl.obj
 0001:00003430       ?DataDormant@CRadio@@QAAJPAVCResponse@@@Z 00104430 f   callctrl.obj
 0001:000034a8       ?GetCallList@CRadio@@QAAJPAVCResponse@@@Z 001044a8 f   callctrl.obj
 0001:00003694       ?ManageGSMCall@CRadio@@QAAJPAVCResponse@@PAX@Z 00104694 f   callctrl.obj
 0001:00003db4       ?SendDTMF@CRadio@@QAAJPAVCResponse@@PAX@Z 00104db4 f   callctrl.obj
 0001:000041e0       ?SetCallStatus@CRadio@@QAAHKKKH@Z 001051e0 f   callctrl.obj
 0001:0000432c       ?AddCall@CRadio@@QAAHKEKKKKPAGKK@Z 0010532c f   callctrl.obj
 0001:000045e0       ?RemCall@CRadio@@QAAHK@Z   001055e0 f   callctrl.obj
 0001:000046e4       ?InitiateDataCall@CRadio@@AAAJPAU__Dial_Data@@PAVCResponse@@@Z 001056e4 f   callctrl.obj
 0001:00004bf4       ?HandleSWI_NOTIFY_CallConnecting@CRadio@@QAAXPAUSwiNotifyVariant@@@Z 00105bf4 f   callctrl.obj
 0001:00004e30       ?HandleSWI_NOTIFY_CallConnected@CRadio@@QAAXPAUSwiNotifyVariant@@@Z 00105e30 f   callctrl.obj
 0001:000052a4       ?HandleSWI_NOTIFY_PktSessionCall@CRadio@@QAAXPAUSwiNotifyVariant@@@Z 001062a4 f   callctrl.obj
 0001:00005438       ?DataCallDisconnected@CRadio@@QAAHW4SWI_TYPE_EndReason@@@Z 00106438 f   callctrl.obj
 0001:00005638       ?RILDrv_Dial@@YAJKPBDKK@Z  00106638 f   callctrl.obj
 0001:000059b8       ?HangUp@CRadio@@QAAJPAVCResponse@@@Z 001069b8 f   callctrl.obj
 0001:00005cd8       ?ManageCDMACall@CRadio@@QAAJPAVCResponse@@PAX@Z 00106cd8 f   callctrl.obj
 0001:00005f00       ?SendFlash@CRadio@@QAAJPAVCResponse@@PAX@Z 00106f00 f   callctrl.obj
 0001:0000621c       ?AddNewVoiceCall@CRadio@@QAAHAAKEKKKKPAGKK@Z 0010721c f   callctrl.obj
 0001:000062b4       ?HandleSWI_NOTIFY_CallDisconnected@CRadio@@QAAXPAUSwiNotifyVariant@@@Z 001072b4 f   callctrl.obj
 0001:00006730       ?HandleSWI_NOTIFY_CallIncomming@CRadio@@QAAXPAUSwiNotifyVariant@@@Z 00107730 f   callctrl.obj
 0001:00006f4c       ?HandleSWI_NOTIFY_COLP@CRadio@@QAAXPAUSwiNotifyVariant@@@Z 00107f4c f   callctrl.obj
 0001:0000711c       ?HandleSWI_NOTIFY_CallCallerID@CRadio@@QAAXPAUSwiNotifyVariant@@@Z 0010811c f   callctrl.obj
 0001:000072e4       ?UpdateAndBroadcastOnSWICallNotification@CRadio@@QAAXPAUSwiNotifyVariant@@@Z 001082e4 f   callctrl.obj
 0001:00007588       ?IsEmergencyNumber@CRadio@@AAAHPBG@Z 00108588 f   callctrl.obj
 0001:000076d8       ?GetEmergencyNumberCategory@CRadio@@AAAEPBG@Z 001086d8 f   callctrl.obj
 0001:0000784c       ?Dial@CRadio@@QAAJPAVCResponse@@PAX@Z 0010884c f   callctrl.obj
 0001:000083c8       ?ManageCall@CRadio@@QAAJPAVCResponse@@PAX@Z 001093c8 f   callctrl.obj
 0001:00008454       ?RILDrv_GetDevCaps@@YAJKK@Z 00109454 f   caps.obj
 0001:00008504       ?GetDevCaps@CRadio@@QAAJPAVCResponse@@PAX@Z 00109504 f   caps.obj
 0001:00008794       ??0CChannel@@QAA@PAGJ@Z    00109794 f   channel.obj
 0001:00008844       ?SetupChannel@CChannel@@QAAXXZ 00109844 f   channel.obj
 0001:00008958       ?CloseChannel@CChannel@@QAAXXZ 00109958 f   channel.obj
 0001:000089dc       ?DeviceIOCtrl@CChannel@@QAAHKPAXK0KPAKPAU_OVERLAPPED@@@Z 001099dc f   channel.obj
 0001:00008a50       ?InternalRecv@CChannel@@QAAHPAJPAE@Z 00109a50 f i channel.obj
 0001:00008b84       ??_ECChannel@@UAAPAXI@Z    00109b84 f i channel.obj
 0001:00008b84       ??_GCChannel@@UAAPAXI@Z    00109b84 f i channel.obj
 0001:00008bc8       ?RecvThread@@YAXPAX@Z      00109bc8 f   channel.obj
 0001:00008c78       ?CreateChannel@CChannel@@QAAPAXP6AKKPAE@Z@Z 00109c78 f   channel.obj
 0001:00008da0       ??0CCommand@@QAA@XZ        00109da0 f   command.obj
 0001:00008dcc       ?Init@CCommand@@QAAHQAVCRilInstanceHandle@@KKKPAXW4APIID@@K@Z 00109dcc f   command.obj
 0001:00008ea8       ?IsDataDialCommand@CCommand@@QAAHXZ 00109ea8 f   command.obj
 0001:00008ee4       ??1CCommand@@QAA@XZ        00109ee4 f   command.obj
 0001:00008fa8       ?SendResponse@CCommand@@QBAHKQBXI@Z 00109fa8 f   command.obj
 0001:00009208       ?RILDrv_GetHSCSDCallSettings@@YAJK@Z 0010a208 f   data.obj
 0001:00009268       ?RILDrv_GetBearerServiceOptions@@YAJK@Z 0010a268 f   data.obj
 0001:000092c8       ?RILDrv_GetRLPOptions@@YAJK@Z 0010a2c8 f   data.obj
 0001:00009330       ?RILDrv_SetRLPOptions@@YAJKPBUrilrlpinfo_tag@@@Z 0010a330 f   data.obj
 0001:000098bc       ?RILDrv_GetDataCompression@@YAJK@Z 0010a8bc f   data.obj
 0001:00009924       ?RILDrv_SetDataCompression@@YAJKPBUrildatacompinfo_tag@@@Z 0010a924 f   data.obj
 0001:00009d58       ?RILDrv_GetErrorCorrection@@YAJK@Z 0010ad58 f   data.obj
 0001:00009dc0       ?RILDrv_SetErrorCorrection@@YAJKPBUrilerrorcorrectioninfo_tag@@@Z 0010adc0 f   data.obj
 0001:0000a140       ?ParseString@CDatERI@@IAAXPAEG_NPAG@Z 0010b140 f   DatERI.obj
 0001:0000a1bc       ?GetVersion@CDatERI@@QAAGXZ 0010b1bc f   DatERI.obj
 0001:0000a1c4       ?CalcCRC16@CDatERI@@IAAGPAEG@Z 0010b1c4 f   DatERI.obj
 0001:0000a288       ??8const_iterator@?$_Tree@V?$_Tmap_traits@GPAUSWI_STRUCT_RoamInd@CDatERI@@U?$less@G@std@@V?$allocator@U?$pair@$$CBGPAUSWI_STRUCT_RoamInd@CDatERI@@@std@@@4@$0A@@std@@@std@@QBA_NABV012@@Z 0010b288 f i DatERI.obj
 0001:0000a2d0       ??8const_iterator@?$_Tree@V?$_Tmap_traits@GPAUSWI_STRUCT_CallPrompt@CDatERI@@U?$less@G@std@@V?$allocator@U?$pair@$$CBGPAUSWI_STRUCT_CallPrompt@CDatERI@@@std@@@4@$0A@@std@@@std@@QBA_NABV012@@Z 0010b2d0 f i DatERI.obj
 0001:0000a318       ?_Dec@const_iterator@?$_Tree@V?$_Tmap_traits@GPAUSWI_STRUCT_RoamInd@CDatERI@@U?$less@G@std@@V?$allocator@U?$pair@$$CBGPAUSWI_STRUCT_RoamInd@CDatERI@@@std@@@4@$0A@@std@@@std@@QAAXXZ 0010b318 f i DatERI.obj
 0001:0000a3e8       ?_Dec@const_iterator@?$_Tree@V?$_Tmap_traits@GPAUSWI_STRUCT_CallPrompt@CDatERI@@U?$less@G@std@@V?$allocator@U?$pair@$$CBGPAUSWI_STRUCT_CallPrompt@CDatERI@@@std@@@4@$0A@@std@@@std@@QAAXXZ 0010b3e8 f i DatERI.obj
 0001:0000a4b8       ??$_Allocate@U_Node@?$_Tree_nod@V?$_Tmap_traits@GPAUSWI_STRUCT_RoamInd@CDatERI@@U?$less@G@std@@V?$allocator@U?$pair@$$CBGPAUSWI_STRUCT_RoamInd@CDatERI@@@std@@@4@$0A@@std@@@std@@@std@@YAPAU_Node@?$_Tree_nod@V?$_Tmap_traits@GPAUSWI_STRUCT_RoamInd@CDatERI@@U?$less@G@std@@V?$allocator@U?$pair@$$CBGPAUSWI_STRUCT_RoamInd@CDatERI@@@std@@@4@$0A@@std@@@0@IPAU120@@Z 0010b4b8 f i DatERI.obj
 0001:0000a528       ??$_Allocate@U_Node@?$_Tree_nod@V?$_Tmap_traits@GPAUSWI_STRUCT_CallPrompt@CDatERI@@U?$less@G@std@@V?$allocator@U?$pair@$$CBGPAUSWI_STRUCT_CallPrompt@CDatERI@@@std@@@4@$0A@@std@@@std@@@std@@YAPAU_Node@?$_Tree_nod@V?$_Tmap_traits@GPAUSWI_STRUCT_CallPrompt@CDatERI@@U?$less@G@std@@V?$allocator@U?$pair@$$CBGPAUSWI_STRUCT_CallPrompt@CDatERI@@@std@@@4@$0A@@std@@@0@IPAU120@@Z 0010b528 f i DatERI.obj
 0001:0000a598       ?ParseCallPrompt@CDatERI@@IAA_NPAUSWI_STRUCT_CallPrompt@1@PAEGAAG@Z 0010b598 f   DatERI.obj
 0001:0000a67c       ?ParseRoamInd@CDatERI@@IAA_NPAUSWI_STRUCT_RoamInd@1@PAEGAAG@Z 0010b67c f   DatERI.obj
 0001:0000a778       ?_Lbound@?$_Tree@V?$_Tmap_traits@GPAUSWI_STRUCT_RoamInd@CDatERI@@U?$less@G@std@@V?$allocator@U?$pair@$$CBGPAUSWI_STRUCT_RoamInd@CDatERI@@@std@@@4@$0A@@std@@@std@@IBAPAU_Node@?$_Tree_nod@V?$_Tmap_traits@GPAUSWI_STRUCT_RoamInd@CDatERI@@U?$less@G@std@@V?$allocator@U?$pair@$$CBGPAUSWI_STRUCT_RoamInd@CDatERI@@@std@@@4@$0A@@std@@@2@ABG@Z 0010b778 f i DatERI.obj
 0001:0000a7d0       ?_Lbound@?$_Tree@V?$_Tmap_traits@GPAUSWI_STRUCT_CallPrompt@CDatERI@@U?$less@G@std@@V?$allocator@U?$pair@$$CBGPAUSWI_STRUCT_CallPrompt@CDatERI@@@std@@@4@$0A@@std@@@std@@IBAPAU_Node@?$_Tree_nod@V?$_Tmap_traits@GPAUSWI_STRUCT_CallPrompt@CDatERI@@U?$less@G@std@@V?$allocator@U?$pair@$$CBGPAUSWI_STRUCT_CallPrompt@CDatERI@@@std@@@4@$0A@@std@@@2@ABG@Z 0010b7d0 f i DatERI.obj
 0001:0000a828       ?_Lrotate@?$_Tree@V?$_Tmap_traits@GPAUSWI_STRUCT_RoamInd@CDatERI@@U?$less@G@std@@V?$allocator@U?$pair@$$CBGPAUSWI_STRUCT_RoamInd@CDatERI@@@std@@@4@$0A@@std@@@std@@IAAXPAU_Node@?$_Tree_nod@V?$_Tmap_traits@GPAUSWI_STRUCT_RoamInd@CDatERI@@U?$less@G@std@@V?$allocator@U?$pair@$$CBGPAUSWI_STRUCT_RoamInd@CDatERI@@@std@@@4@$0A@@std@@@2@@Z 0010b828 f i DatERI.obj
 0001:0000a890       ?_Rrotate@?$_Tree@V?$_Tmap_traits@GPAUSWI_STRUCT_RoamInd@CDatERI@@U?$less@G@std@@V?$allocator@U?$pair@$$CBGPAUSWI_STRUCT_RoamInd@CDatERI@@@std@@@4@$0A@@std@@@std@@IAAXPAU_Node@?$_Tree_nod@V?$_Tmap_traits@GPAUSWI_STRUCT_RoamInd@CDatERI@@U?$less@G@std@@V?$allocator@U?$pair@$$CBGPAUSWI_STRUCT_RoamInd@CDatERI@@@std@@@4@$0A@@std@@@2@@Z 0010b890 f i DatERI.obj
 0001:0000a900       ?_Lrotate@?$_Tree@V?$_Tmap_traits@GPAUSWI_STRUCT_CallPrompt@CDatERI@@U?$less@G@std@@V?$allocator@U?$pair@$$CBGPAUSWI_STRUCT_CallPrompt@CDatERI@@@std@@@4@$0A@@std@@@std@@IAAXPAU_Node@?$_Tree_nod@V?$_Tmap_traits@GPAUSWI_STRUCT_CallPrompt@CDatERI@@U?$less@G@std@@V?$allocator@U?$pair@$$CBGPAUSWI_STRUCT_CallPrompt@CDatERI@@@std@@@4@$0A@@std@@@2@@Z 0010b900 f i DatERI.obj
 0001:0000a968       ?_Rrotate@?$_Tree@V?$_Tmap_traits@GPAUSWI_STRUCT_CallPrompt@CDatERI@@U?$less@G@std@@V?$allocator@U?$pair@$$CBGPAUSWI_STRUCT_CallPrompt@CDatERI@@@std@@@4@$0A@@std@@@std@@IAAXPAU_Node@?$_Tree_nod@V?$_Tmap_traits@GPAUSWI_STRUCT_CallPrompt@CDatERI@@U?$less@G@std@@V?$allocator@U?$pair@$$CBGPAUSWI_STRUCT_CallPrompt@CDatERI@@@std@@@4@$0A@@std@@@2@@Z 0010b968 f i DatERI.obj
 0001:0000a9d8       ?_Inc@const_iterator@?$_Tree@V?$_Tmap_traits@GPAUSWI_STRUCT_RoamInd@CDatERI@@U?$less@G@std@@V?$allocator@U?$pair@$$CBGPAUSWI_STRUCT_RoamInd@CDatERI@@@std@@@4@$0A@@std@@@std@@QAAXXZ 0010b9d8 f i DatERI.obj
 0001:0000aa74       ?_Inc@const_iterator@?$_Tree@V?$_Tmap_traits@GPAUSWI_STRUCT_CallPrompt@CDatERI@@U?$less@G@std@@V?$allocator@U?$pair@$$CBGPAUSWI_STRUCT_CallPrompt@CDatERI@@@std@@@4@$0A@@std@@@std@@QAAXXZ 0010ba74 f i DatERI.obj
 0001:0000ab10       ?_Erase@?$_Tree@V?$_Tmap_traits@GPAUSWI_STRUCT_RoamInd@CDatERI@@U?$less@G@std@@V?$allocator@U?$pair@$$CBGPAUSWI_STRUCT_RoamInd@CDatERI@@@std@@@4@$0A@@std@@@std@@IAAXPAU_Node@?$_Tree_nod@V?$_Tmap_traits@GPAUSWI_STRUCT_RoamInd@CDatERI@@U?$less@G@std@@V?$allocator@U?$pair@$$CBGPAUSWI_STRUCT_RoamInd@CDatERI@@@std@@@4@$0A@@std@@@2@@Z 0010bb10 f i DatERI.obj
 0001:0000ab58       ?_Erase@?$_Tree@V?$_Tmap_traits@GPAUSWI_STRUCT_CallPrompt@CDatERI@@U?$less@G@std@@V?$allocator@U?$pair@$$CBGPAUSWI_STRUCT_CallPrompt@CDatERI@@@std@@@4@$0A@@std@@@std@@IAAXPAU_Node@?$_Tree_nod@V?$_Tmap_traits@GPAUSWI_STRUCT_CallPrompt@CDatERI@@U?$less@G@std@@V?$allocator@U?$pair@$$CBGPAUSWI_STRUCT_CallPrompt@CDatERI@@@std@@@4@$0A@@std@@@2@@Z 0010bb58 f i DatERI.obj
 0001:0000aba0       ?_Buynode@?$_Tree@V?$_Tmap_traits@GPAUSWI_STRUCT_RoamInd@CDatERI@@U?$less@G@std@@V?$allocator@U?$pair@$$CBGPAUSWI_STRUCT_RoamInd@CDatERI@@@std@@@4@$0A@@std@@@std@@IAAPAU_Node@?$_Tree_nod@V?$_Tmap_traits@GPAUSWI_STRUCT_RoamInd@CDatERI@@U?$less@G@std@@V?$allocator@U?$pair@$$CBGPAUSWI_STRUCT_RoamInd@CDatERI@@@std@@@4@$0A@@std@@@2@XZ 0010bba0 f i DatERI.obj
 0001:0000abdc       ?_Buynode@?$_Tree@V?$_Tmap_traits@GPAUSWI_STRUCT_RoamInd@CDatERI@@U?$less@G@std@@V?$allocator@U?$pair@$$CBGPAUSWI_STRUCT_RoamInd@CDatERI@@@std@@@4@$0A@@std@@@std@@IAAPAU_Node@?$_Tree_nod@V?$_Tmap_traits@GPAUSWI_STRUCT_RoamInd@CDatERI@@U?$less@G@std@@V?$allocator@U?$pair@$$CBGPAUSWI_STRUCT_RoamInd@CDatERI@@@std@@@4@$0A@@std@@@2@PAU342@00ABU?$pair@$$CBGPAUSWI_STRUCT_RoamInd@CDatERI@@@2@D@Z 0010bbdc f i DatERI.obj
 0001:0000ac34       ?_Buynode@?$_Tree@V?$_Tmap_traits@GPAUSWI_STRUCT_CallPrompt@CDatERI@@U?$less@G@std@@V?$allocator@U?$pair@$$CBGPAUSWI_STRUCT_CallPrompt@CDatERI@@@std@@@4@$0A@@std@@@std@@IAAPAU_Node@?$_Tree_nod@V?$_Tmap_traits@GPAUSWI_STRUCT_CallPrompt@CDatERI@@U?$less@G@std@@V?$allocator@U?$pair@$$CBGPAUSWI_STRUCT_CallPrompt@CDatERI@@@std@@@4@$0A@@std@@@2@XZ 0010bc34 f i DatERI.obj
 0001:0000ac70       ?_Buynode@?$_Tree@V?$_Tmap_traits@GPAUSWI_STRUCT_CallPrompt@CDatERI@@U?$less@G@std@@V?$allocator@U?$pair@$$CBGPAUSWI_STRUCT_CallPrompt@CDatERI@@@std@@@4@$0A@@std@@@std@@IAAPAU_Node@?$_Tree_nod@V?$_Tmap_traits@GPAUSWI_STRUCT_CallPrompt@CDatERI@@U?$less@G@std@@V?$allocator@U?$pair@$$CBGPAUSWI_STRUCT_CallPrompt@CDatERI@@@std@@@4@$0A@@std@@@2@PAU342@00ABU?$pair@$$CBGPAUSWI_STRUCT_CallPrompt@CDatERI@@@2@D@Z 0010bc70 f i DatERI.obj
 0001:0000acc8       ?_Init@?$_Tree@V?$_Tmap_traits@GPAUSWI_STRUCT_RoamInd@CDatERI@@U?$less@G@std@@V?$allocator@U?$pair@$$CBGPAUSWI_STRUCT_RoamInd@CDatERI@@@std@@@4@$0A@@std@@@std@@IAAXXZ 0010bcc8 f i DatERI.obj
 0001:0000ad04       ?_Init@?$_Tree@V?$_Tmap_traits@GPAUSWI_STRUCT_CallPrompt@CDatERI@@U?$less@G@std@@V?$allocator@U?$pair@$$CBGPAUSWI_STRUCT_CallPrompt@CDatERI@@@std@@@4@$0A@@std@@@std@@IAAXXZ 0010bd04 f i DatERI.obj
 0001:0000ad40       ?find@?$_Tree@V?$_Tmap_traits@GPAUSWI_STRUCT_RoamInd@CDatERI@@U?$less@G@std@@V?$allocator@U?$pair@$$CBGPAUSWI_STRUCT_RoamInd@CDatERI@@@std@@@4@$0A@@std@@@std@@QAA?AViterator@12@ABG@Z 0010bd40 f i DatERI.obj
 0001:0000addc       ?Reset@CDatERI@@QAAXXZ     0010bddc f   DatERI.obj
 0001:0000af64       ?GetRoamDetails@CDatERI@@QAA_NHAAUSWI_STRUCT_ERI@@@Z 0010bf64 f   DatERI.obj
 0001:0000b05c       ??1out_of_range@std@@UAA@XZ 0010c05c f i DatERI.obj
 0001:0000b088       ??_Gout_of_range@std@@UAAPAXI@Z 0010c088 f i DatERI.obj
 0001:0000b088       ??_Eout_of_range@std@@UAAPAXI@Z 0010c088 f i DatERI.obj
 0001:0000b0d0       ?erase@?$_Tree@V?$_Tmap_traits@GPAUSWI_STRUCT_RoamInd@CDatERI@@U?$less@G@std@@V?$allocator@U?$pair@$$CBGPAUSWI_STRUCT_RoamInd@CDatERI@@@std@@@4@$0A@@std@@@std@@QAA?AViterator@12@V312@@Z 0010c0d0 f i DatERI.obj
 0001:0000b53c       ??0out_of_range@std@@QAA@ABV01@@Z 0010c53c f i DatERI.obj
 0001:0000b564       ?erase@?$_Tree@V?$_Tmap_traits@GPAUSWI_STRUCT_CallPrompt@CDatERI@@U?$less@G@std@@V?$allocator@U?$pair@$$CBGPAUSWI_STRUCT_CallPrompt@CDatERI@@@std@@@4@$0A@@std@@@std@@QAA?AViterator@12@V312@@Z 0010c564 f i DatERI.obj
 0001:0000b9d0       ?erase@?$_Tree@V?$_Tmap_traits@GPAUSWI_STRUCT_RoamInd@CDatERI@@U?$less@G@std@@V?$allocator@U?$pair@$$CBGPAUSWI_STRUCT_RoamInd@CDatERI@@@std@@@4@$0A@@std@@@std@@QAA?AViterator@12@V312@0@Z 0010c9d0 f i DatERI.obj
 0001:0000bae4       ?_Insert@?$_Tree@V?$_Tmap_traits@GPAUSWI_STRUCT_RoamInd@CDatERI@@U?$less@G@std@@V?$allocator@U?$pair@$$CBGPAUSWI_STRUCT_RoamInd@CDatERI@@@std@@@4@$0A@@std@@@std@@IAA?AViterator@12@_NPAU_Node@?$_Tree_nod@V?$_Tmap_traits@GPAUSWI_STRUCT_RoamInd@CDatERI@@U?$less@G@std@@V?$allocator@U?$pair@$$CBGPAUSWI_STRUCT_RoamInd@CDatERI@@@std@@@4@$0A@@std@@@2@ABU?$pair@$$CBGPAUSWI_STRUCT_RoamInd@CDatERI@@@2@@Z 0010cae4 f i DatERI.obj
 0001:0000bd30       ?erase@?$_Tree@V?$_Tmap_traits@GPAUSWI_STRUCT_CallPrompt@CDatERI@@U?$less@G@std@@V?$allocator@U?$pair@$$CBGPAUSWI_STRUCT_CallPrompt@CDatERI@@@std@@@4@$0A@@std@@@std@@QAA?AViterator@12@V312@0@Z 0010cd30 f i DatERI.obj
 0001:0000be44       ?_Insert@?$_Tree@V?$_Tmap_traits@GPAUSWI_STRUCT_CallPrompt@CDatERI@@U?$less@G@std@@V?$allocator@U?$pair@$$CBGPAUSWI_STRUCT_CallPrompt@CDatERI@@@std@@@4@$0A@@std@@@std@@IAA?AViterator@12@_NPAU_Node@?$_Tree_nod@V?$_Tmap_traits@GPAUSWI_STRUCT_CallPrompt@CDatERI@@U?$less@G@std@@V?$allocator@U?$pair@$$CBGPAUSWI_STRUCT_CallPrompt@CDatERI@@@std@@@4@$0A@@std@@@2@ABU?$pair@$$CBGPAUSWI_STRUCT_CallPrompt@CDatERI@@@2@@Z 0010ce44 f i DatERI.obj
 0001:0000c090       ?_Tidy@?$_Tree@V?$_Tmap_traits@GPAUSWI_STRUCT_RoamInd@CDatERI@@U?$less@G@std@@V?$allocator@U?$pair@$$CBGPAUSWI_STRUCT_RoamInd@CDatERI@@@std@@@4@$0A@@std@@@std@@IAAXXZ 0010d090 f i DatERI.obj
 0001:0000c0d4       ?_Tidy@?$_Tree@V?$_Tmap_traits@GPAUSWI_STRUCT_CallPrompt@CDatERI@@U?$less@G@std@@V?$allocator@U?$pair@$$CBGPAUSWI_STRUCT_CallPrompt@CDatERI@@@std@@@4@$0A@@std@@@std@@IAAXXZ 0010d0d4 f i DatERI.obj
 0001:0000c118       ?insert@?$_Tree@V?$_Tmap_traits@GPAUSWI_STRUCT_RoamInd@CDatERI@@U?$less@G@std@@V?$allocator@U?$pair@$$CBGPAUSWI_STRUCT_RoamInd@CDatERI@@@std@@@4@$0A@@std@@@std@@QAA?AU?$pair@Viterator@?$_Tree@V?$_Tmap_traits@GPAUSWI_STRUCT_RoamInd@CDatERI@@U?$less@G@std@@V?$allocator@U?$pair@$$CBGPAUSWI_STRUCT_RoamInd@CDatERI@@@std@@@4@$0A@@std@@@std@@_N@2@ABU?$pair@$$CBGPAUSWI_STRUCT_RoamInd@CDatERI@@@2@@Z 0010d118 f i DatERI.obj
 0001:0000c250       ?insert@?$_Tree@V?$_Tmap_traits@GPAUSWI_STRUCT_CallPrompt@CDatERI@@U?$less@G@std@@V?$allocator@U?$pair@$$CBGPAUSWI_STRUCT_CallPrompt@CDatERI@@@std@@@4@$0A@@std@@@std@@QAA?AU?$pair@Viterator@?$_Tree@V?$_Tmap_traits@GPAUSWI_STRUCT_CallPrompt@CDatERI@@U?$less@G@std@@V?$allocator@U?$pair@$$CBGPAUSWI_STRUCT_CallPrompt@CDatERI@@@std@@@4@$0A@@std@@@std@@_N@2@ABU?$pair@$$CBGPAUSWI_STRUCT_CallPrompt@CDatERI@@@2@@Z 0010d250 f i DatERI.obj
 0001:0000c388       ?insert@?$_Tree@V?$_Tmap_traits@GPAUSWI_STRUCT_RoamInd@CDatERI@@U?$less@G@std@@V?$allocator@U?$pair@$$CBGPAUSWI_STRUCT_RoamInd@CDatERI@@@std@@@4@$0A@@std@@@std@@QAA?AViterator@12@V312@ABU?$pair@$$CBGPAUSWI_STRUCT_RoamInd@CDatERI@@@2@@Z 0010d388 f i DatERI.obj
 0001:0000c600       ?insert@?$_Tree@V?$_Tmap_traits@GPAUSWI_STRUCT_CallPrompt@CDatERI@@U?$less@G@std@@V?$allocator@U?$pair@$$CBGPAUSWI_STRUCT_CallPrompt@CDatERI@@@std@@@4@$0A@@std@@@std@@QAA?AViterator@12@V312@ABU?$pair@$$CBGPAUSWI_STRUCT_CallPrompt@CDatERI@@@2@@Z 0010d600 f i DatERI.obj
 0001:0000c878       ??1?$map@GPAUSWI_STRUCT_RoamInd@CDatERI@@U?$less@G@std@@V?$allocator@U?$pair@$$CBGPAUSWI_STRUCT_RoamInd@CDatERI@@@std@@@4@@std@@QAA@XZ 0010d878 f i DatERI.obj
 0001:0000c87c       ??1?$map@GPAUSWI_STRUCT_CallPrompt@CDatERI@@U?$less@G@std@@V?$allocator@U?$pair@$$CBGPAUSWI_STRUCT_CallPrompt@CDatERI@@@std@@@4@@std@@QAA@XZ 0010d87c f i DatERI.obj
 0001:0000c888       ??1CDatERI@@QAA@XZ         0010d888 f   DatERI.obj
 0001:0000c8f4       ??A?$map@GPAUSWI_STRUCT_RoamInd@CDatERI@@U?$less@G@std@@V?$allocator@U?$pair@$$CBGPAUSWI_STRUCT_RoamInd@CDatERI@@@std@@@4@@std@@QAAAAPAUSWI_STRUCT_RoamInd@CDatERI@@ABG@Z 0010d8f4 f i DatERI.obj
 0001:0000c9ac       ??A?$map@GPAUSWI_STRUCT_CallPrompt@CDatERI@@U?$less@G@std@@V?$allocator@U?$pair@$$CBGPAUSWI_STRUCT_CallPrompt@CDatERI@@@std@@@4@@std@@QAAAAPAUSWI_STRUCT_CallPrompt@CDatERI@@ABG@Z 0010d9ac f i DatERI.obj
 0001:0000ca6c       ??0CDatERI@@QAA@XZ         0010da6c f   DatERI.obj
 0001:0000cb3c       ?Load@CDatERI@@QAAHPAEG@Z  0010db3c f   DatERI.obj
 0001:0000cde4       ?EnableNotifications@CRadio@@QAAX_N@Z 0010dde4 f   FakeResponse.obj
 0001:0000d990       ?EnableTechHDRNotifications@CRadio@@QAAX_N@Z 0010e990 f   FakeResponse.obj
 0001:0000d9d0       ??$_Allocate@U_Node@?$_List_nod@PAVCCommand@@V?$allocator@PAVCCommand@@@std@@@std@@@std@@YAPAU_Node@?$_List_nod@PAVCCommand@@V?$allocator@PAVCCommand@@@std@@@0@IPAU120@@Z 0010e9d0 f i FakeResponse.obj
 0001:0000da40       ??D?$_Deque_const_iterator@PAUSwiNotifyVariant@@V?$allocator@PAUSwiNotifyVariant@@@std@@$00@std@@QBAABQAUSwiNotifyVariant@@XZ 0010ea40 f i FakeResponse.obj
 0001:0000da9c       ??1CSafeEntry@@QAA@XZ      0010ea9c f i FakeResponse.obj
 0001:0000dabc       ?InitThreadProc@@YAKPAX@Z  0010eabc f   FakeResponse.obj
 0001:0000dcf8       ?HandleRsp@CRilHandle@@QAAHAAPAVCCommand@@AAPAVCResponse@@@Z 0010ecf8 f   FakeResponse.obj
 0001:0000de28       ??0?$_Deque_const_iterator@PAUSwiNotifyVariant@@V?$allocator@PAUSwiNotifyVariant@@@std@@$00@std@@QAA@IPBU_Container_base@1@@Z 0010ee28 f i FakeResponse.obj
 0001:0000de74       ?_Buynode@?$list@PAVCCommand@@V?$allocator@PAVCCommand@@@std@@@std@@IAAPAU_Node@?$_List_nod@PAVCCommand@@V?$allocator@PAVCCommand@@@std@@@2@PAU342@0ABQAVCCommand@@@Z 0010ee74 f i FakeResponse.obj
 0001:0000deb0       ?pop_front@?$deque@PAUSwiNotifyVariant@@V?$allocator@PAUSwiNotifyVariant@@@std@@@std@@QAAXXZ 0010eeb0 f i FakeResponse.obj
 0001:0000def8       ?Pop_Front@?$CThreadSafeQueue@PAUSwiNotifyVariant@@@@QAAPAUSwiNotifyVariant@@XZ 0010eef8 f i FakeResponse.obj
 0001:0000df88       ?ResponseThread@CRilHandle@@QAAKXZ 0010ef88 f   FakeResponse.obj
 0001:0000e0bc       ?_Incsize@?$list@PAVCCommand@@V?$allocator@PAVCCommand@@@std@@@std@@IAAXI@Z 0010f0bc f i FakeResponse.obj
 0001:0000e16c       ?QueueCommandForDelayedResponse@CRilHandle@@QAAHPAVCCommand@@PAVCResponse@@@Z 0010f16c f   FakeResponse.obj
 0001:0000e2a8       ?HandleCommand@CRilHandle@@QAAHPAVCCommand@@@Z 0010f2a8 f   FakeResponse.obj
 0001:0000e748       ?RILDrv_GetGPRSContextList@@YAJK@Z 0010f748 f   gprs.obj
 0001:0000e7a8       ?RILDrv_SetGPRSContext@@YAJKPBUrilgprscontext_tag@@@Z 0010f7a8 f   gprs.obj
 0001:0000e810       ?RILDrv_NdisSetGPRSContextActivated@@YAJKPBUrilndisgprscontext_tag@@@Z 0010f810 f   gprs.obj
 0001:0000e858       ?RILDrv_DeleteGPRSContext@@YAJKK@Z 0010f858 f   gprs.obj
 0001:0000e8c4       ?RILDrv_GetRequestedQualityOfServiceList@@YAJK@Z 0010f8c4 f   gprs.obj
 0001:0000e924       ?RILDrv_GetMinimumQualityOfServiceList@@YAJK@Z 0010f924 f   gprs.obj
 0001:0000e98c       ?SetQOS@@YAJKPBUrilgprsqosprofile_tag@@PBDW4APIID@@@Z 0010f98c f   gprs.obj
 0001:0000eee8       ?RILDrv_SetRequestedQualityOfService@@YAJKPBUrilgprsqosprofile_tag@@@Z 0010fee8 f   gprs.obj
 0001:0000eef8       ?RILDrv_SetMinimumQualityOfService@@YAJKPBUrilgprsqosprofile_tag@@@Z 0010fef8 f   gprs.obj
 0001:0000ef10       ?DeleteQOS@@YAJKKPBDW4APIID@@@Z 0010ff10 f   gprs.obj
 0001:0000efb4       ?RILDrv_DeleteRequestedQualityOfService@@YAJKK@Z 0010ffb4 f   gprs.obj
 0001:0000efc4       ?RILDrv_DeleteMinimumQualityOfService@@YAJKK@Z 0010ffc4 f   gprs.obj
 0001:0000efdc       ?RILDrv_SetGPRSAttached@@YAJKH@Z 0010ffdc f   gprs.obj
 0001:0000f07c       ?RILDrv_GetGPRSAttached@@YAJK@Z 0011007c f   gprs.obj
 0001:0000f0dc       ?RILDrv_SetGPRSContextActivated@@YAJKKH@Z 001100dc f   gprs.obj
 0001:0000f188       ?RILDrv_GetGPRSContextActivatedList@@YAJK@Z 00110188 f   gprs.obj
 0001:0000f1f0       ?RILDrv_EnterGPRSDataMode@@YAJKPBUrilentergprsdatamode_tag@@@Z 001101f0 f   gprs.obj
 0001:0000f3e8       ?RILDrv_GetGPRSAddress@@YAJKK@Z 001103e8 f   gprs.obj
 0001:0000f488       ?RILDrv_GPRSAnswer@@YAJKPBUrilgprsanswer_tag@@@Z 00110488 f   gprs.obj
 0001:0000f6bc       ?RILDrv_SendSimCmd@@YAJKPBEK@Z 001106bc f   gprs.obj
 0001:0000f7b4       ?RILDrv_SendRestrictedSimCmd@@YAJKKPBUrilsimcmdparameters_tag@@PBEK@Z 001107b4 f   gprs.obj
 0001:0000f8e0       ?RILDrv_GetSimRecordStatus@@YAJKK@Z 001108e0 f   gprs.obj
 0001:0000f948       ?RILDrv_GetGPRSRegistrationStatus@@YAJK@Z 00110948 f   gprs.obj
 0001:0000f9a8       ?RILDrv_GetGPRSClass@@YAJK@Z 001109a8 f   gprs.obj
 0001:0000fa10       ?RILDrv_SetGPRSClass@@YAJKK@Z 00110a10 f   gprs.obj
 0001:0000fac8       ?RILDrv_GetMOSMSService@@YAJK@Z 00110ac8 f   gprs.obj
 0001:0000fb30       ?RILDrv_SetMOSMSService@@YAJKK@Z 00110b30 f   gprs.obj
 0001:0000fbe8       ?GetGPRSRegistrationStatus@CRadio@@QAAJPAVCResponse@@@Z 00110be8 f   gprs.obj
 0001:0000fc94       ?DeleteGPRSContext@CRadio@@QAAJPAVCResponse@@PAX@Z 00110c94 f   gprs.obj
 0001:0000fce8       ?GetGPRSAttached@CRadio@@QAAJPAVCResponse@@@Z 00110ce8 f   gprs.obj
 0001:0000fd3c       ?SetGPRSContextActivated@CRadio@@QAAJPAVCResponse@@PAX@Z 00110d3c f   gprs.obj
 0001:0000fdec       ?SendSimCmd@CRadio@@QAAJPAVCResponse@@PAX@Z 00110dec f   gprs.obj
 0001:0000ffbc       ?SendRestrictedSimCmd@CRadio@@QAAJPAVCResponse@@PAX@Z 00110fbc f   gprs.obj
 0001:000103e8       ?GetSimRecordStatus@CRadio@@QAAJPAVCResponse@@PAX@Z 001113e8 f   gprs.obj
 0001:00010580       ?GetGPRSContextList@CRadio@@QAAJPAVCResponse@@@Z 00111580 f   gprs.obj
 0001:000107bc       ?GPRSActivate@CRadio@@QAAJKH@Z 001117bc f   gprs.obj
 0001:000108a8       ?SetGPRSContext@CRadio@@QAAJPAVCResponse@@PAX@Z 001118a8 f   gprs.obj
 0001:00010b94       ?RILDrv_HandleSuspend@@YAJKJW4_CEDEVICE_POWER_STATE@@@Z 00111b94 f   misc.obj
 0001:00010c84       ?RILDrv_AuxPowerGet@@YAJKPAW4_CEDEVICE_POWER_STATE@@@Z 00111c84 f   misc.obj
 0001:00010cb0       ?RILDrv_GetEquipmentInfo@@YAJK@Z 00111cb0 f   misc.obj
 0001:00010d10       ?RILDrv_GetEquipmentState@@YAJK@Z 00111d10 f   misc.obj
 0001:00010e30       ?RILDrv_SetEquipmentState@@YAJKK@Z 00111e30 f   misc.obj
 0001:00010f10       ?RILDrv_GetSignalQuality@@YAJK@Z 00111f10 f   misc.obj
 0001:00010f70       ?RILDrv_GetCellTowerInfo@@YAJK@Z 00111f70 f   misc.obj
 0001:00010fd0       ?RILDrv_GetPacketByteCount@@YAJK@Z 00111fd0 f   misc.obj
 0001:00011030       ?RILDrv_ResetPacketByteCount@@YAJK@Z 00112030 f   misc.obj
 0001:00011090       ?RILDrv_GetSystemTime@@YAJK@Z 00112090 f   misc.obj
 0001:000110f0       ?RILDrv_DevSpecific@@YAJKPBEK@Z 001120f0 f   misc.obj
 0001:000114ac       ?SetEquipmentCachedState@CRadio@@QAAXK@Z 001124ac f   misc.obj
 0001:000115f4       ?GetEquipmentState@CRadio@@QAAJPAVCResponse@@@Z 001125f4 f   misc.obj
 0001:000116c8       ?ForceModemPowerOff@CRadio@@QAAXXZ 001126c8 f   misc.obj
 0001:0001174c       ?NotifyHardResetModemRequired@CRadio@@QAAXXZ 0011274c f   misc.obj
 0001:00011798       ?SetEquipmentState@CRadio@@QAAJPAVCResponse@@PAX@Z 00112798 f   misc.obj
 0001:00011b4c       ?FillSignalQualityStruct@CRadio@@QAAXPAUrilsignalquality_tag@@II@Z 00112b4c f   misc.obj
 0001:00011e60       ?GetSignalQuality@CRadio@@QAAJPAVCResponse@@@Z 00112e60 f   misc.obj
 0001:00011fb4       ?GetCellTowerInfo@CRadio@@QAAJPAVCResponse@@@Z 00112fb4 f   misc.obj
 0001:00012234       ?GetPacketByteCount@CRadio@@QAAJPAVCResponse@@@Z 00113234 f   misc.obj
 0001:00012340       ?ResetPacketByteCount@CRadio@@QAAJPAVCResponse@@@Z 00113340 f   misc.obj
 0001:00012384       ?GetSystemTime@CRadio@@QAAJPAVCResponse@@@Z 00113384 f   misc.obj
 0001:00012448       ?GetEquipmentInfo@CRadio@@QAAJPAVCResponse@@@Z 00113448 f   misc.obj
 0001:000127dc       ?GetLocationStatus@CRadio@@QAAJXZ 001137dc f   misc.obj
 0001:00012828       ?StopDMMode@CRadio@@QAAJXZ 00113828 f   misc.obj
 0001:00012944       ?StartPTMode@CRadio@@QAAJXZ 00113944 f   misc.obj
 0001:00012a10       ?StopPTMode@CRadio@@QAAJXZ 00113a10 f   misc.obj
 0001:00012ae8       ?SetGpsOneXtra@CRadio@@QAAJK@Z 00113ae8 f   misc.obj
 0001:00012b60       ?SetGpsDefault@CRadio@@QAAJKEKK@Z 00113b60 f   misc.obj
 0001:00012c44       ?SetNMEAConfig@CRadio@@QAAJEEEPAG@Z 00113c44 f   misc.obj
 0001:00012d2c       ?RILDrv_GetPhonebookOptions@@YAJK@Z 00113d2c f   misc.obj
 0001:00012d8c       ?RilToQmiSimPbStoreLocation@@YAKK@Z 00113d8c f   misc.obj
 0001:00012e3c       ?GetPhonebookOptions@CRadio@@QAAJPAVCResponse@@@Z 00113e3c f   misc.obj
 0001:00012fd4       ?RILDrv_SetPhonebookOptions@@YAJKPBUrilphonebookinfo_tag@@@Z 00113fd4 f   misc.obj
 0001:000130a8       ?SetPhonebookOptions@CRadio@@QAAJPAVCResponse@@PAX@Z 001140a8 f   misc.obj
 0001:000130e4       ?RILDrv_ReadPhonebookEntries@@YAJKKK@Z 001140e4 f   misc.obj
 0001:000131ac       ?ReadPhonebookEntries@CRadio@@QAAJPAVCResponse@@PAX@Z 001141ac f   misc.obj
 0001:000135e4       ?UpdateAndBroadcastOnSWIPhoneBookNotification@CRadio@@QAAXPAUSwiNotifyVariant@@@Z 001145e4 f   misc.obj
 0001:000137a8       ?cmp_emergency_num_info@@YA_NABUtagEMERGENCY_NUM_INFO@@0@Z 001147a8 f   misc.obj
 0001:000137d0       ?cmp_emergency_num_info_equal@@YA_NABUtagEMERGENCY_NUM_INFO@@0@Z 001147d0 f   misc.obj
 0001:000137f8       ?RILDrv_WritePhonebookEntry@@YAJKPBUrilphonebookentry_tag@@@Z 001147f8 f   misc.obj
 0001:0001389c       ?WritePhonebookEntry@CRadio@@QAAJPAVCResponse@@PAX@Z 0011489c f   misc.obj
 0001:00013a7c       ?RILDrv_DeletePhonebookEntry@@YAJKK@Z 00114a7c f   misc.obj
 0001:00013ae4       ?DeletePhonebookEntry@CRadio@@QAAJPAVCResponse@@PAX@Z 00114ae4 f   misc.obj
 0001:00013bcc       ?IsSafeImage@CRadio@@QAAHXZ 00114bcc f   misc.obj
 0001:00013e80       ?GetFwImagePreference@CRadio@@QAAHPAKQAE@Z 00114e80 f   misc.obj
 0001:00014004       ?SetFwImagePreference@CRadio@@QAAHPAKQAE@Z 00115004 f   misc.obj
 0001:0001415c       ??$_Allocate@U_Node@?$_List_nod@UtagEMERGENCY_NUM_INFO@@V?$allocator@UtagEMERGENCY_NUM_INFO@@@std@@@std@@@std@@YAPAU_Node@?$_List_nod@UtagEMERGENCY_NUM_INFO@@V?$allocator@UtagEMERGENCY_NUM_INFO@@@std@@@0@IPAU120@@Z 0011515c f i misc.obj
 0001:000141c8       ?RILDrv_HandleResume@@YAJKW4_CEDEVICE_POWER_STATE@@@Z 001151c8 f   misc.obj
 0001:00014330       ?RILDrv_AuxPowerSet@@YAJKPAW4_CEDEVICE_POWER_STATE@@@Z 00115330 f   misc.obj
 0001:000143e0       ?HardResetModem@CRadio@@QAAXXZ 001153e0 f   misc.obj
 0001:00014410       ?StartDMMode@CRadio@@QAAJW4eDM_MODE@@@Z 00115410 f   misc.obj
 0001:00014654       ?DevSpecific@CRadio@@QAAJPAVCResponse@@PAX@Z 00115654 f   misc.obj
 0001:00017908       ?clear@?$list@UtagEMERGENCY_NUM_INFO@@V?$allocator@UtagEMERGENCY_NUM_INFO@@@std@@@std@@QAAXXZ 00118908 f i misc.obj
 0001:0001794c       ?_Buynode@?$list@UtagEMERGENCY_NUM_INFO@@V?$allocator@UtagEMERGENCY_NUM_INFO@@@std@@@std@@IAAPAU_Node@?$_List_nod@UtagEMERGENCY_NUM_INFO@@V?$allocator@UtagEMERGENCY_NUM_INFO@@@std@@@2@XZ 0011894c f i misc.obj
 0001:00017970       ?_Buynode@?$list@UtagEMERGENCY_NUM_INFO@@V?$allocator@UtagEMERGENCY_NUM_INFO@@@std@@@std@@IAAPAU_Node@?$_List_nod@UtagEMERGENCY_NUM_INFO@@V?$allocator@UtagEMERGENCY_NUM_INFO@@@std@@@2@PAU342@0ABUtagEMERGENCY_NUM_INFO@@@Z 00118970 f i misc.obj
 0001:000179b4       ?erase@?$list@UtagEMERGENCY_NUM_INFO@@V?$allocator@UtagEMERGENCY_NUM_INFO@@@std@@@std@@QAA?AV?$_Iterator@$00@12@V312@@Z 001189b4 f i misc.obj
 0001:00017a3c       ??1?$list@UtagEMERGENCY_NUM_INFO@@V?$allocator@UtagEMERGENCY_NUM_INFO@@@std@@@std@@QAA@XZ 00118a3c f i misc.obj
 0001:00017a5c       ??$unique@P6A_NABUtagEMERGENCY_NUM_INFO@@0@Z@?$list@UtagEMERGENCY_NUM_INFO@@V?$allocator@UtagEMERGENCY_NUM_INFO@@@std@@@std@@QAAXP6A_NABUtagEMERGENCY_NUM_INFO@@0@Z@Z 00118a5c f i misc.obj
 0001:00017b4c       ??0?$list@UtagEMERGENCY_NUM_INFO@@V?$allocator@UtagEMERGENCY_NUM_INFO@@@std@@@std@@QAA@XZ 00118b4c f i misc.obj
 0001:00017b74       ?_Incsize@?$list@UtagEMERGENCY_NUM_INFO@@V?$allocator@UtagEMERGENCY_NUM_INFO@@@std@@@std@@IAAXI@Z 00118b74 f i misc.obj
 0001:00017c20       ?_Splice@?$list@UtagEMERGENCY_NUM_INFO@@V?$allocator@UtagEMERGENCY_NUM_INFO@@@std@@@std@@QAAXV?$_Iterator@$00@12@AAV12@00I_N@Z 00118c20 f i misc.obj
 0001:00017c94       ??$merge@P6A_NABUtagEMERGENCY_NUM_INFO@@0@Z@?$list@UtagEMERGENCY_NUM_INFO@@V?$allocator@UtagEMERGENCY_NUM_INFO@@@std@@@std@@QAAXAAV01@P6A_NABUtagEMERGENCY_NUM_INFO@@1@Z@Z 00118c94 f i misc.obj
 0001:00017e4c       ?splice@?$list@UtagEMERGENCY_NUM_INFO@@V?$allocator@UtagEMERGENCY_NUM_INFO@@@std@@@std@@QAAXV?$_Iterator@$00@12@AAV12@@Z 00118e4c f i misc.obj
 0001:00017ec4       ??$sort@P6A_NABUtagEMERGENCY_NUM_INFO@@0@Z@?$list@UtagEMERGENCY_NUM_INFO@@V?$allocator@UtagEMERGENCY_NUM_INFO@@@std@@@std@@QAAXP6A_NABUtagEMERGENCY_NUM_INFO@@0@Z@Z 00118ec4 f i misc.obj
 0001:00018120       ?HandleSWIEmergencyListNotification@CRadio@@QAAXPAUSwiNotifyVariant@@@Z 00119120 f   misc.obj
 0001:0001834c       ?MonitorThreadProc@@YAKPAX@Z 0011934c f   monitor.obj
 0001:00018460       ??0CMonitor@@QAA@XZ        00119460 f   monitor.obj
 0001:0001847c       ?Init@CMonitor@@QAAHQAXKK@Z 0011947c f   monitor.obj
 0001:0001869c       ??1CMonitor@@QAA@XZ        0011969c f   monitor.obj
 0001:000186f4       ??1SWISYNCBLOCK@@QAA@XZ    001196f4 f i msg.obj
 0001:00018708       ?Hex2Dec@@YAGE@Z           00119708 f   msg.obj
 0001:00018758       ?ValidateMsgDCS@@YAJABUrilmsgdcs_tag@@@Z 00119758 f   msg.obj
 0001:00018820       ?ValidateMsgAddress@@YAJABUriladdress_tag@@@Z 00119820 f   msg.obj
 0001:00018880       ?ValidateSubmitMsg@@YAJABUrilmessage_tag@@@Z 00119880 f   msg.obj
 0001:00018934       ?ValidateCmdMsg@@YAJABUrilmessage_tag@@@Z 00119934 f   msg.obj
 0001:000189bc       ?ValidateDeliverMsg@@YAJABUrilmessage_tag@@@Z 001199bc f   msg.obj
 0001:00018a44       ?ValidateStatusMsg@@YAJABUrilmessage_tag@@@Z 00119a44 f   msg.obj
 0001:00018af8       ?ValidateMessage@@YAJABUrilmessage_tag@@@Z 00119af8 f   msg.obj
 0001:00018bec       ?RILDrv_GetMsgServiceOptions@@YAJK@Z 00119bec f   msg.obj
 0001:00018c4c       ?RILDrv_GetMsgConfig@@YAJK@Z 00119c4c f   msg.obj
 0001:00018cac       ?RILDrv_SetMsgConfig@@YAJKPBUrilmsgconfig_tag@@@Z 00119cac f   msg.obj
 0001:00018da8       ?RILDrv_GetCellBroadcastMsgConfig@@YAJK@Z 00119da8 f   msg.obj
 0001:00018e08       ?RILDrv_SetCellBroadcastMsgConfig@@YAJKPBUrilcbmsgconfig_tag@@@Z 00119e08 f   msg.obj
 0001:00018ecc       ?RILDrv_ReadMsg@@YAJKK@Z   00119ecc f   msg.obj
 0001:00018f3c       ?RILDrv_DeleteMsg@@YAJKK@Z 00119f3c f   msg.obj
 0001:00019054       ?RILDrv_SendMsg@@YAJKPBUrilmessage_tag@@K@Z 0011a054 f   msg.obj
 0001:000191a0       ?RILDrv_SendStoredMsg@@YAJKKK@Z 0011a1a0 f   msg.obj
 0001:00019208       ?RILDrv_SendMsgAcknowledgement@@YAJKH@Z 0011a208 f   msg.obj
 0001:00019268       ?MsgSendThreadProc@@YAKPAX@Z 0011a268 f   msg.obj
 0001:000193cc       ?ReceiveMsg@CRadio@@QAAXPAUrilmessage_tag@@@Z 0011a3cc f   msg.obj
 0001:00019778       ?GetMsgServiceOptions@CRadio@@QAAJPAVCResponse@@@Z 0011a778 f   msg.obj
 0001:00019810       ?GetMsgConfig@CRadio@@QAAJPAVCResponse@@@Z 0011a810 f   msg.obj
 0001:000199ec       ?SetMsgConfig@CRadio@@QAAJPAVCResponse@@PAX@Z 0011a9ec f   msg.obj
 0001:00019b24       ?SmsMtSetRilAddressNumberType@CRadio@@QAAKE@Z 0011ab24 f   msg.obj
 0001:00019b90       ?SmsMtSetRilAddressNumberPlan@CRadio@@QAAKE@Z 0011ab90 f   msg.obj
 0001:00019c00       ?IsEmailAddr@CRadio@@IAAHPAG@Z 0011ac00 f   msg.obj
 0001:00019ca0       ?InitSMSSendHdr@CRadio@@QAAXPAUSWI_STRUCT_SMS_CdmaHeader@@@Z 0011aca0 f   msg.obj
 0001:00019d40       ?RILDrv_WriteMsg@@YAJKPBUrilmessage_tag@@K@Z 0011ad40 f   msg.obj
 0001:00019da8       ??_GCriticalSection@@UAAPAXI@Z 0011ada8 f i msg.obj
 0001:00019da8       ??_ECriticalSection@@UAAPAXI@Z 0011ada8 f i msg.obj
 0001:00019de0       ?RILDrv_SetMsgServiceOptions@@YAJKPBUrilmsgserviceinfo_tag@@@Z 0011ade0 f   msg.obj
 0001:0001a0e4       ?MsgReceiveOnNotifyThreadProcGsm@@YAKPAX@Z 0011b0e4 f   msg.obj
 0001:0001a940       ?MsgReceiveOnNotifyThreadProc@@YAKPAX@Z 0011b940 f   msg.obj
 0001:0001b3f4       ?SendMsg@CRadio@@QAAJPAVCResponse@@PAX@Z 0011c3f4 f   msg.obj
 0001:0001c4d4       ?UpdateAndBroadcastOnSWISMSNotification@CRadio@@QAAXPAUSwiNotifyVariant@@@Z 0011d4d4 f   msg.obj
 0001:0001c978       ?RILDrv_GetSubscriberNumbers@@YAJK@Z 0011d978 f   network.obj
 0001:0001c9d8       ?RILDrv_GetCurrentOperator@@YAJKK@Z 0011d9d8 f   network.obj
 0001:0001ca38       ?RILDrv_GetOperatorList@@YAJK@Z 0011da38 f   network.obj
 0001:0001ca98       ?RILDrv_GetRegistrationStatus@@YAJK@Z 0011da98 f   network.obj
 0001:0001caf8       ?RILDrv_GetCurrentSystemType@@YAJK@Z 0011daf8 f   network.obj
 0001:0001cb58       ?RILDrv_GetRoamingMode@@YAJK@Z 0011db58 f   network.obj
 0001:0001cbb8       ?RILDrv_SetRoamingMode@@YAJKK@Z 0011dbb8 f   network.obj
 0001:0001cc20       ?RILDrv_GetPreferredPrivacyMode@@YAJK@Z 0011dc20 f   network.obj
 0001:0001cc80       ?RILDrv_SetPreferredPrivacyMode@@YAJKK@Z 0011dc80 f   network.obj
 0001:0001ccf0       ?GetSubscriberNumbers@CRadio@@QAAJPAVCResponse@@@Z 0011dcf0 f   network.obj
 0001:0001cda8       ?GetCurrentOperator@CRadio@@QAAJPAVCResponse@@@Z 0011dda8 f   network.obj
 0001:0001ceb8       ?AddPreferredOperator@CRadio@@QAAJPAVCResponse@@PAX@Z 0011deb8 f   network.obj
 0001:0001d098       ?RemovePreferredOperator@CRadio@@QAAJPAVCResponse@@PAX@Z 0011e098 f   network.obj
 0001:0001d16c       ?GetPreferredOperatorList@CRadio@@QAAJPAVCResponse@@PAX@Z 0011e16c f   network.obj
 0001:0001d648       ?GetOperatorList@CRadio@@QAAJPAVCResponse@@@Z 0011e648 f   network.obj
 0001:0001d7b0       ?UnRegisterFromNetwork@CRadio@@QAAJPAVCResponse@@@Z 0011e7b0 f   network.obj
 0001:0001d8f4       ?UpdateEVDONetworkType@CRadio@@QAAXK@Z 0011e8f4 f   network.obj
 0001:0001d940       ?GetRegistrationStatus@CRadio@@QAAJPAVCResponse@@@Z 0011e940 f   network.obj
 0001:0001da48       ?GetCurrentSystemType@CRadio@@QAAJPAVCResponse@@@Z 0011ea48 f   network.obj
 0001:0001db1c       ?GetRoamingMode@CRadio@@QAAJPAVCResponse@@@Z 0011eb1c f   network.obj
 0001:0001dc40       ?SetRoamingMode@CRadio@@QAAJPAVCResponse@@PAX@Z 0011ec40 f   network.obj
 0001:0001dd88       ?GetPreferredPrivacyMode@CRadio@@QAAJPAVCResponse@@@Z 0011ed88 f   network.obj
 0001:0001dd94       ?SetPreferredPrivacyMode@CRadio@@QAAJPAVCResponse@@PAX@Z 0011ed94 f   network.obj
 0001:0001dda0       ?SetHomeAndCurrentOperator@CRadio@@QAAXK@Z 0011eda0 f   network.obj
 0001:0001df74       ?RILDrv_RegisterOnNetwork@@YAJKKPBUriloperatornames_tag@@@Z 0011ef74 f   network.obj
 0001:0001e048       ?RILDrv_GetPreferredOperatorList@@YAJKK@Z 0011f048 f   network.obj
 0001:0001e0b0       ?RILDrv_AddPreferredOperator@@YAJKKPBUriloperatornames_tag@@@Z 0011f0b0 f   network.obj
 0001:0001e1a4       ?RILDrv_RemovePreferredOperator@@YAJKK@Z 0011f1a4 f   network.obj
 0001:0001e214       ?GetAllOperatorsList@CRadio@@QAAJPAVCResponse@@@Z 0011f214 f   network.obj
 0001:0001e34c       ?RILDrv_GetAllOperatorsList@@YAJK@Z 0011f34c f   network.obj
 0001:0001e3ac       ?RILDrv_UnregisterFromNetwork@@YAJK@Z 0011f3ac f   network.obj
 0001:0001e434       ?CheckCurrentRUIM@CRadio@@QAAHXZ 0011f434 f   network.obj
 0001:0001e504       ?RegisterOnNetwork@CRadio@@QAAJPAVCResponse@@PAX@Z 0011f504 f   network.obj
 0001:0001eb30       ?ConvertToRILSystem@CRadio@@QAAKK@Z 0011fb30 f   Radio.obj
 0001:0001ebe8       ?UnloadSwiAux@CRadio@@QAAXXZ 0011fbe8 f   Radio.obj
 0001:0001ec50       ?GetUserNetworkPreference@CRadio@@QAAHXZ 0011fc50 f   Radio.obj
 0001:0001ec64       ?GetRuimLockStatus@CRadio@@QAAKXZ 0011fc64 f   Radio.obj
 0001:0001ee5c       ?UpdateUserNetworkPreference@CRadio@@QAAXH@Z 0011fe5c f   Radio.obj
 0001:0001ee6c       ?SetSwiWirelessTech@CRadio@@QAAXK@Z 0011fe6c f   Radio.obj
 0001:0001ef50       ?PreExecCmd@CRadio@@QAAJPAVCCommand@@PAVCResponse@@@Z 0011ff50 f   Radio.obj
 0001:0001eff0       ?LaunchWapIOTA@CRadio@@QAAXG@Z 0011fff0 f   Radio.obj
 0001:0001f0b8       ?ReceiveNotification@CRadio@@QAAXKPAXI@Z 001200b8 f   Radio.obj
 0001:0001f0c8       ?UpdateCombinedServiceStatus@CRadio@@QAAHKK@Z 001200c8 f   Radio.obj
 0001:0001f648       ?SendDelayedNITZThreadProc@@YAKPAX@Z 00120648 f   Radio.obj
 0001:0001f744       ?DataDormancyPollingThread@CRadio@@QAAXXZ 00120744 f   Radio.obj
 0001:0001f974       ?OnIdle@CRadio@@QAAXXZ     00120974 f   Radio.obj
 0001:0001fa50       ?DecBasedOrder@@YAKK@Z     00120a50 f   Radio.obj
 0001:0001fa88       ?HandleRssi@CRadio@@QAAXH@Z 00120a88 f   Radio.obj
 0001:0001fb00       ?HandleGsmSystemStatus@CRadio@@QAAXPAUSWI_STRUCT_GsmSystemStatus@@@Z 00120b00 f   Radio.obj
 0001:0001ff1c       ?UpdateSIMStatus@CRadio@@QAAXK@Z 00120f1c f   Radio.obj
 0001:0001ff48       ?UpdatePhLockedState@CRadio@@QAAXK@Z 00120f48 f   Radio.obj
 0001:0001ff94       ?GetPhLockedState@CRadio@@QAAKXZ 00120f94 f   Radio.obj
 0001:0001ffa8       ?GetPhoneBookEntry@CRadio@@QAAHXZ 00120fa8 f   Radio.obj
 0001:00020190       ?UpdateMDNNumber@CRadio@@QAAHXZ 00121190 f   Radio.obj
 0001:000202cc       ?BroadcastMinActiveStateNotification@CRadio@@QAAXXZ 001212cc f   Radio.obj
 0001:00020308       ?BroadcastEquipmentStateNotification@CRadio@@QAAXKK@Z 00121308 f   Radio.obj
 0001:0002038c       ?ResetCallState@CRadio@@AAAXXZ 0012138c f   Radio.obj
 0001:0002049c       ??8?$_Const_iterator@$00@?$list@PAVCCommand@@V?$allocator@PAVCCommand@@@std@@@std@@QBA_NABV012@@Z 0012149c f i Radio.obj
 0001:000204e4       ??E?$_Const_iterator@$00@?$list@PAVCCommand@@V?$allocator@PAVCCommand@@@std@@@std@@QAAAAV012@XZ 001214e4 f i Radio.obj
 0001:00020520       ??8const_iterator@?$_Tree@V?$_Tmap_traits@KU__Fail_Cmd_Data_tag@@U?$less@K@std@@V?$allocator@U?$pair@$$CBKU__Fail_Cmd_Data_tag@@@std@@@3@$0A@@std@@@std@@QBA_NABV012@@Z 00121520 f i Radio.obj
 0001:00020568       ??8const_iterator@?$_Tree@V?$_Tmap_traits@KKU?$less@K@std@@V?$allocator@U?$pair@$$CBKK@std@@@2@$0A@@std@@@std@@QBA_NABV012@@Z 00121568 f i Radio.obj
 0001:000205b0       ?_Rrotate@?$_Tree@V?$_Tmap_traits@KU__Fail_Cmd_Data_tag@@U?$less@K@std@@V?$allocator@U?$pair@$$CBKU__Fail_Cmd_Data_tag@@@std@@@3@$0A@@std@@@std@@IAAXPAU_Node@?$_Tree_nod@V?$_Tmap_traits@KU__Fail_Cmd_Data_tag@@U?$less@K@std@@V?$allocator@U?$pair@$$CBKU__Fail_Cmd_Data_tag@@@std@@@3@$0A@@std@@@2@@Z 001215b0 f i Radio.obj
 0001:00020620       ?_Rrotate@?$_Tree@V?$_Tmap_traits@KKU?$less@K@std@@V?$allocator@U?$pair@$$CBKK@std@@@2@$0A@@std@@@std@@IAAXPAU_Node@?$_Tree_nod@V?$_Tmap_traits@KKU?$less@K@std@@V?$allocator@U?$pair@$$CBKK@std@@@2@$0A@@std@@@2@@Z 00121620 f i Radio.obj
 0001:00020690       ?_Inc@const_iterator@?$_Tree@V?$_Tmap_traits@KU__Fail_Cmd_Data_tag@@U?$less@K@std@@V?$allocator@U?$pair@$$CBKU__Fail_Cmd_Data_tag@@@std@@@3@$0A@@std@@@std@@QAAXXZ 00121690 f i Radio.obj
 0001:0002072c       ?_Dec@const_iterator@?$_Tree@V?$_Tmap_traits@KKU?$less@K@std@@V?$allocator@U?$pair@$$CBKK@std@@@2@$0A@@std@@@std@@QAAXXZ 0012172c f i Radio.obj
 0001:000207fc       ?_Inc@const_iterator@?$_Tree@V?$_Tmap_traits@KKU?$less@K@std@@V?$allocator@U?$pair@$$CBKK@std@@@2@$0A@@std@@@std@@QAAXXZ 001217fc f i Radio.obj
 0001:00020898       ??$_Allocate@U_Node@?$_Tree_nod@V?$_Tmap_traits@KU__Fail_Cmd_Data_tag@@U?$less@K@std@@V?$allocator@U?$pair@$$CBKU__Fail_Cmd_Data_tag@@@std@@@3@$0A@@std@@@std@@@std@@YAPAU_Node@?$_Tree_nod@V?$_Tmap_traits@KU__Fail_Cmd_Data_tag@@U?$less@K@std@@V?$allocator@U?$pair@$$CBKU__Fail_Cmd_Data_tag@@@std@@@3@$0A@@std@@@0@IPAU120@@Z 00121898 f i Radio.obj
 0001:00020908       ??$_Allocate@U_Node@?$_Tree_nod@V?$_Tmap_traits@KKU?$less@K@std@@V?$allocator@U?$pair@$$CBKK@std@@@2@$0A@@std@@@std@@@std@@YAPAU_Node@?$_Tree_nod@V?$_Tmap_traits@KKU?$less@K@std@@V?$allocator@U?$pair@$$CBKK@std@@@2@$0A@@std@@@0@IPAU120@@Z 00121908 f i Radio.obj
 0001:00020978       ??$_Allocate@PAUSwiNotifyVariant@@@std@@YAPAPAUSwiNotifyVariant@@IPAPAU1@@Z 00121978 f i Radio.obj
 0001:000209e4       ??$_Allocate@PAPAUSwiNotifyVariant@@@std@@YAPAPAPAUSwiNotifyVariant@@IPAPAPAU1@@Z 001219e4 f i Radio.obj
 0001:00020a50       ?DataDormancyPollingThreadProc@@YAKPAX@Z 00121a50 f   Radio.obj
 0001:00020a60       ?ExecuteCommand@CRadio@@QAAJPAVCCommand@@PAVCResponse@@@Z 00121a60 f   Radio.obj
 0001:000212e4       ?_Lbound@?$_Tree@V?$_Tmap_traits@KKU?$less@K@std@@V?$allocator@U?$pair@$$CBKK@std@@@2@$0A@@std@@@std@@IBAPAU_Node@?$_Tree_nod@V?$_Tmap_traits@KKU?$less@K@std@@V?$allocator@U?$pair@$$CBKK@std@@@2@$0A@@std@@@2@ABK@Z 001222e4 f i Radio.obj
 0001:0002133c       ?_Lrotate@?$_Tree@V?$_Tmap_traits@KU__Fail_Cmd_Data_tag@@U?$less@K@std@@V?$allocator@U?$pair@$$CBKU__Fail_Cmd_Data_tag@@@std@@@3@$0A@@std@@@std@@IAAXPAU_Node@?$_Tree_nod@V?$_Tmap_traits@KU__Fail_Cmd_Data_tag@@U?$less@K@std@@V?$allocator@U?$pair@$$CBKU__Fail_Cmd_Data_tag@@@std@@@3@$0A@@std@@@2@@Z 0012233c f i Radio.obj
 0001:000213a4       ?_Lrotate@?$_Tree@V?$_Tmap_traits@KKU?$less@K@std@@V?$allocator@U?$pair@$$CBKK@std@@@2@$0A@@std@@@std@@IAAXPAU_Node@?$_Tree_nod@V?$_Tmap_traits@KKU?$less@K@std@@V?$allocator@U?$pair@$$CBKK@std@@@2@$0A@@std@@@2@@Z 001223a4 f i Radio.obj
 0001:0002140c       ?erase@?$list@PAVCCommand@@V?$allocator@PAVCCommand@@@std@@@std@@QAA?AV?$_Iterator@$00@12@V312@@Z 0012240c f i Radio.obj
 0001:00021494       ?_Buynode@?$_Tree@V?$_Tmap_traits@KU__Fail_Cmd_Data_tag@@U?$less@K@std@@V?$allocator@U?$pair@$$CBKU__Fail_Cmd_Data_tag@@@std@@@3@$0A@@std@@@std@@IAAPAU_Node@?$_Tree_nod@V?$_Tmap_traits@KU__Fail_Cmd_Data_tag@@U?$less@K@std@@V?$allocator@U?$pair@$$CBKU__Fail_Cmd_Data_tag@@@std@@@3@$0A@@std@@@2@XZ 00122494 f i Radio.obj
 0001:000214d0       ?_Buynode@?$_Tree@V?$_Tmap_traits@KKU?$less@K@std@@V?$allocator@U?$pair@$$CBKK@std@@@2@$0A@@std@@@std@@IAAPAU_Node@?$_Tree_nod@V?$_Tmap_traits@KKU?$less@K@std@@V?$allocator@U?$pair@$$CBKK@std@@@2@$0A@@std@@@2@XZ 001224d0 f i Radio.obj
 0001:0002150c       ?_Buynode@?$_Tree@V?$_Tmap_traits@KKU?$less@K@std@@V?$allocator@U?$pair@$$CBKK@std@@@2@$0A@@std@@@std@@IAAPAU_Node@?$_Tree_nod@V?$_Tmap_traits@KKU?$less@K@std@@V?$allocator@U?$pair@$$CBKK@std@@@2@$0A@@std@@@2@PAU342@00ABU?$pair@$$CBKK@2@D@Z 0012250c f i Radio.obj
 0001:00021564       ?_Erase@?$_Tree@V?$_Tmap_traits@KU__Fail_Cmd_Data_tag@@U?$less@K@std@@V?$allocator@U?$pair@$$CBKU__Fail_Cmd_Data_tag@@@std@@@3@$0A@@std@@@std@@IAAXPAU_Node@?$_Tree_nod@V?$_Tmap_traits@KU__Fail_Cmd_Data_tag@@U?$less@K@std@@V?$allocator@U?$pair@$$CBKU__Fail_Cmd_Data_tag@@@std@@@3@$0A@@std@@@2@@Z 00122564 f i Radio.obj
 0001:000215ac       ?_Erase@?$_Tree@V?$_Tmap_traits@KKU?$less@K@std@@V?$allocator@U?$pair@$$CBKK@std@@@2@$0A@@std@@@std@@IAAXPAU_Node@?$_Tree_nod@V?$_Tmap_traits@KKU?$less@K@std@@V?$allocator@U?$pair@$$CBKK@std@@@2@$0A@@std@@@2@@Z 001225ac f i Radio.obj
 0001:000215f4       ?GetDataDialCmd@CRadio@@QAAPAVCCommand@@XZ 001225f4 f   Radio.obj
 0001:000216dc       ?UpdateEmergencyRegistry@CRadio@@AAAXXZ 001226dc f   Radio.obj
 0001:00021a38       ?remove@?$list@PAVCCommand@@V?$allocator@PAVCCommand@@@std@@@std@@QAAXABQAVCCommand@@@Z 00122a38 f i Radio.obj
 0001:00021ae8       ?_Init@?$_Tree@V?$_Tmap_traits@KU__Fail_Cmd_Data_tag@@U?$less@K@std@@V?$allocator@U?$pair@$$CBKU__Fail_Cmd_Data_tag@@@std@@@3@$0A@@std@@@std@@IAAXXZ 00122ae8 f i Radio.obj
 0001:00021b24       ?_Init@?$_Tree@V?$_Tmap_traits@KKU?$less@K@std@@V?$allocator@U?$pair@$$CBKK@std@@@2@$0A@@std@@@std@@IAAXXZ 00122b24 f i Radio.obj
 0001:00021b68       ?Wait4ATConnect@CRadio@@QAAXXZ 00122b68 f   Radio.obj
 0001:0002237c       ?erase@?$_Tree@V?$_Tmap_traits@KU__Fail_Cmd_Data_tag@@U?$less@K@std@@V?$allocator@U?$pair@$$CBKU__Fail_Cmd_Data_tag@@@std@@@3@$0A@@std@@@std@@QAA?AViterator@12@V312@@Z 0012337c f i Radio.obj
 0001:000227f0       ?erase@?$_Tree@V?$_Tmap_traits@KKU?$less@K@std@@V?$allocator@U?$pair@$$CBKK@std@@@2@$0A@@std@@@std@@QAA?AViterator@12@V312@@Z 001237f0 f i Radio.obj
 0001:00022c64       ?_Xlen@?$deque@PAUSwiNotifyVariant@@V?$allocator@PAUSwiNotifyVariant@@@std@@@std@@KAXXZ 00123c64 f i Radio.obj
 0001:00022cd0       ?erase@?$_Tree@V?$_Tmap_traits@KU__Fail_Cmd_Data_tag@@U?$less@K@std@@V?$allocator@U?$pair@$$CBKU__Fail_Cmd_Data_tag@@@std@@@3@$0A@@std@@@std@@QAA?AViterator@12@V312@0@Z 00123cd0 f i Radio.obj
 0001:00022ddc       ?erase@?$_Tree@V?$_Tmap_traits@KKU?$less@K@std@@V?$allocator@U?$pair@$$CBKK@std@@@2@$0A@@std@@@std@@QAA?AViterator@12@V312@0@Z 00123ddc f i Radio.obj
 0001:00022ef0       ?_Insert@?$_Tree@V?$_Tmap_traits@KKU?$less@K@std@@V?$allocator@U?$pair@$$CBKK@std@@@2@$0A@@std@@@std@@IAA?AViterator@12@_NPAU_Node@?$_Tree_nod@V?$_Tmap_traits@KKU?$less@K@std@@V?$allocator@U?$pair@$$CBKK@std@@@2@$0A@@std@@@2@ABU?$pair@$$CBKK@2@@Z 00123ef0 f i Radio.obj
 0001:0002313c       ?_Growmap@?$deque@PAUSwiNotifyVariant@@V?$allocator@PAUSwiNotifyVariant@@@std@@@std@@IAAXI@Z 0012413c f i Radio.obj
 0001:000232c8       ?_Tidy@?$_Tree@V?$_Tmap_traits@KU__Fail_Cmd_Data_tag@@U?$less@K@std@@V?$allocator@U?$pair@$$CBKU__Fail_Cmd_Data_tag@@@std@@@3@$0A@@std@@@std@@IAAXXZ 001242c8 f i Radio.obj
 0001:0002330c       ?_Tidy@?$_Tree@V?$_Tmap_traits@KKU?$less@K@std@@V?$allocator@U?$pair@$$CBKK@std@@@2@$0A@@std@@@std@@IAAXXZ 0012430c f i Radio.obj
 0001:00023350       ?insert@?$_Tree@V?$_Tmap_traits@KKU?$less@K@std@@V?$allocator@U?$pair@$$CBKK@std@@@2@$0A@@std@@@std@@QAA?AU?$pair@Viterator@?$_Tree@V?$_Tmap_traits@KKU?$less@K@std@@V?$allocator@U?$pair@$$CBKK@std@@@2@$0A@@std@@@std@@_N@2@ABU?$pair@$$CBKK@2@@Z 00124350 f i Radio.obj
 0001:00023488       ?push_back@?$deque@PAUSwiNotifyVariant@@V?$allocator@PAUSwiNotifyVariant@@@std@@@std@@QAAXABQAUSwiNotifyVariant@@@Z 00124488 f i Radio.obj
 0001:00023528       ?insert@?$_Tree@V?$_Tmap_traits@KKU?$less@K@std@@V?$allocator@U?$pair@$$CBKK@std@@@2@$0A@@std@@@std@@QAA?AViterator@12@V312@ABU?$pair@$$CBKK@2@@Z 00124528 f i Radio.obj
 0001:000237a0       ??1?$map@KU__Fail_Cmd_Data_tag@@U?$less@K@std@@V?$allocator@U?$pair@$$CBKU__Fail_Cmd_Data_tag@@@std@@@3@@std@@QAA@XZ 001247a0 f i Radio.obj
 0001:000237a4       ??1?$map@KKU?$less@K@std@@V?$allocator@U?$pair@$$CBKK@std@@@2@@std@@QAA@XZ 001247a4 f i Radio.obj
 0001:000237b0       ??1CRadio@@QAA@XZ          001247b0 f   Radio.obj
 0001:00023950       ?InitializeEmergencyList@CRadio@@AAAXXZ 00124950 f   Radio.obj
 0001:00023dac       ??A?$map@KKU?$less@K@std@@V?$allocator@U?$pair@$$CBKK@std@@@2@@std@@QAAAAKABK@Z 00124dac f i Radio.obj
 0001:00023e64       ?Push_Back@?$CThreadSafeQueue@PAUSwiNotifyVariant@@@@QAAXABQAUSwiNotifyVariant@@@Z 00124e64 f i Radio.obj
 0001:00023eb0       ?Init@CRadio@@QAAJXZ       00124eb0 f   Radio.obj
 0001:000241c0       ?SWIEventCallback@@YAXPAUSwiNotifyVariant@@@Z 001251c0 f   Radio.obj
 0001:00024228       ?InitializeRadioStateMachine@CRadio@@QAAXH@Z 00125228 f   Radio.obj
 0001:00024978       ?LoadSwiAux@CRadio@@QAAXXZ 00125978 f   Radio.obj
 0001:00024c0c       ?UpdateAndBroadcastOnSWINotification@CRadio@@QAAXPAUSwiNotifyVariant@@@Z 00125c0c f   Radio.obj
 0001:00026abc       ??0CRadio@@QAA@PAVCRilHandle@@@Z 00127abc f   Radio.obj
 0001:00026d90       ??0CRadioCaps@@QAA@XZ      00127d90 f   RadioCaps.obj
 0001:00026da0       ??1CRadioCaps@@QAA@XZ      00127da0 f   RadioCaps.obj
 0001:00026db8       ?Init@CRadioCaps@@QAAJXZ   00127db8 f   RadioCaps.obj
 0001:00027264       ?SetDevCapsLockFacilities@CRadioCaps@@QAAXKH@Z 00128264 f   RadioCaps.obj
 0001:000272f8       ??0CResponse@@QAA@XZ       001282f8 f   response.obj
 0001:0002731c       ??1CResponse@@QAA@XZ       0012831c f   response.obj
 0001:00027338       ?SetBlob@CResponse@@QAAHQBXI@Z 00128338 f   response.obj
 0001:00027468       ?MakeError@CResponse@@QAAHJ@Z 00128468 f   response.obj
 0001:000274a8       ??0CNotificationData@@QAA@XZ 001284a8 f   response.obj
 0001:000274bc       ??1CNotificationData@@QAA@XZ 001284bc f   response.obj
 0001:000274c4       ?InitFromDWORDBlob@CNotificationData@@QAAHKK@Z 001284c4 f   response.obj
 0001:000275a4       ?InitFromRealBlob@CNotificationData@@QAAHKQBXI@Z 001285a4 f   response.obj
 0001:00027688       ??_ECEvent@@UAAPAXI@Z      00128688 f i rilhand.obj
 0001:00027688       ??_GCEvent@@UAAPAXI@Z      00128688 f i rilhand.obj
 0001:000276c4       ?Init@CUniquelyNamedEvent@@QAAHHHPAG@Z 001286c4 f i rilhand.obj
 0001:00027774       ??1CUniquelyNamedEvent@@UAA@XZ 00128774 f i rilhand.obj
 0001:00027798       ??_GEvent@@UAAPAXI@Z       00128798 f i rilhand.obj
 0001:00027798       ??_EEvent@@UAAPAXI@Z       00128798 f i rilhand.obj
 0001:000277d4       ??0CRilHandle@@QAA@XZ      001287d4 f   rilhand.obj
 0001:00027984       ?GetNextCmdID@CRilHandle@@QAAJXZ 00128984 f   rilhand.obj
 0001:000279c8       ?RegisterWithCPM@CRilHandle@@QAAHXZ 001289c8 f   rilhand.obj
 0001:00027a70       ?GetAPIInfo@CRilHandle@@QAAXW4APIID@@AAUAPIINFO@@@Z 00128a70 f   rilhand.obj
 0001:00027cb4       ?NotificationItemDtor@@YAXPAX@Z 00128cb4 f   rilhand.obj
 0001:00027cb8       ?FEnoughStorage@@YAHPAXK@Z 00128cb8 f   rilhand.obj
 0001:00027d28       ?ImgPref2Ids@@YAXKQAEQAG111@Z 00128d28 f   rilhand.obj
 0001:00027e24       ?Ids2ImgPref@@YAXPAKQAEQAG222@Z 00128e24 f   rilhand.obj
 0001:00027fd0       ?CheckVoiceMailBox@CRilHandle@@QAAXXZ 00128fd0 f   rilhand.obj
 0001:00028178       ?CloseSWI@CRilHandle@@QAAHXZ 00129178 f   rilhand.obj
 0001:000282ec       ?SwitchUnattendedMode@CRilHandle@@QAAXH@Z 001292ec f   rilhand.obj
 0001:0002840c       ?Add@?$CDblList@VCRilInstanceHandle@@@@QAAHQAVCRilInstanceHandle@@@Z 0012940c f i rilhand.obj
 0001:0002845c       ?Remove@?$CDblList@VCRilInstanceHandle@@@@QAAHQBVCRilInstanceHandle@@@Z 0012945c f i rilhand.obj
 0001:000284d8       ?Enum@?$CDblList@VCRilInstanceHandle@@@@QAAXQ6AHPAXK@ZK@Z 001294d8 f i rilhand.obj
 0001:00028554       ??0?$CUnboundedQueue@Urildrvnotification_tag@@@@QAA@P6AXPAX@Z@Z 00129554 f i rilhand.obj
 0001:000285ac       ??1?$CUnboundedQueue@Urildrvnotification_tag@@@@UAA@XZ 001295ac f i rilhand.obj
 0001:0002868c       ?Init@?$CUnboundedQueue@Urildrvnotification_tag@@@@QAAHK@Z 0012968c f i rilhand.obj
 0001:00028704       ?ConditionalGet@?$CUnboundedQueue@Urildrvnotification_tag@@@@QAAJQ6AHPAXK@ZKPAPAUrildrvnotification_tag@@@Z 00129704 f i rilhand.obj
 0001:000287ec       ??_G?$CUnboundedQueue@Urildrvnotification_tag@@@@UAAPAXI@Z 001297ec f i rilhand.obj
 0001:000287ec       ??_E?$CUnboundedQueue@Urildrvnotification_tag@@@@UAAPAXI@Z 001297ec f i rilhand.obj
 0001:00028810       ?GrowQueue@?$CUnboundedQueue@Urildrvnotification_tag@@@@IAAHXZ 00129810 f i rilhand.obj
 0001:0002886c       ??_GCUniquelyNamedEvent@@UAAPAXI@Z 0012986c f i rilhand.obj
 0001:0002886c       ??_ECUniquelyNamedEvent@@UAAPAXI@Z 0012986c f i rilhand.obj
 0001:000288a8       ?WaitForCommandOrCancel@CRilHandle@@QBAHXZ 001298a8 f   rilhand.obj
 0001:00028a0c       ?AddToList@CRilHandle@@QAAHQAVCRilInstanceHandle@@@Z 00129a0c f   rilhand.obj
 0001:00028a14       ?RemoveFromList@CRilHandle@@QAAHQAVCRilInstanceHandle@@@Z 00129a14 f   rilhand.obj
 0001:00028a1c       ??0CRilInstanceHandle@@QAA@XZ 00129a1c f   rilhand.obj
 0001:00028a60       ?Init@CRilInstanceHandle@@QAAHQAVCRilHandle@@@Z 00129a60 f   rilhand.obj
 0001:00028abc       ?GetNextNotification@CRilInstanceHandle@@QAAHAAUrildrvnotification_tag@@@Z 00129abc f   rilhand.obj
 0001:00028cec       ?CreateNotificationQueue@CRilInstanceHandle@@QAAHPBGPAEKPAK@Z 00129cec f   rilhand.obj
 0001:00028e24       ?DeInitializeSWI@CRilHandle@@QAAHH@Z 00129e24 f   rilhand.obj
 0001:00028ffc       ?Put@?$CUnboundedQueue@Urildrvnotification_tag@@@@QAAHQAUrildrvnotification_tag@@@Z 00129ffc f i rilhand.obj
 0001:00029098       ??1CRilInstanceHandle@@QAA@XZ 0012a098 f   rilhand.obj
 0001:00029108       ?Notify@CRilInstanceHandle@@QAAXKJQBXI@Z 0012a108 f   rilhand.obj
 0001:00029210       ?_Buynode@?$list@PAVCCommand@@V?$allocator@PAVCCommand@@@std@@@std@@IAAPAU_Node@?$_List_nod@PAVCCommand@@V?$allocator@PAVCCommand@@@std@@@2@XZ 0012a210 f i rilhand.obj
 0001:00029234       ?clear@?$list@PAVCCommand@@V?$allocator@PAVCCommand@@@std@@@std@@QAAXXZ 0012a234 f i rilhand.obj
 0001:00029278       ?NotifyHandle@@YAHPAXK@Z   0012a278 f   rilhand.obj
 0001:00029354       ?_Tidy@?$deque@PAVCCommand@@V?$allocator@PAVCCommand@@@std@@@std@@IAAXXZ 0012a354 f i rilhand.obj
 0001:000293e8       ?_Tidy@?$deque@PAUSwiNotifyVariant@@V?$allocator@PAUSwiNotifyVariant@@@std@@@std@@IAAXXZ 0012a3e8 f i rilhand.obj
 0001:0002947c       ?DeleteInstanceHandle@@YAHPAXK@Z 0012a47c f   rilhand.obj
 0001:000294f0       ?PreBroadcastNotification@CRilHandle@@QAAHPAVCNotificationData@@@Z 0012a4f0 f   rilhand.obj
 0001:00029e64       ?CheckDelayedRspCmdTimeout@CRilHandle@@QAAXXZ 0012ae64 f   rilhand.obj
 0001:0002a150       ?BroadcastNotification@CRilHandle@@QAAXPAVCNotificationData@@@Z 0012b150 f   rilhand.obj
 0001:0002a228       ?BroadcastRealBlobNotification@CRilHandle@@QAAHKQBXI@Z 0012b228 f   rilhand.obj
 0001:0002a3ac       ?BroadcastDWORDBlobNotification@CRilHandle@@QAAHKK@Z 0012b3ac f   rilhand.obj
 0001:0002a44c       ?SendReadyStateNotification@CRilHandle@@QAAXKH@Z 0012b44c f   rilhand.obj
 0001:0002a4cc       ?GeneralInitDone@CRilHandle@@QAAXH@Z 0012b4cc f   rilhand.obj
 0001:0002a704       ?InitializeSWI@CRilHandle@@QAAHXZ 0012b704 f   rilhand.obj
 0001:0002c270       ??0?$CThreadSafeQueue@PAVCCommand@@@@QAA@XZ 0012d270 f i rilhand.obj
 0001:0002c2e0       ??1?$CThreadSafeQueue@PAVCCommand@@@@QAA@XZ 0012d2e0 f i rilhand.obj
 0001:0002c330       ??0?$CThreadSafeQueue@PAUSwiNotifyVariant@@@@QAA@XZ 0012d330 f i rilhand.obj
 0001:0002c3a0       ??1?$CThreadSafeQueue@PAUSwiNotifyVariant@@@@QAA@XZ 0012d3a0 f i rilhand.obj
 0001:0002c3f8       ?LaunchThreads@CRilHandle@@QAAHXZ 0012d3f8 f   rilhand.obj
 0001:0002c6b4       ??1CRilHandle@@QAA@XZ      0012d6b4 f   rilhand.obj
 0001:0002c9c0       ?StartInit@CRilHandle@@QAAHXZ 0012d9c0 f   rilhand.obj
 0001:0002ce28       ?NdisGetIPAddress@CRilHandle@@QAAHKPAUSWI_STRUCT_IPConfigurationGobi@@@Z 0012de28 f   rilhandndis.obj
 0001:0002ce8c       ?NdisStop@CRilHandle@@AAAXXZ 0012de8c f   rilhandndis.obj
 0001:0002cef0       ?NdisCountEvents@CRilHandle@@AAAKXZ 0012def0 f   rilhandndis.obj
 0001:0002cf20       ?NdisGetFreeNdisEntry@CRilHandle@@QAAJPAK@Z 0012df20 f   rilhandndis.obj
 0001:0002cf7c       ?NdisRemoveNdisEntry@CRilHandle@@QAAXPAX@Z 0012df7c f   rilhandndis.obj
 0001:0002cfe4       ?NdisCidFromHandle@CRilHandle@@QAAJPAXPAK@Z 0012dfe4 f   rilhandndis.obj
 0001:0002d054       ?NdisHandleFromCid@CRilHandle@@QAAJKPAPAX@Z 0012e054 f   rilhandndis.obj
 0001:0002d0cc       ?NdisRilCallbacksFromCID@CRilHandle@@QAAXKPAPAXPAP6AXPAXPAUrilndispacket_tag@@@Z3PAP6AX1PAUrilndisstatus_tag@@@Z@Z 0012e0cc f   rilhandndis.obj
 0001:0002d168       ?NdisRemoveCallbacks@CRilHandle@@QAAXK@Z 0012e168 f   rilhandndis.obj
 0001:0002d1cc       ?NdisAddNdisEntry@CRilHandle@@QAAXKKPAXPBXPBUrilndisgprscontext_tag@@@Z 0012e1cc f   rilhandndis.obj
 0001:0002d22c       ?myinet_addr@@YAKPBEE@Z    0012e22c f   rilhandndis.obj
 0001:0002d26c       ?myinet_ipv6addr@@YA?AUrilndisipv6addr_tag@@PBEE@Z 0012e26c f   rilhandndis.obj
 0001:0002d2a4       ?NdisConvertConfig@CRilHandle@@QAAXPBUoemndisconfiguration_tag@@PAUrilndisipconfig_tag@@@Z 0012e2a4 f   rilhandndis.obj
 0001:0002d508       ?NdisAddNotifyEvent@CRilHandle@@QAAJPAX@Z 0012e508 f   rilhandndis.obj
 0001:0002d58c       ?NdisRemoveNotifyEvent@CRilHandle@@QAAJPAX@Z 0012e58c f   rilhandndis.obj
 0001:0002d650       ?NdisInterfaceReceiveEvent@CRilHandle@@QAAHPAXPAUoemndisevent_tag@@PAH@Z 0012e650 f   rilhandndis.obj
 0001:0002d6b0       ?NdisInterfaceTransmitEvent@CRilHandle@@QAAHPAXPBUoemndisevent_tag@@@Z 0012e6b0 f   rilhandndis.obj
 0001:0002d7a0       ??0AsyncResponse@@QAA@XZ   0012e7a0 f   rilhandndis.obj
 0001:0002d7bc       ??1AsyncResponse@@QAA@XZ   0012e7bc f   rilhandndis.obj
 0001:0002d808       ?AddListItem@AsyncResponse@@AAAJPAUasyncresponse_tag@@@Z 0012e808 f   rilhandndis.obj
 0001:0002d874       ?RemoveListItem@AsyncResponse@@AAAJPAUasyncresponse_tag@@@Z 0012e874 f   rilhandndis.obj
 0001:0002d920       ??0NdisRxPacketQueue@@QAA@XZ 0012e920 f   rilhandndis.obj
 0001:0002d93c       ??1NdisRxPacketQueue@@QAA@XZ 0012e93c f   rilhandndis.obj
 0001:0002d988       ?FindPacket@NdisRxPacketQueue@@QAAPAUrilndispacket_tag@@XZ 0012e988 f   rilhandndis.obj
 0001:0002d9dc       ?NdisShutdownConnection@CRilHandle@@QAAXPAXH@Z 0012e9dc f   rilhandndis.obj
 0001:0002dab0       ?AddCommand@AsyncResponse@@QAAJPAUoemndisapireference_tag@@@Z 0012eab0 f   rilhandndis.obj
 0001:0002db10       ?RemoveCommand@AsyncResponse@@QAAJJ@Z 0012eb10 f   rilhandndis.obj
 0001:0002db84       ?ProcessCommand@AsyncResponse@@QAAHPBUoemndisapireference_tag@@@Z 0012eb84 f   rilhandndis.obj
 0001:0002dcd0       ?_Lbound@?$_Tree@V?$_Tmap_traits@KU__Fail_Cmd_Data_tag@@U?$less@K@std@@V?$allocator@U?$pair@$$CBKU__Fail_Cmd_Data_tag@@@std@@@3@$0A@@std@@@std@@IBAPAU_Node@?$_Tree_nod@V?$_Tmap_traits@KU__Fail_Cmd_Data_tag@@U?$less@K@std@@V?$allocator@U?$pair@$$CBKU__Fail_Cmd_Data_tag@@@std@@@3@$0A@@std@@@2@ABK@Z 0012ecd0 f i rilhandndis.obj
 0001:0002dd28       ?_Dec@const_iterator@?$_Tree@V?$_Tmap_traits@KU__Fail_Cmd_Data_tag@@U?$less@K@std@@V?$allocator@U?$pair@$$CBKU__Fail_Cmd_Data_tag@@@std@@@3@$0A@@std@@@std@@QAAXXZ 0012ed28 f i rilhandndis.obj
 0001:0002ddf8       ?NdisCloseAllConnections@CRilHandle@@QAAXH@Z 0012edf8 f   rilhandndis.obj
 0001:0002de3c       ?NdisNotifyThread@CRilHandle@@QAAKXZ 0012ee3c f   rilhandndis.obj
 0001:0002ead0       ?NdisAllocateCommand@CRilHandle@@QAAJW4oemndiseventtype_tag@@PAX1@Z 0012fad0 f   rilhandndis.obj
 0001:0002eb44       ?NdisNotifyThreadProc@@YAKPAX@Z 0012fb44 f   rilhandndis.obj
 0001:0002eb48       ?_Buynode@?$_Tree@V?$_Tmap_traits@KU__Fail_Cmd_Data_tag@@U?$less@K@std@@V?$allocator@U?$pair@$$CBKU__Fail_Cmd_Data_tag@@@std@@@3@$0A@@std@@@std@@IAAPAU_Node@?$_Tree_nod@V?$_Tmap_traits@KU__Fail_Cmd_Data_tag@@U?$less@K@std@@V?$allocator@U?$pair@$$CBKU__Fail_Cmd_Data_tag@@@std@@@3@$0A@@std@@@2@PAU342@00ABU?$pair@$$CBKU__Fail_Cmd_Data_tag@@@2@D@Z 0012fb48 f i rilhandndis.obj
 0001:0002eba0       ?NdisStart@CRilHandle@@AAAHXZ 0012fba0 f   rilhandndis.obj
 0001:0002ec58       ?_Insert@?$_Tree@V?$_Tmap_traits@KU__Fail_Cmd_Data_tag@@U?$less@K@std@@V?$allocator@U?$pair@$$CBKU__Fail_Cmd_Data_tag@@@std@@@3@$0A@@std@@@std@@IAA?AViterator@12@_NPAU_Node@?$_Tree_nod@V?$_Tmap_traits@KU__Fail_Cmd_Data_tag@@U?$less@K@std@@V?$allocator@U?$pair@$$CBKU__Fail_Cmd_Data_tag@@@std@@@3@$0A@@std@@@2@ABU?$pair@$$CBKU__Fail_Cmd_Data_tag@@@2@@Z 0012fc58 f i rilhandndis.obj
 0001:0002eeb0       ?insert@?$_Tree@V?$_Tmap_traits@KU__Fail_Cmd_Data_tag@@U?$less@K@std@@V?$allocator@U?$pair@$$CBKU__Fail_Cmd_Data_tag@@@std@@@3@$0A@@std@@@std@@QAA?AU?$pair@Viterator@?$_Tree@V?$_Tmap_traits@KU__Fail_Cmd_Data_tag@@U?$less@K@std@@V?$allocator@U?$pair@$$CBKU__Fail_Cmd_Data_tag@@@std@@@3@$0A@@std@@@std@@_N@2@ABU?$pair@$$CBKU__Fail_Cmd_Data_tag@@@2@@Z 0012feb0 f i rilhandndis.obj
 0001:0002efe8       ?insert@?$_Tree@V?$_Tmap_traits@KU__Fail_Cmd_Data_tag@@U?$less@K@std@@V?$allocator@U?$pair@$$CBKU__Fail_Cmd_Data_tag@@@std@@@3@$0A@@std@@@std@@QAA?AViterator@12@V312@ABU?$pair@$$CBKU__Fail_Cmd_Data_tag@@@2@@Z 0012ffe8 f i rilhandndis.obj
 0001:0002f260       ??A?$map@KU__Fail_Cmd_Data_tag@@U?$less@K@std@@V?$allocator@U?$pair@$$CBKU__Fail_Cmd_Data_tag@@@std@@@3@@std@@QAAAAU__Fail_Cmd_Data_tag@@ABK@Z 00130260 f i rilhandndis.obj
 0001:0002f340       ?PreExecNDISCmd@CRilInstanceHandle@@AAAJK@Z 00130340 f   rilhandndis.obj
 0001:0002f3c0       ?NdisSetGPRSContextActivated@CRilInstanceHandle@@QAAJPBV1@PBUrilndisgprscontext_tag@@@Z 001303c0 f   rilhandndis.obj
 0001:0002f848       ?RILDrv_GetAudioDevices@@YAJK@Z 00130848 f   rilmain.obj
 0001:0002f894       ?RILDrv_SetHideConnectedIdStatus@@YAJKK@Z 00130894 f   rilmain.obj
 0001:0002f8e0       DllMain                    001308e0 f   rilmain.obj
 0001:0002f9d4       ?RIL_Deinit@@YAHK@Z        001309d4 f   rilmain.obj
 0001:0002fa94       ?RIL_Read@@YAKKPAXK@Z      00130a94 f   rilmain.obj
 0001:0002fa9c       ?RIL_Write@@YAKKPBXK@Z     00130a9c f   rilmain.obj
 0001:0002faa4       ?RIL_Seek@@YAKKJK@Z        00130aa4 f   rilmain.obj
 0001:0002faac       ?RIL_PowerDown@@YAXK@Z     00130aac f   rilmain.obj
 0001:0002fab0       ?RIL_PowerUp@@YAXK@Z       00130ab0 f   rilmain.obj
 0001:0002fab4       ?ExtractHandle@@YAQAVCRilInstanceHandle@@K@Z 00130ab4 f   rilmain.obj
 0001:0002fb1c       ?hex2bin@@YAEEE@Z          00130b1c f   rilmain.obj
 0001:0002fb78       ?DoFirmwareUpgrade@CRadio@@QAAHH@Z 00130b78 f   rilmain.obj
 0001:000304f4       ?Enum@?$CDblList@VCCommand@@@@QAAXQ6AHPAXK@ZK@Z 001314f4 f i rilmain.obj
 0001:00030578       ?RIL_Init@@YAKK@Z          00131578 f   rilmain.obj
 0001:0003078c       ?RIL_Open@@YAKKKK@Z        0013178c f   rilmain.obj
 0001:000308e0       ?RILDrv_GetNextNotification@@YAJKPAUrildrvnotification_tag@@@Z 001318e0 f   rilmain.obj
 0001:00030928       ?RIL_IOControl@@YAHKKPAEK0KPAK@Z 00131928 f   rilmain.obj
 0001:00032f38       ?ClearCmdHandle@@YAHPAXK@Z 00133f38 f   rilmain.obj
 0001:0003305c       ?RIL_Close@@YAHK@Z         0013405c f   rilmain.obj
 0001:00033198       ?SwiGetProcAddress@@YAP6AHXZPAUHINSTANCE__@@PBG@Z 00134198 f   SDK7Wrapper.obj
 0001:000331f8       ?Cleanup@CSDK7@@QAAXXZ     001341f8 f   SDK7Wrapper.obj
 0001:000334fc       ?Initialize@CSDK7@@QAA_NXZ 001344fc f   SDK7Wrapper.obj
 0001:0003421c       ??0CSDK7@@QAA@XZ           0013521c f   SDK7Wrapper.obj
 0001:00034248       ??1CSDK7@@QAA@XZ           00135248 f   SDK7Wrapper.obj
 0001:0003424c       ?RILDrv_GetPhoneLockedState@@YAJK@Z 0013524c f   secur.obj
 0001:000342b0       ?GetPhoneLockedState@CRadio@@QAAJPAVCResponse@@@Z 001352b0 f   secur.obj
 0001:000343fc       ?RILDrv_UnlockPhone@@YAJKPBD0@Z 001353fc f   secur.obj
 0001:0003454c       ?UnlockPhone@CRadio@@QAAJPAVCResponse@@PAX@Z 0013554c f   secur.obj
 0001:00034730       ?RILDrv_ChangeLockingPassword@@YAJKKKPBD0@Z 00135730 f   secur.obj
 0001:00034974       ?ChangeLockingPassword@CRadio@@QAAJPAVCResponse@@PAX@Z 00135974 f   secur.obj
 0001:00034b7c       ?RILDrv_SetLockingStatus@@YAJKKPBDK@Z 00135b7c f   secur.obj
 0001:00034c68       ?SetLockingStatus@CRadio@@QAAJPAVCResponse@@PAX@Z 00135c68 f   secur.obj
 0001:00034dc8       ?RILDrv_GetLockingStatus@@YAJKKPBD@Z 00135dc8 f   secur.obj
 0001:00034eac       ?GetLockingStatus@CRadio@@QAAJPAVCResponse@@PAX@Z 00135eac f   secur.obj
 0001:00035018       ?RILDrv_GetUserIdentity@@YAJK@Z 00136018 f   secur.obj
 0001:00035080       ?GetUserIdentity@CRadio@@QAAJPAVCResponse@@@Z 00136080 f   secur.obj
 0001:00035320       ?RILDrv_GetCallBarringStatus@@YAJKKKPBD@Z 00136320 f   secur.obj
 0001:000354c0       ?RILDrv_SetCallBarringStatus@@YAJKKKPBDK@Z 001364c0 f   secur.obj
 0001:000356f8       ?RILDrv_ChangeCallBarringPassword@@YAJKKPBD0@Z 001366f8 f   secur.obj
 0001:000358ec       ?GetCallBarringStatus@CRadio@@QAAJPAVCResponse@@PAX@Z 001368ec f   secur.obj
 0001:00035a74       ?SetCallBarringStatus@CRadio@@QAAJPAVCResponse@@PAX@Z 00136a74 f   secur.obj
 0001:00035c34       ?ChangeCallBarringPassword@CRadio@@QAAJPAVCResponse@@PAX@Z 00136c34 f   secur.obj
 0001:00036024       ?ParseCellBroadcastMessage@@YAJPBEIAAUrilmessage_tag@@@Z 00137024 f   smscb.obj
 0001:000361c8       ?RILDrv_GetCallerIdSettings@@YAJK@Z 001371c8 f   supsvc.obj
 0001:00036264       ?RILDrv_SetCallerIdStatus@@YAJKK@Z 00137264 f   supsvc.obj
 0001:00036368       ?RILDrv_GetHideIdSettings@@YAJK@Z 00137368 f   supsvc.obj
 0001:000363c8       ?RILDrv_SetHideIdStatus@@YAJKK@Z 001373c8 f   supsvc.obj
 0001:000364f4       ?RILDrv_GetDialedIdSettings@@YAJK@Z 001374f4 f   supsvc.obj
 0001:00036594       ?RILDrv_SetDialedIdStatus@@YAJKK@Z 00137594 f   supsvc.obj
 0001:000366d0       ?RILDrv_GetHideConnectedIdSettings@@YAJK@Z 001376d0 f   supsvc.obj
 0001:00036730       ?RILDrv_GetCallForwardingSettings@@YAJKKK@Z 00137730 f   supsvc.obj
 0001:000368b0       ?RILDrv_AddCallForwarding@@YAJKKPBUrilcallforwardingsettings_tag@@@Z 001378b0 f   supsvc.obj
 0001:00036a94       ?RILDrv_RemoveCallForwarding@@YAJKKK@Z 00137a94 f   supsvc.obj
 0001:00036c0c       ?RILDrv_SetCallForwardingStatus@@YAJKKKK@Z 00137c0c f   supsvc.obj
 0001:00036de4       ?RILDrv_GetCallWaitingSettings@@YAJKK@Z 00137de4 f   supsvc.obj
 0001:00036f50       ?RILDrv_SetCallWaitingStatus@@YAJKKK@Z 00137f50 f   supsvc.obj
 0001:000372c4       ?RILDrv_SendSupServiceData@@YAJKPBEK@Z 001382c4 f   supsvc.obj
 0001:0003748c       ?RILDrv_CancelSupServiceDataSession@@YAJK@Z 0013848c f   supsvc.obj
 0001:0003752c       ?GetCallerIdSettings@CRadio@@QAAJPAVCResponse@@@Z 0013852c f   supsvc.obj
 0001:0003765c       ?SetCallerIdStatus@CRadio@@QAAJPAVCResponse@@PAX@Z 0013865c f   supsvc.obj
 0001:00037704       ?GetHideIdSettings@CRadio@@QAAJPAVCResponse@@@Z 00138704 f   supsvc.obj
 0001:00037920       ?SetHideIdStatus@CRadio@@QAAJPAVCResponse@@PAX@Z 00138920 f   supsvc.obj
 0001:00037a70       ?GetDialedIdSettings@CRadio@@QAAJPAVCResponse@@@Z 00138a70 f   supsvc.obj
 0001:00037bbc       ?SetDialedIdStatus@CRadio@@QAAJPAVCResponse@@PAX@Z 00138bbc f   supsvc.obj
 0001:00037bd4       ?GetCallForwardingSettings@CRadio@@QAAJPAVCResponse@@PAX@Z 00138bd4 f   supsvc.obj
 0001:000380a4       ?AddCallForwarding@CRadio@@QAAJPAVCResponse@@PAX@Z 001390a4 f   supsvc.obj
 0001:00038318       ?SetCallForwarding@CRadio@@QAAJPAVCResponse@@PAX@Z 00139318 f   supsvc.obj
 0001:0003852c       ?RemoveCallForwarding@CRadio@@QAAJPAVCResponse@@PAX@Z 0013952c f   supsvc.obj
 0001:00038698       ?GetCallWaitingSettings@CRadio@@QAAJPAVCResponse@@PAX@Z 00139698 f   supsvc.obj
 0001:00038904       ?SetCallWaitingStatus@CRadio@@QAAJPAVCResponse@@PAX@Z 00139904 f   supsvc.obj
 0001:00038a94       ?SendUSSD@CRadio@@QAAXPAG@Z 00139a94 f   supsvc.obj
 0001:00038dbc       ?CancelSupServiceDataSession@CRadio@@QAAJPAVCResponse@@@Z 00139dbc f   supsvc.obj
 0001:00038e44       ?GetHideConnectedIdSettings@CRadio@@QAAJPAVCResponse@@@Z 00139e44 f   supsvc.obj
 0001:00038f90       ?SetEnum@CRadio@@QAAJPAD@Z 00139f90 f   supsvc.obj
 0001:00039080       ?ClearEnum@CRadio@@QAAJXZ  0013a080 f   supsvc.obj
 0001:00039164       ?SendSupSvcsThreadProc@@YAKPAX@Z 0013a164 f   supsvc.obj
 0001:00039210       ?SendSupServiceData@CRadio@@QAAJPAVCResponse@@PAX@Z 0013a210 f   supsvc.obj
 0001:000393a8       ?_tcsncpyz@@YAPAGQAGQBGI@Z 0013a3a8 f   toolbox.obj
 0001:000393f4       ?_tcsncatz@@YAPAGQAGQBGI@Z 0013a3f4 f   toolbox.obj
 0001:00039450       ?strncpyz@@YAPADQADQBDI@Z  0013a450 f   toolbox.obj
 0001:0003949c       ?_sntprintfz@@YAHQAGIQBGZZ 0013a49c f   toolbox.obj
 0001:000394fc       ?_snprintfz@@YAHQADIQBDZZ  0013a4fc f   toolbox.obj
 0001:0003955c       ?GetRegistryDWORD@@YA_NQAUHKEY__@@QBG1QAK@Z 0013a55c f   toolbox.obj
 0001:00039618       ?SetRegistryDWORD@@YA_NQAUHKEY__@@QBG1K@Z 0013a618 f   toolbox.obj
 0001:000396b8       ??0AnsiString@@QAA@QBGG@Z  0013a6b8 f   toolbox.obj
 0001:000397b0       ??1AnsiString@@QAA@XZ      0013a7b0 f   toolbox.obj
 0001:000397c8       ??0WideString@@QAA@QBDD@Z  0013a7c8 f   toolbox.obj
 0001:000398ac       ??1WideString@@QAA@XZ      0013a8ac f   toolbox.obj
 0001:000398c4       ??0VerboseString@@QAA@QBGGG@Z 0013a8c4 f   toolbox.obj
 0001:00039a38       ??1VerboseString@@QAA@XZ   0013aa38 f   toolbox.obj
 0001:00039a50       ??0CCheckPoint@@QAA@XZ     0013aa50 f   toolbox.obj
 0001:00039a78       ??1CCheckPoint@@QAA@XZ     0013aa78 f   toolbox.obj
 0001:00039ac4       ?Init@CCheckPoint@@QAA_NI@Z 0013aac4 f   toolbox.obj
 0001:00039b2c       ?Reached@CCheckPoint@@QAAXXZ 0013ab2c f   toolbox.obj
 0001:00039b74       ?Wait@CCheckPoint@@QAA_NK@Z 0013ab74 f   toolbox.obj
 0001:00039bd4       ?bsearch@@YAPAXPBX0IIP6AH00@Z@Z 0013abd4 f   toolbox.obj
 0001:00039c88       ?WaitForSingleObjectReset@@YAKPAXK@Z 0013ac88 f   toolbox.obj
 0001:00039d04       ?ValueFromFlag@@YAHIQBULISTVALUEMAP@@IAAI@Z 0013ad04 f   util.obj
 0001:00039d50       ?StringFromFlag@@YAHIQBULISTSTRINGMAP@@IAAPBD@Z 0013ad50 f   util.obj
 0001:00039d9c       ?UpdateStatStore@@YAXXZ    0013ad9c f   util.obj
 0001:00039e30       ??0CBuffer@@QAA@XZ         0013ae30 f   util.obj
 0001:00039e44       ??1CBuffer@@QAA@XZ         0013ae44 f   util.obj
 0001:00039e54       ?InitializeCarrierIndex@CRilHandle@@QAAXXZ 0013ae54 f   util.obj
 0001:00039fe4       ?UpdateLocalCarrierIndex@CRilHandle@@QAAXW4SWI_TYPE_CarrierID@@@Z 0013afe4 f   util.obj
 0001:0003a3c0       ?MessageBoxFunction@@YAIPAX@Z 0013b3c0 f   util.obj
 0001:0003a434       ?MessageBoxOnSeparateThread@@YAXPBG0I@Z 0013b434 f   util.obj
 0001:0003a4ec       ?ConvertToSwiAudioMode@@YAEK@Z 0013b4ec f   voice.obj
 0001:0003a5b4       ?RILDrv_GetAudioGain@@YAJK@Z 0013b5b4 f   voice.obj
 0001:0003a614       ?RILDrv_SetAudioGain@@YAJKPBUrilgaininfo_tag@@@Z 0013b614 f   voice.obj
 0001:0003a70c       ?RILDrv_SetAudioDevices@@YAJKPBUrilaudiodeviceinfo_tag@@@Z 0013b70c f   voice.obj
 0001:0003a79c       ?RILDrv_GetAudioMuting@@YAJK@Z 0013b79c f   voice.obj
 0001:0003a7fc       ?RILDrv_SetAudioMuting@@YAJKH@Z 0013b7fc f   voice.obj
 0001:0003a864       ?GetAudioGain@CRadio@@QAAJPAVCResponse@@@Z 0013b864 f   voice.obj
 0001:0003a8d0       ?SetAudioGain@CRadio@@QAAJPAVCResponse@@PAX@Z 0013b8d0 f   voice.obj
 0001:0003ac84       ?SetAudioDevices@CRadio@@QAAJPAVCResponse@@PAX@Z 0013bc84 f   voice.obj
 0001:0003affc       ?GetAudioMuting@CRadio@@QAAJPAVCResponse@@@Z 0013bffc f   voice.obj
 0001:0003b070       ?ProgramAudioParameter9090@CRadio@@QAAJXZ 0013c070 f   voice.obj
 0001:0003c100       ?HWSetMicMute@CRadio@@QAAJH@Z 0013d100 f   voice.obj
 0001:0003c2d0       ?HWSetSpeakerMute@CRadio@@QAAJH@Z 0013d2d0 f   voice.obj
 0001:0003c484       ?HWPlayAudioTone@CRadio@@QAAJPAEPAG@Z 0013d484 f   voice.obj
 0001:0003c5b8       ?SetAudioMuting@CRadio@@QAAJPAVCResponse@@PAX@Z 0013d5b8 f   voice.obj
 0001:0003c644       ?ProgramAudioParameterSwiM2MAV@CRadio@@QAAJXZ 0013d644 f   voice.obj
 0001:0003d160       ?ProgramAudioParameter@CRadio@@QAAJXZ 0013e160 f   voice.obj
 0001:0003d1c8       ValidateAPIPermission      0013e1c8 f   ossvcs:ossvcs.dll
 0001:0003d1d8       GetStatStore               0013e1d8 f   ossvcs:ossvcs.dll
 0001:0003d1e8       _DllMainCRTStartup         0013e1e8 f   corelibc:pegdmain.obj
 0001:0003d280       __security_check_cookie    0013e280     corelibc:armsecgs.obj
 0001:0003d294       __gsfailure                0013e294     corelibc:armsecgs.obj
 0001:0003d2d8       _onexit                    0013e2d8 f   corelibc:onexit.obj
 0001:0003d384       atexit                     0013e384 f   corelibc:onexit.obj
 0001:0003d3a4       _cinit                     0013e3a4 f   corelibc:crt0dat.obj
 0001:0003d514       _cexit                     0013e514 f   corelibc:crt0dat.obj
 0001:0003d530       __security_init_cookie     0013e530 f   corelibc:seccinit.obj
 0001:0003d580       PHGetFeatureLevel          0013e580 f   ccoreutl:ccoreutl.dll
 0001:0003d590       htonl                      0013e590 f   winsock:WINSOCK.dll
 0001:0003d5a0       EventModify                0013e5a0 f   coredll:COREDLL.dll
 0001:0003d5b0       EnterCriticalSection       0013e5b0 f   coredll:COREDLL.dll
 0001:0003d5c0       LeaveCriticalSection       0013e5c0 f   coredll:COREDLL.dll
 0001:0003d5d0       strlen                     0013e5d0 f   coredll:COREDLL.dll
 0001:0003d5e0       ??0exception@std@@QAA@PBD@Z 0013e5e0 f   coredll:COREDLL.dll
 0001:0003d5f0       ?what@exception@std@@UBAPBDXZ 0013e5f0 f   coredll:COREDLL.dll
 0001:0003d600       ??1exception@std@@UAA@XZ   0013e600 f   coredll:COREDLL.dll
 0001:0003d610       ??3@YAXPAX@Z               0013e610 f   coredll:COREDLL.dll
 0001:0003d620       SetThreadPriority          0013e620 f   coredll:COREDLL.dll
 0001:0003d630       ??2@YAPAXI@Z               0013e630 f   coredll:COREDLL.dll
 0001:0003d640       __CxxThrowException        0013e640 f   coredll:COREDLL.dll
 0001:0003d650       ??_7type_info@@6B@         0013e650 f   coredll:COREDLL.dll
 0001:0003d660       ??0exception@std@@QAA@ABV01@@Z 0013e660 f   coredll:COREDLL.dll
 0001:0003d670       ??0exception@std@@QAA@XZ   0013e670 f   coredll:COREDLL.dll
 0001:0003d680       GetTickCount               0013e680 f   coredll:COREDLL.dll
 0001:0003d690       wcsstr                     0013e690 f   coredll:COREDLL.dll
 0001:0003d6a0       ??_V@YAXPAX@Z              0013e6a0 f   coredll:COREDLL.dll
 0001:0003d6b0       ??_U@YAPAXI@Z              0013e6b0 f   coredll:COREDLL.dll
 0001:0003d6c0       memset                     0013e6c0 f   coredll:COREDLL.dll
 0001:0003d6d0       Sleep                      0013e6d0 f   coredll:COREDLL.dll
 0001:0003d6e0       _isctype                   0013e6e0 f   coredll:COREDLL.dll
 0001:0003d6f0       wcscpy                     0013e6f0 f   coredll:COREDLL.dll
 0001:0003d700       wcslen                     0013e700 f   coredll:COREDLL.dll
 0001:0003d710       memcpy                     0013e710 f   coredll:COREDLL.dll
 0001:0003d720       _wcsicmp                   0013e720 f   coredll:COREDLL.dll
 0001:0003d730       NKDbgPrintfW               0013e730 f   coredll:COREDLL.dll
 0001:0003d740       CloseHandle                0013e740 f   coredll:COREDLL.dll
 0001:0003d750       EscapeCommFunction         0013e750 f   coredll:COREDLL.dll
 0001:0003d760       MultiByteToWideChar        0013e760 f   coredll:COREDLL.dll
 0001:0003d770       swprintf                   0013e770 f   coredll:COREDLL.dll
 0001:0003d780       strchr                     0013e780 f   coredll:COREDLL.dll
 0001:0003d790       CreateThread               0013e790 f   coredll:COREDLL.dll
 0001:0003d7a0       WriteFile                  0013e7a0 f   coredll:COREDLL.dll
 0001:0003d7b0       PurgeComm                  0013e7b0 f   coredll:COREDLL.dll
 0001:0003d7c0       SetCommMask                0013e7c0 f   coredll:COREDLL.dll
 0001:0003d7d0       SetCommTimeouts            0013e7d0 f   coredll:COREDLL.dll
 0001:0003d7e0       GetCommModemStatus         0013e7e0 f   coredll:COREDLL.dll
 0001:0003d7f0       SetCommState               0013e7f0 f   coredll:COREDLL.dll
 0001:0003d800       CreateFileW                0013e800 f   coredll:COREDLL.dll
 0001:0003d810       MessageBoxW                0013e810 f   coredll:COREDLL.dll
 0001:0003d820       ShowWindow                 0013e820 f   coredll:COREDLL.dll
 0001:0003d830       FindWindowW                0013e830 f   coredll:COREDLL.dll
 0001:0003d840       strcat                     0013e840 f   coredll:COREDLL.dll
 0001:0003d850       SetSystemPowerState        0013e850 f   coredll:COREDLL.dll
 0001:0003d860       wcscmp                     0013e860 f   coredll:COREDLL.dll
 0001:0003d870       CreateProcessW             0013e870 f   coredll:COREDLL.dll
 0001:0003d880       strcpy                     0013e880 f   coredll:COREDLL.dll
 0001:0003d890       CreateMutexW               0013e890 f   coredll:COREDLL.dll
 0001:0003d8a0       wcscat                     0013e8a0 f   coredll:COREDLL.dll
 0001:0003d8b0       GetLastError               0013e8b0 f   coredll:COREDLL.dll
 0001:0003d8c0       TerminateThread            0013e8c0 f   coredll:COREDLL.dll
 0001:0003d8d0       WaitForSingleObject        0013e8d0 f   coredll:COREDLL.dll
 0001:0003d8e0       DeviceIoControl            0013e8e0 f   coredll:COREDLL.dll
 0001:0003d8f0       ReadFile                   0013e8f0 f   coredll:COREDLL.dll
 0001:0003d900       WaitCommEvent              0013e900 f   coredll:COREDLL.dll
 0001:0003d910       __C_specific_handler       0013e910 f   coredll:COREDLL.dll
 0001:0003d920       WaitForMultipleObjects     0013e920 f   coredll:COREDLL.dll
 0001:0003d930       wcsncpy                    0013e930 f   coredll:COREDLL.dll
 0001:0003d940       wcschr                     0013e940 f   coredll:COREDLL.dll
 0001:0003d950       _snwprintf                 0013e950 f   coredll:COREDLL.dll
 0001:0003d960       WideCharToMultiByte        0013e960 f   coredll:COREDLL.dll
 0001:0003d970       wsprintfW                  0013e970 f   coredll:COREDLL.dll
 0001:0003d980       strncat                    0013e980 f   coredll:COREDLL.dll
 0001:0003d990       _snprintf                  0013e990 f   coredll:COREDLL.dll
 0001:0003d9a0       wcsncat                    0013e9a0 f   coredll:COREDLL.dll
 0001:0003d9b0       _wtol                      0013e9b0 f   coredll:COREDLL.dll
 0001:0003d9c0       strncpy                    0013e9c0 f   coredll:COREDLL.dll
 0001:0003d9d0       ??_M@YAXPAXIHP6AX0@Z@Z     0013e9d0 f   coredll:COREDLL.dll
 0001:0003d9e0       ??_L@YAXPAXIHP6AX0@Z1@Z    0013e9e0 f   coredll:COREDLL.dll
 0001:0003d9f0       KernelIoControl            0013e9f0 f   coredll:COREDLL.dll
 0001:0003da00       InitializeCriticalSection  0013ea00 f   coredll:COREDLL.dll
 0001:0003da10       DeleteCriticalSection      0013ea10 f   coredll:COREDLL.dll
 0001:0003da20       iswctype                   0013ea20 f   coredll:COREDLL.dll
 0001:0003da30       FileTimeToSystemTime       0013ea30 f   coredll:COREDLL.dll
 0001:0003da40       LocalFileTimeToFileTime    0013ea40 f   coredll:COREDLL.dll
 0001:0003da50       SystemTimeToFileTime       0013ea50 f   coredll:COREDLL.dll
 0001:0003da60       sprintf                    0013ea60 f   coredll:COREDLL.dll
 0001:0003da70       _itoa                      0013ea70 f   coredll:COREDLL.dll
 0001:0003da80       atoi                       0013ea80 f   coredll:COREDLL.dll
 0001:0003da90       FreeLibrary                0013ea90 f   coredll:COREDLL.dll
 0001:0003daa0       wcsncmp                    0013eaa0 f   coredll:COREDLL.dll
 0001:0003dab0       RegCreateKeyExW            0013eab0 f   coredll:COREDLL.dll
 0001:0003dac0       RegCloseKey                0013eac0 f   coredll:COREDLL.dll
 0001:0003dad0       RegSetValueExW             0013ead0 f   coredll:COREDLL.dll
 0001:0003dae0       RegOpenKeyExW              0013eae0 f   coredll:COREDLL.dll
 0001:0003daf0       StringCchPrintfW           0013eaf0 f   coredll:COREDLL.dll
 0001:0003db00       strstr                     0013eb00 f   coredll:COREDLL.dll
 0001:0003db10       wcstok                     0013eb10 f   coredll:COREDLL.dll
 0001:0003db20       RegQueryValueExW           0013eb20 f   coredll:COREDLL.dll
 0001:0003db30       CreateEventW               0013eb30 f   coredll:COREDLL.dll
 0001:0003db40       _itow                      0013eb40 f   coredll:COREDLL.dll
 0001:0003db50       GetProcAddressW            0013eb50 f   coredll:COREDLL.dll
 0001:0003db60       LoadLibraryW               0013eb60 f   coredll:COREDLL.dll
 0001:0003db70       _wcsupr                    0013eb70 f   coredll:COREDLL.dll
 0001:0003db80       CeSetThreadPriority        0013eb80 f   coredll:COREDLL.dll
 0001:0003db90       SetSystemTime              0013eb90 f   coredll:COREDLL.dll
 0001:0003dba0       LocalFree                  0013eba0 f   coredll:COREDLL.dll
 0001:0003dbb0       TryEnterCriticalSection    0013ebb0 f   coredll:COREDLL.dll
 0001:0003dbc0       PowerPolicyNotify          0013ebc0 f   coredll:COREDLL.dll
 0001:0003dbd0       memmove                    0013ebd0 f   coredll:COREDLL.dll
 0001:0003dbe0       LocalAlloc                 0013ebe0 f   coredll:COREDLL.dll
 0001:0003dbf0       swscanf                    0013ebf0 f   coredll:COREDLL.dll
 0001:0003dc00       CeSafeCopyMemory           0013ec00 f   coredll:COREDLL.dll
 0001:0003dc10       free                       0013ec10 f   coredll:COREDLL.dll
 0001:0003dc20       malloc                     0013ec20 f   coredll:COREDLL.dll
 0001:0003dc30       wcstoul                    0013ec30 f   coredll:COREDLL.dll
 0001:0003dc40       wcstombs                   0013ec40 f   coredll:COREDLL.dll
 0001:0003dc50       SystemIdleTimerReset       0013ec50 f   coredll:COREDLL.dll
 0001:0003dc60       OutputDebugStringW         0013ec60 f   coredll:COREDLL.dll
 0001:0003dc70       _vsnwprintf                0013ec70 f   coredll:COREDLL.dll
 0001:0003dc80       _vsnprintf                 0013ec80 f   coredll:COREDLL.dll
 0001:0003dc90       LocalReAlloc               0013ec90 f   coredll:COREDLL.dll
 0001:0003dca0       strcmp                     0013eca0 f   coredll:COREDLL.dll
 0001:0003dcb0       CopyFileW                  0013ecb0 f   coredll:COREDLL.dll
 0001:0003dcc0       DeleteFileW                0013ecc0 f   coredll:COREDLL.dll
 0001:0003dcd0       SetFileAttributesW         0013ecd0 f   coredll:COREDLL.dll
 0001:0003dce0       MoveFileW                  0013ece0 f   coredll:COREDLL.dll
 0001:0003dcf0       strtoul                    0013ecf0 f   coredll:COREDLL.dll
 0001:0003dd00       strtok                     0013ed00 f   coredll:COREDLL.dll
 0001:0003dd10       RegEnumKeyExW              0013ed10 f   coredll:COREDLL.dll
 0001:0003dd20       __report_gsfailure         0013ed20 f   coredll:COREDLL.dll
 0001:0003dd30       LocalSize                  0013ed30 f   coredll:COREDLL.dll
 0001:0003dd40       __security_gen_cookie      0013ed40 f   coredll:COREDLL.dll
 0001:0003dd58       ?_Xlen@_String_base@std@@SAXXZ 0013ed58 f   libcpmt:string.obj
 0001:0003dde8       ?_Xran@_String_base@std@@SAXXZ 0013ede8 f   libcpmt:string.obj
 0001:0003de70       memcpy_s                   0013ee70 f   LIBCMT:memcpy_s.obj
 0001:0003df58       memmove_s                  0013ef58 f   LIBCMT:memmove_s.obj
 0001:0003e010       _invalid_parameter_noinfo  0013f010 f   LIBCMT:invarg.obj
 0001:0003e04c       _invoke_watson             0013f04c f   LIBCMT:invarg.obj
 0001:0003e080       __FrameUnwindToState       0013f080 f   LIBCMT:frame_ce.obj
 0001:0003e3f8       ?_DestructExceptionObject@@YAXPAUEHExceptionRecord@@E@Z 0013f3f8 f   LIBCMT:frame_ce.obj
 0001:0003e464       ?_OffsetToAddress@@YAPAXHPAKK@Z 0013f464 f   LIBCMT:frame_ce.obj
 0001:0003e4b0       ?FindFrameInfo@@YAPAU_FrameInfo@@PAK@Z 0013f4b0 f   LIBCMT:frame_ce.obj
 0001:0003e4f0       ?FindCatchFrameInfo@@YAPAU_FrameInfo@@PAK@Z 0013f4f0 f   LIBCMT:frame_ce.obj
 0001:0003e530       ?_GetRangeOfTrysToCheck@@YAPBU_s_TryBlockMapEntry@@PBU_s_FuncInfo@@HHPAI1@Z 0013f530 f   LIBCMT:frame_ce.obj
 0001:0003ef3c       __InternalCxxFrameHandler  0013ff3c f   LIBCMT:frame_ce.obj
 0001:0003f094       __CxxFrameHandler3         00140094 f   LIBCMT:frame_ce.obj
 0001:0003f0cc       __GSHandlerCheck_EH        001400cc f   LIBCMT:gshandlereh.obj
 0001:0003f160       __GSHandlerCheckCommon     00140160 f   LIBCMT:gshandler.obj
 0001:0003f1a8       __GSHandlerCheck           001401a8 f   LIBCMT:gshandler.obj
 0001:0003f1d8       _invalid_parameter         001401d8 f   LIBCMT:invarginternal.obj
 0001:0003f204       GetCRTStorage              00140204 f   LIBCMT:corecrt.obj
 0001:0003f2d0       _CallSettingFrame          001402d0     LIBCMT:handlers_arm.obj
 0001:0003f314       ?FindFrameForUnwind@@YAPAKPAKPBU_s_FuncInfo@@@Z 00140314 f   LIBCMT:mdframe_arm.obj
 0001:0003f35c       ?FindCatchFrame@@YAPAKPAKK@Z 0014035c f   LIBCMT:mdframe_arm.obj
 0001:0003f3a8       ?AdjustFrameForCatch@@YAPAKPAKPBU_s_FuncInfo@@@Z 001403a8 f   LIBCMT:mdframe_arm.obj
 0001:0003f3e0       ?GetCurrentState@@YAHPAKPAU_DISPATCHER_CONTEXT@@PBU_s_FuncInfo@@@Z 001403e0 f   LIBCMT:ehstate_arm_mips.obj
 0001:0003f43c       RaiseException             0014043c f   coredll:COREDLL.dll
 0001:0003f44c       ?terminate@std@@YAXXZ      0014044c f   coredll:COREDLL.dll
 0001:0003f45c       TlsCall                    0014045c f   coredll:COREDLL.dll
 0001:0003f46c       TlsSetValue                0014046c f   coredll:COREDLL.dll
 0001:0003f47c       TlsGetValue                0014047c f   coredll:COREDLL.dll
 0001:0003f48c       InterlockedCompareExchange 0014048c f   coredll:COREDLL.dll
 0002:00000000       ??_C@_1CO@IHAJILFA@?$AAS?$AAw?$AAi?$AAM?$AA2?$AAM?$AAA?$AAV?$AA_?$AAA?$AAu?$AAd?$AAi?$AAo?$AAP?$AAl?$AAa?$AAy?$AAT?$AAo?$AAn?$AAe?$AA?$AA@ 00141000     atcmd.obj
 0002:00000030       ??_C@_1CM@POMOKKD@?$AAS?$AAw?$AAi?$AAM?$AA2?$AAM?$AAA?$AAV?$AA_?$AAA?$AAu?$AAd?$AAi?$AAo?$AAS?$AAe?$AAt?$AAA?$AAV?$AAN?$AAS?$AA?$AA@ 00141030     atcmd.obj
 0002:0000005c       ??_C@_1CM@DNPKJILK@?$AAS?$AAw?$AAi?$AAM?$AA2?$AAM?$AAA?$AAV?$AA_?$AAA?$AAu?$AAd?$AAi?$AAo?$AAG?$AAe?$AAt?$AAA?$AAV?$AAN?$AAS?$AA?$AA@ 0014105c     atcmd.obj
 0002:00000088       ??_C@_1CM@DFDCENPP@?$AAS?$AAw?$AAi?$AAM?$AA2?$AAM?$AAA?$AAV?$AA_?$AAA?$AAu?$AAd?$AAi?$AAo?$AAS?$AAe?$AAt?$AAA?$AAV?$AAE?$AAC?$AA?$AA@ 00141088     atcmd.obj
 0002:000000b4       ??_C@_1CM@HCEDPOG@?$AAS?$AAw?$AAi?$AAM?$AA2?$AAM?$AAA?$AAV?$AA_?$AAA?$AAu?$AAd?$AAi?$AAo?$AAG?$AAe?$AAt?$AAA?$AAV?$AAE?$AAC?$AA?$AA@ 001410b4     atcmd.obj
 0002:000000e0       ??_C@_1CO@ICOFFPID@?$AAS?$AAw?$AAi?$AAM?$AA2?$AAM?$AAA?$AAV?$AA_?$AAA?$AAu?$AAd?$AAi?$AAo?$AAS?$AAe?$AAt?$AAA?$AAV?$AAR?$AAX?$AAG?$AA?$AA@ 001410e0     atcmd.obj
 0002:00000110       ??_C@_1CO@KHOONEJN@?$AAS?$AAw?$AAi?$AAM?$AA2?$AAM?$AAA?$AAV?$AA_?$AAA?$AAu?$AAd?$AAi?$AAo?$AAG?$AAe?$AAt?$AAA?$AAV?$AAR?$AAX?$AAG?$AA?$AA@ 00141110     atcmd.obj
 0002:00000140       ??_C@_1CO@EEIKFGAE@?$AAS?$AAw?$AAi?$AAM?$AA2?$AAM?$AAA?$AAV?$AA_?$AAA?$AAu?$AAd?$AAi?$AAo?$AAS?$AAe?$AAt?$AAA?$AAV?$AAT?$AAX?$AAG?$AA?$AA@ 00141140     atcmd.obj
 0002:00000170       ??_C@_1CO@GBIBNNBK@?$AAS?$AAw?$AAi?$AAM?$AA2?$AAM?$AAA?$AAV?$AA_?$AAA?$AAu?$AAd?$AAi?$AAo?$AAG?$AAe?$AAt?$AAA?$AAV?$AAT?$AAX?$AAG?$AA?$AA@ 00141170     atcmd.obj
 0002:000001a0       ??_C@_1DE@DBJHGPIE@?$AAS?$AAw?$AAi?$AAM?$AA2?$AAM?$AAA?$AAV?$AA_?$AAA?$AAu?$AAd?$AAi?$AAo?$AAS?$AAe?$AAt?$AAR?$AAX?$AAP?$AAC?$AAM?$AAI?$AAI?$AAR?$AA?$AA@ 001411a0     atcmd.obj
 0002:000001d4       ??_C@_1DE@CHPKIOOG@?$AAS?$AAw?$AAi?$AAM?$AA2?$AAM?$AAA?$AAV?$AA_?$AAA?$AAu?$AAd?$AAi?$AAo?$AAG?$AAe?$AAt?$AAR?$AAX?$AAP?$AAC?$AAM?$AAI?$AAI?$AAR?$AA?$AA@ 001411d4     atcmd.obj
 0002:00000208       ??_C@_1DE@DPOLNDAB@?$AAS?$AAw?$AAi?$AAM?$AA2?$AAM?$AAA?$AAV?$AA_?$AAA?$AAu?$AAd?$AAi?$AAo?$AAS?$AAe?$AAt?$AAT?$AAX?$AAP?$AAC?$AAM?$AAI?$AAI?$AAR?$AA?$AA@ 00141208     atcmd.obj
 0002:0000023c       ??_C@_1DE@CJIGDCGD@?$AAS?$AAw?$AAi?$AAM?$AA2?$AAM?$AAA?$AAV?$AA_?$AAA?$AAu?$AAd?$AAi?$AAo?$AAG?$AAe?$AAt?$AAT?$AAX?$AAP?$AAC?$AAM?$AAI?$AAI?$AAR?$AA?$AA@ 0014123c     atcmd.obj
 0002:00000270       ??_C@_1CO@LNAOIBJP@?$AAS?$AAw?$AAi?$AAM?$AA2?$AAM?$AAA?$AAV?$AA_?$AAA?$AAu?$AAd?$AAi?$AAo?$AAS?$AAe?$AAt?$AAV?$AAo?$AAl?$AAD?$AAB?$AA?$AA@ 00141270     atcmd.obj
 0002:000002a0       ??_C@_1CO@JIAFAKIB@?$AAS?$AAw?$AAi?$AAM?$AA2?$AAM?$AAA?$AAV?$AA_?$AAA?$AAu?$AAd?$AAi?$AAo?$AAG?$AAe?$AAt?$AAV?$AAo?$AAl?$AAD?$AAB?$AA?$AA@ 001412a0     atcmd.obj
 0002:000002d0       ??_C@_1DC@HAOBKDAK@?$AAS?$AAw?$AAi?$AAM?$AA2?$AAM?$AAA?$AAV?$AA_?$AAA?$AAu?$AAd?$AAi?$AAo?$AAS?$AAe?$AAt?$AAM?$AAi?$AAc?$AAG?$AAa?$AAi?$AAn?$AA?$AA@ 001412d0     atcmd.obj
 0002:00000304       ??_C@_1DC@IFLHHKEL@?$AAS?$AAw?$AAi?$AAM?$AA2?$AAM?$AAA?$AAV?$AA_?$AAA?$AAu?$AAd?$AAi?$AAo?$AAG?$AAe?$AAt?$AAM?$AAi?$AAc?$AAG?$AAa?$AAi?$AAn?$AA?$AA@ 00141304     atcmd.obj
 0002:00000338       ??_C@_1DE@EOBBNMFH@?$AAS?$AAw?$AAi?$AAM?$AA2?$AAM?$AAA?$AAV?$AA_?$AAA?$AAu?$AAd?$AAi?$AAo?$AAS?$AAe?$AAt?$AAT?$AAx?$AAV?$AAo?$AAl?$AAu?$AAm?$AAe?$AA?$AA@ 00141338     atcmd.obj
 0002:0000036c       ??_C@_1DE@FIHMDNDF@?$AAS?$AAw?$AAi?$AAM?$AA2?$AAM?$AAA?$AAV?$AA_?$AAA?$AAu?$AAd?$AAi?$AAo?$AAG?$AAe?$AAt?$AAT?$AAx?$AAV?$AAo?$AAl?$AAu?$AAm?$AAe?$AA?$AA@ 0014136c     atcmd.obj
 0002:000003a0       ??_C@_1CK@OPKNLJIB@?$AAS?$AAw?$AAi?$AAM?$AA2?$AAM?$AAA?$AAV?$AA_?$AAA?$AAu?$AAd?$AAi?$AAo?$AAS?$AAe?$AAt?$AAS?$AAT?$AAG?$AA?$AA@ 001413a0     atcmd.obj
 0002:000003cc       ??_C@_1CK@JALDAKPG@?$AAS?$AAw?$AAi?$AAM?$AA2?$AAM?$AAA?$AAV?$AA_?$AAA?$AAu?$AAd?$AAi?$AAo?$AAG?$AAe?$AAt?$AAS?$AAT?$AAG?$AA?$AA@ 001413cc     atcmd.obj
 0002:000003f8       ??_C@_1CM@NOBCNHJP@?$AAS?$AAw?$AAi?$AAM?$AA2?$AAM?$AAA?$AAV?$AA_?$AAA?$AAu?$AAd?$AAi?$AAo?$AAS?$AAe?$AAt?$AAL?$AAP?$AAB?$AAK?$AA?$AA@ 001413f8     atcmd.obj
 0002:00000424       ??_C@_1CI@NOFGKEE@?$AAS?$AAw?$AAi?$AAM?$AA2?$AAM?$AAA?$AAV?$AA_?$AAA?$AAu?$AAd?$AAi?$AAo?$AAN?$AAV?$AAD?$AAe?$AAf?$AA?$AA@ 00141424     atcmd.obj
 0002:0000044c       ??_C@_1CO@COCDIGMD@?$AAS?$AAw?$AAi?$AAM?$AA2?$AAM?$AAA?$AAV?$AA_?$AAA?$AAu?$AAd?$AAi?$AAo?$AAG?$AAe?$AAt?$AAA?$AAV?$AAC?$AAF?$AAG?$AA?$AA@ 0014144c     atcmd.obj
 0002:0000047c       ??_C@_1CO@LCIANNN@?$AAS?$AAw?$AAi?$AAM?$AA2?$AAM?$AAA?$AAV?$AA_?$AAA?$AAu?$AAd?$AAi?$AAo?$AAS?$AAe?$AAt?$AAA?$AAV?$AAC?$AAF?$AAG?$AA?$AA@ 0014147c     atcmd.obj
 0002:000004ac       ??_C@_1DA@HPJBJKKE@?$AAS?$AAw?$AAi?$AAM?$AA2?$AAM?$AAA?$AAV?$AA_?$AAA?$AAu?$AAd?$AAi?$AAo?$AAG?$AAe?$AAt?$AAA?$AAV?$AAM?$AAu?$AAt?$AAe?$AA?$AA@ 001414ac     atcmd.obj
 0002:000004dc       ??_C@_1DA@NBLKNKNI@?$AAS?$AAw?$AAi?$AAM?$AA2?$AAM?$AAA?$AAV?$AA_?$AAA?$AAu?$AAd?$AAi?$AAo?$AAS?$AAe?$AAt?$AAA?$AAV?$AAM?$AAu?$AAt?$AAe?$AA?$AA@ 001414dc     atcmd.obj
 0002:0000050c       ??_C@_1DA@NPADHLFM@?$AAS?$AAw?$AAi?$AAM?$AA2?$AAM?$AAA?$AAV?$AA_?$AAA?$AAu?$AAd?$AAi?$AAo?$AAS?$AAe?$AAt?$AAV?$AAo?$AAl?$AAu?$AAm?$AAe?$AA?$AA@ 0014150c     atcmd.obj
 0002:0000053c       ??_C@_1DA@HBCIDLCA@?$AAS?$AAw?$AAi?$AAM?$AA2?$AAM?$AAA?$AAV?$AA_?$AAA?$AAu?$AAd?$AAi?$AAo?$AAG?$AAe?$AAt?$AAV?$AAo?$AAl?$AAu?$AAm?$AAe?$AA?$AA@ 0014153c     atcmd.obj
 0002:0000056c       ??_C@_1DC@EHLKPACE@?$AAS?$AAw?$AAi?$AAM?$AA2?$AAM?$AAA?$AAV?$AA_?$AAA?$AAu?$AAd?$AAi?$AAo?$AAS?$AAe?$AAt?$AAP?$AAr?$AAo?$AAf?$AAi?$AAl?$AAe?$AA?$AA@ 0014156c     atcmd.obj
 0002:000005a0       ??_C@_1DC@LCOMCJGF@?$AAS?$AAw?$AAi?$AAM?$AA2?$AAM?$AAA?$AAV?$AA_?$AAA?$AAu?$AAd?$AAi?$AAo?$AAG?$AAe?$AAt?$AAP?$AAr?$AAo?$AAf?$AAi?$AAl?$AAe?$AA?$AA@ 001415a0     atcmd.obj
 0002:000005d4       ??_C@_1CI@EKPGHNKM@?$AAS?$AAW?$AAI?$AAO?$AAM?$AAA?$AAE?$AAX?$AAS?$AAh?$AAu?$AAt?$AAd?$AAo?$AAw?$AAn?$AAA?$AAp?$AAi?$AA?$AA@ 001415d4     atcmd.obj
 0002:000005fc       ??_C@_1CA@LIDENJBL@?$AAS?$AAW?$AAI?$AAO?$AAM?$AAA?$AAE?$AAX?$AAI?$AAn?$AAi?$AAt?$AAA?$AAp?$AAi?$AA?$AA@ 001415fc     atcmd.obj
 0002:0000061c       ??_C@_1CO@LLKDCJKA@?$AAS?$AAW?$AAI?$AAO?$AAM?$AAA?$AAE?$AAX?$AAS?$AAe?$AAs?$AAs?$AAi?$AAo?$AAn?$AAG?$AAe?$AAt?$AAI?$AAn?$AAf?$AAo?$AA?$AA@ 0014161c     atcmd.obj
 0002:0000064c       ??_C@_1CI@HCLCIPMF@?$AAS?$AAW?$AAI?$AAO?$AAM?$AAA?$AAE?$AAX?$AAS?$AAe?$AAt?$AAS?$AAe?$AAt?$AAt?$AAi?$AAn?$AAg?$AAs?$AA?$AA@ 0014164c     atcmd.obj
 0002:00000674       ??_C@_1CI@GENPGOKH@?$AAS?$AAW?$AAI?$AAO?$AAM?$AAA?$AAE?$AAX?$AAG?$AAe?$AAt?$AAS?$AAe?$AAt?$AAt?$AAi?$AAn?$AAg?$AAs?$AA?$AA@ 00141674     atcmd.obj
 0002:0000069c       ??_C@_1CE@GPIKLGLD@?$AAS?$AAW?$AAI?$AAO?$AAM?$AAA?$AAE?$AAX?$AAS?$AAe?$AAl?$AAe?$AAc?$AAt?$AAi?$AAo?$AAn?$AA?$AA@ 0014169c     atcmd.obj
 0002:000006c0       ??_C@_1CM@KMPDFMLJ@?$AAS?$AAW?$AAI?$AAO?$AAM?$AAA?$AAE?$AAX?$AAS?$AAe?$AAs?$AAs?$AAi?$AAo?$AAn?$AAC?$AAa?$AAn?$AAc?$AAe?$AAl?$AA?$AA@ 001416c0     atcmd.obj
 0002:000006ec       ??_C@_1CK@IHNDAJDA@?$AAS?$AAW?$AAI?$AAO?$AAM?$AAA?$AAE?$AAX?$AAS?$AAe?$AAs?$AAs?$AAi?$AAo?$AAn?$AAS?$AAt?$AAa?$AAr?$AAt?$AA?$AA@ 001416ec     atcmd.obj
 0002:00000718       ??_C@_1CO@LGPNPECH@?$AAS?$AAW?$AAI?$AAO?$AAM?$AAA?$AAE?$AAX?$AAS?$AAe?$AAt?$AAE?$AAv?$AAe?$AAn?$AAt?$AAR?$AAe?$AAp?$AAo?$AAr?$AAt?$AA?$AA@ 00141718     atcmd.obj
 0002:00000748       ??_C@_1CG@NFCINIOE@?$AAG?$AAe?$AAt?$AAI?$AAP?$AAC?$AAo?$AAn?$AAf?$AAi?$AAg?$AAu?$AAr?$AAa?$AAt?$AAi?$AAo?$AAn?$AA?$AA@ 00141748     atcmd.obj
 0002:00000770       ??_C@_1CG@DMPJHODC@?$AAO?$AAM?$AAA?$AAD?$AAM?$AAS?$AAe?$AAn?$AAd?$AAS?$AAe?$AAl?$AAe?$AAc?$AAt?$AAi?$AAo?$AAn?$AA?$AA@ 00141770     atcmd.obj
 0002:00000798       ??_C@_1CG@HKOMINGG@?$AAO?$AAM?$AAA?$AAD?$AAM?$AAG?$AAe?$AAt?$AAP?$AAe?$AAn?$AAd?$AAi?$AAn?$AAg?$AAN?$AAI?$AAA?$AA?$AA@ 00141798     atcmd.obj
 0002:000007c0       ??_C@_1CG@HPMHKNDG@?$AAO?$AAM?$AAA?$AAD?$AAM?$AAC?$AAa?$AAn?$AAc?$AAe?$AAl?$AAS?$AAe?$AAs?$AAs?$AAi?$AAo?$AAn?$AA?$AA@ 001417c0     atcmd.obj
 0002:000007e8       ??_C@_1CE@NFPGDNPI@?$AAO?$AAM?$AAA?$AAD?$AAM?$AAS?$AAt?$AAa?$AAr?$AAt?$AAS?$AAe?$AAs?$AAs?$AAi?$AAo?$AAn?$AA?$AA@ 001417e8     atcmd.obj
 0002:0000080c       ??_C@_1DC@KHFMANMB@?$AAO?$AAM?$AAA?$AAD?$AAM?$AAS?$AAe?$AAt?$AAP?$AAR?$AAL?$AAU?$AAp?$AAd?$AAa?$AAt?$AAe?$AAF?$AAe?$AAa?$AAt?$AAu?$AAr?$AAe?$AA?$AA@ 0014180c     atcmd.obj
 0002:00000840       ??_C@_1DI@LBKFFHPH@?$AAO?$AAM?$AAA?$AAD?$AAM?$AAS?$AAe?$AAt?$AAP?$AAr?$AAo?$AAv?$AAi?$AAs?$AAi?$AAo?$AAn?$AAi?$AAn?$AAg?$AAF?$AAe?$AAa?$AAt?$AAu?$AAr?$AAe?$AA?$AA@ 00141840     atcmd.obj
 0002:00000878       ??_C@_1CI@JIPGCIG@?$AAO?$AAM?$AAA?$AAD?$AAM?$AAG?$AAe?$AAt?$AAS?$AAe?$AAs?$AAs?$AAi?$AAo?$AAn?$AAI?$AAn?$AAf?$AAo?$AA?$AA@ 00141878     atcmd.obj
 0002:000008a0       ??_C@_1DA@IDBJEHNH@?$AAO?$AAM?$AAA?$AAD?$AAM?$AAG?$AAe?$AAt?$AAF?$AAe?$AAa?$AAt?$AAu?$AAr?$AAe?$AAS?$AAe?$AAt?$AAt?$AAi?$AAn?$AAg?$AAs?$AA?$AA@ 001418a0     atcmd.obj
 0002:000008d0       ??_C@_1CG@LJKPPMHK@?$AAG?$AAe?$AAt?$AAA?$AAc?$AAt?$AAi?$AAv?$AAa?$AAt?$AAi?$AAo?$AAn?$AAS?$AAt?$AAa?$AAt?$AAe?$AA?$AA@ 001418d0     atcmd.obj
 0002:000008f8       ??_C@_1CE@HJFAADDN@?$AAA?$AAc?$AAt?$AAi?$AAv?$AAa?$AAt?$AAe?$AAA?$AAu?$AAt?$AAo?$AAm?$AAa?$AAt?$AAi?$AAc?$AA?$AA@ 001418f8     atcmd.obj
 0002:0000091c       ??_C@_1BC@HFJKMGOB@?$AAS?$AAe?$AAt?$AAP?$AAo?$AAw?$AAe?$AAr?$AA?$AA@ 0014191c     atcmd.obj
 0002:00000930       ??_C@_1DI@LOOEAKEM@?$AAS?$AAw?$AAi?$AAS?$AAe?$AAt?$AAD?$AAe?$AAv?$AAi?$AAc?$AAe?$AAR?$AAe?$AAm?$AAo?$AAv?$AAa?$AAl?$AAC?$AAa?$AAl?$AAl?$AAb?$AAa?$AAc?$AAk?$AA?$AA@ 00141930     atcmd.obj
 0002:00000968       ??_C@_1BO@LDFOMHLP@?$AAG?$AAe?$AAt?$AAI?$AAm?$AAa?$AAg?$AAe?$AAS?$AAt?$AAo?$AAr?$AAe?$AAW?$AA?$AA@ 00141968     atcmd.obj
 0002:00000988       ??_C@_1BM@LMCPNJMJ@?$AAG?$AAe?$AAt?$AAI?$AAm?$AAa?$AAg?$AAe?$AAI?$AAn?$AAf?$AAo?$AAW?$AA?$AA@ 00141988     atcmd.obj
 0002:000009a4       ??_C@_1CG@HGNNBAKA@?$AAU?$AAp?$AAg?$AAr?$AAa?$AAd?$AAe?$AAF?$AAi?$AAr?$AAm?$AAw?$AAa?$AAr?$AAe?$AA2?$AAk?$AAW?$AA?$AA@ 001419a4     atcmd.obj
 0002:000009cc       ??_C@_1BA@FDMAHHFC@?$AAG?$AAe?$AAt?$AAI?$AAM?$AAS?$AAI?$AA?$AA@ 001419cc     atcmd.obj
 0002:000009dc       ??_C@_1CC@BFFFCEKD@?$AAG?$AAe?$AAt?$AAS?$AAe?$AAr?$AAi?$AAa?$AAl?$AAN?$AAu?$AAm?$AAb?$AAe?$AAr?$AAs?$AA?$AA@ 001419dc     atcmd.obj
 0002:00000a00       ??_C@_1BO@DCEMMFDN@?$AAG?$AAe?$AAt?$AAV?$AAo?$AAi?$AAc?$AAe?$AAN?$AAu?$AAm?$AAb?$AAe?$AAr?$AA?$AA@ 00141a00     atcmd.obj
 0002:00000a20       ??_C@_1CI@PIMIADNL@?$AAG?$AAe?$AAt?$AAH?$AAa?$AAr?$AAd?$AAw?$AAa?$AAr?$AAe?$AAR?$AAe?$AAv?$AAi?$AAs?$AAi?$AAo?$AAn?$AA?$AA@ 00141a20     atcmd.obj
 0002:00000a48       ??_C@_1BG@GEINAGNB@?$AAG?$AAe?$AAt?$AAM?$AAo?$AAd?$AAe?$AAl?$AAI?$AAD?$AA?$AA@ 00141a48     atcmd.obj
 0002:00000a60       ??_C@_1CA@PPLNCIKK@?$AAG?$AAe?$AAt?$AAM?$AAa?$AAn?$AAu?$AAf?$AAa?$AAc?$AAt?$AAu?$AAr?$AAe?$AAr?$AA?$AA@ 00141a60     atcmd.obj
 0002:00000a80       ??_C@_1CE@OAPGAKBB@?$AAS?$AAw?$AAi?$AAG?$AAe?$AAt?$AAC?$AAw?$AAe?$AAP?$AAk?$AAg?$AAs?$AAI?$AAn?$AAf?$AAo?$AA?$AA@ 00141a80     atcmd.obj
 0002:00000aa4       ??_C@_1CA@GLALHLMI@?$AAG?$AAe?$AAt?$AAF?$AAi?$AAr?$AAm?$AAw?$AAa?$AAr?$AAe?$AAI?$AAn?$AAf?$AAo?$AA?$AA@ 00141aa4     atcmd.obj
 0002:00000ac4       ??_C@_1CI@DDKIELDP@?$AAG?$AAe?$AAt?$AAF?$AAi?$AAr?$AAm?$AAw?$AAa?$AAr?$AAe?$AAR?$AAe?$AAv?$AAi?$AAs?$AAi?$AAo?$AAn?$AA?$AA@ 00141ac4     atcmd.obj
 0002:00000aec       ??_C@_1BO@KDNAPCGO@?$AAG?$AAe?$AAt?$AAH?$AAo?$AAm?$AAe?$AAN?$AAe?$AAt?$AAw?$AAo?$AAr?$AAk?$AA?$AA@ 00141aec     atcmd.obj
 0002:00000b0c       ??_C@_1CE@GLLOHEPH@?$AAG?$AAe?$AAt?$AAS?$AAe?$AAr?$AAv?$AAi?$AAn?$AAg?$AAN?$AAe?$AAt?$AAw?$AAo?$AAr?$AAk?$AA?$AA@ 00141b0c     atcmd.obj
 0002:00000b30       ??_C@_1CE@KOCPNJOP@?$AAG?$AAe?$AAt?$AAC?$AAo?$AAn?$AAn?$AAe?$AAc?$AAt?$AAi?$AAo?$AAn?$AAR?$AAa?$AAt?$AAe?$AA?$AA@ 00141b30     atcmd.obj
 0002:00000b54       ??_C@_1DM@IPJHDBDK@?$AAG?$AAe?$AAt?$AAS?$AAe?$AAr?$AAv?$AAi?$AAn?$AAg?$AAN?$AAe?$AAt?$AAw?$AAo?$AAr?$AAk?$AAC?$AAa?$AAp?$AAa?$AAb?$AAi?$AAl?$AAi?$AAt?$AAi?$AAe?$AAs?$AA?$AA@ 00141b54     atcmd.obj
 0002:00000b90       ??_C@_1CG@FELIKJGA@?$AAG?$AAe?$AAt?$AAS?$AAi?$AAg?$AAn?$AAa?$AAl?$AAS?$AAt?$AAr?$AAe?$AAn?$AAg?$AAt?$AAh?$AAs?$AA?$AA@ 00141b90     atcmd.obj
 0002:00000bb8       ??_C@_1CG@HOIPIAHO@?$AAG?$AAe?$AAt?$AAS?$AAe?$AAs?$AAs?$AAi?$AAo?$AAn?$AAD?$AAu?$AAr?$AAa?$AAt?$AAi?$AAo?$AAn?$AA?$AA@ 00141bb8     atcmd.obj
 0002:00000be0       ??_C@_1DA@DKMHBAKK@?$AAG?$AAe?$AAt?$AAD?$AAa?$AAt?$AAa?$AAB?$AAe?$AAa?$AAr?$AAe?$AAr?$AAT?$AAe?$AAc?$AAh?$AAn?$AAo?$AAl?$AAo?$AAg?$AAy?$AA?$AA@ 00141be0     atcmd.obj
 0002:00000c10       ??_C@_1BO@EKIOKBPL@?$AAG?$AAe?$AAt?$AAD?$AAu?$AAn?$AAC?$AAa?$AAl?$AAl?$AAI?$AAn?$AAf?$AAo?$AA?$AA@ 00141c10     atcmd.obj
 0002:00000c30       ??_C@_1CC@NHFMMBGI@?$AAG?$AAe?$AAt?$AAD?$AAo?$AAr?$AAm?$AAa?$AAn?$AAc?$AAy?$AAS?$AAt?$AAa?$AAt?$AAe?$AA?$AA@ 00141c30     atcmd.obj
 0002:00000c54       ??_C@_1CK@KIBDCEK@?$AAW?$AAr?$AAi?$AAt?$AAe?$AAP?$AAh?$AAo?$AAn?$AAe?$AAb?$AAo?$AAo?$AAk?$AAR?$AAe?$AAc?$AAo?$AAr?$AAd?$AA?$AA@ 00141c54     atcmd.obj
 0002:00000c80       ??_C@_1CM@NEKOPCMI@?$AAD?$AAe?$AAl?$AAe?$AAt?$AAe?$AAP?$AAh?$AAo?$AAn?$AAe?$AAb?$AAo?$AAo?$AAk?$AAR?$AAe?$AAc?$AAo?$AAr?$AAd?$AA?$AA@ 00141c80     atcmd.obj
 0002:00000cac       ??_C@_1CK@DFIMJAHF@?$AAR?$AAe?$AAa?$AAd?$AAP?$AAh?$AAo?$AAn?$AAe?$AAb?$AAo?$AAo?$AAk?$AAR?$AAe?$AAc?$AAo?$AAr?$AAd?$AAs?$AA?$AA@ 00141cac     atcmd.obj
 0002:00000cd8       ??_C@_1DC@FBPBHONH@?$AAG?$AAe?$AAt?$AAP?$AAh?$AAo?$AAn?$AAe?$AAb?$AAo?$AAo?$AAk?$AAC?$AAa?$AAp?$AAa?$AAb?$AAi?$AAl?$AAi?$AAt?$AAi?$AAe?$AAs?$AA?$AA@ 00141cd8     atcmd.obj
 0002:00000d0c       ??_C@_1BK@EMHIBMDL@?$AAR?$AAe?$AAs?$AAe?$AAt?$AAP?$AAD?$AAS?$AAD?$AAa?$AAt?$AAa?$AA?$AA@ 00141d0c     atcmd.obj
 0002:00000d28       ??_C@_1DC@BGGGMCCN@?$AAS?$AAe?$AAt?$AAP?$AAo?$AAr?$AAt?$AAA?$AAu?$AAt?$AAo?$AAm?$AAa?$AAt?$AAi?$AAc?$AAT?$AAr?$AAa?$AAc?$AAk?$AAi?$AAn?$AAg?$AA?$AA@ 00141d28     atcmd.obj
 0002:00000d5c       ??_C@_1DC@EFBNBNHH@?$AAG?$AAe?$AAt?$AAP?$AAo?$AAr?$AAt?$AAA?$AAu?$AAt?$AAo?$AAm?$AAa?$AAt?$AAi?$AAc?$AAT?$AAr?$AAa?$AAc?$AAk?$AAi?$AAn?$AAg?$AA?$AA@ 00141d5c     atcmd.obj
 0002:00000d90       ??_C@_1DI@HGHGBMHG@?$AAS?$AAe?$AAt?$AAS?$AAe?$AAr?$AAv?$AAi?$AAc?$AAe?$AAA?$AAu?$AAt?$AAo?$AAm?$AAa?$AAt?$AAi?$AAc?$AAT?$AAr?$AAa?$AAc?$AAk?$AAi?$AAn?$AAg?$AA?$AA@ 00141d90     atcmd.obj
 0002:00000dc8       ??_C@_1DI@CACGIBL@?$AAG?$AAe?$AAt?$AAS?$AAe?$AAr?$AAv?$AAi?$AAc?$AAe?$AAA?$AAu?$AAt?$AAo?$AAm?$AAa?$AAt?$AAi?$AAc?$AAT?$AAr?$AAa?$AAc?$AAk?$AAi?$AAn?$AAg?$AA?$AA@ 00141dc8     atcmd.obj
 0002:00000e00       ??_C@_1BM@IELCHDP@?$AAS?$AAe?$AAt?$AAA?$AAG?$AAP?$AAS?$AAC?$AAo?$AAn?$AAf?$AAi?$AAg?$AA?$AA@ 00141e00     atcmd.obj
 0002:00000e1c       ??_C@_1BM@BFMDACJL@?$AAG?$AAe?$AAt?$AAA?$AAG?$AAP?$AAS?$AAC?$AAo?$AAn?$AAf?$AAi?$AAg?$AA?$AA@ 00141e1c     atcmd.obj
 0002:00000e38       ??_C@_1CE@NCLCCBKH@?$AAF?$AAo?$AAr?$AAc?$AAe?$AAX?$AAT?$AAR?$AAA?$AAD?$AAo?$AAw?$AAn?$AAl?$AAo?$AAa?$AAd?$AA?$AA@ 00141e38     atcmd.obj
 0002:00000e5c       ??_C@_1CM@DDKEFNNN@?$AAS?$AAe?$AAt?$AAX?$AAT?$AAR?$AAA?$AAE?$AAm?$AAb?$AAe?$AAd?$AAd?$AAe?$AAd?$AAC?$AAl?$AAi?$AAe?$AAn?$AAt?$AA?$AA@ 00141e5c     atcmd.obj
 0002:00000e88       ??_C@_1BM@DFJCJMOH@?$AAG?$AAe?$AAt?$AAN?$AAM?$AAE?$AAA?$AAC?$AAo?$AAn?$AAf?$AAi?$AAg?$AA?$AA@ 00141e88     atcmd.obj
 0002:00000ea4       ??_C@_1BM@CIBKLJED@?$AAS?$AAe?$AAt?$AAN?$AAM?$AAE?$AAA?$AAC?$AAo?$AAn?$AAf?$AAi?$AAg?$AA?$AA@ 00141ea4     atcmd.obj
 0002:00000ec0       ??_C@_1CA@KMIGBNMK@?$AAS?$AAe?$AAt?$AAX?$AAT?$AAR?$AAA?$AAV?$AAa?$AAl?$AAi?$AAd?$AAi?$AAt?$AAy?$AA?$AA@ 00141ec0     atcmd.obj
 0002:00000ee0       ??_C@_1CA@MAFFGJAJ@?$AAG?$AAe?$AAt?$AAX?$AAT?$AAR?$AAA?$AAV?$AAa?$AAl?$AAi?$AAd?$AAi?$AAt?$AAy?$AA?$AA@ 00141ee0     atcmd.obj
 0002:00000f00       ??_C@_1BO@CMMMIKIK@?$AAS?$AAe?$AAt?$AAX?$AAT?$AAR?$AAA?$AAN?$AAe?$AAt?$AAw?$AAo?$AAr?$AAk?$AA?$AA@ 00141f00     atcmd.obj
 0002:00000f20       ??_C@_1BO@KNKDDKKI@?$AAG?$AAe?$AAt?$AAX?$AAT?$AAR?$AAA?$AAN?$AAe?$AAt?$AAw?$AAo?$AAr?$AAk?$AA?$AA@ 00141f20     atcmd.obj
 0002:00000f40       ??_C@_1DC@HPMMEIMG@?$AAS?$AAe?$AAt?$AAX?$AAT?$AAR?$AAA?$AAA?$AAu?$AAt?$AAo?$AAm?$AAa?$AAt?$AAi?$AAc?$AAD?$AAo?$AAw?$AAn?$AAl?$AAo?$AAa?$AAd?$AA?$AA@ 00141f40     atcmd.obj
 0002:00000f74       ??_C@_1DC@CMLHJHJM@?$AAG?$AAe?$AAt?$AAX?$AAT?$AAR?$AAA?$AAA?$AAu?$AAt?$AAo?$AAm?$AAa?$AAt?$AAi?$AAc?$AAD?$AAo?$AAw?$AAn?$AAl?$AAo?$AAa?$AAd?$AA?$AA@ 00141f74     atcmd.obj
 0002:00000fa8       ??_C@_1BO@LKBLACJA@?$AAS?$AAe?$AAt?$AAP?$AAD?$AAS?$AAD?$AAe?$AAf?$AAa?$AAu?$AAl?$AAt?$AAs?$AA?$AA@ 00141fa8     atcmd.obj
 0002:00000fc8       ??_C@_1BO@DLHELCLC@?$AAG?$AAe?$AAt?$AAP?$AAD?$AAS?$AAD?$AAe?$AAf?$AAa?$AAu?$AAl?$AAt?$AAs?$AA?$AA@ 00141fc8     atcmd.obj
 0002:00000fe8       ??_C@_1CO@NGELCAG@?$AAP?$AAD?$AAS?$AAI?$AAn?$AAj?$AAe?$AAc?$AAt?$AAT?$AAi?$AAm?$AAe?$AAR?$AAe?$AAf?$AAe?$AAr?$AAe?$AAn?$AAc?$AAe?$AA?$AA@ 00141fe8     atcmd.obj
 0002:00001018       ??_C@_1BI@NEKGNCEE@?$AAS?$AAe?$AAt?$AAP?$AAD?$AAS?$AAS?$AAt?$AAa?$AAt?$AAe?$AA?$AA@ 00142018     atcmd.obj
 0002:00001030       ??_C@_1BI@MCMLDDCG@?$AAG?$AAe?$AAt?$AAP?$AAD?$AAS?$AAS?$AAt?$AAa?$AAt?$AAe?$AA?$AA@ 00142030     atcmd.obj
 0002:00001048       ??_C@_1CO@KFNELFLK@?$AAR?$AAe?$AAs?$AAe?$AAt?$AAT?$AAo?$AAF?$AAa?$AAc?$AAt?$AAo?$AAr?$AAy?$AAD?$AAe?$AAf?$AAa?$AAu?$AAl?$AAt?$AAs?$AA?$AA@ 00142048     atcmd.obj
 0002:00001078       ??_C@_1BK@GJHIJMBE@?$AAU?$AAI?$AAM?$AAC?$AAh?$AAa?$AAn?$AAg?$AAe?$AAP?$AAI?$AAN?$AA?$AA@ 00142078     atcmd.obj
 0002:00001094       ??_C@_1CI@IDBLGFEF@?$AAU?$AAI?$AAM?$AAS?$AAe?$AAt?$AAP?$AAI?$AAN?$AAP?$AAr?$AAo?$AAt?$AAe?$AAc?$AAt?$AAi?$AAo?$AAn?$AA?$AA@ 00142094     atcmd.obj
 0002:000010bc       ??_C@_1BM@KMFJODPI@?$AAU?$AAI?$AAM?$AAU?$AAn?$AAb?$AAl?$AAo?$AAc?$AAk?$AAP?$AAI?$AAN?$AA?$AA@ 001420bc     atcmd.obj
 0002:000010d8       ??_C@_1BK@FNIKCFGA@?$AAU?$AAI?$AAM?$AAV?$AAe?$AAr?$AAi?$AAf?$AAy?$AAP?$AAI?$AAN?$AA?$AA@ 001420d8     atcmd.obj
 0002:000010f4       ??_C@_1CC@MAOGAOLF@?$AAU?$AAI?$AAM?$AAG?$AAe?$AAt?$AAC?$AAa?$AAr?$AAd?$AAS?$AAt?$AAa?$AAt?$AAu?$AAs?$AA?$AA@ 001420f4     atcmd.obj
 0002:00001118       ??_C@_1DA@GHLIECNF@?$AAD?$AAM?$AAS?$AAU?$AAI?$AAM?$AAU?$AAn?$AAb?$AAl?$AAo?$AAc?$AAk?$AAC?$AAo?$AAn?$AAt?$AAr?$AAo?$AAl?$AAK?$AAe?$AAy?$AA?$AA@ 00142118     atcmd.obj
 0002:00001148       ??_C@_1DM@PICNGJDJ@?$AAD?$AAM?$AAS?$AAU?$AAI?$AAM?$AAS?$AAe?$AAt?$AAC?$AAo?$AAn?$AAt?$AAr?$AAo?$AAl?$AAK?$AAe?$AAy?$AAP?$AAr?$AAo?$AAt?$AAe?$AAc?$AAt?$AAi?$AAo?$AAn?$AA?$AA@ 00142148     atcmd.obj
 0002:00001184       ??_C@_1DE@KJIFEPBC@?$AAD?$AAM?$AAS?$AAU?$AAI?$AAM?$AAG?$AAe?$AAt?$AAC?$AAo?$AAn?$AAt?$AAr?$AAo?$AAl?$AAK?$AAe?$AAy?$AAS?$AAt?$AAa?$AAt?$AAu?$AAs?$AA?$AA@ 00142184     atcmd.obj
 0002:000011b8       ??_C@_1BO@BDMAADME@?$AAD?$AAM?$AAS?$AAU?$AAI?$AAM?$AAG?$AAe?$AAt?$AAI?$AAC?$AAC?$AAI?$AAD?$AA?$AA@ 001421b8     atcmd.obj
 0002:000011d8       ??_C@_1CG@GOOPNCGG@?$AAD?$AAM?$AAS?$AAU?$AAI?$AAM?$AAG?$AAe?$AAt?$AAP?$AAI?$AAN?$AAS?$AAt?$AAa?$AAt?$AAu?$AAs?$AA?$AA@ 001421d8     atcmd.obj
 0002:00001200       ??_C@_1CA@ECNLMANC@?$AAD?$AAM?$AAS?$AAU?$AAI?$AAM?$AAC?$AAh?$AAa?$AAn?$AAg?$AAe?$AAP?$AAI?$AAN?$AA?$AA@ 00142200     atcmd.obj
 0002:00001220       ??_C@_1CC@FDCEKFEM@?$AAD?$AAM?$AAS?$AAU?$AAI?$AAM?$AAU?$AAn?$AAb?$AAl?$AAo?$AAc?$AAk?$AAP?$AAI?$AAN?$AA?$AA@ 00142220     atcmd.obj
 0002:00001244       ??_C@_1CA@HGCJHJKG@?$AAD?$AAM?$AAS?$AAU?$AAI?$AAM?$AAV?$AAe?$AAr?$AAi?$AAf?$AAy?$AAP?$AAI?$AAN?$AA?$AA@ 00142244     atcmd.obj
 0002:00001264       ??_C@_1CO@IAPGNGBB@?$AAD?$AAM?$AAS?$AAU?$AAI?$AAM?$AAS?$AAe?$AAt?$AAP?$AAI?$AAN?$AAP?$AAr?$AAo?$AAt?$AAe?$AAc?$AAt?$AAi?$AAo?$AAn?$AA?$AA@ 00142264     atcmd.obj
 0002:00001294       ??_C@_1BO@PHBFFHLB@?$AAS?$AAe?$AAt?$AAS?$AAM?$AAS?$AAC?$AAA?$AAd?$AAd?$AAr?$AAe?$AAs?$AAs?$AA?$AA@ 00142294     atcmd.obj
 0002:000012b4       ??_C@_1BO@HGHKOHJD@?$AAG?$AAe?$AAt?$AAS?$AAM?$AAS?$AAC?$AAA?$AAd?$AAd?$AAr?$AAe?$AAs?$AAs?$AA?$AA@ 001422b4     atcmd.obj
 0002:000012d4       ??_C@_1BA@FCBDHPLP@?$AAS?$AAe?$AAn?$AAd?$AAS?$AAM?$AAS?$AA?$AA@ 001422d4     atcmd.obj
 0002:000012e4       ??_C@_1BA@KOGJAAJI@?$AAS?$AAa?$AAv?$AAe?$AAS?$AAM?$AAS?$AA?$AA@ 001422e4     atcmd.obj
 0002:000012f4       ??_C@_1CA@JHJDBCGM@?$AAM?$AAo?$AAd?$AAi?$AAf?$AAy?$AAS?$AAM?$AAS?$AAS?$AAt?$AAa?$AAt?$AAu?$AAs?$AA?$AA@ 001422f4     atcmd.obj
 0002:00001314       ??_C@_1CO@LFANFNEA@?$AAS?$AAe?$AAt?$AAB?$AAr?$AAo?$AAa?$AAd?$AAc?$AAa?$AAs?$AAt?$AAA?$AAc?$AAt?$AAi?$AAv?$AAa?$AAt?$AAi?$AAo?$AAn?$AA?$AA@ 00142314     atcmd.obj
 0002:00001344       ??_C@_1BE@HLBMIMG@?$AAS?$AAe?$AAt?$AAR?$AAo?$AAu?$AAt?$AAe?$AAs?$AA?$AA@ 00142344     atcmd.obj
 0002:00001358       ??_C@_1BO@MAJBHHDN@?$AAS?$AAe?$AAt?$AAS?$AAM?$AAS?$AAP?$AAr?$AAo?$AAt?$AAo?$AAc?$AAo?$AAl?$AA?$AA@ 00142358     atcmd.obj
 0002:00001378       ??_C@_1O@PELEKICI@?$AAG?$AAe?$AAt?$AAS?$AAM?$AAS?$AA?$AA@ 00142378     atcmd.obj
 0002:00001388       ??_C@_1BG@EAPBFHAO@?$AAG?$AAe?$AAt?$AAS?$AAM?$AAS?$AAL?$AAi?$AAs?$AAt?$AA?$AA@ 00142388     atcmd.obj
 0002:000013a0       ??_C@_1BE@LPEGABOF@?$AAD?$AAe?$AAl?$AAe?$AAt?$AAe?$AAS?$AAM?$AAS?$AA?$AA@ 001423a0     atcmd.obj
 0002:000013b4       ??_C@_1BI@LBBBPLGJ@?$AAV?$AAa?$AAl?$AAi?$AAd?$AAa?$AAt?$AAe?$AAS?$AAP?$AAC?$AA?$AA@ 001423b4     atcmd.obj
 0002:000013cc       ??_C@_1BO@DANEGBA@?$AAG?$AAe?$AAt?$AAN?$AAe?$AAt?$AAw?$AAo?$AAr?$AAk?$AAT?$AAi?$AAm?$AAe?$AA?$AA@ 001423cc     atcmd.obj
 0002:000013ec       ??_C@_1CC@JNFHEGAK@?$AAG?$AAe?$AAt?$AAO?$AAf?$AAf?$AAl?$AAi?$AAn?$AAe?$AAR?$AAe?$AAa?$AAs?$AAo?$AAn?$AA?$AA@ 001423ec     atcmd.obj
 0002:00001410       ??_C@_1BC@FAJBENPP@?$AAG?$AAe?$AAt?$AAP?$AAo?$AAw?$AAe?$AAr?$AA?$AA@ 00142410     atcmd.obj
 0002:00001424       ??_C@_1BO@EMLBJBFB@?$AAA?$AAc?$AAt?$AAi?$AAv?$AAa?$AAt?$AAe?$AAM?$AAa?$AAn?$AAu?$AAa?$AAl?$AA?$AA@ 00142424     atcmd.obj
 0002:00001444       ??_C@_1BG@COEJJNAO@?$AAG?$AAe?$AAt?$AAE?$AAR?$AAI?$AAF?$AAi?$AAl?$AAe?$AA?$AA@ 00142444     atcmd.obj
 0002:0000145c       ??_C@_1DC@BLOBPCMC@?$AAG?$AAe?$AAt?$AA3?$AAG?$AAp?$AAp?$AA2?$AAS?$AAu?$AAb?$AAs?$AAc?$AAr?$AAi?$AAp?$AAt?$AAi?$AAo?$AAn?$AAI?$AAn?$AAf?$AAo?$AA?$AA@ 0014245c     atcmd.obj
 0002:00001490       ??_C@_1DC@EIJKCNJI@?$AAS?$AAe?$AAt?$AA3?$AAG?$AAp?$AAp?$AA2?$AAS?$AAu?$AAb?$AAs?$AAc?$AAr?$AAi?$AAp?$AAt?$AAi?$AAo?$AAn?$AAI?$AAn?$AAf?$AAo?$AA?$AA@ 00142490     atcmd.obj
 0002:000014c4       ??_C@_1BM@CPGDMEDL@?$AAG?$AAe?$AAt?$AAP?$AAR?$AAL?$AAV?$AAe?$AAr?$AAs?$AAi?$AAo?$AAn?$AA?$AA@ 001424c4     atcmd.obj
 0002:000014e0       ??_C@_1CK@MAFKIOPO@?$AAG?$AAe?$AAt?$AAF?$AAi?$AAr?$AAm?$AAw?$AAa?$AAr?$AAe?$AAR?$AAe?$AAv?$AAi?$AAs?$AAi?$AAo?$AAn?$AAs?$AA?$AA@ 001424e0     atcmd.obj
 0002:0000150c       ??_C@_1CM@EDIJFBLL@?$AAG?$AAe?$AAt?$AAD?$AAe?$AAv?$AAi?$AAc?$AAe?$AAC?$AAa?$AAp?$AAa?$AAb?$AAi?$AAl?$AAi?$AAt?$AAi?$AAe?$AAs?$AA?$AA@ 0014250c     atcmd.obj
 0002:00001538       ??_C@_1DK@FDHAHLGB@?$AAG?$AAe?$AAt?$AAA?$AAN?$AAA?$AAA?$AAA?$AAA?$AAu?$AAt?$AAh?$AAe?$AAn?$AAt?$AAi?$AAc?$AAa?$AAt?$AAi?$AAo?$AAn?$AAS?$AAt?$AAa?$AAt?$AAu?$AAs?$AA?$AA@ 00142538     atcmd.obj
 0002:00001574       ??_C@_1BE@GNJLFGAD@?$AAS?$AAe?$AAt?$AAA?$AAC?$AAC?$AAO?$AAL?$AAC?$AA?$AA@ 00142574     atcmd.obj
 0002:00001588       ??_C@_1BE@MDLABGHP@?$AAG?$AAe?$AAt?$AAA?$AAC?$AAC?$AAO?$AAL?$AAC?$AA?$AA@ 00142588     atcmd.obj
 0002:0000159c       ??_C@_1DC@MGKINNOP@?$AAG?$AAe?$AAt?$AAC?$AAD?$AAM?$AAA?$AAN?$AAe?$AAt?$AAw?$AAo?$AAr?$AAk?$AAP?$AAa?$AAr?$AAa?$AAm?$AAe?$AAt?$AAe?$AAr?$AAs?$AA?$AA@ 0014259c     atcmd.obj
 0002:000015d0       ??_C@_1DC@JFNDACLF@?$AAS?$AAe?$AAt?$AAC?$AAD?$AAM?$AAA?$AAN?$AAe?$AAt?$AAw?$AAo?$AAr?$AAk?$AAP?$AAa?$AAr?$AAa?$AAm?$AAe?$AAt?$AAe?$AAr?$AAs?$AA?$AA@ 001425d0     atcmd.obj
 0002:00001604       ??_C@_1CK@EGBLJME@?$AAS?$AAe?$AAt?$AAN?$AAe?$AAt?$AAw?$AAo?$AAr?$AAk?$AAP?$AAr?$AAe?$AAf?$AAe?$AAr?$AAe?$AAn?$AAc?$AAe?$AA?$AA@ 00142604     atcmd.obj
 0002:00001630       ??_C@_1CK@POCCMJNB@?$AAG?$AAe?$AAt?$AAN?$AAe?$AAt?$AAw?$AAo?$AAr?$AAk?$AAP?$AAr?$AAe?$AAf?$AAe?$AAr?$AAe?$AAn?$AAc?$AAe?$AA?$AA@ 00142630     atcmd.obj
 0002:0000165c       ??_C@_1CK@JIMFDDIE@?$AAI?$AAn?$AAi?$AAt?$AAi?$AAa?$AAt?$AAe?$AAD?$AAo?$AAm?$AAa?$AAi?$AAn?$AAA?$AAt?$AAt?$AAa?$AAc?$AAh?$AA?$AA@ 0014265c     atcmd.obj
 0002:00001688       ??_C@_1DI@CIBLKDLK@?$AAI?$AAn?$AAi?$AAt?$AAi?$AAa?$AAt?$AAe?$AAN?$AAe?$AAt?$AAw?$AAo?$AAr?$AAk?$AAR?$AAe?$AAg?$AAi?$AAs?$AAt?$AAr?$AAa?$AAt?$AAi?$AAo?$AAn?$AA?$AA@ 00142688     atcmd.obj
 0002:000016c0       ??_C@_1CM@KHNJMIGB@?$AAP?$AAe?$AAr?$AAf?$AAo?$AAr?$AAm?$AAN?$AAe?$AAt?$AAw?$AAo?$AAr?$AAk?$AAR?$AAA?$AAT?$AAS?$AAc?$AAa?$AAn?$AA?$AA@ 001426c0     atcmd.obj
 0002:000016ec       ??_C@_1CG@KIPBFHFH@?$AAP?$AAe?$AAr?$AAf?$AAo?$AAr?$AAm?$AAN?$AAe?$AAt?$AAw?$AAo?$AAr?$AAk?$AAS?$AAc?$AAa?$AAn?$AA?$AA@ 001426ec     atcmd.obj
 0002:00001714       ??_C@_1BE@CPONLMAP@?$AAG?$AAe?$AAt?$AAR?$AAF?$AAI?$AAn?$AAf?$AAo?$AA?$AA@ 00142714     atcmd.obj
 0002:00001728       ??_C@_1BM@INJOIDEM@?$AAG?$AAe?$AAt?$AAB?$AAy?$AAt?$AAe?$AAT?$AAo?$AAt?$AAa?$AAl?$AAs?$AA?$AA@ 00142728     atcmd.obj
 0002:00001744       ??_C@_1CE@ENGLIMHE@?$AAG?$AAe?$AAt?$AAD?$AAe?$AAf?$AAa?$AAu?$AAl?$AAt?$AAP?$AAr?$AAo?$AAf?$AAi?$AAl?$AAe?$AA?$AA@ 00142744     atcmd.obj
 0002:00001768       ??_C@_1CE@JEHKLGLP@?$AAS?$AAe?$AAt?$AAD?$AAe?$AAf?$AAa?$AAu?$AAl?$AAt?$AAP?$AAr?$AAo?$AAf?$AAi?$AAl?$AAe?$AA?$AA@ 00142768     atcmd.obj
 0002:0000178c       ??_C@_1BO@PCFFIAAI@?$AAS?$AAe?$AAt?$AAA?$AAu?$AAt?$AAo?$AAC?$AAo?$AAn?$AAn?$AAe?$AAc?$AAt?$AA?$AA@ 0014278c     atcmd.obj
 0002:000017ac       ??_C@_1BO@HDDKDACK@?$AAG?$AAe?$AAt?$AAA?$AAu?$AAt?$AAo?$AAC?$AAo?$AAn?$AAn?$AAe?$AAc?$AAt?$AA?$AA@ 001427ac     atcmd.obj
 0002:000017cc       ??_C@_1CK@MBMHNBNM@?$AAG?$AAe?$AAt?$AAL?$AAa?$AAs?$AAt?$AAM?$AAo?$AAb?$AAi?$AAl?$AAe?$AAI?$AAP?$AAE?$AAr?$AAr?$AAo?$AAr?$AA?$AA@ 001427cc     atcmd.obj
 0002:000017f8       ??_C@_1CM@IGBGPKHE@?$AAG?$AAe?$AAt?$AAM?$AAo?$AAb?$AAi?$AAl?$AAe?$AAI?$AAP?$AAP?$AAa?$AAr?$AAa?$AAm?$AAe?$AAt?$AAe?$AAr?$AAs?$AA?$AA@ 001427f8     atcmd.obj
 0002:00001824       ??_C@_1CM@OBKGJHBP@?$AAS?$AAe?$AAt?$AAM?$AAo?$AAb?$AAi?$AAl?$AAe?$AAI?$AAP?$AAP?$AAa?$AAr?$AAa?$AAm?$AAe?$AAt?$AAe?$AAr?$AAs?$AA?$AA@ 00142824     atcmd.obj
 0002:00001850       ??_C@_1CG@COPLLMPK@?$AAG?$AAe?$AAt?$AAM?$AAo?$AAb?$AAi?$AAl?$AAe?$AAI?$AAP?$AAP?$AAr?$AAo?$AAf?$AAi?$AAl?$AAe?$AA?$AA@ 00142850     atcmd.obj
 0002:00001878       ??_C@_1CG@MAPJLCNM@?$AAS?$AAe?$AAt?$AAM?$AAo?$AAb?$AAi?$AAl?$AAe?$AAI?$AAP?$AAP?$AAr?$AAo?$AAf?$AAi?$AAl?$AAe?$AA?$AA@ 00142878     atcmd.obj
 0002:000018a0       ??_C@_1DC@LKPLPLHN@?$AAG?$AAe?$AAt?$AAA?$AAc?$AAt?$AAi?$AAv?$AAe?$AAM?$AAo?$AAb?$AAi?$AAl?$AAe?$AAI?$AAP?$AAP?$AAr?$AAo?$AAf?$AAi?$AAl?$AAe?$AA?$AA@ 001428a0     atcmd.obj
 0002:000018d4       ??_C@_1DC@OJIACECH@?$AAS?$AAe?$AAt?$AAA?$AAc?$AAt?$AAi?$AAv?$AAe?$AAM?$AAo?$AAb?$AAi?$AAl?$AAe?$AAI?$AAP?$AAP?$AAr?$AAo?$AAf?$AAi?$AAl?$AAe?$AA?$AA@ 001428d4     atcmd.obj
 0002:00001908       ??_C@_1BI@FFMCFILE@?$AAG?$AAe?$AAt?$AAM?$AAo?$AAb?$AAi?$AAl?$AAe?$AAI?$AAP?$AA?$AA@ 00142908     atcmd.obj
 0002:00001920       ??_C@_1BI@EDKPLJNG@?$AAS?$AAe?$AAt?$AAM?$AAo?$AAb?$AAi?$AAl?$AAe?$AAI?$AAP?$AA?$AA@ 00142920     atcmd.obj
 0002:00001938       ??_C@_1CA@EINFGIBA@?$AAG?$AAe?$AAt?$AAP?$AAa?$AAc?$AAk?$AAe?$AAt?$AAS?$AAt?$AAa?$AAt?$AAu?$AAs?$AA?$AA@ 00142938     atcmd.obj
 0002:00001958       ??_C@_1BK@DCHGBAOJ@?$AAG?$AAe?$AAt?$AAI?$AAP?$AAA?$AAd?$AAd?$AAr?$AAe?$AAs?$AAs?$AA?$AA@ 00142958     atcmd.obj
 0002:00001974       ??_C@_1CA@JMBMOINF@?$AAG?$AAe?$AAt?$AAS?$AAe?$AAs?$AAs?$AAi?$AAo?$AAn?$AAS?$AAt?$AAa?$AAt?$AAe?$AA?$AA@ 00142974     atcmd.obj
 0002:00001994       ??_C@_1CA@FFLEDDOC@?$AAS?$AAt?$AAo?$AAp?$AAD?$AAa?$AAt?$AAa?$AAS?$AAe?$AAs?$AAs?$AAi?$AAo?$AAn?$AA?$AA@ 00142994     atcmd.obj
 0002:000019b4       ??_C@_1CE@LOHPJLLL@?$AAS?$AAt?$AAa?$AAr?$AAt?$AAD?$AAa?$AAt?$AAa?$AAS?$AAe?$AAs?$AAs?$AAi?$AAo?$AAn?$AA2?$AA?$AA@ 001429b4     atcmd.obj
 0002:000019d8       ??_C@_1CI@GFOILFKB@?$AAG?$AAe?$AAt?$AAC?$AAe?$AAl?$AAl?$AAL?$AAo?$AAc?$AAa?$AAt?$AAi?$AAo?$AAn?$AAI?$AAn?$AAf?$AAo?$AA?$AA@ 001429d8     atcmd.obj
 0002:00001a00       ??_C@_1CE@CJHGMCHL@?$AAG?$AAe?$AAt?$AAW?$AAa?$AAi?$AAt?$AAi?$AAn?$AAg?$AAM?$AAs?$AAg?$AAI?$AAn?$AAf?$AAo?$AA?$AA@ 00142a00     atcmd.obj
 0002:00001a24       ??_C@_1CO@NJMGNGIC@?$AAS?$AAe?$AAt?$AAC?$AAa?$AAl?$AAl?$AAB?$AAa?$AAr?$AAr?$AAi?$AAn?$AAg?$AAP?$AAa?$AAs?$AAs?$AAw?$AAo?$AAr?$AAd?$AA?$AA@ 00142a24     atcmd.obj
 0002:00001a54       ??_C@_1BG@JMOHBGIL@?$AAA?$AAb?$AAo?$AAr?$AAt?$AAs?$AAU?$AAS?$AAS?$AAD?$AA?$AA@ 00142a54     atcmd.obj
 0002:00001a6c       ??_C@_1BA@JNDIFGHG@?$AAA?$AAn?$AAs?$AAU?$AAS?$AAS?$AAD?$AA?$AA@ 00142a6c     atcmd.obj
 0002:00001a7c       ??_C@_1BC@OIGJILDE@?$AAO?$AAr?$AAi?$AAg?$AAU?$AAS?$AAS?$AAD?$AA?$AA@ 00142a7c     atcmd.obj
 0002:00001a90       ??_C@_1CG@GALIHLLO@?$AAA?$AAu?$AAd?$AAi?$AAo?$AAP?$AAl?$AAa?$AAy?$AAA?$AAu?$AAd?$AAi?$AAo?$AAT?$AAo?$AAn?$AAe?$AA?$AA@ 00142a90     atcmd.obj
 0002:00001ab8       ??_C@_1CK@NFNPLDHL@?$AAA?$AAu?$AAd?$AAi?$AAo?$AAS?$AAe?$AAt?$AAV?$AAo?$AAl?$AAT?$AAL?$AAB?$AAC?$AAo?$AAn?$AAf?$AAi?$AAg?$AA?$AA@ 00142ab8     atcmd.obj
 0002:00001ae4       ??_C@_1CM@LIFDNPFB@?$AAA?$AAu?$AAd?$AAi?$AAo?$AAG?$AAe?$AAt?$AAP?$AAa?$AAt?$AAh?$AAP?$AAC?$AAM?$AAF?$AAi?$AAl?$AAt?$AAe?$AAr?$AA?$AA@ 00142ae4     atcmd.obj
 0002:00001b10       ??_C@_1CC@KGCLAPBJ@?$AAA?$AAu?$AAd?$AAi?$AAo?$AAG?$AAe?$AAt?$AAP?$AAa?$AAt?$AAh?$AAW?$AAo?$AAr?$AAd?$AA?$AA@ 00142b10     atcmd.obj
 0002:00001b34       ??_C@_1CC@LDJNPJGB@?$AAA?$AAu?$AAd?$AAi?$AAo?$AAG?$AAe?$AAt?$AAP?$AAa?$AAt?$AAh?$AAB?$AAy?$AAt?$AAe?$AA?$AA@ 00142b34     atcmd.obj
 0002:00001b58       ??_C@_1CE@NEFGGJGB@?$AAA?$AAu?$AAd?$AAi?$AAo?$AAS?$AAe?$AAt?$AAA?$AAu?$AAd?$AAi?$AAo?$AAP?$AAa?$AAt?$AAh?$AA?$AA@ 00142b58     atcmd.obj
 0002:00001b7c       ??_C@_1CA@CJLLLPJJ@?$AAA?$AAu?$AAd?$AAi?$AAo?$AAG?$AAe?$AAt?$AAP?$AAr?$AAo?$AAf?$AAi?$AAl?$AAe?$AA?$AA@ 00142b7c     atcmd.obj
 0002:00001b9c       ??_C@_1CA@NMONGGNI@?$AAA?$AAu?$AAd?$AAi?$AAo?$AAS?$AAe?$AAt?$AAP?$AAr?$AAo?$AAf?$AAi?$AAl?$AAe?$AA?$AA@ 00142b9c     atcmd.obj
 0002:00001bbc       ??_C@_1CI@LOMIGCGI@?$AAS?$AAe?$AAt?$AAI?$AAm?$AAa?$AAg?$AAe?$AAs?$AAP?$AAr?$AAe?$AAf?$AAe?$AAr?$AAe?$AAn?$AAc?$AAe?$AA?$AA@ 00142bbc     atcmd.obj
 0002:00001be4       ??_C@_1CI@JKKOCCEJ@?$AAG?$AAe?$AAt?$AAI?$AAm?$AAa?$AAg?$AAe?$AAs?$AAP?$AAr?$AAe?$AAf?$AAe?$AAr?$AAe?$AAn?$AAc?$AAe?$AA?$AA@ 00142be4     atcmd.obj
 0002:00001c0c       ??_C@_1DC@LEEDOOEP@?$AAS?$AAe?$AAt?$AAS?$AAW?$AAI?$AAO?$AAM?$AAA?$AAE?$AAX?$AAE?$AAv?$AAe?$AAn?$AAt?$AAC?$AAa?$AAl?$AAl?$AAb?$AAa?$AAc?$AAk?$AA?$AA@ 00142c0c     atcmd.obj
 0002:00001c40       ??_C@_1DO@IOPPEPMM@?$AAS?$AAe?$AAt?$AAS?$AAy?$AAs?$AAt?$AAe?$AAm?$AAS?$AAe?$AAl?$AAe?$AAc?$AAt?$AAi?$AAo?$AAn?$AAP?$AAr?$AAe?$AAf?$AAC?$AAa?$AAl?$AAl?$AAb?$AAa?$AAc?$AAk?$AA?$AA@ 00142c40     atcmd.obj
 0002:00001c80       ??_C@_1CO@FGFKLCLK@?$AAS?$AAe?$AAt?$AAN?$AAe?$AAt?$AAw?$AAo?$AAr?$AAk?$AAT?$AAi?$AAm?$AAe?$AAC?$AAa?$AAl?$AAl?$AAb?$AAa?$AAc?$AAk?$AA?$AA@ 00142c80     atcmd.obj
 0002:00001cb0       ??_C@_1DC@MBGELGLO@?$AAS?$AAe?$AAt?$AAE?$AAm?$AAe?$AAr?$AAg?$AAe?$AAn?$AAc?$AAy?$AAL?$AAi?$AAs?$AAt?$AAC?$AAa?$AAl?$AAl?$AAb?$AAa?$AAc?$AAk?$AA?$AA@ 00142cb0     atcmd.obj
 0002:00001ce8       ??_C@_1EA@INMGDAJH@?$AAS?$AAe?$AAt?$AAA?$AAl?$AAl?$AAP?$AAh?$AAo?$AAn?$AAe?$AAb?$AAo?$AAo?$AAk?$AAI?$AAn?$AAi?$AAt?$AAD?$AAo?$AAn?$AAe?$AAC?$AAa?$AAl?$AAl?$AAb?$AAa?$AAc?$AAk?$AA?$AA@ 00142ce8     atcmd.obj
 0002:00001d28       ??_C@_1DO@DLOHKDJD@?$AAS?$AAe?$AAt?$AAP?$AAh?$AAo?$AAn?$AAe?$AAb?$AAo?$AAo?$AAk?$AAR?$AAe?$AAc?$AAo?$AAr?$AAd?$AAR?$AAe?$AAa?$AAd?$AAC?$AAa?$AAl?$AAl?$AAb?$AAa?$AAc?$AAk?$AA?$AA@ 00142d28     atcmd.obj
 0002:00001d68       ??_C@_1CM@HCOEPPEB@?$AAS?$AAe?$AAt?$AAO?$AAM?$AAA?$AAD?$AAM?$AAA?$AAl?$AAe?$AAr?$AAt?$AAC?$AAa?$AAl?$AAl?$AAb?$AAa?$AAc?$AAk?$AA?$AA@ 00142d68     atcmd.obj
 0002:00001d94       ??_C@_1CM@LPNPGND@?$AAS?$AAe?$AAt?$AAO?$AAM?$AAA?$AAD?$AAM?$AAS?$AAt?$AAa?$AAt?$AAe?$AAC?$AAa?$AAl?$AAl?$AAb?$AAa?$AAc?$AAk?$AA?$AA@ 00142d94     atcmd.obj
 0002:00001dc0       ??_C@_1CM@JPEMOGPL@?$AAS?$AAe?$AAt?$AAB?$AAy?$AAt?$AAe?$AAT?$AAo?$AAt?$AAa?$AAl?$AAs?$AAC?$AAa?$AAl?$AAl?$AAb?$AAa?$AAc?$AAk?$AA?$AA@ 00142dc0     atcmd.obj
 0002:00001dec       ??_C@_1DI@NCMMIEFA@?$AAS?$AAe?$AAt?$AAD?$AAa?$AAt?$AAa?$AAC?$AAa?$AAp?$AAa?$AAb?$AAi?$AAl?$AAi?$AAt?$AAi?$AAe?$AAs?$AAC?$AAa?$AAl?$AAl?$AAb?$AAa?$AAc?$AAk?$AA?$AA@ 00142dec     atcmd.obj
 0002:00001e24       ??_C@_1CM@ODEGDLPB@?$AAS?$AAe?$AAt?$AAM?$AAs?$AAg?$AAW?$AAa?$AAi?$AAt?$AAi?$AAn?$AAg?$AAC?$AAa?$AAl?$AAl?$AAb?$AAa?$AAc?$AAk?$AA?$AA@ 00142e24     atcmd.obj
 0002:00001e50       ??_C@_1CI@MKCNFE@?$AAS?$AAe?$AAt?$AAN?$AAe?$AAw?$AAS?$AAM?$AAS?$AAC?$AAB?$AAC?$AAa?$AAl?$AAl?$AAb?$AAa?$AAc?$AAk?$AA?$AA@ 00142e50     atcmd.obj
 0002:00001e78       ??_C@_1CE@DABFEIP@?$AAS?$AAe?$AAt?$AAN?$AAe?$AAw?$AAS?$AAM?$AAS?$AAC?$AAa?$AAl?$AAl?$AAb?$AAa?$AAc?$AAk?$AA?$AA@ 00142e78     atcmd.obj
 0002:00001e9c       ??_C@_1CE@FLDCNMCI@?$AAS?$AAe?$AAt?$AAR?$AAF?$AAI?$AAn?$AAf?$AAo?$AAC?$AAa?$AAl?$AAl?$AAb?$AAa?$AAc?$AAk?$AA?$AA@ 00142e9c     atcmd.obj
 0002:00001ec0       ??_C@_1DE@DAEJPNFC@?$AAS?$AAe?$AAt?$AAS?$AAi?$AAg?$AAn?$AAa?$AAl?$AAS?$AAt?$AAr?$AAe?$AAn?$AAg?$AAt?$AAh?$AAC?$AAa?$AAl?$AAl?$AAb?$AAa?$AAc?$AAk?$AA?$AA@ 00142ec0     atcmd.obj
 0002:00001ef4       ??_C@_1DI@OAEMGPHA@?$AAS?$AAe?$AAt?$AAR?$AAo?$AAa?$AAm?$AAi?$AAn?$AAg?$AAI?$AAn?$AAd?$AAi?$AAc?$AAa?$AAt?$AAo?$AAr?$AAC?$AAa?$AAl?$AAl?$AAb?$AAa?$AAc?$AAk?$AA?$AA@ 00142ef4     atcmd.obj
 0002:00001f2c       ??_C@_1CC@BKDJJPFD@?$AAS?$AAe?$AAt?$AAP?$AAo?$AAw?$AAe?$AAr?$AAC?$AAa?$AAl?$AAl?$AAb?$AAa?$AAc?$AAk?$AA?$AA@ 00142f2c     atcmd.obj
 0002:00001f50       ??_C@_1DI@PLBJFEGC@?$AAS?$AAe?$AAt?$AAA?$AAc?$AAt?$AAi?$AAv?$AAa?$AAt?$AAi?$AAo?$AAn?$AAS?$AAt?$AAa?$AAt?$AAu?$AAs?$AAC?$AAa?$AAl?$AAl?$AAb?$AAa?$AAc?$AAk?$AA?$AA@ 00142f50     atcmd.obj
 0002:00001f88       ??_C@_1DE@IIMOCCEI@?$AAS?$AAe?$AAt?$AAM?$AAo?$AAb?$AAi?$AAl?$AAe?$AAI?$AAP?$AAS?$AAt?$AAa?$AAt?$AAu?$AAs?$AAC?$AAa?$AAl?$AAl?$AAb?$AAa?$AAc?$AAk?$AA?$AA@ 00142f88     atcmd.obj
 0002:00001fbc       ??_C@_1DE@NMHAIBGI@?$AAS?$AAe?$AAt?$AAD?$AAo?$AAr?$AAm?$AAa?$AAn?$AAc?$AAy?$AAS?$AAt?$AAa?$AAt?$AAu?$AAs?$AAC?$AAa?$AAl?$AAl?$AAb?$AAa?$AAc?$AAk?$AA?$AA@ 00142fbc     atcmd.obj
 0002:00001ff0       ??_C@_1CM@JIDPIPCP@?$AAS?$AAe?$AAt?$AAD?$AAa?$AAt?$AAa?$AAB?$AAe?$AAa?$AAr?$AAe?$AAr?$AAC?$AAa?$AAl?$AAl?$AAb?$AAa?$AAc?$AAk?$AA?$AA@ 00142ff0     atcmd.obj
 0002:0000201c       ??_C@_1DA@JDCAJDBL@?$AAS?$AAe?$AAt?$AAS?$AAe?$AAs?$AAs?$AAi?$AAo?$AAn?$AAS?$AAt?$AAa?$AAt?$AAe?$AAC?$AAa?$AAl?$AAl?$AAb?$AAa?$AAc?$AAk?$AA?$AA@ 0014301c     atcmd.obj
 0002:0000204c       ??_C@_1DG@PCCFMBCH@?$AAQ?$AAC?$AAW?$AAW?$AAA?$AAN?$AAG?$AAe?$AAt?$AAC?$AAo?$AAn?$AAn?$AAe?$AAc?$AAt?$AAe?$AAd?$AAD?$AAe?$AAv?$AAi?$AAc?$AAe?$AAI?$AAD?$AA?$AA@ 0014304c     atcmd.obj
 0002:00002084       ??_C@_1CC@JBHNEBD@?$AAQ?$AAC?$AAW?$AAW?$AAA?$AAN?$AAD?$AAi?$AAs?$AAc?$AAo?$AAn?$AAn?$AAe?$AAc?$AAt?$AA?$AA@ 00143084     atcmd.obj
 0002:000020a8       ??_C@_1BM@ICODGDCC@?$AAQ?$AAC?$AAW?$AAW?$AAA?$AAN?$AAC?$AAo?$AAn?$AAn?$AAe?$AAc?$AAt?$AA?$AA@ 001430a8     atcmd.obj
 0002:000020c4       ??_C@_1BM@HKEBDPIM@?$AAG?$AAe?$AAt?$AAR?$AAT?$AAR?$AAE?$AAC?$AAo?$AAn?$AAf?$AAi?$AAg?$AA?$AA@ 001430c4     atcmd.obj
 0002:000020e0       ??_C@_1BK@JPAMOEJH@?$AAS?$AAt?$AAo?$AAp?$AAC?$AAo?$AAn?$AAt?$AAD?$AAT?$AAM?$AAF?$AA?$AA@ 001430e0     atcmd.obj
 0002:000020fc       ??_C@_1BM@BBOAIDPB@?$AAS?$AAt?$AAa?$AAr?$AAt?$AAC?$AAo?$AAn?$AAt?$AAD?$AAT?$AAM?$AAF?$AA?$AA@ 001430fc     atcmd.obj
 0002:00002118       ??_C@_1BE@HONOAGGK@?$AAS?$AAe?$AAn?$AAd?$AAF?$AAl?$AAa?$AAs?$AAh?$AA?$AA@ 00143118     atcmd.obj
 0002:0000212c       ??_C@_1BO@GPPPCEIO@?$AAG?$AAe?$AAt?$AAA?$AAl?$AAl?$AAC?$AAa?$AAl?$AAl?$AAI?$AAn?$AAf?$AAo?$AA?$AA@ 0014312c     atcmd.obj
 0002:0000214c       ??_C@_1BO@NMMIKEEG@?$AAG?$AAe?$AAt?$AAC?$AAa?$AAl?$AAl?$AAW?$AAa?$AAi?$AAt?$AAi?$AAn?$AAg?$AA?$AA@ 0014314c     atcmd.obj
 0002:0000216c       ??_C@_1CE@LMIADLLA@?$AAG?$AAe?$AAt?$AAC?$AAa?$AAl?$AAl?$AAF?$AAo?$AAr?$AAw?$AAa?$AAr?$AAd?$AAi?$AAn?$AAg?$AA?$AA@ 0014316c     atcmd.obj
 0002:00002190       ??_C@_1BA@KNBNBGGG@?$AAG?$AAe?$AAt?$AAC?$AAL?$AAI?$AAR?$AA?$AA@ 00143190     atcmd.obj
 0002:000021a0       ??_C@_1BO@JOMDFNKA@?$AAS?$AAe?$AAt?$AAS?$AAu?$AAp?$AAs?$AAS?$AAe?$AAr?$AAv?$AAi?$AAc?$AAe?$AA?$AA@ 001431a0     atcmd.obj
 0002:000021c0       ??_C@_1BO@DACCHOHL@?$AAG?$AAe?$AAt?$AAC?$AAa?$AAl?$AAl?$AAB?$AAa?$AAr?$AAr?$AAi?$AAn?$AAg?$AA?$AA@ 001431c0     atcmd.obj
 0002:000021e0       ??_C@_1BI@BPLGPDPM@?$AAM?$AAa?$AAn?$AAa?$AAg?$AAe?$AAC?$AAa?$AAl?$AAl?$AAs?$AA?$AA@ 001431e0     atcmd.obj
 0002:000021f8       ??_C@_1DI@LJBDKNNH@?$AAS?$AAe?$AAt?$AAU?$AAS?$AAS?$AAD?$AAN?$AAo?$AAt?$AAi?$AAf?$AAi?$AAc?$AAa?$AAt?$AAi?$AAo?$AAn?$AAC?$AAa?$AAl?$AAl?$AAb?$AAa?$AAc?$AAk?$AA?$AA@ 001431f8     atcmd.obj
 0002:00002230       ??_C@_1CG@JABLONJK@?$AAS?$AAe?$AAt?$AAI?$AAn?$AAf?$AAo?$AAR?$AAe?$AAc?$AAC?$AAa?$AAl?$AAl?$AAb?$AAa?$AAc?$AAk?$AA?$AA@ 00143230     atcmd.obj
 0002:00002258       ??_C@_1CI@OOGJCAEL@?$AAS?$AAe?$AAt?$AAC?$AAa?$AAl?$AAl?$AAI?$AAn?$AAf?$AAo?$AAC?$AAa?$AAl?$AAl?$AAb?$AAa?$AAc?$AAk?$AA?$AA@ 00143258     atcmd.obj
 0002:00002280       ??_C@_1BA@EMHLIJIE@?$AAE?$AAn?$AAd?$AAC?$AAa?$AAl?$AAl?$AA?$AA@ 00143280     atcmd.obj
 0002:00002290       ??_C@_1BG@BKDINFBH@?$AAA?$AAn?$AAs?$AAw?$AAe?$AAr?$AAC?$AAa?$AAl?$AAl?$AA?$AA@ 00143290     atcmd.obj
 0002:000022a8       ??_C@_1BC@JGHLMAEH@?$AAD?$AAi?$AAa?$AAl?$AAC?$AAa?$AAl?$AAl?$AA?$AA@ 001432a8     atcmd.obj
 0002:000022bc       ??_C@_1BI@PLMCJPHK@?$AAG?$AAo?$AAb?$AAi?$AAA?$AAp?$AAi?$AA?4?$AAd?$AAl?$AAl?$AA?$AA@ 001432bc     atcmd.obj
 0002:000022d4       ??_C@_0P@GHFPNOJB@bad?5allocation?$AA@ 001432d4     atcmd.obj
 0002:000022e4       ??_C@_1CC@IENOLDBP@?$AAS?$AAw?$AAi?$AAG?$AAe?$AAt?$AAP?$AAr?$AAi?$AAV?$AAe?$AAr?$AAs?$AAi?$AAo?$AAn?$AA?$AA@ 001432e4     atcmd.obj
 0002:00002308       ??_C@_1DI@JFCKKIP@?$AAS?$AAw?$AAi?$AAG?$AAe?$AAt?$AAC?$AAD?$AAM?$AAA?$AAN?$AAe?$AAt?$AAw?$AAo?$AAr?$AAk?$AAP?$AAa?$AAr?$AAa?$AAm?$AAe?$AAt?$AAe?$AAr?$AAs?$AA?$AA@ 00143308     atcmd.obj
 0002:00002340       ??_C@_1DI@MEGMPGPH@?$AAS?$AAw?$AAi?$AAS?$AAe?$AAt?$AAN?$AAe?$AAt?$AAw?$AAo?$AAr?$AAk?$AAP?$AAr?$AAe?$AAf?$AAe?$AAr?$AAe?$AAn?$AAc?$AAe?$AAG?$AAo?$AAb?$AAi?$AA?$AA@ 00143340     atcmd.obj
 0002:00002378       ??_C@_1DC@IENBGJHF@?$AAS?$AAw?$AAi?$AAG?$AAe?$AAt?$AAS?$AAe?$AAr?$AAv?$AAi?$AAn?$AAg?$AAN?$AAe?$AAt?$AAw?$AAo?$AAr?$AAk?$AAG?$AAo?$AAb?$AAi?$AA?$AA@ 00143378     atcmd.obj
 0002:000023ac       ??_C@_1DI@KLEAJEI@?$AAS?$AAw?$AAi?$AAA?$AAd?$AAd?$AAP?$AAr?$AAe?$AAf?$AAe?$AAr?$AAr?$AAe?$AAd?$AAO?$AAp?$AAe?$AAr?$AAa?$AAt?$AAo?$AAr?$AAG?$AAo?$AAb?$AAi?$AA?$AA@ 001433ac     atcmd.obj
 0002:000023e4       ??_C@_1DO@CDLJFFKE@?$AAS?$AAw?$AAi?$AAR?$AAe?$AAm?$AAo?$AAv?$AAe?$AAP?$AAr?$AAe?$AAf?$AAe?$AAr?$AAr?$AAe?$AAd?$AAO?$AAp?$AAe?$AAr?$AAa?$AAt?$AAo?$AAr?$AAG?$AAo?$AAb?$AAi?$AA?$AA@ 001433e4     atcmd.obj
 0002:00002428       ??_C@_1EA@HHNEOJEB@?$AAS?$AAw?$AAi?$AAG?$AAe?$AAt?$AAP?$AAr?$AAe?$AAf?$AAe?$AAr?$AAr?$AAe?$AAd?$AAO?$AAp?$AAe?$AAr?$AAa?$AAt?$AAo?$AAr?$AAL?$AAi?$AAs?$AAt?$AAG?$AAo?$AAb?$AAi?$AA?$AA@ 00143428     atcmd.obj
 0002:00002468       ??_C@_1CE@KMDCCBPL@?$AAS?$AAw?$AAi?$AAS?$AAe?$AAt?$AAG?$AAs?$AAm?$AAS?$AAM?$AAS?$AAC?$AAA?$AAd?$AAd?$AAr?$AA?$AA@ 00143468     atcmd.obj
 0002:0000248c       ??_C@_1CE@CNFNJBNJ@?$AAS?$AAw?$AAi?$AAG?$AAe?$AAt?$AAG?$AAs?$AAm?$AAS?$AAM?$AAS?$AAC?$AAA?$AAd?$AAd?$AAr?$AA?$AA@ 0014348c     atcmd.obj
 0002:000024b0       ??_C@_1CA@ECPEKBFP@?$AAS?$AAw?$AAi?$AAS?$AAe?$AAt?$AAP?$AAo?$AAw?$AAe?$AAr?$AAD?$AAo?$AAw?$AAn?$AA?$AA@ 001434b0     atcmd.obj
 0002:000024d0       ??_C@_1CA@CMCFIBHO@?$AAS?$AAw?$AAi?$AAG?$AAe?$AAt?$AAP?$AAi?$AAn?$AAS?$AAt?$AAa?$AAt?$AAu?$AAs?$AA?$AA@ 001434d0     atcmd.obj
 0002:000024f0       ??_C@_1BM@JIANFDKK@?$AAS?$AAw?$AAi?$AAG?$AAe?$AAt?$AAM?$AAE?$AAI?$AAD?$AAE?$AAS?$AAN?$AA?$AA@ 001434f0     atcmd.obj
 0002:0000250c       ??_C@_1BM@HALENEKC@?$AAS?$AAw?$AAi?$AAG?$AAe?$AAt?$AAE?$AAS?$AAN?$AAG?$AAo?$AAb?$AAi?$AA?$AA@ 0014350c     atcmd.obj
 0002:00002528       ??_C@_1CA@IDGPCPEM@?$AAS?$AAw?$AAi?$AAH?$AAa?$AAn?$AAd?$AAl?$AAe?$AAR?$AAe?$AAs?$AAu?$AAm?$AAe?$AA?$AA@ 00143528     atcmd.obj
 0002:00002548       ??_C@_1CC@NEIIFDKE@?$AAS?$AAw?$AAi?$AAH?$AAa?$AAn?$AAd?$AAl?$AAe?$AAS?$AAu?$AAs?$AAp?$AAe?$AAn?$AAd?$AA?$AA@ 00143548     atcmd.obj
 0002:0000256c       ??_C@_1DE@OJPFFICG@?$AAS?$AAw?$AAi?$AAG?$AAe?$AAt?$AAI?$AAP?$AAC?$AAo?$AAn?$AAf?$AAi?$AAg?$AAu?$AAr?$AAa?$AAt?$AAi?$AAo?$AAn?$AAG?$AAo?$AAb?$AAi?$AA?$AA@ 0014356c     atcmd.obj
 0002:000025a0       ??_C@_1CI@EKKPBEMO@?$AAS?$AAw?$AAi?$AAS?$AAe?$AAt?$AAS?$AAi?$AAm?$AAV?$AAe?$AAr?$AAi?$AAf?$AAy?$AAG?$AAo?$AAb?$AAi?$AA?$AA@ 001435a0     atcmd.obj
 0002:000025c8       ??_C@_1CI@PNBAEJLF@?$AAS?$AAw?$AAi?$AAG?$AAe?$AAt?$AAS?$AAi?$AAm?$AAV?$AAe?$AAr?$AAi?$AAf?$AAy?$AAG?$AAo?$AAb?$AAi?$AA?$AA@ 001435c8     atcmd.obj
 0002:000025f0       ??_C@_1CM@ICKBFCJL@?$AAS?$AAw?$AAi?$AAS?$AAe?$AAt?$AAS?$AAi?$AAm?$AAP?$AAa?$AAs?$AAs?$AAw?$AAo?$AAr?$AAd?$AAG?$AAo?$AAb?$AAi?$AA?$AA@ 001435f0     atcmd.obj
 0002:0000261c       ??_C@_1CE@HICGHFBG@?$AAS?$AAw?$AAi?$AAS?$AAe?$AAt?$AAS?$AAi?$AAm?$AAL?$AAo?$AAc?$AAk?$AAG?$AAo?$AAb?$AAi?$AA?$AA@ 0014361c     atcmd.obj
 0002:00002640       ??_C@_1CE@PJEJMFDE@?$AAS?$AAw?$AAi?$AAG?$AAe?$AAt?$AAS?$AAi?$AAm?$AAL?$AAo?$AAc?$AAk?$AAG?$AAo?$AAb?$AAi?$AA?$AA@ 00143640     atcmd.obj
 0002:00002664       ??_C@_1CA@EOLOMMOG@?$AAS?$AAw?$AAi?$AAG?$AAe?$AAt?$AAI?$AAP?$AAA?$AAd?$AAd?$AAr?$AAe?$AAs?$AAs?$AA?$AA@ 00143664     atcmd.obj
 0002:00002684       ??_C@_1CM@DMBPHJBN@?$AAS?$AAw?$AAi?$AAG?$AAe?$AAt?$AAG?$AAs?$AAm?$AAS?$AAy?$AAs?$AAt?$AAe?$AAm?$AAS?$AAt?$AAa?$AAt?$AAu?$AAs?$AA?$AA@ 00143684     atcmd.obj
 0002:000026b0       ??_C@_1CK@OHEKEBLG@?$AAS?$AAw?$AAi?$AAG?$AAe?$AAt?$AAP?$AAh?$AAo?$AAn?$AAe?$AAb?$AAo?$AAo?$AAk?$AAE?$AAn?$AAt?$AAr?$AAy?$AA?$AA@ 001436b0     atcmd.obj
 0002:000026dc       ??_C@_1CM@PIBNMFKG@?$AAS?$AAw?$AAi?$AAS?$AAe?$AAt?$AAG?$AAs?$AAm?$AAP?$AAr?$AAo?$AAf?$AAi?$AAl?$AAe?$AAB?$AAa?$AAs?$AAi?$AAc?$AA?$AA@ 001436dc     atcmd.obj
 0002:00002708       ??_C@_1BG@PHLKENOP@?$AAS?$AAw?$AAi?$AAG?$AAe?$AAt?$AAI?$AAm?$AAe?$AAi?$AA?$AA@ 00143708     atcmd.obj
 0002:00002720       ??_C@_1DC@DPCECLCK@?$AAS?$AAw?$AAi?$AAS?$AAe?$AAn?$AAd?$AAG?$AAe?$AAn?$AAe?$AAr?$AAi?$AAc?$AAS?$AAi?$AAm?$AAC?$AAo?$AAm?$AAm?$AAa?$AAn?$AAd?$AA?$AA@ 00143720     atcmd.obj
 0002:00002754       ??_C@_1CM@PNDIGLJM@?$AAS?$AAw?$AAi?$AAG?$AAe?$AAt?$AAS?$AAI?$AAM?$AAR?$AAe?$AAc?$AAo?$AAr?$AAd?$AAS?$AAt?$AAa?$AAt?$AAu?$AAs?$AA?$AA@ 00143754     atcmd.obj
 0002:00002780       ??_C@_1DA@FEPOGCNF@?$AAS?$AAw?$AAi?$AAS?$AAe?$AAn?$AAd?$AAR?$AAe?$AAs?$AAt?$AAr?$AAi?$AAc?$AAt?$AAe?$AAd?$AAS?$AAI?$AAM?$AAC?$AAm?$AAd?$AA?$AA@ 00143780     atcmd.obj
 0002:000027b0       ??_C@_1BM@NMEPFPPD@?$AAS?$AAw?$AAi?$AAS?$AAe?$AAt?$AAP?$AAr?$AAo?$AAf?$AAi?$AAl?$AAe?$AA?$AA@ 001437b0     atcmd.obj
 0002:000027cc       ??_C@_1BO@CIHFPALC@?$AAS?$AAw?$AAi?$AAS?$AAe?$AAt?$AAP?$AAL?$AAM?$AAN?$AAM?$AAo?$AAd?$AAe?$AA?$AA@ 001437cc     atcmd.obj
 0002:000027ec       ??_C@_1CG@KHGPLFG@?$AAS?$AAw?$AAi?$AAA?$AAc?$AAt?$AAi?$AAv?$AAa?$AAt?$AAe?$AAP?$AAr?$AAo?$AAf?$AAi?$AAl?$AAe?$AA?$AA@ 001437ec     atcmd.obj
 0002:00002814       ??_C@_1BM@JPFBKOLP@?$AAS?$AAw?$AAi?$AAG?$AAe?$AAt?$AAG?$AAs?$AAm?$AAI?$AAM?$AAS?$AAI?$AA?$AA@ 00143814     atcmd.obj
 0002:00002830       ??_C@_1DA@ENPHNEFA@?$AAS?$AAw?$AAi?$AAG?$AAe?$AAt?$AAT?$AAr?$AAa?$AAf?$AAf?$AAi?$AAc?$AAS?$AAt?$AAa?$AAt?$AAi?$AAs?$AAt?$AAi?$AAc?$AAs?$AA?$AA@ 00143830     atcmd.obj
 0002:00002860       ??_C@_1CG@IFHAOAAO@?$AAS?$AAw?$AAi?$AAS?$AAt?$AAa?$AAr?$AAt?$AAP?$AAL?$AAM?$AAN?$AAS?$AAe?$AAa?$AAr?$AAc?$AAh?$AA?$AA@ 00143860     atcmd.obj
 0002:00002888       ??_C@_1CI@GGJBIKFN@?$AAS?$AAw?$AAi?$AAG?$AAe?$AAt?$AAP?$AAL?$AAM?$AAN?$AAS?$AAe?$AAl?$AAe?$AAc?$AAt?$AAi?$AAo?$AAn?$AA?$AA@ 00143888     atcmd.obj
 0002:000028b0       ??_C@_1DA@IAEGLCBE@?$AAS?$AAw?$AAi?$AAG?$AAe?$AAt?$AAG?$AAs?$AAm?$AAP?$AAr?$AAo?$AAf?$AAi?$AAl?$AAe?$AAS?$AAu?$AAm?$AAm?$AAa?$AAr?$AAy?$AA?$AA@ 001438b0     atcmd.obj
 0002:000028e0       ??_C@_1CM@BGBPMLIA@?$AAS?$AAw?$AAi?$AAG?$AAe?$AAt?$AAG?$AAs?$AAm?$AAP?$AAr?$AAo?$AAf?$AAi?$AAl?$AAe?$AAB?$AAa?$AAs?$AAi?$AAc?$AA?$AA@ 001438e0     atcmd.obj
 0002:0000290c       ??_C@_1CE@EBJOMJIK@?$AAS?$AAw?$AAi?$AAS?$AAe?$AAt?$AAH?$AAo?$AAs?$AAt?$AAS?$AAt?$AAa?$AAr?$AAt?$AAu?$AAp?$AA?$AA@ 0014390c     atcmd.obj
 0002:00002930       ??_C@_1CK@DFCLIICL@?$AAS?$AAw?$AAi?$AAP?$AAr?$AAi?$AAG?$AAe?$AAt?$AAM?$AAa?$AAx?$AAM?$AAo?$AAs?$AAm?$AAs?$AAL?$AAe?$AAn?$AA?$AA@ 00143930     atcmd.obj
 0002:0000295c       ??_C@_1DA@GLBAEJEH@?$AAS?$AAw?$AAi?$AAP?$AAr?$AAi?$AAG?$AAe?$AAt?$AAA?$AAc?$AAt?$AAi?$AAv?$AAa?$AAt?$AAi?$AAo?$AAn?$AAM?$AAa?$AAs?$AAk?$AA?$AA@ 0014395c     atcmd.obj
 0002:0000298c       ??_C@_1CK@IMNEHMJE@?$AAS?$AAw?$AAi?$AAP?$AAs?$AAt?$AAG?$AAe?$AAt?$AAH?$AAd?$AAr?$AAP?$AAa?$AAs?$AAs?$AAw?$AAo?$AAr?$AAd?$AA?$AA@ 0014398c     atcmd.obj
 0002:000029b8       ??_C@_1CG@GEHBLOPO@?$AAS?$AAw?$AAi?$AAP?$AAs?$AAt?$AAG?$AAe?$AAt?$AAH?$AAd?$AAr?$AAU?$AAs?$AAe?$AAr?$AAI?$AAd?$AA?$AA@ 001439b8     atcmd.obj
 0002:000029e0       ??_C@_1CE@BLMCHMOH@?$AAS?$AAw?$AAi?$AAP?$AAs?$AAt?$AAS?$AAe?$AAt?$AAI?$AAm?$AAs?$AAi?$AA1?$AA1?$AA1?$AA2?$AA?$AA@ 001439e0     atcmd.obj
 0002:00002a04       ??_C@_1CC@ODNPEKIG@?$AAS?$AAw?$AAi?$AAP?$AAs?$AAt?$AAS?$AAe?$AAt?$AAI?$AAm?$AAs?$AAi?$AAM?$AAc?$AAc?$AA?$AA@ 00143a04     atcmd.obj
 0002:00002a28       ??_C@_1DI@JPANBIKM@?$AAS?$AAw?$AAi?$AAG?$AAe?$AAt?$AAG?$AAe?$AAn?$AAe?$AAr?$AAa?$AAl?$AAF?$AAe?$AAa?$AAt?$AAu?$AAr?$AAe?$AAS?$AAu?$AAp?$AAp?$AAo?$AAr?$AAt?$AA?$AA@ 00143a28     atcmd.obj
 0002:00002a60       ??_C@_1CI@ICBPPJIN@?$AAS?$AAw?$AAi?$AAR?$AAe?$AAs?$AAe?$AAt?$AAB?$AAy?$AAt?$AAe?$AAC?$AAo?$AAu?$AAn?$AAt?$AAe?$AAr?$AA?$AA@ 00143a60     atcmd.obj
 0002:00002a88       ??_C@_1BG@LJHLEDEM@?$AAS?$AAw?$AAi?$AAS?$AAe?$AAt?$AAA?$AAK?$AAe?$AAy?$AA?$AA@ 00143a88     atcmd.obj
 0002:00002aa0       ??_C@_1BM@CDMOPMHM@?$AAS?$AAw?$AAi?$AAS?$AAe?$AAt?$AAD?$AAo?$AAr?$AAm?$AAa?$AAn?$AAt?$AA?$AA@ 00143aa0     atcmd.obj
 0002:00002abc       ??_C@_1CC@NKMHGHPM@?$AAS?$AAw?$AAi?$AAP?$AAo?$AAw?$AAe?$AAr?$AAS?$AAa?$AAv?$AAe?$AAE?$AAx?$AAi?$AAt?$AA?$AA@ 00143abc     atcmd.obj
 0002:00002ae0       ??_C@_1CM@NCJAHMAJ@?$AAS?$AAw?$AAi?$AAG?$AAe?$AAt?$AAA?$AAv?$AAa?$AAi?$AAl?$AAA?$AAi?$AAr?$AAS?$AAe?$AAr?$AAv?$AAe?$AAr?$AAs?$AA?$AA@ 00143ae0     atcmd.obj
 0002:00002b0c       ??_C@_1BG@PEENOIKK@?$AAS?$AAw?$AAi?$AAG?$AAe?$AAt?$AAE?$AAC?$AAI?$AAO?$AA?$AA@ 00143b0c     atcmd.obj
 0002:00002b24       ??_C@_1BG@KKEIBLHB@?$AAS?$AAw?$AAi?$AAP?$AAs?$AAt?$AAL?$AAo?$AAc?$AAk?$AA?$AA@ 00143b24     atcmd.obj
 0002:00002b3c       ??_C@_1BK@EMFGHDEM@?$AAS?$AAw?$AAi?$AAP?$AAs?$AAt?$AAS?$AAe?$AAt?$AAS?$AAc?$AAi?$AA?$AA@ 00143b3c     atcmd.obj
 0002:00002b58       ??_C@_1CG@GHILBCDP@?$AAS?$AAw?$AAi?$AAS?$AAe?$AAt?$AAN?$AAD?$AAI?$AAS?$AAP?$AAr?$AAe?$AAf?$AAM?$AAo?$AAd?$AAe?$AA?$AA@ 00143b58     atcmd.obj
 0002:00002b80       ??_C@_1BO@PBJOKDAH@?$AAS?$AAw?$AAi?$AAG?$AAe?$AAt?$AAN?$AAD?$AAI?$AAS?$AAM?$AAo?$AAd?$AAe?$AA?$AA@ 00143b80     atcmd.obj
 0002:00002ba0       ??_C@_1BM@CIGLOAEP@?$AAS?$AAw?$AAi?$AAR?$AAe?$AAs?$AAe?$AAt?$AAM?$AAo?$AAd?$AAe?$AAm?$AA?$AA@ 00143ba0     atcmd.obj
 0002:00002bbc       ??_C@_1BM@IEIJNEJG@?$AAS?$AAw?$AAi?$AAS?$AAt?$AAo?$AAp?$AAN?$AAo?$AAt?$AAi?$AAf?$AAy?$AA?$AA@ 00143bbc     atcmd.obj
 0002:00002bd8       ??_C@_1BE@GOLJPDNF@?$AAS?$AAw?$AAi?$AAN?$AAo?$AAt?$AAi?$AAf?$AAy?$AA?$AA@ 00143bd8     atcmd.obj
 0002:00002bec       ??_C@_1CM@BCIHGEPN@?$AAS?$AAw?$AAi?$AAD?$AAe?$AAR?$AAe?$AAg?$AAi?$AAs?$AAt?$AAe?$AAr?$AAC?$AAa?$AAl?$AAl?$AAb?$AAa?$AAc?$AAk?$AA?$AA@ 00143bec     atcmd.obj
 0002:00002c18       ??_C@_1CI@NCCHBDEC@?$AAS?$AAw?$AAi?$AAR?$AAe?$AAg?$AAi?$AAs?$AAt?$AAe?$AAr?$AAC?$AAa?$AAl?$AAl?$AAb?$AAa?$AAc?$AAk?$AA?$AA@ 00143c18     atcmd.obj
 0002:00002c40       ??_C@_1DA@JGJOPAHE@?$AAS?$AAw?$AAi?$AAG?$AAe?$AAt?$AAT?$AAe?$AAc?$AAh?$AAP?$AAo?$AAw?$AAe?$AAr?$AAs?$AAa?$AAv?$AAe?$AAM?$AAo?$AAd?$AAe?$AA?$AA@ 00143c40     atcmd.obj
 0002:00002c70       ??_C@_1CA@CGACPPEE@?$AAS?$AAw?$AAi?$AAG?$AAe?$AAt?$AAC?$AAa?$AAr?$AAr?$AAi?$AAe?$AAr?$AAI?$AAD?$AA?$AA@ 00143c70     atcmd.obj
 0002:00002c90       ??_C@_1BI@GIKGBDNP@?$AAS?$AAw?$AAi?$AAG?$AAe?$AAt?$AAE?$AAF?$AAi?$AAl?$AAe?$AA?$AA@ 00143c90     atcmd.obj
 0002:00002ca8       ??_C@_1CA@PFCKLJGN@?$AAS?$AAw?$AAi?$AAG?$AAe?$AAt?$AAE?$AAF?$AAi?$AAl?$AAe?$AAI?$AAn?$AAf?$AAo?$AA?$AA@ 00143ca8     atcmd.obj
 0002:00002cc8       ??_C@_1BI@KAAOJHKJ@?$AAS?$AAw?$AAi?$AAR?$AAt?$AAn?$AAR?$AAe?$AAs?$AAe?$AAt?$AA?$AA@ 00143cc8     atcmd.obj
 0002:00002ce0       ??_C@_1CG@HMDNHHOA@?$AAS?$AAw?$AAi?$AAP?$AAr?$AAi?$AAG?$AAe?$AAt?$AAM?$AAD?$AAN?$AAL?$AAe?$AAn?$AAg?$AAt?$AAh?$AA?$AA@ 00143ce0     atcmd.obj
 0002:00002d08       ??_C@_1CA@JCINPHO@?$AAS?$AAw?$AAi?$AAG?$AAe?$AAt?$AAA?$AAc?$AAt?$AAi?$AAv?$AAe?$AAN?$AAa?$AAm?$AA?$AA@ 00143d08     atcmd.obj
 0002:00002d28       ??_C@_1CE@BGEAEHEA@?$AAS?$AAw?$AAi?$AAG?$AAe?$AAt?$AAP?$AAh?$AAo?$AAn?$AAe?$AAN?$AAu?$AAm?$AAb?$AAe?$AAr?$AA?$AA@ 00143d28     atcmd.obj
 0002:00002d4c       ??_C@_1CI@IGEDNCOH@?$AAS?$AAw?$AAi?$AAG?$AAe?$AAt?$AAT?$AAe?$AAc?$AAh?$AAB?$AAa?$AAn?$AAd?$AAC?$AAl?$AAa?$AAs?$AAs?$AA?$AA@ 00143d4c     atcmd.obj
 0002:00002d74       ??_C@_1CI@HIEDPAC@?$AAS?$AAw?$AAi?$AAG?$AAe?$AAt?$AAC?$AAh?$AAa?$AAn?$AAn?$AAe?$AAl?$AAN?$AAu?$AAm?$AAb?$AAe?$AAr?$AA?$AA@ 00143d74     atcmd.obj
 0002:00002d9c       ??_C@_1BM@FJMIBGDK@?$AAS?$AAw?$AAi?$AAG?$AAe?$AAt?$AAT?$AAe?$AAc?$AAh?$AAN?$AAI?$AAD?$AA?$AA@ 00143d9c     atcmd.obj
 0002:00002db8       ??_C@_1BM@LOHGDCMA@?$AAS?$AAw?$AAi?$AAG?$AAe?$AAt?$AAT?$AAe?$AAc?$AAh?$AAS?$AAI?$AAD?$AA?$AA@ 00143db8     atcmd.obj
 0002:00002dd4       ??_C@_1DG@LDNMCDKH@?$AAS?$AAw?$AAi?$AAP?$AAs?$AAt?$AAG?$AAe?$AAt?$AAD?$AAi?$AAs?$AAp?$AAl?$AAa?$AAy?$AAB?$AAa?$AAn?$AAn?$AAe?$AAr?$AAN?$AAa?$AAm?$AAe?$AA?$AA@ 00143dd4     atcmd.obj
 0002:00002e0c       ??_C@_1CG@KHNBCGJA@?$AAS?$AAw?$AAi?$AAS?$AAe?$AAt?$AAT?$AAe?$AAm?$AAp?$AAM?$AAo?$AAd?$AAe?$AAP?$AAr?$AAe?$AAf?$AA?$AA@ 00143e0c     atcmd.obj
 0002:00002e34       ??_C@_1CI@FBNKOANF@?$AAS?$AAw?$AAi?$AAP?$AAs?$AAt?$AAG?$AAe?$AAt?$AAS?$AAy?$AAs?$AAt?$AAe?$AAm?$AAP?$AAr?$AAe?$AAf?$AA?$AA@ 00143e34     atcmd.obj
 0002:00002e5c       ??_C@_1DG@IHICJCIB@?$AAS?$AAw?$AAi?$AAG?$AAe?$AAt?$AAC?$AAd?$AAm?$AAa?$AAS?$AAM?$AAS?$AAM?$AAe?$AAs?$AAs?$AAa?$AAg?$AAe?$AAS?$AAt?$AAa?$AAt?$AAu?$AAs?$AA?$AA@ 00143e5c     atcmd.obj
 0002:00002e94       ??_C@_1DE@PJGLKFBD@?$AAS?$AAw?$AAi?$AAR?$AAe?$AAt?$AAr?$AAi?$AAe?$AAv?$AAe?$AAC?$AAd?$AAm?$AAa?$AAS?$AAM?$AAS?$AAM?$AAe?$AAs?$AAs?$AAa?$AAg?$AAe?$AA?$AA@ 00143e94     atcmd.obj
 0002:00002ec8       ??_C@_1CO@LPDMDDCF@?$AAS?$AAw?$AAi?$AAS?$AAt?$AAo?$AAr?$AAe?$AAC?$AAd?$AAm?$AAa?$AAS?$AAM?$AAS?$AAM?$AAe?$AAs?$AAs?$AAa?$AAg?$AAe?$AA?$AA@ 00143ec8     atcmd.obj
 0002:00002ef8       ??_C@_1BO@BHHMHHMC@?$AAS?$AAw?$AAi?$AAS?$AAe?$AAn?$AAd?$AAC?$AAd?$AAm?$AAa?$AAS?$AAM?$AAS?$AA?$AA@ 00143ef8     atcmd.obj
 0002:00002f18       ??_C@_1BG@HNAOGMNK@?$AAS?$AAw?$AAi?$AAS?$AAe?$AAn?$AAd?$AAS?$AAM?$AAS?$AA?$AA@ 00143f18     atcmd.obj
 0002:00002f30       ??_C@_1CO@MOBKEOCJ@?$AAS?$AAw?$AAi?$AAS?$AAt?$AAo?$AAr?$AAe?$AAS?$AAM?$AAS?$AAM?$AAe?$AAs?$AAs?$AAa?$AAg?$AAe?$AAG?$AAo?$AAb?$AAi?$AA?$AA@ 00143f30     atcmd.obj
 0002:00002f60       ??_C@_1DE@IIENNIBP@?$AAS?$AAw?$AAi?$AAR?$AAe?$AAt?$AAr?$AAi?$AAe?$AAv?$AAe?$AAS?$AAM?$AAS?$AAM?$AAe?$AAs?$AAs?$AAa?$AAg?$AAe?$AAG?$AAo?$AAb?$AAi?$AA?$AA@ 00143f60     atcmd.obj
 0002:00002f94       ??_C@_1CO@PMNEBND@?$AAS?$AAw?$AAi?$AAG?$AAe?$AAt?$AAS?$AAM?$AAS?$AAM?$AAe?$AAs?$AAs?$AAa?$AAg?$AAe?$AAS?$AAt?$AAa?$AAt?$AAu?$AAs?$AA?$AA@ 00143f94     atcmd.obj
 0002:00002fc4       ??_C@_1CE@OPALKDKA@?$AAS?$AAw?$AAi?$AAP?$AAs?$AAt?$AAS?$AAe?$AAt?$AAP?$AAr?$AAe?$AAf?$AAM?$AAo?$AAd?$AAe?$AA?$AA@ 00143fc4     atcmd.obj
 0002:00002fe8       ??_C@_1CE@PJGGECMC@?$AAS?$AAw?$AAi?$AAP?$AAs?$AAt?$AAG?$AAe?$AAt?$AAP?$AAr?$AAe?$AAf?$AAM?$AAo?$AAd?$AAe?$AA?$AA@ 00143fe8     atcmd.obj
 0002:0000300c       ??_C@_1CE@DGMHLNJL@?$AAS?$AAw?$AAi?$AAS?$AAe?$AAt?$AAH?$AAd?$AAr?$AAH?$AAy?$AAb?$AAr?$AAP?$AAr?$AAe?$AAf?$AA?$AA@ 0014400c     atcmd.obj
 0002:00003030       ??_C@_1CE@LHKIANLJ@?$AAS?$AAw?$AAi?$AAG?$AAe?$AAt?$AAH?$AAd?$AAr?$AAH?$AAy?$AAb?$AAr?$AAP?$AAr?$AAe?$AAf?$AA?$AA@ 00144030     atcmd.obj
 0002:00003054       ??_C@_1DC@ONDMGNIP@?$AAS?$AAw?$AAi?$AAP?$AAs?$AAt?$AAS?$AAe?$AAt?$AAD?$AAs?$AAM?$AAi?$AAp?$AAA?$AAc?$AAt?$AAi?$AAv?$AAe?$AAP?$AAr?$AAo?$AAf?$AA?$AA@ 00144054     atcmd.obj
 0002:00003088       ??_C@_1DC@EIIONCMM@?$AAS?$AAw?$AAi?$AAP?$AAs?$AAt?$AAS?$AAe?$AAt?$AAD?$AAs?$AAM?$AAi?$AAp?$AAS?$AAs?$AAU?$AAs?$AAe?$AAr?$AAP?$AAr?$AAo?$AAf?$AA?$AA@ 00144088     atcmd.obj
 0002:000030bc       ??_C@_1CM@LMPPEFNJ@?$AAS?$AAw?$AAi?$AAP?$AAs?$AAt?$AAS?$AAe?$AAt?$AAD?$AAs?$AAM?$AAi?$AAp?$AAG?$AAe?$AAn?$AAU?$AAs?$AAe?$AAr?$AA?$AA@ 001440bc     atcmd.obj
 0002:000030e8       ??_C@_1DC@KGIMNMOK@?$AAS?$AAw?$AAi?$AAP?$AAs?$AAt?$AAG?$AAe?$AAt?$AAD?$AAs?$AAM?$AAi?$AAp?$AAS?$AAs?$AAU?$AAs?$AAe?$AAr?$AAP?$AAr?$AAo?$AAf?$AA?$AA@ 001440e8     atcmd.obj
 0002:0000311c       ??_C@_1CM@NACMDBBK@?$AAS?$AAw?$AAi?$AAP?$AAs?$AAt?$AAG?$AAe?$AAt?$AAD?$AAs?$AAM?$AAi?$AAp?$AAG?$AAe?$AAn?$AAU?$AAs?$AAe?$AAr?$AA?$AA@ 0014411c     atcmd.obj
 0002:00003148       ??_C@_1DC@MNMJAGLB@?$AAS?$AAw?$AAi?$AAP?$AAs?$AAt?$AAG?$AAe?$AAt?$AAD?$AAs?$AAM?$AAi?$AAp?$AAE?$AAn?$AAa?$AAb?$AAl?$AAe?$AAP?$AAr?$AAo?$AAf?$AA?$AA@ 00144148     atcmd.obj
 0002:0000317c       ??_C@_1DC@DDOGDKJ@?$AAS?$AAw?$AAi?$AAP?$AAs?$AAt?$AAG?$AAe?$AAt?$AAD?$AAs?$AAM?$AAi?$AAp?$AAA?$AAc?$AAt?$AAi?$AAv?$AAe?$AAP?$AAr?$AAo?$AAf?$AA?$AA@ 0014417c     atcmd.obj
 0002:000031b0       ??_C@_1CC@LCPFLGML@?$AAS?$AAw?$AAi?$AAP?$AAs?$AAt?$AAG?$AAe?$AAt?$AAD?$AAs?$AAQ?$AAc?$AAM?$AAi?$AAp?$AA?$AA@ 001441b0     atcmd.obj
 0002:000031d4       ??_C@_1CC@EHKDGPIK@?$AAS?$AAw?$AAi?$AAP?$AAs?$AAt?$AAS?$AAe?$AAt?$AAD?$AAs?$AAQ?$AAc?$AAM?$AAi?$AAp?$AA?$AA@ 001441d4     atcmd.obj
 0002:000031f8       ??_C@_1CK@NLLMMLG@?$AAS?$AAw?$AAi?$AAP?$AAs?$AAt?$AAS?$AAe?$AAt?$AAH?$AAd?$AAr?$AAP?$AAa?$AAs?$AAs?$AAw?$AAo?$AAr?$AAd?$AA?$AA@ 001441f8     atcmd.obj
 0002:00003224       ??_C@_1CG@OELHHDFI@?$AAS?$AAw?$AAi?$AAP?$AAs?$AAt?$AAS?$AAe?$AAt?$AAH?$AAd?$AAr?$AAU?$AAs?$AAe?$AAr?$AAI?$AAd?$AA?$AA@ 00144224     atcmd.obj
 0002:0000324c       ??_C@_1CA@JOJODJAB@?$AAS?$AAw?$AAi?$AAP?$AAs?$AAt?$AAS?$AAe?$AAt?$AAA?$AAc?$AAc?$AAo?$AAl?$AAc?$AA?$AA@ 0014424c     atcmd.obj
 0002:0000326c       ??_C@_1BG@EOMLBGCO@?$AAS?$AAw?$AAi?$AAS?$AAe?$AAt?$AAI?$AAM?$AAS?$AAI?$AA?$AA@ 0014426c     atcmd.obj
 0002:00003284       ??_C@_1CG@LDLFMJAC@?$AAS?$AAw?$AAi?$AAS?$AAe?$AAt?$AAM?$AAo?$AAb?$AAi?$AAl?$AAe?$AAD?$AAi?$AAr?$AAN?$AAu?$AAm?$AA?$AA@ 00144284     atcmd.obj
 0002:000032ac       ??_C@_1CI@EABJILOD@?$AAS?$AAw?$AAi?$AAP?$AAs?$AAt?$AAS?$AAe?$AAt?$AAH?$AAo?$AAm?$AAe?$AAS?$AAi?$AAd?$AAN?$AAi?$AAd?$AA?$AA@ 001442ac     atcmd.obj
 0002:000032d4       ??_C@_1CI@CFIKJPKB@?$AAS?$AAw?$AAi?$AAP?$AAs?$AAt?$AAS?$AAe?$AAt?$AAC?$AAu?$AAr?$AAr?$AAe?$AAn?$AAt?$AAN?$AAa?$AAm?$AA?$AA@ 001442d4     atcmd.obj
 0002:000032fc       ??_C@_1BK@DDEIMADL@?$AAS?$AAw?$AAi?$AAP?$AAs?$AAt?$AAG?$AAe?$AAt?$AAS?$AAc?$AAi?$AA?$AA@ 001442fc     atcmd.obj
 0002:00003318       ??_C@_1CA@DALFHJHN@?$AAS?$AAw?$AAi?$AAP?$AAs?$AAt?$AAG?$AAe?$AAt?$AAA?$AAc?$AAc?$AAo?$AAl?$AAc?$AA?$AA@ 00144318     atcmd.obj
 0002:00003338       ??_C@_1CI@FNJBKOEH@?$AAS?$AAw?$AAi?$AAP?$AAs?$AAt?$AAG?$AAe?$AAt?$AAH?$AAo?$AAm?$AAe?$AAS?$AAi?$AAd?$AAN?$AAi?$AAd?$AA?$AA@ 00144338     atcmd.obj
 0002:00003360       ??_C@_1BO@HIPDKKAL@?$AAS?$AAw?$AAi?$AAG?$AAe?$AAt?$AAC?$AAd?$AAm?$AAa?$AAI?$AAM?$AAS?$AAI?$AA?$AA@ 00144360     atcmd.obj
 0002:00003380       ??_C@_1CE@NKPJNIF@?$AAS?$AAw?$AAi?$AAP?$AAs?$AAt?$AAG?$AAe?$AAt?$AAI?$AAm?$AAs?$AAi?$AA1?$AA1?$AA1?$AA2?$AA?$AA@ 00144380     atcmd.obj
 0002:000033a4       ??_C@_1CC@BGIJJDMH@?$AAS?$AAw?$AAi?$AAP?$AAs?$AAt?$AAG?$AAe?$AAt?$AAI?$AAm?$AAs?$AAi?$AAM?$AAc?$AAc?$AA?$AA@ 001443a4     atcmd.obj
 0002:000033c8       ??_C@_1CC@OKDAABBP@?$AAS?$AAw?$AAi?$AAP?$AAs?$AAt?$AAG?$AAe?$AAt?$AAT?$AAe?$AAr?$AAm?$AAN?$AAi?$AAd?$AA?$AA@ 001443c8     atcmd.obj
 0002:000033ec       ??_C@_1CC@NIOCFOF@?$AAS?$AAw?$AAi?$AAP?$AAs?$AAt?$AAG?$AAe?$AAt?$AAT?$AAe?$AAr?$AAm?$AAS?$AAi?$AAd?$AA?$AA@ 001443ec     atcmd.obj
 0002:00003410       ??_C@_1CE@FKNLPLAB@?$AAS?$AAw?$AAi?$AAP?$AAs?$AAt?$AAG?$AAe?$AAt?$AAT?$AAe?$AAr?$AAm?$AAH?$AAo?$AAm?$AAe?$AA?$AA@ 00144410     atcmd.obj
 0002:00003434       ??_C@_1CM@DCILJAJM@?$AAS?$AAw?$AAi?$AAG?$AAe?$AAt?$AAH?$AAa?$AAr?$AAd?$AAw?$AAa?$AAr?$AAe?$AAV?$AAe?$AAr?$AAs?$AAi?$AAo?$AAn?$AA?$AA@ 00144434     atcmd.obj
 0002:00003460       ??_C@_1BM@LMJBLBBE@?$AAS?$AAw?$AAi?$AAG?$AAe?$AAt?$AAP?$AAr?$AAi?$AAI?$AAn?$AAf?$AAo?$AA?$AA@ 00144460     atcmd.obj
 0002:0000347c       ??_C@_1BK@IJBENDFB@?$AAS?$AAw?$AAi?$AAP?$AAs?$AAt?$AAU?$AAn?$AAl?$AAo?$AAc?$AAk?$AA?$AA@ 0014447c     atcmd.obj
 0002:00003498       ??_C@_1CE@BIKCGOEC@?$AAS?$AAw?$AAi?$AAG?$AAe?$AAt?$AAB?$AAo?$AAo?$AAt?$AAV?$AAe?$AAr?$AAs?$AAi?$AAo?$AAn?$AA?$AA@ 00144498     atcmd.obj
 0002:000034bc       ??_C@_1CC@CHJODKMD@?$AAS?$AAw?$AAi?$AAG?$AAe?$AAt?$AAP?$AAR?$AAL?$AAV?$AAe?$AAr?$AAs?$AAi?$AAo?$AAn?$AA?$AA@ 001444bc     atcmd.obj
 0002:000034e0       ??_C@_1CM@BCJCCGNN@?$AAS?$AAw?$AAi?$AAG?$AAe?$AAt?$AAF?$AAi?$AAr?$AAm?$AAw?$AAa?$AAr?$AAe?$AAV?$AAe?$AAr?$AAs?$AAi?$AAo?$AAn?$AA?$AA@ 001444e0     atcmd.obj
 0002:0000350c       ??_C@_1CC@GKKJAOIA@?$AAS?$AAw?$AAi?$AAG?$AAe?$AAt?$AAS?$AAy?$AAs?$AAt?$AAe?$AAm?$AAT?$AAi?$AAm?$AAe?$AA?$AA@ 0014450c     atcmd.obj
 0002:00003530       ??_C@_1CE@GEIKJBFI@?$AAS?$AAw?$AAi?$AAG?$AAe?$AAt?$AAB?$AAy?$AAt?$AAe?$AAC?$AAo?$AAu?$AAn?$AAt?$AAe?$AAr?$AA?$AA@ 00144530     atcmd.obj
 0002:00003554       ??_C@_1BI@MMKFLMNO@?$AAS?$AAw?$AAi?$AAG?$AAe?$AAt?$AAP?$AAo?$AAw?$AAe?$AAr?$AA?$AA@ 00144554     atcmd.obj
 0002:0000356c       ??_C@_1BI@OJKODHMA@?$AAS?$AAw?$AAi?$AAS?$AAe?$AAt?$AAP?$AAo?$AAw?$AAe?$AAr?$AA?$AA@ 0014456c     atcmd.obj
 0002:00003584       ??_C@_1CE@LKAKPCBN@?$AAS?$AAw?$AAi?$AAG?$AAe?$AAt?$AAI?$AAO?$AAT?$AAA?$AAD?$AAi?$AAs?$AAa?$AAb?$AAl?$AAe?$AA?$AA@ 00144584     atcmd.obj
 0002:000035a8       ??_C@_1CC@EDNLMIL@?$AAS?$AAw?$AAi?$AAG?$AAe?$AAt?$AAM?$AAi?$AAp?$AAE?$AAr?$AAr?$AAC?$AAo?$AAd?$AAe?$AA?$AA@ 001445a8     atcmd.obj
 0002:000035cc       ??_C@_1CC@EAGJOJPC@?$AAS?$AAw?$AAi?$AAO?$AAM?$AAA?$AAE?$AAX?$AAS?$AAh?$AAu?$AAt?$AAd?$AAo?$AAw?$AAn?$AA?$AA@ 001445cc     atcmd.obj
 0002:000035f0       ??_C@_1BK@KFFNGFCM@?$AAS?$AAw?$AAi?$AAO?$AAM?$AAA?$AAE?$AAX?$AAI?$AAn?$AAi?$AAt?$AA?$AA@ 001445f0     atcmd.obj
 0002:0000360c       ??_C@_1CO@HHFKDDGI@?$AAS?$AAw?$AAi?$AAO?$AAM?$AAA?$AAE?$AAX?$AAG?$AAe?$AAt?$AAS?$AAe?$AAs?$AAs?$AAi?$AAo?$AAn?$AAI?$AAn?$AAf?$AAo?$AA?$AA@ 0014460c     atcmd.obj
 0002:0000363c       ??_C@_1CI@NLFFKNKH@?$AAS?$AAw?$AAi?$AAO?$AAM?$AAA?$AAE?$AAX?$AAS?$AAe?$AAt?$AAS?$AAe?$AAt?$AAt?$AAi?$AAn?$AAg?$AAs?$AA?$AA@ 0014463c     atcmd.obj
 0002:00003664       ??_C@_1CI@MNDIEMMF@?$AAS?$AAw?$AAi?$AAO?$AAM?$AAA?$AAE?$AAX?$AAG?$AAe?$AAt?$AAS?$AAe?$AAt?$AAt?$AAi?$AAn?$AAg?$AAs?$AA?$AA@ 00144664     atcmd.obj
 0002:0000368c       ??_C@_1CE@BOFEFICH@?$AAS?$AAw?$AAi?$AAO?$AAM?$AAA?$AAE?$AAX?$AAS?$AAe?$AAl?$AAe?$AAc?$AAt?$AAi?$AAo?$AAn?$AA?$AA@ 0014468c     atcmd.obj
 0002:000036b0       ??_C@_1CM@LICAIPNI@?$AAS?$AAw?$AAi?$AAO?$AAM?$AAA?$AAE?$AAX?$AAS?$AAe?$AAs?$AAs?$AAi?$AAo?$AAn?$AAC?$AAa?$AAn?$AAc?$AAe?$AAl?$AA?$AA@ 001446b0     atcmd.obj
 0002:000036dc       ??_C@_1CK@FHIOIBG@?$AAS?$AAw?$AAi?$AAO?$AAM?$AAA?$AAE?$AAX?$AAS?$AAe?$AAs?$AAs?$AAi?$AAo?$AAn?$AAS?$AAt?$AAa?$AAr?$AAt?$AA?$AA@ 001446dc     atcmd.obj
 0002:00003708       ??_C@_1CO@DMKHMAJN@?$AAS?$AAw?$AAi?$AAS?$AAe?$AAt?$AAO?$AAM?$AAA?$AAE?$AAX?$AAE?$AAv?$AAe?$AAn?$AAt?$AAR?$AAe?$AAp?$AAo?$AAr?$AAt?$AA?$AA@ 00144708     atcmd.obj
 0002:00003738       ??_C@_1DG@KIMPHPML@?$AAS?$AAw?$AAi?$AAS?$AAe?$AAt?$AAO?$AAM?$AAA?$AAD?$AAM?$AAN?$AAI?$AAA?$AAl?$AAe?$AAr?$AAt?$AAR?$AAe?$AAs?$AAp?$AAo?$AAn?$AAs?$AAe?$AA?$AA@ 00144738     atcmd.obj
 0002:00003770       ??_C@_1CG@LNDMJEE@?$AAS?$AAw?$AAi?$AAG?$AAe?$AAt?$AAO?$AAM?$AAA?$AAD?$AAM?$AAN?$AAI?$AAA?$AAl?$AAe?$AAr?$AAt?$AA?$AA@ 00144770     atcmd.obj
 0002:00003798       ??_C@_1CM@MPIBCJGP@?$AAS?$AAw?$AAi?$AAC?$AAa?$AAn?$AAc?$AAe?$AAl?$AAO?$AAM?$AAA?$AAD?$AAM?$AAS?$AAe?$AAs?$AAs?$AAi?$AAo?$AAn?$AA?$AA@ 00144798     atcmd.obj
 0002:000037c4       ??_C@_1CK@DBOLMJBK@?$AAS?$AAw?$AAi?$AAS?$AAt?$AAa?$AAr?$AAt?$AAO?$AAM?$AAA?$AAD?$AAM?$AAS?$AAe?$AAs?$AAs?$AAi?$AAo?$AAn?$AA?$AA@ 001447c4     atcmd.obj
 0002:000037f0       ??_C@_1CE@MOABMDJN@?$AAS?$AAw?$AAi?$AAS?$AAe?$AAt?$AAO?$AAM?$AAA?$AAD?$AAM?$AAC?$AAo?$AAn?$AAf?$AAi?$AAg?$AA?$AA@ 001447f0     atcmd.obj
 0002:00003814       ??_C@_1DA@JOLCEBDL@?$AAS?$AAw?$AAi?$AAG?$AAe?$AAt?$AAO?$AAM?$AAA?$AAD?$AAM?$AAS?$AAe?$AAs?$AAs?$AAi?$AAo?$AAn?$AAS?$AAt?$AAa?$AAt?$AAe?$AA?$AA@ 00144814     atcmd.obj
 0002:00003844       ??_C@_1CE@EPGOHDLP@?$AAS?$AAw?$AAi?$AAG?$AAe?$AAt?$AAO?$AAM?$AAA?$AAD?$AAM?$AAC?$AAo?$AAn?$AAf?$AAi?$AAg?$AA?$AA@ 00144844     atcmd.obj
 0002:00003868       ??_C@_1DA@IFJBBOPH@?$AAS?$AAw?$AAi?$AAS?$AAe?$AAt?$AAC?$AAa?$AAl?$AAl?$AAD?$AAi?$AAs?$AAc?$AAo?$AAn?$AAn?$AAe?$AAc?$AAt?$AAC?$AAm?$AAd?$AA?$AA@ 00144868     atcmd.obj
 0002:00003898       ??_C@_1CO@NEOJGBMN@?$AAS?$AAw?$AAi?$AAS?$AAe?$AAt?$AAC?$AAa?$AAl?$AAl?$AAO?$AAr?$AAi?$AAg?$AAi?$AAn?$AAa?$AAt?$AAe?$AAC?$AAm?$AAd?$AA?$AA@ 00144898     atcmd.obj
 0002:000038c8       ??_C@_1DE@LHBHLGKL@?$AAS?$AAw?$AAi?$AAG?$AAe?$AAt?$AAC?$AAa?$AAl?$AAl?$AAC?$AAo?$AAn?$AAn?$AAe?$AAc?$AAt?$AAi?$AAo?$AAn?$AAS?$AAt?$AAa?$AAt?$AAe?$AA?$AA@ 001448c8     atcmd.obj
 0002:000038fc       ??_C@_1DC@DNOMEIAB@?$AAS?$AAw?$AAi?$AAG?$AAe?$AAt?$AAC?$AAu?$AAr?$AAr?$AAe?$AAn?$AAt?$AAB?$AAa?$AAs?$AAe?$AAS?$AAt?$AAa?$AAt?$AAi?$AAo?$AAn?$AA?$AA@ 001448fc     atcmd.obj
 0002:00003930       ??_C@_1DA@PDCJHJEP@?$AAS?$AAw?$AAi?$AAG?$AAe?$AAt?$AAS?$AAe?$AAr?$AAv?$AAi?$AAc?$AAe?$AAI?$AAn?$AAd?$AAi?$AAc?$AAa?$AAt?$AAi?$AAo?$AAn?$AA?$AA@ 00144930     atcmd.obj
 0002:00003960       ??_C@_1CE@KMDAMGCA@?$AAS?$AAw?$AAi?$AAG?$AAe?$AAt?$AAH?$AAd?$AAr?$AAS?$AAr?$AAv?$AAS?$AAt?$AAa?$AAt?$AAe?$AA?$AA@ 00144960     atcmd.obj
 0002:00003984       ??_C@_1CI@FHPBAGN@?$AAS?$AAw?$AAi?$AAG?$AAe?$AAt?$AAH?$AAd?$AAr?$AAR?$AAo?$AAa?$AAm?$AAS?$AAt?$AAa?$AAt?$AAu?$AAs?$AA?$AA@ 00144984     atcmd.obj
 0002:000039ac       ??_C@_1CI@OLPCIGGN@?$AAS?$AAw?$AAi?$AAG?$AAe?$AAt?$AAR?$AAo?$AAa?$AAm?$AAi?$AAn?$AAg?$AAS?$AAt?$AAa?$AAt?$AAu?$AAs?$AA?$AA@ 001449ac     atcmd.obj
 0002:000039d4       ??_C@_1BO@NPIBNNMI@?$AAS?$AAw?$AAi?$AAG?$AAe?$AAt?$AAR?$AAs?$AAs?$AAi?$AAE?$AAc?$AAi?$AAo?$AA?$AA@ 001449d4     atcmd.obj
 0002:000039f4       ??_C@_1BG@JEEKPFGP@?$AAS?$AAw?$AAi?$AAG?$AAe?$AAt?$AAR?$AAs?$AAs?$AAi?$AA?$AA@ 001449f4     atcmd.obj
 0002:00003a0c       ??_C@_1BE@LNEKMFOL@?$AAS?$AAw?$AAi?$AAG?$AAe?$AAt?$AAE?$AAS?$AAN?$AA?$AA@ 00144a0c     atcmd.obj
 0002:00003a20       ??_C@_1CA@CEJEGIEG@?$AAS?$AAw?$AAi?$AAI?$AAs?$AAM?$AAo?$AAd?$AAe?$AAm?$AAR?$AAe?$AAa?$AAd?$AAy?$AA?$AA@ 00144a20     atcmd.obj
 0002:00003a40       ??_C@_1BM@DPLLEFED@?$AAS?$AAw?$AAi?$AAM?$AAo?$AAd?$AAe?$AAm?$AAR?$AAe?$AAs?$AAe?$AAt?$AA?$AA@ 00144a40     atcmd.obj
 0002:00003a5c       ??_C@_1CI@DLHEBEPN@?$AAS?$AAw?$AAi?$AAG?$AAe?$AAt?$AAA?$AAi?$AAr?$AAS?$AAe?$AAr?$AAv?$AAe?$AAr?$AAI?$AAn?$AAf?$AAo?$AA?$AA@ 00144a5c     atcmd.obj
 0002:00003a84       ??_C@_1BM@IKJGPLPF@?$AAS?$AAw?$AAi?$AAG?$AAe?$AAt?$AAM?$AAo?$AAd?$AAe?$AAl?$AAI?$AAD?$AA?$AA@ 00144a84     atcmd.obj
 0002:00003aa0       ??_C@_1CG@DMEGCIBF@?$AAS?$AAw?$AAi?$AAS?$AAe?$AAl?$AAe?$AAc?$AAt?$AAA?$AAi?$AAr?$AAS?$AAe?$AAr?$AAv?$AAe?$AAr?$AA?$AA@ 00144aa0     atcmd.obj
 0002:00003ac8       ??_C@_1CO@NMNJOKLM@?$AAS?$AAw?$AAi?$AAG?$AAe?$AAt?$AAA?$AAc?$AAt?$AAi?$AAv?$AAa?$AAt?$AAi?$AAo?$AAn?$AAS?$AAt?$AAa?$AAt?$AAu?$AAs?$AA?$AA@ 00144ac8     atcmd.obj
 0002:00003af8       ??_C@_1CK@PIODAMEA@?$AAS?$AAw?$AAi?$AAA?$AAc?$AAt?$AAi?$AAv?$AAa?$AAt?$AAe?$AAA?$AAu?$AAt?$AAo?$AAm?$AAa?$AAt?$AAi?$AAc?$AA?$AA@ 00144af8     atcmd.obj
 0002:00003b24       ??_C@_1CG@GPFEELC@?$AAS?$AAw?$AAi?$AAS?$AAt?$AAo?$AAp?$AAD?$AAa?$AAt?$AAa?$AAS?$AAe?$AAs?$AAs?$AAi?$AAo?$AAn?$AA?$AA@ 00144b24     atcmd.obj
 0002:00003b4c       ??_C@_1CI@KDNDFGHI@?$AAS?$AAw?$AAi?$AAS?$AAt?$AAa?$AAr?$AAt?$AAD?$AAa?$AAt?$AAa?$AAS?$AAe?$AAs?$AAs?$AAi?$AAo?$AAn?$AA?$AA@ 00144b4c     atcmd.obj
 0002:00003b74       ??_C@_1BO@JENOOCNI@?$AAS?$AAw?$AAi?$AAA?$AAp?$AAi?$AAS?$AAh?$AAu?$AAt?$AAd?$AAo?$AAw?$AAn?$AA?$AA@ 00144b74     atcmd.obj
 0002:00003b94       ??_C@_1BM@PPHCOJDH@?$AAS?$AAw?$AAi?$AAA?$AAp?$AAi?$AAS?$AAt?$AAa?$AAr?$AAt?$AAu?$AAp?$AA?$AA@ 00144b94     atcmd.obj
 0002:00003bb0       ??_C@_1DA@PGKJGMLC@?$AAS?$AAw?$AAi?$AAA?$AAT?$AAG?$AAe?$AAt?$AAP?$AAr?$AAo?$AAv?$AAi?$AAs?$AAi?$AAo?$AAn?$AAS?$AAt?$AAa?$AAt?$AAu?$AAs?$AA?$AA@ 00144bb0     atcmd.obj
 0002:00003be0       ??_C@_1BM@FLKGECGM@?$AAS?$AAw?$AAi?$AAA?$AAT?$AAR?$AAt?$AAn?$AAR?$AAe?$AAs?$AAe?$AAt?$AA?$AA@ 00144be0     atcmd.obj
 0002:00003bfc       ??_C@_1BG@PLNNLANE@?$AAS?$AAw?$AAi?$AAA?$AAT?$AAR?$AAe?$AAs?$AAe?$AAt?$AA?$AA@ 00144bfc     atcmd.obj
 0002:00003c14       ??_C@_1CK@GCHOJML@?$AAS?$AAw?$AAi?$AAA?$AAT?$AAS?$AAe?$AAt?$AAS?$AAi?$AAd?$AAe?$AAT?$AAo?$AAn?$AAe?$AAG?$AAa?$AAi?$AAn?$AA?$AA@ 00144c14     atcmd.obj
 0002:00003c40       ??_C@_1BK@JIOEKFJJ@?$AAS?$AAw?$AAi?$AAA?$AAT?$AAS?$AAe?$AAt?$AAE?$AAn?$AAu?$AAm?$AA?$AA@ 00144c40     atcmd.obj
 0002:00003c5c       ??_C@_1BO@CNFCHCOA@?$AAS?$AAw?$AAi?$AAM?$AAa?$AAn?$AAa?$AAg?$AAe?$AAC?$AAa?$AAl?$AAl?$AAs?$AA?$AA@ 00144c5c     atcmd.obj
 0002:00003c7c       ??_C@_1BK@EJNNAMHO@?$AAS?$AAw?$AAi?$AAA?$AAn?$AAs?$AAe?$AAr?$AAC?$AAa?$AAl?$AAl?$AA?$AA@ 00144c7c     atcmd.obj
 0002:00003c98       ??_C@_1BG@GDGGJKOB@?$AAS?$AAw?$AAi?$AAE?$AAn?$AAd?$AAC?$AAa?$AAl?$AAl?$AA?$AA@ 00144c98     atcmd.obj
 0002:00003cb0       ??_C@_1CC@PPKPAHLI@?$AAS?$AAw?$AAi?$AAA?$AAT?$AAR?$AAe?$AAl?$AAe?$AAa?$AAs?$AAe?$AAC?$AAa?$AAl?$AAl?$AA?$AA@ 00144cb0     atcmd.obj
 0002:00003cd4       ??_C@_1BK@BJANHLJN@?$AAS?$AAw?$AAi?$AAA?$AAT?$AAG?$AAe?$AAt?$AAC?$AAO?$AAL?$AAR?$AA?$AA@ 00144cd4     atcmd.obj
 0002:00003cf0       ??_C@_1BK@CLBLAJIE@?$AAS?$AAw?$AAi?$AAA?$AAT?$AAS?$AAe?$AAt?$AAC?$AAO?$AAL?$AAR?$AA?$AA@ 00144cf0     atcmd.obj
 0002:00003d0c       ??_C@_1BK@LDAELDBG@?$AAS?$AAw?$AAi?$AAA?$AAT?$AAG?$AAe?$AAt?$AAC?$AAO?$AAL?$AAP?$AA?$AA@ 00144d0c     atcmd.obj
 0002:00003d28       ??_C@_1BK@IBBCMBAP@?$AAS?$AAw?$AAi?$AAA?$AAT?$AAS?$AAe?$AAt?$AAC?$AAO?$AAL?$AAP?$AA?$AA@ 00144d28     atcmd.obj
 0002:00003d44       ??_C@_1BK@MHEPONMN@?$AAS?$AAw?$AAi?$AAA?$AAT?$AAG?$AAe?$AAt?$AAC?$AAL?$AAI?$AAR?$AA?$AA@ 00144d44     atcmd.obj
 0002:00003d60       ??_C@_1BK@PFFJJPNE@?$AAS?$AAw?$AAi?$AAA?$AAT?$AAS?$AAe?$AAt?$AAC?$AAL?$AAI?$AAR?$AA?$AA@ 00144d60     atcmd.obj
 0002:00003d7c       ??_C@_1BK@GNEGCFEG@?$AAS?$AAw?$AAi?$AAA?$AAT?$AAG?$AAe?$AAt?$AAC?$AAL?$AAI?$AAP?$AA?$AA@ 00144d7c     atcmd.obj
 0002:00003d98       ??_C@_1BK@FPFAFHFP@?$AAS?$AAw?$AAi?$AAA?$AAT?$AAS?$AAe?$AAt?$AAC?$AAL?$AAI?$AAP?$AA?$AA@ 00144d98     atcmd.obj
 0002:00003db4       ??_C@_1BI@KEPDBGG@?$AAS?$AAw?$AAi?$AAD?$AAi?$AAa?$AAl?$AAC?$AAa?$AAl?$AAl?$AA?$AA@ 00144db4     atcmd.obj
 0002:00003dcc       ??_C@_1CG@JDNDNGNF@?$AAS?$AAw?$AAi?$AAU?$AAp?$AAg?$AAr?$AAa?$AAd?$AAe?$AAF?$AAi?$AAr?$AAm?$AAw?$AAa?$AAr?$AAe?$AA?$AA@ 00144dcc     atcmd.obj
 0002:00003df4       ??_C@_1CM@OOMOMHGB@?$AAS?$AAw?$AAi?$AAS?$AAe?$AAt?$AAI?$AAm?$AAa?$AAg?$AAe?$AAP?$AAr?$AAe?$AAf?$AAe?$AAr?$AAe?$AAn?$AAc?$AAe?$AA?$AA@ 00144df4     atcmd.obj
 0002:00003e20       ??_C@_1CM@MMMJEH@?$AAS?$AAw?$AAi?$AAG?$AAe?$AAt?$AAI?$AAm?$AAa?$AAg?$AAe?$AAP?$AAr?$AAe?$AAf?$AAe?$AAr?$AAe?$AAn?$AAc?$AAe?$AA?$AA@ 00144e20     atcmd.obj
 0002:00003e4c       ??_C@_1BG@KPNEMHOH@?$AAS?$AAD?$AAK?$AAR?$AAI?$AAL?$AA?4?$AAd?$AAl?$AAl?$AA?$AA@ 00144e4c     atcmd.obj
 0002:00003e64       ??_C@_1CC@JJFJLKM@?$AAR?$AAI?$AAL?$AA?5?$AAH?$AAa?$AAn?$AAd?$AAl?$AAe?$AA?5?$AAN?$AAU?$AAL?$AAL?$AA?$CB?$AA?$AA@ 00144e64     atcmd.obj
 0002:00003e88       ??_C@_1IK@IKNNEHFL@?$AAc?$AA?3?$AA?2?$AAo?$AAf?$AAf?$AAi?$AAc?$AAa?$AAl?$AA_?$AAb?$AAu?$AAi?$AAl?$AAd?$AA?2?$AAr?$AAi?$AAl?$AAg?$AAo?$AAb?$AAi?$AA?2?$AAs?$AAw?$AA?2?$AAd?$AAl?$AAl?$AAs@ 00144e88     atcmd.obj
 0002:00003f18       ??_C@_1FE@KJJCAGGP@?$AAA?$AAS?$AAS?$AAE?$AAR?$AAT?$AAI?$AAO?$AAN?$AA?5?$AAF?$AAA?$AAI?$AAL?$AAU?$AAR?$AAE?$AA?3?$AA?5?$AA?$DN?$AA?$DN?$AA?$DN?$AA?$DO?$AAF?$AAA?$AAL?$AAS?$AAE?$AA?5?$AA?$CB?$AA?$DN?$AA?5@ 00144f18     atcmd.obj
 0002:00003f70       ??_C@_1FG@FGKKPHPP@?$AAR?$AAe?$AAa?$AAd?$AAT?$AAh?$AAr?$AAe?$AAa?$AAd?$AAP?$AAr?$AAo?$AAc?$AA?5?$AA?3?$AA?5?$AAE?$AAn?$AAt?$AAe?$AAr?$AAi?$AAn?$AAg?$AA?0?$AA?5?$AAp?$AAR?$AAi?$AAl?$AAD@ 00144f70     atcmd.obj
 0002:00003fc8       ??_C@_1GE@BMGBJBJK@?$AAR?$AAe?$AAa?$AAd?$AAT?$AAh?$AAr?$AAe?$AAa?$AAd?$AAP?$AAr?$AAo?$AAc?$AA?5?$AA?3?$AA?5?$AAT?$AAH?$AAR?$AAE?$AAA?$AAD?$AA?5?$AAI?$AAS?$AA?5?$AAE?$AAX?$AAI?$AAT?$AAI@ 00144fc8     atcmd.obj
 0002:00004030       ??_C@_1HG@FHAGDNPC@?$AAR?$AAe?$AAa?$AAd?$AAT?$AAh?$AAr?$AAe?$AAa?$AAd?$AAP?$AAr?$AAo?$AAc?$AA?5?$AA?3?$AA?5?$AAU?$AAn?$AAa?$AAb?$AAl?$AAe?$AA?5?$AAt?$AAo?$AA?5?$AAr?$AAa?$AAi?$AAs?$AAe@ 00145030     atcmd.obj
 0002:000040a8       ??_C@_1BI@KBDHFJMO@?$AA?4?$AA?2?$AAa?$AAt?$AAc?$AAm?$AAd?$AA?4?$AAc?$AAp?$AAp?$AA?$AA@ 001450a8     atcmd.obj
 0002:000040c0       ??_C@_1FG@MLHHDNMH@?$AAA?$AAS?$AAS?$AAE?$AAR?$AAT?$AAI?$AAO?$AAN?$AA?5?$AAF?$AAA?$AAI?$AAL?$AAU?$AAR?$AAE?$AA?3?$AA?5?$AA?$DN?$AA?$DN?$AA?$DN?$AA?$DO?$AAl?$AAp?$AAP?$AAa?$AAr?$AAa?$AAm?$AAe?$AAt@ 001450c0     atcmd.obj
 0002:0000423c       ??_C@_0BC@KBDMBKEH@deque?$DMT?$DO?5too?5long?$AA@ 0014523c     atcmd.obj
 0002:00004288       ??_C@_1ME@OKAODALA@?$AAC?$AAo?$AAm?$AAm?$AAa?$AAn?$AAd?$AAT?$AAh?$AAr?$AAe?$AAa?$AAd?$AA?3?$AA?5?$AAC?$AAa?$AAn?$AAn?$AAo?$AAt?$AA?5?$AAR?$AAe?$AAm?$AAo?$AAv?$AAe?$AA?5?$AAc?$AAm?$AAd@ 00145288     atcmd.obj
 0002:00004350       ??_C@_1HI@DAMBEHME@?$AAC?$AAR?$AAi?$AAl?$AAH?$AAa?$AAn?$AAd?$AAl?$AAe?$AA?3?$AA?3?$AAC?$AAo?$AAm?$AAm?$AAa?$AAn?$AAd?$AAT?$AAh?$AAr?$AAe?$AAa?$AAd?$AA?5?$AA?3?$AA?5?$AAp?$AAC?$AAm?$AAd@ 00145350     atcmd.obj
 0002:000043c8       ??_C@_1FG@CGMOIEOK@?$AAC?$AAR?$AAi?$AAl?$AAH?$AAa?$AAn?$AAd?$AAl?$AAe?$AA?3?$AA?3?$AAC?$AAo?$AAm?$AAm?$AAa?$AAn?$AAd?$AAT?$AAh?$AAr?$AAe?$AAa?$AAd?$AA?5?$AA?3?$AA?5?$AAC?$AAa?$AAn?$AAc@ 001453c8     atcmd.obj
 0002:00004420       ??_C@_1HM@CMCEDNAJ@?$AAC?$AAm?$AAd?$AAI?$AAD?$AA?5?$AA?$DN?$AA?5?$AA?$CF?$AAd?$AA?0?$AA?5?$AAA?$AAP?$AAI?$AAI?$AAD?$AA?5?$AA?$DN?$AA?5?$AA?$CF?$AAd?$AA?5?$AAh?$AAa?$AAs?$AA?5?$AAn?$AAo?$AA?5?$AAm?$AAo@ 00145420     atcmd.obj
 0002:000044a0       ??_C@_1FE@CPCDJHBC@?$AAC?$AAm?$AAd?$AAT?$AAh?$AAr?$AAe?$AAa?$AAd?$AAP?$AAr?$AAo?$AAc?$AA?5?$AA?3?$AA?5?$AAE?$AAn?$AAt?$AAe?$AAr?$AAi?$AAn?$AAg?$AA?0?$AA?5?$AAp?$AAR?$AAi?$AAl?$AAD?$AAe@ 001454a0     atcmd.obj
 0002:000044f8       ??_C@_1GC@NCMHGCFD@?$AAC?$AAm?$AAd?$AAT?$AAh?$AAr?$AAe?$AAa?$AAd?$AAP?$AAr?$AAo?$AAc?$AA?5?$AA?3?$AA?5?$AAT?$AAH?$AAR?$AAE?$AAA?$AAD?$AA?5?$AAI?$AAS?$AA?5?$AAE?$AAX?$AAI?$AAT?$AAI?$AAN@ 001454f8     atcmd.obj
 0002:000045a8       ??_C@_1HG@MPPBHIHD@?$AAQ?$AAu?$AAe?$AAu?$AAe?$AAC?$AAm?$AAd?$AAW?$AAi?$AAt?$AAh?$AAT?$AAi?$AAm?$AAe?$AAo?$AAu?$AAt?$AA?5?$AA?3?$AA?5?$AAU?$AAn?$AAa?$AAb?$AAl?$AAe?$AA?5?$AAt?$AAo?$AA?5@ 001455a8     atcmd.obj
 0002:00004620       ??_C@_1GM@CJNHKFGA@?$AAF?$AAa?$AAi?$AAl?$AA?5?$AAt?$AAo?$AA?5?$AAa?$AAd?$AAd?$AA?5?$AAc?$AAm?$AAd?$AA?5?$AAA?$AAP?$AAI?$AAI?$AAD?$AA?$DN?$AA?$CF?$AAd?$AA?5?$AAt?$AAo?$AA?5?$AAt?$AAh?$AAe?$AA?5@ 00145620     atcmd.obj
 0002:00004690       ??_C@_1JA@BGMBFCCG@?$AAQ?$AAu?$AAe?$AAu?$AAe?$AAC?$AAm?$AAd?$AA?5?$AAs?$AAu?$AAc?$AAc?$AAe?$AAs?$AAs?$AA?5?$AAA?$AAP?$AAP?$AAI?$AAD?$AA?5?$AA?$DN?$AA?5?$AA?$CF?$AAd?$AA?0?$AA?5?$AAR?$AAI?$AAL@ 00145690     atcmd.obj
 0002:00004720       ??_C@_1EC@KPKGMADJ@?$AAQ?$AAu?$AAe?$AAu?$AAe?$AAi?$AAn?$AAg?$AA?5?$AAc?$AAo?$AAm?$AAm?$AAa?$AAn?$AAd?$AA?5?$AAw?$AAi?$AAt?$AAh?$AA?5?$AAI?$AAD?$AA?3?$AA?5?$AA0?$AAx?$AA?$CF?$AA0?$AA8?$AAx@ 00145720     atcmd.obj
 0002:00004768       ??_C@_1LC@KGPNPBBC@?$AAI?$AAn?$AAc?$AAo?$AAr?$AAr?$AAe?$AAc?$AAt?$AA?5?$AAu?$AAs?$AAe?$AA?5?$AAo?$AAf?$AA?5?$AAQ?$AAu?$AAe?$AAu?$AAe?$AAC?$AAm?$AAd?$AA?5?$AAp?$AAa?$AAr?$AAa?$AAm?$AAs@ 00145768     atcmd.obj
 0002:00004820       ??_C@_1FE@NBHPGEDJ@?$AAA?$AAS?$AAS?$AAE?$AAR?$AAT?$AAI?$AAO?$AAN?$AA?5?$AAF?$AAA?$AAI?$AAL?$AAU?$AAR?$AAE?$AA?3?$AA?5?$AA?$DN?$AA?$DN?$AA?$DN?$AA?$DO?$AAN?$AAU?$AAL?$AAL?$AA?5?$AA?$CB?$AA?$DN?$AA?5?$AAp@ 00145820     atcmd.obj
 0002:00004874       ??_C@_00CNPNBAHC@?$AA@     00145874     callctrl.obj
 0002:00004878       ??_C@_11LOCGONAA@?$AA?$AA@ 00145878     callctrl.obj
 0002:0000487c       ??_C@_1CE@JANOHFNC@?$AAR?$AAa?$AAd?$AAi?$AAo?$AA?5?$AAH?$AAa?$AAn?$AAd?$AAl?$AAe?$AA?5?$AAN?$AAU?$AAL?$AAL?$AA?$AA@ 0014587c     callctrl.obj
 0002:00004900       ??_C@_1HI@EKLFFCGI@?$AAR?$AAI?$AAL?$AAD?$AAr?$AAv?$AA_?$AAS?$AAe?$AAn?$AAd?$AAD?$AAT?$AAM?$AAF?$AA?5?$AA?3?$AA?5?$AAS?$AAe?$AAn?$AAd?$AAi?$AAn?$AAg?$AA?5?$AAD?$AAT?$AAM?$AAF?$AA?0?$AA?5@ 00145900     callctrl.obj
 0002:00004978       ??_C@_1FK@LEPAKGPK@?$AAA?$AAS?$AAS?$AAE?$AAR?$AAT?$AAI?$AAO?$AAN?$AA?5?$AAF?$AAA?$AAI?$AAL?$AAU?$AAR?$AAE?$AA?3?$AA?5?$AA?$DN?$AA?$DN?$AA?$DN?$AA?$DO?$AA0?$AA?5?$AA?$DM?$AA?5?$AAs?$AAt?$AAr?$AAl?$AAe@ 00145978     callctrl.obj
 0002:000049d4       ??_C@_1BO@CGJHHAKI@?$AA?4?$AA?2?$AAc?$AAa?$AAl?$AAl?$AAc?$AAt?$AAr?$AAl?$AA?4?$AAc?$AAp?$AAp?$AA?$AA@ 001459d4     callctrl.obj
 0002:000049f8       ??_C@_1FC@FDJOMKME@?$AAA?$AAS?$AAS?$AAE?$AAR?$AAT?$AAI?$AAO?$AAN?$AA?5?$AAF?$AAA?$AAI?$AAL?$AAU?$AAR?$AAE?$AA?3?$AA?5?$AA?$DN?$AA?$DN?$AA?$DN?$AA?$DO?$AAN?$AAU?$AAL?$AAL?$AA?5?$AA?$CB?$AA?$DN?$AA?5?$AAl@ 001459f8     callctrl.obj
 0002:00004a4c       ??_C@_1CG@CGLLMFLF@?$AAR?$AAI?$AAL?$AAD?$AAr?$AAv?$AA_?$AAG?$AAe?$AAt?$AAC?$AAa?$AAl?$AAl?$AAL?$AAi?$AAs?$AAt?$AA?$AA@ 00145a4c     callctrl.obj
 0002:00004a78       ??_C@_1EK@KIPDDKFI@?$AAR?$AAI?$AAL?$AAD?$AAr?$AAv?$AA_?$AAM?$AAa?$AAn?$AAa?$AAg?$AAe?$AAC?$AAa?$AAl?$AAl?$AAs?$AA?5?$AAc?$AAo?$AAm?$AAm?$AAa?$AAn?$AAd?$AA?5?$AA?$CF?$AAd?$AA?0?$AA?5?$AAi@ 00145a78     callctrl.obj
 0002:00004ac4       ??_C@_1CK@FCLFBFHP@?$AAR?$AAI?$AAL?$AAD?$AAr?$AAv?$AA_?$AAG?$AAe?$AAt?$AAL?$AAi?$AAn?$AAe?$AAS?$AAt?$AAa?$AAt?$AAu?$AAs?$AA?$AA@ 00145ac4     callctrl.obj
 0002:00004b50       ??_C@_1EM@FGGFAEGL@?$AAA?$AAS?$AAS?$AAE?$AAR?$AAT?$AAI?$AAO?$AAN?$AA?5?$AAF?$AAA?$AAI?$AAL?$AAU?$AAR?$AAE?$AA?3?$AA?5?$AA?$DN?$AA?$DN?$AA?$DN?$AA?$DO?$AAp?$AAR?$AAi?$AAl?$AAC?$AAI?$AA?5?$AA?$CB?$AA?$DN@ 00145b50     callctrl.obj
 0002:00004be8       ??_C@_1EA@KEMMJNOJ@?$AAG?$AAe?$AAt?$AAL?$AAi?$AAn?$AAe?$AAS?$AAt?$AAa?$AAt?$AAu?$AAs?$AA?3?$AA?5?$AAL?$AAi?$AAn?$AAe?$AAS?$AAt?$AAa?$AAt?$AAu?$AAs?$AA?3?$AA?5?$AA0?$AAx?$AA?$CF?$AAx?$AA?$AA@ 00145be8     callctrl.obj
 0002:00004c28       ??_C@_1GO@KIFACNAJ@?$AAC?$AAR?$AAa?$AAd?$AAi?$AAo?$AA?3?$AA?3?$AAG?$AAe?$AAt?$AAL?$AAi?$AAn?$AAe?$AAS?$AAt?$AAa?$AAt?$AAu?$AAs?$AA?5?$AAm?$AA_?$AAd?$AAw?$AAC?$AAu?$AAr?$AAr?$AAe?$AAn@ 00145c28     callctrl.obj
 0002:00004c98       ??_C@_1EK@MOLNCJBP@?$AAR?$AAe?$AAa?$AAd?$AAC?$AAu?$AAr?$AAr?$AAe?$AAn?$AAt?$AAP?$AAr?$AAi?$AAv?$AAa?$AAc?$AAy?$AAS?$AAt?$AAa?$AAt?$AAu?$AAs?$AA?5?$AAu?$AAn?$AAs?$AAu?$AAp?$AAp?$AAo@ 00145c98     callctrl.obj
 0002:00004d60       ??_C@_1FC@EPHLCJEL@?$AAT?$AAo?$AAo?$AA?5?$AAm?$AAa?$AAn?$AAy?$AA?5?$AAl?$AAi?$AAn?$AAe?$AAs?$AA?0?$AA?5?$AAA?$AAd?$AAd?$AAr?$AAe?$AAs?$AAs?$AAI?$AAd?$AA?5?$AAw?$AAa?$AAs?$AA?5?$AAn?$AAo@ 00145d60     callctrl.obj
 0002:00004db4       ??_C@_1CG@JLBDJBPE@?$AAI?$AAn?$AAv?$AAa?$AAl?$AAi?$AAd?$AA?5?$AAA?$AAd?$AAd?$AAr?$AAe?$AAs?$AAs?$AA?5?$AAI?$AAD?$AA?$AA@ 00145db4     callctrl.obj
 0002:00004e18       ??_C@_1EO@IKBLPLFP@?$AAA?$AAS?$AAS?$AAE?$AAR?$AAT?$AAI?$AAO?$AAN?$AA?5?$AAF?$AAA?$AAI?$AAL?$AAU?$AAR?$AAE?$AA?3?$AA?5?$AA?$DN?$AA?$DN?$AA?$DN?$AA?$DO?$AAp?$AAR?$AAi?$AAl?$AAA?$AAd?$AAd?$AA?5?$AA?$CB@ 00145e18     callctrl.obj
 0002:00004e68       ??_C@_1BA@LEPJIIOK@?$AAU?$AAn?$AAk?$AAn?$AAo?$AAw?$AAn?$AA?$AA@ 00145e68     callctrl.obj
 0002:00004e78       ??_C@_1BA@BOLKEAKD@?$AAP?$AAr?$AAi?$AAv?$AAa?$AAt?$AAe?$AA?$AA@ 00145e78     callctrl.obj
 0002:00004e88       ??_C@_1BG@OCCAHMJC@?$AAR?$AAE?$AAS?$AAT?$AAR?$AAI?$AAC?$AAT?$AAE?$AAD?$AA?$AA@ 00145e88     callctrl.obj
 0002:00004ea0       ??_C@_1EK@IJCFBGIL@?$AAD?$AAW?$AAO?$AAR?$AAD?$AA?5?$AAC?$AAR?$AAa?$AAd?$AAi?$AAo?$AA?3?$AA?3?$AAC?$AAa?$AAl?$AAl?$AAE?$AAx?$AAi?$AAs?$AAt?$AAs?$AA?$CI?$AA?$CF?$AAd?$AA?$CJ?$AA?5?$AAf?$AAa?$AAi@ 00145ea0     callctrl.obj
 0002:00004f58       ??_C@_1EG@BAPAAGIF@?$AAU?$AAp?$AAd?$AAa?$AAt?$AAe?$AAL?$AAi?$AAn?$AAe?$AAS?$AAt?$AAa?$AAt?$AAu?$AAs?$AA?5?$AAm?$AA_?$AAd?$AAw?$AAL?$AAi?$AAn?$AAe?$AAS?$AAt?$AAa?$AAt?$AAu?$AAs?$AA?5@ 00145f58     callctrl.obj
 0002:00004fa0       ??_C@_1CC@DEHKJFIH@?$AAG?$AAe?$AAt?$AAC?$AAa?$AAl?$AAl?$AAI?$AAn?$AAf?$AAo?$AA?3?$AA?$CF?$AAd?$AA?$AN?$AA?6?$AA?$AA@ 00145fa0     callctrl.obj
 0002:00004fc8       ??_C@_1GI@OGKAKGJH@?$AAC?$AAl?$AAo?$AAs?$AAe?$AAD?$AAa?$AAt?$AAa?$AAP?$AAo?$AAr?$AAt?$AA?5?$AAN?$AAO?$AAO?$AAP?$AA?5?$AAb?$AAc?$AAo?$AAs?$AA?5?$AAD?$AAa?$AAt?$AAa?$AA?5?$AAp?$AAo?$AAr@ 00145fc8     callctrl.obj
 0002:00005030       ??_C@_1HI@IEKCFOOE@?$AAC?$AAl?$AAo?$AAs?$AAe?$AAD?$AAa?$AAt?$AAa?$AAP?$AAo?$AAr?$AAt?$AA?3?$AA?5?$AAb?$AAe?$AAf?$AAo?$AAr?$AAe?$AA?5?$AAc?$AAl?$AAo?$AAs?$AAi?$AAn?$AAg?$AA?5?$AAh?$AAa@ 00146030     callctrl.obj
 0002:000050a8       ??_C@_1KK@NEPDCEBI@?$AAU?$AAn?$AAh?$AAa?$AAn?$AAd?$AAl?$AAe?$AAd?$AA?5?$AAO?$AAT?$AAA?$AAS?$AAP?$AAS?$AAt?$AAa?$AAt?$AAe?$AA?4?$AAe?$AAS?$AAt?$AAa?$AAt?$AAe?$AA?5?$AA?$DN?$AA?5?$AA?$CF?$AAd@ 001460a8     callctrl.obj
 0002:00005154       ??_C@_1CO@LHJDEFDH@?$AAO?$AAT?$AAA?$AAS?$AAP?$AA?5?$AAf?$AAa?$AAi?$AAl?$AAe?$AAd?$AA?5?$AAt?$AAo?$AA?5?$AAc?$AAo?$AAm?$AAm?$AAi?$AAt?$AA?$AA@ 00146154     callctrl.obj
 0002:00005184       ??_C@_1DG@GBMNGKJJ@?$AAC?$AAo?$AAd?$AAi?$AAn?$AAg?$AA?5?$AAS?$AAc?$AAh?$AAe?$AAm?$AAe?$AA?5?$AAn?$AAo?$AAt?$AA?5?$AAs?$AAu?$AAp?$AAp?$AAo?$AAr?$AAt?$AA?$CB?$AA?$AA@ 00146184     callctrl.obj
 0002:000051c0       ??_C@_1FE@KLKMAOPE@?$AAU?$AAS?$AAS?$AAD?$AA?5?$AAc?$AAo?$AAd?$AAi?$AAn?$AAg?$AA?5?$AAs?$AAc?$AAh?$AAe?$AAm?$AAe?$AA?5?$AA?$DN?$AA?5?$AA?5?$AAU?$AAC?$AAS?$AA2?$AA?0?$AA?5?$AAd?$AAa?$AAt?$AAa@ 001461c0     callctrl.obj
 0002:00005214       ??_C@_1DE@EBCHHMPP@?$AAR?$AAI?$AAL?$AAS?$AAU?$AAP?$AAS?$AAE?$AAR?$AAV?$AAI?$AAC?$AAE?$AAD?$AAA?$AAT?$AAA?$AA?5?$AAi?$AAs?$AA?5?$AAN?$AAU?$AAL?$AAL?$AA?$AA@ 00146214     callctrl.obj
 0002:00005248       ??_C@_1GK@CLIGCDEL@?$AAm?$AA_?$AAb?$AAA?$AAn?$AAs?$AAU?$AAS?$AAS?$AAD?$AA?3?$AA?3?$AAR?$AAI?$AAL?$AA_?$AAS?$AAU?$AAP?$AAS?$AAV?$AAC?$AAD?$AAA?$AAT?$AAA?$AAS?$AAT?$AAA?$AAT?$AAU?$AAS@ 00146248     callctrl.obj
 0002:000052b4       ??_C@_1CM@EDMAIFEF@?$AAH?$AAa?$AAn?$AAd?$AAl?$AAe?$AAS?$AAW?$AAI?$AA_?$AAN?$AAO?$AAT?$AAI?$AAF?$AAY?$AA_?$AAU?$AAS?$AAS?$AAD?$AA?$AA@ 001462b4     callctrl.obj
 0002:00005348       ??_C@_1BO@CPBFMBMJ@?$AAC?$AAR?$AAa?$AAd?$AAi?$AAo?$AA?3?$AA?3?$AAA?$AAn?$AAs?$AAw?$AAe?$AAr?$AA?$AA@ 00146348     callctrl.obj
 0002:000053a8       ??_C@_1NA@GIKKEANA@?$AAG?$AAe?$AAt?$AAC?$AAa?$AAl?$AAl?$AAL?$AAi?$AAs?$AAt?$AA?3?$AA?5?$AAC?$AAa?$AAl?$AAl?$AAI?$AAD?$AA?5?$AA?$CF?$AAd?$AA?5?$AAQ?$AAm?$AAi?$AAI?$AAD?$AA?5?$AA?$CF?$AAd?$AA?0@ 001463a8     callctrl.obj
 0002:000054ac       ??_C@_1CG@BACOLJLE@?$AAC?$AAR?$AAa?$AAd?$AAi?$AAo?$AA?3?$AA?3?$AAM?$AAa?$AAn?$AAa?$AAg?$AAe?$AAC?$AAa?$AAl?$AAl?$AA?$AA@ 001464ac     callctrl.obj
 0002:000054d4       ??_C@_1CO@JDLGIDGF@?$AAR?$AAI?$AAL?$AA_?$AAC?$AAA?$AAL?$AAL?$AAC?$AAM?$AAD?$AA_?$AAI?$AAN?$AAV?$AAO?$AAK?$AAE?$AAC?$AAC?$AAB?$AAS?$AA?$AA@ 001464d4     callctrl.obj
 0002:00005508       ??_C@_1EK@NEJCEMML@?$AAR?$AAI?$AAL?$AA_?$AAC?$AAA?$AAL?$AAL?$AAC?$AAM?$AAD?$AA_?$AAA?$AAD?$AAD?$AAH?$AAE?$AAL?$AAD?$AAT?$AAO?$AAC?$AAO?$AAN?$AAF?$AA_?$AAD?$AAI?$AAS?$AAC?$AAO?$AAN@ 00146508     callctrl.obj
 0002:00005554       ??_C@_1DE@DKJKEBOE@?$AAR?$AAI?$AAL?$AA_?$AAC?$AAA?$AAL?$AAL?$AAC?$AAM?$AAD?$AA_?$AAA?$AAD?$AAD?$AAH?$AAE?$AAL?$AAD?$AAT?$AAO?$AAC?$AAO?$AAN?$AAF?$AA?$AA@ 00146554     callctrl.obj
 0002:00005588       ??_C@_1GM@GAEIJGAL@?$AAR?$AAI?$AAL?$AA_?$AAC?$AAA?$AAL?$AAL?$AAC?$AAM?$AAD?$AA_?$AAH?$AAO?$AAL?$AAD?$AAA?$AAL?$AAL?$AAB?$AAU?$AAT?$AAO?$AAN?$AAE?$AA?5?$AAL?$AAo?$AAo?$AAk?$AAu?$AAp@ 00146588     callctrl.obj
 0002:000055f4       ??_C@_1DE@DEHHCOMF@?$AAR?$AAI?$AAL?$AA_?$AAC?$AAA?$AAL?$AAL?$AAC?$AAM?$AAD?$AA_?$AAH?$AAO?$AAL?$AAD?$AAA?$AAL?$AAL?$AAB?$AAU?$AAT?$AAO?$AAN?$AAE?$AA?$AA@ 001465f4     callctrl.obj
 0002:00005628       ??_C@_1IA@BIKFJMID@?$AAM?$AAa?$AAn?$AAa?$AAg?$AAe?$AAC?$AAa?$AAl?$AAl?$AA?5?$AAL?$AAo?$AAo?$AAk?$AAu?$AAp?$AAC?$AAa?$AAl?$AAl?$AAI?$AAd?$AAB?$AAy?$AAC?$AAa?$AAl?$AAl?$AAS?$AAt?$AAa@ 00146628     callctrl.obj
 0002:000056a8       ??_C@_1EE@FDJNIFNI@?$AAR?$AAI?$AAL?$AA_?$AAC?$AAA?$AAL?$AAL?$AAC?$AAM?$AAD?$AA_?$AAH?$AAO?$AAL?$AAD?$AAA?$AAC?$AAT?$AAI?$AAV?$AAE?$AA_?$AAA?$AAC?$AAC?$AAE?$AAP?$AAT?$AAH?$AAE?$AAL@ 001466a8     callctrl.obj
 0002:000056ec       ??_C@_1DA@JEBNEJIP@?$AAR?$AAI?$AAL?$AA_?$AAC?$AAA?$AAL?$AAL?$AAC?$AAM?$AAD?$AA_?$AAR?$AAE?$AAL?$AAE?$AAA?$AAS?$AAE?$AAC?$AAA?$AAL?$AAL?$AA?$AA@ 001466ec     callctrl.obj
 0002:00005720       ??_C@_1EK@DCLLNKIF@?$AAR?$AAI?$AAL?$AA_?$AAC?$AAA?$AAL?$AAL?$AAC?$AAM?$AAD?$AA_?$AAR?$AAE?$AAL?$AAE?$AAA?$AAS?$AAE?$AAA?$AAC?$AAT?$AAI?$AAV?$AAE?$AA_?$AAA?$AAC?$AAC?$AAE?$AAP?$AAT@ 00146720     callctrl.obj
 0002:00005770       ??_C@_1EC@NOAMHBJP@?$AAM?$AAa?$AAn?$AAa?$AAg?$AAe?$AAC?$AAa?$AAl?$AAl?$AA?5?$AAf?$AAa?$AAi?$AAl?$AAu?$AAr?$AAe?$AA?4?$AA?5?$AAE?$AAr?$AAr?$AAC?$AAo?$AAd?$AAe?$AA?5?$AA?$DN?$AA?5?$AA?$CF?$AAd@ 00146770     callctrl.obj
 0002:000057b4       ??_C@_1DA@CNADJEGN@?$AAR?$AAI?$AAL?$AA_?$AAC?$AAA?$AAL?$AAL?$AAC?$AAM?$AAD?$AA_?$AAR?$AAE?$AAL?$AAE?$AAA?$AAS?$AAE?$AAH?$AAE?$AAL?$AAD?$AA?$AA@ 001467b4     callctrl.obj
 0002:000057e8       ??_C@_1FE@JLNEAPD@?$AAC?$AAR?$AAa?$AAd?$AAi?$AAo?$AA?3?$AA?3?$AAM?$AAa?$AAn?$AAa?$AAg?$AAe?$AAC?$AAa?$AAl?$AAl?$AA?5?$AAc?$AAm?$AAd?$AA?5?$AA?$DN?$AA?5?$AA?$CF?$AAd?$AA?0?$AA?5?$AAd?$AAw?$AAQ@ 001467e8     callctrl.obj
 0002:00005840       ??_C@_1FC@IIPADAAF@?$AAC?$AAR?$AAa?$AAd?$AAi?$AAo?$AA?3?$AA?3?$AAM?$AAa?$AAn?$AAa?$AAg?$AAe?$AAC?$AAa?$AAl?$AAl?$AA?5?$AAc?$AAm?$AAd?$AA?5?$AA?$DN?$AA?5?$AA?$CF?$AAd?$AA?0?$AA?5?$AAc?$AAa?$AAl@ 00146840     callctrl.obj
 0002:000058e0       ??_C@_1EC@NABPKBOI@?$AAS?$AAt?$AAo?$AAp?$AAD?$AAT?$AAM?$AAF?$AAK?$AAe?$AAy?$AA?5?$AAf?$AAa?$AAi?$AAl?$AAe?$AAd?$AA?$CB?$AA?5?$AAD?$AAT?$AAM?$AAF?$AAK?$AAe?$AAy?$AA?5?$AA?$DN?$AA?5?$AA?$CF?$AAd@ 001468e0     callctrl.obj
 0002:00005928       ??_C@_1EE@MMOHIGBP@?$AAS?$AAt?$AAa?$AAr?$AAt?$AAD?$AAT?$AAM?$AAF?$AAK?$AAe?$AAy?$AA?5?$AAf?$AAa?$AAi?$AAl?$AAe?$AAd?$AA?$CB?$AA?5?$AAD?$AAT?$AAM?$AAF?$AAK?$AAe?$AAy?$AA?5?$AA?$DN?$AA?5?$AA?$CF@ 00146928     callctrl.obj
 0002:00005970       ??_C@_1GE@DFKGMNGB@?$AAm?$AAp?$AAF?$AAn?$AAP?$AAl?$AAa?$AAy?$AAA?$AAu?$AAd?$AAi?$AAo?$AAT?$AAo?$AAn?$AAe?$AA?5?$AAf?$AAa?$AAi?$AAl?$AAe?$AAd?$AA?$CB?$AA?5?$AAr?$AAe?$AAt?$AA?5?$AA?$DN?$AA?5@ 00146970     callctrl.obj
 0002:000059d8       ??_C@_1EM@JLNHOFMJ@?$AAS?$AAE?$AAN?$AAD?$AA?5?$AAD?$AAT?$AAM?$AAF?$AA?3?$AA?5?$AAt?$AAo?$AAn?$AAe?$AA?5?$AA0?$AAx?$AA?$CF?$AAx?$AA?0?$AA?5?$AAD?$AAu?$AAr?$AAa?$AAt?$AAi?$AAo?$AAn?$AA?5?$AA?$DN@ 001469d8     callctrl.obj
 0002:00005a24       ??_C@_1BE@IKEPKMAH@?$AAR?$AAI?$AAL?$AA?2?$AAA?$AAu?$AAd?$AAi?$AAo?$AA?$AA@ 00146a24     callctrl.obj
 0002:00005a38       ??_C@_1DK@DFOPCCDF@?$AAS?$AAo?$AAf?$AAt?$AAw?$AAa?$AAr?$AAe?$AA?2?$AAS?$AAi?$AAe?$AAr?$AAr?$AAa?$AA?5?$AAW?$AAi?$AAr?$AAe?$AAl?$AAe?$AAs?$AAs?$AA?5?$AAI?$AAn?$AAc?$AA?$AA@ 00146a38     callctrl.obj
 0002:00005a74       ??_C@_1M@DFKENGJN@?$AA?$CF?$AAs?$AA?2?$AA?$CF?$AAs?$AA?$AA@ 00146a74     callctrl.obj
 0002:00005a80       ??_C@_1BK@NMBDBCCI@?$AAD?$AAT?$AAM?$AAF?$AAT?$AAo?$AAn?$AAe?$AAT?$AAy?$AAp?$AAe?$AA?$AA@ 00146a80     callctrl.obj
 0002:00005a9c       ??_C@_1BK@LJACFJAI@?$AAD?$AAT?$AAM?$AAF?$AAD?$AAu?$AAr?$AAa?$AAt?$AAi?$AAo?$AAn?$AA?$AA@ 00146a9c     callctrl.obj
 0002:00005ab8       ??_C@_0N@MHBNBAPM@?$CD?$CK0123456789?$AA@ 00146ab8     callctrl.obj
 0002:00005b00       ??_C@_1FE@CNJACHEJ@?$AAS?$AAe?$AAt?$AAC?$AAa?$AAl?$AAl?$AAS?$AAt?$AAa?$AAt?$AAu?$AAs?$AA?5?$AAc?$AAa?$AAl?$AAl?$AAi?$AAn?$AAg?$AA?5?$AAu?$AAp?$AAd?$AAa?$AAt?$AAe?$AAl?$AAi?$AAn?$AAe@ 00146b00     callctrl.obj
 0002:00005b58       ??_C@_1JG@FJCPOCJC@?$AAS?$AAe?$AAt?$AAC?$AAa?$AAl?$AAl?$AAS?$AAt?$AAa?$AAt?$AAu?$AAs?$AA?5?$AAd?$AAw?$AAI?$AAD?$AA?5?$AA?$DN?$AA?5?$AA?$CF?$AAd?$AA?0?$AA?5?$AAc?$AAa?$AAl?$AAl?$AAS?$AAt?$AAa@ 00146b58     callctrl.obj
 0002:00005c30       ??_C@_1MG@HMNNACJP@?$AAA?$AAd?$AAd?$AAC?$AAa?$AAl?$AAl?$AA?5?$AAd?$AAw?$AAC?$AAa?$AAl?$AAl?$AAI?$AAD?$AA?5?$AA?$CF?$AAd?$AA?0?$AA?5?$AAQ?$AAm?$AAi?$AAI?$AAD?$AA?5?$AA?$DN?$AA?5?$AA?$CF?$AAd?$AA?0@ 00146c30     callctrl.obj
 0002:00005cf8       ??_C@_1EO@LHFLAJIE@?$AAr?$AAe?$AAf?$AAu?$AAs?$AAe?$AA?5?$AAt?$AAo?$AA?5?$AAa?$AAd?$AAd?$AA?5?$AAt?$AAh?$AAe?$AA?5?$AAs?$AAa?$AAm?$AAe?$AA?5?$AAQ?$AAm?$AAi?$AAI?$AAd?$AA?5?$AAa?$AAg?$AAa@ 00146cf8     callctrl.obj
 0002:00005d48       ??_C@_1IC@MBKLFGFB@?$AAM?$AAo?$AAd?$AAe?$AAm?$AA?5?$AAa?$AAl?$AAr?$AAe?$AAa?$AAd?$AAy?$AA?5?$AAh?$AAa?$AAs?$AA?5?$AAa?$AA?5?$AAd?$AAa?$AAt?$AAa?$AA?5?$AAc?$AAa?$AAl?$AAl?$AA?5?$AAw?$AAi@ 00146d48     callctrl.obj
 0002:00005dd0       ??_C@_1PO@HONNGKJD@?$AAC?$AAR?$AAa?$AAd?$AAi?$AAo?$AA?3?$AA?3?$AAA?$AAd?$AAd?$AAC?$AAa?$AAl?$AAl?$AA?5?$AA?9?$AA?5?$AAd?$AAw?$AAC?$AAa?$AAl?$AAl?$AAI?$AAD?$AA?5?$AA?$CF?$AAd?$AA?0?$AA?5?$AAQ@ 00146dd0     callctrl.obj
 0002:00005f04       ??_C@_1CM@KEODMBGO@?$AAR?$AAe?$AAm?$AAC?$AAa?$AAl?$AAl?$AA?5?$AAd?$AAw?$AAC?$AAa?$AAl?$AAl?$AAI?$AAD?$AA?5?$AA?$DN?$AA?5?$AA?$CF?$AAd?$AA?$AA@ 00146f04     callctrl.obj
 0002:00005f30       ??_C@_1DC@EEKGAKCA@?$AAI?$AAn?$AAi?$AAt?$AAi?$AAa?$AAt?$AAe?$AAD?$AAa?$AAt?$AAa?$AAC?$AAa?$AAl?$AAl?$AA?5?$AAs?$AAu?$AAc?$AAc?$AAe?$AAe?$AAd?$AA?$AA@ 00146f30     callctrl.obj
 0002:00005f68       ??_C@_1GA@JAECKCGN@?$AAC?$AAr?$AAe?$AAa?$AAt?$AAe?$AAF?$AAi?$AAl?$AAe?$AA?5?$AAf?$AAa?$AAi?$AAl?$AAe?$AAd?$AA?5?$AAo?$AAn?$AA?5?$AAd?$AAa?$AAt?$AAa?$AA?5?$AAp?$AAo?$AAr?$AAt?$AA?0?$AA?5@ 00146f68     callctrl.obj
 0002:00005fc8       ??_C@_1DC@CKPNGNII@?$AAf?$AAa?$AAi?$AAl?$AAe?$AAd?$AA?0?$AA?5?$AAc?$AAl?$AAo?$AAs?$AAi?$AAn?$AAg?$AA?5?$AAc?$AAo?$AAm?$AA?5?$AAp?$AAo?$AAr?$AAt?$AA?$AA@ 00146fc8     callctrl.obj
 0002:00006000       ??_C@_1EC@PGNPHEGD@?$AAI?$AAn?$AAi?$AAt?$AAi?$AAa?$AAt?$AAe?$AAD?$AAa?$AAt?$AAa?$AAC?$AAa?$AAl?$AAl?$AA?5?$AAC?$AAr?$AAe?$AAa?$AAt?$AAe?$AAT?$AAh?$AAr?$AAe?$AAa?$AAd?$AA?5?$AA?$CF?$AAx@ 00147000     callctrl.obj
 0002:00006044       ??_C@_1CC@LGKBMPDP@?$AAW?$AAr?$AAi?$AAt?$AAe?$AAF?$AAi?$AAl?$AAe?$AA?5?$AAf?$AAa?$AAi?$AAl?$AAe?$AAd?$AA?$AA@ 00147044     callctrl.obj
 0002:00006068       ??_C@_04ONBPMAIJ@ATZD?$AA@ 00147068     callctrl.obj
 0002:00006070       ??_C@_01LIIJDEN@?$AN?$AA@  00147070     callctrl.obj
 0002:00006078       ??_C@_1FA@KDIDLJNN@?$AAS?$AAe?$AAt?$AAC?$AAo?$AAm?$AAm?$AAT?$AAi?$AAm?$AAe?$AAo?$AAu?$AAt?$AAs?$AA?$CI?$AA?$CJ?$AA?5?$AAD?$AAa?$AAt?$AAa?$AA?5?$AAp?$AAo?$AAr?$AAt?$AA?5?$AAe?$AAr?$AAr?$AAo@ 00147078     callctrl.obj
 0002:000060c8       ??_C@_1CM@COIMMFCE@?$AAR?$AAo?$AAa?$AAm?$AAi?$AAn?$AAg?$AA?5?$AAC?$AAa?$AAl?$AAl?$AA?5?$AAR?$AAe?$AAm?$AAi?$AAn?$AAd?$AAe?$AAr?$AA?$AA@ 001470c8     callctrl.obj
 0002:000060f8       ??_C@_1HK@KGLHFJJJ@?$AAR?$AAo?$AAa?$AAm?$AAi?$AAn?$AAg?$AA?5?$AAR?$AAa?$AAt?$AAe?$AA?5?$AAa?$AAp?$AAp?$AAl?$AAi?$AAe?$AAs?$AA?5?$AAf?$AAo?$AAr?$AA?5?$AAt?$AAh?$AAi?$AAs?$AA?5?$AAc?$AAa@ 001470f8     callctrl.obj
 0002:00006174       ??_C@_1BM@KGGCDICL@?$AAC?$AAo?$AAn?$AAn?$AAe?$AAc?$AAt?$AAi?$AAn?$AAg?$AA?4?$AA?4?$AA?4?$AA?$AA@ 00147174     callctrl.obj
 0002:00006190       ??_C@_1FO@NINIOGNH@?$AAC?$AAR?$AAa?$AAd?$AAi?$AAo?$AA?3?$AA?3?$AAD?$AAi?$AAa?$AAl?$AA?5?$AAG?$AAe?$AAt?$AAR?$AAe?$AAg?$AAi?$AAs?$AAt?$AAr?$AAy?$AAD?$AAW?$AAO?$AAR?$AAD?$AA?5?$AAR?$AAo@ 00147190     callctrl.obj
 0002:000061f0       ??_C@_1CC@LPFDJFMA@?$AAI?$AAn?$AAi?$AAt?$AAi?$AAa?$AAt?$AAe?$AAD?$AAa?$AAt?$AAa?$AAC?$AAa?$AAl?$AAl?$AA?$AA@ 001471f0     callctrl.obj
 0002:00006214       ??_C@_1BE@OIBEOKIJ@?$AAR?$AAo?$AAa?$AAm?$AAG?$AAu?$AAa?$AAr?$AAd?$AA?$AA@ 00147214     callctrl.obj
 0002:00006228       ??_C@_1EK@CPPGCLPN@?$AA?2?$AAS?$AAo?$AAf?$AAt?$AAw?$AAa?$AAr?$AAe?$AA?2?$AAS?$AAi?$AAe?$AAr?$AAr?$AAa?$AA?5?$AAW?$AAi?$AAr?$AAe?$AAl?$AAe?$AAs?$AAs?$AA?5?$AAI?$AAn?$AAc?$AA?2?$AAS?$AAy@ 00147228     callctrl.obj
 0002:00006278       ??_C@_1GI@EDLIHAOA@?$AAS?$AAW?$AAI?$AA_?$AAN?$AAO?$AAT?$AAI?$AAF?$AAY?$AA_?$AAC?$AAa?$AAl?$AAl?$AAC?$AAo?$AAn?$AAn?$AAe?$AAc?$AAt?$AAi?$AAn?$AAg?$AA?3?$AA?5?$AAu?$AAn?$AAh?$AAa?$AAn@ 00147278     callctrl.obj
 0002:000062e0       ??_C@_1HG@HIEDOBNM@?$AAA?$AAs?$AAy?$AAn?$AAc?$AAD?$AAa?$AAt?$AAa?$AA?5?$AAc?$AAa?$AAl?$AAl?$AA?5?$AAc?$AAo?$AAn?$AAn?$AAe?$AAc?$AAt?$AAi?$AAn?$AAg?$AA?4?$AA?5?$AAA?$AAd?$AAd?$AA?5?$AAR@ 001472e0     callctrl.obj
 0002:00006358       ??_C@_1IO@FNBPCBIC@?$AAA?$AAs?$AAy?$AAn?$AAc?$AAD?$AAa?$AAt?$AAa?$AA?5?$AAc?$AAa?$AAl?$AAl?$AA?5?$AAc?$AAo?$AAn?$AAn?$AAe?$AAc?$AAt?$AAi?$AAn?$AAg?$AA?4?$AA?5?$AAR?$AAI?$AAL?$AA_?$AAD@ 00147358     callctrl.obj
 0002:000063e8       ??_C@_1EA@EHHDMDIN@?$AAH?$AAa?$AAn?$AAd?$AAl?$AAe?$AAS?$AAW?$AAI?$AA_?$AAN?$AAO?$AAT?$AAI?$AAF?$AAY?$AA_?$AAC?$AAa?$AAl?$AAl?$AAC?$AAo?$AAn?$AAn?$AAe?$AAc?$AAt?$AAi?$AAn?$AAg?$AA?$AA@ 001473e8     callctrl.obj
 0002:00006428       ??_C@_1FC@GBLIJDLA@?$AAA?$AAn?$AAy?$AA?5?$AAO?$AAT?$AAH?$AAE?$AAR?$AA?5?$AAC?$AAa?$AAl?$AAl?$AA?5?$AAC?$AAo?$AAn?$AAn?$AAe?$AAc?$AAt?$AAe?$AAd?$AA?5?$AAe?$AAS?$AAt?$AAa?$AAt?$AAe?$AA?5@ 00147428     callctrl.obj
 0002:00006480       ??_C@_1EE@KHKLMBPK@?$AAD?$AAa?$AAt?$AAa?$AAC?$AAa?$AAl?$AAl?$AAC?$AAo?$AAn?$AAn?$AAe?$AAc?$AAt?$AAe?$AAd?$AA?5?$AAe?$AAS?$AAt?$AAa?$AAt?$AAe?$AA?5?$AA?$DN?$AA?5?$AA0?$AAx?$AA?$CF?$AAx?$AA?4@ 00147480     callctrl.obj
 0002:000064c8       ??_C@_1FE@NNDOCCDL@?$AAD?$AAO?$AAR?$AAM?$AAA?$AAN?$AAT?$AA?5?$AAD?$AAa?$AAt?$AAa?$AAC?$AAa?$AAl?$AAl?$AAC?$AAo?$AAn?$AAn?$AAe?$AAc?$AAt?$AAe?$AAd?$AA?5?$AAe?$AAS?$AAt?$AAa?$AAt?$AAe@ 001474c8     callctrl.obj
 0002:00006520       ??_C@_1GA@EFFPIFNA@?$AAM?$AAo?$AAd?$AAe?$AAm?$AA?5?$AAs?$AAt?$AAa?$AAr?$AAt?$AAs?$AA?5?$AAa?$AA?5?$AAd?$AAa?$AAt?$AAa?$AA?5?$AAc?$AAa?$AAl?$AAl?$AA?5?$AAo?$AAn?$AA?5?$AAi?$AAt?$AAs?$AA?5@ 00147520     callctrl.obj
 0002:00006580       ??_C@_1IE@JIAHGKIJ@?$AAN?$AAo?$AA?5?$AAc?$AAo?$AAn?$AAn?$AAe?$AAc?$AAt?$AAi?$AAo?$AAn?$AA?5?$AAi?$AAn?$AA?5?$AAl?$AAi?$AAs?$AAt?$AA?5?$AAw?$AAh?$AAe?$AAn?$AA?5?$AAS?$AAW?$AAI?$AA_?$AAN@ 00147580     callctrl.obj
 0002:00006604       ??_C@_1CC@FAHGNPFK@?$AAb?$AAe?$AAf?$AAo?$AAr?$AAe?$AA?5?$AAu?$AAp?$AAd?$AAa?$AAt?$AAe?$AA?5?$AA?$CF?$AAd?$AA?$AA@ 00147604     callctrl.obj
 0002:00006628       ??_C@_1CA@MFPLFNFK@?$AAa?$AAf?$AAt?$AAe?$AAr?$AA?5?$AAu?$AAp?$AAd?$AAa?$AAt?$AAe?$AA?5?$AA?$CF?$AAd?$AA?$AA@ 00147628     callctrl.obj
 0002:00006648       ??_C@_1CK@MHHFEIOJ@?$AAc?$AAa?$AAl?$AAl?$AA?5?$AAa?$AAr?$AAr?$AAa?$AAy?$AA?5?$AAn?$AAo?$AAt?$AA?5?$AAf?$AAo?$AAu?$AAn?$AAd?$AA?$AA@ 00147648     callctrl.obj
 0002:00006674       ??_C@_1CC@IEAMMAJA@?$AAc?$AAa?$AAl?$AAl?$AA?5?$AAa?$AAr?$AAr?$AAa?$AAy?$AA?5?$AAf?$AAo?$AAu?$AAn?$AAd?$AA?$AA@ 00147674     callctrl.obj
 0002:00006698       ??_C@_1FK@FKKIKCKC@?$AAH?$AAa?$AAn?$AAd?$AAl?$AAe?$AAS?$AAW?$AAI?$AA_?$AAN?$AAO?$AAT?$AAI?$AAF?$AAY?$AA_?$AAC?$AAa?$AAl?$AAl?$AAC?$AAo?$AAn?$AAn?$AAe?$AAc?$AAt?$AAe?$AAd?$AA?5?$AAe@ 00147698     callctrl.obj
 0002:000066f8       ??_C@_1LE@DOINKOGB@?$AAS?$AAW?$AAI?$AA_?$AAN?$AAO?$AAT?$AAI?$AAF?$AAY?$AA_?$AAP?$AAk?$AAt?$AAS?$AAe?$AAs?$AAs?$AAi?$AAo?$AAn?$AAC?$AAa?$AAl?$AAl?$AA?5?$AAr?$AAe?$AAc?$AAe?$AAi?$AAv@ 001476f8     callctrl.obj
 0002:000067b0       ??_C@_1IE@BJFLNPLE@?$AAD?$AAa?$AAt?$AAa?$AA?5?$AAC?$AAa?$AAl?$AAl?$AA?5?$AAD?$AAi?$AAs?$AAc?$AAo?$AAn?$AAn?$AAe?$AAc?$AAt?$AA?5?$AAr?$AAe?$AAc?$AAe?$AAi?$AAv?$AAe?$AAd?$AA?4?$AA?5?$AAR@ 001477b0     callctrl.obj
 0002:00006838       ??_C@_1JC@LJOAEDFN@?$AAH?$AAa?$AAn?$AAd?$AAl?$AAe?$AAS?$AAW?$AAI?$AA_?$AAN?$AAO?$AAT?$AAI?$AAF?$AAY?$AA_?$AAP?$AAk?$AAt?$AAS?$AAe?$AAs?$AAs?$AAi?$AAo?$AAn?$AAC?$AAa?$AAl?$AAl?$AA?5@ 00147838     callctrl.obj
 0002:000068d0       ??_C@_1KI@HBAGLKGH@?$AAH?$AAa?$AAn?$AAd?$AAl?$AAe?$AAS?$AAW?$AAI?$AA_?$AAN?$AAO?$AAT?$AAI?$AAF?$AAY?$AA_?$AAP?$AAk?$AAt?$AAS?$AAe?$AAs?$AAs?$AAi?$AAo?$AAn?$AAC?$AAa?$AAl?$AAl?$AA?5@ 001478d0     callctrl.obj
 0002:00006978       ??_C@_1FI@OEHEBGBG@?$AAR?$AAI?$AAL?$AA_?$AAD?$AAA?$AAT?$AAA?$AA_?$AAC?$AAA?$AAL?$AAL?$AAI?$AAD?$AA?5?$AAa?$AAl?$AAr?$AAe?$AAa?$AAd?$AAy?$AA?5?$AAe?$AAx?$AAi?$AAs?$AAt?$AAe?$AAd?$AA?4@ 00147978     callctrl.obj
 0002:000069d0       ??_C@_1EA@IGNNHOIP@?$AAH?$AAa?$AAn?$AAd?$AAl?$AAe?$AAS?$AAW?$AAI?$AA_?$AAN?$AAO?$AAT?$AAI?$AAF?$AAY?$AA_?$AAP?$AAk?$AAt?$AAS?$AAe?$AAs?$AAs?$AAi?$AAo?$AAn?$AAC?$AAa?$AAl?$AAl?$AA?$AA@ 001479d0     callctrl.obj
 0002:00006a48       ??_C@_1KC@HJKBINN@?$AAS?$AAw?$AAi?$AAG?$AAe?$AAt?$AAM?$AAi?$AAp?$AAE?$AAr?$AAr?$AAC?$AAo?$AAd?$AAe?$AA?0?$AA?5?$AAr?$AAC?$AAo?$AAd?$AAe?$AA?5?$AA?$DN?$AA?5?$AA?$CF?$AAd?$AA?0?$AA?5?$AAe?$AAr@ 00147a48     callctrl.obj
 0002:00006af0       ??_C@_1HA@MHPBIKKP@?$AAM?$AAI?$AAP?$AA?5?$AAe?$AAr?$AAr?$AAo?$AAr?$AA?5?$AA?$DN?$AA?5?$AA?$CF?$AAd?$AA?0?$AA?5?$AAd?$AAw?$AAD?$AAi?$AAs?$AAc?$AAo?$AAn?$AAn?$AAe?$AAc?$AAt?$AAC?$AAa?$AAu?$AAs@ 00147af0     callctrl.obj
 0002:00006b60       ??_C@_1BEI@HNKHBMNO@?$AAR?$AAi?$AAl?$AA?5?$AAi?$AAs?$AA?5?$AAi?$AAg?$AAn?$AAo?$AAr?$AAi?$AAn?$AAg?$AA?5?$AAt?$AAh?$AAe?$AA?5?$AAS?$AAW?$AAI?$AA_?$AAN?$AAO?$AAT?$AAI?$AAF?$AAY?$AA_?$AAC@ 00147b60     callctrl.obj
 0002:00006d18       ??_C@_1BK@BEPAKJNC@?$AAR?$AAI?$AAL?$AAD?$AAr?$AAv?$AA_?$AAD?$AAi?$AAa?$AAl?$AA?9?$AA?$AA@ 00147d18     callctrl.obj
 0002:00006d34       ??_C@_19BGDFMPBJ@?$AAl?$AAe?$AAo?$AA?5?$AA?$AA@ 00147d34     callctrl.obj
 0002:00006d40       ??_C@_1HE@EMKBDIKF@?$AAC?$AAu?$AAr?$AAr?$AAe?$AAn?$AAt?$AA?5?$AAi?$AAn?$AAt?$AAe?$AAr?$AAn?$AAa?$AAl?$AA?5?$AAd?$AAa?$AAt?$AAa?$AA?5?$AAc?$AAa?$AAl?$AAl?$AA?5?$AAs?$AAt?$AAa?$AAt?$AAu@ 00147d40     callctrl.obj
 0002:00006db4       ??_C@_1CM@OKBAAH@?$AAF?$AAa?$AAi?$AAl?$AA?5?$AAt?$AAo?$AA?5?$AAA?$AAd?$AAd?$AA?5?$AAD?$AAa?$AAt?$AAa?$AA?5?$AAC?$AAa?$AAl?$AAl?$AA?$AA@ 00147db4     callctrl.obj
 0002:00006de0       ??_C@_1BK@DBJLPGAO@?$AAR?$AAI?$AAL?$AAD?$AAr?$AAv?$AA_?$AAD?$AAi?$AAa?$AAl?$AA?$CL?$AA?$AA@ 00147de0     callctrl.obj
 0002:00006e40       ??_C@_1FI@IBALLLCM@?$AAH?$AAa?$AAn?$AAg?$AAu?$AAp?$AA?5?$AAg?$AAo?$AAt?$AA?5?$AAt?$AAh?$AAo?$AAu?$AAg?$AAh?$AA?5?$AAD?$AAa?$AAt?$AAa?$AA?5?$AAf?$AAe?$AAa?$AAt?$AAu?$AAr?$AAe?$AAs?$AA?5@ 00147e40     callctrl.obj
 0002:00006e98       ??_C@_1FK@HCNBLKIN@?$AAH?$AAa?$AAn?$AAg?$AAu?$AAp?$AA?5?$AAg?$AAo?$AAt?$AA?5?$AAt?$AAh?$AAo?$AAu?$AAg?$AAh?$AA?5?$AAV?$AAo?$AAi?$AAc?$AAe?$AA?5?$AAf?$AAe?$AAa?$AAt?$AAu?$AAr?$AAe?$AAs@ 00147e98     callctrl.obj
 0002:00006ef4       ??_C@_1DE@GGCLGMIO@?$AAH?$AAa?$AAn?$AAg?$AAu?$AAp?$AA?5?$AAf?$AAa?$AAi?$AAl?$AAe?$AAd?$AA?$CB?$AA?$CB?$AA?$CB?$AA?5?$AA?$CF?$AAd?$AA?5?$AA?$CF?$AAd?$AA?5?$AA?$CF?$AAd?$AA?$AA@ 00147ef4     callctrl.obj
 0002:00006f28       ??_C@_1BO@PDEPFFKN@?$AAC?$AAR?$AAa?$AAd?$AAi?$AAo?$AA?3?$AA?3?$AAH?$AAa?$AAn?$AAg?$AAU?$AAp?$AA?$AA@ 00147f28     callctrl.obj
 0002:00006f80       ??_C@_1EA@GCEHDDNC@?$AAR?$AAI?$AAL?$AA?5?$AAM?$AAa?$AAn?$AAa?$AAg?$AAe?$AA?5?$AAN?$AAO?$AAO?$AAP?$AA?5?$AAf?$AAo?$AAr?$AA?5?$AAc?$AAa?$AAl?$AAl?$AAI?$AAD?$AA?5?$AA?$DN?$AA?5?$AA?$CF?$AAd?$AA?$AA@ 00147f80     callctrl.obj
 0002:00006fc0       ??_C@_1IK@BLJKHNPH@?$AAR?$AAI?$AAL?$AA_?$AAM?$AAa?$AAn?$AAa?$AAg?$AAe?$AA?5?$AAw?$AAa?$AAn?$AAt?$AAs?$AA?5?$AAt?$AAo?$AA?5?$AAc?$AAa?$AAn?$AAc?$AAe?$AAl?$AA?5?$AAa?$AA?5?$AAd?$AAi?$AAa@ 00147fc0     callctrl.obj
 0002:00007050       ??_C@_1FG@NDIJHFGI@?$AAC?$AAR?$AAa?$AAd?$AAi?$AAo?$AA?3?$AA?3?$AAM?$AAa?$AAn?$AAa?$AAg?$AAe?$AAC?$AAa?$AAl?$AAl?$AA?5?$AAc?$AAm?$AAd?$AA?5?$AA?$DN?$AA?5?$AA?$CF?$AAd?$AA?0?$AA?5?$AAc?$AAa?$AAl@ 00148050     callctrl.obj
 0002:000070a8       ??_C@_1CI@BJKFDKFL@?$AAS?$AAe?$AAn?$AAd?$AAF?$AAl?$AAa?$AAs?$AAh?$AA?5?$AAF?$AAa?$AAi?$AAl?$AAe?$AAd?$AA?$CB?$AA?$CB?$AA?$CB?$AA?$AA@ 001480a8     callctrl.obj
 0002:000070d0       ??_C@_1EC@MJHJCKKJ@?$AAT?$AAh?$AAi?$AAs?$AA?5?$AAi?$AAs?$AA?5?$AAa?$AAn?$AAs?$AAw?$AAe?$AAr?$AAi?$AAn?$AAg?$AA?5?$AAa?$AA?5?$AAw?$AAa?$AAi?$AAt?$AAi?$AAn?$AAg?$AA?5?$AAc?$AAa?$AAl?$AAl@ 001480d0     callctrl.obj
 0002:00007118       ??_C@_1GK@GDHCDGHP@?$AAF?$AAl?$AAa?$AAs?$AAh?$AA?5?$AAw?$AAi?$AAt?$AAh?$AA?5?$AAP?$AAh?$AAo?$AAn?$AAe?$AA?5?$AAI?$AAn?$AAf?$AAo?$AA?0?$AA?5?$AAa?$AAt?$AAt?$AAe?$AAm?$AAp?$AAt?$AA?5?$AAt@ 00148118     callctrl.obj
 0002:00007188       ??_C@_1GE@GEOMAJIJ@?$AAA?$AAS?$AAS?$AAE?$AAR?$AAT?$AAI?$AAO?$AAN?$AA?5?$AAF?$AAA?$AAI?$AAL?$AAU?$AAR?$AAE?$AA?3?$AA?5?$AA?$DN?$AA?$DN?$AA?$DN?$AA?$DO?$AA_?$AAt?$AAc?$AAs?$AAl?$AAe?$AAn?$AA?5?$AA?$CI@ 00148188     callctrl.obj
 0002:000071f0       ??_C@_1FC@GGEGCOBB@?$AAU?$AAn?$AAh?$AAa?$AAn?$AAd?$AAl?$AAe?$AAd?$AA?5?$AAS?$AAe?$AAn?$AAd?$AAF?$AAl?$AAa?$AAs?$AAh?$AA?5?$AAw?$AAi?$AAt?$AAh?$AA?5?$AAc?$AAa?$AAl?$AAl?$AAS?$AAt?$AAa@ 001481f0     callctrl.obj
 0002:00007248       ??_C@_1GG@KCCNHKEE@?$AAC?$AAR?$AAa?$AAd?$AAi?$AAo?$AA?3?$AA?3?$AAS?$AAe?$AAn?$AAd?$AAF?$AAl?$AAa?$AAs?$AAh?$AA?5?$AAa?$AAd?$AAd?$AAr?$AAe?$AAs?$AAs?$AA?5?$AAi?$AAs?$AA?5?$AA?$CF?$AAs?$AA?5@ 00148248     callctrl.obj
 0002:000072b0       ??_C@_1GE@NNJADOND@?$AAS?$AAW?$AAI?$AA_?$AAN?$AAO?$AAT?$AAI?$AAF?$AAY?$AA_?$AAC?$AAa?$AAl?$AAl?$AAD?$AAi?$AAs?$AAc?$AAo?$AAn?$AAn?$AAe?$AAc?$AAt?$AAe?$AAd?$AA?5?$AAf?$AAa?$AAi?$AAl@ 001482b0     callctrl.obj
 0002:00007318       ??_C@_1FM@CBHPJHLM@?$AAr?$AAe?$AAm?$AAc?$AAc?$AAa?$AAl?$AAl?$AA?5?$AAf?$AAo?$AAr?$AA?5?$AAd?$AAa?$AAt?$AAa?$AA?5?$AAc?$AAa?$AAl?$AAl?$AA?0?$AA?5?$AAQ?$AAm?$AAi?$AAI?$AAD?$AA?5?$AA?$CF?$AAd@ 00148318     callctrl.obj
 0002:00007378       ??_C@_1KO@DPFKFMGJ@?$AAC?$AAA?$AAL?$AAL?$AA_?$AAE?$AAN?$AAD?$AA?0?$AA?5?$AAm?$AA_?$AAb?$AAA?$AAc?$AAt?$AAi?$AAv?$AAa?$AAt?$AAi?$AAo?$AAn?$AAP?$AAa?$AAs?$AAs?$AAe?$AAd?$AA?5?$AA?$DN?$AA?$DN@ 00148378     callctrl.obj
 0002:00007428       ??_C@_1FC@CKJHCLP@?$AAc?$AAo?$AAu?$AAl?$AAd?$AA?5?$AAn?$AAo?$AAt?$AA?5?$AAf?$AAi?$AAn?$AAd?$AA?5?$AAc?$AAa?$AAl?$AAl?$AA?5?$AAt?$AAo?$AA?5?$AAR?$AAe?$AAm?$AAC?$AAa?$AAl?$AAl?$AA?0?$AA?5@ 00148428     callctrl.obj
 0002:0000747c       ??_C@_1DM@BOGHFOID@?$AAR?$AAe?$AAm?$AAC?$AAa?$AAl?$AAl?$AA?0?$AA?5?$AAQ?$AAm?$AAi?$AAI?$AAD?$AA?5?$AA?$CF?$AAd?$AA?5?$AAd?$AAw?$AAC?$AAa?$AAl?$AAl?$AAI?$AAD?$AA?5?$AA?$CF?$AAd?$AA?$AA@ 0014847c     callctrl.obj
 0002:000074b8       ??_C@_1JO@OCICMPDH@?$AAS?$AAW?$AAI?$AA_?$AAN?$AAO?$AAT?$AAI?$AAF?$AAY?$AA_?$AAC?$AAa?$AAl?$AAl?$AAD?$AAi?$AAs?$AAc?$AAo?$AAn?$AAn?$AAe?$AAc?$AAt?$AAe?$AAd?$AA?5?$AAe?$AAS?$AAt?$AAa@ 001484b8     callctrl.obj
 0002:00007558       ??_C@_1M@ENKMPMBE@?$AAP?$AAh?$AAo?$AAn?$AAe?$AA?$AA@ 00148558     callctrl.obj
 0002:00007568       ??_C@_1NG@HLKLBKFB@?$AAY?$AAo?$AAu?$AAr?$AA?5?$AAc?$AAa?$AAl?$AAl?$AA?5?$AAb?$AAa?$AAr?$AAr?$AAi?$AAn?$AAg?$AA?5?$AAs?$AAe?$AAt?$AAt?$AAi?$AAn?$AAg?$AAs?$AA?5?$AAd?$AAo?$AA?5?$AAn?$AAo@ 00148568     callctrl.obj
 0002:00007640       ??_C@_1FA@HGPBKHGI@?$AAf?$AAa?$AAi?$AAl?$AAe?$AAd?$AA?5?$AAt?$AAo?$AA?5?$AAa?$AAd?$AAd?$AA?5?$AAc?$AAa?$AAl?$AAl?$AA?0?$AA?5?$AAc?$AAa?$AAl?$AAl?$AA?5?$AAf?$AAu?$AAl?$AAl?$AA?$DP?$AA?5?$AAQ@ 00148640     callctrl.obj
 0002:00007690       ??_C@_1EC@GKBKHJKD@?$AAc?$AAa?$AAl?$AAl?$AA?5?$AAa?$AAd?$AAd?$AAe?$AAd?$AA?5?$AAt?$AAo?$AA?5?$AAC?$AAa?$AAl?$AAl?$AAI?$AAD?$AA?5?$AA?$CF?$AAd?$AA?5?$AAQ?$AAm?$AAi?$AAI?$AAd?$AA?5?$AA?$CF?$AAd@ 00148690     callctrl.obj
 0002:000076d4       ??_C@_1DO@BEALADKP@?$AAs?$AAe?$AAc?$AAo?$AAn?$AAd?$AA?5?$AAR?$AAi?$AAn?$AAg?$AA?5?$AAC?$AAa?$AAl?$AAl?$AAI?$AAD?$AA?5?$AA?$CF?$AAd?$AA?5?$AAQ?$AAm?$AAi?$AAI?$AAd?$AA?5?$AA?$CF?$AAd?$AA?$AA@ 001486d4     callctrl.obj
 0002:00007714       ??_C@_1CO@PHFNMKCH@?$AAc?$AAa?$AAl?$AAl?$AA?5?$AAi?$AAn?$AAc?$AAo?$AAm?$AAi?$AAn?$AAg?$AA?5?$AAQ?$AAM?$AAI?$AAI?$AAD?$AA?5?$AA?$CF?$AAd?$AA?$AA@ 00148714     callctrl.obj
 0002:00007748       ??_C@_1GA@FNJCGOCD@?$AAf?$AAa?$AAi?$AAl?$AAe?$AAd?$AA?5?$AAt?$AAo?$AA?5?$AAa?$AAd?$AAd?$AA?5?$AAw?$AAa?$AAi?$AAt?$AAi?$AAn?$AAg?$AA?5?$AAc?$AAa?$AAl?$AAl?$AA?0?$AA?5?$AAc?$AAa?$AAl?$AAl@ 00148748     callctrl.obj
 0002:000077a8       ??_C@_1FC@GKIFNMGO@?$AAw?$AAa?$AAi?$AAt?$AAi?$AAn?$AAg?$AA?5?$AAc?$AAa?$AAl?$AAl?$AA?5?$AAa?$AAd?$AAd?$AAe?$AAd?$AA?5?$AAt?$AAo?$AA?5?$AAC?$AAa?$AAl?$AAl?$AAI?$AAD?$AA?5?$AA?$CF?$AAd?$AA?5@ 001487a8     callctrl.obj
 0002:00007800       ??_C@_1FI@DKEJGKNM@?$AAs?$AAe?$AAc?$AAo?$AAn?$AAd?$AA?5?$AAc?$AAa?$AAl?$AAl?$AA?5?$AAw?$AAa?$AAi?$AAt?$AAi?$AAn?$AAg?$AA?5?$AAR?$AAi?$AAn?$AAg?$AA?5?$AAC?$AAa?$AAl?$AAl?$AAI?$AAD?$AA?5@ 00148800     callctrl.obj
 0002:00007858       ??_C@_1CM@OKNPHJDO@?$AAc?$AAa?$AAl?$AAl?$AA?5?$AAw?$AAa?$AAi?$AAt?$AAi?$AAn?$AAg?$AA?5?$AAQ?$AAM?$AAI?$AAI?$AAD?$AA?5?$AA?$CF?$AAd?$AA?$AA@ 00148858     callctrl.obj
 0002:00007888       ??_C@_1FA@FLJNKOAC@?$AAi?$AAg?$AAn?$AAo?$AAr?$AAi?$AAn?$AAg?$AA?5?$AAi?$AAt?$AA?5?$AAi?$AAs?$AA?5?$AAa?$AAl?$AAr?$AAe?$AAa?$AAd?$AAy?$AA?5?$AAi?$AAn?$AA?5?$AAc?$AAa?$AAl?$AAl?$AA?5?$AAa@ 00148888     callctrl.obj
 0002:000078d8       ??_C@_1DO@PECHBACL@?$AAH?$AAa?$AAn?$AAd?$AAl?$AAe?$AAS?$AAW?$AAI?$AA_?$AAN?$AAO?$AAT?$AAI?$AAF?$AAY?$AA_?$AAC?$AAa?$AAl?$AAl?$AAI?$AAn?$AAc?$AAo?$AAm?$AAm?$AAi?$AAn?$AAg?$AA?$AA@ 001488d8     callctrl.obj
 0002:00007918       ??_C@_1CE@DHBOHBAM@?$AAi?$AAn?$AAc?$AAo?$AAm?$AAi?$AAn?$AAg?$AA?5?$AAQ?$AAm?$AAi?$AAI?$AAD?$AA?5?$AA?$CF?$AAd?$AA?$AA@ 00148918     callctrl.obj
 0002:00007940       ??_C@_1LA@PNIJKBGF@?$AAR?$AAe?$AAc?$AAe?$AAi?$AAv?$AAe?$AA?5?$AAS?$AAW?$AAI?$AA_?$AAN?$AAO?$AAT?$AAI?$AAF?$AAY?$AA_?$AAC?$AAa?$AAl?$AAl?$AAC?$AAa?$AAl?$AAl?$AAe?$AAr?$AAI?$AAD?$AA?5@ 00148940     callctrl.obj
 0002:000079f0       ??_C@_1CA@BPEBMMHF@?$AAS?$AAW?$AAI?$AA_?$AAN?$AAO?$AAT?$AAI?$AAF?$AAY?$AA_?$AAC?$AAO?$AAL?$AAP?$AA?$AA@ 001489f0     callctrl.obj
 0002:00007a10       ??_C@_1BI@EHAJMBKH@?$AAP?$AAh?$AAo?$AAn?$AAe?$AA?3?$AA?5?$AAC?$AAO?$AAL?$AAP?$AA?$AA@ 00148a10     callctrl.obj
 0002:00007a28       ??_C@_1DA@LPMKKOFJ@?$AAS?$AAW?$AAI?$AA_?$AAN?$AAO?$AAT?$AAI?$AAF?$AAY?$AA_?$AAC?$AAa?$AAl?$AAl?$AAC?$AAa?$AAl?$AAl?$AAe?$AAr?$AAI?$AAD?$AA?$AA@ 00148a28     callctrl.obj
 0002:00007a9c       ??_C@_1BM@HEJKBNGE@?$AAp?$AAN?$AAo?$AAt?$AAi?$AAf?$AAy?$AA?5?$AAN?$AAU?$AAL?$AAL?$AA?$CB?$AA?$AA@ 00148a9c     callctrl.obj
 0002:00007ab8       ??_C@_1KC@JDBOEBBI@?$AAU?$AAp?$AAd?$AAa?$AAt?$AAe?$AAA?$AAn?$AAd?$AAB?$AAr?$AAo?$AAa?$AAd?$AAc?$AAa?$AAs?$AAt?$AAO?$AAn?$AAS?$AAW?$AAI?$AAC?$AAa?$AAl?$AAl?$AAN?$AAo?$AAt?$AAi?$AAf@ 00148ab8     callctrl.obj
 0002:00007b60       ??_C@_1GE@PANHFAFF@?$AAI?$AAs?$AAE?$AAm?$AAe?$AAr?$AAg?$AAe?$AAn?$AAc?$AAy?$AAN?$AAu?$AAm?$AAb?$AAe?$AAr?$AA?5?$AAs?$AAk?$AAi?$AAp?$AAp?$AAi?$AAn?$AAg?$AA?5?$AA?$CK?$AA?5?$AAo?$AAr?$AA?5@ 00148b60     callctrl.obj
 0002:00007bc8       ??_C@_1GK@ICLPNICN@?$AAG?$AAe?$AAt?$AAE?$AAm?$AAe?$AAr?$AAg?$AAe?$AAn?$AAc?$AAy?$AAN?$AAu?$AAm?$AAb?$AAe?$AAr?$AAC?$AAa?$AAt?$AAe?$AAg?$AAo?$AAr?$AAy?$AA?0?$AA?5?$AAn?$AAo?$AAt?$AA?5@ 00148bc8     callctrl.obj
 0002:00007c38       ??_C@_1GC@EGIBFBHI@?$AAC?$AAR?$AAa?$AAd?$AAi?$AAo?$AA?3?$AA?3?$AAD?$AAi?$AAa?$AAl?$AA?5?$AAN?$AAo?$AA?5?$AAs?$AAu?$AAp?$AAp?$AAo?$AAr?$AAt?$AA?5?$AAf?$AAo?$AAr?$AA?5?$AAF?$AAa?$AAx?$AA?5@ 00148c38     callctrl.obj
 0002:00007ca0       ??_C@_1JO@CIJPFHLI@?$AAC?$AAR?$AAa?$AAd?$AAi?$AAo?$AA?3?$AA?3?$AAD?$AAi?$AAa?$AAl?$AA?5?$AAV?$AAo?$AAi?$AAc?$AAe?$AA?5?$AAc?$AAa?$AAl?$AAl?$AA?5?$AAs?$AAu?$AAp?$AAp?$AAo?$AAr?$AAt?$AA?5@ 00148ca0     callctrl.obj
 0002:00007d40       ??_C@_1GK@PONBHAMA@?$AAC?$AAR?$AAa?$AAd?$AAi?$AAo?$AA?3?$AA?3?$AAD?$AAi?$AAa?$AAl?$AA?5?$AAS?$AAw?$AAi?$AAS?$AAe?$AAt?$AAC?$AAa?$AAl?$AAl?$AAO?$AAr?$AAi?$AAg?$AAi?$AAn?$AAa?$AAt?$AAe@ 00148d40     callctrl.obj
 0002:00007dac       ??_C@_1DC@CLNBHDJA@?$AAa?$AAf?$AAt?$AAe?$AAr?$AA?5?$AAm?$AA_?$AAp?$AAS?$AAD?$AAK?$AAR?$AAI?$AAL?$AA?4?$AAD?$AAi?$AAa?$AAl?$AAC?$AAa?$AAl?$AAl?$AA?$AA@ 00148dac     callctrl.obj
 0002:00007de0       ??_C@_1CG@NMJCGEN@?$AAm?$AA_?$AAp?$AAS?$AAD?$AAK?$AAR?$AAI?$AAL?$AA?4?$AAD?$AAi?$AAa?$AAl?$AAC?$AAa?$AAl?$AAl?$AA?$AA@ 00148de0     callctrl.obj
 0002:00007e08       ??_C@_1GE@OLNMLEFO@?$AAC?$AAR?$AAa?$AAd?$AAi?$AAo?$AA?3?$AA?3?$AAD?$AAi?$AAa?$AAl?$AA?5?$AAG?$AAe?$AAt?$AAR?$AAe?$AAg?$AAi?$AAs?$AAt?$AAr?$AAy?$AAD?$AAW?$AAO?$AAR?$AAD?$AA?5?$AAf?$AAa@ 00148e08     callctrl.obj
 0002:00007e6c       ??_C@_1BG@NJIJAMEF@?$AAR?$AAI?$AAL?$AA?2?$AAS?$AAu?$AAp?$AAs?$AAv?$AAc?$AA?$AA@ 00148e6c     callctrl.obj
 0002:00007e84       ??_C@_1BG@HCFOPAG@?$AAC?$AAL?$AAI?$AAR?$AAS?$AAt?$AAa?$AAt?$AAu?$AAs?$AA?$AA@ 00148e84     callctrl.obj
 0002:00007ea0       ??_C@_1EA@IIIILGID@?$AAC?$AAR?$AAa?$AAd?$AAi?$AAo?$AA?3?$AA?3?$AAD?$AAi?$AAa?$AAl?$AA?5?$AAd?$AAw?$AAR?$AAi?$AAl?$AAC?$AAL?$AAI?$AAR?$AAS?$AAt?$AAa?$AAt?$AAu?$AAs?$AA?5?$AA?$CF?$AAd?$AA?$AA@ 00148ea0     callctrl.obj
 0002:00007ee0       ??_C@_1FE@LBCMLCGG@?$AAC?$AAR?$AAa?$AAd?$AAi?$AAo?$AA?3?$AA?3?$AAD?$AAi?$AAa?$AAl?$AA?5?$AAo?$AAs?$AA?5?$AAs?$AAa?$AAy?$AA?5?$AAR?$AAI?$AAL?$AA_?$AAD?$AAI?$AAA?$AAL?$AAO?$AAP?$AAT?$AA_@ 00148ee0     callctrl.obj
 0002:00007f38       ??_C@_1FG@BJPPGOIP@?$AAC?$AAR?$AAa?$AAd?$AAi?$AAo?$AA?3?$AA?3?$AAD?$AAi?$AAa?$AAl?$AA?5?$AAo?$AAs?$AA?5?$AAs?$AAa?$AAy?$AA?5?$AAR?$AAI?$AAL?$AA_?$AAD?$AAI?$AAA?$AAL?$AAO?$AAP?$AAT?$AA_@ 00148f38     callctrl.obj
 0002:00007f90       ??_C@_1DM@KHOJAHIK@?$AAC?$AAR?$AAa?$AAd?$AAi?$AAo?$AA?3?$AA?3?$AAD?$AAi?$AAa?$AAl?$AA?5?$AAd?$AAw?$AAO?$AAp?$AAt?$AAi?$AAo?$AAn?$AAs?$AA?3?$AA?$CF?$AAx?$AA?0?$AA?5?$AA?$CF?$AAx?$AA?$AA@ 00148f90     callctrl.obj
 0002:00007fd0       ??_C@_1FO@HKFJIGMK@?$AAb?$AAI?$AAs?$AAE?$AAm?$AAe?$AAr?$AAg?$AAe?$AAn?$AAc?$AAy?$AAN?$AAu?$AAm?$AAb?$AAe?$AAr?$AA?0?$AA?5?$AAs?$AAe?$AAr?$AAv?$AAi?$AAc?$AAe?$AA?5?$AAc?$AAo?$AAn?$AAd@ 00148fd0     callctrl.obj
 0002:00008030       ??_C@_15LCCIEICG@?$AA?$CK?$AA2?$AA?$AA@ 00149030     callctrl.obj
 0002:00008038       ??_C@_1HA@HBNPFLK@?$AAC?$AAR?$AAa?$AAd?$AAi?$AAo?$AA?3?$AA?3?$AAD?$AAi?$AAa?$AAl?$AA?5?$AAn?$AAo?$AAt?$AA?5?$AAa?$AAn?$AA?5?$AAe?$AAm?$AAe?$AAr?$AAg?$AAe?$AAn?$AAc?$AAy?$AA?5?$AAn?$AAu@ 00149038     callctrl.obj
 0002:000080a8       ??_C@_1CG@HOGAHMIN@?$AAb?$AAI?$AAs?$AAE?$AAm?$AAe?$AAr?$AAg?$AAe?$AAn?$AAc?$AAy?$AAN?$AAu?$AAm?$AAb?$AAe?$AAr?$AA?$AA@ 001490a8     callctrl.obj
 0002:000080d0       ??_C@_1DC@KFAFKKAM@?$AAU?$AAn?$AAa?$AAb?$AAl?$AAe?$AA?5?$AAt?$AAo?$AA?5?$AAL?$AAa?$AAu?$AAn?$AAc?$AAh?$AA?5?$AAp?$AAi?$AAn?$AAl?$AAo?$AAc?$AAk?$AA?$AA@ 001490d0     callctrl.obj
 0002:00008104       ??_C@_1CK@ODHIAEAO@?$AA?2?$AAW?$AAi?$AAn?$AAd?$AAo?$AAw?$AAs?$AA?2?$AAp?$AAi?$AAn?$AAl?$AAo?$AAc?$AAk?$AA?4?$AAe?$AAx?$AAe?$AA?$AA@ 00149104     callctrl.obj
 0002:00008130       ??_C@_1IC@KNAPPLNJ@?$AAC?$AAR?$AAa?$AAd?$AAi?$AAo?$AA?3?$AA?3?$AAD?$AAi?$AAa?$AAl?$AA?5?$AAv?$AAo?$AAi?$AAc?$AAe?$AA?5?$AAc?$AAa?$AAl?$AAl?$AA?5?$AA?$CI?$AAd?$AAw?$AAC?$AAa?$AAl?$AAl?$AAI@ 00149130     callctrl.obj
 0002:000081b8       ??_C@_1FA@NDMNJCDJ@?$AAm?$AAp?$AAF?$AAn?$AAS?$AAw?$AAi?$AAG?$AAe?$AAt?$AAC?$AAa?$AAl?$AAl?$AAC?$AAo?$AAn?$AAn?$AAe?$AAc?$AAt?$AAi?$AAo?$AAn?$AAS?$AAt?$AAa?$AAt?$AAe?$AA?5?$AAf?$AAa@ 001491b8     callctrl.obj
 0002:00008208       ??_C@_1BBI@FMECGKAP@?$AAM?$AAi?$AAc?$AAr?$AAo?$AAs?$AAo?$AAf?$AAt?$AA?5?$AAs?$AAe?$AAe?$AAs?$AA?5?$AAn?$AAo?$AA?5?$AAd?$AAa?$AAt?$AAa?$AA?5?$AAc?$AAa?$AAl?$AAl?$AA?5?$AAb?$AAe?$AAc?$AAa@ 00149208     callctrl.obj
 0002:00008320       ??_C@_1PC@KBDFCBBJ@?$AAM?$AAi?$AAc?$AAr?$AAo?$AAs?$AAo?$AAf?$AAt?$AA?5?$AAs?$AAe?$AAe?$AAs?$AA?5?$AAn?$AAo?$AA?5?$AAd?$AAa?$AAt?$AAa?$AA?5?$AAc?$AAa?$AAl?$AAl?$AA?5?$AAb?$AAe?$AAc?$AAa@ 00149320     callctrl.obj
 0002:00008418       ??_C@_1HI@JJIKFOMM@?$AAF?$AAa?$AAi?$AAl?$AA?5?$AAd?$AAa?$AAt?$AAa?$AA?5?$AAc?$AAa?$AAl?$AAl?$AA?5?$AAb?$AAe?$AAc?$AAa?$AAu?$AAs?$AAe?$AA?5?$AAm?$AA_?$AAw?$AAA?$AAc?$AAt?$AAi?$AAv?$AAe@ 00149418     callctrl.obj
 0002:00008490       ??_C@_1JA@KCMKDFM@?$AAC?$AAR?$AAa?$AAd?$AAi?$AAo?$AA?3?$AA?3?$AAD?$AAi?$AAa?$AAl?$AA?3?$AA?3?$AA?5?$AAF?$AAA?$AAI?$AAL?$AAE?$AAD?$AA?0?$AA?5?$AAb?$AAe?$AAc?$AAa?$AAu?$AAs?$AAe?$AA?5?$AAS@ 00149490     callctrl.obj
 0002:00008520       ??_C@_1LK@EFIOHHGG@?$AAC?$AAR?$AAa?$AAd?$AAi?$AAo?$AA?3?$AA?3?$AAD?$AAi?$AAa?$AAl?$AA?3?$AA?3?$AA?5?$AAF?$AAA?$AAI?$AAL?$AAE?$AAD?$AA?0?$AA?5?$AAb?$AAe?$AAc?$AAa?$AAu?$AAs?$AAe?$AA?5?$AAm@ 00149520     callctrl.obj
 0002:000085e0       ??_C@_1IK@BKDOEPJM@?$AAC?$AAR?$AAa?$AAd?$AAi?$AAo?$AA?3?$AA?3?$AAD?$AAi?$AAa?$AAl?$AA?3?$AA?3?$AA?5?$AAF?$AAA?$AAI?$AAL?$AAE?$AAD?$AA?0?$AA?5?$AAb?$AAe?$AAc?$AAa?$AAu?$AAs?$AAe?$AA?5?$AAc@ 001495e0     callctrl.obj
 0002:00008670       ??_C@_1FA@DHALLCOO@?$AAD?$AAi?$AAa?$AAl?$AA?5?$AAd?$AAa?$AAt?$AAa?$AA?5?$AAb?$AAu?$AAt?$AA?5?$AAv?$AAo?$AAi?$AAc?$AAe?$AA?5?$AAc?$AAa?$AAl?$AAl?$AA?5?$AAe?$AAx?$AAi?$AAs?$AAt?$AA?5?$AA?$DN@ 00149670     callctrl.obj
 0002:000086c0       ??_C@_1FA@GKCHIPPE@?$AAC?$AAR?$AAa?$AAd?$AAi?$AAo?$AA?3?$AA?3?$AAD?$AAi?$AAa?$AAl?$AA?5?$AAD?$AAA?$AAT?$AAA?$AA?5?$AAC?$AAA?$AAL?$AAL?$AA?5?$AAi?$AAs?$AA?5?$AAn?$AAo?$AAt?$AA?5?$AAs?$AAu@ 001496c0     callctrl.obj
 0002:00008710       ??_C@_1LG@IJPICA@?$AAD?$AAi?$AAa?$AAl?$AA?5?$AAc?$AAa?$AAl?$AAl?$AAT?$AAy?$AAp?$AAe?$AA?5?$AA?$DN?$AA?5?$AA?$CF?$AAd?$AA?5?$AAw?$AAi?$AAt?$AAh?$AA?5?$AAp?$AAo?$AAw?$AAe?$AAr?$AAS?$AAa?$AAv@ 00149710     callctrl.obj
 0002:000087c8       ??_C@_1FA@LDFJHLAO@?$AAC?$AAR?$AAa?$AAd?$AAi?$AAo?$AA?3?$AA?3?$AAD?$AAi?$AAa?$AAl?$AA?5?$AAc?$AAa?$AAl?$AAl?$AAT?$AAy?$AAp?$AAe?$AA?5?$AA?$DN?$AA?5?$AA?$CF?$AAd?$AA?0?$AA?5?$AAn?$AAu?$AAm?$AAb@ 001497c8     callctrl.obj
 0002:00008818       ??_C@_1DO@OIOJFKCC@?$AAC?$AAR?$AAa?$AAd?$AAi?$AAo?$AA?3?$AA?3?$AAD?$AAi?$AAa?$AAl?$AA?5?$AAw?$AAi?$AAt?$AAh?$AA?5?$AAe?$AAm?$AAp?$AAt?$AAy?$AA?5?$AAn?$AAu?$AAm?$AAb?$AAe?$AAr?$AA?$AA@ 00149818     callctrl.obj
 0002:00008858       ??_C@_1DG@EKCGJMJE@?$AAu?$AAn?$AAd?$AAe?$AAf?$AAi?$AAn?$AAe?$AAd?$AA?5?$AAw?$AAi?$AAr?$AAe?$AAl?$AAe?$AAs?$AAs?$AA?5?$AAt?$AAe?$AAc?$AAh?$AA?5?$AA?$CF?$AAd?$AA?$AA@ 00149858     callctrl.obj
 0002:00008890       ??_C@_1EO@GAENICFH@?$AAQ?$AAu?$AAe?$AAr?$AAy?$AAi?$AAn?$AAg?$AA?5?$AAD?$AAe?$AAv?$AAC?$AAa?$AAp?$AAs?$AA?3?$AA?5?$AAS?$AAe?$AAt?$AAB?$AAl?$AAo?$AAb?$AA?5?$AAF?$AAa?$AAi?$AAl?$AAe?$AAd@ 00149890     caps.obj
 0002:000088e0       ??_C@_1FI@EEMBPANB@?$AAQ?$AAu?$AAe?$AAr?$AAy?$AAi?$AAn?$AAg?$AA?5?$AAD?$AAe?$AAv?$AAC?$AAa?$AAp?$AAs?$AA?3?$AA?5?$AAU?$AAn?$AAh?$AAa?$AAn?$AAd?$AAl?$AAe?$AAd?$AA?5?$AAC?$AAa?$AAp?$AAs@ 001498e0     caps.obj
 0002:00008938       ??_C@_1CO@JIINKCMH@?$AAQ?$AAu?$AAe?$AAr?$AAy?$AAi?$AAn?$AAg?$AA?5?$AAD?$AAe?$AAv?$AAC?$AAa?$AAp?$AAs?$AA?3?$AA?5?$AA?$DN?$AA?5?$AA?$CF?$AAx?$AA?$AA@ 00149938     caps.obj
 0002:00008968       ??_C@_1BG@FOMBEGIH@?$AA?4?$AA?2?$AAc?$AAa?$AAp?$AAs?$AA?4?$AAc?$AAp?$AAp?$AA?$AA@ 00149968     caps.obj
 0002:00008980       ??_C@_1EI@PMCAHCLO@?$AAA?$AAS?$AAS?$AAE?$AAR?$AAT?$AAI?$AAO?$AAN?$AA?5?$AAF?$AAA?$AAI?$AAL?$AAU?$AAR?$AAE?$AA?3?$AA?5?$AA?$DN?$AA?$DN?$AA?$DN?$AA?$DO?$AAp?$AAD?$AAa?$AAt?$AAa?$AA?5?$AA?$CB?$AA?$DN?$AAN@ 00149980     caps.obj
 0002:000089c8       ??_7CChannel@@6B@          001499c8     channel.obj
 0002:000089cc       ??_C@_1BK@HEEOHIKH@?$AAC?$AAh?$AAa?$AAn?$AAn?$AAe?$AAl?$AAM?$AAu?$AAt?$AAe?$AAx?$AA?$AA@ 001499cc     channel.obj
 0002:000089e8       ??_C@_1FE@JCODGOLL@?$AAS?$AAe?$AAt?$AAC?$AAo?$AAm?$AAm?$AAT?$AAi?$AAm?$AAe?$AAo?$AAu?$AAt?$AAs?$AA?$CI?$AA?$CJ?$AA?5?$AAD?$AAa?$AAt?$AAa?$AA?5?$AAp?$AAo?$AAr?$AAt?$AA?5?$AAe?$AAr?$AAr?$AAo@ 001499e8     channel.obj
 0002:00008a40       ??_C@_1JM@JKCLEOIB@?$AAD?$AAe?$AAv?$AAi?$AAc?$AAe?$AAI?$AAO?$AAC?$AAt?$AAr?$AAl?$AA?5?$AAn?$AAO?$AAu?$AAt?$AAB?$AAu?$AAf?$AAS?$AAi?$AAz?$AAe?$AA?5?$AA?$DN?$AA?5?$AA?$CF?$AAd?$AA?5?$AAb?$AAu@ 00149a40     channel.obj
 0002:00008ae0       ??_C@_1EM@HHCPHIDC@?$AAW?$AAa?$AAi?$AAt?$AAC?$AAo?$AAm?$AAm?$AAE?$AAv?$AAe?$AAn?$AAt?$AA?5?$AAr?$AAe?$AAt?$AAu?$AAr?$AAn?$AAs?$AA?5?$AAw?$AAi?$AAn?$AAE?$AAr?$AAr?$AAo?$AAr?$AA?5?$AA?$DN@ 00149ae0     channel.obj
 0002:00008b30       ??_C@_1IE@GJFPDDGH@?$AAW?$AAa?$AAi?$AAt?$AAC?$AAo?$AAm?$AAE?$AAv?$AAe?$AAn?$AAt?$AA?5?$AAr?$AAe?$AAt?$AAu?$AAr?$AAn?$AAs?$AA?5?$AAT?$AAR?$AAU?$AAE?$AA?5?$AAw?$AAi?$AAt?$AAh?$AA?5?$AAc@ 00149b30     channel.obj
 0002:00008bb8       ??_C@_1EC@DAOPNPPB@?$AAR?$AAe?$AAa?$AAd?$AAF?$AAi?$AAl?$AAe?$AA?5?$AAr?$AAe?$AAt?$AAu?$AAr?$AAn?$AAs?$AA?5?$AAw?$AAi?$AAn?$AAE?$AAr?$AAr?$AAo?$AAr?$AA?5?$AA?$DN?$AA?5?$AA0?$AAx?$AA?$CF?$AAx@ 00149bb8     channel.obj
 0002:00008c00       ??_C@_1FK@FHNPFMOH@?$AAF?$AAa?$AAi?$AAl?$AA?5?$AAt?$AAo?$AA?5?$AAr?$AAu?$AAn?$AA?5?$AAR?$AAe?$AAc?$AAv?$AAT?$AAh?$AAr?$AAe?$AAa?$AAd?$AA?0?$AA?5?$AAp?$AAC?$AAh?$AAa?$AAn?$AAn?$AAe?$AAl@ 00149c00     channel.obj
 0002:00008c5c       ??_C@_1O@IHEKMJDI@?$AAC?$AAO?$AAM?$AA?$CF?$AAd?$AA?3?$AA?$AA@ 00149c5c     channel.obj
 0002:00008c6c       ??_C@_15GANGMFKL@?$AA?$CF?$AAs?$AA?$AA@ 00149c6c     channel.obj
 0002:00008c74       ??_C@_13EBCNDICG@?$AA?3?$AA?$AA@ 00149c74     channel.obj
 0002:00008c78       ??_C@_1GI@FKGOEPMF@?$AAA?$AAS?$AAS?$AAE?$AAR?$AAT?$AAI?$AAO?$AAN?$AA?5?$AAF?$AAA?$AAI?$AAL?$AAU?$AAR?$AAE?$AA?3?$AA?5?$AA?$DN?$AA?$DN?$AA?$DN?$AA?$DO?$AAp?$AAH?$AAa?$AAn?$AAd?$AAl?$AAe?$AA?9?$AA?$DO@ 00149c78     command.obj
 0002:00008ce0       ??_C@_1BM@FHKKBHCP@?$AA?4?$AA?2?$AAc?$AAo?$AAm?$AAm?$AAa?$AAn?$AAd?$AA?4?$AAc?$AAp?$AAp?$AA?$AA@ 00149ce0     command.obj
 0002:00008d30       ??_C@_1LO@MCDADINP@?$AAC?$AAC?$AAo?$AAm?$AAm?$AAa?$AAn?$AAd?$AA?3?$AA?3?$AA?$HO?$AAC?$AAC?$AAo?$AAm?$AAm?$AAa?$AAn?$AAd?$AA?$CI?$AA?$CJ?$AA?5?$AAT?$AAh?$AAi?$AAs?$AA?5?$AAc?$AAo?$AAm?$AAm?$AAa@ 00149d30     command.obj
 0002:00008df0       ??_C@_1LC@FPJHEFJF@?$AAA?$AAh?$AAa?$AA?$CB?$AA?5?$AAS?$AAe?$AAn?$AAd?$AAR?$AAe?$AAp?$AAo?$AAn?$AAs?$AAe?$AA?$CL?$AA?$CL?$AA?5?$AAf?$AAo?$AAr?$AA?5?$AAc?$AAm?$AAd?$AAI?$AAD?$AA?5?$AA?$DN?$AA?5?$AA?$CF@ 00149df0     command.obj
 0002:00008ea8       ??_C@_1JM@MIAFDJIK@?$AAA?$AAh?$AAa?$AA?$CB?$AA?5?$AAR?$AAI?$AAL?$AA?5?$AAc?$AAl?$AAi?$AAe?$AAn?$AAt?$AA?5?$AA?$CI?$AAp?$AAH?$AAa?$AAn?$AAd?$AAl?$AAe?$AA?5?$AA?$DN?$AA?5?$AA0?$AAx?$AA?$CF?$AAx?$AA?$CJ@ 00149ea8     command.obj
 0002:00008f48       ??_C@_1LC@JAEMIJMB@?$AAS?$AAe?$AAn?$AAd?$AAR?$AAe?$AAs?$AAp?$AAo?$AAn?$AAs?$AAe?$AA?5?$AA?$CI?$AAR?$AAe?$AAm?$AAo?$AAv?$AAe?$AA?5?$AAe?$AAx?$AAc?$AAe?$AAp?$AAt?$AAi?$AAo?$AAn?$AA?$CJ?$AA?$CB@ 00149f48     command.obj
 0002:00009000       ??_C@_1LK@ELFKFMH@?$AAA?$AAh?$AAa?$AA?$CB?$AA?5?$AAS?$AAe?$AAn?$AAd?$AAR?$AAe?$AAs?$AAp?$AAo?$AAn?$AAs?$AAe?$AA?5?$AAr?$AAe?$AAd?$AAu?$AAn?$AAd?$AAe?$AAn?$AAt?$AA?5?$AAf?$AAo?$AAr?$AA?5@ 0014a000     command.obj
 0002:00009174       ??_C@_01IHBHIGKO@?0?$AA@   0014a174     data.obj
 0002:00009178       ??_C@_02GMHACPFF@?$CFu?$AA@ 0014a178     data.obj
 0002:0000917c       ??_C@_1BG@EGGALAJL@?$AA?4?$AA?2?$AAd?$AAa?$AAt?$AAa?$AA?4?$AAc?$AAp?$AAp?$AA?$AA@ 0014a17c     data.obj
 0002:00009198       ??_C@_1EM@MIOLNEAM@?$AAA?$AAS?$AAS?$AAE?$AAR?$AAT?$AAI?$AAO?$AAN?$AA?5?$AAF?$AAA?$AAI?$AAL?$AAU?$AAR?$AAE?$AA?3?$AA?5?$AA?$DN?$AA?$DN?$AA?$DN?$AA?$DO?$AAN?$AAU?$AAL?$AAL?$AA?5?$AA?$CB?$AA?$DN?$AA?5?$AAs@ 0014a198     data.obj
 0002:000091e4       ??_C@_08NAEAAJKN@AT?$CLCRLP?$DN?$AA@ 0014a1e4     data.obj
 0002:000091f0       ??_C@_06LBIFBNIF@AT?$CLDS?$DN?$AA@ 0014a1f0     data.obj
 0002:000091f8       ??_C@_06JDJHKOA@AT?$CLES?$DN?$AA@ 0014a1f8     data.obj
 0002:00009200       ??_C@_1CO@PFFMHNAH@?$AAS?$AAo?$AAf?$AAt?$AAw?$AAa?$AAr?$AAe?$AA?2?$AAM?$AAi?$AAc?$AAr?$AAo?$AAs?$AAo?$AAf?$AAt?$AA?2?$AAR?$AAI?$AAL?$AA?$AA@ 0014a200     data.obj
 0002:00009470       ??_C@_0BM@PAPJHAGI@invalid?5map?1set?$DMT?$DO?5iterator?$AA@ 0014a470     DatERI.obj
 0002:00009520       ??_C@_0BE@JONHPENG@map?1set?$DMT?$DO?5too?5long?$AA@ 0014a520     DatERI.obj
 0002:0000961c       ??_C@_1DA@CGKFLEDF@?$AA2?$AA?9?$AAp?$AAR?$AAo?$AAa?$AAm?$AAI?$AAn?$AAd?$AA?9?$AA?$DO?$AAn?$AAI?$AAD?$AA?5?$AA?$DN?$AA?5?$AA?$CF?$AAd?$AA?5?$AA?$AN?$AA?6?$AA?$AA@ 0014a61c     DatERI.obj
 0002:0000964c       ??_C@_1DA@GAHHIBFB@?$AA1?$AA?9?$AAp?$AAR?$AAo?$AAa?$AAm?$AAI?$AAn?$AAd?$AA?9?$AA?$DO?$AAn?$AAI?$AAD?$AA?5?$AA?$DN?$AA?5?$AA?$CF?$AAd?$AA?5?$AA?$AN?$AA?6?$AA?$AA@ 0014a64c     DatERI.obj
 0002:0000967c       ??_C@_1DG@OMFIFHKA@?$AA2?$AA?9?$AAp?$AAC?$AAa?$AAl?$AAl?$AAP?$AAr?$AAo?$AAm?$AAp?$AAt?$AA?9?$AA?$DO?$AAn?$AAI?$AAD?$AA?5?$AA?$DN?$AA?5?$AA?$CF?$AAd?$AA?5?$AA?$AN?$AA?6?$AA?$AA@ 0014a67c     DatERI.obj
 0002:000096b4       ??_C@_1DG@OOLGKNHK@?$AA1?$AA?9?$AAp?$AAC?$AAa?$AAl?$AAl?$AAP?$AAr?$AAo?$AAm?$AAp?$AAt?$AA?9?$AA?$DO?$AAn?$AAI?$AAD?$AA?5?$AA?$DN?$AA?5?$AA?$CF?$AAd?$AA?5?$AA?$AN?$AA?6?$AA?$AA@ 0014a6b4     DatERI.obj
 0002:000096f0       ??_C@_1GO@LJICMMHB@?$AAS?$AAw?$AAi?$AAS?$AAt?$AAo?$AAp?$AAN?$AAo?$AAt?$AAi?$AAf?$AAy?$AA?$CI?$AAS?$AAW?$AAI?$AA_?$AAN?$AAO?$AAT?$AAI?$AAF?$AAY?$AA_?$AAP?$AAD?$AAS?$AAM?$AAP?$AAa?$AAr@ 0014a6f0     FakeResponse.obj
 0002:00009760       ??_C@_1GE@OBDECEGI@?$AAS?$AAw?$AAi?$AAN?$AAo?$AAt?$AAi?$AAf?$AAy?$AA?$CI?$AAS?$AAW?$AAI?$AA_?$AAN?$AAO?$AAT?$AAI?$AAF?$AAY?$AA_?$AAP?$AAD?$AAS?$AAM?$AAP?$AAa?$AAr?$AAa?$AAm?$AAN?$AAo@ 0014a760     FakeResponse.obj
 0002:000097c8       ??_C@_1GA@MEBCPOIB@?$AAS?$AAw?$AAi?$AAN?$AAo?$AAt?$AAi?$AAf?$AAy?$AA?$CI?$AAS?$AAW?$AAI?$AA_?$AAN?$AAO?$AAT?$AAI?$AAF?$AAY?$AA_?$AAH?$AAd?$AAr?$AA_?$AAP?$AAo?$AAw?$AAe?$AAr?$AAS?$AAa@ 0014a7c8     FakeResponse.obj
 0002:00009828       ??_C@_1GC@ELMPAJAN@?$AAS?$AAw?$AAi?$AAN?$AAo?$AAt?$AAi?$AAf?$AAy?$AA?$CI?$AAS?$AAW?$AAI?$AA_?$AAN?$AAO?$AAT?$AAI?$AAF?$AAY?$AA_?$AAH?$AAd?$AAr?$AA_?$AAP?$AAo?$AAw?$AAe?$AAr?$AAS?$AAa@ 0014a828     FakeResponse.obj
 0002:00009890       ??_C@_1FG@JNIEFLFM@?$AAS?$AAw?$AAi?$AAN?$AAo?$AAt?$AAi?$AAf?$AAy?$AA?$CI?$AAS?$AAW?$AAI?$AA_?$AAN?$AAO?$AAT?$AAI?$AAF?$AAY?$AA_?$AAH?$AAd?$AAr?$AA_?$AAH?$AAy?$AAb?$AAr?$AA_?$AAP?$AAr@ 0014a890     FakeResponse.obj
 0002:000098e8       ??_C@_1FG@BKMEHNDI@?$AAS?$AAw?$AAi?$AAN?$AAo?$AAt?$AAi?$AAf?$AAy?$AA?$CI?$AAS?$AAW?$AAI?$AA_?$AAN?$AAO?$AAT?$AAI?$AAF?$AAY?$AA_?$AAH?$AAd?$AAr?$AA_?$AAS?$AAr?$AAv?$AA_?$AAS?$AAt?$AAa@ 0014a8e8     FakeResponse.obj
 0002:00009940       ??_C@_1FK@NEJLJNGO@?$AAS?$AAw?$AAi?$AAN?$AAo?$AAt?$AAi?$AAf?$AAy?$AA?$CI?$AAS?$AAW?$AAI?$AA_?$AAN?$AAO?$AAT?$AAI?$AAF?$AAY?$AA_?$AAH?$AAd?$AAr?$AA_?$AAR?$AAo?$AAa?$AAm?$AA_?$AAS?$AAt@ 0014a940     FakeResponse.obj
 0002:000099a0       ??_C@_1EO@PGGCIPK@?$AAS?$AAw?$AAi?$AAN?$AAo?$AAt?$AAi?$AAf?$AAy?$AA?$CI?$AAS?$AAW?$AAI?$AA_?$AAN?$AAO?$AAT?$AAI?$AAF?$AAY?$AA_?$AAR?$AAs?$AAs?$AAi?$AA_?$AAE?$AAc?$AAi?$AAo?$AA?$CJ?$AA?5@ 0014a9a0     FakeResponse.obj
 0002:000099f0       ??_C@_1EM@EBCKDCEA@?$AAS?$AAw?$AAi?$AAN?$AAo?$AAt?$AAi?$AAf?$AAy?$AA?$CI?$AAS?$AAW?$AAI?$AA_?$AAN?$AAO?$AAT?$AAI?$AAF?$AAY?$AA_?$AAH?$AAd?$AAr?$AA_?$AAR?$AAs?$AAs?$AAi?$AA?$CJ?$AA?5?$AAF@ 0014a9f0     FakeResponse.obj
 0002:00009a40       ??_C@_1EE@CFLJNOEN@?$AAS?$AAw?$AAi?$AAN?$AAo?$AAt?$AAi?$AAf?$AAy?$AA?$CI?$AAS?$AAW?$AAI?$AA_?$AAN?$AAO?$AAT?$AAI?$AAF?$AAY?$AA_?$AAE?$AAc?$AAi?$AAo?$AA?$CJ?$AA?5?$AAF?$AAa?$AAi?$AAl?$AAe@ 0014aa40     FakeResponse.obj
 0002:00009a84       ??_C@_1DA@PHDOKMHP@?$AAS?$AAW?$AAI?$AA_?$AAN?$AAO?$AAT?$AAI?$AAF?$AAY?$AA_?$AAR?$AAs?$AAs?$AAi?$AA?5?$AAe?$AAn?$AAa?$AAb?$AAl?$AAe?$AAd?$AA?$AA@ 0014aa84     FakeResponse.obj
 0002:00009ab8       ??_C@_1EE@JCIELJDK@?$AAS?$AAw?$AAi?$AAN?$AAo?$AAt?$AAi?$AAf?$AAy?$AA?$CI?$AAS?$AAW?$AAI?$AA_?$AAN?$AAO?$AAT?$AAI?$AAF?$AAY?$AA_?$AAR?$AAs?$AAs?$AAi?$AA?$CJ?$AA?5?$AAF?$AAa?$AAi?$AAl?$AAe@ 0014aab8     FakeResponse.obj
 0002:00009b00       ??_C@_1EM@PAMJBOAF@?$AAS?$AAw?$AAi?$AAN?$AAo?$AAt?$AAi?$AAf?$AAy?$AA?$CI?$AAS?$AAW?$AAI?$AA_?$AAN?$AAO?$AAT?$AAI?$AAF?$AAY?$AA_?$AAE?$AA9?$AA1?$AA1?$AAM?$AAo?$AAd?$AAe?$AA?$CJ?$AA?5?$AAF@ 0014ab00     FakeResponse.obj
 0002:00009b50       ??_C@_1FC@NMGLBJDL@?$AAS?$AAw?$AAi?$AAN?$AAo?$AAt?$AAi?$AAf?$AAy?$AA?$CI?$AAS?$AAW?$AAI?$AA_?$AAN?$AAO?$AAT?$AAI?$AAF?$AAY?$AA_?$AAC?$AAa?$AAl?$AAl?$AAP?$AAr?$AAi?$AAv?$AAa?$AAc?$AAy@ 0014ab50     FakeResponse.obj
 0002:00009ba8       ??_C@_1GE@OBECEJLJ@?$AAS?$AAw?$AAi?$AAN?$AAo?$AAt?$AAi?$AAf?$AAy?$AA?$CI?$AAS?$AAW?$AAI?$AA_?$AAN?$AAO?$AAT?$AAI?$AAF?$AAY?$AA_?$AAC?$AAa?$AAl?$AAl?$AAE?$AAx?$AAt?$AAe?$AAn?$AAd?$AAe@ 0014aba8     FakeResponse.obj
 0002:00009c10       ??_C@_1FE@MKDICCBG@?$AAS?$AAw?$AAi?$AAN?$AAo?$AAt?$AAi?$AAf?$AAy?$AA?$CI?$AAS?$AAW?$AAI?$AA_?$AAN?$AAO?$AAT?$AAI?$AAF?$AAY?$AA_?$AAC?$AAa?$AAl?$AAl?$AAC?$AAa?$AAl?$AAl?$AAe?$AAr?$AAI@ 0014ac10     FakeResponse.obj
 0002:00009c68       ??_C@_1GI@FLEDOOEG@?$AAS?$AAw?$AAi?$AAN?$AAo?$AAt?$AAi?$AAf?$AAy?$AA?$CI?$AAS?$AAW?$AAI?$AA_?$AAN?$AAO?$AAT?$AAI?$AAF?$AAY?$AA_?$AAC?$AAa?$AAl?$AAl?$AAN?$AAo?$AAt?$AAi?$AAf?$AAi?$AAc@ 0014ac68     FakeResponse.obj
 0002:00009cd0       ??_C@_1FG@OOIEMAFG@?$AAS?$AAw?$AAi?$AAN?$AAo?$AAt?$AAi?$AAf?$AAy?$AA?$CI?$AAS?$AAW?$AAI?$AA_?$AAN?$AAO?$AAT?$AAI?$AAF?$AAY?$AA_?$AAS?$AAm?$AAs?$AAS?$AAe?$AAn?$AAd?$AAS?$AAt?$AAa?$AAt@ 0014acd0     FakeResponse.obj
 0002:00009d28       ??_C@_1EO@OHFEFLFL@?$AAS?$AAw?$AAi?$AAN?$AAo?$AAt?$AAi?$AAf?$AAy?$AA?$CI?$AAS?$AAW?$AAI?$AA_?$AAN?$AAO?$AAT?$AAI?$AAF?$AAY?$AA_?$AAS?$AAm?$AAs?$AAS?$AAt?$AAa?$AAt?$AAu?$AAs?$AA?$CJ?$AA?5@ 0014ad28     FakeResponse.obj
 0002:00009d78       ??_C@_1FI@NJCIAJGG@?$AAS?$AAw?$AAi?$AAN?$AAo?$AAt?$AAi?$AAf?$AAy?$AA?$CI?$AAS?$AAW?$AAI?$AA_?$AAN?$AAO?$AAT?$AAI?$AAF?$AAY?$AA_?$AAO?$AAM?$AAA?$AAD?$AAM?$AA_?$AAN?$AAI?$AA_?$AAA?$AAl@ 0014ad78     FakeResponse.obj
 0002:00009dd0       ??_C@_1FC@PJMAPKCN@?$AAS?$AAw?$AAi?$AAN?$AAo?$AAt?$AAi?$AAf?$AAy?$AA?$CI?$AAS?$AAW?$AAI?$AA_?$AAN?$AAO?$AAT?$AAI?$AAF?$AAY?$AA_?$AAO?$AAM?$AAA?$AAD?$AAM?$AA_?$AAS?$AAt?$AAa?$AAt?$AAe@ 0014add0     FakeResponse.obj
 0002:00009e28       ??_C@_1FI@PPAAHGOP@?$AAS?$AAw?$AAi?$AAN?$AAo?$AAt?$AAi?$AAf?$AAy?$AA?$CI?$AAS?$AAW?$AAI?$AA_?$AAN?$AAO?$AAT?$AAI?$AAF?$AAY?$AA_?$AAP?$AAk?$AAt?$AAS?$AAe?$AAs?$AAs?$AAi?$AAo?$AAn?$AAC@ 0014ae28     FakeResponse.obj
 0002:00009e80       ??_C@_1FC@FPCLHPIH@?$AAS?$AAw?$AAi?$AAN?$AAo?$AAt?$AAi?$AAf?$AAy?$AA?$CI?$AAS?$AAW?$AAI?$AA_?$AAN?$AAO?$AAT?$AAI?$AAF?$AAY?$AA_?$AAS?$AAe?$AAr?$AAv?$AAi?$AAc?$AAe?$AAI?$AAc?$AAo?$AAn@ 0014ae80     FakeResponse.obj
 0002:00009ed8       ??_C@_1FK@IDAJMJPM@?$AAS?$AAw?$AAi?$AAN?$AAo?$AAt?$AAi?$AAf?$AAy?$AA?$CI?$AAS?$AAW?$AAI?$AA_?$AAN?$AAO?$AAT?$AAI?$AAF?$AAY?$AA_?$AAG?$AAs?$AAm?$AAS?$AAy?$AAs?$AAt?$AAe?$AAm?$AAS?$AAt@ 0014aed8     FakeResponse.obj
 0002:00009f38       ??_C@_1FG@JOKNKDEJ@?$AAS?$AAw?$AAi?$AAN?$AAo?$AAt?$AAi?$AAf?$AAy?$AA?$CI?$AAS?$AAW?$AAI?$AA_?$AAN?$AAO?$AAT?$AAI?$AAF?$AAY?$AA_?$AAP?$AAl?$AAm?$AAn?$AAA?$AAv?$AAa?$AAi?$AAl?$AAa?$AAb@ 0014af38     FakeResponse.obj
 0002:00009f90       ??_C@_1FK@CIDEBECM@?$AAS?$AAw?$AAi?$AAN?$AAo?$AAt?$AAi?$AAf?$AAy?$AA?$CI?$AAS?$AAW?$AAI?$AA_?$AAN?$AAO?$AAT?$AAI?$AAF?$AAY?$AA_?$AAA?$AAi?$AAr?$AAS?$AAe?$AAr?$AAv?$AAe?$AAr?$AAC?$AAh@ 0014af90     FakeResponse.obj
 0002:00009ff0       ??_C@_1FC@BIKKABHO@?$AAS?$AAw?$AAi?$AAN?$AAo?$AAt?$AAi?$AAf?$AAy?$AA?$CI?$AAS?$AAW?$AAI?$AA_?$AAN?$AAO?$AAT?$AAI?$AAF?$AAY?$AA_?$AAD?$AAe?$AAv?$AAi?$AAc?$AAe?$AA_?$AAT?$AAi?$AAm?$AAe@ 0014aff0     FakeResponse.obj
 0002:0000a048       ??_C@_1FG@NIFANPHI@?$AAS?$AAw?$AAi?$AAN?$AAo?$AAt?$AAi?$AAf?$AAy?$AA?$CI?$AAS?$AAW?$AAI?$AA_?$AAN?$AAO?$AAT?$AAI?$AAF?$AAY?$AA_?$AAP?$AAo?$AAw?$AAe?$AAr?$AAS?$AAa?$AAv?$AAe?$AAE?$AAx@ 0014b048     FakeResponse.obj
 0002:0000a0a0       ??_C@_1FI@MCNIFPOF@?$AAS?$AAw?$AAi?$AAN?$AAo?$AAt?$AAi?$AAf?$AAy?$AA?$CI?$AAS?$AAW?$AAI?$AA_?$AAN?$AAO?$AAT?$AAI?$AAF?$AAY?$AA_?$AAP?$AAo?$AAw?$AAe?$AAr?$AAS?$AAa?$AAv?$AAe?$AAE?$AAn@ 0014b0a0     FakeResponse.obj
 0002:0000a0f8       ??_C@_1FM@IJCNJEEO@?$AAS?$AAw?$AAi?$AAN?$AAo?$AAt?$AAi?$AAf?$AAy?$AA?$CI?$AAS?$AAW?$AAI?$AA_?$AAN?$AAO?$AAT?$AAI?$AAF?$AAY?$AA_?$AAE?$AAx?$AAc?$AAe?$AAs?$AAs?$AAS?$AAP?$AAC?$AAF?$AAa@ 0014b0f8     FakeResponse.obj
 0002:0000a158       ??_C@_1FG@IEEJNODA@?$AAS?$AAw?$AAi?$AAN?$AAo?$AAt?$AAi?$AAf?$AAy?$AA?$CI?$AAS?$AAW?$AAI?$AA_?$AAN?$AAO?$AAT?$AAI?$AAF?$AAY?$AA_?$AAR?$AAo?$AAa?$AAm?$AAi?$AAn?$AAg?$AAS?$AAt?$AAa?$AAt@ 0014b158     FakeResponse.obj
 0002:0000a1b0       ??_C@_1CG@FMFDONOL@?$AA?4?$AA?2?$AAF?$AAa?$AAk?$AAe?$AAR?$AAe?$AAs?$AAp?$AAo?$AAn?$AAs?$AAe?$AA?4?$AAc?$AAp?$AAp?$AA?$AA@ 0014b1b0     FakeResponse.obj
 0002:0000a1d8       ??_C@_1FO@OKBMGKBN@?$AAS?$AAw?$AAi?$AAN?$AAo?$AAt?$AAi?$AAf?$AAy?$AA?$CI?$AAS?$AAW?$AAI?$AA_?$AAN?$AAO?$AAT?$AAI?$AAF?$AAY?$AA_?$AAS?$AAe?$AAr?$AAv?$AAi?$AAc?$AAe?$AAI?$AAn?$AAd?$AAi@ 0014b1d8     FakeResponse.obj
 0002:0000a238       ??_C@_1EO@PJKKADKC@?$AAE?$AAn?$AAa?$AAb?$AAl?$AAe?$AAT?$AAe?$AAc?$AAh?$AAH?$AAD?$AAR?$AAN?$AAo?$AAt?$AAi?$AAf?$AAi?$AAc?$AAa?$AAt?$AAi?$AAo?$AAn?$AAs?$AA?5?$AAu?$AAn?$AAs?$AAu?$AAp@ 0014b238     FakeResponse.obj
 0002:0000a2bc       ??_C@_1DO@MJNLKBEJ@?$AAM?$AAo?$AAd?$AAe?$AAm?$AA?5?$AAi?$AAs?$AA?5?$AAn?$AAo?$AAt?$AA?5?$AAr?$AAe?$AAa?$AAd?$AAy?$AA?$CB?$AA?5?$AAF?$AAa?$AAi?$AAl?$AAO?$AAn?$AAI?$AAn?$AAi?$AAt?$AA?$AA@ 0014b2bc     FakeResponse.obj
 0002:0000a300       ??_C@_1FE@HLEJDPGF@?$AAO?$AAu?$AAr?$AA?5?$AAD?$AAE?$AAV?$AAI?$AAC?$AAE?$AA?5?$AAA?$AAR?$AAR?$AAI?$AAV?$AAE?$AAS?$AA?4?$AA?5?$AAC?$AAa?$AAl?$AAl?$AA?5?$AAI?$AAn?$AAi?$AAt?$AAi?$AAa?$AAl@ 0014b300     FakeResponse.obj
 0002:0000a358       ??_C@_1EC@BGBPKHNO@?$AAC?$AAa?$AAn?$AAc?$AAe?$AAl?$AAE?$AAv?$AAe?$AAn?$AAt?$AA?5?$AAs?$AAt?$AAo?$AAp?$AAs?$AA?5?$AAI?$AAn?$AAi?$AAt?$AAT?$AAh?$AAr?$AAe?$AAa?$AAd?$AAP?$AAr?$AAo?$AAc@ 0014b358     FakeResponse.obj
 0002:0000a3a0       ??_C@_1GK@ENKFFFPJ@?$AAw?$AAa?$AAi?$AAt?$AAO?$AAb?$AAj?$AAe?$AAc?$AAt?$AAR?$AAe?$AAs?$AAu?$AAl?$AAt?$AA?5?$AA?$DN?$AA?5?$AA?$CF?$AAd?$AA?5?$AAs?$AAt?$AAo?$AAp?$AAs?$AA?5?$AAI?$AAn?$AAi?$AAt@ 0014b3a0     FakeResponse.obj
 0002:0000a410       ??_C@_1HC@DOBDFIMD@?$AAM?$AAo?$AAd?$AAe?$AAm?$AA?5?$AAs?$AAt?$AAi?$AAl?$AAl?$AA?5?$AAI?$AAN?$AA?5?$AAa?$AAt?$AA?5?$AAI?$AAn?$AAi?$AAt?$AAT?$AAh?$AAr?$AAe?$AAa?$AAd?$AAP?$AAr?$AAo?$AAc@ 0014b410     FakeResponse.obj
 0002:0000a488       ??_C@_1EK@FNPFGGOL@?$AAA?$AAS?$AAS?$AAE?$AAR?$AAT?$AAI?$AAO?$AAN?$AA?5?$AAF?$AAA?$AAI?$AAL?$AAU?$AAR?$AAE?$AA?3?$AA?5?$AA?$DN?$AA?$DN?$AA?$DN?$AA?$DO?$AAr?$AAp?$AAR?$AAs?$AAp?$AA?5?$AA?$CB?$AA?$DN?$AA?5@ 0014b488     FakeResponse.obj
 0002:0000a4d8       ??_C@_1EK@GPNFAKEM@?$AAA?$AAS?$AAS?$AAE?$AAR?$AAT?$AAI?$AAO?$AAN?$AA?5?$AAF?$AAA?$AAI?$AAL?$AAU?$AAR?$AAE?$AA?3?$AA?5?$AA?$DN?$AA?$DN?$AA?$DN?$AA?$DO?$AAr?$AAp?$AAC?$AAm?$AAd?$AA?5?$AA?$CB?$AA?$DN?$AA?5@ 0014b4d8     FakeResponse.obj
 0002:0000a528       ??_C@_1FE@KMFGMDEF@?$AAU?$AAn?$AAh?$AAa?$AAn?$AAd?$AAl?$AAe?$AAd?$AA?5?$AAs?$AAi?$AAg?$AAn?$AAa?$AAl?$AA?5?$AA?$DN?$AA?5?$AA0?$AAx?$AA?$CF?$AAx?$AA?0?$AA?5?$AAl?$AAa?$AAs?$AAt?$AAE?$AAr?$AAr@ 0014b528     FakeResponse.obj
 0002:0000a5bc       ??_C@_0BB@MOGOBHAF@list?$DMT?$DO?5too?5long?$AA@ 0014b5bc     FakeResponse.obj
 0002:0000a610       ??_C@_1GC@DMCBKNID@?$AAR?$AAI?$AAL?$AA_?$AAR?$AAE?$AAS?$AAU?$AAL?$AAT?$AA_?$AAX?$AA?5?$AAn?$AAo?$AAt?$AA?5?$AAs?$AAe?$AAt?$AA?5?$AAf?$AAo?$AAr?$AA?5?$AAA?$AAP?$AAI?$AAI?$AAD?$AA?5?$AA?$DN@ 0014b610     FakeResponse.obj
 0002:0000a6b0       ??_C@_1EI@HMGKPBJ@?$AAA?$AAS?$AAS?$AAE?$AAR?$AAT?$AAI?$AAO?$AAN?$AA?5?$AAF?$AAA?$AAI?$AAL?$AAU?$AAR?$AAE?$AA?3?$AA?5?$AA?$DN?$AA?$DN?$AA?$DN?$AA?$DO?$AAN?$AAU?$AAL?$AAL?$AA?5?$AA?$DN?$AA?$DN?$AA?5?$AAp@ 0014b6b0     FakeResponse.obj
 0002:0000a6f8       ??_C@_1EK@PEDLHPLJ@?$AAA?$AAS?$AAS?$AAE?$AAR?$AAT?$AAI?$AAO?$AAN?$AA?5?$AAF?$AAA?$AAI?$AAL?$AAU?$AAR?$AAE?$AA?3?$AA?5?$AA?$DN?$AA?$DN?$AA?$DN?$AA?$DO?$AAN?$AAU?$AAL?$AAL?$AA?5?$AA?$DN?$AA?$DN?$AA?5?$AAr@ 0014b6f8     FakeResponse.obj
 0002:0000a748       ??_C@_1HA@IIAMPOLA@?$AAH?$AAa?$AAn?$AAd?$AAl?$AAe?$AAR?$AAs?$AAp?$AA?5?$AA?3?$AA?5?$AAU?$AAn?$AAa?$AAb?$AAl?$AAe?$AA?5?$AAt?$AAo?$AA?5?$AAH?$AAa?$AAn?$AAd?$AAl?$AAe?$AA?5?$AAR?$AAe?$AAs@ 0014b748     FakeResponse.obj
 0002:0000a7b8       ??_C@_1IO@COLNIMCG@?$AAE?$AAx?$AAe?$AAc?$AAu?$AAt?$AAe?$AAC?$AAo?$AAm?$AAm?$AAa?$AAn?$AAd?$AA?5?$AA?3?$AA?5?$AAF?$AAa?$AAi?$AAl?$AAe?$AAd?$AA?5?$AAt?$AAo?$AA?5?$AAe?$AAx?$AAe?$AAc?$AAu@ 0014b7b8     FakeResponse.obj
 0002:0000a848       ??_C@_1KK@MDBJPCHO@?$AAE?$AAx?$AAe?$AAc?$AAu?$AAt?$AAe?$AAC?$AAo?$AAm?$AAm?$AAa?$AAn?$AAd?$AA?5?$AA?3?$AA?5?$AAF?$AAa?$AAi?$AAl?$AAe?$AAd?$AA?5?$AAt?$AAo?$AA?5?$AAe?$AAx?$AAe?$AAc?$AAu@ 0014b848     FakeResponse.obj
 0002:0000a8f8       ??_C@_1IM@NBBCMIKG@?$AAE?$AAx?$AAe?$AAc?$AAu?$AAt?$AAe?$AAC?$AAo?$AAm?$AAm?$AAa?$AAn?$AAd?$AA?5?$AA?3?$AA?5?$AAF?$AAa?$AAi?$AAl?$AAe?$AAd?$AA?5?$AAt?$AAo?$AA?5?$AAe?$AAx?$AAe?$AAc?$AAu@ 0014b8f8     FakeResponse.obj
 0002:0000a984       ??_C@_1BM@CKLAAKNF@?$AAO?$AAu?$AAt?$AA?5?$AAo?$AAf?$AA?5?$AAm?$AAe?$AAm?$AAo?$AAr?$AAy?$AA?$AA@ 0014b984     FakeResponse.obj
 0002:0000a9a0       ??_C@_1KE@DMNPMKBK@?$AAP?$AAl?$AAa?$AAc?$AAe?$AA?5?$AAt?$AAh?$AAe?$AA?5?$AAA?$AAP?$AAI?$AAI?$AAD?$AA_?$AAS?$AAE?$AAT?$AAE?$AAQ?$AAU?$AAI?$AAP?$AAM?$AAE?$AAN?$AAT?$AAS?$AAT?$AAA?$AAT@ 0014b9a0     FakeResponse.obj
 0002:0000aa48       ??_C@_1KI@NFPDHMML@?$AAE?$AAx?$AAe?$AAc?$AAu?$AAt?$AAe?$AAC?$AAo?$AAm?$AAm?$AAa?$AAn?$AAd?$AA?5?$AAo?$AAf?$AA?5?$AAA?$AAP?$AAI?$AAI?$AAD?$AA?5?$AA?$DN?$AA?5?$AA?$CF?$AAd?$AA?0?$AA?5?$AAc?$AAm@ 0014ba48     FakeResponse.obj
 0002:0000aaf0       ??_C@_1IE@OKPIEGGI@?$AAR?$AAI?$AAL?$AA?5?$AAs?$AAu?$AAs?$AAp?$AAe?$AAn?$AAd?$AAe?$AAd?$AA?5?$AA?$CI?$AAg?$AAL?$AAa?$AAs?$AAt?$AAD?$AAe?$AAv?$AAi?$AAc?$AAe?$AAD?$AAx?$AA?5?$AA?$DN?$AA?5?$AA?$CF@ 0014baf0     FakeResponse.obj
 0002:0000ab74       ??_C@_02MNFKMMLG@CG?$AA@   0014bb74     gprs.obj
 0002:0000ab78       ??_C@_02KJDGAJLC@CC?$AA@   0014bb78     gprs.obj
 0002:0000ab7c       ??_C@_01GFHCPBMG@C?$AA@    0014bb7c     gprs.obj
 0002:0000ab80       ??_C@_01HMGJMAIH@B?$AA@    0014bb80     gprs.obj
 0002:0000ab84       ??_C@_01FHEEJDEE@A?$AA@    0014bb84     gprs.obj
 0002:0000ab88       ??_C@_03FFNMPEOG@X25?$AA@  0014bb88     gprs.obj
 0002:0000ab8c       ??_C@_03MDLBFMKF@PPP?$AA@  0014bb8c     gprs.obj
 0002:0000ab90       ??_C@_03PAPLECLH@PAD?$AA@  0014bb90     gprs.obj
 0002:0000ab94       ??_C@_04HIBGFPH@NULL?$AA@  0014bb94     gprs.obj
 0002:0000ad70       ??_C@_1BG@PMEIPKCD@?$AA?4?$AA?2?$AAg?$AAp?$AAr?$AAs?$AA?4?$AAc?$AAp?$AAp?$AA?$AA@ 0014bd70     gprs.obj
 0002:0000ad88       ??_C@_08LEBGIKFD@AT?$CFs?$DN?$CFu?0?$AA@ 0014bd88     gprs.obj
 0002:0000ad94       ??_C@_07OIPJAJMK@?$CLCGQREQ?$AA@ 0014bd94     gprs.obj
 0002:0000ad9c       ??_C@_07CEMDLJPJ@?$CLCGQMIN?$AA@ 0014bd9c     gprs.obj
 0002:0000ada4       ??_C@_08DIIJJPLA@AT?$CFs?$DN?$CFu?$AN?$AA@ 0014bda4     gprs.obj
 0002:0000adb0       ??_C@_0N@EJFFPICF@AT?$CLCGATT?$DN?$CFu?$AN?$AA@ 0014bdb0     gprs.obj
 0002:0000ae18       ??_C@_1FG@PJFBHKIC@?$AAA?$AAP?$AAI?$AAI?$AAD?$AA_?$AAE?$AAN?$AAT?$AAE?$AAR?$AAG?$AAP?$AAR?$AAS?$AAD?$AAA?$AAT?$AAA?$AAM?$AAO?$AAD?$AAE?$AA?5?$AAF?$AAa?$AAi?$AAl?$AA?5?$AAt?$AAo?$AA?5@ 0014be18     gprs.obj
 0002:0000ae70       ??_C@_02IPBLKABJ@?$CD?$AN?$AA@ 0014be70     gprs.obj
 0002:0000ae74       ??_C@_09JONDINHO@ATD?$CK99?$CK?$CK?$CK?$AA@ 0014be74     gprs.obj
 0002:0000ae80       ??_C@_0P@IMFDNHHB@AT?$CLCGPADDR?$DN?$CFu?$AN?$AA@ 0014be80     gprs.obj
 0002:0000ae90       ??_C@_03FIJBDJNN@?0?$CFu?$AA@ 0014be90     gprs.obj
 0002:0000ae94       ??_C@_04OEDFLLKD@?$CC?$CFs?$CC?$AA@ 0014be94     gprs.obj
 0002:0000ae9c       ??_C@_0N@BLGBBOPO@AT?$CLCGANS?$DN?$CFu?0?$AA@ 0014be9c     gprs.obj
 0002:0000aeb0       ??_C@_1FM@PHPKMKEN@?$AAR?$AAI?$AAL?$AAD?$AAr?$AAv?$AA_?$AAS?$AAe?$AAn?$AAd?$AAS?$AAi?$AAm?$AAC?$AAm?$AAd?$AA?3?$AA?5?$AAL?$AAe?$AAn?$AAg?$AAt?$AAh?$AA?5?$AAo?$AAf?$AA?5?$AAt?$AAh?$AAe@ 0014beb0     gprs.obj
 0002:0000af10       ??_C@_1OC@LIAPPLBN@?$AAR?$AAI?$AAL?$AAD?$AAr?$AAv?$AA_?$AAS?$AAe?$AAn?$AAd?$AAR?$AAe?$AAs?$AAt?$AAr?$AAi?$AAc?$AAt?$AAe?$AAd?$AAS?$AAi?$AAm?$AAC?$AAm?$AAd?$AA?3?$AA?5?$AAd?$AAw?$AAP@ 0014bf10     gprs.obj
 0002:0000aff4       ??_C@_0BB@FMDCNBOF@AT?$CLCGCLASS?$DN?$CC?$CFs?$CC?$AN?$AA@ 0014bff4     gprs.obj
 0002:0000b008       ??_C@_0N@JIIICHNG@AT?$CLCGSMS?$DN?$CFu?$AN?$AA@ 0014c008     gprs.obj
 0002:0000b018       ??_C@_1IO@CFJLAAL@?$AAA?$AAS?$AAS?$AAE?$AAR?$AAT?$AAI?$AAO?$AAN?$AA?5?$AAF?$AAA?$AAI?$AAL?$AAU?$AAR?$AAE?$AA?3?$AA?5?$AA?$DN?$AA?$DN?$AA?$DN?$AA?$DO?$AAm?$AA_?$AAd?$AAw?$AAS?$AAw?$AAi?$AAW?$AAi@ 0014c018     gprs.obj
 0002:0000b0a8       ??_C@_1DK@ODIIFDJH@?$AAD?$AAe?$AAl?$AAe?$AAt?$AAe?$AAG?$AAP?$AAR?$AAS?$AAC?$AAo?$AAn?$AAt?$AAe?$AAx?$AAt?$AA?5?$AAu?$AAn?$AAs?$AAp?$AAp?$AAo?$AAr?$AAt?$AAe?$AAd?$AA?$AA@ 0014c0a8     gprs.obj
 0002:0000b0e8       ??_C@_1IA@KOOLNGCI@?$AAS?$AAe?$AAt?$AAG?$AAP?$AAR?$AAS?$AAC?$AAo?$AAn?$AAt?$AAe?$AAx?$AAt?$AAA?$AAc?$AAt?$AAi?$AAv?$AAa?$AAt?$AAe?$AAd?$AA?9?$AA?$DO?$AAS?$AAw?$AAi?$AAA?$AAc?$AAt?$AAi@ 0014c0e8     gprs.obj
 0002:0000b168       ??_C@_1GK@FLJPAMMA@?$AAS?$AAe?$AAn?$AAd?$AAS?$AAi?$AAm?$AAC?$AAm?$AAd?$AA?3?$AA?3?$AAE?$AAR?$AAR?$AAO?$AAR?$AA?5?$AAc?$AAo?$AAm?$AAm?$AAa?$AAn?$AAd?$AA?5?$AAw?$AAi?$AAt?$AAh?$AA?5?$AAl@ 0014c168     gprs.obj
 0002:0000b1d8       ??_C@_1IA@IMMDJIB@?$AAS?$AAe?$AAn?$AAd?$AAS?$AAi?$AAm?$AAC?$AAm?$AAd?$AA?3?$AA?3?$AAE?$AAR?$AAR?$AAO?$AAR?$AA?5?$AAS?$AAw?$AAi?$AAS?$AAe?$AAn?$AAd?$AAG?$AAe?$AAn?$AAe?$AAr?$AAi?$AAc@ 0014c1d8     gprs.obj
 0002:0000b258       ??_C@_1HA@HODKDLJD@?$AAS?$AAe?$AAn?$AAd?$AAS?$AAi?$AAm?$AAC?$AAm?$AAd?$AA?3?$AA?3?$AAS?$AAw?$AAi?$AAS?$AAe?$AAn?$AAd?$AAG?$AAe?$AAn?$AAe?$AAr?$AAi?$AAc?$AAS?$AAi?$AAm?$AAC?$AAo?$AAm@ 0014c258     gprs.obj
 0002:0000b2c8       ??_C@_1FO@JLBCMGAL@?$AAS?$AAw?$AAi?$AAR?$AAe?$AAs?$AAt?$AAr?$AAi?$AAc?$AAt?$AAe?$AAd?$AAS?$AAi?$AAm?$AAC?$AAm?$AAd?$AA?5?$AAd?$AAi?$AAd?$AA?5?$AAn?$AAo?$AAt?$AA?5?$AAr?$AAe?$AAt?$AAu@ 0014c2c8     gprs.obj
 0002:0000b328       ??_C@_1GE@JJBKFBKH@?$AAS?$AAw?$AAi?$AAR?$AAe?$AAs?$AAt?$AAr?$AAi?$AAc?$AAt?$AAe?$AAd?$AAS?$AAi?$AAm?$AAC?$AAm?$AAd?$AAR?$AAs?$AAp?$AA?4?$AAd?$AAw?$AAE?$AAx?$AAt?$AAr?$AAa?$AAP?$AAa@ 0014c328     gprs.obj
 0002:0000b38c       ??_C@_1DI@DAGIMKEA@?$AAm?$AAp?$AAF?$AAn?$AAS?$AAw?$AAi?$AAG?$AAe?$AAt?$AAP?$AAi?$AAn?$AAS?$AAt?$AAa?$AAt?$AAu?$AAs?$AA?5?$AAi?$AAs?$AA?5?$AAN?$AAU?$AAL?$AAL?$AA?$AA@ 0014c38c     gprs.obj
 0002:0000b3c8       ??_C@_1FG@EDACBJFO@?$AAS?$AAw?$AAi?$AAS?$AAe?$AAn?$AAd?$AAR?$AAe?$AAs?$AAt?$AAr?$AAi?$AAc?$AAt?$AAe?$AAd?$AAS?$AAI?$AAM?$AAC?$AAm?$AAd?$AA?5?$AAF?$AAA?$AAI?$AAL?$AAE?$AAD?$AA?0?$AA?5@ 0014c3c8     gprs.obj
 0002:0000b420       ??_C@_1FM@GIFNGKMB@?$AAS?$AAe?$AAn?$AAd?$AAR?$AAe?$AAs?$AAt?$AAr?$AAi?$AAc?$AAt?$AAe?$AAd?$AAS?$AAi?$AAm?$AAC?$AAm?$AAd?$AA?5?$AAc?$AAa?$AAl?$AAl?$AAe?$AAd?$AA?5?$AAw?$AAi?$AAt?$AAh@ 0014c420     gprs.obj
 0002:0000b480       ??_C@_1IA@EEKFNKAH@?$AAS?$AAw?$AAi?$AAG?$AAe?$AAt?$AAS?$AAI?$AAM?$AAR?$AAe?$AAc?$AAo?$AAr?$AAd?$AAS?$AAt?$AAa?$AAt?$AAu?$AAs?$AA?5?$AAf?$AAa?$AAi?$AAl?$AAs?$AA?0?$AA?5?$AAR?$AAe?$AAt@ 0014c480     gprs.obj
 0002:0000b500       ??_C@_1FI@FENEHLFH@?$AAG?$AAe?$AAt?$AAS?$AAi?$AAm?$AAR?$AAe?$AAc?$AAo?$AAr?$AAd?$AAS?$AAt?$AAa?$AAt?$AAu?$AAs?$AA?5?$AAc?$AAa?$AAl?$AAl?$AAe?$AAd?$AA?5?$AAw?$AAi?$AAt?$AAh?$AA?5?$AAf@ 0014c500     gprs.obj
 0002:0000b558       ??_C@_1GA@JHJLLNH@?$AAF?$AAa?$AAi?$AAl?$AA?5?$AAt?$AAo?$AA?5?$AAo?$AAb?$AAt?$AAa?$AAi?$AAn?$AA?5?$AAd?$AAw?$AAP?$AAr?$AAo?$AAt?$AAo?$AAc?$AAo?$AAl?$AAT?$AAy?$AAp?$AAe?$AA?0?$AA?5?$AAw@ 0014c558     gprs.obj
 0002:0000b5b8       ??_C@_1EI@CJINFDBB@?$AAF?$AAa?$AAi?$AAl?$AA?5?$AAS?$AAw?$AAi?$AAG?$AAe?$AAt?$AAG?$AAS?$AAM?$AAP?$AAr?$AAo?$AAf?$AAi?$AAl?$AAe?$AAB?$AAa?$AAs?$AAi?$AAc?$AA?0?$AA?5?$AAr?$AAc?$AA?5?$AA?$DN@ 0014c5b8     gprs.obj
 0002:0000b600       ??_C@_1MC@DEICCILN@?$AAG?$AAP?$AAR?$AAS?$AAA?$AAc?$AAt?$AAi?$AAv?$AAa?$AAt?$AAe?$AA?5?$AA?$CI?$AAd?$AAw?$AAC?$AAo?$AAn?$AAt?$AAe?$AAx?$AAt?$AA?5?$AA?$DN?$AA?5?$AA?$CF?$AAd?$AA?0?$AA?5?$AAb?$AAA@ 0014c600     gprs.obj
 0002:0000b6c8       ??_C@_1EC@EMNBEADF@?$AAF?$AAa?$AAi?$AAl?$AA?5?$AAS?$AAw?$AAi?$AAA?$AAc?$AAt?$AAi?$AAv?$AAa?$AAt?$AAe?$AAP?$AAr?$AAo?$AAf?$AAi?$AAl?$AAe?$AA?0?$AA?5?$AAr?$AAc?$AA?5?$AA?$DN?$AA?5?$AA?$CF?$AAd@ 0014c6c8     gprs.obj
 0002:0000b710       ??_C@_1IE@LPMCJJEG@?$AAS?$AAe?$AAt?$AAG?$AAP?$AAR?$AAS?$AAC?$AAo?$AAn?$AAt?$AAe?$AAx?$AAt?$AA?5?$AAc?$AAa?$AAl?$AAl?$AAe?$AAd?$AA?5?$AAw?$AAh?$AAi?$AAl?$AAe?$AA?5?$AAt?$AAe?$AAc?$AAh@ 0014c710     gprs.obj
 0002:0000b798       ??_C@_1EI@FNPJCHHM@?$AAF?$AAa?$AAi?$AAl?$AA?5?$AAS?$AAw?$AAi?$AAS?$AAe?$AAt?$AAG?$AAS?$AAM?$AAP?$AAr?$AAo?$AAf?$AAi?$AAl?$AAe?$AAB?$AAa?$AAs?$AAi?$AAc?$AA?0?$AA?5?$AAr?$AAc?$AA?5?$AA?$DN@ 0014c798     gprs.obj
 0002:0000b7e0       ??_C@_1JK@KJMKHFKH@?$AAI?$AAS?$AAS?$AAU?$AAE?$AA?3?$AA?5?$AAR?$AAI?$AAL?$AAG?$AAP?$AAR?$AAS?$AAC?$AAO?$AAN?$AAT?$AAE?$AAX?$AAT?$AA?5?$AAN?$AAe?$AAe?$AAd?$AA?5?$AAt?$AAo?$AA?5?$AAF?$AAi@ 0014c7e0     gprs.obj
 0002:0000b880       ??_C@_1FE@OFLAGLLJ@?$AAF?$AAa?$AAi?$AAl?$AA?5?$AAt?$AAo?$AA?5?$AAo?$AAb?$AAt?$AAa?$AAi?$AAn?$AA?5?$AAP?$AAD?$AAP?$AA?5?$AAt?$AAy?$AAp?$AAe?$AA?0?$AA?5?$AAw?$AAh?$AAa?$AAt?$AA?5?$AAi?$AAs@ 0014c880     gprs.obj
 0002:0000b8d4       ??_C@_1DE@EMJBEPGN@?$AA?2?$AAS?$AAt?$AAr?$AAi?$AAn?$AAg?$AAF?$AAi?$AAl?$AAe?$AAI?$AAn?$AAf?$AAo?$AA?2?$AA0?$AA4?$AA0?$AA9?$AA0?$AA4?$AAB?$AA0?$AA?2?$AA?$AA@ 0014c8d4     misc.obj
 0002:0000b908       ??_C@_1BG@EEIGADGG@?$AA?4?$AA?2?$AAm?$AAi?$AAs?$AAc?$AA?4?$AAc?$AAp?$AAp?$AA?$AA@ 0014c908     misc.obj
 0002:0000b920       ??_C@_1GA@GMEPHDIK@?$AAT?$AAh?$AAe?$AA?5?$AAm?$AAo?$AAd?$AAe?$AAm?$AA?5?$AAs?$AAh?$AAo?$AAu?$AAl?$AAd?$AA?5?$AAf?$AAo?$AAr?$AAc?$AAe?$AA?5?$AAd?$AAa?$AAt?$AAa?$AA?5?$AAc?$AAa?$AAl?$AAl@ 0014c920     misc.obj
 0002:0000b980       ??_C@_1FE@FEMPENEA@?$AAR?$AAI?$AAL?$AAD?$AAr?$AAv?$AA_?$AAG?$AAe?$AAt?$AAE?$AAq?$AAu?$AAi?$AAp?$AAm?$AAe?$AAn?$AAt?$AAS?$AAt?$AAa?$AAt?$AAe?$AA?0?$AA?5?$AAQ?$AAu?$AAe?$AAu?$AAe?$AAC@ 0014c980     misc.obj
 0002:0000b9d8       ??_C@_1FC@BLGLIFKB@?$AAR?$AAI?$AAL?$AAD?$AAr?$AAv?$AA_?$AAG?$AAe?$AAt?$AAE?$AAq?$AAu?$AAi?$AAp?$AAm?$AAe?$AAn?$AAt?$AAS?$AAt?$AAa?$AAt?$AAe?$AA?0?$AA?5?$AAp?$AAH?$AAa?$AAn?$AAd?$AAl@ 0014c9d8     misc.obj
 0002:0000ba2c       ??_C@_1DC@KGLEAOJN@?$AAR?$AAI?$AAL?$AAD?$AAr?$AAv?$AA_?$AAG?$AAe?$AAt?$AAE?$AAq?$AAu?$AAi?$AAp?$AAm?$AAe?$AAn?$AAt?$AAS?$AAt?$AAa?$AAt?$AAe?$AA?$AA@ 0014ca2c     misc.obj
 0002:0000ba60       ??_C@_1EE@MELFAAB@?$AAU?$AAn?$AAh?$AAa?$AAn?$AAd?$AAl?$AAe?$AAd?$AA?5?$AAS?$AAe?$AAt?$AA?5?$AAE?$AAq?$AAu?$AAi?$AAp?$AAm?$AAe?$AAn?$AAt?$AAS?$AAt?$AAa?$AAt?$AAe?$AA?5?$AA?$DN?$AA?5?$AA?$CF@ 0014ca60     misc.obj
 0002:0000baa4       ??_C@_1CI@LDJJKLLA@?$AAp?$AAb?$AAD?$AAe?$AAv?$AAS?$AAp?$AAe?$AAc?$AAD?$AAa?$AAt?$AAa?$AA?5?$AAN?$AAU?$AAL?$AAL?$AA?$CB?$AA?$AA@ 0014caa4     misc.obj
 0002:0000bad0       ??_C@_1GM@KONOKCLC@?$AAR?$AAI?$AAL?$AA_?$AAD?$AAe?$AAv?$AAS?$AAp?$AAe?$AAc?$AAi?$AAf?$AAi?$AAc?$AA?5?$AAr?$AAe?$AAt?$AAu?$AAr?$AAn?$AAs?$AA?5?$AAE?$AA_?$AAN?$AAO?$AAT?$AAI?$AAM?$AAP@ 0014cad0     misc.obj
 0002:0000bb40       ??_C@_1HE@NLBFEBFJ@?$AAD?$AAS?$AA_?$AAX?$AAX?$AAX?$AA_?$AAC?$AAI?$AAD?$AA?5?$AA?$DN?$AA?5?$AA?$CF?$AAd?$AA?5?$AAu?$AAn?$AAh?$AAa?$AAn?$AAd?$AAl?$AAe?$AAd?$AA?5?$AAd?$AAu?$AAe?$AA?5?$AAt?$AAo@ 0014cb40     misc.obj
 0002:0000bbb8       ??_C@_1EE@EEDENINA@?$AAA?$AAS?$AAS?$AAE?$AAR?$AAT?$AAI?$AAO?$AAN?$AA?5?$AAF?$AAA?$AAI?$AAL?$AAU?$AAR?$AAE?$AA?3?$AA?5?$AA?$DN?$AA?$DN?$AA?$DN?$AA?$DO?$AAd?$AAw?$AAS?$AAi?$AAz?$AAe?$AA?5?$AA?$DO?$AA?5@ 0014cbb8     misc.obj
 0002:0000bc00       ??_C@_1FC@DCIECDIA@?$AAA?$AAS?$AAS?$AAE?$AAR?$AAT?$AAI?$AAO?$AAN?$AA?5?$AAF?$AAA?$AAI?$AAL?$AAU?$AAR?$AAE?$AA?3?$AA?5?$AA?$DN?$AA?$DN?$AA?$DN?$AA?$DO?$AAN?$AAU?$AAL?$AAL?$AA?5?$AA?$CB?$AA?$DN?$AA?5?$AAl@ 0014cc00     misc.obj
 0002:0000bc88       ??_C@_1HA@PEBFJIHG@?$AAS?$AAe?$AAt?$AAE?$AAq?$AAu?$AAi?$AAp?$AAm?$AAe?$AAn?$AAt?$AAC?$AAa?$AAc?$AAh?$AAe?$AAS?$AAt?$AAa?$AAt?$AAe?$AA?5?$AAN?$AAO?$AAO?$AAP?$AA?5?$AAs?$AAi?$AAn?$AAc@ 0014cc88     misc.obj
 0002:0000bcf8       ??_C@_1CG@KFJKIMKK@?$AAL?$AAa?$AAs?$AAt?$AAE?$AAq?$AAu?$AAi?$AAp?$AAm?$AAe?$AAn?$AAt?$AAS?$AAt?$AAa?$AAt?$AAe?$AA?$AA@ 0014ccf8     misc.obj
 0002:0000bd20       ??_C@_1BAI@OHMCGNDD@?$AAG?$AAe?$AAt?$AAE?$AAq?$AAu?$AAi?$AAp?$AAm?$AAe?$AAn?$AAt?$AAS?$AAt?$AAa?$AAt?$AAe?$AA?5?$AAr?$AAe?$AAt?$AAu?$AAr?$AAn?$AAs?$AA?5?$AAh?$AAr?$AA?5?$AA?$DN?$AA?5?$AA0@ 0014cd20     misc.obj
 0002:0000be28       ??_C@_1FA@MJNFAOON@?$AAD?$AAo?$AAn?$AAe?$AA?5?$AAf?$AAo?$AAr?$AAc?$AAi?$AAn?$AAg?$AA?5?$AAt?$AAh?$AAe?$AA?5?$AAm?$AAo?$AAd?$AAe?$AAm?$AA?5?$AAo?$AAf?$AAf?$AA?5?$AA?$CI?$AAl?$AAo?$AAw?$AA?5@ 0014ce28     misc.obj
 0002:0000be78       ??_C@_1FM@MHHHFEPK@?$AAR?$AAI?$AAL?$AA?5?$AAa?$AAu?$AAt?$AAo?$AA?5?$AAp?$AAo?$AAw?$AAe?$AAr?$AA?5?$AAc?$AAy?$AAc?$AAl?$AAe?$AA?5?$AAi?$AAn?$AAs?$AAt?$AAe?$AAa?$AAd?$AA?5?$AAo?$AAf?$AA?5@ 0014ce78     misc.obj
 0002:0000bed4       ??_C@_1BO@FEFGDBAP@?$AAR?$AAe?$AAs?$AAe?$AAt?$AAi?$AAn?$AAg?$AA?5?$AAm?$AAo?$AAd?$AAe?$AAm?$AA?$AA@ 0014ced4     misc.obj
 0002:0000bef8       ??_C@_1FE@NMEJPKAK@?$AAF?$AAa?$AAi?$AAl?$AA?5?$AAt?$AAo?$AA?5?$AAt?$AAu?$AAr?$AAn?$AA?5?$AAo?$AAf?$AAf?$AA?5?$AAm?$AAo?$AAd?$AAe?$AAm?$AA?5?$AAH?$AAW?$AA?4?$AA?5?$AAT?$AAr?$AAy?$AA?5?$AAS@ 0014cef8     misc.obj
 0002:0000bf50       ??_C@_1EK@MGODGNKC@?$AAF?$AAa?$AAi?$AAl?$AA?5?$AAt?$AAo?$AA?5?$AAS?$AAe?$AAt?$AAP?$AAo?$AAw?$AAe?$AAr?$AAD?$AAo?$AAw?$AAn?$AA?0?$AA?5?$AAr?$AAc?$AAP?$AAo?$AAw?$AAe?$AAr?$AAO?$AAp?$AA?5@ 0014cf50     misc.obj
 0002:0000bfa0       ??_C@_1HO@BDBDHIOO@?$AAF?$AAa?$AAi?$AAl?$AA?5?$AAt?$AAo?$AA?5?$AAt?$AAu?$AAr?$AAn?$AA?5?$AAo?$AAn?$AA?5?$AAm?$AAo?$AAd?$AAe?$AAm?$AA?5?$AAH?$AAW?$AA?0?$AA?5?$AAm?$AA_?$AAp?$AAS?$AAe?$AAt@ 0014cfa0     misc.obj
 0002:0000c020       ??_C@_1GE@DPCBLCOO@?$AAS?$AAe?$AAt?$AAE?$AAq?$AAu?$AAi?$AAp?$AAm?$AAe?$AAn?$AAt?$AAS?$AAt?$AAa?$AAt?$AAe?$AA?5?$AAt?$AAo?$AA?5?$AAs?$AAt?$AAa?$AAt?$AAe?$AA?5?$AA?$DN?$AA?5?$AA?$CF?$AAd?$AA?5@ 0014d020     misc.obj
 0002:0000c088       ??_C@_1KM@FGPIFFGK@?$AAF?$AAi?$AAl?$AAl?$AAS?$AAi?$AAg?$AAn?$AAa?$AAl?$AAQ?$AAu?$AAa?$AAl?$AAi?$AAt?$AAy?$AAS?$AAt?$AAr?$AAu?$AAc?$AAt?$AA?5?$AAc?$AAa?$AAl?$AAl?$AAe?$AAd?$AA?5?$AAw@ 0014d088     misc.obj
 0002:0000c138       ??_C@_1BEO@FFMKOHED@?$AAU?$AAp?$AAd?$AAa?$AAt?$AAe?$AA?5?$AAs?$AAe?$AAr?$AAv?$AAi?$AAc?$AAe?$AA?5?$AAi?$AAn?$AAd?$AAi?$AAc?$AAa?$AAt?$AAi?$AAo?$AAn?$AA?5?$AAm?$AAa?$AAn?$AAu?$AAa?$AAl@ 0014d138     misc.obj
 0002:0000c288       ??_C@_1EK@BPLLLANG@?$AAC?$AAa?$AAn?$AAn?$AAo?$AAt?$AA?5?$AAp?$AAo?$AAl?$AAl?$AA?5?$AAR?$AAS?$AAS?$AAI?$AA?5?$AAd?$AAu?$AAe?$AA?5?$AAt?$AAo?$AA?5?$AAu?$AAn?$AAk?$AAn?$AAo?$AAw?$AAn?$AA?5@ 0014d288     misc.obj
 0002:0000c2d8       ??_C@_1HC@EFLNCBLC@?$AAG?$AAe?$AAt?$AAC?$AAe?$AAl?$AAl?$AAT?$AAo?$AAw?$AAe?$AAr?$AAI?$AAn?$AAf?$AAo?$AA?5?$AAU?$AAM?$AAT?$AAS?$AA?3?$AA?5?$AAC?$AAe?$AAl?$AAl?$AA?5?$AAI?$AAD?$AA?$DN?$AA?$CF@ 0014d2d8     misc.obj
 0002:0000c350       ??_C@_1MA@IMPJFHNA@?$AAG?$AAe?$AAt?$AAC?$AAe?$AAl?$AAl?$AAT?$AAo?$AAw?$AAe?$AAr?$AAI?$AAn?$AAf?$AAo?$AA?5?$AAG?$AAS?$AAM?$AA?3?$AA?5?$AAC?$AAe?$AAl?$AAl?$AA?5?$AAI?$AAD?$AA?$DN?$AA?$CF?$AAd@ 0014d350     misc.obj
 0002:0000c410       ??_C@_1JC@JJGLMAMM@?$AAG?$AAe?$AAt?$AAC?$AAe?$AAl?$AAl?$AAT?$AAo?$AAw?$AAe?$AAr?$AAI?$AAn?$AAf?$AAo?$AA?5?$AAC?$AAD?$AAM?$AAA?$AA?3?$AA?5?$AAS?$AAy?$AAs?$AAt?$AAe?$AAm?$AA?5?$AAI?$AAD@ 0014d410     misc.obj
 0002:0000c4a4       ??_C@_1DC@CDJMMJGK@?$AAC?$AAR?$AAa?$AAd?$AAi?$AAo?$AA?3?$AA?3?$AAG?$AAe?$AAt?$AAC?$AAe?$AAl?$AAl?$AAT?$AAo?$AAw?$AAe?$AAr?$AAI?$AAn?$AAf?$AAo?$AA?$AA@ 0014d4a4     misc.obj
 0002:0000c4d8       ??_C@_1DE@IIPFICIA@?$AAS?$AAw?$AAi?$AAG?$AAe?$AAt?$AAB?$AAy?$AAt?$AAe?$AAC?$AAo?$AAu?$AAn?$AAt?$AAe?$AAr?$AA?$CI?$AA?$CF?$AAd?$AA?0?$AA?5?$AA?$CF?$AAd?$AA?$CJ?$AA?$AA@ 0014d4d8     misc.obj
 0002:0000c510       ??_C@_1EG@JJEMINIM@?$AAm?$AAp?$AAF?$AAn?$AAS?$AAw?$AAi?$AAG?$AAe?$AAt?$AAI?$AAm?$AAe?$AAi?$AA?5?$AAf?$AAa?$AAi?$AAl?$AAe?$AAd?$AA?0?$AA?5?$AAe?$AAr?$AAr?$AAo?$AAr?$AA?5?$AA?$DN?$AA?5?$AA?$CF@ 0014d510     misc.obj
 0002:0000c558       ??_C@_17FKMEKEMI@?$AA?$CF?$AAl?$AAX?$AA?$AA@ 0014d558     misc.obj
 0002:0000c560       ??_C@_1M@OOOOBAIH@?$AA?$CF?$AAs?$AA?3?$AA?$CF?$AAd?$AA?$AA@ 0014d560     misc.obj
 0002:0000c56c       ??_C@_1CA@KOBFOPFD@?$AAS?$AAi?$AAe?$AAr?$AAr?$AAa?$AA?5?$AAW?$AAi?$AAr?$AAe?$AAl?$AAe?$AAs?$AAs?$AA?$AA@ 0014d56c     misc.obj
 0002:0000c590       ??_C@_1EO@BDMPPGAO@?$AAm?$AAp?$AAF?$AAn?$AAS?$AAw?$AAi?$AAG?$AAe?$AAt?$AAP?$AAd?$AAs?$AAm?$AAP?$AAa?$AAG?$AAp?$AAs?$AAL?$AAo?$AAc?$AAk?$AA?5?$AAf?$AAa?$AAi?$AAl?$AAe?$AAd?$AA?5?$AAr@ 0014d590     misc.obj
 0002:0000c5e0       ??_C@_1GG@JOMNGKOM@?$AAD?$AAM?$AA?5?$AAm?$AAo?$AAd?$AAe?$AA?5?$AAs?$AAt?$AAo?$AAp?$AAp?$AAe?$AAd?$AA?5?$AAO?$AAK?$AA?$CB?$AA?5?$AAA?$AAu?$AAt?$AAo?$AA?5?$AAp?$AAo?$AAw?$AAe?$AAr?$AA?5?$AAc@ 0014d5e0     misc.obj
 0002:0000c648       ??_C@_1CK@JOONJNHB@?$AAF?$AAa?$AAi?$AAl?$AA?5?$AAt?$AAo?$AA?5?$AAs?$AAt?$AAo?$AAp?$AA?5?$AAD?$AAM?$AA?5?$AAM?$AAo?$AAd?$AAe?$AA?$AA@ 0014d648     misc.obj
 0002:0000c678       ??_C@_1EI@IGMMHOJI@?$AAS?$AAt?$AAo?$AAp?$AAD?$AAM?$AAM?$AAo?$AAd?$AAe?$AA?5?$AAf?$AAa?$AAi?$AAl?$AAs?$AA?5?$AAb?$AAe?$AAc?$AAa?$AAu?$AAs?$AAe?$AA?5?$AAP?$AAT?$AA?5?$AAm?$AAo?$AAd?$AAe@ 0014d678     misc.obj
 0002:0000c6c0       ??_C@_1GA@GLELEKNE@?$AAS?$AAt?$AAa?$AAr?$AAt?$AAP?$AAT?$AAM?$AAo?$AAd?$AAe?$AA?5?$AAf?$AAa?$AAi?$AAl?$AAe?$AAd?$AA?5?$AAt?$AAo?$AA?5?$AAm?$AA_?$AAp?$AAS?$AAe?$AAt?$AAT?$AAe?$AAt?$AAh@ 0014d6c0     misc.obj
 0002:0000c720       ??_C@_1EK@DFKCMBJD@?$AAS?$AAt?$AAa?$AAr?$AAt?$AAP?$AAT?$AAM?$AAo?$AAd?$AAe?$AA?5?$AAf?$AAa?$AAi?$AAl?$AAs?$AA?5?$AAb?$AAe?$AAc?$AAa?$AAu?$AAs?$AAe?$AA?5?$AAD?$AAM?$AA?5?$AAm?$AAo?$AAd@ 0014d720     misc.obj
 0002:0000c770       ??_C@_1GA@PMPBONJ@?$AAS?$AAt?$AAo?$AAp?$AAP?$AAT?$AAM?$AAo?$AAd?$AAe?$AA?5?$AAf?$AAa?$AAi?$AAl?$AAe?$AAd?$AA?5?$AAt?$AAo?$AA?5?$AAm?$AA_?$AAp?$AAS?$AAe?$AAt?$AAT?$AAe?$AAt?$AAh?$AAe@ 0014d770     misc.obj
 0002:0000c7d0       ??_C@_1EI@BIDKHPHK@?$AAS?$AAt?$AAo?$AAp?$AAP?$AAT?$AAM?$AAo?$AAd?$AAe?$AA?5?$AAf?$AAa?$AAi?$AAl?$AAs?$AA?5?$AAb?$AAe?$AAc?$AAa?$AAu?$AAs?$AAe?$AA?5?$AAD?$AAM?$AA?5?$AAm?$AAo?$AAd?$AAe@ 0014d7d0     misc.obj
 0002:0000c818       ??_C@_1GM@BCLCIKDI@?$AAC?$AAR?$AAa?$AAd?$AAi?$AAo?$AA?3?$AA?3?$AAS?$AAe?$AAt?$AAX?$AAT?$AAR?$AAA?$AAE?$AAm?$AAb?$AAe?$AAd?$AAd?$AAe?$AAd?$AAC?$AAl?$AAi?$AAe?$AAn?$AAt?$AA?3?$AA?5?$AAS@ 0014d818     misc.obj
 0002:0000c888       ??_C@_1HC@EGPFMAKE@?$AAC?$AAR?$AAa?$AAd?$AAi?$AAo?$AA?3?$AA?3?$AAS?$AAe?$AAt?$AAG?$AAp?$AAs?$AAD?$AAe?$AAf?$AAa?$AAu?$AAl?$AAt?$AA?3?$AA?5?$AAS?$AAe?$AAt?$AAP?$AAD?$AAS?$AAD?$AAe?$AAf@ 0014d888     misc.obj
 0002:0000c900       ??_C@_1LA@OLIBJKIM@?$AAC?$AAR?$AAa?$AAd?$AAi?$AAo?$AA?3?$AA?3?$AAS?$AAe?$AAt?$AAG?$AAp?$AAs?$AAD?$AAe?$AAf?$AAa?$AAu?$AAl?$AAt?$AA?3?$AA?5?$AAn?$AAO?$AAp?$AAe?$AAr?$AAa?$AAt?$AAi?$AAo@ 0014d900     misc.obj
 0002:0000c9b0       ??_C@_1FC@BIGANALK@?$AAC?$AAR?$AAa?$AAd?$AAi?$AAo?$AA?3?$AA?3?$AAS?$AAe?$AAt?$AAN?$AAM?$AAE?$AAA?$AAC?$AAo?$AAn?$AAf?$AAi?$AAg?$AA?5?$AAf?$AAa?$AAi?$AAl?$AAe?$AAd?$AA?0?$AA?5?$AAr?$AAc@ 0014d9b0     misc.obj
 0002:0000ca08       ??_C@_1MI@OILNKMFF@?$AAC?$AAR?$AAa?$AAd?$AAi?$AAo?$AA?3?$AA?3?$AAS?$AAe?$AAt?$AAN?$AAM?$AAE?$AAA?$AAC?$AAo?$AAn?$AAf?$AAi?$AAg?$AA?3?$AA?5?$AAN?$AAM?$AAE?$AAA?$AAC?$AAo?$AAn?$AAf?$AAi@ 0014da08     misc.obj
 0002:0000cad0       ??_C@_1IC@LEMCGGIP@?$AAC?$AAR?$AAa?$AAd?$AAi?$AAo?$AA?3?$AA?5?$AAR?$AAe?$AAa?$AAd?$AAP?$AAh?$AAo?$AAn?$AAe?$AAb?$AAo?$AAo?$AAk?$AAE?$AAn?$AAt?$AAr?$AAi?$AAe?$AAs?$AA?3?$AA?5?$AAE?$AAR@ 0014dad0     misc.obj
 0002:0000cb58       ??_C@_1BAM@NAHKKLL@?$AAC?$AAR?$AAa?$AAd?$AAi?$AAo?$AA?3?$AA?3?$AAG?$AAe?$AAt?$AAP?$AAh?$AAo?$AAn?$AAe?$AAb?$AAo?$AAo?$AAk?$AAC?$AAa?$AAp?$AAa?$AAb?$AAi?$AAl?$AAi?$AAt?$AAi?$AAe?$AAs@ 0014db58     misc.obj
 0002:0000cc68       ??_C@_1JM@OMMIDNMJ@?$AAC?$AAR?$AAa?$AAd?$AAi?$AAo?$AA?3?$AA?3?$AAG?$AAe?$AAt?$AAP?$AAh?$AAo?$AAn?$AAe?$AAb?$AAo?$AAo?$AAk?$AAC?$AAa?$AAp?$AAa?$AAb?$AAi?$AAl?$AAi?$AAt?$AAi?$AAe?$AAs@ 0014dc68     misc.obj
 0002:0000cd38       ??_C@_1CG@NMENLFLO@?$AAW?$AAa?$AAi?$AAt?$AA?5?$AAE?$AAv?$AAe?$AAn?$AAt?$AA?5?$AAT?$AAi?$AAm?$AAe?$AAo?$AAu?$AAt?$AA?$AA@ 0014dd38     misc.obj
 0002:0000cd60       ??_C@_1JO@EKLJEOOG@?$AAC?$AAR?$AAa?$AAd?$AAi?$AAo?$AA?3?$AA?5?$AAR?$AAe?$AAa?$AAd?$AAP?$AAh?$AAo?$AAn?$AAe?$AAb?$AAo?$AAo?$AAk?$AAE?$AAn?$AAt?$AAr?$AAi?$AAe?$AAs?$AA?3?$AA?5?$AAA?$AAt@ 0014dd60     misc.obj
 0002:0000ce00       ??_C@_1IM@LPNAEMDI@?$AAQ?$AAM?$AAI?$AA?5?$AAR?$AAe?$AAa?$AAd?$AAP?$AAh?$AAo?$AAn?$AAe?$AAb?$AAo?$AAo?$AAk?$AAR?$AAe?$AAc?$AAo?$AAr?$AAd?$AAs?$AA?5?$AAE?$AAR?$AAR?$AAO?$AAR?$AA?$CB?$AA?$CB@ 0014de00     misc.obj
 0002:0000ce90       ??_C@_1GK@JFNPDAPG@?$AAC?$AAR?$AAa?$AAd?$AAi?$AAo?$AA?3?$AA?5?$AAR?$AAe?$AAa?$AAd?$AAP?$AAh?$AAo?$AAn?$AAe?$AAb?$AAo?$AAo?$AAk?$AAE?$AAn?$AAt?$AAr?$AAi?$AAe?$AAs?$AA?3?$AA?5?$AAE?$AAR@ 0014de90     misc.obj
 0002:0000cf00       ??_C@_1GI@MODMLKDJ@?$AAC?$AAR?$AAa?$AAd?$AAi?$AAo?$AA?3?$AA?5?$AAR?$AAe?$AAa?$AAd?$AAP?$AAh?$AAo?$AAn?$AAe?$AAb?$AAo?$AAo?$AAk?$AAE?$AAn?$AAt?$AAr?$AAi?$AAe?$AAs?$AA?3?$AA?5?$AAE?$AAR@ 0014df00     misc.obj
 0002:0000cf68       ??_C@_1HA@HKCHNNDK@?$AAC?$AAR?$AAa?$AAd?$AAi?$AAo?$AA?3?$AA?5?$AAR?$AAe?$AAa?$AAd?$AAP?$AAh?$AAo?$AAn?$AAe?$AAb?$AAo?$AAo?$AAk?$AAE?$AAn?$AAt?$AAr?$AAi?$AAe?$AAs?$AA?3?$AA?5?$AAE?$AAR@ 0014df68     misc.obj
 0002:0000cfd8       ??_C@_1JE@KICINDAF@?$AAA?$AAS?$AAS?$AAE?$AAR?$AAT?$AAI?$AAO?$AAN?$AA?5?$AAF?$AAA?$AAI?$AAL?$AAU?$AAR?$AAE?$AA?3?$AA?5?$AA?$DN?$AA?$DN?$AA?$DN?$AA?$DO?$AA?$CI?$AAp?$AAP?$AAB?$AAE?$AAD?$AAa?$AAt?$AAa@ 0014dfd8     misc.obj
 0002:0000d070       ??_C@_1EK@GIFGGHIK@?$AAA?$AAS?$AAS?$AAE?$AAR?$AAT?$AAI?$AAO?$AAN?$AA?5?$AAF?$AAA?$AAI?$AAL?$AAU?$AAR?$AAE?$AA?3?$AA?5?$AA?$DN?$AA?$DN?$AA?$DN?$AA?$DO?$AAp?$AAD?$AAa?$AAt?$AAa?$AA?5?$AA?$CB?$AA?$DN?$AA?5@ 0014e070     misc.obj
 0002:0000d0c0       ??_C@_1GG@JDOBCDLN@?$AAS?$AAW?$AAI?$AA_?$AAN?$AAO?$AAT?$AAI?$AAF?$AAY?$AA_?$AAP?$AAh?$AAo?$AAn?$AAe?$AAb?$AAo?$AAo?$AAk?$AAE?$AAn?$AAt?$AAr?$AAy?$AA?5?$AAr?$AAe?$AAc?$AAe?$AAi?$AAv@ 0014e0c0     misc.obj
 0002:0000d128       ??_C@_1EO@DHGAIBAF@?$AAW?$AAr?$AAi?$AAt?$AAe?$AAP?$AAh?$AAo?$AAn?$AAe?$AAb?$AAo?$AAo?$AAk?$AAR?$AAe?$AAc?$AAo?$AAr?$AAd?$AA?5?$AAf?$AAa?$AAi?$AAl?$AAe?$AAd?$AA?0?$AA?5?$AAr?$AAc?$AA?5@ 0014e128     misc.obj
 0002:0000d178       ??_C@_1EO@MIMLBPGP@?$AAD?$AAe?$AAl?$AAe?$AAt?$AAe?$AAP?$AAh?$AAo?$AAn?$AAe?$AAb?$AAo?$AAo?$AAk?$AAE?$AAn?$AAt?$AAr?$AAy?$AA?5?$AAf?$AAa?$AAi?$AAl?$AAe?$AAd?$AA?0?$AA?5?$AAr?$AAc?$AA?5@ 0014e178     misc.obj
 0002:0000d1c8       ??_C@_1FO@NMDDADBK@?$AAI?$AAs?$AAS?$AAa?$AAf?$AAe?$AAI?$AAm?$AAa?$AAg?$AAe?$AA?5?$AAm?$AAp?$AAF?$AAn?$AAS?$AAw?$AAi?$AAG?$AAe?$AAt?$AAF?$AAi?$AAr?$AAm?$AAw?$AAa?$AAr?$AAe?$AAV?$AAe@ 0014e1c8     misc.obj
 0002:0000d228       ??_C@_1O@ICDCMGEE@?$AAS?$AAL?$AA9?$AA0?$AA9?$AA0?$AA?$AA@ 0014e228     misc.obj
 0002:0000d238       ??_C@_1EI@NEECAIND@?$AAI?$AAs?$AAS?$AAa?$AAf?$AAe?$AAI?$AAm?$AAa?$AAg?$AAe?$AA?5?$AAS?$AAw?$AAi?$AAG?$AAe?$AAt?$AAB?$AAo?$AAo?$AAt?$AAV?$AAe?$AAr?$AAs?$AAi?$AAo?$AAn?$AA?5?$AA?3?$AA?5@ 0014e238     misc.obj
 0002:0000d280       ??_C@_1FM@MIKHCGDH@?$AAI?$AAs?$AAS?$AAa?$AAf?$AAe?$AAI?$AAm?$AAa?$AAg?$AAe?$AA?5?$AAS?$AAw?$AAi?$AAG?$AAe?$AAt?$AAB?$AAo?$AAo?$AAt?$AAV?$AAe?$AAr?$AAs?$AAi?$AAo?$AAn?$AA?5?$AAf?$AAa@ 0014e280     misc.obj
 0002:0000d2e0       ??_C@_1EG@DMELMCAA@?$AAI?$AAs?$AAS?$AAa?$AAf?$AAe?$AAI?$AAm?$AAa?$AAg?$AAe?$AA?5?$AAS?$AAw?$AAi?$AAG?$AAe?$AAt?$AAP?$AAR?$AAL?$AAV?$AAe?$AAr?$AAs?$AAi?$AAo?$AAn?$AA?5?$AA?3?$AA?5?$AA?$CF@ 0014e2e0     misc.obj
 0002:0000d328       ??_C@_1FK@NGCGOECF@?$AAI?$AAs?$AAS?$AAa?$AAf?$AAe?$AAI?$AAm?$AAa?$AAg?$AAe?$AA?5?$AAS?$AAw?$AAi?$AAG?$AAe?$AAt?$AAP?$AAR?$AAL?$AAV?$AAe?$AAr?$AAs?$AAi?$AAo?$AAn?$AA?5?$AAf?$AAa?$AAi@ 0014e328     misc.obj
 0002:0000d388       ??_C@_1FA@FHJNFDAM@?$AAI?$AAs?$AAS?$AAa?$AAf?$AAe?$AAI?$AAm?$AAa?$AAg?$AAe?$AA?5?$AAS?$AAw?$AAi?$AAG?$AAe?$AAt?$AAH?$AAa?$AAr?$AAd?$AAw?$AAa?$AAr?$AAe?$AAV?$AAe?$AAr?$AAs?$AAi?$AAo@ 0014e388     misc.obj
 0002:0000d3d8       ??_C@_1GE@NLGGKPPK@?$AAI?$AAs?$AAS?$AAa?$AAf?$AAe?$AAI?$AAm?$AAa?$AAg?$AAe?$AA?5?$AAS?$AAw?$AAi?$AAG?$AAe?$AAt?$AAH?$AAa?$AAr?$AAd?$AAw?$AAa?$AAr?$AAe?$AAV?$AAe?$AAr?$AAs?$AAi?$AAo@ 0014e3d8     misc.obj
 0002:0000d440       ??_C@_1FA@BCCPDENC@?$AAI?$AAs?$AAS?$AAa?$AAf?$AAe?$AAI?$AAm?$AAa?$AAg?$AAe?$AA?5?$AAS?$AAw?$AAi?$AAG?$AAe?$AAt?$AAF?$AAi?$AAr?$AAm?$AAw?$AAa?$AAr?$AAe?$AAV?$AAe?$AAr?$AAs?$AAi?$AAo@ 0014e440     misc.obj
 0002:0000d490       ??_C@_1GE@CMFBFOKH@?$AAI?$AAs?$AAS?$AAa?$AAf?$AAe?$AAI?$AAm?$AAa?$AAg?$AAe?$AA?5?$AAS?$AAw?$AAi?$AAG?$AAe?$AAt?$AAF?$AAi?$AAr?$AAm?$AAw?$AAa?$AAr?$AAe?$AAV?$AAe?$AAr?$AAs?$AAi?$AAo@ 0014e490     misc.obj
 0002:0000d4f4       ??_C@_1BA@FEAMADEO@?$AA0?$AAx?$AA?$CF?$AA0?$AA2?$AAX?$AA?5?$AA?$AA@ 0014e4f4     misc.obj
 0002:0000d504       ??_C@_19HHMHINIL@?$AA?$CF?$AA0?$AA2?$AAX?$AA?$AA@ 0014e504     misc.obj
 0002:0000d510       ??_C@_1FE@IGHJNBKC@?$AA?$CK?$AAm?$AAp?$AAF?$AAn?$AAS?$AAw?$AAi?$AAG?$AAe?$AAt?$AAI?$AAm?$AAa?$AAg?$AAe?$AAP?$AAr?$AAe?$AAf?$AAe?$AAr?$AAe?$AAn?$AAc?$AAe?$AA?5?$AAf?$AAa?$AAi?$AAl?$AAe@ 0014e510     misc.obj
 0002:0000d568       ??_C@_1GC@FGFFPJCG@?$AAS?$AAe?$AAt?$AAF?$AAw?$AAI?$AAm?$AAa?$AAg?$AAe?$AAP?$AAr?$AAe?$AAf?$AAe?$AAr?$AAe?$AAn?$AAc?$AAe?$AA?3?$AA?5?$AAF?$AAa?$AAi?$AAl?$AAe?$AAd?$AA?5?$AAt?$AAo?$AA?5@ 0014e568     misc.obj
 0002:0000d5d0       ??_C@_1HO@CNKGJMEN@?$AAS?$AAe?$AAt?$AAF?$AAw?$AAI?$AAm?$AAa?$AAg?$AAe?$AAP?$AAr?$AAe?$AAf?$AAe?$AAr?$AAe?$AAn?$AAc?$AAe?$AA?3?$AA?5?$AAF?$AAa?$AAi?$AAl?$AAe?$AAd?$AA?5?$AAt?$AAo?$AA?5@ 0014e5d0     misc.obj
 0002:0000d650       ??_C@_1FG@NAKDFHMF@?$AAm?$AAp?$AAF?$AAn?$AAS?$AAw?$AAi?$AAS?$AAe?$AAt?$AAI?$AAm?$AAa?$AAg?$AAe?$AAP?$AAr?$AAe?$AAf?$AAe?$AAr?$AAe?$AAn?$AAc?$AAe?$AA?5?$AAf?$AAa?$AAi?$AAl?$AAe?$AAd@ 0014e650     misc.obj
 0002:0000d6a8       ??_C@_1DC@GGMFGHGM@?$AAH?$AAa?$AAn?$AAd?$AAl?$AAe?$AAR?$AAe?$AAs?$AAu?$AAm?$AAe?$AA?5?$AAG?$AAe?$AAt?$AAH?$AAW?$AAP?$AAo?$AAw?$AAe?$AAr?$AA?$DP?$AA?$AA@ 0014e6a8     misc.obj
 0002:0000d6e0       ??_C@_1GA@NHLIPGDN@?$AAS?$AAy?$AAn?$AAc?$AA?5?$AAU?$AAp?$AA?5?$AAC?$AAa?$AAl?$AAl?$AA?5?$AAs?$AAt?$AAa?$AAt?$AAe?$AAs?$AA?5?$AAw?$AAi?$AAt?$AAh?$AA?5?$AAt?$AAh?$AAe?$AA?5?$AAm?$AAo?$AAd@ 0014e6e0     misc.obj
 0002:0000d740       ??_C@_1EE@BHOLLJBE@?$AAH?$AAW?$AA?5?$AAO?$AAf?$AAf?$AA?5?$AAd?$AAu?$AAr?$AAi?$AAn?$AAg?$AA?5?$AAD?$AAM?$AA?5?$AAm?$AAo?$AAd?$AAe?$AA?4?$AA?5?$AAT?$AAu?$AAr?$AAn?$AA?5?$AAH?$AAW?$AA?5?$AAo@ 0014e740     misc.obj
 0002:0000d788       ??_C@_1FE@HAAECLEM@?$AAD?$AAM?$AA?5?$AAm?$AAo?$AAd?$AAe?$AA?5?$AAs?$AAt?$AAa?$AAr?$AAt?$AAe?$AAd?$AA?5?$AAO?$AAK?$AA?5?$AAm?$AA_?$AAe?$AAC?$AAu?$AAr?$AAr?$AAe?$AAn?$AAt?$AAD?$AAM?$AAM@ 0014e788     misc.obj
 0002:0000d7dc       ??_C@_1CM@CINOGJE@?$AAF?$AAa?$AAi?$AAl?$AA?5?$AAt?$AAo?$AA?5?$AAs?$AAt?$AAa?$AAr?$AAt?$AA?5?$AAD?$AAM?$AA?5?$AAM?$AAo?$AAd?$AAe?$AA?$AA@ 0014e7dc     misc.obj
 0002:0000d808       ??_C@_1MA@EJHDDJOJ@?$AAS?$AAt?$AAa?$AAr?$AAt?$AAD?$AAM?$AAM?$AAo?$AAd?$AAe?$AA?5?$AA?$CI?$AAd?$AAe?$AAs?$AAi?$AAr?$AAe?$AAd?$AA?5?$AAm?$AAo?$AAd?$AAe?$AA?5?$AA?$DN?$AA?5?$AA?$CF?$AAd?$AA?5?$AA?$FL@ 0014e808     misc.obj
 0002:0000d8c8       ??_C@_1HA@FCAJBEHF@?$AAS?$AAt?$AAa?$AAr?$AAt?$AAD?$AAM?$AAM?$AAo?$AAd?$AAe?$AA?5?$AA?$CI?$AAR?$AAI?$AAL?$AA_?$AAP?$AAU?$AAR?$AAE?$AA_?$AAD?$AAM?$AA_?$AAM?$AAO?$AAD?$AAE?$AA?$CJ?$AA?5?$AAf@ 0014e8c8     misc.obj
 0002:0000d938       ??_C@_1GM@LEIAEKMM@?$AAE?$AAn?$AAd?$AA?5?$AAt?$AAh?$AAe?$AA?5?$AAP?$AAT?$AA?5?$AAm?$AAo?$AAd?$AAe?$AA?5?$AAb?$AAe?$AAf?$AAo?$AAr?$AAe?$AA?5?$AAs?$AAt?$AAa?$AAr?$AAt?$AAi?$AAn?$AAg?$AA?5@ 0014e938     misc.obj
 0002:0000db18       ??_C@_1HG@GCPALFPO@?$AAD?$AAE?$AAV?$AAS?$AAP?$AAE?$AAC?$AAI?$AAF?$AAI?$AAC?$AAD?$AAA?$AAT?$AAA?$AA?5?$AAi?$AAs?$AA?5?$AAN?$AAU?$AAL?$AAL?$AA?0?$AA?5?$AAr?$AAe?$AAt?$AAu?$AAr?$AAn?$AA?5@ 0014eb18     misc.obj
 0002:0000db90       ??_C@_1FM@FHKBGKCA@?$AAD?$AAE?$AAV?$AA_?$AAS?$AAP?$AAE?$AAC?$AAI?$AAF?$AAI?$AAC?$AA?0?$AA?5?$AAd?$AAw?$AAA?$AAc?$AAt?$AAi?$AAo?$AAn?$AA?5?$AA?$DN?$AA?5?$AA?$CF?$AAd?$AA?5?$AAn?$AAo?$AAt?$AA?5@ 0014eb90     misc.obj
 0002:0000dbec       ??_C@_1DK@BGCLKBGF@?$AAm?$AA_?$AAp?$AAI?$AAn?$AAi?$AAt?$AAi?$AAa?$AAt?$AAe?$AAH?$AAo?$AAs?$AAt?$AAB?$AAo?$AAo?$AAt?$AA?$CI?$AA?$CJ?$AA?5?$AAf?$AAa?$AAi?$AAl?$AAe?$AAd?$AA?$AA@ 0014ebec     misc.obj
 0002:0000dc28       ??_C@_1DI@NGMHFBAA@?$AAm?$AA_?$AAp?$AAI?$AAn?$AAi?$AAt?$AAi?$AAa?$AAt?$AAe?$AAH?$AAo?$AAs?$AAt?$AAB?$AAo?$AAo?$AAt?$AA?5?$AAi?$AAs?$AA?5?$AAN?$AAU?$AAL?$AAL?$AA?$AA@ 0014ec28     misc.obj
 0002:0000dc60       ??_C@_1FO@CCACCIBK@?$AAU?$AAn?$AAe?$AAx?$AAp?$AAe?$AAc?$AAt?$AAe?$AAd?$AA?5?$AAd?$AAw?$AAW?$AAa?$AAi?$AAt?$AAO?$AAb?$AAj?$AA?5?$AA?$DN?$AA?5?$AA?$CF?$AAd?$AA?0?$AA?5?$AAG?$AAe?$AAt?$AAL?$AAa@ 0014ec60     misc.obj
 0002:0000dcc0       ??_C@_1HA@HGNPJAC@?$AAU?$AAs?$AAe?$AAr?$AA?5?$AAw?$AAa?$AAn?$AAt?$AAs?$AA?5?$AAt?$AAo?$AA?5?$AAi?$AAn?$AAi?$AAt?$AAi?$AAa?$AAt?$AAe?$AA?5?$AAb?$AAo?$AAo?$AAt?$AA?5?$AA?$DN?$AA?5?$AA?$CF?$AAd@ 0014ecc0     misc.obj
 0002:0000dd30       ??_C@_1FA@OOHIDILK@?$AAD?$AAS?$AA_?$AAG?$AAE?$AAT?$AA_?$AAO?$AAM?$AAA?$AAD?$AAM?$AA_?$AAC?$AAO?$AAN?$AAF?$AAI?$AAG?$AA_?$AAC?$AAI?$AAD?$AA?5?$AAf?$AAa?$AAi?$AAl?$AAe?$AAd?$AA?0?$AA?5@ 0014ed30     misc.obj
 0002:0000dd80       ??_C@_1MM@LHJJDAEH@?$AAn?$AAO?$AAM?$AAA?$AAD?$AAM?$AAC?$AAa?$AAp?$AAa?$AAb?$AAi?$AAl?$AAi?$AAt?$AAy?$AA?5?$AA?$DN?$AA?5?$AA?$CF?$AAd?$AA?0?$AA?5?$AAd?$AAw?$AAF?$AAe?$AAa?$AAt?$AAu?$AAr?$AAe@ 0014ed80     misc.obj
 0002:0000de4c       ??_C@_1CM@NIENMKNP@?$AAS?$AAw?$AAi?$AAR?$AAt?$AAn?$AAR?$AAe?$AAs?$AAe?$AAt?$AA?$CI?$AA?$CJ?$AA?5?$AAs?$AAu?$AAc?$AAc?$AAe?$AAs?$AAs?$AA?$AA@ 0014ee4c     misc.obj
 0002:0000de78       ??_C@_1DC@HKGPFLDO@?$AAS?$AAw?$AAi?$AAR?$AAt?$AAn?$AAR?$AAe?$AAs?$AAe?$AAt?$AA?$CI?$AA?$CJ?$AA?5?$AAf?$AAa?$AAi?$AAl?$AAe?$AAd?$AA?3?$AA?5?$AA?$CF?$AAd?$AA?$AA@ 0014ee78     misc.obj
 0002:0000deb0       ??_C@_1HG@HNALKAFB@?$AAD?$AAS?$AA_?$AAG?$AAE?$AAT?$AA_?$AAP?$AAA?$AAC?$AAK?$AAE?$AAT?$AA_?$AAD?$AAA?$AAT?$AAA?$AA_?$AAS?$AAT?$AAA?$AAT?$AAU?$AAS?$AA_?$AAC?$AAI?$AAD?$AA?5?$AAt?$AAo@ 0014eeb0     misc.obj
 0002:0000df28       ??_C@_1DI@HEIHJLFI@?$AAS?$AAw?$AAi?$AAP?$AAo?$AAw?$AAe?$AAr?$AAS?$AAa?$AAv?$AAe?$AAE?$AAx?$AAi?$AAt?$AA?5?$AAF?$AAa?$AAi?$AAl?$AAe?$AAd?$AA?3?$AA?5?$AA?$CF?$AAi?$AA?$AA@ 0014ef28     misc.obj
 0002:0000df60       ??_C@_1FE@EOKOBAIM@?$AAD?$AAi?$AAa?$AAl?$AAE?$AAx?$AA?5?$AAw?$AAr?$AAo?$AAn?$AAg?$AA?5?$AAc?$AAa?$AAl?$AAl?$AAt?$AAy?$AAp?$AAe?$AA?5?$AA?$DN?$AA?5?$AA?$CF?$AAd?$AA?0?$AA?5?$AA?$CI?$AAo?$AAp?$AAt@ 0014ef60     misc.obj
 0002:0000dfb8       ??_C@_1FI@FPPLPBDF@?$AAm?$AAp?$AAF?$AAn?$AAS?$AAw?$AAi?$AAS?$AAe?$AAt?$AAC?$AAa?$AAl?$AAl?$AAO?$AAr?$AAi?$AAg?$AAi?$AAn?$AAa?$AAt?$AAe?$AAS?$AAo?$AAC?$AAm?$AAd?$AA?5?$AAf?$AAa?$AAi@ 0014efb8     misc.obj
 0002:0000e010       ??_C@_1GK@BIEJFHNH@?$AAF?$AAa?$AAi?$AAl?$AAe?$AAd?$AA?5?$AAt?$AAo?$AA?5?$AAr?$AAe?$AAa?$AAd?$AA?5?$AAO?$AAE?$AAM?$AA?5?$AAH?$AAa?$AAr?$AAd?$AAw?$AAa?$AAr?$AAe?$AA?5?$AAA?$AAu?$AAx?$AA?5@ 0014f010     misc.obj
 0002:0000e080       ??_C@_1EA@GEJFKMBN@?$AAO?$AAE?$AAM?$AA?5?$AAH?$AAa?$AAr?$AAd?$AAw?$AAa?$AAr?$AAe?$AA?5?$AAA?$AAu?$AAx?$AA?5?$AAV?$AAe?$AAr?$AAs?$AAi?$AAo?$AAn?$AA?5?$AAi?$AAs?$AA?3?$AA?5?$AA?$CF?$AAs?$AA?$AA@ 0014f080     misc.obj
 0002:0000e0c0       ??_C@_1DM@GPBOJDAJ@?$AAR?$AAe?$AAa?$AAd?$AA?5?$AAP?$AAR?$AAI?$AA?5?$AAv?$AAe?$AAr?$AAs?$AAi?$AAo?$AAn?$AA?$CI?$AA?$CJ?$AA?5?$AAF?$AAA?$AAI?$AAL?$AAE?$AAD?$AA?$DN?$AA?$CF?$AAd?$AA?6?$AA?$AA@ 0014f0c0     misc.obj
 0002:0000e100       ??_C@_1GE@INNNKLJJ@?$AAR?$AAe?$AAa?$AAd?$AA?5?$AAP?$AAR?$AAI?$AA?5?$AAv?$AAe?$AAr?$AAs?$AAi?$AAo?$AAn?$AA?$CI?$AA?$CJ?$AA?5?$AAS?$AAw?$AAi?$AAG?$AAe?$AAt?$AAP?$AAr?$AAi?$AAI?$AAn?$AAf?$AAo@ 0014f100     misc.obj
 0002:0000e164       ??_C@_1DM@MBCCOPAF@?$AAG?$AAe?$AAt?$AAP?$AAr?$AAo?$AAd?$AAu?$AAc?$AAt?$AAV?$AAe?$AAr?$AAs?$AAi?$AAo?$AAn?$AAS?$AAt?$AAr?$AA?5?$AAU?$AAS?$AAB?$AA?3?$AA?5?$AA?$CF?$AAs?$AA?5?$AA?$AA@ 0014f164     misc.obj
 0002:0000e1a0       ??_C@_1DO@MGKMODMF@?$AAU?$AAS?$AAB?$AA?5?$AAd?$AAr?$AAi?$AAv?$AAe?$AAr?$AA?5?$AAv?$AAe?$AAr?$AAs?$AAi?$AAo?$AAn?$AA?5?$AAu?$AAn?$AAv?$AAa?$AAi?$AAl?$AAa?$AAb?$AAl?$AAe?$AA?$CB?$AA?$AA@ 0014f1a0     misc.obj
 0002:0000e1e0       ??_C@_1BG@IBIGOCCD@?$AAs?$AAw?$AAi?$AAv?$AAs?$AAp?$AA?4?$AAd?$AAl?$AAl?$AA?$AA@ 0014f1e0     misc.obj
 0002:0000e1f8       ??_C@_1BI@FEHOKEFI@?$AAs?$AAw?$AAi?$AAc?$AAo?$AAm?$AAp?$AA?4?$AAd?$AAl?$AAl?$AA?$AA@ 0014f1f8     misc.obj
 0002:0000e210       ??_C@_1DM@HKNGGKCL@?$AAG?$AAe?$AAt?$AAP?$AAr?$AAo?$AAd?$AAu?$AAc?$AAt?$AAV?$AAe?$AAr?$AAs?$AAi?$AAo?$AAn?$AAS?$AAt?$AAr?$AA?5?$AAS?$AAD?$AAK?$AA?3?$AA?5?$AA?$CF?$AAs?$AA?5?$AA?$AA@ 0014f210     misc.obj
 0002:0000e24c       ??_C@_1BI@JIPDBAMF@?$AAs?$AAw?$AAi?$AAg?$AAo?$AAb?$AAi?$AA?4?$AAd?$AAl?$AAl?$AA?$AA@ 0014f24c     misc.obj
 0002:0000e264       ??_C@_1BI@LCJLEBHI@?$AAU?$AAN?$AAA?$AAV?$AAA?$AAI?$AAL?$AAA?$AAB?$AAL?$AAE?$AA?$AA@ 0014f264     misc.obj
 0002:0000e27c       ??_C@_1DA@JIIOIDF@?$AAS?$AAD?$AAK?$AA?5?$AAv?$AAe?$AAr?$AAs?$AAi?$AAo?$AAn?$AA?5?$AAu?$AAn?$AAv?$AAa?$AAi?$AAl?$AAa?$AAb?$AAl?$AAe?$AA?$CB?$AA?$AA@ 0014f27c     misc.obj
 0002:0000e2ac       ??_C@_1BM@IJDGBKNP@?$AAs?$AAw?$AAi?$AAr?$AAi?$AAl?$AAg?$AAs?$AAm?$AA?4?$AAd?$AAl?$AAl?$AA?$AA@ 0014f2ac     misc.obj
 0002:0000e2c8       ??_C@_1BO@DOEDCFIE@?$AAs?$AAw?$AAi?$AA_?$AAe?$AAv?$AAd?$AAo?$AAm?$AAx?$AA?4?$AAd?$AAl?$AAl?$AA?$AA@ 0014f2c8     misc.obj
 0002:0000e2e8       ??_C@_1BG@KCJLGFEC@?$AAs?$AAd?$AAk?$AAr?$AAi?$AAl?$AA?4?$AAd?$AAl?$AAl?$AA?$AA@ 0014f2e8     misc.obj
 0002:0000e300       ??_C@_1BI@BCCLBKHN@?$AAg?$AAo?$AAb?$AAi?$AAa?$AAp?$AAi?$AA?4?$AAd?$AAl?$AAl?$AA?$AA@ 0014f300     misc.obj
 0002:0000e318       ??_C@_1CO@FOGODAOI@?$AAm?$AAp?$AAF?$AAn?$AAS?$AAw?$AAi?$AAG?$AAe?$AAt?$AAI?$AAm?$AAe?$AAi?$AA?5?$AAi?$AAs?$AA?5?$AAN?$AAU?$AAL?$AAL?$AA?$AA@ 0014f318     misc.obj
 0002:0000e348       ??_C@_1CM@FGOALGJ@?$AAS?$AAw?$AAi?$AAG?$AAe?$AAt?$AAI?$AAm?$AAe?$AAi?$AA?5?$AAF?$AAA?$AAI?$AAL?$AAE?$AAD?$AA?5?$AA?$CF?$AAd?$AA?5?$AA?$AA@ 0014f348     misc.obj
 0002:0000e374       ??_C@_1DE@LEDHIPBL@?$AAm?$AAp?$AAF?$AAn?$AAS?$AAw?$AAi?$AAG?$AAe?$AAt?$AAG?$AAs?$AAm?$AAI?$AAM?$AAS?$AAI?$AA?5?$AAi?$AAs?$AA?5?$AAN?$AAU?$AAL?$AAL?$AA?$AA@ 0014f374     misc.obj
 0002:0000e3a8       ??_C@_1EM@IPHBPMH@?$AAm?$AAp?$AAF?$AAn?$AAS?$AAw?$AAi?$AAG?$AAe?$AAt?$AAG?$AAs?$AAm?$AAI?$AAM?$AAS?$AAI?$AA?5?$AAf?$AAa?$AAi?$AAl?$AAe?$AAd?$AA?0?$AA?5?$AAe?$AAr?$AAr?$AAo?$AAr?$AA?5@ 0014f3a8     misc.obj
 0002:0000e3f4       ??_C@_1O@JPOJDKNI@?$AA?$CF?$AAd?$AA?$CF?$AAd?$AA?$CF?$AAs?$AA?$AA@ 0014f3f4     misc.obj
 0002:0000e404       ??_C@_1DE@DIONHALM@?$AAm?$AAp?$AAF?$AAn?$AAS?$AAw?$AAi?$AAG?$AAe?$AAt?$AAE?$AAS?$AAN?$AAG?$AAo?$AAb?$AAi?$AA?5?$AAi?$AAs?$AA?5?$AAN?$AAU?$AAL?$AAL?$AA?$AA@ 0014f404     misc.obj
 0002:0000e438       ??_C@_1DK@EPIKMMNP@?$AAm?$AAp?$AAF?$AAn?$AAS?$AAw?$AAi?$AAG?$AAe?$AAt?$AAE?$AAS?$AAN?$AAG?$AAo?$AAb?$AAi?$AA?5?$AAF?$AAA?$AAI?$AAL?$AAE?$AAD?$AA?5?$AA?$CF?$AAd?$AA?5?$AA?$AA@ 0014f438     misc.obj
 0002:0000e474       ??_C@_1DA@MICMOHLL@?$AAm?$AAp?$AAF?$AAn?$AAS?$AAw?$AAi?$AAG?$AAe?$AAt?$AAE?$AAS?$AAN?$AAG?$AAo?$AAb?$AAi?$AA?5?$AA?3?$AA?5?$AA?$CF?$AAs?$AA?5?$AA?$AA@ 0014f474     misc.obj
 0002:0000e4a4       ??_C@_1DE@OMBBGIGA@?$AAm?$AAp?$AAF?$AAn?$AAS?$AAw?$AAi?$AAG?$AAe?$AAt?$AAM?$AAE?$AAI?$AAD?$AAE?$AAS?$AAN?$AA?5?$AAi?$AAs?$AA?5?$AAN?$AAU?$AAL?$AAL?$AA?$AA@ 0014f4a4     misc.obj
 0002:0000e4d8       ??_C@_1EM@DPBONAON@?$AAm?$AAp?$AAF?$AAn?$AAS?$AAw?$AAi?$AAG?$AAe?$AAt?$AAM?$AAE?$AAI?$AAD?$AAE?$AAS?$AAN?$AA?5?$AAf?$AAa?$AAi?$AAl?$AAe?$AAd?$AA?0?$AA?5?$AAe?$AAr?$AAr?$AAo?$AAr?$AA?5@ 0014f4d8     misc.obj
 0002:0000e528       ??_C@_1GE@NEIGAJEI@?$AAM?$AAE?$AAI?$AAD?$AA?5?$AAi?$AAs?$AA?5?$AAN?$AAO?$AAT?$AA?5?$AAe?$AAn?$AAa?$AAb?$AAl?$AAe?$AAd?$AA?0?$AA?5?$AAT?$AAR?$AAU?$AAE?$AA?5?$AAE?$AAS?$AAN?$AA?5?$AAm?$AAa@ 0014f528     misc.obj
 0002:0000e590       ??_C@_1HC@EJOMLCBB@?$AAM?$AAE?$AAI?$AAD?$AA?5?$AAi?$AAs?$AA?5?$AAe?$AAn?$AAa?$AAb?$AAl?$AAe?$AAd?$AA?5?$AAb?$AAu?$AAt?$AA?5?$AAN?$AAO?$AAT?$AA?5?$AAp?$AAr?$AAo?$AAv?$AAi?$AAs?$AAi?$AAo@ 0014f590     misc.obj
 0002:0000e604       ??_C@_05FOJCDADK@?$CF06lX?$AA@ 0014f604     misc.obj
 0002:0000e60c       ??_C@_05LOENEHAJ@?$CF08lX?$AA@ 0014f60c     misc.obj
 0002:0000e614       ??_C@_1DA@IEHKLHNK@?$AAS?$AAw?$AAi?$AAG?$AAe?$AAt?$AAB?$AAo?$AAo?$AAt?$AAV?$AAe?$AAr?$AAs?$AAi?$AAo?$AAn?$AA?5?$AA?3?$AA?5?$AA?$CF?$AAs?$AA?5?$AA?$AA@ 0014f614     misc.obj
 0002:0000e644       ??_C@_1CO@CKOLGFGF@?$AAS?$AAw?$AAi?$AAG?$AAe?$AAt?$AAP?$AAR?$AAL?$AAV?$AAe?$AAr?$AAs?$AAi?$AAo?$AAn?$AA?5?$AA?3?$AA?5?$AA?$CF?$AAd?$AA?5?$AA?$AA@ 0014f644     misc.obj
 0002:0000e674       ??_C@_1DI@EONFDNGF@?$AAS?$AAw?$AAi?$AAG?$AAe?$AAt?$AAH?$AAa?$AAr?$AAd?$AAw?$AAa?$AAr?$AAe?$AAV?$AAe?$AAr?$AAs?$AAi?$AAo?$AAn?$AA?5?$AA?3?$AA?5?$AA?$CF?$AAs?$AA?5?$AA?$AA@ 0014f674     misc.obj
 0002:0000e6ac       ??_C@_1DI@LGHFKLL@?$AAS?$AAw?$AAi?$AAG?$AAe?$AAt?$AAF?$AAi?$AAr?$AAm?$AAw?$AAa?$AAr?$AAe?$AAV?$AAe?$AAr?$AAs?$AAi?$AAo?$AAn?$AA?5?$AA?3?$AA?5?$AA?$CF?$AAs?$AA?5?$AA?$AA@ 0014f6ac     misc.obj
 0002:0000e6e8       ??_C@_1FE@DLEBKKKE@?$AAA?$AAS?$AAS?$AAE?$AAR?$AAT?$AAI?$AAO?$AAN?$AA?5?$AAF?$AAA?$AAI?$AAL?$AAU?$AAR?$AAE?$AA?3?$AA?5?$AA?$DN?$AA?$DN?$AA?$DN?$AA?$DO?$AAr?$AAc?$AA?5?$AA?$DN?$AA?$DN?$AA?5?$AAS?$AAW?$AAI@ 0014f6e8     misc.obj
 0002:0000e73c       ??_C@_1BI@FBPCKNIP@?$AAr?$AAi?$AAl?$AAc?$AAd?$AAm?$AAa?$AA?4?$AAd?$AAl?$AAl?$AA?$AA@ 0014f73c     misc.obj
 0002:0000e754       ??_C@_17DJMMGLBL@?$AAD?$AAl?$AAl?$AA?$AA@ 0014f754     misc.obj
 0002:0000e75c       ??_C@_1CI@IKLNBDDE@?$AAD?$AAr?$AAi?$AAv?$AAe?$AAr?$AAs?$AA?2?$AAB?$AAu?$AAi?$AAl?$AAt?$AAi?$AAn?$AA?2?$AAR?$AAI?$AAL?$AA?$AA@ 0014f75c     misc.obj
 0002:0000e784       ??_C@_1DM@PJADDEFD@?$AAG?$AAe?$AAt?$AAP?$AAr?$AAo?$AAd?$AAu?$AAc?$AAt?$AAV?$AAe?$AAr?$AAs?$AAi?$AAo?$AAn?$AAS?$AAt?$AAr?$AA?5?$AAR?$AAI?$AAL?$AA?3?$AA?5?$AA?$CF?$AAs?$AA?5?$AA?$AA@ 0014f784     misc.obj
 0002:0000e7c0       ??_C@_1DI@EFMHHOFE@?$AAm?$AAp?$AAF?$AAn?$AAS?$AAw?$AAi?$AAP?$AAs?$AAt?$AAG?$AAe?$AAt?$AAA?$AAc?$AAc?$AAo?$AAl?$AAc?$AA?5?$AAf?$AAa?$AAi?$AAl?$AAe?$AAd?$AA?4?$AA?$AA@ 0014f7c0     misc.obj
 0002:0000e7f8       ??_C@_1DO@CAPCDODC@?$AAm?$AAp?$AAF?$AAn?$AAS?$AAw?$AAi?$AAP?$AAs?$AAt?$AAG?$AAe?$AAt?$AAH?$AAo?$AAm?$AAe?$AAS?$AAi?$AAd?$AAN?$AAi?$AAd?$AA?5?$AAf?$AAa?$AAi?$AAl?$AAe?$AAd?$AA?$AA@ 0014f7f8     misc.obj
 0002:0000e838       ??_C@_1EO@BHJKNAAC@?$AAm?$AAp?$AAF?$AAn?$AAS?$AAw?$AAi?$AAG?$AAe?$AAt?$AAC?$AAD?$AAM?$AAA?$AAN?$AAe?$AAt?$AAw?$AAo?$AAr?$AAk?$AAP?$AAa?$AAr?$AAa?$AAm?$AAe?$AAt?$AAe?$AAr?$AAs?$AA?5@ 0014f838     misc.obj
 0002:0000e888       ??_C@_1EC@GOOCDHMA@?$AAS?$AAw?$AAi?$AAP?$AAs?$AAt?$AAS?$AAe?$AAt?$AAD?$AAs?$AAM?$AAi?$AAp?$AAA?$AAc?$AAt?$AAi?$AAv?$AAe?$AAP?$AAr?$AAo?$AAf?$AA?5?$AAr?$AAc?$AA?5?$AA?$DN?$AA?5?$AA?$CF?$AAd@ 0014f888     misc.obj
 0002:0000e8d0       ??_C@_1EG@BLCIAECM@?$AAT?$AAh?$AAe?$AA?5?$AAs?$AAy?$AAs?$AAt?$AAe?$AAm?$AA?5?$AAp?$AAr?$AAe?$AAf?$AAe?$AAr?$AAr?$AAe?$AAd?$AA?5?$AAm?$AAo?$AAd?$AAe?$AA?5?$AA?$DN?$AA?5?$AA?$CF?$AAd?$AA?0?$AA?5@ 0014f8d0     misc.obj
 0002:0000e918       ??_C@_1FC@LENIGPEJ@?$AAS?$AAw?$AAi?$AAP?$AAs?$AAt?$AAG?$AAe?$AAt?$AAD?$AAs?$AAM?$AAi?$AAp?$AAE?$AAn?$AAa?$AAb?$AAl?$AAe?$AAP?$AAr?$AAo?$AAf?$AA?5?$AAr?$AAe?$AAt?$AAu?$AAr?$AAn?$AAs@ 0014f918     misc.obj
 0002:0000e970       ??_C@_1EI@NOAGCHD@?$AAS?$AAw?$AAi?$AAS?$AAe?$AAt?$AAP?$AAs?$AAt?$AAL?$AAo?$AAc?$AAk?$AA?5?$AAr?$AAe?$AAt?$AAu?$AAr?$AAn?$AAs?$AA?5?$AAe?$AAr?$AAr?$AAo?$AAr?$AA?5?$AAr?$AAc?$AA?5?$AA?$DN@ 0014f970     misc.obj
 0002:0000e9b8       ??_C@_1IM@NHKEICMM@?$AAP?$AAo?$AAs?$AAs?$AAi?$AAb?$AAl?$AAe?$AA?5?$AAP?$AAr?$AAo?$AAv?$AAi?$AAs?$AAi?$AAo?$AAn?$AAn?$AAi?$AAn?$AAg?$AA?5?$AAp?$AAr?$AAo?$AAb?$AAl?$AAe?$AAm?$AA?0?$AA?5@ 0014f9b8     misc.obj
 0002:0000ea48       ??_C@_1EM@EIIIBLIF@?$AAS?$AAw?$AAi?$AAP?$AAs?$AAt?$AAS?$AAe?$AAt?$AAE?$AAv?$AAr?$AAc?$AAV?$AAo?$AAi?$AAc?$AAe?$AAS?$AAe?$AAr?$AAv?$AAi?$AAc?$AAe?$AA?5?$AAu?$AAn?$AAs?$AAu?$AAp?$AAp@ 0014fa48     misc.obj
 0002:0000ea98       ??_C@_1EC@GEGJODHJ@?$AAU?$AAn?$AAs?$AAu?$AAp?$AAp?$AAo?$AAr?$AAt?$AAe?$AAd?$AA?5?$AAe?$AAR?$AAo?$AAa?$AAm?$AAP?$AAr?$AAe?$AAf?$AAC?$AAa?$AAl?$AAl?$AAS?$AAO?$AA?5?$AA?$DN?$AA?5?$AA?$CF?$AAd@ 0014fa98     misc.obj
 0002:0000eae0       ??_C@_1EK@MAFGMDGL@?$AAU?$AAn?$AAs?$AAu?$AAp?$AAp?$AAo?$AAr?$AAt?$AAe?$AAd?$AA?5?$AAe?$AAH?$AAo?$AAm?$AAe?$AAO?$AAr?$AAi?$AAg?$AAP?$AAr?$AAe?$AAf?$AAC?$AAa?$AAl?$AAl?$AAS?$AAO?$AA?5@ 0014fae0     misc.obj
 0002:0000eb30       ??_C@_1EK@LMMBKFIJ@?$AAU?$AAn?$AAs?$AAu?$AAp?$AAp?$AAo?$AAr?$AAt?$AAe?$AAd?$AA?5?$AAe?$AAH?$AAo?$AAm?$AAe?$AAP?$AAa?$AAg?$AAe?$AAP?$AAr?$AAe?$AAf?$AAC?$AAa?$AAl?$AAl?$AAS?$AAO?$AA?5@ 0014fb30     misc.obj
 0002:0000eb80       ??_C@_1GG@DMAKKFML@?$AAU?$AAs?$AAe?$AAr?$AA?5?$AAh?$AAa?$AAs?$AA?5?$AAe?$AAn?$AAt?$AAe?$AAr?$AAe?$AAd?$AA?5?$AAa?$AAn?$AA?5?$AAi?$AAn?$AAv?$AAa?$AAl?$AAi?$AAd?$AA?5?$AAM?$AAI?$AAN?$AA1@ 0014fb80     misc.obj
 0002:0000ebe8       ??_C@_1CO@ICEELGH@?$AAR?$AAe?$AAa?$AAd?$AA?5?$AAE?$AAS?$AAN?$AA?5?$AAf?$AAa?$AAi?$AAl?$AA?0?$AA?5?$AAr?$AAc?$AA?5?$AA?$DN?$AA?5?$AA?$CF?$AAd?$AA?$AA@ 0014fbe8     misc.obj
 0002:0000ec18       ??_C@_1EO@FLPHODML@?$AAT?$AAh?$AAe?$AA?5?$AAM?$AAI?$AAN?$AA?5?$AA?$CI?$AA?$DN?$AA?$CF?$AAs?$AA?$CJ?$AA?5?$AAi?$AAs?$AA?5?$AAn?$AAo?$AAt?$AA?5?$AAi?$AAn?$AA?5?$AAp?$AAr?$AAo?$AAp?$AAe?$AAr?$AA?5?$AAf@ 0014fc18     misc.obj
 0002:0000ec68       ??_C@_15KNBIKKIN@?$AA?$CF?$AAd?$AA?$AA@ 0014fc68     misc.obj
 0002:0000ec70       ??_C@_1EG@EFNMIGIA@?$AAG?$AAe?$AAt?$AA?5?$AAN?$AAV?$AA?5?$AAi?$AAt?$AAe?$AAm?$AA?5?$AA?$DN?$AA?5?$AA?$CF?$AAd?$AA?5?$AAn?$AAo?$AAt?$AA?5?$AAs?$AAu?$AAp?$AAp?$AAo?$AAr?$AAt?$AAe?$AAd?$AA?5?$AAy@ 0014fc70     misc.obj
 0002:0000ecb8       ??_C@_1EA@KEPNAKLJ@?$AAS?$AAw?$AAi?$AAP?$AAs?$AAt?$AAG?$AAe?$AAt?$AAT?$AAe?$AAr?$AAm?$AAN?$AAi?$AAd?$AA?5?$AAf?$AAa?$AAi?$AAl?$AAe?$AAd?$AA?5?$AAr?$AAc?$AA?5?$AA?$DN?$AA?5?$AA?$CF?$AAd?$AA?$AA@ 0014fcb8     misc.obj
 0002:0000ecf8       ??_C@_1EA@HABGADOL@?$AAS?$AAw?$AAi?$AAP?$AAs?$AAt?$AAG?$AAe?$AAt?$AAT?$AAe?$AAr?$AAm?$AAS?$AAi?$AAd?$AA?5?$AAf?$AAa?$AAi?$AAl?$AAe?$AAd?$AA?5?$AAr?$AAc?$AA?5?$AA?$DN?$AA?5?$AA?$CF?$AAd?$AA?$AA@ 0014fcf8     misc.obj
 0002:0000ed38       ??_C@_1EC@DEOJOPGM@?$AAS?$AAw?$AAi?$AAP?$AAs?$AAt?$AAG?$AAe?$AAt?$AAT?$AAe?$AAr?$AAm?$AAH?$AAo?$AAm?$AAe?$AA?5?$AAf?$AAa?$AAi?$AAl?$AAe?$AAd?$AA?5?$AAr?$AAc?$AA?5?$AA?$DN?$AA?5?$AA?$CF?$AAd@ 0014fd38     misc.obj
 0002:0000ed80       ??_C@_1EA@MNEKFDHO@?$AAS?$AAw?$AAi?$AAP?$AAs?$AAt?$AAG?$AAe?$AAt?$AAD?$AAs?$AAQ?$AAc?$AAM?$AAi?$AAp?$AA?5?$AAf?$AAa?$AAi?$AAl?$AAe?$AAd?$AA?5?$AAr?$AAc?$AA?5?$AA?$DN?$AA?5?$AA?$CF?$AAd?$AA?$AA@ 0014fd80     misc.obj
 0002:0000edc0       ??_C@_1EI@HAHPDCJA@?$AAS?$AAw?$AAi?$AAP?$AAs?$AAt?$AAG?$AAe?$AAt?$AAH?$AAd?$AAr?$AAP?$AAa?$AAs?$AAs?$AAw?$AAo?$AAr?$AAd?$AA?5?$AAf?$AAa?$AAi?$AAl?$AAe?$AAd?$AA?5?$AAr?$AAc?$AA?5?$AA?$DN@ 0014fdc0     misc.obj
 0002:0000ee08       ??_C@_1EE@DNNAMKOK@?$AAS?$AAw?$AAi?$AAP?$AAs?$AAt?$AAG?$AAe?$AAt?$AAH?$AAd?$AAr?$AAU?$AAs?$AAe?$AAr?$AAI?$AAd?$AA?5?$AAf?$AAa?$AAi?$AAl?$AAe?$AAd?$AA?5?$AAr?$AAc?$AA?5?$AA?$DN?$AA?5?$AA?$CF@ 0014fe08     misc.obj
 0002:0000ee50       ??_C@_1FG@GDCGKDKJ@?$AAS?$AAw?$AAi?$AAG?$AAe?$AAt?$AAG?$AAe?$AAn?$AAe?$AAr?$AAa?$AAl?$AAF?$AAe?$AAa?$AAt?$AAu?$AAr?$AAe?$AAS?$AAu?$AAp?$AAp?$AAo?$AAr?$AAt?$AA?5?$AAf?$AAa?$AAi?$AAl@ 0014fe50     misc.obj
 0002:0000eea8       ??_C@_1DK@NLFMMHEP@?$AAS?$AAw?$AAi?$AAG?$AAe?$AAt?$AAE?$AAS?$AAN?$AAG?$AAo?$AAb?$AAi?$AA?5?$AAf?$AAa?$AAi?$AAl?$AAe?$AAd?$AA?5?$AAr?$AAc?$AA?5?$AA?$DN?$AA?5?$AA?$CF?$AAd?$AA?$AA@ 0014fea8     misc.obj
 0002:0000eee8       ??_C@_1EA@JLHCHKJO@?$AAS?$AAw?$AAi?$AAP?$AAs?$AAt?$AAS?$AAe?$AAt?$AAD?$AAs?$AAQ?$AAc?$AAM?$AAi?$AAp?$AA?5?$AAf?$AAa?$AAi?$AAl?$AAe?$AAd?$AA?5?$AAr?$AAc?$AA?5?$AA?$DN?$AA?5?$AA?$CF?$AAd?$AA?$AA@ 0014fee8     misc.obj
 0002:0000ef28       ??_C@_1EE@EJKELOIH@?$AAS?$AAw?$AAi?$AAP?$AAs?$AAt?$AAS?$AAe?$AAt?$AAH?$AAd?$AAr?$AAU?$AAs?$AAe?$AAr?$AAI?$AAd?$AA?5?$AAf?$AAa?$AAi?$AAl?$AAe?$AAd?$AA?5?$AAr?$AAc?$AA?5?$AA?$DN?$AA?5?$AA?$CF@ 0014ff28     misc.obj
 0002:0000ef70       ??_C@_1EI@PGPANEBF@?$AAS?$AAw?$AAi?$AAP?$AAs?$AAt?$AAS?$AAe?$AAt?$AAH?$AAd?$AAr?$AAP?$AAa?$AAs?$AAs?$AAw?$AAo?$AAr?$AAd?$AA?5?$AAf?$AAa?$AAi?$AAl?$AAe?$AAd?$AA?5?$AAr?$AAc?$AA?5?$AA?$DN@ 0014ff70     misc.obj
 0002:0000efb8       ??_C@_1EG@GNABPEBK@?$AAS?$AAe?$AAt?$AA?5?$AAN?$AAV?$AA?5?$AAi?$AAt?$AAe?$AAm?$AA?5?$AA?$DN?$AA?5?$AA?$CF?$AAd?$AA?5?$AAn?$AAo?$AAt?$AA?5?$AAs?$AAu?$AAp?$AAp?$AAo?$AAr?$AAt?$AAe?$AAd?$AA?5?$AAy@ 0014ffb8     misc.obj
 0002:0000f000       ??_C@_1DO@KFPIBDIM@?$AAF?$AAa?$AAi?$AAl?$AA?5?$AAV?$AAa?$AAl?$AAi?$AAd?$AAa?$AAt?$AAe?$AA?5?$AAS?$AAP?$AAC?$AA?0?$AA?5?$AAr?$AAc?$AAC?$AAo?$AAd?$AAe?$AA?5?$AA?$DN?$AA?5?$AA?$CF?$AAd?$AA?$AA@ 00150000     misc.obj
 0002:0000f128       ??_C@_1GE@LPBGGGMO@?$AAH?$AAa?$AAn?$AAd?$AAl?$AAe?$AAS?$AAW?$AAI?$AAE?$AAm?$AAe?$AAr?$AAg?$AAe?$AAn?$AAc?$AAy?$AAL?$AAi?$AAs?$AAt?$AAN?$AAo?$AAt?$AAi?$AAf?$AAi?$AAc?$AAa?$AAt?$AAi@ 00150128     misc.obj
 0002:0000f190       ??_C@_1GM@DNPBGNNM@?$AAR?$AAI?$AAL?$AA?3?$AA?5?$AAC?$AAr?$AAi?$AAt?$AAi?$AAc?$AAa?$AAl?$AA?5?$AAe?$AAr?$AAr?$AAo?$AAr?$AA?5?$AAh?$AAa?$AAs?$AA?5?$AAo?$AAc?$AAc?$AAu?$AAr?$AAr?$AAe?$AAd@ 00150190     monitor.obj
 0002:0000f1fc       ??_C@_1BM@HDMPKJOP@?$AA?4?$AA?2?$AAm?$AAo?$AAn?$AAi?$AAt?$AAo?$AAr?$AA?4?$AAc?$AAp?$AAp?$AA?$AA@ 001501fc     monitor.obj
 0002:0000f218       ??_C@_1FA@JPDJNKKN@?$AAA?$AAS?$AAS?$AAE?$AAR?$AAT?$AAI?$AAO?$AAN?$AA?5?$AAF?$AAA?$AAI?$AAL?$AAU?$AAR?$AAE?$AA?3?$AA?5?$AA?$DN?$AA?$DN?$AA?$DN?$AA?$DO?$AAN?$AAU?$AAL?$AAL?$AA?5?$AA?$CB?$AA?$DN?$AA?5?$AAp@ 00150218     monitor.obj
 0002:0000f2a8       ??_C@_1GK@HMOLFDND@?$AAA?$AAS?$AAS?$AAE?$AAR?$AAT?$AAI?$AAO?$AAN?$AA?5?$AAF?$AAA?$AAI?$AAL?$AAU?$AAR?$AAE?$AA?3?$AA?5?$AA?$DN?$AA?$DN?$AA?$DN?$AA?$DO?$AAN?$AAU?$AAL?$AAL?$AA?5?$AA?$CB?$AA?$DN?$AA?5?$AAg@ 001502a8     monitor.obj
 0002:0000f318       ??_C@_1FG@CBHIFPKF@?$AAA?$AAS?$AAS?$AAE?$AAR?$AAT?$AAI?$AAO?$AAN?$AA?5?$AAF?$AAA?$AAI?$AAL?$AAU?$AAR?$AAE?$AA?3?$AA?5?$AA?$DN?$AA?$DN?$AA?$DN?$AA?$DO?$AA0?$AA?5?$AA?$CB?$AA?$DN?$AA?5?$AAd?$AAw?$AAR?$AAe@ 00150318     monitor.obj
 0002:0000f370       ??_C@_1FE@LOHMDHBM@?$AAA?$AAS?$AAS?$AAE?$AAR?$AAT?$AAI?$AAO?$AAN?$AA?5?$AAF?$AAA?$AAI?$AAL?$AAU?$AAR?$AAE?$AA?3?$AA?5?$AA?$DN?$AA?$DN?$AA?$DN?$AA?$DO?$AA0?$AA?5?$AA?$CB?$AA?$DN?$AA?5?$AAd?$AAw?$AAC?$AAm@ 00150370     monitor.obj
 0002:0000f3c8       ??_C@_1FI@OLMELOGJ@?$AAA?$AAS?$AAS?$AAE?$AAR?$AAT?$AAI?$AAO?$AAN?$AA?5?$AAF?$AAA?$AAI?$AAL?$AAU?$AAR?$AAE?$AA?3?$AA?5?$AA?$DN?$AA?$DN?$AA?$DN?$AA?$DO?$AAN?$AAU?$AAL?$AAL?$AA?5?$AA?$CB?$AA?$DN?$AA?5?$AAh@ 001503c8     monitor.obj
 0002:0000f444       ??_7CriticalSection@@6B@   00150444     msg.obj
 0002:0000f448       ??_C@_15BHOFONJE@?$AA?$CF?$AAX?$AA?$AA@ 00150448     msg.obj
 0002:0000f4b0       ??_C@_1BAG@HDODIGMH@?$AAM?$AAs?$AAg?$AAS?$AAe?$AAn?$AAd?$AAT?$AAh?$AAr?$AAe?$AAa?$AAd?$AAP?$AAr?$AAo?$AAc?$AA?5?$AAS?$AAM?$AAS?$AA_?$AAS?$AAe?$AAn?$AAd?$AAS?$AAt?$AAa?$AAt?$AAu?$AAs@ 001504b0     msg.obj
 0002:0000f5b8       ??_C@_1IM@NEIOCGIM@?$AAM?$AAs?$AAg?$AAS?$AAe?$AAn?$AAd?$AAT?$AAh?$AAr?$AAe?$AAa?$AAd?$AAP?$AAr?$AAo?$AAc?$AA?5?$AAS?$AAM?$AAS?$AA_?$AAS?$AAe?$AAn?$AAd?$AAS?$AAt?$AAa?$AAt?$AAu?$AAs@ 001505b8     msg.obj
 0002:0000f648       ??_C@_1JA@EGDPDKLI@?$AAM?$AAs?$AAg?$AAS?$AAe?$AAn?$AAd?$AAT?$AAh?$AAr?$AAe?$AAa?$AAd?$AAP?$AAr?$AAo?$AAc?$AA?5?$AAS?$AAM?$AAS?$AA_?$AAS?$AAe?$AAn?$AAd?$AAS?$AAt?$AAa?$AAt?$AAu?$AAs@ 00150648     msg.obj
 0002:0000f6d8       ??_C@_1BE@OONLMPMN@?$AA?4?$AA?2?$AAm?$AAs?$AAg?$AA?4?$AAc?$AAp?$AAp?$AA?$AA@ 001506d8     msg.obj
 0002:0000f6f0       ??_C@_1EO@JNNJILDK@?$AAA?$AAS?$AAS?$AAE?$AAR?$AAT?$AAI?$AAO?$AAN?$AA?5?$AAF?$AAA?$AAI?$AAL?$AAU?$AAR?$AAE?$AA?3?$AA?5?$AA?$DN?$AA?$DN?$AA?$DN?$AA?$DO?$AAp?$AAN?$AAo?$AAt?$AAi?$AAf?$AAy?$AA?5?$AA?$CB@ 001506f0     msg.obj
 0002:0000f740       ??_C@_1FK@CFJMENGE@?$AAR?$AAe?$AAc?$AAe?$AAi?$AAv?$AAe?$AAM?$AAs?$AAg?$AA?$CI?$AA?$CJ?$AA?3?$AAB?$AAr?$AAo?$AAa?$AAd?$AAc?$AAa?$AAs?$AAt?$AAR?$AAe?$AAa?$AAl?$AAB?$AAl?$AAo?$AAb?$AAN?$AAo@ 00150740     msg.obj
 0002:0000f7a0       ??_C@_1EG@GFBIDOM@?$AAR?$AAe?$AAc?$AAe?$AAi?$AAv?$AAe?$AAM?$AAs?$AAg?$AA?$CI?$AAR?$AAI?$AAL?$AA_?$AAM?$AAS?$AAG?$AAT?$AAY?$AAP?$AAE?$AA_?$AAI?$AAN?$AA_?$AAD?$AAE?$AAL?$AAI?$AAV?$AAE@ 001507a0     msg.obj
 0002:0000f7e8       ??_C@_1EE@IBDKAMFK@?$AAR?$AAe?$AAc?$AAe?$AAi?$AAv?$AAe?$AAM?$AAs?$AAg?$AA?$CI?$AAR?$AAI?$AAL?$AA_?$AAM?$AAS?$AAG?$AAT?$AAY?$AAP?$AAE?$AA_?$AAI?$AAN?$AA_?$AAS?$AAT?$AAA?$AAT?$AAU?$AAS@ 001507e8     msg.obj
 0002:0000f830       ??_C@_1FO@NBMOBOMO@?$AAR?$AAe?$AAc?$AAe?$AAi?$AAv?$AAe?$AAM?$AAs?$AAg?$AA?$CI?$AAR?$AAI?$AAL?$AA_?$AAM?$AAS?$AAG?$AAT?$AAY?$AAP?$AAE?$AA_?$AAB?$AAC?$AA_?$AAG?$AAE?$AAN?$AAE?$AAR?$AAA@ 00150830     msg.obj
 0002:0000f890       ??_C@_1EI@OIODJANI@?$AAR?$AAe?$AAc?$AAe?$AAi?$AAv?$AAe?$AAM?$AAs?$AAg?$AA?$CI?$AAn?$AAo?$AAt?$AA?5?$AAp?$AAr?$AAo?$AAc?$AAe?$AAs?$AAs?$AAe?$AAd?$AA?5?$AAt?$AAy?$AAp?$AAe?$AA?5?$AA?$DN?$AA?5@ 00150890     msg.obj
 0002:0000f8d8       ??_C@_1FC@IIAIDPO@?$AAR?$AAe?$AAc?$AAe?$AAi?$AAv?$AAe?$AAM?$AAs?$AAg?$AA?$CI?$AA?$CJ?$AA?3?$AA?5?$AAM?$AAs?$AAg?$AA?5?$AAm?$AAa?$AAs?$AAk?$AA?5?$AA?$DN?$AA?5?$AA0?$AAx?$AA?$CF?$AAx?$AA?0?$AA?5?$AAt@ 001508d8     msg.obj
 0002:0000f930       ??_C@_1BPK@GEGJNKEE@?$AAA?$AAS?$AAS?$AAE?$AAR?$AAT?$AAI?$AAO?$AAN?$AA?5?$AAF?$AAA?$AAI?$AAL?$AAU?$AAR?$AAE?$AA?3?$AA?5?$AA?$DN?$AA?$DN?$AA?$DN?$AA?$DO?$AAp?$AAR?$AAi?$AAl?$AAM?$AAs?$AAg?$AA?9?$AA?$DO@ 00150930     msg.obj
 0002:0000fb30       ??_C@_1EO@FCJHGAHF@?$AAA?$AAS?$AAS?$AAE?$AAR?$AAT?$AAI?$AAO?$AAN?$AA?5?$AAF?$AAA?$AAI?$AAL?$AAU?$AAR?$AAE?$AA?3?$AA?5?$AA?$DN?$AA?$DN?$AA?$DN?$AA?$DO?$AAp?$AAR?$AAi?$AAl?$AAM?$AAs?$AAg?$AA?5?$AA?$CB@ 00150b30     msg.obj
 0002:0000fb80       ??_C@_1CG@HFDCNKMN@?$AAC?$AAR?$AAa?$AAd?$AAi?$AAo?$AA?3?$AA?3?$AAR?$AAe?$AAc?$AAe?$AAi?$AAv?$AAe?$AAM?$AAs?$AAg?$AA?$AA@ 00150b80     msg.obj
 0002:0000fba8       ??_C@_1EM@CMOAHOKC@?$AAm?$AAp?$AAF?$AAn?$AAS?$AAw?$AAi?$AAG?$AAe?$AAt?$AAG?$AAs?$AAm?$AAS?$AAM?$AAS?$AAC?$AAA?$AAd?$AAd?$AAr?$AA?5?$AAf?$AAa?$AAi?$AAl?$AAe?$AAd?$AA?0?$AA?5?$AAr?$AAc@ 00150ba8     msg.obj
 0002:0000fbf8       ??_C@_1GE@MFOHMJEN@?$AAm?$AAp?$AAF?$AAn?$AAS?$AAw?$AAi?$AAG?$AAe?$AAt?$AAG?$AAs?$AAm?$AAS?$AAM?$AAS?$AAC?$AAA?$AAd?$AAd?$AAr?$AA?5?$AAr?$AAe?$AAt?$AAu?$AAr?$AAn?$AAe?$AAd?$AA?5?$AAE@ 00150bf8     msg.obj
 0002:0000fc60       ??_C@_1FC@IAIJAKKC@?$AAT?$AAh?$AAe?$AAr?$AAe?$AA?5?$AAi?$AAs?$AA?5?$AAn?$AAo?$AA?5?$AAS?$AAM?$AAS?$AAC?$AA?5?$AAa?$AAd?$AAd?$AAr?$AAe?$AAs?$AAs?$AA?5?$AAi?$AAn?$AA?5?$AAt?$AAh?$AAe?$AA?5@ 00150c60     msg.obj
 0002:0000fcb8       ??_C@_1EM@CDHNNDGO@?$AAm?$AAp?$AAF?$AAn?$AAS?$AAw?$AAi?$AAS?$AAe?$AAt?$AAG?$AAs?$AAm?$AAS?$AAM?$AAS?$AAC?$AAA?$AAd?$AAd?$AAr?$AA?5?$AAf?$AAa?$AAi?$AAl?$AAe?$AAd?$AA?0?$AA?5?$AAr?$AAc@ 00150cb8     msg.obj
 0002:0000fd60       ??_C@_1FI@CONEDHG@?$AAA?$AAS?$AAS?$AAE?$AAR?$AAT?$AAI?$AAO?$AAN?$AA?5?$AAF?$AAA?$AAI?$AAL?$AAU?$AAR?$AAE?$AA?3?$AA?5?$AA?$DN?$AA?$DN?$AA?$DN?$AA?$DO?$AAN?$AAU?$AAM?$AA_?$AAM?$AAS?$AAG?$AAL?$AAO@ 00150d60     msg.obj
 0002:0000fdb8       ??_C@_1BBI@IOLAIKB@?$AAA?$AAS?$AAS?$AAE?$AAR?$AAT?$AAI?$AAO?$AAN?$AA?5?$AAF?$AAA?$AAI?$AAL?$AAU?$AAR?$AAE?$AA?3?$AA?5?$AA?$DN?$AA?$DN?$AA?$DN?$AA?$DO?$AA?$CI?$AAR?$AAI?$AAL?$AA_?$AAM?$AAS?$AAG?$AAS@ 00150db8     msg.obj
 0002:0000ff40       ??_C@_1EI@EFHIJHHH@?$AAS?$AAw?$AAi?$AAR?$AAe?$AAt?$AAr?$AAi?$AAe?$AAv?$AAe?$AAS?$AAM?$AAS?$AAM?$AAe?$AAs?$AAs?$AAa?$AAg?$AAe?$AAG?$AAo?$AAb?$AAi?$AA?5?$AAF?$AAa?$AAi?$AAl?$AAe?$AAd@ 00150f40     msg.obj
 0002:0000ff88       ??_C@_1EA@ONBBBAOE@?$AAm?$AAs?$AAg?$AAc?$AAo?$AAu?$AAn?$AAt?$AA?5?$AAi?$AAs?$AA?5?$AAz?$AAe?$AAr?$AAo?$AA?5?$AAn?$AAo?$AA?5?$AAN?$AAe?$AAw?$AA?5?$AAm?$AAe?$AAs?$AAs?$AAa?$AAg?$AAe?$AA?$AA@ 00150f88     msg.obj
 0002:0000ffc8       ??_C@_1GI@OLKLDGE@?$AAS?$AAw?$AAi?$AAG?$AAe?$AAt?$AAS?$AAM?$AAS?$AAM?$AAe?$AAs?$AAs?$AAa?$AAg?$AAe?$AAS?$AAt?$AAa?$AAt?$AAu?$AAs?$AA?5?$AAF?$AAa?$AAi?$AAl?$AAe?$AAd?$AA?5?$AA?$CF?$AAd@ 00150fc8     msg.obj
 0002:00010030       ??_C@_1EM@FABCKFPE@?$AAA?$AAS?$AAS?$AAE?$AAR?$AAT?$AAI?$AAO?$AAN?$AA?5?$AAF?$AAA?$AAI?$AAL?$AAU?$AAR?$AAE?$AA?3?$AA?5?$AA?$DN?$AA?$DN?$AA?$DN?$AA?$DO?$AAp?$AAR?$AAa?$AAd?$AAi?$AAo?$AA?5?$AA?$CB?$AA?$DN@ 00151030     msg.obj
 0002:00010080       ??_C@_1EE@OMKBAFMP@?$AAM?$AAs?$AAg?$AAR?$AAe?$AAc?$AAe?$AAi?$AAv?$AAe?$AAO?$AAn?$AAN?$AAo?$AAt?$AAi?$AAf?$AAy?$AAT?$AAh?$AAr?$AAe?$AAa?$AAd?$AAP?$AAr?$AAo?$AAc?$AAG?$AAs?$AAm?$AA?$CI@ 00151080     msg.obj
 0002:00010138       ??_C@_1EI@GJIDJKBA@?$AAS?$AAw?$AAi?$AAR?$AAe?$AAt?$AAr?$AAi?$AAe?$AAv?$AAe?$AAC?$AAd?$AAm?$AAa?$AAS?$AAM?$AAS?$AAM?$AAe?$AAs?$AAs?$AAa?$AAg?$AAe?$AA?5?$AAF?$AAa?$AAi?$AAl?$AAe?$AAd@ 00151138     msg.obj
 0002:00010180       ??_C@_1KE@NBNMDBCI@?$AAV?$AAZ?$AAW?$AA?5?$AAi?$AAs?$AA?5?$AAm?$AAa?$AAk?$AAi?$AAn?$AAg?$AA?5?$AAa?$AA?5?$AAj?$AAo?$AAk?$AAe?$AA?4?$AA?5?$AAT?$AAh?$AAe?$AAy?$AA?5?$AAs?$AAe?$AAn?$AAd?$AA?5@ 00151180     msg.obj
 0002:00010228       ??_C@_1EE@DNNGFBLK@?$AAA?$AAd?$AAd?$AAr?$AAe?$AAs?$AAs?$AA?5?$AA?$DN?$AA?5?$AA?$CC?$AA6?$AA2?$AA4?$AA5?$AA?$CC?$AA?5?$AAa?$AAn?$AAd?$AA?5?$AAU?$AAS?$AAE?$AAR?$AA_?$AAD?$AAA?$AAT?$AAA?$AA?5?$AA?$DN@ 00151228     msg.obj
 0002:0001026c       ??_C@_19OGGOHMNO@?$AA6?$AA2?$AA4?$AA5?$AA?$AA@ 0015126c     msg.obj
 0002:00010278       ??_C@_1LG@IOCKJJCD@?$AAR?$AAI?$AAL?$AA?5?$AAd?$AAe?$AAt?$AAe?$AAc?$AAt?$AAs?$AA?5?$AAu?$AAn?$AAs?$AAu?$AAp?$AAp?$AAo?$AAr?$AAt?$AAe?$AAd?$AA?5?$AAe?$AAn?$AAc?$AAo?$AAd?$AAi?$AAn?$AAg@ 00151278     msg.obj
 0002:00010330       ??_C@_1EO@ENHPOGGF@?$AAS?$AAw?$AAi?$AAR?$AAe?$AAt?$AAr?$AAi?$AAe?$AAv?$AAe?$AAC?$AAd?$AAm?$AAa?$AAS?$AAM?$AAS?$AAM?$AAe?$AAs?$AAs?$AAa?$AAg?$AAe?$AA?$CI?$AA?$CJ?$AA?5?$AAM?$AAs?$AAg?$AAI@ 00151330     msg.obj
 0002:00010380       ??_C@_1CK@JOHCANCG@?$AAI?$AAn?$AAi?$AAt?$AAi?$AAa?$AAl?$AA?5?$AAO?$AAr?$AAi?$AAg?$AA?5?$AAA?$AAd?$AAd?$AAr?$AA?5?$AA?$DN?$AA?5?$AA?$AA@ 00151380     msg.obj
 0002:000103b0       ??_C@_1FC@GJDDLFPG@?$AAF?$AAI?$AAN?$AAA?$AAL?$AA?5?$AAI?$AAn?$AAc?$AAo?$AAm?$AAi?$AAn?$AAg?$AA?5?$AAC?$AAD?$AAM?$AAA?$AA?5?$AAM?$AAe?$AAs?$AAs?$AAa?$AAg?$AAe?$AA?5?$AAt?$AAy?$AAp?$AAe@ 001513b0     msg.obj
 0002:00010404       ??_C@_1DM@JBLLCNNG@?$AAW?$AAA?$AAP?$AA?5?$AAS?$AAM?$AAS?$AA?5?$AAr?$AAe?$AAc?$AAe?$AAi?$AAv?$AAe?$AAd?$AA?4?$AA?5?$AAI?$AAg?$AAn?$AAo?$AAr?$AAe?$AAd?$AA?5?$AAi?$AAt?$AA?$CB?$AA?$AA@ 00151404     msg.obj
 0002:00010440       ??_C@_1DE@HJIJLINA@?$AAU?$AAn?$AAh?$AAa?$AAn?$AAd?$AAl?$AAe?$AAd?$AA?5?$AAM?$AAS?$AAG?$AAI?$AAD?$AA?5?$AAT?$AAy?$AAp?$AAe?$AA?5?$AA?$DN?$AA?5?$AA?$CF?$AAd?$AA?$AA@ 00151440     msg.obj
 0002:00010474       ??_C@_1DI@PEONACEF@?$AAG?$AAo?$AAt?$AA?5?$AAD?$AAi?$AAl?$AAv?$AAe?$AAr?$AAy?$AA?5?$AAA?$AAc?$AAk?$AA?5?$AAo?$AAr?$AA?5?$AAU?$AAs?$AAe?$AAr?$AA?5?$AAA?$AAc?$AAk?$AA?$AA@ 00151474     msg.obj
 0002:000104b0       ??_C@_1IK@FIMKIPMD@?$AAR?$AAe?$AAc?$AAe?$AAi?$AAv?$AAe?$AAd?$AA?5?$AAS?$AAM?$AAS?$AA?5?$AAm?$AAe?$AAs?$AAs?$AAa?$AAg?$AAe?$AA?5?$AAw?$AAi?$AAt?$AAh?$AA?5?$AAM?$AAs?$AAg?$AAI?$AAd?$AA?5@ 001514b0     msg.obj
 0002:00010540       ??_C@_1GO@CGMMPELJ@?$AAS?$AAw?$AAi?$AAG?$AAe?$AAt?$AAC?$AAd?$AAm?$AAa?$AAM?$AAS?$AAM?$AAe?$AAs?$AAs?$AAa?$AAg?$AAe?$AAS?$AAt?$AAa?$AAt?$AAu?$AAs?$AA?5?$AAF?$AAa?$AAi?$AAl?$AAe?$AAd@ 00151540     msg.obj
 0002:000105b0       ??_C@_1DO@DHCPOLEI@?$AAM?$AAs?$AAg?$AAR?$AAe?$AAc?$AAe?$AAi?$AAv?$AAe?$AAO?$AAn?$AAN?$AAo?$AAt?$AAi?$AAf?$AAy?$AAT?$AAh?$AAr?$AAe?$AAa?$AAd?$AAP?$AAr?$AAo?$AAc?$AA?$CI?$AA?$CJ?$AA?$AA@ 001515b0     msg.obj
 0002:00010630       ??_C@_1BCC@FKINOFAB@?$AAS?$AAe?$AAn?$AAd?$AAi?$AAn?$AAg?$AA?5?$AAS?$AAM?$AAS?$AA?5?$AAm?$AAe?$AAs?$AAs?$AAa?$AAg?$AAe?$AA?5?$AAw?$AAi?$AAt?$AAh?$AA?5?$AAg?$AA_?$AAn?$AAM?$AAs?$AAg?$AAI@ 00151630     msg.obj
 0002:00010758       ??_C@_1HA@KIPMFHFK@?$AAM?$AAO?$AA?5?$AAS?$AAM?$AAS?$AA?5?$AAp?$AAa?$AAy?$AAl?$AAo?$AAa?$AAd?$AA?5?$AAc?$AAo?$AAr?$AAr?$AAu?$AAp?$AAt?$AAi?$AAo?$AAn?$AA?$CB?$AA?$CB?$AA?$CB?$AA?0?$AA?5?$AAs?$AAC@ 00151758     msg.obj
 0002:000107c8       ??_C@_1DI@HPKENKAE@?$AAU?$AAn?$AAh?$AAa?$AAn?$AAd?$AAl?$AAe?$AAd?$AA?5?$AAR?$AAI?$AAL?$AA?5?$AAp?$AAr?$AAi?$AAo?$AAr?$AAi?$AAt?$AAy?$AA?5?$AA?$DN?$AA?5?$AA?$CF?$AAd?$AA?$AA@ 001517c8     msg.obj
 0002:00010800       ??_C@_1IM@BPNDMKJA@?$AAM?$AAS?$AA?5?$AAs?$AAe?$AAt?$AAs?$AA?5?$AAB?$AAE?$AAA?$AAR?$AAE?$AAR?$AAR?$AAE?$AAP?$AAL?$AAY?$AAA?$AAC?$AAK?$AA?5?$AAb?$AAu?$AAt?$AA?5?$AAb?$AAe?$AAa?$AAr?$AAe@ 00151800     msg.obj
 0002:00010890       ??_C@_1JI@HHLFCEAB@?$AAN?$AAo?$AA?5?$AAd?$AAe?$AAs?$AAt?$AAi?$AAn?$AAa?$AAt?$AAi?$AAo?$AAn?$AA?5?$AAn?$AAu?$AAm?$AAb?$AAe?$AAr?$AA?5?$AAf?$AAo?$AAu?$AAn?$AAd?$AA?4?$AA?5?$AAW?$AAh?$AAe@ 00151890     msg.obj
 0002:00010928       ??_C@_1NI@DPMFOOG@?$AAN?$AAo?$AA?5?$AAd?$AAe?$AAs?$AAt?$AAi?$AAn?$AAa?$AAt?$AAi?$AAo?$AAn?$AA?5?$AAn?$AAu?$AAm?$AAb?$AAe?$AAr?$AA?5?$AAf?$AAo?$AAu?$AAn?$AAd?$AA?4?$AA?5?$AAW?$AAh?$AAe@ 00151928     msg.obj
 0002:00010a00       ??_C@_13KJIIAINM@?$AA?$CL?$AA?$AA@ 00151a00     msg.obj
 0002:00010a08       ??_C@_1JK@MCDKECGG@?$AA?3?$AA?3?$AAS?$AAe?$AAn?$AAd?$AAM?$AAs?$AAg?$AA?$CB?$AA?5?$AAp?$AAR?$AAs?$AAp?$AA?5?$AA?$DN?$AA?5?$AA0?$AAx?$AA?$CF?$AAx?$AA?0?$AA?5?$AAg?$AA_?$AAn?$AAM?$AAs?$AAg?$AAI?$AAD@ 00151a08     msg.obj
 0002:00010aa8       ??_C@_1EG@LHBODBOI@?$AAm?$AAp?$AAF?$AAn?$AAS?$AAw?$AAi?$AAS?$AAe?$AAn?$AAd?$AAS?$AAM?$AAS?$AA?5?$AAr?$AAe?$AAt?$AAu?$AAr?$AAn?$AAe?$AAd?$AA?5?$AAE?$AAR?$AAR?$AAO?$AAR?$AA?5?$AA?$DN?$AA?5@ 00151aa8     msg.obj
 0002:00010af0       ??_C@_1FO@IOBOEKG@?$AAm?$AAp?$AAF?$AAn?$AAS?$AAw?$AAi?$AAS?$AAt?$AAo?$AAr?$AAe?$AAS?$AAM?$AAS?$AAM?$AAe?$AAs?$AAs?$AAa?$AAg?$AAe?$AAG?$AAo?$AAb?$AAi?$AA?5?$AAr?$AAe?$AAt?$AAu?$AAr@ 00151af0     msg.obj
 0002:00010b50       ??_C@_1GC@EAKIEFHA@?$AAI?$AAn?$AAv?$AAa?$AAl?$AAi?$AAd?$AA?5?$AAO?$AAr?$AAi?$AAg?$AAi?$AAn?$AAa?$AAl?$AA?5?$AAd?$AAe?$AAs?$AAt?$AAi?$AAn?$AAa?$AAt?$AAi?$AAo?$AAn?$AA?5?$AAa?$AAd?$AAd@ 00151b50     msg.obj
 0002:00010bb8       ??_C@_1FM@GAKCBAIE@?$AAI?$AAn?$AAv?$AAa?$AAl?$AAi?$AAd?$AA?5?$AAF?$AAi?$AAn?$AAa?$AAl?$AA?5?$AAd?$AAe?$AAs?$AAt?$AAi?$AAn?$AAa?$AAt?$AAi?$AAo?$AAn?$AA?5?$AAa?$AAd?$AAd?$AAr?$AAe?$AAs@ 00151bb8     msg.obj
 0002:00010c14       ??_C@_1M@BNIGDGDD@?$AA3?$AA6?$AA2?$AA4?$AA5?$AA?$AA@ 00151c14     msg.obj
 0002:00010c20       ??_C@_17KDKBICID@?$AA5?$AA0?$AA0?$AA?$AA@ 00151c20     msg.obj
 0002:00010c28       ??_C@_1BC@NMOKCBPG@?$AAT?$AA?9?$AAM?$AAo?$AAb?$AAi?$AAl?$AAe?$AA?$AA@ 00151c28     msg.obj
 0002:00010c40       ??_C@_1GI@COMLJFLD@?$AAC?$AAu?$AAr?$AAr?$AAe?$AAn?$AAt?$AAl?$AAy?$AA?5?$AAw?$AAe?$AA?5?$AAd?$AAo?$AA?5?$AAN?$AAO?$AAT?$AA?5?$AAh?$AAa?$AAn?$AAd?$AAl?$AAe?$AA?5?$AAt?$AAh?$AAe?$AA?5?$AAm@ 00151c40     msg.obj
 0002:00010ca8       ??_C@_1EI@PGOLDMFC@?$AA?3?$AA?3?$AAS?$AAe?$AAn?$AAd?$AAM?$AAs?$AAg?$AA?$CB?$AA?5?$AAp?$AAR?$AAi?$AAl?$AAM?$AAs?$AAg?$AA?9?$AA?$DO?$AAd?$AAw?$AAP?$AAa?$AAr?$AAa?$AAm?$AAs?$AA?5?$AA?$DN?$AA?5?$AA0@ 00151ca8     msg.obj
 0002:00010cf0       ??_C@_1DA@HEPIIPAO@?$AA?3?$AA?3?$AAS?$AAe?$AAn?$AAd?$AAM?$AAs?$AAg?$AA?$CB?$AA?5?$AAp?$AAR?$AAi?$AAl?$AAM?$AAs?$AAg?$AA?5?$AAN?$AAU?$AAL?$AAL?$AA?$AA@ 00151cf0     msg.obj
 0002:00010d20       ??_C@_1FI@HIJGOPNJ@?$AAA?$AAS?$AAS?$AAE?$AAR?$AAT?$AAI?$AAO?$AAN?$AA?5?$AAF?$AAA?$AAI?$AAL?$AAU?$AAR?$AAE?$AA?3?$AA?5?$AA?$DN?$AA?$DN?$AA?$DN?$AA?$DO?$AAh?$AAS?$AAM?$AAS?$AAS?$AAt?$AAa?$AAt?$AAu@ 00151d20     msg.obj
 0002:00010d78       ??_C@_1HM@LCGPEIGN@?$AAU?$AAp?$AAd?$AAa?$AAt?$AAe?$AAA?$AAn?$AAd?$AAB?$AAr?$AAo?$AAa?$AAd?$AAc?$AAa?$AAs?$AAt?$AAO?$AAn?$AAS?$AAW?$AAI?$AAS?$AAM?$AAS?$AAN?$AAo?$AAt?$AAi?$AAf?$AAi@ 00151d78     msg.obj
 0002:00010df8       ??_C@_1HO@BGKIIBCF@?$AAU?$AAp?$AAd?$AAa?$AAt?$AAe?$AAA?$AAn?$AAd?$AAB?$AAr?$AAo?$AAa?$AAd?$AAc?$AAa?$AAs?$AAt?$AAO?$AAn?$AAS?$AAW?$AAI?$AAS?$AAM?$AAS?$AAN?$AAo?$AAt?$AAi?$AAf?$AAi@ 00151df8     msg.obj
 0002:00010e78       ??_C@_1IC@BGGCDPNM@?$AAG?$AAS?$AAM?$AA?3?$AA?5?$AAR?$AAI?$AAL?$AA_?$AAN?$AAO?$AAT?$AAI?$AAF?$AAY?$AA_?$AAS?$AAM?$AAS?$AA_?$AAS?$AAE?$AAN?$AAD?$AA_?$AAS?$AAT?$AAA?$AAT?$AAU?$AAS?$AA?5@ 00151e78     msg.obj
 0002:00010f00       ??_C@_1IC@GKMJPJI@?$AAC?$AAD?$AAM?$AAA?$AA?3?$AA?5?$AAR?$AAI?$AAL?$AA_?$AAN?$AAO?$AAT?$AAI?$AAF?$AAY?$AA_?$AAS?$AAM?$AAS?$AA_?$AAS?$AAE?$AAN?$AAD?$AA_?$AAS?$AAT?$AAA?$AAT?$AAU?$AAS@ 00151f00     msg.obj
 0002:00010f88       ??_C@_1IE@LJBDIDB@?$AAU?$AAp?$AAd?$AAa?$AAt?$AAe?$AAA?$AAn?$AAd?$AAB?$AAr?$AAo?$AAa?$AAd?$AAc?$AAa?$AAs?$AAt?$AAO?$AAn?$AAS?$AAW?$AAI?$AAS?$AAM?$AAS?$AAN?$AAo?$AAt?$AAi?$AAf?$AAi@ 00151f88     msg.obj
 0002:00011010       ??_C@_1HE@EPENBEEP@?$AAU?$AAp?$AAd?$AAa?$AAt?$AAe?$AAA?$AAn?$AAd?$AAB?$AAr?$AAo?$AAa?$AAd?$AAc?$AAa?$AAs?$AAt?$AAO?$AAn?$AAS?$AAW?$AAI?$AAS?$AAM?$AAS?$AAN?$AAo?$AAt?$AAi?$AAf?$AAi@ 00152010     msg.obj
 0002:00011084       ??_C@_1DE@PJFGBEO@?$AAB?$AAe?$AAf?$AAo?$AAr?$AAe?$AA?5?$AAs?$AAe?$AAn?$AAd?$AA?5?$AAM?$AAe?$AAs?$AAs?$AAa?$AAg?$AAe?$AA?5?$AAt?$AAo?$AA?5?$AAU?$AAI?$AA?$AA@ 00152084     msg.obj
 0002:000110b8       ??_C@_1DA@PIJIFMKJ@?$AAC?$AAD?$AAM?$AAA?$AA?5?$AAn?$AAo?$AAt?$AA?5?$AAs?$AAu?$AAp?$AAp?$AAo?$AAr?$AAt?$AA?5?$AAS?$AAM?$AAS?$AA?9?$AAC?$AAB?$AA?$AA@ 001520b8     msg.obj
 0002:000110e8       ??_C@_1HG@HFLFAAKB@?$AAU?$AAp?$AAd?$AAa?$AAt?$AAe?$AAA?$AAn?$AAd?$AAB?$AAr?$AAo?$AAa?$AAd?$AAc?$AAa?$AAs?$AAt?$AAO?$AAn?$AAS?$AAW?$AAI?$AAS?$AAM?$AAS?$AAN?$AAo?$AAt?$AAi?$AAf?$AAi@ 001520e8     msg.obj
 0002:00011160       ??_C@_1DO@GCAJAHAO@?$AAB?$AAe?$AAf?$AAo?$AAr?$AAe?$AA?5?$AAs?$AAe?$AAn?$AAd?$AA?5?$AAV?$AAo?$AAi?$AAc?$AAe?$AAM?$AAe?$AAs?$AAs?$AAa?$AAg?$AAe?$AA?5?$AAt?$AAo?$AA?5?$AAU?$AAI?$AA?$AA@ 00152160     msg.obj
 0002:000111a0       ??_C@_1EK@MHHPODOE@?$AAs?$AAe?$AAt?$AAt?$AAi?$AAn?$AAg?$AA?5?$AAv?$AAo?$AAi?$AAc?$AAe?$AAm?$AAa?$AAi?$AAl?$AA?5?$AAn?$AAu?$AAm?$AAb?$AAe?$AAr?$AA?5?$AAb?$AAy?$AA?5?$AAr?$AAe?$AAg?$AAi@ 001521a0     msg.obj
 0002:000111f0       ??_C@_1FC@EEMOLNHA@?$AAS?$AAy?$AAs?$AAt?$AAe?$AAm?$AA?2?$AAS?$AAt?$AAa?$AAt?$AAe?$AA?2?$AAM?$AAe?$AAs?$AAs?$AAa?$AAg?$AAe?$AAs?$AA?2?$AAv?$AAm?$AAa?$AAi?$AAl?$AA?2?$AAL?$AAi?$AAn?$AAe@ 001521f0     msg.obj
 0002:00011244       ??_C@_1M@NBCIMFHI@?$AAC?$AAo?$AAu?$AAn?$AAt?$AA?$AA@ 00152244     msg.obj
 0002:00011250       ??_C@_1FC@BMAEDEOP@?$AAS?$AAy?$AAs?$AAt?$AAe?$AAm?$AA?2?$AAS?$AAt?$AAa?$AAt?$AAe?$AA?2?$AAM?$AAe?$AAs?$AAs?$AAa?$AAg?$AAe?$AAs?$AA?2?$AAv?$AAm?$AAa?$AAi?$AAl?$AA?2?$AAT?$AAo?$AAt?$AAa@ 00152250     msg.obj
 0002:000112a8       ??_C@_1FC@BPAKOKOC@?$AAS?$AAW?$AAI?$AA_?$AAN?$AAO?$AAT?$AAI?$AAF?$AAY?$AA_?$AAV?$AAo?$AAi?$AAc?$AAe?$AAM?$AAe?$AAs?$AAs?$AAa?$AAg?$AAe?$AA?5?$AAr?$AAe?$AAv?$AAi?$AAc?$AAe?$AAd?$AA?$CB@ 001522a8     msg.obj
 0002:00011300       ??_C@_1GE@BJCLHOAF@?$AAU?$AAp?$AAd?$AAa?$AAt?$AAe?$AAA?$AAn?$AAd?$AAB?$AAr?$AAo?$AAa?$AAd?$AAc?$AAa?$AAs?$AAt?$AAO?$AAn?$AAS?$AAW?$AAI?$AAS?$AAM?$AAS?$AAN?$AAo?$AAt?$AAi?$AAf?$AAi@ 00152300     msg.obj
 0002:00011368       ??_C@_1EM@ONMBGJKG@?$AAA?$AAS?$AAS?$AAE?$AAR?$AAT?$AAI?$AAO?$AAN?$AA?5?$AAF?$AAA?$AAI?$AAL?$AAU?$AAR?$AAE?$AA?3?$AA?5?$AA?$DN?$AA?$DN?$AA?$DN?$AA?$DO?$AAh?$AAD?$AAu?$AAm?$AAm?$AAy?$AA?5?$AA?$CB?$AA?$DN@ 00152368     msg.obj
 0002:000113b4       ??_C@_07IPEJGJKK@Thuraya?$AA@ 001523b4     network.obj
 0002:000113bc       ??_C@_02OGMJIJNC@SR?$AA@   001523bc     network.obj
 0002:000113c0       ??_C@_04MELNFAN@ICMS?$AA@  001523c0     network.obj
 0002:000113c8       ??_C@_05BOJJOFMO@PY?502?$AA@ 001523c8     network.obj
 0002:000113d0       ??_C@_02HHLOOEA@PY?$AA@    001523d0     network.obj
 0002:000113d4       ??_C@_03DJHJGNDM@VOX?$AA@  001523d4     network.obj
 0002:000113d8       ??_C@_05JIJJPEHM@ENTEL?$AA@ 001523d8     network.obj
 0002:000113e0       ??_C@_02EEBCMIJ@BO?$AA@    001523e0     network.obj
 0002:000113e4       ??_C@_08NFOFNJHM@NUEVATEL?$AA@ 001523e4     network.obj
 0002:000113f0       ??_C@_07MPNFALBA@DIGITEL?$AA@ 001523f0     network.obj
 0002:000113f8       ??_C@_02OFIBMPKP@VE?$AA@   001523f8     network.obj
 0002:000113fc       ??_C@_07GINECJOI@INFONET?$AA@ 001523fc     network.obj
 0002:00011404       ??_C@_02COKOBFHN@CL?$AA@   00152404     network.obj
 0002:00011408       ??_C@_09CEPFPDKF@ENTEL?5PCS?$AA@ 00152408     network.obj
 0002:00011414       ??_C@_06DEILFLKD@BrTCel?$AA@ 00152414     network.obj
 0002:0001141c       ??_C@_05KNLJOHOC@Claro?$AA@ 0015241c     network.obj
 0002:00011424       ??_C@_02PLCNEAJF@BR?$AA@   00152424     network.obj
 0002:00011428       ??_C@_0L@OFGFOAIG@TIM?5BRASIL?$AA@ 00152428     network.obj
 0002:00011434       ??_C@_0L@ODNOKFCA@PORT?9HABLE?$AA@ 00152434     network.obj
 0002:00011440       ??_C@_0BB@CCJOKBAE@Telecom?5Personal?$AA@ 00152440     network.obj
 0002:00011454       ??_C@_02PJGLPOMM@AR?$AA@   00152454     network.obj
 0002:00011458       ??_C@_06NIIMBICC@UNIFON?$AA@ 00152458     network.obj
 0002:00011460       ??_C@_02OBAMLDBN@PE?$AA@   00152460     network.obj
 0002:00011464       ??_C@_07CBLGEDG@DIGICEL?$AA@ 00152464     network.obj
 0002:0001146c       ??_C@_02ICKFEMNG@SV?$AA@   0015246c     network.obj
 0002:00011470       ??_C@_08LIHFODAB@PERSONAL?$AA@ 00152470     network.obj
 0002:0001147c       ??_C@_0BB@LFNDMJBC@Cell?5C?5?$CIPty?$CJ?5Ltd?$AA@ 0015247c     network.obj
 0002:00011490       ??_C@_02IIPHPDMP@ZA?$AA@   00152490     network.obj
 0002:00011494       ??_C@_02COBAADNK@SZ?$AA@   00152494     network.obj
 0002:00011498       ??_C@_08ILNHBGKG@SwaziMTN?$AA@ 00152498     network.obj
 0002:000114a4       ??_C@_05JKGGNHOK@VISTA?$AA@ 001524a4     network.obj
 0002:000114ac       ??_C@_02IGFKLENA@BW?$AA@   001524ac     network.obj
 0002:000114b0       ??_C@_06ELEIFEIM@MASCOM?$AA@ 001524b0     network.obj
 0002:000114b8       ??_C@_02OIKIFMNO@LS?$AA@   001524b8     network.obj
 0002:000114bc       ??_C@_02INAGPDON@MW?$AA@   001524bc     network.obj
 0002:000114c0       ??_C@_0N@PMKNDHNJ@CALLPOINT?590?$AA@ 001524c0     network.obj
 0002:000114d0       ??_C@_02JDNIPIGD@NA?$AA@   001524d0     network.obj
 0002:000114d4       ??_C@_03HCEDKKJ@MTC?$AA@   001524d4     network.obj
 0002:000114d8       ??_C@_02JEGPEGBI@ZW?$AA@   001524d8     network.obj
 0002:000114dc       ??_C@_07JIOKIEDC@NET?$CKONE?$AA@ 001524dc     network.obj
 0002:000114e4       ??_C@_0M@IDJJAGAM@SFR?5Reunion?$AA@ 001524e4     network.obj
 0002:000114f0       ??_C@_02OCIIGHHD@RE?$AA@   001524f0     network.obj
 0002:000114f4       ??_C@_0P@CODDPBOL@Orange?5Reunion?$AA@ 001524f4     network.obj
 0002:00011504       ??_C@_07BGILKICI@ANTARIS?$AA@ 00152504     network.obj
 0002:0001150c       ??_C@_02MHMEOBLM@MG?$AA@   0015250c     network.obj
 0002:00011510       ??_C@_07IIPIGCFA@Madacom?$AA@ 00152510     network.obj
 0002:00011518       ??_C@_07JJFEFGNM@ZAMCELL?$AA@ 00152518     network.obj
 0002:00011520       ??_C@_04FGIKGBKN@mCel?$AA@ 00152520     network.obj
 0002:00011528       ??_C@_07JAEDENAH@SAFARIS?$AA@ 00152528     network.obj
 0002:00011530       ??_C@_02FCBLILAP@BI?$AA@   00152530     network.obj
 0002:00011534       ??_C@_0M@GCAINNJK@UTL?5TELECEL?$AA@ 00152534     network.obj
 0002:00011540       ??_C@_0L@KOGBGKLA@MTN?9UGANDA?$AA@ 00152540     network.obj
 0002:0001154c       ??_C@_02NFPBBDHE@UG?$AA@   0015254c     network.obj
 0002:00011550       ??_C@_06NALAPOFF@CelTel?$AA@ 00152550     network.obj
 0002:00011558       ??_C@_07PJBGDEHA@Vodacom?$AA@ 00152558     network.obj
 0002:00011560       ??_C@_06KIADHOEO@ZANTEL?$AA@ 00152560     network.obj
 0002:00011568       ??_C@_02CLFPBFFP@TZ?$AA@   00152568     network.obj
 0002:0001156c       ??_C@_06MPFOKJDG@TRITEL?$AA@ 0015256c     network.obj
 0002:00011574       ??_C@_07FLJODBNE@KENCELL?$AA@ 00152574     network.obj
 0002:0001157c       ??_C@_02PBHPPPIM@KE?$AA@   0015257c     network.obj
 0002:00011580       ??_C@_09FGIIKJKE@Safaricom?$AA@ 00152580     network.obj
 0002:0001158c       ??_C@_02BJKFOFMO@SO?$AA@   0015258c     network.obj
 0002:00011590       ??_C@_08NPOPAKFD@BARAKAAT?$AA@ 00152590     network.obj
 0002:0001159c       ??_C@_02KIDIPBJG@ET?$AA@   0015259c     network.obj
 0002:000115a0       ??_C@_05LAAKMIIP@ETMTN?$AA@ 001525a0     network.obj
 0002:000115a8       ??_C@_02JKHMBHKA@RW?$AA@   001525a8     network.obj
 0002:000115ac       ??_C@_0L@MIPIDLDD@Rwandacell?$AA@ 001525ac     network.obj
 0002:000115b8       ??_C@_02DIKIINKA@MZ?$AA@   001525b8     network.obj
 0002:000115bc       ??_C@_06IEJJEOJE@AIRTEL?$AA@ 001525bc     network.obj
 0002:000115c4       ??_C@_02LFBAKKMC@SC?$AA@   001525c4     network.obj
 0002:000115c8       ??_C@_06LJAEFNDP@SEYCEL?$AA@ 001525c8     network.obj
 0002:000115d0       ??_C@_05OCMFIPII@OASIS?$AA@ 001525d0     network.obj
 0002:000115d8       ??_C@_06BBJOGCE@CELLCO?$AA@ 001525d8     network.obj
 0002:000115e0       ??_C@_02OGHHJPHF@CD?$AA@   001525e0     network.obj
 0002:000115e4       ??_C@_07BNCIDIGM@CELLNET?$AA@ 001525e4     network.obj
 0002:000115ec       ??_C@_09IKFPFEDK@GO?5Celtel?$AA@ 001525ec     network.obj
 0002:000115f8       ??_C@_02JMAJMDOM@GA?$AA@   001525f8     network.obj
 0002:000115fc       ??_C@_02JOIDOPKG@CV?$AA@   001525fc     network.obj
 0002:00011600       ??_C@_09OKMAGAPH@CPV?5MOVEL?$AA@ 00152600     network.obj
 0002:0001160c       ??_C@_02DHLFCEDM@CM?$AA@   0015260c     network.obj
 0002:00011610       ??_C@_07EOPCJLML@MTN?9CAM?$AA@ 00152610     network.obj
 0002:00011618       ??_C@_08HDOCIBIN@LIBERTIS?$AA@ 00152618     network.obj
 0002:00011624       ??_C@_02PPBOCKIA@TD?$AA@   00152624     network.obj
 0002:00011628       ??_C@_09LNNNJGBC@NITEL?5GSM?$AA@ 00152628     network.obj
 0002:00011634       ??_C@_06PEICDFHA@ECONET?$AA@ 00152634     network.obj
 0002:0001163c       ??_C@_02MFICFPOF@NG?$AA@   0015263c     network.obj
 0002:00011640       ??_C@_03LCIKEEOE@MTN?$AA@  00152640     network.obj
 0002:00011644       ??_C@_08CHMMGLF@ONEtouch?$AA@ 00152644     network.obj
 0002:00011650       ??_C@_02ENMLHIKF@GH?$AA@   00152650     network.obj
 0002:00011654       ??_C@_08FHOPBLIF@SPACEFON?$AA@ 00152654     network.obj
 0002:00011660       ??_C@_02PBLDGNJP@LR?$AA@   00152660     network.obj
 0002:00011664       ??_C@_05OMBHNFGL@Omega?$AA@ 00152664     network.obj
 0002:0001166c       ??_C@_05NPDJIOKM@EMTEL?$AA@ 0015266c     network.obj
 0002:00011674       ??_C@_02LPDAJBGP@MU?$AA@   00152674     network.obj
 0002:00011678       ??_C@_08HGJFAHIC@CELLPLUS?$AA@ 00152678     network.obj
 0002:00011684       ??_C@_09FMDMHDAO@BENINCELL?$AA@ 00152684     network.obj
 0002:00011690       ??_C@_0O@BPPKCCBM@Telecel?5Benin?$AA@ 00152690     network.obj
 0002:000116a0       ??_C@_02HJDGNIMM@BJ?$AA@   001526a0     network.obj
 0002:000116a4       ??_C@_08GOOAKNMG@LIBERCOM?$AA@ 001526a4     network.obj
 0002:000116b0       ??_C@_02NEDDHJED@TG?$AA@   001526b0     network.obj
 0002:000116b4       ??_C@_07JCDAJFIH@TOGOCEL?$AA@ 001526b4     network.obj
 0002:000116bc       ??_C@_02PHLEDNGH@NE?$AA@   001526bc     network.obj
 0002:000116c0       ??_C@_02NFIDJHMA@BF?$AA@   001526c0     network.obj
 0002:000116c4       ??_C@_06LLBELGCF@CELTEL?$AA@ 001526c4     network.obj
 0002:000116cc       ??_C@_07BGDHCCKL@TELECEL?$AA@ 001526cc     network.obj
 0002:000116d4       ??_C@_07MMBFAGHP@Ivoiris?$AA@ 001526d4     network.obj
 0002:000116dc       ??_C@_02FDNJOBDI@CI?$AA@   001526dc     network.obj
 0002:000116e0       ??_C@_04GDKDOGIK@CORA?$AA@ 001526e0     network.obj
 0002:000116e8       ??_C@_05BODLJNCB@LAGUI?$AA@ 001526e8     network.obj
 0002:000116f0       ??_C@_02BLJBNPCD@GN?$AA@   001526f0     network.obj
 0002:000116f4       ??_C@_02CEDADIHH@ML?$AA@   001526f4     network.obj
 0002:000116f8       ??_C@_07IJLCKOJP@MALITEL?$AA@ 001526f8     network.obj
 0002:00011700       ??_C@_06KGAKHJIL@SENTEL?$AA@ 00152700     network.obj
 0002:00011708       ??_C@_02LONEIP@SN?$AA@     00152708     network.obj
 0002:0001170c       ??_C@_05BNADDFEM@ALIZE?$AA@ 0015270c     network.obj
 0002:00011714       ??_C@_02FPBMCAK@TN?$AA@    00152714     network.obj
 0002:00011718       ??_C@_08IBDIKNDC@TUNICELL?$AA@ 00152718     network.obj
 0002:00011724       ??_C@_03MCIOBOL@IAM?$AA@   00152724     network.obj
 0002:00011728       ??_C@_02JBJOEGDK@MA?$AA@   00152728     network.obj
 0002:0001172c       ??_C@_07JFIFNGDD@Meditel?$AA@ 0015272c     network.obj
 0002:00011734       ??_C@_02DHHJLGCP@DZ?$AA@   00152734     network.obj
 0002:00011738       ??_C@_03OLKLGDKD@AMN?$AA@  00152738     network.obj
 0002:0001173c       ??_C@_09JLNPHJJF@CLICK?5GSM?$AA@ 0015273c     network.obj
 0002:00011748       ??_C@_02MJNHLAAE@EG?$AA@   00152748     network.obj
 0002:0001174c       ??_C@_07OEKEKPGD@MobiNiL?$AA@ 0015274c     network.obj
 0002:00011754       ??_C@_02DBHOOGNH@FM?$AA@   00152754     network.obj
 0002:00011758       ??_C@_03ELOJIGKD@FSM?$AA@  00152758     network.obj
 0002:0001175c       ??_C@_02MKCBOANO@PF?$AA@   0015275c     network.obj
 0002:00011760       ??_C@_04DDCNHBLI@VINI?$AA@ 00152760     network.obj
 0002:00011768       ??_C@_02KBOOJKOB@NC?$AA@   00152768     network.obj
 0002:0001176c       ??_C@_07LCGKDMDI@MOBILIS?$AA@ 0015276c     network.obj
 0002:00011774       ??_C@_02OAHAMPIN@AS?$AA@   00152774     network.obj
 0002:00011778       ??_C@_08CKLJHNHH@Blue?5Sky?$AA@ 00152778     network.obj
 0002:00011784       ??_C@_02HODPHABA@FJ?$AA@   00152784     network.obj
 0002:00011788       ??_C@_05HGNGGAKO@SMILE?$AA@ 00152788     network.obj
 0002:00011790       ??_C@_02KPEDNNPO@VU?$AA@   00152790     network.obj
 0002:00011794       ??_C@_02BMOKPDEL@TO?$AA@   00152794     network.obj
 0002:00011798       ??_C@_0M@EMEBJNNF@Tonga?5Comm?4?$AA@ 00152798     network.obj
 0002:000117a4       ??_C@_02DKOODDPJ@NZ?$AA@   001527a4     network.obj
 0002:000117a8       ??_C@_02BNFKBNMI@BN?$AA@   001527a8     network.obj
 0002:000117ac       ??_C@_0L@OMGEGOPF@BRU?5TSTCom?$AA@ 001527ac     network.obj
 0002:000117b8       ??_C@_0M@MMPGCDGD@STARHUB?9SGP?$AA@ 001527b8     network.obj
 0002:000117c4       ??_C@_0M@DGMHDCPN@SGP?9M1?93GSM?$AA@ 001527c4     network.obj
 0002:000117d0       ??_C@_0L@NAAPDKIN@M1?9GSM?9SGP?$AA@ 001527d0     network.obj
 0002:000117dc       ??_C@_0P@FPCCMHFK@ST?9GSM1800?9SGP?$AA@ 001527dc     network.obj
 0002:000117ec       ??_C@_02NBHMGPMG@SG?$AA@   001527ec     network.obj
 0002:000117f0       ??_C@_0L@BLEBBKHE@ST?9GSM?9SGP?$AA@ 001527f0     network.obj
 0002:000117fc       ??_C@_05OCIGMBIP@HELLO?$AA@ 001527fc     network.obj
 0002:00011804       ??_C@_07PCKLHAN@WP?91800?$AA@ 00152804     network.obj
 0002:0001180c       ??_C@_0L@BONOIH@ACT?5Mobile?$AA@ 0015280c     network.obj
 0002:00011818       ??_C@_02FDKLGFIM@TH?$AA@   00152818     network.obj
 0002:0001181c       ??_C@_07MIEMEGDH@AIS?5GSM?$AA@ 0015281c     network.obj
 0002:00011824       ??_C@_07MLPONFMC@Digitel?$AA@ 00152824     network.obj
 0002:0001182c       ??_C@_05PGADOFCL@SMART?$AA@ 0015282c     network.obj
 0002:00011834       ??_C@_05DADOJJDN@Globe?$AA@ 00152834     network.obj
 0002:0001183c       ??_C@_02FEKCMNFA@PH?$AA@   0015283c     network.obj
 0002:00011840       ??_C@_07BEILLNPC@ISLACOM?$AA@ 00152840     network.obj
 0002:00011848       ??_C@_07IAGGKPHN@INDOSAT?$AA@ 00152848     network.obj
 0002:00011850       ??_C@_06KFHNIFDF@GSM?9XL?$AA@ 00152850     network.obj
 0002:00011858       ??_C@_09KNPJMKPN@TELKOMSEL?$AA@ 00152858     network.obj
 0002:00011864       ??_C@_09MNAMJPOA@LIPPO?5TEL?$AA@ 00152864     network.obj
 0002:00011870       ??_C@_0N@KIOPGDPN@SATELINDOCEL?$AA@ 00152870     network.obj
 0002:00011880       ??_C@_02OLOABKKD@ID?$AA@   00152880     network.obj
 0002:00011884       ??_C@_07FEBKHNHG@One?4Tel?$AA@ 00152884     network.obj
 0002:0001188c       ??_C@_05DHKOFDBH@OPTUS?$AA@ 0015288c     network.obj
 0002:00011894       ??_C@_02LGCKGIAL@AU?$AA@   00152894     network.obj
 0002:00011898       ??_C@_09CIGLFGDH@MobileNet?$AA@ 00152898     network.obj
 0002:000118a4       ??_C@_06GCFGGNJE@CELCOM?$AA@ 001528a4     network.obj
 0002:000118ac       ??_C@_04HMLHGAMO@ADAM?$AA@ 001528ac     network.obj
 0002:000118b4       ??_C@_04BDGKAFEJ@DiGi?$AA@ 001528b4     network.obj
 0002:000118bc       ??_C@_08HMEEHLIO@TM?5Touch?$AA@ 001528bc     network.obj
 0002:000118c8       ??_C@_02BDIFNOGD@MY?$AA@   001528c8     network.obj
 0002:000118cc       ??_C@_0N@MAHDPBLB@Maxis?5Mobile?$AA@ 001528cc     network.obj
 0002:000118dc       ??_C@_02JEBNMCKM@MV?$AA@   001528dc     network.obj
 0002:000118e0       ??_C@_09DDMPDHPA@DHIMOBILE?$AA@ 001528e0     network.obj
 0002:000118ec       ??_C@_0M@EFJJBNGG@Mobile?52000?$AA@ 001528ec     network.obj
 0002:000118f8       ??_C@_0L@JFGMLJON@ShebaWorld?$AA@ 001528f8     network.obj
 0002:00011904       ??_C@_05MLOIDJBK@AKTEL?$AA@ 00152904     network.obj
 0002:0001190c       ??_C@_02OHLFPFEC@BD?$AA@   0015290c     network.obj
 0002:00011910       ??_C@_0N@LFJDBKCK@GrameemPhone?$AA@ 00152910     network.obj
 0002:00011920       ??_C@_09BPFIGGNI@TransAsia?$AA@ 00152920     network.obj
 0002:0001192c       ??_C@_07HELOIPKO@TWN?5GSM?$AA@ 0015292c     network.obj
 0002:00011934       ??_C@_07DNOAJJMH@MobiTai?$AA@ 00152934     network.obj
 0002:0001193c       ??_C@_08IJJBKOLJ@Chunghwa?$AA@ 0015293c     network.obj
 0002:00011948       ??_C@_03DJKMPMMK@KGT?$AA@  00152948     network.obj
 0002:0001194c       ??_C@_04KGFIJJE@ACeS?$AA@  0015294c     network.obj
 0002:00011954       ??_C@_06EONFJCML@TUNTEX?$AA@ 00152954     network.obj
 0002:0001195c       ??_C@_02JOPBGLBC@TW?$AA@   0015295c     network.obj
 0002:00011960       ??_C@_0M@IPHMLGFP@Far?5EasTone?$AA@ 00152960     network.obj
 0002:0001196c       ??_C@_0N@OFDBEJDN@China?5Unicom?$AA@ 0015296c     network.obj
 0002:0001197c       ??_C@_02BMJIHHPP@CN?$AA@   0015297c     network.obj
 0002:00011980       ??_C@_0N@KIKOKNBF@China?5Mobile?$AA@ 00152980     network.obj
 0002:00011990       ??_C@_02JAFMCMAN@LA?$AA@   00152990     network.obj
 0002:00011994       ??_C@_07BELCNPGB@LAO?5GSM?$AA@ 00152994     network.obj
 0002:0001199c       ??_C@_0L@PJFMCHGE@SAMART?9GSM?$AA@ 0015299c     network.obj
 0002:000119a8       ??_C@_02EENBIBMB@KH?$AA@   001529a8     network.obj
 0002:000119ac       ??_C@_07EHJOMFFO@MobiTel?$AA@ 001529ac     network.obj
 0002:000119b4       ??_C@_08EHDHLNOI@HT?5Macau?$AA@ 001529b4     network.obj
 0002:000119c0       ??_C@_06NOCFIFJ@CTMGSM?$AA@ 001529c0     network.obj
 0002:000119c8       ??_C@_08IGPJDPIF@SmarTone?$AA@ 001529c8     network.obj
 0002:000119d4       ??_C@_06MFHJGCEH@SUNDAY?$AA@ 001529d4     network.obj
 0002:000119dc       ??_C@_07CJNAFIMF@PEOPLES?$AA@ 001529dc     network.obj
 0002:000119e4       ??_C@_03KEBFICPK@SMC?$AA@  001529e4     network.obj
 0002:000119e8       ??_C@_09NPOEOLMK@NEW?5WORLD?$AA@ 001529e8     network.obj
 0002:000119f4       ??_C@_02GNLKGMFL@HK?$AA@   001529f4     network.obj
 0002:000119f8       ??_C@_03GFCMEHNA@CSL?$AA@  001529f8     network.obj
 0002:000119fc       ??_C@_08BNJCCDIO@VINAFONE?$AA@ 001529fc     network.obj
 0002:00011a08       ??_C@_02GHFBGGE@VN?$AA@    00152a08     network.obj
 0002:00011a0c       ??_C@_08NOJLBOLM@MOBIFONE?$AA@ 00152a0c     network.obj
 0002:00011a18       ??_C@_02CONMJBMJ@TM?$AA@   00152a18     network.obj
 0002:00011a1c       ??_C@_04NIEBIGDI@BCTI?$AA@ 00152a1c     network.obj
 0002:00011a24       ??_C@_02MDEJJNAO@KG?$AA@   00152a24     network.obj
 0002:00011a28       ??_C@_05DHLMBINE@BITEL?$AA@ 00152a28     network.obj
 0002:00011a30       ??_C@_06OKOLKJOP@Coscom?$AA@ 00152a30     network.obj
 0002:00011a38       ??_C@_0P@CBBDGFGC@UZB?5DAEWOO?9GSM?$AA@ 00152a38     network.obj
 0002:00011a48       ??_C@_07GFHANBDC@Uzmacom?$AA@ 00152a48     network.obj
 0002:00011a50       ??_C@_02CKJNHPGI@UZ?$AA@   00152a50     network.obj
 0002:00011a54       ??_C@_06DKIDDKGG@Buztel?$AA@ 00152a54     network.obj
 0002:00011a5c       ??_C@_04KGLICDOJ@KISH?$AA@ 00152a5c     network.obj
 0002:00011a64       ??_C@_02PHHIKPHE@IR?$AA@   00152a64     network.obj
 0002:00011a68       ??_C@_03MJLDHPMD@TCI?$AA@  00152a68     network.obj
 0002:00011a6c       ??_C@_02MAABNLHD@NP?$AA@   00152a6c     network.obj
 0002:00011a70       ??_C@_02BGAGFKPF@MN?$AA@   00152a70     network.obj
 0002:00011a74       ??_C@_07JONMBOOP@MobiCom?$AA@ 00152a74     network.obj
 0002:00011a7c       ??_C@_02IEKCBMCO@QA?$AA@   00152a7c     network.obj
 0002:00011a80       ??_C@_08BLOIAMKE@QATARNET?$AA@ 00152a80     network.obj
 0002:00011a8c       ??_C@_02ELAALKEO@BH?$AA@   00152a8c     network.obj
 0002:00011a90       ??_C@_0M@PKLFECKO@MOBILE?5PLUS?$AA@ 00152a90     network.obj
 0002:00011a9c       ??_C@_06LHJBBAEB@JAWWAL?$AA@ 00152a9c     network.obj
 0002:00011aa4       ??_C@_02CDDJJAKL@IL?$AA@   00152aa4     network.obj
 0002:00011aa8       ??_C@_02PMOIHKFK@AE?$AA@   00152aa8     network.obj
 0002:00011aac       ??_C@_08BMMIPDAN@ETISALAT?$AA@ 00152aac     network.obj
 0002:00011ab8       ??_C@_02DOKPNNFI@OM?$AA@   00152ab8     network.obj
 0002:00011abc       ??_C@_0M@KOCMOMNO@OMAN?5MOBILE?$AA@ 00152abc     network.obj
 0002:00011ac8       ??_C@_02OONNIIJC@YE?$AA@   00152ac8     network.obj
 0002:00011acc       ??_C@_03IOCHNEFL@EAE?$AA@  00152acc     network.obj
 0002:00011ad0       ??_C@_02IHCGMIEA@SA?$AA@   00152ad0     network.obj
 0002:00011ad4       ??_C@_08IFBFHLND@Al?9Jawal?$AA@ 00152ad4     network.obj
 0002:00011ae0       ??_C@_08HCLMILBE@WATANIYA?$AA@ 00152ae0     network.obj
 0002:00011aec       ??_C@_02IJILIPFP@KW?$AA@   00152aec     network.obj
 0002:00011af0       ??_C@_06LBIHMGHH@MTCNet?$AA@ 00152af0     network.obj
 0002:00011af8       ??_C@_0N@HKAEDBKK@MOBILE?5SYRIA?$AA@ 00152af8     network.obj
 0002:00011b08       ??_C@_02FDNFABJ@SY?$AA@    00152b08     network.obj
 0002:00011b0c       ??_C@_08GPADNPEB@Spacetel?$AA@ 00152b0c     network.obj
 0002:00011b18       ??_C@_09EMJGKCCE@MobileCom?$AA@ 00152b18     network.obj
 0002:00011b24       ??_C@_02KFCHNDB@JO?$AA@    00152b24     network.obj
 0002:00011b28       ??_C@_08DLKAMCBL@Fastlink?$AA@ 00152b28     network.obj
 0002:00011b34       ??_C@_09HOOMPKKC@LibanCell?$AA@ 00152b34     network.obj
 0002:00011b40       ??_C@_02LLHBHPMO@LB?$AA@   00152b40     network.obj
 0002:00011b44       ??_C@_06CBGPNJOB@Cellis?$AA@ 00152b44     network.obj
 0002:00011b4c       ??_C@_02DNCLAJDG@MM?$AA@   00152b4c     network.obj
 0002:00011b50       ??_C@_06EDEGGGMG@MM?5900?$AA@ 00152b50     network.obj
 0002:00011b58       ??_C@_07KAJHBHMO@CELLTEL?$AA@ 00152b58     network.obj
 0002:00011b60       ??_C@_02GKLDMEIH@LK?$AA@   00152b60     network.obj
 0002:00011b64       ??_C@_06IKCPKPAM@DIALOG?$AA@ 00152b64     network.obj
 0002:00011b6c       ??_C@_02HPIPJOJD@PK?$AA@   00152b6c     network.obj
 0002:00011b70       ??_C@_08NCJOMIML@Mobilink?$AA@ 00152b70     network.obj
 0002:00011b7c       ??_C@_07LJDFOIJB@hexacom?$AA@ 00152b7c     network.obj
 0002:00011b84       ??_C@_06EJFHCBLC@AIRCEL?$AA@ 00152b84     network.obj
 0002:00011b8c       ??_C@_0N@ENOCILDN@RPG?5Cellular?$AA@ 00152b8c     network.obj
 0002:00011b9c       ??_C@_07LKCMFCDE@SKYCELL?$AA@ 00152b9c     network.obj
 0002:00011ba4       ??_C@_07FBJAHANB@COMMAND?$AA@ 00152ba4     network.obj
 0002:00011bac       ??_C@_04PKDGEDOM@AT?$CGT?$AA@ 00152bac     network.obj
 0002:00011bb4       ??_C@_0L@IJOLIFEK@BPL?5MOBILE?$AA@ 00152bb4     network.obj
 0002:00011bc0       ??_C@_05OFPKHEKA@SPICE?$AA@ 00152bc0     network.obj
 0002:00011bc8       ??_C@_07NEAAHPLI@ESCOTEL?$AA@ 00152bc8     network.obj
 0002:00011bd0       ??_C@_06OPDNAGOE@AirTel?$AA@ 00152bd0     network.obj
 0002:00011bd8       ??_C@_08JDAEGACL@Reliance?$AA@ 00152bd8     network.obj
 0002:00011be4       ??_C@_0O@LCKJHHFC@TATA?5CELLULAR?$AA@ 00152be4     network.obj
 0002:00011bf4       ??_C@_08IBELGOAO@CELFORCE?$AA@ 00152bf4     network.obj
 0002:00011c00       ??_C@_02BBAPPCCJ@IN?$AA@   00152c00     network.obj
 0002:00011c04       ??_C@_05EOHGAIPF@ESSAR?$AA@ 00152c04     network.obj
 0002:00011c0c       ??_C@_06KIODMKLH@K?8CELL?$AA@ 00152c0c     network.obj
 0002:00011c14       ??_C@_02DMCFPBBC@KZ?$AA@   00152c14     network.obj
 0002:00011c18       ??_C@_08MMDBHOHG@K?9MOBILE?$AA@ 00152c18     network.obj
 0002:00011c24       ??_C@_0BB@IDKCIIMC@BAKCELL?5GSM?52000?$AA@ 00152c24     network.obj
 0002:00011c38       ??_C@_02DBLCHEME@AZ?$AA@   00152c38     network.obj
 0002:00011c3c       ??_C@_0N@MNFOGIJG@AZERCELL?5GSM?$AA@ 00152c3c     network.obj
 0002:00011c4c       ??_C@_02MMFADL@DO?$AA@     00152c4c     network.obj
 0002:00011c50       ??_C@_02LFKOLMGF@CU?$AA@   00152c50     network.obj
 0002:00011c54       ??_C@_05GHMLBAKA@C_Com?$AA@ 00152c54     network.obj
 0002:00011c5c       ??_C@_02BPBMKDJB@AN?$AA@   00152c5c     network.obj
 0002:00011c60       ??_C@_0M@HDOFJCEI@Telcell?5GSM?$AA@ 00152c60     network.obj
 0002:00011c6c       ??_C@_02DGHHEOAL@BM?$AA@   00152c6c     network.obj
 0002:00011c70       ??_C@_07GJAEIOO@Telecom?$AA@ 00152c70     network.obj
 0002:00011c78       ??_C@_02MONOBINI@AG?$AA@   00152c78     network.obj
 0002:00011c7c       ??_C@_08NJFGANKC@APUA?5PCS?$AA@ 00152c7c     network.obj
 0002:00011c88       ??_C@_08EPNJAJEP@Bouygues?$AA@ 00152c88     network.obj
 0002:00011c94       ??_C@_02IBFDBMAM@FW?$AA@   00152c94     network.obj
 0002:00011c98       ??_C@_07IJFEMGNF@Orange?5?$AA@ 00152c98     network.obj
 0002:00011ca0       ??_C@_02DIGEBPLD@JM?$AA@   00152ca0     network.obj
 0002:00011ca4       ??_C@_07GDALKOE@Digicel?$AA@ 00152ca4     network.obj
 0002:00011cac       ??_C@_06IEDFABOJ@Nextel?$AA@ 00152cac     network.obj
 0002:00011cb4       ??_C@_02BAABKJLB@?9?9?$AA@ 00152cb4     network.obj
 0002:00011cb8       ??_C@_08ELNGLDFJ@Sprocket?$AA@ 00152cb8     network.obj
 0002:00011cc4       ??_C@_03FHGCJBJ@AWS?$AA@   00152cc4     network.obj
 0002:00011cc8       ??_C@_08CHFBCMDF@PinPoint?$AA@ 00152cc8     network.obj
 0002:00011cd4       ??_C@_0M@NDAGCDLO@Airlink?5PCS?$AA@ 00152cd4     network.obj
 0002:00011ce0       ??_C@_0O@JODLAKDE@Iowa?5Wireless?$AA@ 00152ce0     network.obj
 0002:00011cf0       ??_C@_04KOADLHJ@PTSI?$AA@  00152cf0     network.obj
 0002:00011cf8       ??_C@_0L@JGFBGNGL@Telemetrix?$AA@ 00152cf8     network.obj
 0002:00011d04       ??_C@_09CFBCONOC@Conestoga?$AA@ 00152d04     network.obj
 0002:00011d10       ??_C@_0N@JBAFPDFF@NPI?5Wireless?$AA@ 00152d10     network.obj
 0002:00011d20       ??_C@_0N@KBMAIEL@Einstein?5PCS?$AA@ 00152d20     network.obj
 0002:00011d30       ??_C@_09BDELPFCM@AmeriLink?$AA@ 00152d30     network.obj
 0002:00011d3c       ??_C@_0L@JDBOLJBI@Epic?5Touch?$AA@ 00152d3c     network.obj
 0002:00011d48       ??_C@_08KEPFMAJC@TMP?5Corp?$AA@ 00152d48     network.obj
 0002:00011d54       ??_C@_0O@OJNKGLNJ@AT?$CGT?5Mobility?$AA@ 00152d54     network.obj
 0002:00011d64       ??_C@_08EELOJGDC@Carolina?$AA@ 00152d64     network.obj
 0002:00011d70       ??_C@_08MFJALFNH@WestLink?$AA@ 00152d70     network.obj
 0002:00011d7c       ??_C@_0BG@IGHHLMOI@West?5Central?5Wireless?$AA@ 00152d7c     network.obj
 0002:00011d94       ??_C@_08OLOLPKDO@Cingular?$AA@ 00152d94     network.obj
 0002:00011da0       ??_C@_0O@PJCNKLAA@Wireless?52000?$AA@ 00152da0     network.obj
 0002:00011db0       ??_C@_02PLFPMECB@US?$AA@   00152db0     network.obj
 0002:00011db4       ??_C@_07BJADOGLO@Cellnet?$AA@ 00152db4     network.obj
 0002:00011dbc       ??_C@_0BA@KIONBCLL@Rogers?5Wireless?$AA@ 00152dbc     network.obj
 0002:00011dcc       ??_C@_0M@EFDLFGHM@Rogers?5AT?$CGT?$AA@ 00152dcc     network.obj
 0002:00011dd8       ??_C@_02JLAAGLDA@CA?$AA@   00152dd8     network.obj
 0002:00011ddc       ??_C@_09BCPOLPA@Microcell?$AA@ 00152ddc     network.obj
 0002:00011de8       ??_C@_08FDEMCHIB@LI?5TANGO?$AA@ 00152de8     network.obj
 0002:00011df4       ??_C@_03NPBJFEBE@FL1?$AA@  00152df4     network.obj
 0002:00011df8       ??_C@_06DAHALNHO@MONTEL?$AA@ 00152df8     network.obj
 0002:00011e00       ??_C@_02FIIFKGAF@LI?$AA@   00152e00     network.obj
 0002:00011e04       ??_C@_07CLLJGDM@TELECOM?$AA@ 00152e04     network.obj
 0002:00011e0c       ??_C@_02GLHBKOLA@MK?$AA@   00152e0c     network.obj
 0002:00011e10       ??_C@_07IGNOJCLM@MOBIMAK?$AA@ 00152e10     network.obj
 0002:00011e18       ??_C@_07ODIHLELC@MOBITEL?$AA@ 00152e18     network.obj
 0002:00011e20       ??_C@_02EPPPECEI@SI?$AA@   00152e20     network.obj
 0002:00011e24       ??_C@_08IAIGPNDP@SI?4MOBIL?$AA@ 00152e24     network.obj
 0002:00011e30       ??_C@_0P@KNHAJFCM@TELE?5Greenland?$AA@ 00152e30     network.obj
 0002:00011e40       ??_C@_02DEIIEFF@FO?$AA@    00152e40     network.obj
 0002:00011e44       ??_C@_06DOHIMEAC@FT?5GSM?$AA@ 00152e44     network.obj
 0002:00011e4c       ??_C@_06DNLLPJEI@AYCELL?$AA@ 00152e4c     network.obj
 0002:00011e54       ??_C@_04KLGDHGDJ@ARIA?$AA@ 00152e54     network.obj
 0002:00011e5c       ??_C@_06JELLOEPJ@TELSIM?$AA@ 00152e5c     network.obj
 0002:00011e64       ??_C@_02ODIGJPFH@TR?$AA@   00152e64     network.obj
 0002:00011e68       ??_C@_08GMIOPKID@TURKCELL?$AA@ 00152e68     network.obj
 0002:00011e74       ??_C@_02MMJIKGIB@BG?$AA@   00152e74     network.obj
 0002:00011e78       ??_C@_09FHGFPNLJ@M?9TEL?5GSM?$AA@ 00152e78     network.obj
 0002:00011e84       ??_C@_02DEDBPAFC@AM?$AA@   00152e84     network.obj
 0002:00011e88       ??_C@_06EMCEKKGN@ARMGSM?$AA@ 00152e88     network.obj
 0002:00011e90       ??_C@_06BGDLBAKP@GEO?503?$AA@ 00152e90     network.obj
 0002:00011e98       ??_C@_09DNPEGDFH@Magti?5GSM?$AA@ 00152e98     network.obj
 0002:00011ea4       ??_C@_02PIGFAGOI@GE?$AA@   00152ea4     network.obj
 0002:00011ea8       ??_C@_07MHGNPHDO@GEOCELL?$AA@ 00152ea8     network.obj
 0002:00011eb0       ??_C@_02BJBLPDGJ@CY?$AA@   00152eb0     network.obj
 0002:00011eb4       ??_C@_07FEOALDMB@CYTAGSM?$AA@ 00152eb4     network.obj
 0002:00011ebc       ??_C@_09LKLKAFAL@go?5mobile?$AA@ 00152ebc     network.obj
 0002:00011ec8       ??_C@_02KGCLKACO@MT?$AA@   00152ec8     network.obj
 0002:00011ecc       ??_C@_0P@DBFLDMMF@Vodafone?5Malta?$AA@ 00152ecc     network.obj
 0002:00011edc       ??_C@_02CNCKMBBD@AL?$AA@   00152edc     network.obj
 0002:00011ee0       ??_C@_03FOAFBNOO@AMC?$AA@  00152ee0     network.obj
 0002:00011ee4       ??_C@_06MNFEEHAB@Viking?$AA@ 00152ee4     network.obj
 0002:00011eec       ??_C@_03LHEAFPOI@TAL?$AA@  00152eec     network.obj
 0002:00011ef0       ??_C@_02OOGDJODF@IS?$AA@   00152ef0     network.obj
 0002:00011ef4       ??_C@_06KHIMBAB@SIMINN?$AA@ 00152ef4     network.obj
 0002:00011efc       ??_C@_06IKMIJLMI@METEOR?$AA@ 00152efc     network.obj
 0002:00011f04       ??_C@_08LPJDJOJH@O2?5?9?5IRL?$AA@ 00152f04     network.obj
 0002:00011f10       ??_C@_02PCPLCLOC@IE?$AA@   00152f10     network.obj
 0002:00011f14       ??_C@_0N@GMCBAJFA@Vodafone?5IRL?$AA@ 00152f14     network.obj
 0002:00011f24       ??_C@_05MFEOICMF@TANGO?$AA@ 00152f24     network.obj
 0002:00011f2c       ??_C@_02LOPCPLFI@LU?$AA@   00152f2c     network.obj
 0002:00011f30       ??_C@_06JIPGODOH@LUXGSM?$AA@ 00152f30     network.obj
 0002:00011f38       ??_C@_03IMGMMEAO@TMN?$AA@  00152f38     network.obj
 0002:00011f3c       ??_C@_07BJNGALJF@OPTIMUS?$AA@ 00152f3c     network.obj
 0002:00011f44       ??_C@_02LCNFJAAN@PT?$AA@   00152f44     network.obj
 0002:00011f48       ??_C@_02FENAEJOE@GI?$AA@   00152f48     network.obj
 0002:00011f4c       ??_C@_06IHKJOMCM@GIBTEL?$AA@ 00152f4c     network.obj
 0002:00011f54       ??_C@_08OKLLOFBO@Mobilcom?$AA@ 00152f54     network.obj
 0002:00011f60       ??_C@_07DBMOJLEN@O2?5?9?5DE?$AA@ 00152f60     network.obj
 0002:00011f68       ??_C@_06NAFJGLEJ@E?9Plus?$AA@ 00152f68     network.obj
 0002:00011f70       ??_C@_0M@DFNDEIBL@Vodafone?5D2?$AA@ 00152f70     network.obj
 0002:00011f7c       ??_C@_02PKCDLILB@DE?$AA@   00152f7c     network.obj
 0002:00011f80       ??_C@_04OHHLMMNP@IDEA?$AA@ 00152f80     network.obj
 0002:00011f88       ??_C@_07KPNABPMD@Era?5GSM?$AA@ 00152f88     network.obj
 0002:00011f90       ??_C@_02DAMOAIFE@PL?$AA@   00152f90     network.obj
 0002:00011f94       ??_C@_08DDCJHBBB@Plus?5GSM?$AA@ 00152f94     network.obj
 0002:00011fa0       ??_C@_08EHCBHGAM@MOLDCELL?$AA@ 00152fa0     network.obj
 0002:00011fac       ??_C@_02OMOJLCHP@MD?$AA@   00152fac     network.obj
 0002:00011fb0       ??_C@_06LKAJBHGI@VOXTEL?$AA@ 00152fb0     network.obj
 0002:00011fb8       ??_C@_02BINJJJFO@BY?$AA@   00152fb8     network.obj
 0002:00011fbc       ??_C@_06FHLANOPN@VELCOM?$AA@ 00152fbc     network.obj
 0002:00011fc4       ??_C@_0P@OMJDGDBA@Golden?5Telecom?$AA@ 00152fc4     network.obj
 0002:00011fd4       ??_C@_08DLEIAMGN@Kyivstar?$AA@ 00152fd4     network.obj
 0002:00011fe0       ??_C@_07IIPEOAAA@WellCOM?$AA@ 00152fe0     network.obj
 0002:00011fe8       ??_C@_02IDKLLEPC@UA?$AA@   00152fe8     network.obj
 0002:00011fec       ??_C@_03IBHONNCG@UMC?$AA@  00152fec     network.obj
 0002:00011ff0       ??_C@_08COFFHMHC@Bee?5Line?$AA@ 00152ff0     network.obj
 0002:00011ffc       ??_C@_0BA@IGJACJ@JSC?5Telecom?5XXI?$AA@ 00152ffc     network.obj
 0002:0001200c       ??_C@_07JJFMOFJH@Primtel?$AA@ 0015300c     network.obj
 0002:00012014       ??_C@_09PNELBPEB@Sonic?5Duo?$AA@ 00153014     network.obj
 0002:00012020       ??_C@_06OLNEHMPH@NC?9GSM?$AA@ 00153020     network.obj
 0002:00012028       ??_C@_07IPEACO@Uraltel?$AA@ 00153028     network.obj
 0002:00012030       ??_C@_05HHDJJGFO@EXTEL?$AA@ 00153030     network.obj
 0002:00012038       ??_C@_09PHLOEFLF@Ermak?5RMS?$AA@ 00153038     network.obj
 0002:00012044       ??_C@_03BFJBJFEH@NTC?$AA@  00153044     network.obj
 0002:00012048       ??_C@_09KBMFINNI@Kuban?5GSM?$AA@ 00153048     network.obj
 0002:00012054       ??_C@_08NKAJNIGJ@Far?5East?$AA@ 00153054     network.obj
 0002:00012060       ??_C@_07BOPOFJIN@Orensot?$AA@ 00153060     network.obj
 0002:00012068       ??_C@_03HKCMHFCD@DTC?$AA@  00153068     network.obj
 0002:0001206c       ??_C@_06DNNMPEDC@SMARTS?$AA@ 0015306c     network.obj
 0002:00012074       ??_C@_03OEEJLNKB@SCS?$AA@  00153074     network.obj
 0002:00012078       ??_C@_03MPICALC@NCC?$AA@   00153078     network.obj
 0002:0001207c       ??_C@_0O@OGHLLIJM@NorthWest?5GSM?$AA@ 0015307c     network.obj
 0002:0001208c       ??_C@_02KIEKHFCC@RU?$AA@   0015308c     network.obj
 0002:00012090       ??_C@_03ENOGCIPI@MTS?$AA@  00153090     network.obj
 0002:00012094       ??_C@_05GFMAGLCP@Q?5GSM?$AA@ 00153094     network.obj
 0002:0001209c       ??_C@_03ELDBCICO@RLE?$AA@  0015309c     network.obj
 0002:000120a0       ??_C@_02PLOBNCIG@EE?$AA@   001530a0     network.obj
 0002:000120a4       ??_C@_07KFEMFMGG@EMT?5GSM?$AA@ 001530a4     network.obj
 0002:000120ac       ??_C@_07BBKADELB@BALTCOM?$AA@ 001530ac     network.obj
 0002:000120b4       ??_C@_02JFNPKIJL@LV?$AA@   001530b4     network.obj
 0002:000120b8       ??_C@_07LKADEHEN@LMT?5GSM?$AA@ 001530b8     network.obj
 0002:000120c0       ??_C@_05DNCDPFL@TELE2?$AA@ 001530c0     network.obj
 0002:000120c8       ??_C@_08IKAHPPLA@Bite?5GSM?$AA@ 001530c8     network.obj
 0002:000120d4       ??_C@_02KHOJMKBJ@LT?$AA@   001530d4     network.obj
 0002:000120d8       ??_C@_07EBPPGCJN@OMNITEL?$AA@ 001530d8     network.obj
 0002:000120e0       ??_C@_06EDPDKBKP@SONERA?$AA@ 001530e0     network.obj
 0002:000120e8       ??_C@_03FLIGJJHI@AMT?$AA@  001530e8     network.obj
 0002:000120ec       ??_C@_02JIGJMONB@2G?$AA@   001530ec     network.obj
 0002:000120f0       ??_C@_06FJJBCFDL@FINNET?$AA@ 001530f0     network.obj
 0002:000120f8       ??_C@_0L@OAGBEG@RADIOLINJA?$AA@ 001530f8     network.obj
 0002:00012104       ??_C@_02FFBCCDND@FI?$AA@   00153104     network.obj
 0002:00012108       ??_C@_06DILFJIGH@NetCom?$AA@ 00153108     network.obj
 0002:00012110       ??_C@_02NFLNFON@NO?$AA@    00153110     network.obj
 0002:00012114       ??_C@_07DNILEAHP@TELENOR?$AA@ 00153114     network.obj
 0002:0001211c       ??_C@_02NMFFPMLH@IQ?$AA@   0015311c     network.obj
 0002:00012120       ??_C@_02ODEKANEE@SE?$AA@   00153120     network.obj
 0002:00012124       ??_C@_07FDGKLMOE@Telia?5S?$AA@ 00153124     network.obj
 0002:0001212c       ??_C@_05MCOAAOHC@Telia?$AA@ 0015312c     network.obj
 0002:00012134       ??_C@_07LHIFNKDA@SONOFON?$AA@ 00153134     network.obj
 0002:0001213c       ??_C@_02GEKAJFDP@DK?$AA@   0015313c     network.obj
 0002:00012140       ??_C@_09IOJGJFIN@TDK?9MOBIL?$AA@ 00153140     network.obj
 0002:0001214c       ??_C@_04LCHANMNE@MANX?$AA@ 0015314c     network.obj
 0002:00012154       ??_C@_0N@NBCLDHMI@GUERNSEY?5TEL?$AA@ 00153154     network.obj
 0002:00012164       ??_C@_06PJNIKOHG@JT?5GSM?$AA@ 00153164     network.obj
 0002:0001216c       ??_C@_0M@GFANBEBB@T?9Mobile?5UK?$AA@ 0015316c     network.obj
 0002:00012178       ??_C@_02LHCEJACP@GB?$AA@   00153178     network.obj
 0002:0001217c       ??_C@_07LCKJHPIE@O2?5?9?5UK?$AA@ 0015317c     network.obj
 0002:00012184       ??_C@_09DLIGNEBM@tele?4ring?$AA@ 00153184     network.obj
 0002:00012190       ??_C@_03OKMGHDAC@ONE?$AA@  00153190     network.obj
 0002:00012194       ??_C@_08HENOBEJI@T?9Mobile?$AA@ 00153194     network.obj
 0002:000121a0       ??_C@_02KPDBFJEK@AT?$AA@   001531a0     network.obj
 0002:000121a4       ??_C@_02LHLLMGKI@A1?$AA@   001531a4     network.obj
 0002:000121a8       ??_C@_02HNMJCAMK@SK?$AA@   001531a8     network.obj
 0002:000121ac       ??_C@_07IIOBJACI@GLOBTEL?$AA@ 001531ac     network.obj
 0002:000121b4       ??_C@_05HKEAFEOD@OSKAR?$AA@ 001531b4     network.obj
 0002:000121bc       ??_C@_07HPFKJLLM@EUROTEL?$AA@ 001531bc     network.obj
 0002:000121c4       ??_C@_02DCDGKAKK@CZ?$AA@   001531c4     network.obj
 0002:000121c8       ??_C@_06PDFMEOCC@PAEGAS?$AA@ 001531c8     network.obj
 0002:000121d0       ??_C@_07LPKNGFIO@sunrise?$AA@ 001531d0     network.obj
 0002:000121d8       ??_C@_02EKMCNAHJ@CH?$AA@   001531d8     network.obj
 0002:000121dc       ??_C@_09KJCJOELG@Swiss?5GSM?$AA@ 001531dc     network.obj
 0002:000121e8       ??_C@_06IOAEHBNO@dialog?$AA@ 001531e8     network.obj
 0002:000121f0       ??_C@_08NHEEKBMK@Cosmorom?$AA@ 001531f0     network.obj
 0002:000121fc       ??_C@_02BIGHIPPJ@RO?$AA@   001531fc     network.obj
 0002:00012200       ??_C@_06HBEFKGIN@CONNEX?$AA@ 00153200     network.obj
 0002:00012208       ??_C@_07EDHGMGLJ@Blu?5SpA?$AA@ 00153208     network.obj
 0002:00012210       ??_C@_04LLODCGEF@WIND?$AA@ 00153210     network.obj
 0002:00012218       ??_C@_0M@OKMBHGJ@Vodafone?5IT?$AA@ 00153218     network.obj
 0002:00012224       ??_C@_02KBCCAIPC@IT?$AA@   00153224     network.obj
 0002:00012228       ??_C@_03KAEIDPBB@TIM?$AA@  00153228     network.obj
 0002:0001222c       ??_C@_05PEBFHAAD@MONET?$AA@ 0015322c     network.obj
 0002:00012234       ??_C@_0P@MPOBHJMA@Telekom?5Srbija?$AA@ 00153234     network.obj
 0002:00012244       ??_C@_08MAAACGLG@ProMonte?$AA@ 00153244     network.obj
 0002:00012250       ??_C@_02KEBPJKMD@YU?$AA@   00153250     network.obj
 0002:00012254       ??_C@_06PFIAFAHP@MOBTEL?$AA@ 00153254     network.obj
 0002:0001225c       ??_C@_03PFCNJLIG@VIP?$AA@  0015325c     network.obj
 0002:00012260       ??_C@_02PGLKMFED@HR?$AA@   00153260     network.obj
 0002:00012264       ??_C@_06FPNINBHE@CRONET?$AA@ 00153264     network.obj
 0002:0001226c       ??_C@_07JHAEILOK@GSM?5BiH?$AA@ 0015326c     network.obj
 0002:00012274       ??_C@_0P@NEKBPOMN@Mobilna?5Srpska?$AA@ 00153274     network.obj
 0002:00012284       ??_C@_02JKMCABAH@BA?$AA@   00153284     network.obj
 0002:00012288       ??_C@_06DMAIOEEO@ERONET?$AA@ 00153288     network.obj
 0002:00012290       ??_C@_08ICNAMJMD@Vodafone?$AA@ 00153290     network.obj
 0002:0001229c       ??_C@_06BKDOJOF@Westel?$AA@ 0015329c     network.obj
 0002:000122a4       ??_C@_02LJPLFDIE@HU?$AA@   001532a4     network.obj
 0002:000122a8       ??_C@_0L@CAAMKIMB@Pannon?5GSM?$AA@ 001532a8     network.obj
 0002:000122b4       ??_C@_05JPPJLHMC@Xfera?$AA@ 001532b4     network.obj
 0002:000122bc       ??_C@_05BFPGGNOM@AMENA?$AA@ 001532bc     network.obj
 0002:000122c4       ??_C@_08FAFBDOCG@MoviStar?$AA@ 001532c4     network.obj
 0002:000122d0       ??_C@_02OHHJGHFB@ES?$AA@   001532d0     network.obj
 0002:000122d4       ??_C@_0L@LHCMIBOJ@Vodafone?5E?$AA@ 001532d4     network.obj
 0002:000122e0       ??_C@_02OFPDELBL@AD?$AA@   001532e0     network.obj
 0002:000122e4       ??_C@_08JALCPMOL@Mobiland?$AA@ 001532e4     network.obj
 0002:000122f0       ??_C@_08MHGCNMDA@BOUYGTEL?$AA@ 001532f0     network.obj
 0002:000122fc       ??_C@_03PLJJEOAL@SFR?$AA@  001532fc     network.obj
 0002:00012300       ??_C@_02PMCEOIEJ@FR?$AA@   00153300     network.obj
 0002:00012304       ??_C@_06LMIDBFFB@Orange?$AA@ 00153304     network.obj
 0002:0001230c       ??_C@_08CABKJPP@Mobistar?$AA@ 0015330c     network.obj
 0002:00012318       ??_C@_02POKOMEAD@BE?$AA@   00153318     network.obj
 0002:0001231c       ??_C@_08BEBIDFAG@Proximus?$AA@ 0015331c     network.obj
 0002:00012328       ??_C@_09DNHKCJKO@dutchtone?$AA@ 00153328     network.obj
 0002:00012334       ??_C@_03FKMEPPLH@Ben?$AA@  00153334     network.obj
 0002:00012338       ??_C@_07ONJLKFNC@O2?5?9?5NL?$AA@ 00153338     network.obj
 0002:00012340       ??_C@_03JAOILDOE@KPN?$AA@  00153340     network.obj
 0002:00012344       ??_C@_02CGHGIGCO@NL?$AA@   00153344     network.obj
 0002:00012348       ??_C@_0M@IJPIJJLF@Vodafone?5NL?$AA@ 00153348     network.obj
 0002:00012354       ??_C@_08BIFBEJOF@TELESTET?$AA@ 00153354     network.obj
 0002:00012360       ??_C@_0M@FCGIJNOF@Vodafone?5GR?$AA@ 00153360     network.obj
 0002:0001236c       ??_C@_02PNOGICHO@GR?$AA@   0015336c     network.obj
 0002:00012370       ??_C@_07IEBCKNDM@Cosmote?$AA@ 00153370     network.obj
 0002:00013884       ??_C@_04LLKPOCGK@?$CFd?$CFd?$AA@ 00154884     network.obj
 0002:00013890       ??_C@_1FA@PGKCFFIM@?$AAm?$AAp?$AAF?$AAn?$AAS?$AAw?$AAi?$AAA?$AAd?$AAd?$AAP?$AAr?$AAe?$AAf?$AAe?$AAr?$AAr?$AAe?$AAd?$AAO?$AAp?$AAe?$AAr?$AAa?$AAt?$AAo?$AAr?$AAG?$AAo?$AAb?$AAi?$AA?5@ 00154890     network.obj
 0002:000138e0       ??_C@_1BM@MAJKCELE@?$AA?4?$AA?2?$AAn?$AAe?$AAt?$AAw?$AAo?$AAr?$AAk?$AA?4?$AAc?$AAp?$AAp?$AA?$AA@ 001548e0     network.obj
 0002:00013900       ??_C@_1II@NDFCMCON@?$AAm?$AAp?$AAF?$AAn?$AAS?$AAw?$AAi?$AAA?$AAd?$AAd?$AAP?$AAr?$AAe?$AAf?$AAe?$AAr?$AAr?$AAe?$AAd?$AAO?$AAp?$AAe?$AAr?$AAa?$AAt?$AAo?$AAr?$AAG?$AAo?$AAb?$AAi?$AA?5@ 00154900     network.obj
 0002:00013988       ??_C@_1FG@DOECPHMA@?$AAm?$AAp?$AAF?$AAn?$AAS?$AAw?$AAi?$AAR?$AAe?$AAm?$AAo?$AAv?$AAe?$AAP?$AAr?$AAe?$AAf?$AAe?$AAr?$AAr?$AAe?$AAd?$AAO?$AAp?$AAe?$AAr?$AAa?$AAt?$AAo?$AAr?$AAG?$AAo@ 00154988     network.obj
 0002:000139e0       ??_C@_1IO@OEHGLHMP@?$AAm?$AAp?$AAF?$AAn?$AAS?$AAw?$AAi?$AAR?$AAe?$AAm?$AAo?$AAv?$AAe?$AAP?$AAr?$AAe?$AAf?$AAe?$AAr?$AAr?$AAe?$AAd?$AAO?$AAp?$AAe?$AAr?$AAa?$AAt?$AAo?$AAr?$AAG?$AAo@ 001549e0     network.obj
 0002:00013a70       ??_C@_1FI@HKCAKLDF@?$AAm?$AAp?$AAF?$AAn?$AAS?$AAw?$AAi?$AAG?$AAe?$AAt?$AAP?$AAr?$AAe?$AAf?$AAe?$AAr?$AAr?$AAe?$AAd?$AAO?$AAp?$AAe?$AAr?$AAa?$AAt?$AAo?$AAr?$AAL?$AAi?$AAs?$AAt?$AAG@ 00154a70     network.obj
 0002:00013ac8       ??_C@_1JA@GBGFKCKO@?$AAm?$AAp?$AAF?$AAn?$AAS?$AAw?$AAi?$AAG?$AAe?$AAt?$AAP?$AAr?$AAe?$AAf?$AAe?$AAr?$AAr?$AAe?$AAd?$AAO?$AAp?$AAe?$AAr?$AAa?$AAt?$AAo?$AAr?$AAL?$AAi?$AAs?$AAt?$AAG@ 00154ac8     network.obj
 0002:00013b58       ??_C@_1EO@BBECKLIH@?$AAF?$AAa?$AAi?$AAl?$AAe?$AAd?$AA?5?$AAt?$AAo?$AA?5?$AAs?$AAe?$AAn?$AAd?$AA?5?$AAr?$AAe?$AAs?$AAp?$AAo?$AAn?$AAs?$AAe?$AA?5?$AAt?$AAo?$AA?5?$AAt?$AAh?$AAe?$AA?5?$AAc@ 00154b58     network.obj
 0002:00013ba8       ??_C@_1FI@FKFLJEB@?$AAT?$AAh?$AAe?$AAr?$AAe?$AA?5?$AAa?$AAr?$AAe?$AA?5?$AAN?$AAO?$AA?5?$AAp?$AAr?$AAe?$AAf?$AAe?$AAr?$AAr?$AAe?$AAd?$AA?5?$AAo?$AAp?$AAe?$AAr?$AAa?$AAt?$AAo?$AAr?$AAs@ 00154ba8     network.obj
 0002:00013c00       ??_C@_1CK@LFMAJJKO@?$AAO?$AAp?$AAe?$AAr?$AAa?$AAt?$AAo?$AAr?$AA?5?$AAf?$AAo?$AAr?$AAm?$AAa?$AAt?$AA?5?$AA?$DN?$AA?5?$AA?$CF?$AAd?$AA?$AA@ 00154c00     network.obj
 0002:00013c30       ??_C@_1HI@PIKENFNF@?$AAm?$AAp?$AAF?$AAn?$AAS?$AAw?$AAi?$AAS?$AAt?$AAa?$AAr?$AAt?$AAP?$AAL?$AAM?$AAN?$AAS?$AAe?$AAa?$AAr?$AAc?$AAh?$AA?5?$AAi?$AAs?$AA?5?$AAN?$AAO?$AAT?$AA?5?$AAi?$AAm@ 00154c30     network.obj
 0002:00013ce8       ??_C@_1FG@EKOIBMAI@?$AAF?$AAa?$AAi?$AAl?$AAe?$AAd?$AA?5?$AAt?$AAo?$AA?5?$AAU?$AAn?$AAr?$AAe?$AAg?$AAi?$AAs?$AAt?$AAe?$AAr?$AA?5?$AAF?$AAr?$AAo?$AAm?$AA?5?$AAt?$AAh?$AAe?$AA?5?$AAn?$AAe@ 00154ce8     network.obj
 0002:00013d40       ??_C@_1KK@GLCADCCH@?$AAG?$AAe?$AAt?$AAR?$AAe?$AAg?$AAi?$AAs?$AAt?$AAr?$AAa?$AAt?$AAi?$AAo?$AAn?$AAS?$AAt?$AAa?$AAt?$AAu?$AAs?$AA?3?$AA?5?$AAm?$AA_?$AAd?$AAw?$AA1?$AAx?$AAS?$AAv?$AAr@ 00154d40     network.obj
 0002:00013dec       ??_C@_1DC@HOCICHOG@?$AAG?$AAe?$AAt?$AA?5?$AAI?$AAn?$AAv?$AAa?$AAl?$AAi?$AAd?$AA?5?$AAs?$AAy?$AAs?$AAP?$AAr?$AAe?$AAf?$AA?5?$AA?$DN?$AA?5?$AA?$CF?$AAd?$AA?$AA@ 00154dec     network.obj
 0002:00013e20       ??_C@_1DG@CNKGFEPK@?$AAS?$AAw?$AAi?$AAS?$AAe?$AAt?$AAT?$AAe?$AAm?$AAp?$AAM?$AAo?$AAd?$AAe?$AAP?$AAr?$AAe?$AAf?$AA?5?$AAr?$AAc?$AA?5?$AA?$DN?$AA?5?$AA?$CF?$AAd?$AA?$AA@ 00154e20     network.obj
 0002:00013e58       ??_C@_06LHKKIPJE@Sprint?$AA@ 00154e58     network.obj
 0002:00013e60       ??_C@_07LOKFIKKP@Verizon?$AA@ 00154e60     network.obj
 0002:00013e68       ??_C@_0O@NAKMDDBD@China?5Telecom?$AA@ 00154e68     network.obj
 0002:00013e78       ??_C@_1EC@NLGMBINA@?$AAR?$AAe?$AAa?$AAd?$AA?5?$AAB?$AAa?$AAn?$AAn?$AAe?$AAr?$AA?5?$AAN?$AAa?$AAm?$AAe?$AA?$CB?$AA?5?$AAU?$AAs?$AAe?$AA?5?$AAo?$AAl?$AAd?$AA?5?$AAm?$AAe?$AAt?$AAh?$AAo?$AAd@ 00154e78     network.obj
 0002:00013ef8       ??_C@_1FI@FCAIJPKC@?$AAC?$AAR?$AAa?$AAd?$AAi?$AAo?$AA?3?$AA?3?$AAC?$AAh?$AAe?$AAc?$AAk?$AAC?$AAu?$AAr?$AAr?$AAe?$AAn?$AAt?$AAR?$AAU?$AAI?$AAM?$AA?5?$AAf?$AAa?$AAi?$AAl?$AAe?$AAd?$AA?0@ 00154ef8     network.obj
 0002:00013f50       ??_C@_1DC@KBDHOJEM@?$AAC?$AAR?$AAa?$AAd?$AAi?$AAo?$AA?3?$AA?3?$AAC?$AAh?$AAe?$AAc?$AAk?$AAC?$AAu?$AAr?$AAr?$AAe?$AAn?$AAt?$AAR?$AAU?$AAI?$AAM?$AA?$AA@ 00154f50     network.obj
 0002:00013fc8       ??_C@_1IM@LGFNGCPK@?$AAm?$AAp?$AAF?$AAn?$AAS?$AAw?$AAi?$AAS?$AAe?$AAt?$AAN?$AAe?$AAt?$AAw?$AAo?$AAr?$AAk?$AAP?$AAr?$AAe?$AAf?$AAe?$AAr?$AAe?$AAn?$AAc?$AAe?$AAG?$AAo?$AAb?$AAi?$AA?5@ 00154fc8     network.obj
 0002:00014058       ??_C@_1EC@GCMNOOPM@?$AAm?$AAp?$AAF?$AAn?$AAS?$AAw?$AAi?$AAG?$AAe?$AAt?$AAG?$AAs?$AAm?$AAS?$AAy?$AAs?$AAt?$AAe?$AAm?$AAS?$AAt?$AAa?$AAt?$AAu?$AAs?$AA?5?$AAF?$AAa?$AAi?$AAl?$AAe?$AAd@ 00155058     network.obj
 0002:0001409c       ??_C@_1DI@JDBCIPIH@?$AAF?$AAa?$AAi?$AAl?$AAe?$AAd?$AA?5?$AAt?$AAo?$AA?5?$AAs?$AAe?$AAt?$AA?5?$AAt?$AAh?$AAe?$AA?5?$AAP?$AAL?$AAM?$AAN?$AA?5?$AAm?$AAo?$AAd?$AAe?$AA?$AA@ 0015509c     network.obj
 0002:000140d8       ??_C@_1GO@CLHFKDGJ@?$AAm?$AAp?$AAF?$AAn?$AAS?$AAw?$AAi?$AAS?$AAe?$AAt?$AAP?$AAL?$AAM?$AAN?$AAM?$AAo?$AAd?$AAe?$AA?5?$AAr?$AAe?$AAt?$AAu?$AAr?$AAn?$AAs?$AA?5?$AAr?$AAc?$AA?5?$AA?$DN?$AA?5@ 001550d8     network.obj
 0002:00014148       ??_C@_1FG@LOEMKCNJ@?$AAR?$AAe?$AAg?$AAi?$AAs?$AAt?$AAe?$AAr?$AAO?$AAn?$AAN?$AAe?$AAt?$AAw?$AAo?$AAr?$AAk?$AA?5?$AAc?$AAa?$AAl?$AAl?$AAe?$AAd?$AA?5?$AAw?$AAi?$AAt?$AAh?$AA?5?$AA?$DN?$AA?5@ 00155148     network.obj
 0002:000141a0       ??_C@_1HC@MLCMEIDC@?$AAR?$AAe?$AAg?$AAi?$AAs?$AAt?$AAe?$AAr?$AAO?$AAn?$AAN?$AAe?$AAt?$AAw?$AAo?$AAr?$AAk?$AA?3?$AA?5?$AAd?$AAw?$AA1?$AAx?$AAS?$AAv?$AAr?$AAS?$AAt?$AAa?$AAt?$AAe?$AA?5@ 001551a0     network.obj
 0002:00014218       ??_C@_1EE@DIOLKGFB@?$AAS?$AAw?$AAi?$AAG?$AAe?$AAt?$AAH?$AAd?$AAr?$AAS?$AAr?$AAv?$AAS?$AAt?$AAa?$AAt?$AAe?$AA?5?$AAf?$AAa?$AAi?$AAl?$AAe?$AAd?$AA?0?$AA?5?$AAr?$AAc?$AA?5?$AA?$DN?$AA?5?$AA?$CF@ 00155218     network.obj
 0002:00014260       ??_C@_1FA@FMMOGEGK@?$AAS?$AAw?$AAi?$AAG?$AAe?$AAt?$AAS?$AAe?$AAr?$AAv?$AAi?$AAc?$AAe?$AAI?$AAn?$AAd?$AAi?$AAc?$AAa?$AAt?$AAi?$AAo?$AAn?$AA?5?$AAf?$AAa?$AAi?$AAl?$AAe?$AAd?$AA?0?$AA?5@ 00155260     network.obj
 0002:000142b0       ??_C@_1CK@HFDDBPDA@?$AAR?$AAI?$AAL?$AA_?$AAC?$AAA?$AAL?$AAL?$AAS?$AAT?$AAA?$AAT?$AA_?$AAW?$AAA?$AAI?$AAT?$AAI?$AAN?$AAG?$AA?$AA@ 001552b0     Radio.obj
 0002:000142dc       ??_C@_1CM@GGHFGMNI@?$AAR?$AAI?$AAL?$AA_?$AAC?$AAA?$AAL?$AAL?$AAS?$AAT?$AAA?$AAT?$AA_?$AAI?$AAN?$AAC?$AAO?$AAM?$AAI?$AAN?$AAG?$AA?$AA@ 001552dc     Radio.obj
 0002:00014308       ??_C@_1CM@EHEKOKDB@?$AAR?$AAI?$AAL?$AA_?$AAC?$AAA?$AAL?$AAL?$AAS?$AAT?$AAA?$AAT?$AA_?$AAA?$AAL?$AAE?$AAR?$AAT?$AAI?$AAN?$AAG?$AA?$AA@ 00155308     Radio.obj
 0002:00014334       ??_C@_1CK@LLPADMII@?$AAR?$AAI?$AAL?$AA_?$AAC?$AAA?$AAL?$AAL?$AAS?$AAT?$AAA?$AAT?$AA_?$AAD?$AAI?$AAA?$AAL?$AAI?$AAN?$AAG?$AA?$AA@ 00155334     Radio.obj
 0002:00014360       ??_C@_1CI@GGLFIGAB@?$AAR?$AAI?$AAL?$AA_?$AAC?$AAA?$AAL?$AAL?$AAS?$AAT?$AAA?$AAT?$AA_?$AAO?$AAN?$AAH?$AAO?$AAL?$AAD?$AA?$AA@ 00155360     Radio.obj
 0002:00014388       ??_C@_1CI@NCINPMBG@?$AAR?$AAI?$AAL?$AA_?$AAC?$AAA?$AAL?$AAL?$AAS?$AAT?$AAA?$AAT?$AA_?$AAA?$AAC?$AAT?$AAI?$AAV?$AAE?$AA?$AA@ 00155388     Radio.obj
 0002:000143b0       ??_C@_1M@FGKNGGMD@?$AAd?$AAu?$AAm?$AAm?$AAy?$AA?$AA@ 001553b0     Radio.obj
 0002:000143bc       ??_C@_1BC@JCFAACCD@?$AAe?$AAr?$AAi?$AA_?$AAn?$AAa?$AAm?$AA2?$AA?$AA@ 001553bc     Radio.obj
 0002:000143d0       ??_C@_1BC@IAOFKNMN@?$AAe?$AAr?$AAi?$AA_?$AAn?$AAa?$AAm?$AA1?$AA?$AA@ 001553d0     Radio.obj
 0002:000158d4       ??_C@_1BI@KLDKABLF@?$AA?4?$AA?2?$AAR?$AAa?$AAd?$AAi?$AAo?$AA?4?$AAc?$AAp?$AAp?$AA?$AA@ 001568d4     Radio.obj
 0002:000158f0       ??_C@_1FK@GHLBOOMH@?$AAm?$AAp?$AAF?$AAn?$AAS?$AAw?$AAi?$AAG?$AAe?$AAt?$AAS?$AAe?$AAr?$AAv?$AAi?$AAn?$AAg?$AAN?$AAe?$AAt?$AAw?$AAo?$AAr?$AAk?$AAG?$AAo?$AAb?$AAi?$AA?5?$AAf?$AAa?$AAi@ 001568f0     Radio.obj
 0002:00015950       ??_C@_1IG@HOGPIDEJ@?$AAp?$AAi?$AAn?$AA?5?$AAs?$AAt?$AAa?$AAt?$AAu?$AAs?$AA?3?$AA?$CF?$AAd?$AA?0?$AA?5?$AAi?$AAn?$AAd?$AAe?$AAx?$AA?3?$AA?$CF?$AAd?$AA?0?$AA?5?$AAp?$AAi?$AAn?$AA1?$AA?5?$AAs?$AAt@ 00156950     Radio.obj
 0002:000159d8       ??_C@_1BI@MOONEFEJ@?$AAS?$AAt?$AAa?$AAt?$AAu?$AAs?$AA?5?$AA?$DN?$AA?5?$AA?$CF?$AAd?$AA?$AA@ 001569d8     Radio.obj
 0002:000159f0       ??_C@_1HC@KPCACJAH@?$AAF?$AAa?$AAi?$AAl?$AAe?$AAd?$AA?5?$AAt?$AAo?$AA?5?$AAu?$AAp?$AAd?$AAa?$AAt?$AAe?$AA?5?$AAt?$AAh?$AAe?$AA?5?$AAN?$AAe?$AAt?$AAw?$AAo?$AAr?$AAk?$AAT?$AAy?$AAp?$AAe@ 001569f0     Radio.obj
 0002:00015a68       ??_C@_1GO@PPBJMDAO@?$AAT?$AAh?$AAe?$AA?5?$AAr?$AAa?$AAd?$AAi?$AAo?$AA?5?$AAt?$AAe?$AAc?$AAh?$AAn?$AAo?$AAl?$AAo?$AAg?$AAy?$AA?5?$AAi?$AAs?$AA?3?$AA?5?$AA?$CF?$AAd?$AA?0?$AA?5?$AA0?$AA?9?$AAU@ 00156a68     Radio.obj
 0002:00015ad8       ??_C@_1BI@FJLDDKCH@?$AAN?$AAe?$AAt?$AAw?$AAo?$AAr?$AAk?$AAT?$AAy?$AAp?$AAe?$AA?$AA@ 00156ad8     Radio.obj
 0002:00015af0       ??_C@_1FG@IIMPGLEC@?$AAU?$AAn?$AAa?$AAb?$AAl?$AAe?$AA?5?$AAt?$AAo?$AA?5?$AAs?$AAt?$AAa?$AAr?$AAt?$AA?5?$AAN?$AAI?$AAI?$AAP?$AA?5?$AAI?$AAO?$AAT?$AAA?$AA?5?$AAP?$AAr?$AAo?$AAc?$AAe?$AAs@ 00156af0     Radio.obj
 0002:00015b48       ??_C@_19NJBOMLMI@?$AAs?$AAm?$AAs?$AAf?$AA?$AA@ 00156b48     Radio.obj
 0002:00015b54       ??_C@_17HFOCKFBD@?$AAs?$AAm?$AAs?$AA?$AA@ 00156b54     Radio.obj
 0002:00015b5c       ??_C@_1DI@GBDICIOO@?$AA?2?$AAW?$AAi?$AAn?$AAd?$AAo?$AAw?$AAs?$AA?2?$AAI?$AAO?$AAT?$AAA?$AAT?$AAh?$AAi?$AAn?$AAC?$AAl?$AAi?$AAe?$AAn?$AAt?$AA?4?$AAe?$AAx?$AAe?$AA?$AA@ 00156b5c     Radio.obj
 0002:00015bd8       ??_C@_07HMPBCEOB@Roaming?$AA@ 00156bd8     Radio.obj
 0002:00015be0       ??_C@_1IM@EGBINDMO@?$AAU?$AAn?$AAh?$AAa?$AAn?$AAd?$AAl?$AAe?$AA?5?$AAf?$AAi?$AAn?$AAa?$AAl?$AAE?$AAR?$AAI?$AAI?$AAd?$AA?5?$AA?$DN?$AA?5?$AA?$CF?$AAd?$AA?0?$AA?5?$AAn?$AAe?$AAw?$AAd?$AAw?$AA1@ 00156be0     Radio.obj
 0002:00015c70       ??_C@_1BGM@HFOOMDEB@?$AAU?$AAp?$AAd?$AAa?$AAt?$AAe?$AAC?$AAo?$AAm?$AAb?$AAi?$AAn?$AAe?$AAd?$AAS?$AAe?$AAr?$AAv?$AAi?$AAc?$AAe?$AAS?$AAt?$AAa?$AAt?$AAu?$AAs?$AA?3?$AA?5?$AAm?$AA_?$AAd@ 00156c70     Radio.obj
 0002:00015de0       ??_C@_1EC@IFJAPBHP@?$AAS?$AAw?$AAi?$AAG?$AAe?$AAt?$AAC?$AAu?$AAr?$AAr?$AAe?$AAn?$AAt?$AAB?$AAa?$AAs?$AAe?$AAS?$AAt?$AAa?$AAt?$AAi?$AAo?$AAn?$AA?5?$AAf?$AAa?$AAi?$AAl?$AAe?$AAd?$AA?$CB@ 00156de0     Radio.obj
 0002:00015e28       ??_C@_1II@LEHIBDEM@?$AAJ?$AAu?$AAs?$AAt?$AA?5?$AAs?$AAe?$AAn?$AAt?$AA?5?$AAt?$AAh?$AAe?$AA?5?$AAR?$AAI?$AAL?$AA_?$AAN?$AAO?$AAT?$AAI?$AAF?$AAY?$AA_?$AAN?$AAI?$AAT?$AAZ?$AA?5?$AAa?$AAf@ 00156e28     Radio.obj
 0002:00015eb0       ??_C@_1DC@FOBMFODB@?$AAN?$AAi?$AAt?$AAz?$AAT?$AAi?$AAm?$AAe?$AAD?$AAe?$AAl?$AAa?$AAy?$AAO?$AAn?$AAC?$AAl?$AAe?$AAa?$AAn?$AAb?$AAo?$AAo?$AAt?$AA?$AA@ 00156eb0     Radio.obj
 0002:00015ee4       ??_C@_1O@GINMMDNN@?$AAS?$AAy?$AAs?$AAt?$AAe?$AAm?$AA?$AA@ 00156ee4     Radio.obj
 0002:00015ef8       ??_C@_1EM@FIBFKGCO@?$AAA?$AAS?$AAS?$AAE?$AAR?$AAT?$AAI?$AAO?$AAN?$AA?5?$AAF?$AAA?$AAI?$AAL?$AAU?$AAR?$AAE?$AA?3?$AA?5?$AA?$DN?$AA?$DN?$AA?$DN?$AA?$DO?$AAN?$AAU?$AAL?$AAL?$AA?5?$AA?$CB?$AA?$DN?$AA?5?$AAp@ 00156ef8     Radio.obj
 0002:00015f44       ??_C@_1DG@EJCGFIJL@?$AAu?$AAn?$AAk?$AAn?$AAo?$AAw?$AAn?$AA?5?$AAD?$AAo?$AAr?$AAm?$AAa?$AAn?$AAc?$AAy?$AA?5?$AAs?$AAt?$AAa?$AAt?$AAe?$AA?5?$AA?3?$AA?$CF?$AAd?$AA?$AA@ 00156f44     Radio.obj
 0002:00015f7c       ??_C@_1DO@CHIINPHC@?$AAG?$AAe?$AAt?$AAD?$AAu?$AAn?$AAC?$AAa?$AAl?$AAl?$AAI?$AAn?$AAf?$AAo?$AA?5?$AAf?$AAa?$AAi?$AAl?$AAe?$AAd?$AA?5?$AAr?$AAe?$AAt?$AA?5?$AA?$DN?$AA?5?$AA?$CF?$AAd?$AA?$AA@ 00156f7c     Radio.obj
 0002:00015fc0       ??_C@_1EC@MBOBIEPK@?$AAG?$AAe?$AAt?$AAD?$AAo?$AAr?$AAm?$AAa?$AAn?$AAc?$AAy?$AAS?$AAt?$AAa?$AAt?$AAe?$AA?5?$AAf?$AAa?$AAi?$AAl?$AAe?$AAd?$AA?5?$AAr?$AAe?$AAt?$AA?5?$AA?$DN?$AA?5?$AA?$CF?$AAd@ 00156fc0     Radio.obj
 0002:00016008       ??_C@_1FO@LPIPHICA@?$AAA?$AAS?$AAS?$AAE?$AAR?$AAT?$AAI?$AAO?$AAN?$AA?5?$AAF?$AAA?$AAI?$AAL?$AAU?$AAR?$AAE?$AA?3?$AA?5?$AA?$DN?$AA?$DN?$AA?$DN?$AA?$DO?$AAm?$AAd?$AAm?$AAI?$AAn?$AAf?$AAo?$AA?4?$AAd@ 00157008     Radio.obj
 0002:00016068       ??_C@_1BCE@PLBBKEKL@?$AAE?$AAi?$AAt?$AAh?$AAe?$AAr?$AA?5?$AAM?$AAN?$AAC?$AA?5?$AAo?$AAr?$AA?5?$AAM?$AAC?$AAC?$AA?5?$AAi?$AAs?$AA?5?$AAc?$AAh?$AAa?$AAn?$AAg?$AAe?$AAd?$AA?4?$AA?5?$AAN?$AAe@ 00157068     Radio.obj
 0002:00016190       ??_C@_1GC@KMMLLIHO@?$AAF?$AAo?$AAr?$AAc?$AAi?$AAn?$AAg?$AA?5?$AAt?$AAh?$AAe?$AA?5?$AAm?$AA_?$AAd?$AAw?$AAC?$AAu?$AAr?$AAr?$AAe?$AAn?$AAt?$AAS?$AAy?$AAs?$AAt?$AAe?$AAm?$AAT?$AAy?$AAp@ 00157190     Radio.obj
 0002:000161f8       ??_C@_1KM@IEPMHEJF@?$AAC?$AAo?$AAu?$AAl?$AAd?$AA?5?$AAN?$AAO?$AAT?$AA?5?$AAg?$AAe?$AAt?$AA?5?$AAp?$AAh?$AAo?$AAn?$AAe?$AA?5?$AAn?$AAu?$AAm?$AAb?$AAe?$AAr?$AA?5?$AAf?$AAr?$AAo?$AAm?$AA?5@ 001571f8     Radio.obj
 0002:000162a4       ??_C@_1DO@IAKOFNDC@?$AAE?$AAR?$AAR?$AAO?$AAR?$AA?5?$AAP?$AAh?$AAo?$AAn?$AAe?$AA?5?$AAn?$AAu?$AAm?$AAb?$AAe?$AAr?$AA?5?$AAl?$AAe?$AAn?$AAg?$AAt?$AAh?$AA?5?$AA?$DN?$AA?5?$AA?$CF?$AAd?$AA?$AA@ 001572a4     Radio.obj
 0002:000162e4       ??_C@_1CE@JBFDIICD@?$AAP?$AAh?$AAo?$AAn?$AAe?$AA?5?$AAn?$AAu?$AAm?$AAb?$AAe?$AAr?$AA?5?$AA?$DN?$AA?5?$AA?$CF?$AAs?$AA?$AA@ 001572e4     Radio.obj
 0002:00016308       ??_C@_1EM@GPJGBFFA@?$AAS?$AAw?$AAi?$AAG?$AAe?$AAt?$AAP?$AAh?$AAo?$AAn?$AAe?$AAN?$AAu?$AAm?$AAb?$AAe?$AAr?$AA?5?$AAf?$AAa?$AAi?$AAl?$AAe?$AAd?$AA?0?$AA?5?$AAe?$AAr?$AAr?$AAo?$AAr?$AA?5@ 00157308     Radio.obj
 0002:00016390       ??_C@_1FO@MLPKHIPI@?$AAE?$AAx?$AAe?$AAc?$AAu?$AAt?$AAe?$AAC?$AAo?$AAm?$AAm?$AAa?$AAn?$AAd?$AA?3?$AA?5?$AAD?$AAo?$AAn?$AA?8?$AAt?$AA?5?$AAk?$AAn?$AAo?$AAw?$AA?5?$AAt?$AAo?$AA?5?$AAh?$AAa@ 00157390     Radio.obj
 0002:000163f0       ??_C@_1GO@FIIHCNMN@?$AAG?$AAe?$AAt?$AAE?$AAq?$AAu?$AAi?$AAp?$AAm?$AAe?$AAn?$AAt?$AAS?$AAt?$AAa?$AAt?$AAe?$AA?5?$AAr?$AAe?$AAt?$AAu?$AAr?$AAn?$AAs?$AA?5?$AAh?$AAr?$AA?5?$AA?$DN?$AA?5?$AA0@ 001573f0     Radio.obj
 0002:00016460       ??_C@_1CI@BIKECOH@?$AAE?$AAx?$AAe?$AAc?$AAu?$AAt?$AAi?$AAn?$AAg?$AA?5?$AAA?$AAP?$AAI?$AAI?$AAD?$AA?3?$AA?5?$AA?$CF?$AAd?$AA?$AA@ 00157460     Radio.obj
 0002:00016488       ??_C@_1KC@BNFNCHDA@?$AAF?$AAa?$AAi?$AAl?$AAe?$AAd?$AA?5?$AAt?$AAo?$AA?5?$AAc?$AAr?$AAe?$AAa?$AAt?$AAe?$AA?5?$AAt?$AAh?$AAe?$AA?5?$AAr?$AAe?$AAg?$AAi?$AAs?$AAt?$AAr?$AAy?$AA?5?$AAH?$AAK@ 00157488     Radio.obj
 0002:0001652c       ??_C@_1CK@CECJDBPC@?$AAS?$AAe?$AAc?$AAu?$AAr?$AAi?$AAt?$AAy?$AA?2?$AAP?$AAh?$AAo?$AAn?$AAe?$AA?2?$AAN?$AAo?$AAL?$AAo?$AAg?$AA?$AA@ 0015752c     Radio.obj
 0002:00016558       ??_C@_1KE@GFPLAFFG@?$AAF?$AAa?$AAi?$AAl?$AAe?$AAd?$AA?5?$AAt?$AAo?$AA?5?$AAc?$AAr?$AAe?$AAa?$AAt?$AAe?$AA?5?$AAt?$AAh?$AAe?$AA?5?$AAr?$AAe?$AAg?$AAi?$AAs?$AAt?$AAr?$AAy?$AA?5?$AAH?$AAK@ 00157558     Radio.obj
 0002:000165fc       ??_C@_1CM@NCMBAEHJ@?$AAS?$AAe?$AAc?$AAu?$AAr?$AAi?$AAt?$AAy?$AA?2?$AAE?$AAC?$AAa?$AAl?$AAl?$AAW?$AAi?$AAt?$AAh?$AAS?$AAI?$AAM?$AA?$AA@ 001575fc     Radio.obj
 0002:00016628       ??_C@_1KK@JMEKONJP@?$AAF?$AAa?$AAi?$AAl?$AAe?$AAd?$AA?5?$AAt?$AAo?$AA?5?$AAc?$AAr?$AAe?$AAa?$AAt?$AAe?$AA?5?$AAt?$AAh?$AAe?$AA?5?$AAr?$AAe?$AAg?$AAi?$AAs?$AAt?$AAr?$AAy?$AA?5?$AAH?$AAK@ 00157628     Radio.obj
 0002:000166d4       ??_C@_19DOLMIDJD@?$AAL?$AAi?$AAs?$AAt?$AA?$AA@ 001576d4     Radio.obj
 0002:000166e0       ??_C@_1DC@HDHLKHL@?$AAS?$AAe?$AAc?$AAu?$AAr?$AAi?$AAt?$AAy?$AA?2?$AAE?$AAC?$AAa?$AAl?$AAl?$AAW?$AAi?$AAt?$AAh?$AAo?$AAu?$AAt?$AAS?$AAI?$AAM?$AA?$AA@ 001576e0     Radio.obj
 0002:00016714       ??_C@_17NMIAMFPP@?$AA?$CK?$AA?$CF?$AAs?$AA?$AA@ 00157714     Radio.obj
 0002:0001671c       ??_C@_17MDMPNONE@?$AA?$CD?$AA?$CF?$AAs?$AA?$AA@ 0015771c     Radio.obj
 0002:00016828       ??_C@_1IK@BCLJMHD@?$AAW?$AAa?$AAi?$AAt?$AA4?$AAA?$AAT?$AAC?$AAo?$AAn?$AAn?$AAe?$AAc?$AAt?$AAe?$AAd?$AA?5?$AAS?$AAe?$AAt?$AAC?$AAa?$AAl?$AAl?$AAS?$AAt?$AAa?$AAt?$AAu?$AAs?$AA?$CI?$AAR@ 00157828     Radio.obj
 0002:000168b4       ??_C@_1DO@HOEMIDAL@?$AAs?$AAe?$AAn?$AAd?$AAi?$AAn?$AAg?$AA?5?$AAo?$AAu?$AAt?$AA?5?$AAR?$AAI?$AAL?$AA_?$AAN?$AAO?$AAT?$AAI?$AAF?$AAY?$AA_?$AAC?$AAO?$AAN?$AAN?$AAE?$AAC?$AAT?$AA?$AA@ 001578b4     Radio.obj
 0002:000168f4       ??_C@_1DI@CJMPANKH@?$AAD?$AAa?$AAt?$AAa?$AAD?$AAo?$AAr?$AAm?$AAa?$AAn?$AAc?$AAy?$AAP?$AAo?$AAl?$AAl?$AAi?$AAn?$AAg?$AAI?$AAn?$AAt?$AAe?$AAr?$AAv?$AAa?$AAl?$AA?$AA@ 001578f4     Radio.obj
 0002:0001692c       ??_C@_17HEELGIAM@?$AAR?$AAI?$AAL?$AA?$AA@ 0015792c     Radio.obj
 0002:00016938       ??_C@_1JC@KPHFCMDA@?$AAF?$AAa?$AAi?$AAl?$AA?5?$AAt?$AAo?$AA?5?$AAw?$AAa?$AAi?$AAt?$AA?5?$AAf?$AAo?$AAr?$AA?5?$AAC?$AAO?$AAN?$AAN?$AAE?$AAC?$AAT?$AA?5?$AAs?$AAt?$AAr?$AAi?$AAn?$AAg?$AA?5@ 00157938     Radio.obj
 0002:000169d0       ??_C@_1HA@CCAONHF@?$AAW?$AAa?$AAi?$AAt?$AAi?$AAn?$AAg?$AA?5?$AAf?$AAo?$AAr?$AA?5?$AAA?$AAT?$AA?5?$AAC?$AAO?$AAN?$AAN?$AAE?$AAC?$AAT?$AA?5?$AAF?$AAA?$AAI?$AAL?$AA?3?$AA?5?$AAC?$AAl?$AAo@ 001579d0     Radio.obj
 0002:00016a40       ??_C@_1EA@GBJPDKFM@?$AAb?$AAe?$AAf?$AAo?$AAr?$AAe?$AA?5?$AAc?$AAl?$AAo?$AAs?$AAi?$AAn?$AAg?$AA?5?$AAd?$AAa?$AAt?$AAa?$AA?5?$AAp?$AAo?$AAr?$AAt?$AA?5?$AAb?$AAu?$AAf?$AA?3?$AA?$CF?$AAs?$AA?$AA@ 00157a40     Radio.obj
 0002:00016a80       ??_C@_1IG@DFHOCMDG@?$AAG?$AAi?$AAv?$AAe?$AAu?$AAp?$AA?5?$AAo?$AAn?$AA?5?$AAW?$AAa?$AAi?$AAt?$AA?5?$AAf?$AAo?$AAr?$AA?5?$AAA?$AAT?$AA?5?$AAC?$AAO?$AAN?$AAN?$AAE?$AAC?$AAT?$AA?5?$AAb?$AAe@ 00157a80     Radio.obj
 0002:00016b08       ??_C@_1GC@PEKCALMO@?$AAN?$AAo?$AAt?$AA?5?$AAw?$AAo?$AAr?$AAt?$AAh?$AAy?$AA?5?$AAt?$AAo?$AA?5?$AAc?$AAo?$AAn?$AAt?$AAi?$AAn?$AAu?$AAe?$AA?5?$AAb?$AAc?$AAo?$AAs?$AA?5?$AAr?$AAe?$AAt?$AAu@ 00157b08     Radio.obj
 0002:00016b6c       ??_C@_1BC@LDNMIJDI@?$AAb?$AAu?$AAf?$AA?5?$AAc?$AA?3?$AA?$CF?$AAs?$AA?$AA@ 00157b6c     Radio.obj
 0002:00016b80       ??_C@_1HM@INJPKNLB@?$AAN?$AAo?$AAt?$AA?5?$AAw?$AAo?$AAr?$AAt?$AAh?$AAy?$AA?5?$AAt?$AAo?$AA?5?$AAc?$AAo?$AAn?$AAt?$AAi?$AAn?$AAu?$AAe?$AA?5?$AAb?$AAc?$AAo?$AAs?$AA?5?$AAO?$AAK?$AA?5?$AAr@ 00157b80     Radio.obj
 0002:00016c00       ??_C@_1EA@OBBPJGPO@?$AAg?$AAo?$AAt?$AA?5?$AAp?$AAp?$AAp?$AA?5?$AAp?$AAa?$AAc?$AAk?$AAe?$AAt?$AAi?$AAn?$AAg?$AA?0?$AA?5?$AAc?$AAo?$AAn?$AAt?$AAi?$AAn?$AAu?$AAe?$AA?0?$AA?5?$AA?$CF?$AAs?$AA?$AA@ 00157c00     Radio.obj
 0002:00016c40       ??_C@_1DG@LAPDCGFO@?$AAG?$AAo?$AAt?$AA?5?$AA?$CC?$AAC?$AAO?$AAN?$AAN?$AAE?$AAC?$AAT?$AA?$CC?$AA?5?$AAc?$AAo?$AAn?$AAt?$AAi?$AAn?$AAu?$AAe?$AA?0?$AA?5?$AA?$CF?$AAs?$AA?$AA@ 00157c40     Radio.obj
 0002:00016c78       ??_C@_1BC@FMBOOCAG@?$AAb?$AAu?$AAf?$AA?5?$AAb?$AA?3?$AA?$CF?$AAs?$AA?$AA@ 00157c78     Radio.obj
 0002:00016c90       ??_C@_1GI@MDBHNADI@?$AAD?$AAe?$AAt?$AAe?$AAc?$AAt?$AA?5?$AAE?$AAV?$AA_?$AAP?$AAO?$AAW?$AAE?$AAR?$AA?5?$AAw?$AAh?$AAi?$AAl?$AAe?$AA?5?$AAw?$AAa?$AAi?$AAt?$AAi?$AAn?$AAg?$AA?5?$AAf?$AAo@ 00157c90     Radio.obj
 0002:00016cf8       ??_C@_1HK@PMJGKLKG@?$AAK?$AAe?$AAe?$AAp?$AA?5?$AAt?$AAr?$AAy?$AAi?$AAn?$AAg?$AA?5?$AAb?$AAc?$AAo?$AAs?$AA?5?$AAw?$AAa?$AAi?$AAt?$AAi?$AAn?$AAg?$AA?5?$AAf?$AAo?$AAr?$AA?5?$AAA?$AAT?$AA?5@ 00157cf8     Radio.obj
 0002:00016d74       ??_C@_02GIPFHKNO@OK?$AA@   00157d74     Radio.obj
 0002:00016d78       ??_C@_0L@KDDNELKK@NO?5CARRIER?$AA@ 00157d78     Radio.obj
 0002:00016d84       ??_C@_05MBDEGLCK@ERROR?$AA@ 00157d84     Radio.obj
 0002:00016d8c       ??_C@_01PJKLJHI@?$HO?$AA@  00157d8c     Radio.obj
 0002:00016d90       ??_C@_1EO@CMANFHIK@?$AAS?$AAo?$AAr?$AAr?$AAy?$AA?0?$AA?5?$AAi?$AAt?$AA?8?$AAs?$AA?5?$AAa?$AA?5?$AAj?$AAo?$AAk?$AAe?$AA?5?$AAf?$AAr?$AAo?$AAm?$AA?5?$AAM?$AAS?$AA?4?$AA?5?$AAK?$AAe?$AAe?$AAp@ 00157d90     Radio.obj
 0002:00016de0       ??_C@_1FC@NBGHAKCH@?$AAG?$AAo?$AAt?$AA?5?$AA?$CC?$AAC?$AAO?$AAN?$AAN?$AAE?$AAC?$AAT?$AA?$CC?$AA?$DP?$AA?5?$AAb?$AAu?$AAf?$AAf?$AAe?$AAr?$AA?5?$AA?$DN?$AA?5?$AA?$CF?$AAs?$AA?5?$AA?0?$AA?5?$AAd?$AAw?$AAR@ 00157de0     Radio.obj
 0002:00016e34       ??_C@_1BC@LHCJFJAF@?$AAb?$AAu?$AAf?$AA?5?$AAa?$AA?3?$AA?$CF?$AAs?$AA?$AA@ 00157e34     Radio.obj
 0002:00016e48       ??_C@_07FNNMGOPK@CONNECT?$AA@ 00157e48     Radio.obj
 0002:00017028       ??_C@_1DC@ILLNCPI@?$AA0?$AA?4?$AA?5?$AAE?$AAm?$AAe?$AAr?$AAg?$AAe?$AAn?$AAc?$AAy?$AA?5?$AAl?$AAi?$AAs?$AAt?$AA?5?$AA?$CF?$AAd?$AA?3?$AA?5?$AA?$CF?$AAs?$AA?$AA@ 00158028     Radio.obj
 0002:00017060       ??_C@_1EK@EHBADBPN@?$AAR?$AAI?$AAL?$AAE?$AAm?$AAe?$AAr?$AAg?$AAe?$AAn?$AAc?$AAy?$AA?5?$AAn?$AAu?$AAm?$AAb?$AAe?$AAr?$AA?5?$AAr?$AAe?$AAg?$AAi?$AAs?$AAt?$AAr?$AAy?$AA?5?$AAa?$AAb?$AAs@ 00158060     Radio.obj
 0002:000170ac       ??_C@_1CA@PEHDDLFM@?$AAS?$AAe?$AAt?$AAE?$AAn?$AAu?$AAm?$AA?5?$AAf?$AAa?$AAi?$AAl?$AAe?$AAd?$AA?$CB?$AA?$AA@ 001580ac     Radio.obj
 0002:000170cc       ??_C@_1DI@FBIJAMBO@?$AAR?$AAe?$AAa?$AAd?$AAi?$AAn?$AAg?$AA?5?$AAE?$AAm?$AAe?$AAr?$AAg?$AAe?$AAn?$AAc?$AAy?$AA?5?$AAN?$AAu?$AAm?$AAb?$AAe?$AAr?$AA?5?$AA?$CF?$AAs?$AA?$AA@ 001580cc     Radio.obj
 0002:00017104       ??_C@_13DEFPDAGF@?$AA?0?$AA?$AA@ 00158104     Radio.obj
 0002:00017108       ??_C@_1CA@FAHDNPE@?$AAR?$AAi?$AAl?$AAE?$AAm?$AAe?$AAr?$AAg?$AAe?$AAn?$AAc?$AAy?$AAN?$AAu?$AAm?$AA?$AA@ 00158108     Radio.obj
 0002:00017128       ??_C@_1CE@PKINJKKB@?$AAC?$AAl?$AAe?$AAa?$AAr?$AAE?$AAn?$AAu?$AAm?$AA?5?$AAf?$AAa?$AAi?$AAl?$AAe?$AAd?$AA?$CB?$AA?$AA@ 00158128     Radio.obj
 0002:0001714c       ??_C@_1BM@BDJPLGHF@?$AAR?$AAI?$AAL?$AA?2?$AAE?$AAm?$AAe?$AAr?$AAg?$AAe?$AAn?$AAc?$AAy?$AA?$AA@ 0015814c     Radio.obj
 0002:00017168       ??_C@_1BI@MACJDEKE@?$AAF?$AAo?$AAr?$AAc?$AAe?$AAU?$AAp?$AAd?$AAa?$AAt?$AAe?$AA?$AA@ 00158168     Radio.obj
 0002:000171d0       ??_C@_1HG@EOIBBOLJ@?$AAF?$AAa?$AAi?$AAl?$AAe?$AAd?$AA?5?$AAt?$AAo?$AA?5?$AAr?$AAe?$AAa?$AAd?$AA?5?$AAt?$AAh?$AAe?$AA?5?$AAI?$AAs?$AAO?$AAS?$AAE?$AAx?$AAp?$AAe?$AAc?$AAt?$AAN?$AAI?$AAT@ 001581d0     Radio.obj
 0002:00017248       ??_C@_1BO@OCKECDNL@?$AAI?$AAs?$AAO?$AAS?$AAE?$AAx?$AAp?$AAe?$AAc?$AAt?$AAN?$AAI?$AAT?$AAZ?$AA?$AA@ 00158248     Radio.obj
 0002:00017268       ??_C@_1IK@BDHLMAM@?$AAF?$AAa?$AAi?$AAl?$AAe?$AAd?$AA?5?$AAt?$AAo?$AA?5?$AAr?$AAe?$AAs?$AAe?$AAt?$AA?5?$AAD?$AAe?$AAl?$AAa?$AAy?$AAN?$AAI?$AAT?$AAZ?$AAN?$AAo?$AAt?$AAi?$AAf?$AAi?$AAc@ 00158268     Radio.obj
 0002:000172f8       ??_C@_1EC@LKEECJMO@?$AAD?$AAe?$AAl?$AAa?$AAy?$AAN?$AAI?$AAT?$AAZ?$AAN?$AAo?$AAt?$AAi?$AAf?$AAi?$AAc?$AAa?$AAt?$AAi?$AAo?$AAn?$AAO?$AAn?$AAC?$AAl?$AAe?$AAa?$AAn?$AAB?$AAo?$AAo?$AAt@ 001582f8     Radio.obj
 0002:00017340       ??_C@_1KG@ILFOMHIB@?$AAR?$AAI?$AAL?$AA?5?$AAs?$AAt?$AAa?$AAt?$AAe?$AA?5?$AAh?$AAa?$AAs?$AA?5?$AAe?$AAq?$AAS?$AAt?$AAa?$AAt?$AAe?$AA?5?$AA?$DN?$AA?5?$AA?$CF?$AAd?$AA?5?$AAb?$AAu?$AAt?$AA?5?$AAr@ 00158340     Radio.obj
 0002:000173e8       ??_C@_1CO@CNNDJLME@?$AAI?$AAn?$AAf?$AAe?$AAr?$AA?5?$AAM?$AAo?$AAd?$AAe?$AAm?$AA?5?$AAr?$AAe?$AAs?$AAe?$AAt?$AAt?$AAi?$AAn?$AAg?$AA?$CB?$AA?$AA@ 001583e8     Radio.obj
 0002:00017418       ??_C@_1HO@DGEMOOIL@?$AAC?$AAa?$AAn?$AAn?$AAo?$AAt?$AA?5?$AAd?$AAe?$AAt?$AAe?$AAr?$AAm?$AAi?$AAn?$AAe?$AA?5?$AAa?$AAc?$AAt?$AAi?$AAv?$AAe?$AA?5?$AAi?$AAn?$AAd?$AAe?$AAx?$AA?0?$AA?5?$AAr@ 00158418     Radio.obj
 0002:00017498       ??_C@_1EI@DPIPNIBI@?$AAm?$AAp?$AAF?$AAn?$AAS?$AAw?$AAi?$AAG?$AAe?$AAt?$AAE?$AAF?$AAi?$AAl?$AAe?$AAI?$AAn?$AAf?$AAo?$AA?5?$AAf?$AAa?$AAi?$AAl?$AAe?$AAd?$AA?0?$AA?5?$AAr?$AAc?$AA?5?$AA?$DN@ 00158498     Radio.obj
 0002:000174e0       ??_C@_1DA@FDKGGDNN@?$AAA?$AAc?$AAt?$AAi?$AAv?$AAa?$AAt?$AAe?$AAd?$AA?5?$AA?$DN?$AA?5?$AA?$CF?$AAd?$AA?0?$AA?5?$AAr?$AAc?$AA?5?$AA?$DN?$AA?5?$AA?$CF?$AAd?$AA?$AA@ 001584e0     Radio.obj
 0002:00017510       ??_C@_1DG@FKGAPPCC@?$AAF?$AAa?$AAi?$AAl?$AA?5?$AAt?$AAo?$AA?5?$AAp?$AAu?$AAb?$AAl?$AAi?$AAs?$AAh?$AA?5?$AAM?$AAD?$AAN?$AA?5?$AAl?$AAe?$AAn?$AAg?$AAt?$AAh?$AA?$AA@ 00158510     Radio.obj
 0002:00017548       ??_C@_1O@JGODHDHF@?$AAM?$AAD?$AAN?$AAL?$AAe?$AAn?$AA?$AA@ 00158548     Radio.obj
 0002:00017558       ??_C@_1EC@NHKFHNNI@?$AAS?$AAw?$AAi?$AAG?$AAe?$AAt?$AAT?$AAe?$AAc?$AAh?$AAP?$AAo?$AAw?$AAe?$AAr?$AAs?$AAa?$AAv?$AAe?$AAM?$AAo?$AAd?$AAe?$AA?$CI?$AA?$CJ?$AA?5?$AAF?$AAa?$AAi?$AAl?$AAe?$AAd@ 00158558     Radio.obj
 0002:000175a0       ??_C@_1JK@OBPPCMDP@?$AAS?$AAw?$AAi?$AAH?$AAW?$AAI?$AAn?$AAi?$AAt?$AAi?$AAa?$AAl?$AAi?$AAz?$AAe?$AAd?$AA?5?$AAf?$AAa?$AAi?$AAl?$AAe?$AAd?$AA?0?$AA?5?$AAm?$AA_?$AAp?$AAH?$AAW?$AAI?$AAn@ 001585a0     Radio.obj
 0002:0001763c       ??_C@_1BG@MJHELIBO@?$AAS?$AAw?$AAi?$AAA?$AAu?$AAx?$AAD?$AAL?$AAL?$AA?$DP?$AA?$AA@ 0015863c     Radio.obj
 0002:00017654       ??_C@_1CE@LNNMKKNE@?$AAH?$AAW?$AAS?$AAe?$AAt?$AAT?$AAe?$AAt?$AAh?$AAe?$AAr?$AAe?$AAd?$AAM?$AAo?$AAd?$AAe?$AA?$AA@ 00158654     Radio.obj
 0002:00017678       ??_C@_1CM@BGMEFFMM@?$AAH?$AAW?$AAS?$AAe?$AAt?$AAD?$AAe?$AAv?$AAi?$AAc?$AAe?$AAP?$AAo?$AAw?$AAe?$AAr?$AAS?$AAt?$AAa?$AAt?$AAe?$AA?$AA@ 00158678     Radio.obj
 0002:000176a8       ??_C@_1FG@BIKHNBHN@?$AAF?$AAa?$AAi?$AAl?$AA?5?$AAt?$AAo?$AA?5?$AAg?$AAe?$AAt?$AA?5?$AAa?$AAd?$AAd?$AAr?$AAe?$AAs?$AAs?$AA?5?$AAf?$AAo?$AAr?$AA?5?$AAH?$AAW?$AAI?$AAN?$AAI?$AAT?$AAI?$AAA@ 001586a8     Radio.obj
 0002:00017700       ??_C@_1CA@KAIDLGAK@?$AAS?$AAw?$AAi?$AAH?$AAW?$AAI?$AAn?$AAi?$AAt?$AAi?$AAa?$AAl?$AAi?$AAz?$AAe?$AA?$AA@ 00158700     Radio.obj
 0002:00017720       ??_C@_1CE@EHDKEFAJ@?$AAS?$AAw?$AAi?$AAH?$AAW?$AAU?$AAn?$AAI?$AAn?$AAi?$AAt?$AAi?$AAa?$AAl?$AAi?$AAz?$AAe?$AA?$AA@ 00158720     Radio.obj
 0002:00017744       ??_C@_1BM@BDMEONAP@?$AAS?$AAw?$AAi?$AAH?$AAW?$AAS?$AAe?$AAt?$AAP?$AAo?$AAw?$AAe?$AAr?$AA?$AA@ 00158744     Radio.obj
 0002:00017760       ??_C@_1BM@DGMPGGBB@?$AAS?$AAw?$AAi?$AAH?$AAW?$AAG?$AAe?$AAt?$AAP?$AAo?$AAw?$AAe?$AAr?$AA?$AA@ 00158760     Radio.obj
 0002:0001777c       ??_C@_1CE@EDGHLLPL@?$AAS?$AAw?$AAi?$AAH?$AAW?$AAG?$AAe?$AAt?$AAO?$AAE?$AAM?$AAI?$AAD?$AAS?$AAt?$AAr?$AAA?$AA?$AA@ 0015877c     Radio.obj
 0002:000177a0       ??_C@_1CM@PHHEGMOO@?$AAS?$AAw?$AAi?$AAH?$AAW?$AAR?$AAe?$AAg?$AAi?$AAs?$AAt?$AAe?$AAr?$AAC?$AAa?$AAl?$AAl?$AAb?$AAa?$AAc?$AAk?$AA?$AA@ 001587a0     Radio.obj
 0002:000177cc       ??_C@_1BM@HDFANJMM@?$AAH?$AAW?$AAE?$AAn?$AAa?$AAb?$AAl?$AAe?$AAA?$AAu?$AAd?$AAi?$AAo?$AA?$AA@ 001587cc     Radio.obj
 0002:000177e8       ??_C@_1BO@BFJGFNIP@?$AAH?$AAW?$AAG?$AAe?$AAt?$AAA?$AAu?$AAd?$AAi?$AAo?$AAP?$AAa?$AAt?$AAh?$AA?$AA@ 001587e8     Radio.obj
 0002:00017808       ??_C@_1CC@CMAGINCM@?$AAH?$AAW?$AAS?$AAe?$AAt?$AAV?$AAo?$AAl?$AAu?$AAm?$AAn?$AAL?$AAe?$AAv?$AAe?$AAl?$AA?$AA@ 00158808     Radio.obj
 0002:0001782c       ??_C@_1CG@MAIIFACA@?$AAH?$AAW?$AAI?$AAn?$AAi?$AAt?$AAi?$AAa?$AAt?$AAe?$AAH?$AAo?$AAs?$AAt?$AAB?$AAo?$AAo?$AAt?$AA?$AA@ 0015882c     Radio.obj
 0002:00017854       ??_C@_1BM@HNCBPPPM@?$AAS?$AAw?$AAi?$AAS?$AAB?$AAL?$AAA?$AAu?$AAx?$AA?4?$AAd?$AAl?$AAl?$AA?$AA@ 00158854     Radio.obj
 0002:00017870       ??_C@_1CC@FNEJBKJG@?$AAS?$AAw?$AAi?$AAA?$AAu?$AAx?$AAA?$AAP?$AAI?$AAD?$AAl?$AAl?$AAN?$AAa?$AAm?$AAe?$AA?$AA@ 00158870     Radio.obj
 0002:00017894       ??_C@_1CC@BJGAIDMD@?$AAR?$AAI?$AAL?$AA?2?$AAP?$AAo?$AAw?$AAe?$AAr?$AAC?$AAo?$AAn?$AAt?$AAr?$AAo?$AAl?$AA?$AA@ 00158894     Radio.obj
 0002:00017a98       ??_C@_1MC@HBKIBEIF@?$AAS?$AAW?$AAI?$AA_?$AAN?$AAO?$AAT?$AAI?$AAF?$AAY?$AA_?$AAO?$AAM?$AAA?$AAD?$AAM?$AA_?$AAS?$AAt?$AAa?$AAt?$AAe?$AA?3?$AA?5?$AAN?$AAe?$AAt?$AAw?$AAo?$AAr?$AAk?$AA?5@ 00158a98     Radio.obj
 0002:00017b60       ??_C@_1EM@GEOBOLKK@?$AAS?$AAW?$AAI?$AA_?$AAN?$AAO?$AAT?$AAI?$AAF?$AAY?$AA_?$AAO?$AAM?$AAA?$AAD?$AAM?$AA_?$AAN?$AAI?$AA_?$AAA?$AAl?$AAe?$AAr?$AAt?$AA?5?$AAi?$AAs?$AA?5?$AAr?$AAe?$AAc@ 00158b60     Radio.obj
 0002:00017bb0       ??_C@_1GM@OFJIGNBC@?$AAm?$AAp?$AAF?$AAn?$AAS?$AAw?$AAi?$AAS?$AAt?$AAa?$AAr?$AAt?$AAP?$AAL?$AAM?$AAN?$AAS?$AAe?$AAa?$AAr?$AAc?$AAh?$AA?5?$AAf?$AAa?$AAi?$AAl?$AAs?$AA?5?$AAo?$AAr?$AA?5@ 00158bb0     Radio.obj
 0002:00017c20       ??_C@_1EA@IMCIBGDP@?$AAm?$AAp?$AAF?$AAn?$AAS?$AAw?$AAi?$AAG?$AAe?$AAt?$AAP?$AAL?$AAM?$AAN?$AAS?$AAe?$AAl?$AAe?$AAc?$AAt?$AAi?$AAo?$AAn?$AA?5?$AAi?$AAs?$AA?5?$AAN?$AAU?$AAL?$AAL?$AA?$AA@ 00158c20     Radio.obj
 0002:00017c60       ??_C@_1GK@GGICLNNB@?$AAN?$AAu?$AAm?$AAb?$AAe?$AAr?$AA?5?$AAo?$AAf?$AA?5?$AAa?$AAv?$AAa?$AAi?$AAl?$AAa?$AAb?$AAl?$AAe?$AA?5?$AAP?$AAL?$AAM?$AAN?$AAs?$AA?5?$AA?$DN?$AA?5?$AA?$CF?$AAd?$AA?0?$AA?5@ 00158c60     Radio.obj
 0002:00017cd0       ??_C@_1FG@LPKCFANI@?$AAm?$AAp?$AAF?$AAn?$AAS?$AAw?$AAi?$AAG?$AAe?$AAt?$AAP?$AAL?$AAM?$AAN?$AAS?$AAe?$AAl?$AAe?$AAc?$AAt?$AAi?$AAo?$AAn?$AA?5?$AAf?$AAa?$AAi?$AAl?$AAe?$AAd?$AA?0?$AA?5@ 00158cd0     Radio.obj
 0002:00017d28       ??_C@_1CA@BPLNCKOJ@?$AAM?$AAo?$AAr?$AAe?$AA?5?$AAP?$AAL?$AAM?$AAN?$AA?$DP?$AA?5?$AA?$DN?$AA?5?$AA?$CF?$AAd?$AA?$AA@ 00158d28     Radio.obj
 0002:00017d48       ??_C@_1EK@JIBOILBL@?$AAC?$AAo?$AAu?$AAl?$AAd?$AA?5?$AAn?$AAo?$AAt?$AA?5?$AAl?$AAo?$AAc?$AAa?$AAt?$AAe?$AA?5?$AAt?$AAh?$AAe?$AA?5?$AAM?$AAC?$AAC?$AA?5?$AAa?$AAn?$AAd?$AA?5?$AAM?$AAN?$AAC@ 00158d48     Radio.obj
 0002:00017d94       ??_C@_07NFANNNEC@UNKNOWN?$AA@ 00158d94     Radio.obj
 0002:00017d9c       ??_C@_04OHGLKFFN@?$CF03d?$AA@ 00158d9c     Radio.obj
 0002:00017da4       ??_C@_04OGKJMPGK@?$CF02d?$AA@ 00158da4     Radio.obj
 0002:00017db0       ??_C@_1FA@KPEOFMMK@?$AAF?$AAa?$AAi?$AAl?$AAe?$AAd?$AA?5?$AAt?$AAo?$AA?5?$AAt?$AAa?$AAl?$AAk?$AA?5?$AAt?$AAo?$AA?5?$AAS?$AAI?$AAM?$AA?4?$AA?4?$AA?4?$AA?4?$AAc?$AAa?$AAn?$AAn?$AAo?$AAt?$AA?5@ 00158db0     Radio.obj
 0002:00017e00       ??_C@_1FG@MHBHDHDJ@?$AAm?$AAp?$AAF?$AAn?$AAS?$AAw?$AAi?$AAG?$AAe?$AAt?$AAG?$AAs?$AAm?$AAS?$AAy?$AAs?$AAt?$AAe?$AAm?$AAS?$AAt?$AAa?$AAt?$AAu?$AAs?$AA?5?$AAi?$AAs?$AA?5?$AAN?$AAO?$AAT@ 00158e00     Radio.obj
 0002:00017e58       ??_C@_1FC@FFMMIHHL@?$AAm?$AAp?$AAF?$AAn?$AAS?$AAw?$AAi?$AAG?$AAe?$AAt?$AAG?$AAs?$AAm?$AAS?$AAy?$AAs?$AAt?$AAe?$AAm?$AAS?$AAt?$AAa?$AAt?$AAu?$AAs?$AA?5?$AAF?$AAa?$AAi?$AAl?$AAe?$AAd@ 00158e58     Radio.obj
 0002:00017eb0       ??_C@_1GE@PPIJHLJG@?$AAH?$AAd?$AAr?$AA_?$AAP?$AAo?$AAw?$AAe?$AAr?$AAS?$AAa?$AAv?$AAe?$AA_?$AAE?$AAx?$AAi?$AAt?$AA?0?$AA?5?$AAf?$AAi?$AAn?$AAa?$AAl?$AA?5?$AAm?$AA_?$AAw?$AAP?$AAo?$AAw@ 00158eb0     Radio.obj
 0002:00017f18       ??_C@_1GG@ICIHBHCO@?$AAH?$AAd?$AAr?$AA_?$AAP?$AAo?$AAw?$AAe?$AAr?$AAS?$AAa?$AAv?$AAe?$AA_?$AAE?$AAn?$AAt?$AAe?$AAr?$AA?0?$AA?5?$AAf?$AAi?$AAn?$AAa?$AAl?$AA?5?$AAm?$AA_?$AAw?$AAP?$AAo@ 00158f18     Radio.obj
 0002:00017f80       ??_C@_1CC@JNAOBFPO@?$AAI?$AAO?$AAT?$AAA?$AA?5?$AAe?$AAv?$AAe?$AAn?$AAt?$AA?$DP?$AA?5?$AA?$DN?$AA?5?$AA?$CF?$AAd?$AA?$AA@ 00158f80     Radio.obj
 0002:00017fa4       ??_C@_1BO@GIFMJGL@?$AAS?$AAt?$AAa?$AAr?$AAt?$AA?5?$AAW?$AAA?$AAP?$AA?5?$AAI?$AAO?$AAT?$AAA?$AA?$AA@ 00158fa4     Radio.obj
 0002:00017fc8       ??_C@_1LM@KCKIFEM@?$AAS?$AAW?$AAI?$AA_?$AAN?$AAO?$AAT?$AAI?$AAF?$AAY?$AA_?$AAI?$AAO?$AAT?$AAA?$AA_?$AAS?$AAt?$AAa?$AAt?$AAu?$AAs?$AA?5?$AAE?$AAv?$AAe?$AAn?$AAt?$AA?9?$AA?$DO?$AA?$CF?$AAd@ 00158fc8     Radio.obj
 0002:00018084       ??_C@_1BK@LKIHCDFH@?$AAW?$AAA?$AAP?$AA?5?$AAU?$AAR?$AAI?$AA?5?$AA?$DN?$AA?5?$AA?$CF?$AAs?$AA?$AA@ 00159084     Radio.obj
 0002:000180a0       ??_C@_1FM@KPENFBCP@?$AAP?$AAo?$AAw?$AAe?$AAr?$AAS?$AAa?$AAv?$AAe?$AAE?$AAn?$AAt?$AAe?$AAr?$AA?0?$AA?5?$AAf?$AAi?$AAn?$AAa?$AAl?$AA?5?$AAm?$AA_?$AAw?$AAP?$AAo?$AAw?$AAe?$AAr?$AAS?$AAa@ 001590a0     Radio.obj
 0002:00018100       ??_C@_1FK@IBFEAEKE@?$AAP?$AAo?$AAw?$AAe?$AAr?$AAS?$AAa?$AAv?$AAe?$AAE?$AAx?$AAi?$AAt?$AA?0?$AA?5?$AAf?$AAi?$AAn?$AAa?$AAl?$AA?5?$AAm?$AA_?$AAw?$AAP?$AAo?$AAw?$AAe?$AAr?$AAS?$AAa?$AAv@ 00159100     Radio.obj
 0002:00018160       ??_C@_1HI@NGCFIAMC@?$AAI?$AAg?$AAn?$AAo?$AAr?$AAi?$AAn?$AAg?$AA?5?$AAS?$AAW?$AAI?$AA_?$AAN?$AAO?$AAT?$AAI?$AAF?$AAY?$AA_?$AAH?$AAd?$AAr?$AA_?$AAR?$AAs?$AAs?$AAi?$AA?5?$AAw?$AAh?$AAi@ 00159160     Radio.obj
 0002:000181d8       ??_C@_1HK@EODJBGNN@?$AAI?$AAg?$AAn?$AAo?$AAr?$AAi?$AAn?$AAg?$AA?5?$AAS?$AAW?$AAI?$AA_?$AAN?$AAO?$AAT?$AAI?$AAF?$AAY?$AA_?$AAR?$AAs?$AAs?$AAi?$AA_?$AAE?$AAc?$AAi?$AAo?$AA?5?$AAw?$AAh@ 001591d8     Radio.obj
 0002:00018258       ??_C@_1GA@DECDMBCE@?$AAO?$AAl?$AAd?$AA?5?$AAm?$AA_?$AAd?$AAw?$AAH?$AAd?$AAr?$AAS?$AAv?$AAr?$AAS?$AAt?$AAa?$AAt?$AAe?$AA?5?$AA?$DN?$AA?5?$AA?$CF?$AAd?$AA?0?$AA?5?$AAn?$AAe?$AAw?$AAd?$AAw?$AAH@ 00159258     Radio.obj
 0002:000182b8       ??_C@_1IA@LPDBEBLL@?$AAC?$AAa?$AAl?$AAl?$AA?5?$AAE?$AAr?$AAr?$AAo?$AAr?$AA?5?$AA?$DN?$AA?5?$AA0?$AAx?$AA?$CF?$AAx?$AA?0?$AA?5?$AAR?$AAi?$AAl?$AA?5?$AAw?$AAi?$AAl?$AAl?$AA?5?$AAS?$AAe?$AAn?$AAd@ 001592b8     Radio.obj
 0002:00018338       ??_C@_1IO@NOJNPNJC@?$AAW?$AAe?$AA?5?$AAh?$AAa?$AAv?$AAe?$AA?5?$AAa?$AA?5?$AAW?$AAP?$AAS?$AA?5?$AAc?$AAa?$AAl?$AAl?$AA?5?$AAg?$AAo?$AAi?$AAn?$AAg?$AA?5?$AAo?$AAn?$AA?0?$AA?5?$AAt?$AAh?$AAe@ 00159338     Radio.obj
 0002:000183c8       ??_C@_1O@BOCOOEDM@?$AAQ?$AAU?$AAE?$AAU?$AAE?$AAD?$AA?$AA@ 001593c8     Radio.obj
 0002:000183d8       ??_C@_1FM@GCBADMD@?$AAO?$AAl?$AAd?$AA?5?$AAm?$AA_?$AAd?$AAw?$AA1?$AAx?$AAS?$AAv?$AAr?$AAS?$AAt?$AAa?$AAt?$AAe?$AA?5?$AA?$DN?$AA?5?$AA?$CF?$AAd?$AA?0?$AA?5?$AAn?$AAe?$AAw?$AAd?$AAw?$AA1?$AAx@ 001593d8     Radio.obj
 0002:00018438       ??_C@_1HA@KNLKLDJF@?$AAI?$AAg?$AAn?$AAo?$AAr?$AAi?$AAn?$AAg?$AA?5?$AAS?$AAW?$AAI?$AA_?$AAN?$AAO?$AAT?$AAI?$AAF?$AAY?$AA_?$AAE?$AAc?$AAi?$AAo?$AA?5?$AAw?$AAh?$AAi?$AAl?$AAe?$AA?5?$AAm@ 00159438     Radio.obj
 0002:000184a8       ??_C@_1KA@IOJCIABB@?$AAR?$AAe?$AAc?$AAe?$AAi?$AAv?$AAe?$AA?5?$AAS?$AAW?$AAI?$AA_?$AAN?$AAO?$AAT?$AAI?$AAF?$AAY?$AA_?$AAA?$AAi?$AAr?$AAS?$AAe?$AAr?$AAv?$AAe?$AAr?$AAC?$AAh?$AAa?$AAn@ 001594a8     Radio.obj
 0002:00018548       ??_C@_1IM@CJHAKONO@?$AAI?$AAg?$AAn?$AAo?$AAr?$AAe?$AA?5?$AAM?$AAo?$AAd?$AAe?$AAm?$AA?5?$AA_?$AAH?$AAW?$AAP?$AAo?$AAw?$AAe?$AAr?$AA?4?$AAS?$AAt?$AAa?$AAt?$AAe?$AA?5?$AA?$CI?$AAS?$AAW?$AAI@ 00159548     Radio.obj
 0002:000185d8       ??_C@_1LO@KBHHCCCI@?$AAM?$AAo?$AAd?$AAe?$AAm?$AA?5?$AA_?$AAH?$AAW?$AAP?$AAo?$AAw?$AAe?$AAr?$AA?4?$AAS?$AAt?$AAa?$AAt?$AAe?$AA?5?$AAc?$AAh?$AAa?$AAn?$AAg?$AAe?$AA?5?$AAt?$AAo?$AA?5?$AA?$CF@ 001595d8     Radio.obj
 0002:00018698       ??_C@_1JA@OEDNNHJL@?$AAR?$AAe?$AAc?$AAe?$AAi?$AAv?$AAe?$AAd?$AA?5?$AAS?$AAW?$AAI?$AA_?$AAT?$AAY?$AAP?$AAE?$AA_?$AAP?$AAo?$AAw?$AAe?$AAr?$AAR?$AAe?$AAs?$AAe?$AAt?$AA?4?$AA?5?$AAE?$AAx@ 00159698     Radio.obj
 0002:00018728       ??_C@_1DG@BMLECOJI@?$AAU?$AAn?$AAh?$AAa?$AAn?$AAd?$AAl?$AAe?$AAd?$AA?5?$AAP?$AAo?$AAw?$AAe?$AAr?$AA?5?$AAN?$AAo?$AAt?$AAi?$AAf?$AA?5?$AA?$DN?$AA?5?$AA?$CF?$AAd?$AA?$AA@ 00159728     Radio.obj
 0002:00018760       ??_C@_1MM@KPDIMMHE@?$AAM?$AAo?$AAd?$AAe?$AAm?$AA?5?$AA_?$AAP?$AAo?$AAw?$AAe?$AAr?$AA?4?$AAS?$AAt?$AAa?$AAt?$AAe?$AA?5?$AAc?$AAh?$AAa?$AAn?$AAg?$AAe?$AA?5?$AAt?$AAo?$AA?5?$AA?$CF?$AAd?$AA?5@ 00159760     Radio.obj
 0002:00018830       ??_C@_1GA@KMLHOBMG@?$AAI?$AAg?$AAn?$AAo?$AAr?$AAi?$AAn?$AAg?$AA?5?$AAS?$AAW?$AAI?$AA_?$AAN?$AAO?$AAT?$AAI?$AAF?$AAY?$AA_?$AAR?$AAs?$AAs?$AAi?$AA?5?$AAw?$AAh?$AAi?$AAl?$AAe?$AA?5?$AAt@ 00159830     Radio.obj
 0002:00018890       ??_C@_1HI@HJPIFCJL@?$AAI?$AAg?$AAn?$AAo?$AAr?$AAe?$AA?5?$AA?$CF?$AAd?$AA?5?$AA?$FL?$AAS?$AAW?$AAI?$AA_?$AAN?$AAO?$AAT?$AAI?$AAF?$AAY?$AA_?$AAR?$AAe?$AAs?$AAe?$AAt?$AA?5?$AA?$DN?$AA?5?$AA?$CF?$AAd@ 00159890     Radio.obj
 0002:00018908       ??_C@_1HG@LNDGGFFK@?$AAS?$AAW?$AAI?$AA_?$AAN?$AAO?$AAT?$AAI?$AAF?$AAY?$AA_?$AAR?$AAe?$AAs?$AAe?$AAt?$AA?5?$AAr?$AAe?$AAc?$AAe?$AAi?$AAv?$AAe?$AAd?$AA?$CB?$AA?5?$AAg?$AA_?$AAI?$AAs?$AAC@ 00159908     Radio.obj
 0002:00018980       ??_C@_1IG@INMMJPOA@?$AAF?$AAa?$AAi?$AAl?$AAe?$AAd?$AA?5?$AAt?$AAo?$AA?5?$AAc?$AAr?$AAe?$AAa?$AAt?$AAe?$AA?5?$AAt?$AAh?$AAr?$AAe?$AAa?$AAd?$AA?5?$AAf?$AAo?$AAr?$AA?5?$AAd?$AAe?$AAl?$AAa@ 00159980     Radio.obj
 0002:00018a08       ??_C@_1KO@KOBJPMHN@?$AAR?$AAe?$AAc?$AAe?$AAi?$AAv?$AAe?$AAd?$AA?5?$AAN?$AAI?$AAT?$AAZ?$AA?5?$AAf?$AAr?$AAo?$AAm?$AA?5?$AAt?$AAh?$AAe?$AA?5?$AAm?$AAo?$AAd?$AAe?$AAm?$AA?4?$AA?5?$AAB?$AAu@ 00159a08     Radio.obj
 0002:00018ab8       ??_C@_1EG@MNPGKKOG@?$AAC?$AAa?$AAl?$AAl?$AA?5?$AAS?$AAe?$AAt?$AAS?$AAy?$AAs?$AAt?$AAe?$AAm?$AAT?$AAi?$AAm?$AAe?$AA?5?$AAo?$AAn?$AA?5?$AAb?$AAe?$AAh?$AAa?$AAl?$AAf?$AA?5?$AAo?$AAf?$AA?5@ 00159ab8     Radio.obj
 0002:00018b88       ??_C@_1FA@MFEFKMCC@?$AAA?$AAS?$AAS?$AAE?$AAR?$AAT?$AAI?$AAO?$AAN?$AA?5?$AAF?$AAA?$AAI?$AAL?$AAU?$AAR?$AAE?$AA?3?$AA?5?$AA?$DN?$AA?$DN?$AA?$DN?$AA?$DO?$AAm?$AA_?$AAp?$AAc?$AAR?$AAi?$AAl?$AAh?$AA?5@ 00159b88     Radio.obj
 0002:00018bd8       ??_C@_1BO@CLDJMABK@?$AAP?$AAo?$AAl?$AAl?$AAi?$AAn?$AAg?$AAF?$AAo?$AAr?$AAR?$AAS?$AAS?$AAI?$AA?$AA@ 00159bd8     RadioCaps.obj
 0002:00018bf8       ??_C@_1FI@MOIBECKB@?$AAS?$AAi?$AAg?$AAn?$AAa?$AAl?$AAC?$AAr?$AAi?$AAt?$AAi?$AAc?$AAa?$AAl?$AAE?$AAr?$AAr?$AAo?$AAr?$AA?$CI?$AAR?$AAI?$AAL?$AAL?$AAO?$AAG?$AA_?$AAE?$AAV?$AAE?$AAN?$AAT@ 00159bf8     response.obj
 0002:00018c50       ??_C@_1EK@OKJBIBM@?$AAA?$AAS?$AAS?$AAE?$AAR?$AAT?$AAI?$AAO?$AAN?$AA?5?$AAF?$AAA?$AAI?$AAL?$AAU?$AAR?$AAE?$AA?3?$AA?5?$AA?$DN?$AA?$DN?$AA?$DN?$AA?$DO?$AAN?$AAU?$AAL?$AAL?$AA?5?$AA?$CB?$AA?$DN?$AA?5?$AAp@ 00159c50     response.obj
 0002:00018c9c       ??_C@_1BO@EKIIPBII@?$AA?4?$AA?2?$AAr?$AAe?$AAs?$AAp?$AAo?$AAn?$AAs?$AAe?$AA?4?$AAc?$AAp?$AAp?$AA?$AA@ 00159c9c     response.obj
 0002:00018cc0       ??_C@_1HA@FCAHIBNB@?$AAA?$AAS?$AAS?$AAE?$AAR?$AAT?$AAI?$AAO?$AAN?$AA?5?$AAF?$AAA?$AAI?$AAL?$AAU?$AAR?$AAE?$AA?3?$AA?5?$AA?$DN?$AA?$DN?$AA?$DN?$AA?$DO?$AAN?$AAU?$AAL?$AAL?$AA?5?$AA?$DN?$AA?$DN?$AA?5?$AAm@ 00159cc0     response.obj
 0002:00018d30       ??_C@_1EK@HFNFPGLO@?$AAA?$AAS?$AAS?$AAE?$AAR?$AAT?$AAI?$AAO?$AAN?$AA?5?$AAF?$AAA?$AAI?$AAL?$AAU?$AAR?$AAE?$AA?3?$AA?5?$AA?$DN?$AA?$DN?$AA?$DN?$AA?$DO?$AA0?$AA?5?$AA?$DN?$AA?$DN?$AA?5?$AAm?$AA_?$AAc?$AAb@ 00159d30     response.obj
 0002:00018d80       ??_C@_1EO@CMABEHNB@?$AAA?$AAS?$AAS?$AAE?$AAR?$AAT?$AAI?$AAO?$AAN?$AA?5?$AAF?$AAA?$AAI?$AAL?$AAU?$AAR?$AAE?$AA?3?$AA?5?$AA?$DN?$AA?$DN?$AA?$DN?$AA?$DO?$AAN?$AAU?$AAL?$AAL?$AA?5?$AA?$DN?$AA?$DN?$AA?5?$AAm@ 00159d80     response.obj
 0002:00018dd0       ??_C@_1EA@PLHLMFLC@?$AAS?$AAo?$AAf?$AAt?$AAw?$AAa?$AAr?$AAe?$AA?2?$AAM?$AAi?$AAc?$AAr?$AAo?$AAs?$AAo?$AAf?$AAt?$AA?2?$AAR?$AAI?$AAL?$AA?2?$AAA?$AAP?$AAI?$AAI?$AAn?$AAf?$AAo?$AA?2?$AA?$AA@ 00159dd0     rilhand.obj
 0002:00018e10       ?g_tszRegKeyRIL@@3QBGB     00159e10     rilhand.obj
 0002:00018e14       ?g_tszRegKeyAPIInfo@@3QBGB 00159e14     rilhand.obj
 0002:00018e18       ??_7CEvent@@6B@            00159e18     rilhand.obj
 0002:00018e1c       ??_7CUniquelyNamedEvent@@6B@ 00159e1c     rilhand.obj
 0002:00018e20       ??_C@_19GODENFJI@?$AA?$CF?$AAs?$AA?$CF?$AAx?$AA?$AA@ 00159e20     rilhand.obj
 0002:00018e2c       ??_7Event@@6B@             00159e2c     rilhand.obj
 0002:00018e8c       ??_C@_1BM@FKIIANBE@?$AA?4?$AA?2?$AAr?$AAi?$AAl?$AAh?$AAa?$AAn?$AAd?$AA?4?$AAc?$AAp?$AAp?$AA?$AA@ 00159e8c     rilhand.obj
 0002:00018ea8       ??_C@_1GC@GEGPJNLF@?$AAA?$AAS?$AAS?$AAE?$AAR?$AAT?$AAI?$AAO?$AAN?$AA?5?$AAF?$AAA?$AAI?$AAL?$AAU?$AAR?$AAE?$AA?3?$AA?5?$AA?$DN?$AA?$DN?$AA?$DN?$AA?$DO?$AAg?$AA_?$AAG?$AAl?$AAo?$AAb?$AAa?$AAl?$AAR@ 00159ea8     rilhand.obj
 0002:00018f98       ??_C@_1JO@IHNLPMIO@?$AAC?$AAR?$AAi?$AAl?$AAH?$AAa?$AAn?$AAd?$AAl?$AAe?$AA?3?$AA?3?$AAG?$AAe?$AAt?$AAA?$AAP?$AAI?$AAI?$AAn?$AAf?$AAo?$AA?5?$AA?3?$AA?5?$AAI?$AAn?$AAf?$AAo?$AA?5?$AAf?$AAo@ 00159f98     rilhand.obj
 0002:00019038       ??_C@_1GG@IOGECMLN@?$AAA?$AAS?$AAS?$AAE?$AAR?$AAT?$AAI?$AAO?$AAN?$AA?5?$AAF?$AAA?$AAI?$AAL?$AAU?$AAR?$AAE?$AA?3?$AA?5?$AA?$DN?$AA?$DN?$AA?$DN?$AA?$DO?$AAN?$AAU?$AAL?$AAL?$AA?5?$AA?$CB?$AA?$DN?$AA?5?$AAm@ 0015a038     rilhand.obj
 0002:000190a0       ??_C@_1BA@BKONPLFM@?$AAT?$AAi?$AAm?$AAe?$AAo?$AAu?$AAt?$AA?$AA@ 0015a0a0     rilhand.obj
 0002:000190b0       ??_C@_1BM@PEDHMNHE@?$AAE?$AAx?$AAe?$AAc?$AAu?$AAt?$AAi?$AAo?$AAn?$AAT?$AAi?$AAm?$AAe?$AA?$AA@ 0015a0b0     rilhand.obj
 0002:000190cc       ??_C@_1CK@DKJPDPOJ@?$AAI?$AAn?$AAc?$AAo?$AAr?$AAr?$AAe?$AAc?$AAt?$AA?5?$AAA?$AAP?$AAI?$AAI?$AAD?$AA?5?$AA?$DN?$AA?5?$AA?$CF?$AAd?$AA?$AA@ 0015a0cc     rilhand.obj
 0002:000190f8       ??_C@_1EK@KAOPPKEF@?$AAA?$AAS?$AAS?$AAE?$AAR?$AAT?$AAI?$AAO?$AAN?$AA?5?$AAF?$AAA?$AAI?$AAL?$AAU?$AAR?$AAE?$AA?3?$AA?5?$AA?$DN?$AA?$DN?$AA?$DN?$AA?$DO?$AAN?$AAU?$AAL?$AAL?$AA?5?$AA?$CB?$AA?$DN?$AA?5?$AAp@ 0015a0f8     rilhand.obj
 0002:00019144       ??_C@_1O@JJGPBMPP@?$AA?$CF?$AA0?$AA2?$AAX?$AA?$AA?$AA?$AA?$AA?$AA@ 0015a144     rilhand.obj
 0002:00019154       ??_C@_1DM@NJAKJLNC@?$AAQ?$AAM?$AAI?$AA?5?$AAG?$AAe?$AAt?$AAW?$AAa?$AAi?$AAt?$AAi?$AAn?$AAg?$AAM?$AAe?$AAs?$AAs?$AAa?$AAg?$AAe?$AA?5?$AAf?$AAa?$AAi?$AAl?$AAe?$AAd?$AA?$CB?$AA?$AA@ 0015a154     rilhand.obj
 0002:00019190       ??_C@_1FO@HIDNNNIM@?$AAC?$AAl?$AAo?$AAs?$AAe?$AAS?$AAW?$AAI?$AA?5?$AAN?$AAO?$AAO?$AAP?$AA?5?$AAs?$AAi?$AAn?$AAc?$AAe?$AA?5?$AAD?$AAe?$AAI?$AAn?$AAi?$AAt?$AAi?$AAa?$AAl?$AAi?$AAz?$AAe@ 0015a190     rilhand.obj
 0002:000191f0       ??_C@_1FE@CHLOFECA@?$AAR?$AAi?$AAl?$AAD?$AAr?$AAv?$AA?3?$AA?5?$AAU?$AAn?$AAa?$AAt?$AAt?$AAe?$AAn?$AAd?$AAe?$AAd?$AA?9?$AAM?$AAo?$AAd?$AAe?$AA?5?$AAr?$AAe?$AAq?$AAu?$AAe?$AAs?$AAt?$AA?5@ 0015a1f0     rilhand.obj
 0002:00019248       ??_C@_1HE@NELMMJFF@?$AAR?$AAi?$AAl?$AAD?$AAr?$AAv?$AA?3?$AA?5?$AAU?$AAn?$AAa?$AAt?$AAt?$AAe?$AAn?$AAd?$AAe?$AAd?$AA?9?$AAM?$AAo?$AAd?$AAe?$AA?5?$AAr?$AAe?$AAm?$AAo?$AAv?$AAe?$AA?9?$AAr@ 0015a248     rilhand.obj
 0002:000192c0       ??_C@_1FA@HBHGOHHG@?$AAR?$AAi?$AAl?$AAD?$AAr?$AAv?$AA?3?$AA?5?$AAU?$AAn?$AAa?$AAt?$AAt?$AAe?$AAn?$AAd?$AAe?$AAd?$AA?9?$AAM?$AAo?$AAd?$AAe?$AA?5?$AAr?$AAe?$AAq?$AAu?$AAe?$AAs?$AAt?$AA?5@ 0015a2c0     rilhand.obj
 0002:00019310       ??_C@_1GO@MIDLHICK@?$AAR?$AAi?$AAl?$AAD?$AAr?$AAv?$AA?3?$AA?5?$AAU?$AAn?$AAa?$AAt?$AAt?$AAe?$AAn?$AAd?$AAe?$AAd?$AA?9?$AAM?$AAo?$AAd?$AAe?$AA?5?$AAa?$AAd?$AAd?$AA?9?$AAr?$AAe?$AAq?$AAu@ 0015a310     rilhand.obj
 0002:000193b4       ??_7?$CUnboundedQueue@Urildrvnotification_tag@@@@6B@ 0015a3b4     rilhand.obj
 0002:000193ec       ??_C@_1CC@CMJCLKEP@?$AAC?$AAU?$AAn?$AAb?$AAo?$AAu?$AAn?$AAd?$AAe?$AAd?$AAQ?$AAu?$AAe?$AAu?$AAe?$AA_?$AA?$AA@ 0015a3ec     rilhand.obj
 0002:00019458       ??_C@_1EM@IBKBEHJ@?$AAA?$AAS?$AAS?$AAE?$AAR?$AAT?$AAI?$AAO?$AAN?$AA?5?$AAF?$AAA?$AAI?$AAL?$AAU?$AAR?$AAE?$AA?3?$AA?5?$AA?$DN?$AA?$DN?$AA?$DN?$AA?$DO?$AAd?$AAw?$AAD?$AAa?$AAt?$AAa?$AA?5?$AA?$CB?$AA?$DN@ 0015a458     rilhand.obj
 0002:000194a8       ??_C@_1EK@KFHONFA@?$AAA?$AAS?$AAS?$AAE?$AAR?$AAT?$AAI?$AAO?$AAN?$AA?5?$AAF?$AAA?$AAI?$AAL?$AAU?$AAR?$AAE?$AA?3?$AA?5?$AA?$DN?$AA?$DN?$AA?$DN?$AA?$DO?$AAp?$AAI?$AAt?$AAe?$AAm?$AA?5?$AA?$CB?$AA?$DN?$AA?5@ 0015a4a8     rilhand.obj
 0002:000194f8       ??_C@_1EI@FDJCMHMO@?$AAA?$AAS?$AAS?$AAE?$AAR?$AAT?$AAI?$AAO?$AAN?$AA?5?$AAF?$AAA?$AAI?$AAL?$AAU?$AAR?$AAE?$AA?3?$AA?5?$AA?$DN?$AA?$DN?$AA?$DN?$AA?$DO?$AAT?$AAR?$AAU?$AAE?$AA?5?$AA?$DN?$AA?$DN?$AA?5?$AAf@ 0015a4f8     rilhand.obj
 0002:00019540       ??_C@_1FO@CGHJMELG@?$AAU?$AAn?$AAe?$AAx?$AAp?$AAe?$AAc?$AAt?$AAe?$AAd?$AA?5?$AAw?$AAa?$AAi?$AAt?$AAe?$AAd?$AAO?$AAb?$AAj?$AA?5?$AA?$DN?$AA?5?$AA?$CF?$AAd?$AA?0?$AA?5?$AAG?$AAe?$AAt?$AAL?$AAa@ 0015a540     rilhand.obj
 0002:000195a0       ??_C@_1DA@JKLAGHBF@?$AAg?$AA_?$AAp?$AAC?$AAm?$AAd?$AAQ?$AA?5?$AAg?$AAo?$AAt?$AA?5?$AAa?$AAl?$AAe?$AAr?$AAt?$AA?5?$AAe?$AAv?$AAe?$AAn?$AAt?$AA?$AA@ 0015a5a0     rilhand.obj
 0002:000195d0       ??_C@_1GM@POOCIBKG@?$AAM?$AAe?$AAm?$AAo?$AAr?$AAy?$AA?5?$AAc?$AAo?$AAn?$AAt?$AAe?$AAn?$AAt?$AA?5?$AAo?$AAf?$AA?5?$AAt?$AAh?$AAe?$AA?5?$AAG?$AAe?$AAt?$AAN?$AAe?$AAx?$AAt?$AAN?$AAo?$AAt@ 0015a5d0     rilhand.obj
 0002:00019640       ??_C@_1BEA@IPHGGPKF@?$AAN?$AAo?$AAt?$AAi?$AAf?$AAi?$AAc?$AAa?$AAt?$AAi?$AAo?$AAn?$AA?5?$AAs?$AAi?$AAz?$AAe?$AA?5?$AAi?$AAn?$AAv?$AAa?$AAl?$AAi?$AAd?$AA?0?$AA?5?$AAn?$AAe?$AAx?$AAt?$AA?5@ 0015a640     rilhand.obj
 0002:00019780       ??_C@_1GI@FMBIKGJP@?$AAA?$AAS?$AAS?$AAE?$AAR?$AAT?$AAI?$AAO?$AAN?$AA?5?$AAF?$AAA?$AAI?$AAL?$AAU?$AAR?$AAE?$AA?3?$AA?5?$AA?$DN?$AA?$DN?$AA?$DN?$AA?$DO?$AAN?$AAU?$AAL?$AAL?$AA?5?$AA?$CB?$AA?$DN?$AA?5?$AAp@ 0015a780     rilhand.obj
 0002:000197e8       ??_C@_1EK@GEMHABFC@?$AAA?$AAS?$AAS?$AAE?$AAR?$AAT?$AAI?$AAO?$AAN?$AA?5?$AAF?$AAA?$AAI?$AAL?$AAU?$AAR?$AAE?$AA?3?$AA?5?$AA?$DN?$AA?$DN?$AA?$DN?$AA?$DO?$AAS?$AAU?$AAC?$AAC?$AAE?$AAE?$AAD?$AAE?$AAD@ 0015a7e8     rilhand.obj
 0002:00019838       ??_C@_1HM@EFMNHPFO@?$AAA?$AAS?$AAS?$AAE?$AAR?$AAT?$AAI?$AAO?$AAN?$AA?5?$AAF?$AAA?$AAI?$AAL?$AAU?$AAR?$AAE?$AA?3?$AA?5?$AA?$DN?$AA?$DN?$AA?$DN?$AA?$DO?$AAE?$AAR?$AAR?$AAO?$AAR?$AA_?$AAA?$AAL?$AAR@ 0015a838     rilhand.obj
 0002:000198b4       ??_C@_1CG@PEHJEDAN@?$AAM?$AAo?$AAd?$AAe?$AAm?$AA?5?$AAi?$AAs?$AA?5?$AAr?$AAe?$AAs?$AAe?$AAt?$AAt?$AAi?$AAn?$AAg?$AA?$AA@ 0015a8b4     rilhand.obj
 0002:000198dc       ??_C@_1CI@ELPIMIJB@?$AAD?$AAe?$AAI?$AAn?$AAi?$AAt?$AAi?$AAa?$AAl?$AAi?$AAz?$AAe?$AAS?$AAW?$AAI?$AA?5?$AA?4?$AA?4?$AA?4?$AA?$AA@ 0015a8dc     rilhand.obj
 0002:00019908       ??_C@_1IE@MELJCIBL@?$AAA?$AAl?$AAr?$AAe?$AAa?$AAd?$AAy?$AA?5?$AAh?$AAa?$AAd?$AA?5?$AAa?$AAn?$AA?5?$AAD?$AAe?$AAI?$AAn?$AAi?$AAt?$AAi?$AAa?$AAl?$AAi?$AAz?$AAe?$AAS?$AAw?$AAi?$AA?5?$AAr@ 0015a908     rilhand.obj
 0002:000199c0       ??_C@_1JM@BIMOLACM@?$AAC?$AAR?$AAi?$AAl?$AAI?$AAn?$AAs?$AAt?$AAa?$AAn?$AAc?$AAe?$AAH?$AAa?$AAn?$AAd?$AAl?$AAe?$AA?3?$AA?3?$AAN?$AAo?$AAt?$AAi?$AAf?$AAy?$AA?5?$AA?3?$AA?5?$AAD?$AAr?$AAo@ 0015a9c0     rilhand.obj
 0002:00019b18       ??_C@_1PE@BODAAKMI@?$AAg?$AA_?$AAa?$AAr?$AAr?$AAW?$AAa?$AAi?$AAt?$AAi?$AAn?$AAg?$AAC?$AAo?$AAm?$AAm?$AAa?$AAn?$AAd?$AAs?$AA?5?$AAj?$AAu?$AAs?$AAt?$AA?5?$AAr?$AAe?$AAm?$AAo?$AAv?$AAe@ 0015ab18     rilhand.obj
 0002:00019c0c       ??_C@_1DM@CNCCEAJF@?$AAA?$AAP?$AAI?$AAI?$AAD?$AA_?$AAG?$AAE?$AAT?$AAO?$AAP?$AAE?$AAR?$AAA?$AAT?$AAO?$AAR?$AAL?$AAI?$AAS?$AAT?$AA?5?$AAt?$AAi?$AAm?$AAe?$AAo?$AAu?$AAt?$AA?$AA@ 0015ac0c     rilhand.obj
 0002:00019c48       ??_C@_1CM@LACLALCA@?$AAA?$AAP?$AAI?$AAI?$AAD?$AA_?$AAH?$AAA?$AAN?$AAG?$AAU?$AAP?$AA?5?$AAt?$AAi?$AAm?$AAe?$AAo?$AAu?$AAt?$AA?4?$AA?$AA@ 0015ac48     rilhand.obj
 0002:00019c74       ??_C@_1CO@BMGGEOMG@?$AAA?$AAP?$AAI?$AAI?$AAD?$AA_?$AAS?$AAE?$AAN?$AAD?$AAM?$AAS?$AAG?$AA?5?$AAt?$AAi?$AAm?$AAe?$AAo?$AAu?$AAt?$AA?4?$AA?$AA@ 0015ac74     rilhand.obj
 0002:00019ca4       ??_C@_1DK@LPMMDHGL@?$AAU?$AAn?$AAk?$AAn?$AAo?$AAw?$AAn?$AA?5?$AAc?$AAo?$AAm?$AAm?$AAa?$AAn?$AAd?$AA?$CI?$AA?$CF?$AAd?$AA?$CJ?$AA?5?$AAt?$AAi?$AAm?$AAe?$AAo?$AAu?$AAt?$AA?4?$AA?$AA@ 0015aca4     rilhand.obj
 0002:00019ce0       ??_C@_1FI@PBACLHHF@?$AAD?$AAa?$AAt?$AAa?$AA?5?$AAd?$AAi?$AAa?$AAl?$AA?5?$AAm?$AAi?$AAg?$AAh?$AAt?$AA?5?$AAb?$AAe?$AA?5?$AAs?$AAt?$AAu?$AAc?$AAk?$AA?4?$AA?5?$AAT?$AAr?$AAy?$AA?5?$AAC?$AAl@ 0015ace0     rilhand.obj
 0002:00019d38       ??_C@_1CK@BBNEJOGK@?$AAD?$AAi?$AAa?$AAl?$AA?5?$AAc?$AAo?$AAm?$AAm?$AAa?$AAn?$AAd?$AA?5?$AAt?$AAi?$AAm?$AAe?$AAo?$AAu?$AAt?$AA?$AA@ 0015ad38     rilhand.obj
 0002:00019d64       ??_C@_1CG@NEMBKIBF@?$AAA?$AAP?$AAI?$AAI?$AAD?$AA?5?$AA?$DN?$AA?5?$AA?$CF?$AAd?$AA?5?$AAt?$AAi?$AAm?$AAe?$AAo?$AAu?$AAt?$AA?$AA@ 0015ad64     rilhand.obj
 0002:00019d90       ??_C@_1GI@LDGHPBON@?$AAD?$AAe?$AAl?$AAe?$AAt?$AAe?$AA?5?$AAc?$AAo?$AAm?$AAm?$AAa?$AAn?$AAd?$AA?5?$AAA?$AAP?$AAI?$AAI?$AAD?$AA?5?$AA?$DN?$AA?5?$AA?$CF?$AAd?$AA?5?$AAf?$AAr?$AAo?$AAm?$AA?5?$AAg@ 0015ad90     rilhand.obj
 0002:00019df8       ??_C@_1GO@MJJNBDMN@?$AAR?$AAi?$AAl?$AA?5?$AAw?$AAi?$AAl?$AAl?$AA?5?$AAS?$AAe?$AAn?$AAd?$AAR?$AAe?$AAs?$AAp?$AAo?$AAn?$AAs?$AAe?$AA?5?$AAR?$AAI?$AAL?$AA_?$AAR?$AAE?$AAS?$AAU?$AAL?$AAT@ 0015adf8     rilhand.obj
 0002:00019e68       ??_C@_1DA@POMFHEIG@?$AAC?$AAh?$AAe?$AAc?$AAk?$AAT?$AAi?$AAm?$AAe?$AAO?$AAu?$AAt?$AA?5?$AAA?$AAP?$AAI?$AAI?$AAD?$AA?5?$AA?$DN?$AA?5?$AA?$CF?$AAd?$AA?$AA@ 0015ae68     rilhand.obj
 0002:00019e98       ??_C@_1JM@HPJOOKOC@?$AAE?$AAR?$AAR?$AAO?$AAR?$AA?$CB?$AA?$CB?$AA?$CB?$AA?5?$AAp?$AAR?$AAI?$AAL?$AAG?$AAE?$AAN?$AAE?$AAR?$AAI?$AAC?$AAN?$AAO?$AAT?$AAI?$AAF?$AAI?$AAC?$AAA?$AAT?$AAI?$AAO?$AAN@ 0015ae98     rilhand.obj
 0002:00019f38       ??_C@_1HO@JMFKFENC@?$AAS?$AAe?$AAn?$AAd?$AAR?$AAe?$AAs?$AAp?$AAo?$AAn?$AAs?$AAe?$AA?$CI?$AAR?$AAI?$AAL?$AA_?$AAR?$AAE?$AAS?$AAU?$AAL?$AAT?$AA_?$AAE?$AAR?$AAR?$AAO?$AAR?$AA?$CJ?$AA?0?$AA?5@ 0015af38     rilhand.obj
 0002:00019fb8       ??_C@_1JO@MAIIINFK@?$AAS?$AAe?$AAn?$AAd?$AAR?$AAe?$AAs?$AAp?$AAo?$AAn?$AAs?$AAe?$AA?$CI?$AAR?$AAI?$AAL?$AA_?$AAR?$AAE?$AAS?$AAU?$AAL?$AAT?$AA_?$AAE?$AAR?$AAR?$AAO?$AAR?$AA?$CJ?$AA?0?$AA?5@ 0015afb8     rilhand.obj
 0002:0001a058       ??_C@_1GM@HHBEEBBF@?$AAS?$AAe?$AAn?$AAd?$AAR?$AAe?$AAs?$AAp?$AAo?$AAn?$AAs?$AAe?$AA?$CI?$AAR?$AAI?$AAL?$AA_?$AAR?$AAE?$AAS?$AAU?$AAL?$AAT?$AA_?$AAO?$AAK?$AA?$CJ?$AA?0?$AA?5?$AAm?$AAs?$AAg@ 0015b058     rilhand.obj
 0002:0001a0c8       ??_C@_1PO@LFHAKMGP@?$AAP?$AAr?$AAe?$AAB?$AAr?$AAo?$AAa?$AAd?$AAc?$AAa?$AAs?$AAt?$AA?5?$AAn?$AAo?$AAt?$AAi?$AAf?$AA?5?$AAC?$AAo?$AAd?$AAe?$AA?5?$AA?$DN?$AA?5?$AA0?$AAx?$AA?$CF?$AAx?$AA?0?$AA?5@ 0015b0c8     rilhand.obj
 0002:0001a200       ??_C@_1JE@KKIAIKNK@?$AAC?$AAa?$AAn?$AAn?$AAo?$AAt?$AA?5?$AAa?$AAf?$AAf?$AAo?$AAr?$AAd?$AA?5?$AAt?$AAo?$AA?5?$AAr?$AAe?$AAm?$AAo?$AAv?$AAe?$AA?5?$AAA?$AAP?$AAI?$AAI?$AAD?$AA?5?$AA?$DN?$AA?5@ 0015b200     rilhand.obj
 0002:0001a298       ??_C@_1HE@PDHMMLAI@?$AAC?$AAh?$AAe?$AAc?$AAk?$AAD?$AAe?$AAl?$AAa?$AAy?$AAe?$AAd?$AAR?$AAs?$AAp?$AAC?$AAm?$AAd?$AAT?$AAi?$AAm?$AAe?$AAo?$AAu?$AAt?$AA?5?$AAm?$AAu?$AAs?$AAt?$AA?5?$AAs@ 0015b298     rilhand.obj
 0002:0001a310       ??_C@_1OG@IKJPNOEI@?$AAC?$AAh?$AAe?$AAc?$AAk?$AAD?$AAe?$AAl?$AAa?$AAy?$AAe?$AAd?$AAR?$AAs?$AAp?$AAC?$AAm?$AAd?$AAT?$AAi?$AAm?$AAe?$AAo?$AAu?$AAt?$AA?5?$AA?$CI?$AAc?$AAm?$AAd?$AAI?$AAD@ 0015b310     rilhand.obj
 0002:0001a3f8       ??_C@_1FO@HCFBALNL@?$AAC?$AAh?$AAe?$AAc?$AAk?$AAD?$AAe?$AAl?$AAa?$AAy?$AAe?$AAd?$AAR?$AAs?$AAp?$AAC?$AAm?$AAd?$AAT?$AAi?$AAm?$AAe?$AAo?$AAu?$AAt?$AA?3?$AA?5?$AAA?$AAP?$AAI?$AAI?$AAD@ 0015b3f8     rilhand.obj
 0002:0001a458       ??_C@_1IG@KHAGBDGK@?$AAC?$AAR?$AAi?$AAl?$AAH?$AAa?$AAn?$AAd?$AAl?$AAe?$AA?3?$AA?3?$AAB?$AAr?$AAo?$AAa?$AAd?$AAc?$AAa?$AAs?$AAt?$AAN?$AAo?$AAt?$AAi?$AAf?$AAi?$AAc?$AAa?$AAt?$AAi?$AAo@ 0015b458     rilhand.obj
 0002:0001a4e0       ??_C@_1EI@JJFGCGNE@?$AAA?$AAS?$AAS?$AAE?$AAR?$AAT?$AAI?$AAO?$AAN?$AA?5?$AAF?$AAA?$AAI?$AAL?$AAU?$AAR?$AAE?$AA?3?$AA?5?$AA?$DN?$AA?$DN?$AA?$DN?$AA?$DO?$AAN?$AAU?$AAL?$AAL?$AA?5?$AA?$CB?$AA?$DN?$AA?5?$AAr@ 0015b4e0     rilhand.obj
 0002:0001a568       ??_C@_1OA@DGABLGHP@?$AAI?$AAn?$AAv?$AAa?$AAl?$AAi?$AAd?$AA?5?$AAs?$AAi?$AAz?$AAe?$AA?5?$AAf?$AAo?$AAr?$AA?5?$AAR?$AAI?$AAL?$AA_?$AAN?$AAO?$AAT?$AAI?$AAF?$AAY?$AA_?$AAR?$AAA?$AAD?$AAI@ 0015b568     rilhand.obj
 0002:0001a648       ??_C@_1BDC@OAAGENID@?$AAR?$AAI?$AAL?$AA?5?$AAj?$AAu?$AAs?$AAt?$AA?5?$AAn?$AAo?$AAt?$AAi?$AAf?$AAi?$AAe?$AAs?$AA?5?$AAE?$AAQ?$AAU?$AAI?$AAP?$AAM?$AAE?$AAN?$AAT?$AAS?$AAT?$AAA?$AAT?$AAE@ 0015b648     rilhand.obj
 0002:0001a7b8       ??_C@_1GO@CFPKPHKD@?$AAC?$AAR?$AAi?$AAl?$AAH?$AAa?$AAn?$AAd?$AAl?$AAe?$AA?3?$AA?3?$AAF?$AAi?$AAn?$AAi?$AAs?$AAh?$AAI?$AAn?$AAi?$AAt?$AA?5?$AA?3?$AA?5?$AAM?$AAo?$AAd?$AAu?$AAl?$AAe?$AA?5@ 0015b7b8     rilhand.obj
 0002:0001a828       ??_C@_1HE@JNFMNMKE@?$AAC?$AAR?$AAi?$AAl?$AAH?$AAa?$AAn?$AAd?$AAl?$AAe?$AA?3?$AA?3?$AAF?$AAi?$AAn?$AAi?$AAs?$AAh?$AAI?$AAn?$AAi?$AAt?$AA?5?$AA?3?$AA?5?$AAM?$AAo?$AAd?$AAu?$AAl?$AAe?$AA?5@ 0015b828     rilhand.obj
 0002:0001a8a0       ??_C@_1FO@CADPEKDJ@?$AAN?$AAO?$AAO?$AAP?$AA?5?$AAs?$AAi?$AAn?$AAc?$AAe?$AA?5?$AAS?$AAW?$AAI?$AA?5?$AAi?$AAs?$AA?5?$AAc?$AAl?$AAo?$AAs?$AAe?$AAd?$AA?0?$AA?5?$AAe?$AAq?$AAS?$AAt?$AAa?$AAt@ 0015b8a0     rilhand.obj
 0002:0001a900       ??_C@_1KG@DBIFGCNP@?$AAF?$AAa?$AAi?$AAl?$AAe?$AAd?$AA?5?$AAt?$AAo?$AA?5?$AAg?$AAe?$AAt?$AA?5?$AAt?$AAh?$AAe?$AA?5?$AAL?$AAo?$AAc?$AAk?$AAe?$AAd?$AA?5?$AAS?$AAt?$AAa?$AAt?$AAe?$AA?5?$AAf@ 0015b900     rilhand.obj
 0002:0001a9a8       ??_C@_1FC@GNBAADJ@?$AAE?$AAR?$AAR?$AAO?$AAR?$AA?$CB?$AA?$CB?$AA?$CB?$AA?5?$AAm?$AAp?$AAF?$AAn?$AAS?$AAw?$AAi?$AAG?$AAe?$AAt?$AAS?$AAi?$AAm?$AAV?$AAe?$AAr?$AAi?$AAf?$AAy?$AAG?$AAo?$AAb?$AAi@ 0015b9a8     rilhand.obj
 0002:0001aa00       ??_C@_1KM@JEPOFMIP@?$AAI?$AAn?$AAi?$AAt?$AAi?$AAa?$AAl?$AAi?$AAz?$AAe?$AAS?$AAW?$AAI?$AA?3?$AA?5?$AAm?$AAp?$AAF?$AAn?$AAS?$AAw?$AAi?$AAG?$AAe?$AAt?$AAS?$AAi?$AAm?$AAV?$AAe?$AAr?$AAi@ 0015ba00     rilhand.obj
 0002:0001aaac       ??_C@_1DE@HAGGGFFF@?$AAI?$AAn?$AAi?$AAt?$AAi?$AAa?$AAl?$AAi?$AAz?$AAe?$AAS?$AAW?$AAI?$AA?5?$AAr?$AAe?$AAs?$AAu?$AAl?$AAt?$AA?5?$AA?$DN?$AA?5?$AA?$CF?$AAd?$AA?$AA@ 0015baac     rilhand.obj
 0002:0001aae0       ??_C@_1DO@JGBCHAMG@?$AAF?$AAa?$AAi?$AAl?$AA?5?$AAt?$AAo?$AA?5?$AAg?$AAe?$AAt?$AA?5?$AAC?$AAa?$AAr?$AAr?$AAi?$AAe?$AAr?$AAI?$AAD?$AA?0?$AA?5?$AAr?$AAc?$AA?5?$AA?$DN?$AA?5?$AA?$CF?$AAd?$AA?$AA@ 0015bae0     rilhand.obj
 0002:0001ab20       ??_C@_1II@PDBCNMPI@?$AAF?$AAa?$AAi?$AAl?$AAe?$AAd?$AA?5?$AAt?$AAo?$AA?5?$AAo?$AAp?$AAe?$AAn?$AA?5?$AAS?$AAo?$AAf?$AAt?$AAw?$AAa?$AAr?$AAe?$AA?2?$AAS?$AAi?$AAe?$AAr?$AAr?$AAa?$AAW?$AAi@ 0015bb20     rilhand.obj
 0002:0001aba8       ??_C@_1BK@GIONEDDC@?$AAC?$AAa?$AAr?$AAr?$AAi?$AAe?$AAr?$AAI?$AAn?$AAd?$AAe?$AAx?$AA?$AA@ 0015bba8     rilhand.obj
 0002:0001abc8       ??_C@_1EC@GEHDNBGM@?$AAS?$AAo?$AAf?$AAt?$AAw?$AAa?$AAr?$AAe?$AA?2?$AAS?$AAi?$AAe?$AAr?$AAr?$AAa?$AA?5?$AAW?$AAi?$AAr?$AAe?$AAl?$AAe?$AAs?$AAs?$AA?5?$AAI?$AAn?$AAc?$AA?2?$AAQ?$AAD?$AAL@ 0015bbc8     rilhand.obj
 0002:0001ac0c       ??_C@_1DA@ENICLKHI@?$AAC?$AAa?$AAr?$AAr?$AAi?$AAe?$AAr?$AAI?$AAD?$AA?5?$AA?$DN?$AA?5?$AA?$CF?$AAu?$AA?0?$AA?5?$AAr?$AAc?$AA?5?$AA?$DN?$AA?5?$AA?$CF?$AAd?$AA?$AA@ 0015bc0c     rilhand.obj
 0002:0001ac40       ??_C@_1KG@LALBCDMB@?$AAT?$AAh?$AAi?$AAs?$AA?5?$AAi?$AAs?$AA?5?$AAa?$AA?5?$AAU?$AAN?$AAK?$AAN?$AAO?$AAW?$AAN?$AA?5?$AAt?$AAe?$AAc?$AAh?$AAn?$AAo?$AAl?$AAo?$AAg?$AAy?$AA?5?$AA?$DN?$AA?5?$AA?$CF@ 0015bc40     rilhand.obj
 0002:0001ace8       ??_C@_1GI@NBOOKMLN@?$AAS?$AAw?$AAi?$AAS?$AAe?$AAt?$AAH?$AAo?$AAs?$AAt?$AAS?$AAt?$AAa?$AAr?$AAt?$AAu?$AAp?$AA?5?$AAf?$AAa?$AAi?$AAl?$AAs?$AA?5?$AAt?$AAh?$AAr?$AAe?$AAe?$AA?5?$AAt?$AAi@ 0015bce8     rilhand.obj
 0002:0001ad50       ??_C@_1HC@POEJAHBC@?$AAO?$AAo?$AAp?$AAs?$AA?5?$AAG?$AAS?$AAM?$AA?5?$AAm?$AAo?$AAd?$AAe?$AAm?$AA?5?$AAn?$AAo?$AAt?$AA?5?$AAr?$AAe?$AAa?$AAd?$AAy?$AA?$CB?$AA?0?$AA?5?$AAr?$AAc?$AAP?$AAo?$AAw@ 0015bd50     rilhand.obj
 0002:0001adc8       ??_C@_1FI@LNBLEN@?$AAS?$AAw?$AAi?$AAN?$AAo?$AAt?$AAi?$AAf?$AAy?$AA?$CI?$AAS?$AAW?$AAI?$AA_?$AAN?$AAO?$AAT?$AAI?$AAF?$AAY?$AA_?$AAP?$AAh?$AAo?$AAn?$AAe?$AAb?$AAo?$AAo?$AAk?$AAR?$AAe@ 0015bdc8     rilhand.obj
 0002:0001ae20       ??_C@_1HE@MPAGLBCJ@?$AAO?$AAo?$AAp?$AAs?$AA?5?$AAC?$AAD?$AAM?$AAA?$AA?5?$AAm?$AAo?$AAd?$AAe?$AAm?$AA?5?$AAn?$AAo?$AAt?$AA?5?$AAr?$AAe?$AAa?$AAd?$AAy?$AA?$CB?$AA?0?$AA?5?$AAr?$AAc?$AAP?$AAo@ 0015be20     rilhand.obj
 0002:0001ae98       ??_C@_1FI@MDGNFLJE@?$AAU?$AAn?$AAa?$AAb?$AAl?$AAe?$AA?5?$AAt?$AAo?$AA?5?$AAG?$AAe?$AAt?$AA?5?$AAL?$AAi?$AAs?$AAt?$AA?5?$AAo?$AAf?$AA?5?$AAA?$AAv?$AAa?$AAi?$AAl?$AAa?$AAb?$AAl?$AAe?$AA?5@ 0015be98     rilhand.obj
 0002:0001aef0       ??_C@_1GK@PKELPOMB@?$AAS?$AAw?$AAi?$AAG?$AAe?$AAt?$AAA?$AAv?$AAa?$AAi?$AAl?$AAA?$AAi?$AAr?$AAS?$AAe?$AAr?$AAv?$AAe?$AAr?$AAs?$AA?5?$AAr?$AAe?$AAt?$AAu?$AAr?$AAn?$AAs?$AA?5?$AAZ?$AAE@ 0015bef0     rilhand.obj
 0002:0001af60       ??_C@_1EE@EHCBKDMN@?$AAG?$AAo?$AAb?$AAi?$AA?5?$AAA?$AAi?$AAr?$AAS?$AAe?$AAr?$AAv?$AAe?$AAr?$AA?5?$AAi?$AAs?$AA?5?$AAN?$AAO?$AAT?$AA?5?$AAa?$AAv?$AAa?$AAi?$AAl?$AAa?$AAb?$AAl?$AAe?$AA?4@ 0015bf60     rilhand.obj
 0002:0001afa8       ??_C@_1GG@CFNPNPJL@?$AA?5?$AAC?$AAa?$AAn?$AAn?$AAo?$AAt?$AA?5?$AAt?$AAu?$AAr?$AAn?$AA?5?$AAO?$AAN?$AA?5?$AAt?$AAh?$AAe?$AA?5?$AAm?$AAo?$AAd?$AAe?$AAm?$AA?0?$AA?5?$AAm?$AAp?$AAF?$AAn?$AAS@ 0015bfa8     rilhand.obj
 0002:0001b010       ??_C@_1DO@KNOBMJDK@?$AAR?$AAe?$AAg?$AA?5?$AAC?$AAa?$AAl?$AAl?$AAb?$AAa?$AAc?$AAk?$AA?5?$AAf?$AAa?$AAi?$AAl?$AAe?$AAd?$AA?$CB?$AA?5?$AAr?$AAc?$AA?5?$AA?$DN?$AA?5?$AA?$CI?$AA?$CF?$AAu?$AA?$CJ?$AA?$AA@ 0015c010     rilhand.obj
 0002:0001b050       ??_C@_1FM@HELHNHDN@?$AA?$CK?$AA?$CK?$AA?$CK?$AA?$CK?$AA?$CK?$AAT?$AAh?$AAi?$AAs?$AA?5?$AAi?$AAs?$AA?5?$AAU?$AAN?$AAK?$AAN?$AAO?$AAW?$AAN?$AA?5?$AAW?$AAi?$AAr?$AAe?$AAl?$AAe?$AAs?$AAs?$AA?5?$AAt?$AAe@ 0015c050     rilhand.obj
 0002:0001b0b0       ??_C@_1KC@FPHENCOC@?$AAF?$AAa?$AAi?$AAl?$AAe?$AAd?$AA?5?$AAt?$AAo?$AA?5?$AAu?$AAp?$AAd?$AAa?$AAt?$AAe?$AA?5?$AAH?$AAK?$AAC?$AAU?$AA?2?$AAS?$AAo?$AAf?$AAt?$AAw?$AAa?$AAr?$AAe?$AA?2?$AAS@ 0015c0b0     rilhand.obj
 0002:0001b154       ??_C@_17FKOBBBNL@?$AAG?$AAS?$AAM?$AA?$AA@ 0015c154     rilhand.obj
 0002:0001b15c       ??_C@_1BM@CHNBANCA@?$AAC?$AAa?$AAr?$AAr?$AAi?$AAe?$AAr?$AAS?$AAu?$AAf?$AAf?$AAi?$AAx?$AA?$AA@ 0015c15c     rilhand.obj
 0002:0001b178       ??_C@_1HC@PODCJFNJ@?$AAF?$AAa?$AAi?$AAl?$AAe?$AAd?$AA?5?$AAt?$AAo?$AA?5?$AAu?$AAp?$AAd?$AAa?$AAt?$AAe?$AA?5?$AAS?$AAe?$AAc?$AAu?$AAr?$AAi?$AAt?$AAy?$AA?2?$AAP?$AAh?$AAo?$AAn?$AAe?$AA?2@ 0015c178     rilhand.obj
 0002:0001b1f0       ??_C@_1HK@EJGGKLCH@?$AAF?$AAa?$AAi?$AAl?$AAe?$AAd?$AA?5?$AAt?$AAo?$AA?5?$AAu?$AAp?$AAd?$AAa?$AAt?$AAe?$AA?5?$AAC?$AAo?$AAn?$AAt?$AAr?$AAo?$AAl?$AAP?$AAa?$AAn?$AAe?$AAl?$AA?2?$AAP?$AAh@ 0015c1f0     rilhand.obj
 0002:0001b270       ??_C@_1FE@NGKHCEHE@?$AAG?$AAS?$AAM?$AA?5?$AAd?$AAw?$AAF?$AAe?$AAa?$AAt?$AAu?$AAr?$AAe?$AAs?$AA?5?$AA?$DN?$AA?5?$AAd?$AAw?$AAD?$AAe?$AAf?$AAa?$AAu?$AAl?$AAt?$AAF?$AAe?$AAa?$AAt?$AAu?$AAr@ 0015c270     rilhand.obj
 0002:0001b2c8       ??_C@_1HK@MHHEFKPK@?$AAG?$AAS?$AAM?$AA?5?$AAd?$AAw?$AAF?$AAe?$AAa?$AAt?$AAu?$AAr?$AAe?$AAs?$AA?5?$AA?$DN?$AA?5?$AAd?$AAw?$AAD?$AAe?$AAf?$AAa?$AAu?$AAl?$AAt?$AAF?$AAe?$AAa?$AAt?$AAu?$AAr@ 0015c2c8     rilhand.obj
 0002:0001b348       ??_C@_1HG@HLKDFPLD@?$AAF?$AAa?$AAi?$AAl?$AAe?$AAd?$AA?5?$AAt?$AAo?$AA?5?$AAr?$AAe?$AAa?$AAd?$AA?5?$AAC?$AAo?$AAn?$AAt?$AAr?$AAo?$AAl?$AAP?$AAa?$AAn?$AAe?$AAl?$AA?2?$AAP?$AAh?$AAo?$AAn@ 0015c348     rilhand.obj
 0002:0001b3c0       ??_C@_1FK@PBEAIMHK@?$AAd?$AAw?$AAF?$AAe?$AAa?$AAt?$AAu?$AAr?$AAe?$AAs?$AA?5?$AA?$DN?$AA?5?$AA0?$AAx?$AA?$CF?$AAx?$AA?$DL?$AA?5?$AAu?$AAp?$AAd?$AAa?$AAt?$AAe?$AAd?$AA?5?$AAr?$AAe?$AAg?$AAi?$AAs@ 0015c3c0     rilhand.obj
 0002:0001b420       ??_C@_1HE@IMKCEALP@?$AAF?$AAa?$AAi?$AAl?$AAe?$AAd?$AA?5?$AAt?$AAo?$AA?5?$AAu?$AAp?$AAd?$AAa?$AAt?$AAe?$AA?5?$AAS?$AAe?$AAc?$AAu?$AAr?$AAi?$AAt?$AAy?$AA?2?$AAP?$AAh?$AAo?$AAn?$AAe?$AA?2@ 0015c420     rilhand.obj
 0002:0001b494       ??_C@_1BO@GPKEDHOB@?$AAS?$AAe?$AAc?$AAu?$AAr?$AAi?$AAt?$AAy?$AA?2?$AAP?$AAh?$AAo?$AAn?$AAe?$AA?$AA@ 0015c494     rilhand.obj
 0002:0001b4b8       ??_C@_1HM@MHPMCGHD@?$AAF?$AAa?$AAi?$AAl?$AAe?$AAd?$AA?5?$AAt?$AAo?$AA?5?$AAu?$AAp?$AAd?$AAa?$AAt?$AAe?$AA?5?$AAC?$AAo?$AAn?$AAt?$AAr?$AAo?$AAl?$AAP?$AAa?$AAn?$AAe?$AAl?$AA?2?$AAP?$AAh@ 0015c4b8     rilhand.obj
 0002:0001b538       ??_C@_1HI@GIABGNKN@?$AAF?$AAa?$AAi?$AAl?$AAe?$AAd?$AA?5?$AAt?$AAo?$AA?5?$AAr?$AAe?$AAa?$AAd?$AA?5?$AAC?$AAo?$AAn?$AAt?$AAr?$AAo?$AAl?$AAP?$AAa?$AAn?$AAe?$AAl?$AA?2?$AAP?$AAh?$AAo?$AAn@ 0015c538     rilhand.obj
 0002:0001b5b0       ??_C@_1BC@IGDFDBLI@?$AAF?$AAe?$AAa?$AAt?$AAu?$AAr?$AAe?$AAs?$AA?$AA@ 0015c5b0     rilhand.obj
 0002:0001b5c4       ??_C@_1CG@LJBEDMCE@?$AAC?$AAo?$AAn?$AAt?$AAr?$AAo?$AAl?$AAP?$AAa?$AAn?$AAe?$AAl?$AA?2?$AAP?$AAh?$AAo?$AAn?$AAe?$AA?$AA@ 0015c5c4     rilhand.obj
 0002:0001b5f0       ??_C@_1II@DBDPOKNL@?$AAT?$AAh?$AAe?$AA?5?$AAc?$AAu?$AAr?$AAr?$AAe?$AAn?$AAt?$AA?5?$AAS?$AAW?$AAI?$AA?5?$AAw?$AAi?$AAr?$AAe?$AAl?$AAe?$AAs?$AAs?$AA?5?$AAt?$AAe?$AAc?$AAh?$AAn?$AAo?$AAl@ 0015c5f0     rilhand.obj
 0002:0001b678       ??_C@_1GO@NANGOFMN@?$AAS?$AAe?$AAt?$AA?5?$AAS?$AAo?$AAf?$AAt?$AAw?$AAa?$AAr?$AAe?$AA?2?$AAS?$AAi?$AAe?$AAr?$AAr?$AAa?$AA?5?$AAW?$AAi?$AAr?$AAe?$AAl?$AAe?$AAs?$AAs?$AA?5?$AAI?$AAn?$AAc@ 0015c678     rilhand.obj
 0002:0001b6e8       ??_C@_1BK@GHPPPKCI@?$AAs?$AAz?$AAA?$AAm?$AAs?$AAs?$AAU?$AAi?$AAd?$AA?5?$AA?$CF?$AAs?$AA?$AA@ 0015c6e8     rilhand.obj
 0002:0001b704       ??_C@_1BK@GEIAGMIE@?$AAs?$AAz?$AAA?$AAm?$AAs?$AAs?$AAB?$AAi?$AAd?$AA?5?$AA?$CF?$AAs?$AA?$AA@ 0015c704     rilhand.obj
 0002:0001b720       ??_C@_1BI@DLAOCKKD@?$AAs?$AAz?$AAP?$AAr?$AAi?$AAU?$AAi?$AAd?$AA?5?$AA?$CF?$AAs?$AA?$AA@ 0015c720     rilhand.obj
 0002:0001b738       ??_C@_1BI@DIHBLMAP@?$AAs?$AAz?$AAP?$AAr?$AAi?$AAB?$AAi?$AAd?$AA?5?$AA?$CF?$AAs?$AA?$AA@ 0015c738     rilhand.obj
 0002:0001b750       ??_C@_1HA@EKPJNGHD@?$AAO?$AAp?$AAe?$AAn?$AA?5?$AAS?$AAo?$AAf?$AAt?$AAw?$AAa?$AAr?$AAe?$AA?2?$AAS?$AAi?$AAe?$AAr?$AAr?$AAa?$AA?5?$AAW?$AAi?$AAr?$AAe?$AAl?$AAe?$AAs?$AAs?$AA?5?$AAI?$AAn@ 0015c750     rilhand.obj
 0002:0001b7c0       ??_C@_1KA@MCBPIAGJ@?$AAF?$AAa?$AAi?$AAl?$AA?5?$AAt?$AAo?$AA?5?$AAr?$AAe?$AAa?$AAd?$AA?5?$AAo?$AAn?$AAe?$AA?5?$AAo?$AAf?$AA?5?$AAt?$AAh?$AAe?$AA?5?$AAv?$AAa?$AAl?$AAu?$AAe?$AA?5?$AAu?$AAn@ 0015c7c0     rilhand.obj
 0002:0001b860       ??_C@_1M@OLEMGGOE@?$AA?$CF?$AA0?$AA2?$AAX?$AA?5?$AA?$AA@ 0015c860     rilhand.obj
 0002:0001b86c       ??_C@_1DI@DGELMJDP@?$AAS?$AAe?$AAt?$AAF?$AAw?$AAI?$AAm?$AAa?$AAg?$AAe?$AAP?$AAr?$AAe?$AAf?$AAe?$AAr?$AAe?$AAn?$AAc?$AAe?$AA?5?$AAf?$AAa?$AAi?$AAl?$AAe?$AAd?$AA?$AA@ 0015c86c     rilhand.obj
 0002:0001b8a4       ??_C@_1CC@HLECAKKC@?$AAi?$AAm?$AAa?$AAg?$AAe?$AAL?$AAi?$AAs?$AAt?$AAS?$AAi?$AAz?$AAe?$AA?5?$AA?$CF?$AAd?$AA?$AA@ 0015c8a4     rilhand.obj
 0002:0001b8c8       ??_C@_1BG@NDAHLFMG@?$AAi?$AAm?$AAa?$AAg?$AAe?$AAL?$AAi?$AAs?$AAt?$AA?3?$AA?$AA@ 0015c8c8     rilhand.obj
 0002:0001b8e0       ??_C@_1DO@DFFMONPC@?$AAR?$AAe?$AAs?$AAt?$AAo?$AAr?$AAi?$AAn?$AAg?$AA?5?$AAi?$AAm?$AAa?$AAg?$AAe?$AA?5?$AAp?$AAr?$AAe?$AAf?$AAe?$AAr?$AAe?$AAn?$AAc?$AAe?$AA?5?$AA?4?$AA?4?$AA?4?$AA?$AA@ 0015c8e0     rilhand.obj
 0002:0001b920       ??_C@_1BG@NPGHBPKL@?$AAA?$AAm?$AAs?$AAs?$AAU?$AAi?$AAd?$AA?5?$AA?$CF?$AAs?$AA?$AA@ 0015c920     rilhand.obj
 0002:0001b938       ??_C@_1BG@NMBIIJAH@?$AAA?$AAm?$AAs?$AAs?$AAB?$AAi?$AAd?$AA?5?$AA?$CF?$AAs?$AA?$AA@ 0015c938     rilhand.obj
 0002:0001b950       ??_C@_1BE@BEFALNBB@?$AAP?$AAr?$AAi?$AAU?$AAi?$AAd?$AA?5?$AA?$CF?$AAs?$AA?$AA@ 0015c950     rilhand.obj
 0002:0001b964       ??_C@_1BE@BHCPCLLN@?$AAP?$AAr?$AAi?$AAB?$AAi?$AAd?$AA?5?$AA?$CF?$AAs?$AA?$AA@ 0015c964     rilhand.obj
 0002:0001b978       ??_C@_1BG@IFNFDAIC@?$AAP?$AAR?$AAI?$AAI?$AAm?$AAa?$AAg?$AAe?$AAI?$AAD?$AA?$AA@ 0015c978     rilhand.obj
 0002:0001b990       ??_C@_1BK@NFCMDDIJ@?$AAM?$AAo?$AAd?$AAe?$AAm?$AAI?$AAm?$AAa?$AAg?$AAe?$AAI?$AAD?$AA?$AA@ 0015c990     rilhand.obj
 0002:0001b9ac       ??_C@_1BG@LIKDLEPC@?$AAP?$AAR?$AAI?$AAB?$AAu?$AAi?$AAl?$AAd?$AAI?$AAD?$AA?$AA@ 0015c9ac     rilhand.obj
 0002:0001b9c4       ??_C@_1BK@OIFKLHPJ@?$AAM?$AAo?$AAd?$AAe?$AAm?$AAB?$AAu?$AAi?$AAl?$AAd?$AAI?$AAD?$AA?$AA@ 0015c9c4     rilhand.obj
 0002:0001b9e0       ??_C@_1BI@EKOJIGLA@?$AAS?$AAa?$AAf?$AAe?$AA?5?$AAI?$AAm?$AAa?$AAg?$AAe?$AA?$CB?$AA?$AA@ 0015c9e0     rilhand.obj
 0002:0001b9f8       ??_C@_1FI@JKOFNHKJ@?$AAS?$AAo?$AAf?$AAt?$AAw?$AAa?$AAr?$AAe?$AA?2?$AAS?$AAi?$AAe?$AAr?$AAr?$AAa?$AA?5?$AAW?$AAi?$AAr?$AAe?$AAl?$AAe?$AAs?$AAs?$AA?5?$AAI?$AAn?$AAc?$AA?2?$AAQ?$AAD?$AAL@ 0015c9f8     rilhand.obj
 0002:0001ba50       ??_C@_1GA@DJFHPHBO@?$AAM?$AAo?$AAd?$AAu?$AAl?$AAe?$AA?5?$AAi?$AAs?$AA?5?$AAS?$AAL?$AA9?$AA0?$AA9?$AA0?$AA?5?$AAA?$AAV?$AA?5?$AAc?$AAo?$AAm?$AAp?$AAa?$AAt?$AAi?$AAb?$AAl?$AAe?$AA?0?$AA?5@ 0015ca50     rilhand.obj
 0002:0001bab0       ??_C@_19JKKFOJCB@?$AA0?$AAx?$AAF?$AA1?$AA?$AA@ 0015cab0     rilhand.obj
 0002:0001babc       ??_C@_1M@NDGNLFMH@?$AA?$CF?$AAd?$AA?4?$AA?$CF?$AAd?$AA?$AA@ 0015cabc     rilhand.obj
 0002:0001bac8       ??_C@_1GA@NBJMHFKH@?$AAM?$AAo?$AAd?$AAu?$AAl?$AAe?$AA?5?$AAi?$AAs?$AA?5?$AAS?$AAw?$AAi?$AAM?$AA2?$AAM?$AA?5?$AAA?$AAV?$AA?5?$AAc?$AAo?$AAm?$AAp?$AAa?$AAt?$AAi?$AAb?$AAl?$AAe?$AA?0?$AA?5@ 0015cac8     rilhand.obj
 0002:0001bb28       ??_C@_19BFMHHOHG@?$AA0?$AAx?$AAF?$AA5?$AA?$AA@ 0015cb28     rilhand.obj
 0002:0001bb34       ??_C@_1CG@FJLIKHGJ@?$AAS?$AAW?$AAG?$AAo?$AAb?$AAi?$AAQ?$AAM?$AAI?$AA?2?$AAS?$AAe?$AAr?$AAv?$AAi?$AAc?$AAe?$AAs?$AA?$AA@ 0015cb34     rilhand.obj
 0002:0001bb5c       ??_C@_1CA@FEIADPEA@?$AAI?$AAn?$AA?5?$AAR?$AAU?$AAI?$AAM?$AA?5?$AAm?$AAo?$AAd?$AAe?$AA?5?$AA?$CB?$AA?$CB?$AA?$AA@ 0015cb5c     rilhand.obj
 0002:0001bb80       ??_C@_1IC@DFKIKACA@?$AAU?$AAn?$AAa?$AAb?$AAl?$AAe?$AA?5?$AAt?$AAo?$AA?5?$AAG?$AAe?$AAt?$AA?5?$AAE?$AAx?$AAt?$AAe?$AAn?$AAd?$AAe?$AAd?$AA?5?$AAA?$AAi?$AAr?$AAS?$AAe?$AAr?$AAv?$AAe?$AAr@ 0015cb80     rilhand.obj
 0002:0001bc08       ??_C@_1HG@NHGBBBBF@?$AAU?$AAn?$AAa?$AAb?$AAl?$AAe?$AA?5?$AAt?$AAo?$AA?5?$AAs?$AAe?$AAl?$AAe?$AAc?$AAt?$AA?5?$AAA?$AAi?$AAr?$AAS?$AAe?$AAr?$AAv?$AAe?$AAr?$AA?5?$AA?$DN?$AA?5?$AA?$CF?$AAd?$AA?0@ 0015cc08     rilhand.obj
 0002:0001bc80       ??_C@_1IE@MHMCNCNJ@?$AAU?$AAs?$AAe?$AAr?$AA?5?$AAw?$AAa?$AAn?$AAt?$AAs?$AA?5?$AAt?$AAo?$AA?5?$AAr?$AAe?$AAg?$AAi?$AAs?$AAt?$AAe?$AAr?$AA?5?$AAo?$AAn?$AA?5?$AAa?$AA?5?$AA?$CF?$AAd?$AA?5?$AA?$CI@ 0015cc80     rilhand.obj
 0002:0001bd08       ??_C@_1FM@NFHCLJOJ@?$AAN?$AAe?$AAt?$AAw?$AAo?$AAr?$AAk?$AAP?$AAr?$AAe?$AAf?$AAe?$AAr?$AAe?$AAn?$AAc?$AAe?$AA?5?$AAr?$AAe?$AAg?$AAi?$AAs?$AAt?$AAr?$AAy?$AA?5?$AAk?$AAe?$AAy?$AA?5?$AAd@ 0015cd08     rilhand.obj
 0002:0001bd68       ??_C@_1EE@CPOKLOGM@?$AAY?$AAe?$AAs?$AA?0?$AA?5?$AAG?$AAO?$AAB?$AAI?$AA?5?$AAA?$AAi?$AAr?$AAS?$AAe?$AAr?$AAv?$AAe?$AAr?$AA?5?$AAi?$AAs?$AA?5?$AAa?$AAv?$AAa?$AAi?$AAl?$AAa?$AAb?$AAl?$AAe@ 0015cd68     rilhand.obj
 0002:0001bdac       ??_C@_1CE@CACGJONK@?$AAN?$AAe?$AAt?$AAw?$AAo?$AAr?$AAk?$AAP?$AAr?$AAe?$AAf?$AAe?$AAr?$AAe?$AAn?$AAc?$AAe?$AA?$AA@ 0015cdac     rilhand.obj
 0002:0001bdd0       ??_C@_1DI@MAJHLGJA@?$AAF?$AAa?$AAi?$AAl?$AA?5?$AAS?$AAw?$AAi?$AAA?$AAp?$AAi?$AAS?$AAt?$AAa?$AAr?$AAt?$AAu?$AAp?$AA?0?$AA?5?$AAr?$AAc?$AA?5?$AA?$DN?$AA?5?$AA?$CF?$AAd?$AA?$AA@ 0015cdd0     rilhand.obj
 0002:0001be48       ??_C@_1IA@EJAFMPEI@?$AAC?$AAR?$AAi?$AAl?$AAH?$AAa?$AAn?$AAd?$AAl?$AAe?$AA?3?$AA?3?$AAL?$AAa?$AAu?$AAn?$AAc?$AAh?$AAT?$AAh?$AAr?$AAe?$AAa?$AAd?$AAs?$AA?5?$AA?3?$AA?5?$AAL?$AAa?$AAu?$AAn@ 0015ce48     rilhand.obj
 0002:0001bf3c       ??_C@_1DA@OPKGBPCF@?$AAC?$AAR?$AAi?$AAl?$AAH?$AAa?$AAn?$AAd?$AAl?$AAe?$AA?3?$AA?3?$AA?$HO?$AAC?$AAR?$AAi?$AAl?$AAH?$AAa?$AAn?$AAd?$AAl?$AAe?$AA?$AA@ 0015cf3c     rilhand.obj
 0002:0001bfc8       ??_C@_1GG@EEDJPDMD@?$AAC?$AAR?$AAi?$AAl?$AAH?$AAa?$AAn?$AAd?$AAl?$AAe?$AA?3?$AA?3?$AAS?$AAt?$AAa?$AAr?$AAt?$AAI?$AAn?$AAi?$AAt?$AA?5?$AA?3?$AA?5?$AAV?$AAS?$AAP?$AA?5?$AAi?$AAs?$AA?5?$AAo@ 0015cfc8     rilhand.obj
 0002:0001c030       ??_C@_1DK@PFMIPBAF@?$AAa?$AAc?$AAt?$AAi?$AAv?$AAe?$AAl?$AAo?$AAw?$AA_?$AAs?$AAw?$AAi?$AAm?$AAd?$AAm?$AAr?$AAe?$AAs?$AAe?$AAt?$AA_?$AAs?$AAi?$AAg?$AAn?$AAa?$AAl?$AA?$AA@ 0015d030     rilhand.obj
 0002:0001c06c       ??_C@_1CK@KPOOGEDK@?$AAg?$AA_?$AAd?$AAw?$AAN?$AAe?$AAt?$AAw?$AAo?$AAr?$AAk?$AAT?$AAy?$AAp?$AAe?$AA?5?$AA?$DN?$AA?5?$AA?$CF?$AAd?$AA?$AA@ 0015d06c     rilhand.obj
 0002:0001c098       ??_C@_1FO@OJIAMFBF@?$AAF?$AAa?$AAi?$AAl?$AAe?$AAd?$AA?5?$AAt?$AAo?$AA?5?$AAr?$AAe?$AAa?$AAd?$AA?5?$AAN?$AAe?$AAt?$AAw?$AAo?$AAr?$AAk?$AAT?$AAy?$AAp?$AAe?$AA?5?$AAr?$AAe?$AAg?$AA?5?$AAk@ 0015d098     rilhand.obj
 0002:0001c0f8       ??_C@_1CG@HFKLFDBL@?$AAT?$AAi?$AAm?$AAe?$AAo?$AAu?$AAt?$AAW?$AAa?$AAi?$AAt?$AAF?$AAo?$AAr?$AAI?$AAn?$AAi?$AAt?$AA?$AA@ 0015d0f8     rilhand.obj
 0002:0001c120       ??_C@_1BO@JFNLDEIF@?$AAT?$AAi?$AAm?$AAe?$AAo?$AAu?$AAt?$AAD?$AAT?$AAR?$AAD?$AAr?$AAo?$AAp?$AA?$AA@ 0015d120     rilhand.obj
 0002:0001c140       ??_C@_1CE@OPCAMNLE@?$AAT?$AAi?$AAm?$AAe?$AAo?$AAu?$AAt?$AAA?$AAP?$AAI?$AAD?$AAe?$AAf?$AAa?$AAu?$AAl?$AAt?$AA?$AA@ 0015d140     rilhand.obj
 0002:0001c164       ??_C@_1CC@CDIIGFID@?$AAT?$AAi?$AAm?$AAe?$AAo?$AAu?$AAt?$AAC?$AAm?$AAd?$AAO?$AAn?$AAl?$AAi?$AAn?$AAe?$AA?$AA@ 0015d164     rilhand.obj
 0002:0001c188       ??_C@_1BO@GBIGFFOF@?$AAT?$AAi?$AAm?$AAe?$AAo?$AAu?$AAt?$AAC?$AAm?$AAd?$AAN?$AAo?$AAO?$AAp?$AA?$AA@ 0015d188     rilhand.obj
 0002:0001c1a8       ??_C@_1BO@BBGHDPHO@?$AAT?$AAi?$AAm?$AAe?$AAo?$AAu?$AAt?$AAC?$AAm?$AAd?$AAI?$AAn?$AAi?$AAt?$AA?$AA@ 0015d1a8     rilhand.obj
 0002:0001c1c8       ??_C@_1CE@IOIFLPGB@?$AA?4?$AA?2?$AAr?$AAi?$AAl?$AAh?$AAa?$AAn?$AAd?$AAn?$AAd?$AAi?$AAs?$AA?4?$AAc?$AAp?$AAp?$AA?$AA@ 0015d1c8     rilhandndis.obj
 0002:0001c1f0       ??_C@_1HG@NJPLAELI@?$AAN?$AAd?$AAi?$AAs?$AAI?$AAn?$AAt?$AAe?$AAr?$AAf?$AAa?$AAc?$AAe?$AAT?$AAr?$AAa?$AAn?$AAs?$AAm?$AAi?$AAt?$AAE?$AAv?$AAe?$AAn?$AAt?$AA?5?$AAn?$AAo?$AAt?$AA?5?$AAh@ 0015d1f0     rilhandndis.obj
 0002:0001c2e8       ??_C@_1FE@MEMIIMOL@?$AAR?$AAI?$AAL?$AAN?$AAD?$AAI?$AAS?$AA?5?$AAd?$AAa?$AAt?$AAa?$AA?5?$AAc?$AAa?$AAl?$AAl?$AA?5?$AAd?$AAi?$AAs?$AAc?$AAo?$AAn?$AAn?$AAe?$AAc?$AAt?$AAe?$AAd?$AA?0?$AA?5@ 0015d2e8     rilhandndis.obj
 0002:0001c340       ??_C@_1FI@BIBOBACJ@?$AAR?$AAI?$AAL?$AAN?$AAD?$AAI?$AAS?$AA?5?$AAd?$AAa?$AAt?$AAa?$AA?5?$AAc?$AAa?$AAl?$AAl?$AA?5?$AAc?$AAo?$AAn?$AAn?$AAe?$AAc?$AAt?$AAe?$AAd?$AA?3?$AA?5?$AAc?$AAo?$AAn@ 0015d340     rilhandndis.obj
 0002:0001c398       ??_C@_1DO@JIDKPIAM@?$AAN?$AAo?$AA?5?$AAs?$AAe?$AAc?$AAo?$AAn?$AAd?$AAa?$AAr?$AAy?$AA?5?$AAD?$AAN?$AAS?$AA?5?$AAi?$AAs?$AA?5?$AAr?$AAe?$AAt?$AAr?$AAi?$AAe?$AAv?$AAe?$AAd?$AA?4?$AA?$AA@ 0015d398     rilhandndis.obj
 0002:0001c3d8       ??_C@_13JOFGPIOO@?$AA?4?$AA?$AA@ 0015d3d8     rilhandndis.obj
 0002:0001c3dc       ??_C@_1DK@KMBOGHKG@?$AAN?$AAo?$AA?5?$AAp?$AAr?$AAi?$AAm?$AAa?$AAr?$AAy?$AA?5?$AAD?$AAN?$AAS?$AA?5?$AAi?$AAs?$AA?5?$AAr?$AAe?$AAt?$AAr?$AAi?$AAe?$AAv?$AAe?$AAd?$AA?4?$AA?$AA@ 0015d3dc     rilhandndis.obj
 0002:0001c418       ??_C@_1JG@KMFMDAO@?$AAF?$AAa?$AAi?$AAl?$AA?5?$AAt?$AAo?$AA?5?$AAi?$AAn?$AAs?$AAt?$AAa?$AAn?$AAt?$AAi?$AAa?$AAt?$AAe?$AA?5?$AAc?$AAo?$AAm?$AAm?$AAu?$AAn?$AAi?$AAc?$AAa?$AAt?$AAi?$AAo@ 0015d418     rilhandndis.obj
 0002:0001c4b0       ??_C@_1KO@LPJMGECI@?$AAF?$AAa?$AAi?$AAl?$AA?5?$AAt?$AAo?$AA?5?$AAg?$AAe?$AAt?$AA?5?$AAt?$AAh?$AAe?$AA?5?$AAI?$AAP?$AA?5?$AAa?$AAd?$AAd?$AAr?$AAe?$AAs?$AAs?$AA?5?$AAa?$AAf?$AAt?$AAe?$AAr@ 0015d4b0     rilhandndis.obj
 0002:0001c560       ??_C@_1ME@MCJKALHH@?$AAF?$AAa?$AAi?$AAl?$AA?5?$AAt?$AAo?$AA?5?$AAG?$AAE?$AAT?$AA?5?$AAf?$AAu?$AAn?$AAc?$AAt?$AAi?$AAo?$AAn?$AA?5?$AAp?$AAo?$AAi?$AAn?$AAt?$AAe?$AAr?$AAs?$AA?5?$AAf?$AAr@ 0015d560     rilhandndis.obj
 0002:0001c628       ??_C@_1HA@NNHLCPBG@?$AAF?$AAa?$AAi?$AAl?$AA?5?$AAt?$AAo?$AA?5?$AAS?$AAE?$AAT?$AA?5?$AAC?$AAB?$AA?5?$AAf?$AAu?$AAn?$AAc?$AAt?$AAi?$AAo?$AAn?$AA?5?$AAp?$AAo?$AAi?$AAn?$AAt?$AAe?$AAr?$AAs@ 0015d628     rilhandndis.obj
 0002:0001c698       ??_C@_19MNOLIHKD@?$AAS?$AAW?$AAD?$AA1?$AA?$AA@ 0015d698     rilhandndis.obj
 0002:0001c6a8       ??_C@_1GE@EJAFLBJN@?$AAA?$AAS?$AAS?$AAE?$AAR?$AAT?$AAI?$AAO?$AAN?$AA?5?$AAF?$AAA?$AAI?$AAL?$AAU?$AAR?$AAE?$AA?3?$AA?5?$AA?$DN?$AA?$DN?$AA?$DN?$AA?$DO?$AAl?$AAp?$AAE?$AAv?$AAe?$AAn?$AAt?$AA?9?$AA?$DO@ 0015d6a8     rilhandndis.obj
 0002:0001c710       ??_C@_1FM@BEAGPJOB@?$AAR?$AAI?$AAL?$AAN?$AAD?$AAI?$AAS?$AA?3?$AA?5?$AAh?$AAa?$AAn?$AAd?$AAl?$AAi?$AAn?$AAg?$AA?5?$AAO?$AAE?$AAM?$AA_?$AAN?$AAD?$AAI?$AAS?$AA_?$AAT?$AAX?$AA_?$AAP?$AAA@ 0015d710     rilhandndis.obj
 0002:0001c770       ??_C@_1FE@PEPIOGOD@?$AAR?$AAI?$AAL?$AAN?$AAD?$AAI?$AAS?$AA?3?$AA?5?$AAO?$AAE?$AAM?$AA_?$AAN?$AAD?$AAI?$AAS?$AA_?$AAR?$AAX?$AA_?$AAP?$AAA?$AAC?$AAK?$AAE?$AAT?$AA?5?$AAp?$AAa?$AAc?$AAk@ 0015d770     rilhandndis.obj
 0002:0001c818       ??_C@_1GM@PCKDCBGG@?$AAT?$AAh?$AAe?$AAr?$AAe?$AA?5?$AAi?$AAs?$AA?5?$AAn?$AAo?$AA?5?$AAm?$AAo?$AAr?$AAe?$AA?5?$AAN?$AAD?$AAI?$AAS?$AA?5?$AAd?$AAa?$AAt?$AAa?$AA?5?$AAc?$AAa?$AAl?$AAl?$AA?5@ 0015d818     rilhandndis.obj
 0002:0001c888       ??_C@_1FK@KDOCJOGD@?$AAR?$AAI?$AAL?$AAN?$AAD?$AAI?$AAS?$AA?3?$AA?5?$AAF?$AAa?$AAi?$AAl?$AA?5?$AAS?$AAw?$AAi?$AAS?$AAe?$AAt?$AAG?$AAS?$AAM?$AAP?$AAr?$AAo?$AAf?$AAi?$AAl?$AAe?$AAB?$AAa@ 0015d888     rilhandndis.obj
 0002:0001c8e8       ??_C@_1FK@NHJGOKAO@?$AAR?$AAI?$AAL?$AAN?$AAD?$AAI?$AAS?$AA?3?$AA?5?$AAF?$AAa?$AAi?$AAl?$AA?5?$AAS?$AAw?$AAi?$AAG?$AAe?$AAt?$AAG?$AAS?$AAM?$AAP?$AAr?$AAo?$AAf?$AAi?$AAl?$AAe?$AAB?$AAa@ 0015d8e8     rilhandndis.obj
 0002:0001c948       ??_C@_1HO@GJAJGFKL@?$AAR?$AAI?$AAL?$AAN?$AAD?$AAI?$AAS?$AA?3?$AA?5?$AAN?$AAd?$AAi?$AAs?$AAS?$AAe?$AAt?$AAG?$AAP?$AAR?$AAS?$AAC?$AAo?$AAn?$AAt?$AAe?$AAx?$AAt?$AAA?$AAc?$AAt?$AAi?$AAv@ 0015d948     rilhandndis.obj
 0002:0001c9c8       ??_C@_1BM@DBIICOFC@?$AA?4?$AA?2?$AAr?$AAi?$AAl?$AAm?$AAa?$AAi?$AAn?$AA?4?$AAc?$AAp?$AAp?$AA?$AA@ 0015d9c8     rilmain.obj
 0002:0001c9e8       ??_C@_1EG@KKHADHIJ@?$AAR?$AAI?$AAL?$AAD?$AAr?$AAv?$AA_?$AAG?$AAe?$AAt?$AAA?$AAu?$AAd?$AAi?$AAo?$AAD?$AAe?$AAv?$AAi?$AAc?$AAe?$AAs?$AA?5?$AA?3?$AA?5?$AAE?$AA_?$AAN?$AAO?$AAT?$AAI?$AAM@ 0015d9e8     rilmain.obj
 0002:0001ca30       ??_C@_1FI@GOLKNALO@?$AAR?$AAI?$AAL?$AAD?$AAr?$AAv?$AA_?$AAS?$AAe?$AAt?$AAH?$AAi?$AAd?$AAe?$AAC?$AAo?$AAn?$AAn?$AAe?$AAc?$AAt?$AAe?$AAd?$AAI?$AAd?$AAS?$AAt?$AAa?$AAt?$AAu?$AAs?$AA?5@ 0015da30     rilmain.obj
 0002:0001ca88       ??_C@_1DK@MPAHECIH@?$AAD?$AAl?$AAl?$AAM?$AAa?$AAi?$AAn?$AA?5?$AA?3?$AA?5?$AAD?$AAL?$AAL?$AA_?$AAP?$AAR?$AAO?$AAC?$AAE?$AAS?$AAS?$AA_?$AAD?$AAE?$AAT?$AAA?$AAC?$AAH?$AA?$AA@ 0015da88     rilmain.obj
 0002:0001cac4       ??_C@_1DK@NMBJINHJ@?$AAD?$AAl?$AAl?$AAM?$AAa?$AAi?$AAn?$AA?5?$AA?3?$AA?5?$AAD?$AAL?$AAL?$AA_?$AAP?$AAR?$AAO?$AAC?$AAE?$AAS?$AAS?$AA_?$AAA?$AAT?$AAT?$AAA?$AAC?$AAH?$AA?$AA@ 0015dac4     rilmain.obj
 0002:0001cb00       ??_C@_1EG@OECLAFGC@?$AAA?$AAS?$AAS?$AAE?$AAR?$AAT?$AAI?$AAO?$AAN?$AA?5?$AAF?$AAA?$AAI?$AAL?$AAU?$AAR?$AAE?$AA?3?$AA?5?$AA?$DN?$AA?$DN?$AA?$DN?$AA?$DO?$AAd?$AAw?$AAD?$AAa?$AAt?$AAa?$AA?5?$AA?$CB?$AA?$DN@ 0015db00     rilmain.obj
 0002:0001cb48       ??_C@_1OG@NBMIIGEI@?$AA?$AN?$AA?6?$AAC?$AAG?$AAo?$AAb?$AAi?$AA?3?$AA?3?$AAD?$AAo?$AAF?$AAi?$AAr?$AAm?$AAw?$AAa?$AAr?$AAe?$AAU?$AAp?$AAg?$AAr?$AAa?$AAd?$AAe?$AA?3?$AA?3?$AA?5?$AAF?$AAa?$AAi@ 0015db48     rilmain.obj
 0002:0001cc30       ??_C@_1BAI@PDLHOHON@?$AA?$AN?$AA?6?$AAC?$AAG?$AAo?$AAb?$AAi?$AA?3?$AA?3?$AAD?$AAo?$AAF?$AAi?$AAr?$AAm?$AAw?$AAa?$AAr?$AAe?$AAU?$AAp?$AAg?$AAr?$AAa?$AAd?$AAe?$AA?3?$AA?3?$AA?5?$AAF?$AAa?$AAi@ 0015dc30     rilmain.obj
 0002:0001cd38       ??_C@_1M@PIGKLJLL@?$AA?$CF?$AAs?$AA?2?$AA?$CF?$AAd?$AA?$AA@ 0015dd38     rilmain.obj
 0002:0001cd48       ??_C@_1HA@IHMCMDCH@?$AA?$AN?$AA?6?$AAC?$AAG?$AAo?$AAb?$AAi?$AA?3?$AA?3?$AAD?$AAo?$AAF?$AAi?$AAr?$AAm?$AAw?$AAa?$AAr?$AAe?$AAU?$AAp?$AAg?$AAr?$AAa?$AAd?$AAe?$AA?3?$AA?3?$AA?5?$AAF?$AAa?$AAi@ 0015dd48     rilmain.obj
 0002:0001cdb8       ??_C@_1IM@BKNLIJNE@?$AA?$AN?$AA?6?$AAC?$AAG?$AAo?$AAb?$AAi?$AA?3?$AA?3?$AAD?$AAo?$AAF?$AAi?$AAr?$AAm?$AAw?$AAa?$AAr?$AAe?$AAU?$AAp?$AAg?$AAr?$AAa?$AAd?$AAe?$AA?3?$AA?3?$AA?5?$AAF?$AAa?$AAi@ 0015ddb8     rilmain.obj
 0002:0001ce48       ??_C@_1II@EJEPKAHJ@?$AA?$AN?$AA?6?$AAC?$AAG?$AAo?$AAb?$AAi?$AA?3?$AA?3?$AAD?$AAo?$AAF?$AAi?$AAr?$AAm?$AAw?$AAa?$AAr?$AAe?$AAU?$AAp?$AAg?$AAr?$AAa?$AAd?$AAe?$AA?3?$AA?3?$AA?5?$AAT?$AAh?$AAe@ 0015de48     rilmain.obj
 0002:0001ced0       ??_C@_1IM@HAGKIOKP@?$AA?$AN?$AA?6?$AAC?$AAG?$AAo?$AAb?$AAi?$AA?3?$AA?3?$AAD?$AAo?$AAF?$AAi?$AAr?$AAm?$AAw?$AAa?$AAr?$AAe?$AAU?$AAp?$AAg?$AAr?$AAa?$AAd?$AAe?$AA?3?$AA?3?$AA?5?$AAI?$AAm?$AAa@ 0015ded0     rilmain.obj
 0002:0001cf60       ??_C@_1LA@LJGPHEBP@?$AA?$AN?$AA?6?$AAC?$AAG?$AAo?$AAb?$AAi?$AA?3?$AA?3?$AAD?$AAo?$AAF?$AAi?$AAr?$AAm?$AAw?$AAa?$AAr?$AAe?$AAU?$AAp?$AAg?$AAr?$AAa?$AAd?$AAe?$AA?3?$AA?3?$AA?5?$AAR?$AAe?$AAs@ 0015df60     rilmain.obj
 0002:0001d010       ??_C@_1GM@ICFBNCFO@?$AA?$AN?$AA?6?$AAC?$AAG?$AAo?$AAb?$AAi?$AA?3?$AA?3?$AAD?$AAo?$AAF?$AAi?$AAr?$AAm?$AAw?$AAa?$AAr?$AAe?$AAU?$AAp?$AAg?$AAr?$AAa?$AAd?$AAe?$AA?3?$AA?3?$AA?5?$AA?$CF?$AAs?$AA?5@ 0015e010     rilmain.obj
 0002:0001d080       ??_C@_1GK@GPENKJPG@?$AA?$AN?$AA?6?$AAC?$AAG?$AAo?$AAb?$AAi?$AA?3?$AA?3?$AAD?$AAo?$AAF?$AAi?$AAr?$AAm?$AAw?$AAa?$AAr?$AAe?$AAU?$AAp?$AAg?$AAr?$AAa?$AAd?$AAe?$AA?3?$AA?3?$AA?5?$AA?$CF?$AAs?$AA?5@ 0015e080     rilmain.obj
 0002:0001d0f0       ??_C@_1OM@LOHFDJBL@?$AA?$AN?$AA?6?$AAC?$AAG?$AAo?$AAb?$AAi?$AA?3?$AA?3?$AAD?$AAo?$AAF?$AAi?$AAr?$AAm?$AAw?$AAa?$AAr?$AAe?$AAU?$AAp?$AAg?$AAr?$AAa?$AAd?$AAe?$AA?3?$AA?3?$AA?5?$AAF?$AAa?$AAi@ 0015e0f0     rilmain.obj
 0002:0001d1e0       ??_C@_1GM@NLEFDCFE@?$AA?$AN?$AA?6?$AAC?$AAG?$AAo?$AAb?$AAi?$AA?3?$AA?3?$AAD?$AAo?$AAF?$AAi?$AAr?$AAm?$AAw?$AAa?$AAr?$AAe?$AAU?$AAp?$AAg?$AAr?$AAa?$AAd?$AAe?$AA?3?$AA?3?$AA?5?$AAF?$AAo?$AAr@ 0015e1e0     rilmain.obj
 0002:0001d24c       ??_C@_19HEPLDNLP@?$AA?$CF?$AAs?$AA?$CF?$AAd?$AA?$AA@ 0015e24c     rilmain.obj
 0002:0001d258       ??_C@_1BBA@FHJCDMAI@?$AA?$AN?$AA?6?$AAC?$AAG?$AAo?$AAb?$AAi?$AA?3?$AA?3?$AAD?$AAo?$AAF?$AAi?$AAr?$AAm?$AAw?$AAa?$AAr?$AAe?$AAU?$AAp?$AAg?$AAr?$AAa?$AAd?$AAe?$AA?3?$AA?3?$AA?5?$AAS?$AAu?$AAc@ 0015e258     rilmain.obj
 0002:0001d368       ??_C@_1BAG@CMCLMFHD@?$AA?$AN?$AA?6?$AAC?$AAG?$AAo?$AAb?$AAi?$AA?3?$AA?3?$AAD?$AAo?$AAF?$AAi?$AAr?$AAm?$AAw?$AAa?$AAr?$AAe?$AAU?$AAp?$AAg?$AAr?$AAa?$AAd?$AAe?$AA?3?$AA?3?$AA?5?$AAF?$AAa?$AAi@ 0015e368     rilmain.obj
 0002:0001d470       ??_C@_1CA@BFGBOAIH@?$AAF?$AAo?$AAr?$AAc?$AAe?$AAF?$AAW?$AAD?$AAo?$AAw?$AAn?$AAl?$AAo?$AAa?$AAd?$AA?$AA@ 0015e470     rilmain.obj
 0002:0001d490       ??_C@_1EK@ECJGCHPJ@?$AAn?$AAo?$AA?5?$AAc?$AAa?$AAr?$AAr?$AAi?$AAe?$AAr?$AA?5?$AAw?$AAa?$AAs?$AA?5?$AAs?$AAe?$AAl?$AAe?$AAc?$AAt?$AAe?$AAd?$AA?0?$AA?5?$AAd?$AAo?$AA?5?$AAn?$AAo?$AAt?$AAh@ 0015e490     rilmain.obj
 0002:0001d4dc       ??_C@_1CC@OPPLHLDH@?$AAF?$AAi?$AAr?$AAm?$AAw?$AAa?$AAr?$AAe?$AAL?$AAo?$AAc?$AAa?$AAt?$AAi?$AAo?$AAn?$AA?$AA@ 0015e4dc     rilmain.obj
 0002:0001d570       ??_C@_1EI@HOHMODHF@?$AAR?$AAI?$AAL?$AA_?$AAI?$AAn?$AAi?$AAt?$AA?5?$AA?3?$AA?5?$AAR?$AAI?$AAL?$AA?5?$AAf?$AAa?$AAi?$AAl?$AAe?$AAd?$AA?5?$AAt?$AAo?$AA?5?$AAi?$AAn?$AAi?$AAt?$AAi?$AAa?$AAl@ 0015e570     rilmain.obj
 0002:0001d5b8       ??_C@_1EA@MLENMHGG@?$AAR?$AAI?$AAL?$AA_?$AAI?$AAn?$AAi?$AAt?$AA?5?$AA?3?$AA?5?$AAS?$AAt?$AAa?$AAr?$AAt?$AAe?$AAd?$AA?5?$AAs?$AAu?$AAc?$AAc?$AAe?$AAs?$AAs?$AAf?$AAu?$AAl?$AAl?$AAy?$AA?$AA@ 0015e5b8     rilmain.obj
 0002:0001d5f8       ??_C@_1BO@LGHGDGAG@?$AAR?$AAI?$AAL?$AAD?$AAr?$AAv?$AA_?$AAP?$AAr?$AAe?$AAs?$AAe?$AAn?$AAt?$AA?$AA@ 0015e5f8     rilmain.obj
 0002:0001d618       ??_C@_1DO@CMEBMNLF@?$AAR?$AAI?$AAL?$AA_?$AAI?$AAn?$AAi?$AAt?$AA?5?$AA?3?$AA?5?$AAp?$AAa?$AAr?$AAa?$AAm?$AAs?$AA?3?$AA?5?$AAd?$AAw?$AAI?$AAn?$AAf?$AAo?$AA?5?$AA?$DN?$AA?5?$AA?$CF?$AAd?$AA?$AA@ 0015e618     rilmain.obj
 0002:0001d6a4       ??_C@_1CE@DJLLJBPI@?$AAR?$AAI?$AAL?$AA_?$AAO?$AAp?$AAe?$AAn?$AA?5?$AAr?$AAe?$AAj?$AAe?$AAc?$AAt?$AAs?$AA?$CB?$AA?$AA@ 0015e6a4     rilmain.obj
 0002:0001d6c8       ??_C@_1DE@LDIPIANA@?$AAR?$AAI?$AAL?$AA_?$AAI?$AAO?$AAC?$AAo?$AAn?$AAt?$AAr?$AAo?$AAl?$AA?$CB?$AA?5?$AAI?$AAO?$AAC?$AAT?$AAL?$AA?5?$AA?$DN?$AA?5?$AA?$CF?$AAd?$AA?$AA@ 0015e6c8     rilmain.obj
 0002:0001d700       ??_C@_1OE@LNBLILNA@?$AA?$CB?$AA?$CB?$AA?$CB?$AA?$CB?$AA?$CB?$AA?$CB?$AA?$CB?$AA?5?$AAA?$AA?5?$AAL?$AA?5?$AAO?$AA?5?$AA?$DP?$AA?$DP?$AA?$DP?$AA?$DP?$AA?$DP?$AA?$DP?$AA?5?$AAF?$AAo?$AAr?$AAg?$AAo?$AAt?$AA?5?$AAt?$AAo?$AA?5?$AAu@ 0015e700     rilmain.obj
 0002:0001d7e8       ??_C@_1FC@HIIFJEFC@?$AAV?$AAa?$AAl?$AAi?$AAd?$AAa?$AAt?$AAe?$AAA?$AAP?$AAI?$AAP?$AAe?$AAr?$AAm?$AAi?$AAs?$AAs?$AAi?$AAo?$AAn?$AA?5?$AAf?$AAa?$AAi?$AAl?$AAe?$AAd?$AA?5?$AAo?$AAn?$AA?5@ 0015e7e8     rilmain.obj
 0002:0001d840       ??_C@_1EM@EMKCKLCD@?$AAI?$AAO?$AAC?$AAT?$AAL?$AA_?$AAR?$AAI?$AAL?$AA_?$AAC?$AAA?$AAN?$AAC?$AAE?$AAL?$AAS?$AAU?$AAP?$AAS?$AAE?$AAR?$AAV?$AAI?$AAC?$AAE?$AAD?$AAA?$AAT?$AAA?$AAS?$AAE@ 0015e840     rilmain.obj
 0002:0001d88c       ??_C@_1DK@PKIENGIC@?$AAI?$AAO?$AAC?$AAT?$AAL?$AA_?$AAR?$AAI?$AAL?$AA_?$AAS?$AAE?$AAN?$AAD?$AAS?$AAU?$AAP?$AAS?$AAE?$AAR?$AAV?$AAI?$AAC?$AAE?$AAD?$AAA?$AAT?$AAA?$AA?$AA@ 0015e88c     rilmain.obj
 0002:0001d8c8       ??_C@_1BBC@OOPDDACM@?$AAI?$AAO?$AAC?$AAT?$AAL?$AA_?$AAR?$AAI?$AAL?$AA_?$AAG?$AAE?$AAT?$AAD?$AAR?$AAI?$AAV?$AAE?$AAR?$AAV?$AAE?$AAR?$AAS?$AAI?$AAO?$AAN?$AAE?$AAX?$AA?3?$AA?5?$AAp?$AAR@ 0015e8c8     rilmain.obj
 0002:0001d9e0       ??_C@_1NC@LLDHMPAP@?$AAM?$AAi?$AAc?$AAr?$AAo?$AAs?$AAo?$AAf?$AAt?$AA?5?$AAW?$AAi?$AAn?$AAd?$AAo?$AAw?$AAs?$AA?5?$AAC?$AAE?$AA?3?$AA?5?$AAM?$AAa?$AAj?$AAo?$AAr?$AA?5?$AAv?$AAe?$AAr?$AAs@ 0015e9e0     rilmain.obj
 0002:0001dab4       ??_C@_1BK@CKLBEDFK@?$AAV?$AAe?$AAr?$AAs?$AAi?$AAo?$AAn?$AAi?$AAn?$AAg?$AAE?$AAx?$AA?$AA@ 0015eab4     rilmain.obj
 0002:0001dad0       ??_C@_1BK@PCELPCLA@?$AAA?$AAP?$AAI?$AA?5?$AAR?$AAo?$AAu?$AAt?$AAi?$AAn?$AAe?$AAs?$AA?$AA@ 0015ead0     rilmain.obj
 0002:0001daec       ??_C@_1CK@NGKMNFNC@?$AAN?$AAo?$AAt?$AAi?$AAf?$AAi?$AAc?$AAa?$AAt?$AAi?$AAo?$AAn?$AA?5?$AAC?$AAl?$AAa?$AAs?$AAs?$AAe?$AAs?$AA?$AA@ 0015eaec     rilmain.obj
 0002:0001db18       ??_C@_1BK@COMCHFH@?$AAR?$AAe?$AAs?$AAu?$AAl?$AAt?$AA?5?$AAC?$AAo?$AAd?$AAe?$AAs?$AA?$AA@ 0015eb18     rilmain.obj
 0002:0001db34       ??_C@_1CG@LBCAKCLL@?$AAN?$AAo?$AAt?$AAi?$AAf?$AAi?$AAc?$AAa?$AAt?$AAi?$AAo?$AAn?$AA?5?$AAC?$AAo?$AAd?$AAe?$AAs?$AA?$AA@ 0015eb34     rilmain.obj
 0002:0001db5c       ??_C@_1BM@FFKFMPJP@?$AAE?$AAr?$AAr?$AAo?$AAr?$AA?5?$AAC?$AAl?$AAa?$AAs?$AAs?$AAe?$AAs?$AA?$AA@ 0015eb5c     rilmain.obj
 0002:0001db78       ??_C@_1BI@MEKOKMNO@?$AAE?$AAr?$AAr?$AAo?$AAr?$AA?5?$AAC?$AAo?$AAd?$AAe?$AAs?$AA?$AA@ 0015eb78     rilmain.obj
 0002:0001db90       ??_C@_1FA@ILDHHHFN@?$AAR?$AAI?$AAL?$AA?5?$AAS?$AAE?$AAT?$AAC?$AAU?$AAR?$AAR?$AAE?$AAN?$AAT?$AAA?$AAD?$AAD?$AAR?$AAE?$AAS?$AAS?$AAI?$AAD?$AA?5?$AAr?$AAe?$AAt?$AAu?$AAr?$AAn?$AAs?$AA?5@ 0015eb90     rilmain.obj
 0002:0001dbe0       ??_C@_1FA@LOJCCNAA@?$AAR?$AAI?$AAL?$AA?5?$AAG?$AAE?$AAT?$AAC?$AAU?$AAR?$AAR?$AAE?$AAN?$AAT?$AAA?$AAD?$AAD?$AAR?$AAE?$AAS?$AAS?$AAI?$AAD?$AA?5?$AAr?$AAe?$AAt?$AAu?$AAr?$AAn?$AAs?$AA?5@ 0015ebe0     rilmain.obj
 0002:0001dc30       ??_C@_1EG@DPDFPNIM@?$AAI?$AAO?$AAC?$AAT?$AAL?$AA_?$AAR?$AAI?$AAL?$AA_?$AAS?$AAW?$AAI?$AA_?$AAG?$AAO?$AAB?$AAI?$AA_?$AAC?$AAA?$AAR?$AAR?$AAI?$AAE?$AAR?$AA_?$AAS?$AAW?$AAI?$AAT?$AAC@ 0015ec30     rilmain.obj
 0002:0001dc78       ??_C@_1CA@OKOEHIDM@?$AAW?$AAr?$AAo?$AAn?$AAg?$AA?5?$AAp?$AAa?$AAr?$AAa?$AAm?$AAs?$AA?5?$AA?$CF?$AAd?$AA?$AA@ 0015ec78     rilmain.obj
 0002:0001dc98       ??_C@_1CG@LNBKANIK@?$AAp?$AAR?$AAi?$AAl?$AAD?$AAe?$AAv?$AAi?$AAc?$AAe?$AA?5?$AAi?$AAs?$AA?5?$AAN?$AAU?$AAL?$AAL?$AA?$AA@ 0015ec98     rilmain.obj
 0002:0001dcc0       ??_C@_1BO@KCNEBGOO@?$AAp?$AAR?$AAa?$AAd?$AAi?$AAo?$AA?5?$AAi?$AAs?$AA?5?$AAN?$AAU?$AAL?$AAL?$AA?$AA@ 0015ecc0     rilmain.obj
 0002:0001dce0       ??_C@_1EG@BKFOKCFA@?$AAI?$AAO?$AAC?$AAT?$AAL?$AA_?$AAR?$AAI?$AAL?$AA_?$AAS?$AAW?$AAI?$AA_?$AAG?$AAO?$AAB?$AAI?$AA_?$AAC?$AAA?$AAR?$AAR?$AAI?$AAE?$AAR?$AA_?$AAS?$AAW?$AAI?$AAT?$AAC@ 0015ece0     rilmain.obj
 0002:0001dd28       ??_C@_1FM@EGFMHFAC@?$AAI?$AAO?$AAC?$AAT?$AAL?$AA_?$AAR?$AAI?$AAL?$AA_?$AAS?$AAW?$AAI?$AA_?$AAS?$AAE?$AAT?$AA_?$AAG?$AAP?$AAS?$AAO?$AAN?$AAE?$AAX?$AAT?$AAR?$AAA?$AA?3?$AA?5?$AAW?$AAr@ 0015ed28     rilmain.obj
 0002:0001dd88       ??_C@_1GC@HDFOGNJH@?$AAI?$AAO?$AAC?$AAT?$AAL?$AA_?$AAR?$AAI?$AAL?$AA_?$AAS?$AAW?$AAI?$AA_?$AAS?$AAE?$AAT?$AA_?$AAG?$AAP?$AAS?$AAO?$AAN?$AAE?$AAX?$AAT?$AAR?$AAA?$AA?3?$AA?5?$AAp?$AAR@ 0015ed88     rilmain.obj
 0002:0001ddf0       ??_C@_1FK@INIMCIGI@?$AAI?$AAO?$AAC?$AAT?$AAL?$AA_?$AAR?$AAI?$AAL?$AA_?$AAS?$AAW?$AAI?$AA_?$AAS?$AAE?$AAT?$AA_?$AAG?$AAP?$AAS?$AAO?$AAN?$AAE?$AAX?$AAT?$AAR?$AAA?$AA?3?$AA?5?$AAp?$AAR@ 0015edf0     rilmain.obj
 0002:0001de50       ??_C@_1IM@NGNNEDPB@?$AAI?$AAO?$AAC?$AAT?$AAL?$AA_?$AAR?$AAI?$AAL?$AA_?$AAS?$AAW?$AAI?$AA_?$AAS?$AAE?$AAT?$AA_?$AAG?$AAP?$AAS?$AAO?$AAN?$AAE?$AAX?$AAT?$AAR?$AAA?$AA?3?$AA?5?$AAp?$AAR@ 0015ee50     rilmain.obj
 0002:0001dee0       ??_C@_1FM@GNPAJPMF@?$AAI?$AAO?$AAC?$AAT?$AAL?$AA_?$AAR?$AAI?$AAL?$AA_?$AAS?$AAW?$AAI?$AA_?$AAS?$AAE?$AAT?$AA_?$AAG?$AAP?$AAS?$AAD?$AAE?$AAF?$AAA?$AAU?$AAL?$AAT?$AA?3?$AA?5?$AAW?$AAr@ 0015eee0     rilmain.obj
 0002:0001df40       ??_C@_1GC@COHCJDFJ@?$AAI?$AAO?$AAC?$AAT?$AAL?$AA_?$AAR?$AAI?$AAL?$AA_?$AAS?$AAW?$AAI?$AA_?$AAS?$AAE?$AAT?$AA_?$AAG?$AAP?$AAS?$AAD?$AAE?$AAF?$AAA?$AAU?$AAL?$AAT?$AA?3?$AA?5?$AAp?$AAR@ 0015ef40     rilmain.obj
 0002:0001dfa8       ??_C@_1FK@IKJOOFLP@?$AAI?$AAO?$AAC?$AAT?$AAL?$AA_?$AAR?$AAI?$AAL?$AA_?$AAS?$AAW?$AAI?$AA_?$AAS?$AAE?$AAT?$AA_?$AAG?$AAP?$AAS?$AAD?$AAE?$AAF?$AAA?$AAU?$AAL?$AAT?$AA?3?$AA?5?$AAp?$AAR@ 0015efa8     rilmain.obj
 0002:0001e008       ??_C@_1IM@EBPFJNBF@?$AAI?$AAO?$AAC?$AAT?$AAL?$AA_?$AAR?$AAI?$AAL?$AA_?$AAS?$AAW?$AAI?$AA_?$AAS?$AAE?$AAT?$AA_?$AAG?$AAP?$AAS?$AAD?$AAE?$AAF?$AAA?$AAU?$AAL?$AAT?$AA?3?$AA?5?$AAp?$AAR@ 0015f008     rilmain.obj
 0002:0001e098       ??_C@_1FO@EGAEIKMN@?$AAI?$AAO?$AAC?$AAT?$AAL?$AA_?$AAR?$AAI?$AAL?$AA_?$AAS?$AAW?$AAI?$AA_?$AAS?$AAE?$AAT?$AA_?$AAN?$AAM?$AAE?$AAA?$AA_?$AAC?$AAO?$AAN?$AAF?$AAI?$AAG?$AA?3?$AA?5?$AAW@ 0015f098     rilmain.obj
 0002:0001e0f8       ??_C@_1GE@FHDNCBDH@?$AAI?$AAO?$AAC?$AAT?$AAL?$AA_?$AAR?$AAI?$AAL?$AA_?$AAS?$AAW?$AAI?$AA_?$AAS?$AAE?$AAT?$AA_?$AAN?$AAM?$AAE?$AAA?$AA_?$AAC?$AAO?$AAN?$AAF?$AAI?$AAG?$AA?3?$AA?5?$AAp@ 0015f0f8     rilmain.obj
 0002:0001e160       ??_C@_1FM@BKAPDJFF@?$AAI?$AAO?$AAC?$AAT?$AAL?$AA_?$AAR?$AAI?$AAL?$AA_?$AAS?$AAW?$AAI?$AA_?$AAS?$AAE?$AAT?$AA_?$AAN?$AAM?$AAE?$AAA?$AA_?$AAC?$AAO?$AAN?$AAF?$AAI?$AAG?$AA?3?$AA?5?$AAp@ 0015f160     rilmain.obj
 0002:0001e1c0       ??_C@_1IO@NIMPOHDJ@?$AAI?$AAO?$AAC?$AAT?$AAL?$AA_?$AAR?$AAI?$AAL?$AA_?$AAS?$AAW?$AAI?$AA_?$AAS?$AAE?$AAT?$AA_?$AAN?$AAM?$AAE?$AAA?$AA_?$AAC?$AAO?$AAN?$AAF?$AAI?$AAG?$AA?3?$AA?5?$AAp@ 0015f1c0     rilmain.obj
 0002:0001e250       ??_C@_1DG@LOKOLNHC@?$AAc?$AAa?$AAl?$AAl?$AA?5?$AAp?$AAR?$AAa?$AAd?$AAi?$AAo?$AA?9?$AA?$DO?$AAS?$AAe?$AAt?$AAN?$AAM?$AAE?$AAA?$AAC?$AAo?$AAn?$AAf?$AAi?$AAg?$AA?$AA@ 0015f250     rilmain.obj
 0002:0001e288       ??_C@_1DM@LLKCEOJJ@?$AAI?$AAO?$AAC?$AAT?$AAL?$AA_?$AAR?$AAI?$AAL?$AA_?$AAS?$AAW?$AAI?$AA_?$AAS?$AAE?$AAT?$AA_?$AAN?$AAM?$AAE?$AAA?$AA_?$AAC?$AAO?$AAN?$AAF?$AAI?$AAG?$AA?$AA@ 0015f288     rilmain.obj
 0002:0001e2c8       ??_C@_1NA@LAEKKEOI@?$AAA?$AAS?$AAS?$AAE?$AAR?$AAT?$AAI?$AAO?$AAN?$AA?5?$AAF?$AAA?$AAI?$AAL?$AAU?$AAR?$AAE?$AA?3?$AA?5?$AA?$DN?$AA?$DN?$AA?$DN?$AA?$DO?$AA?$CI?$AAd?$AAw?$AAL?$AAe?$AAn?$AAI?$AAn?$AA?5@ 0015f2c8     rilmain.obj
 0002:0001e398       ??_C@_1KI@PKMONBOL@?$AAF?$AAa?$AAi?$AAl?$AA?5?$AAH?$AAa?$AAn?$AAd?$AAl?$AAe?$AA?5?$AAI?$AAO?$AAC?$AAT?$AAL?$AA_?$AAP?$AAO?$AAW?$AAE?$AAR?$AA_?$AAC?$AAA?$AAP?$AAA?$AAB?$AAI?$AAL?$AAI@ 0015f398     rilmain.obj
 0002:0001e440       ??_C@_1GC@GGCPHFPH@?$AAR?$AAI?$AAL?$AA?5?$AAr?$AAe?$AAt?$AAu?$AAr?$AAn?$AAs?$AA?5?$AAD?$AAx?$AA?$DN?$AA0?$AAx?$AA?$CF?$AAx?$AA?5?$AAf?$AAo?$AAr?$AA?5?$AAI?$AAO?$AAC?$AAT?$AAL?$AA_?$AAP?$AAO@ 0015f440     rilmain.obj
 0002:0001e4a8       ??_C@_1JK@JCKCDBNF@?$AAF?$AAa?$AAi?$AAl?$AA?5?$AAH?$AAa?$AAn?$AAd?$AAl?$AAe?$AA?5?$AAI?$AAO?$AAC?$AAT?$AAL?$AA_?$AAP?$AAO?$AAW?$AAE?$AAR?$AA_?$AAG?$AAE?$AAT?$AA?0?$AA?5?$AAd?$AAw?$AAL@ 0015f4a8     rilmain.obj
 0002:0001e544       ??_C@_1DE@MJGKBKHM@?$AAR?$AAe?$AAc?$AAe?$AAi?$AAv?$AAi?$AAn?$AAg?$AA?5?$AAI?$AAO?$AAC?$AAT?$AAL?$AA_?$AAP?$AAO?$AAW?$AAE?$AAR?$AA_?$AAG?$AAE?$AAT?$AA?$AA@ 0015f544     rilmain.obj
 0002:0001e578       ??_C@_1IO@HIFDEBMH@?$AAF?$AAa?$AAi?$AAl?$AA?5?$AAH?$AAa?$AAn?$AAd?$AAl?$AAe?$AA?5?$AAD?$AA?$CF?$AAd?$AA?5?$AAs?$AAt?$AAa?$AAt?$AAe?$AA?0?$AA?5?$AAd?$AAw?$AAL?$AAe?$AAn?$AAO?$AAu?$AAt?$AA?5@ 0015f578     rilmain.obj
 0002:0001e608       ??_C@_1FG@FPNHLHNG@?$AAH?$AAa?$AAn?$AAd?$AAl?$AAe?$AAd?$AA?5?$AAD?$AA?$CF?$AAd?$AA?5?$AAs?$AAt?$AAa?$AAt?$AAe?$AA?4?$AA?5?$AAp?$AAr?$AAe?$AAv?$AAi?$AAo?$AAu?$AAs?$AAl?$AAy?$AA?5?$AAD?$AA?$CF@ 0015f608     rilmain.obj
 0002:0001e660       ??_C@_1HI@OOCJODDN@?$AAR?$AAI?$AAL?$AAD?$AAr?$AAv?$AA_?$AAA?$AAu?$AAx?$AAP?$AAo?$AAw?$AAe?$AAr?$AAS?$AAe?$AAt?$AA?$CB?$AA?5?$AAr?$AAe?$AAt?$AAu?$AAr?$AAn?$AA?5?$AAh?$AAr?$AA?5?$AA?$DN?$AA?5@ 0015f660     rilmain.obj
 0002:0001e6d8       ??_C@_1HI@GJIJMGFO@?$AAR?$AAI?$AAL?$AAD?$AAr?$AAv?$AA_?$AAA?$AAu?$AAx?$AAP?$AAo?$AAw?$AAe?$AAr?$AAS?$AAe?$AAt?$AA?$CB?$AA?5?$AAr?$AAe?$AAt?$AAu?$AAr?$AAn?$AA?5?$AAh?$AAr?$AA?5?$AA?$DN?$AA?5@ 0015f6d8     rilmain.obj
 0002:0001e750       ??_C@_1BE@PEIFHNGC@?$AAI?$AAO?$AAC?$AAo?$AAn?$AAt?$AAr?$AAo?$AAl?$AA?$AA@ 0015f750     rilmain.obj
 0002:0001e764       ??_C@_1BA@MOAPPNDD@?$AAR?$AAI?$AAL?$AAC?$AAD?$AAM?$AAA?$AA?$AA@ 0015f764     rilmain.obj
 0002:0001e778       ??_C@_1EO@KBDMLHFP@?$AAA?$AAS?$AAS?$AAE?$AAR?$AAT?$AAI?$AAO?$AAN?$AA?5?$AAF?$AAA?$AAI?$AAL?$AAU?$AAR?$AAE?$AA?3?$AA?5?$AA?$DN?$AA?$DN?$AA?$DN?$AA?$DO?$AAd?$AAw?$AAO?$AAp?$AAe?$AAn?$AAD?$AAa?$AAt@ 0015f778     rilmain.obj
 0002:0001e7c8       ??_C@_1FG@IEPONGLA@?$AAC?$AAl?$AAe?$AAa?$AAr?$AAC?$AAm?$AAd?$AAH?$AAa?$AAn?$AAd?$AAl?$AAe?$AA?3?$AA?3?$AA?5?$AAE?$AAR?$AAR?$AAO?$AAR?$AA?4?$AA?4?$AA?4?$AA?4?$AAd?$AAw?$AAD?$AAu?$AAm?$AAm@ 0015f7c8     rilmain.obj
 0002:0001e858       ??_C@_1GK@EJAKHODL@?$AAA?$AAS?$AAS?$AAE?$AAR?$AAT?$AAI?$AAO?$AAN?$AA?5?$AAF?$AAA?$AAI?$AAL?$AAU?$AAR?$AAE?$AA?3?$AA?5?$AA?$DN?$AA?$DN?$AA?$DN?$AA?$DO?$AAp?$AAI?$AAn?$AAs?$AAt?$AAH?$AAa?$AAn?$AAd@ 0015f858     rilmain.obj
 0002:0001e8c8       ??_C@_1FK@PNAJHECC@?$AAG?$AAe?$AAt?$AAP?$AAr?$AAo?$AAc?$AAA?$AAd?$AAd?$AAr?$AAe?$AAs?$AAs?$AA?5?$AAf?$AAa?$AAi?$AAl?$AAe?$AAd?$AA?5?$AAf?$AAo?$AAr?$AA?3?$AA?5?$AA?$CF?$AAs?$AA?5?$AAR?$AAe@ 0015f8c8     SDK7Wrapper.obj
 0002:0001eae8       ??_C@_1BI@PMAAAENI@?$AA?4?$AA?2?$AAs?$AAe?$AAc?$AAu?$AAr?$AA?4?$AAc?$AAp?$AAp?$AA?$AA@ 0015fae8     secur.obj
 0002:0001eb00       ??_C@_1KA@CEJDPJIK@?$AAF?$AAa?$AAi?$AAl?$AAe?$AAd?$AA?5?$AAt?$AAo?$AA?5?$AAg?$AAe?$AAt?$AA?5?$AAt?$AAh?$AAe?$AA?5?$AAL?$AAo?$AAc?$AAk?$AAe?$AAd?$AA?5?$AAS?$AAt?$AAa?$AAt?$AAe?$AA?5?$AAf@ 0015fb00     secur.obj
 0002:0001eba0       ??_C@_1FI@ONBAEPFP@?$AAA?$AAS?$AAS?$AAE?$AAR?$AAT?$AAI?$AAO?$AAN?$AA?5?$AAF?$AAA?$AAI?$AAL?$AAU?$AAR?$AAE?$AA?3?$AA?5?$AA?$DN?$AA?$DN?$AA?$DN?$AA?$DO?$AAN?$AAU?$AAL?$AAL?$AA?5?$AA?$CB?$AA?$DN?$AA?5?$AAl@ 0015fba0     secur.obj
 0002:0001ebf8       ??_C@_1HA@OPIOGMHB@?$AAS?$AAw?$AAi?$AAS?$AAe?$AAt?$AAS?$AAi?$AAm?$AAV?$AAe?$AAr?$AAi?$AAf?$AAy?$AAG?$AAo?$AAb?$AAi?$AA?5?$AAr?$AAe?$AAt?$AAu?$AAr?$AAn?$AAe?$AAd?$AA?5?$AAe?$AAr?$AAr@ 0015fbf8     secur.obj
 0002:0001ec68       ??_C@_1MK@EGFAJAEG@?$AAA?$AAS?$AAS?$AAE?$AAR?$AAT?$AAI?$AAO?$AAN?$AA?5?$AAF?$AAA?$AAI?$AAL?$AAU?$AAR?$AAE?$AA?3?$AA?5?$AA?$DN?$AA?$DN?$AA?$DN?$AA?$DO?$AAR?$AAI?$AAL?$AA_?$AAL?$AAO?$AAC?$AAK?$AAF@ 0015fc68     secur.obj
 0002:0001ed38       ??_C@_1FO@DLCHJPDI@?$AAA?$AAS?$AAS?$AAE?$AAR?$AAT?$AAI?$AAO?$AAN?$AA?5?$AAF?$AAA?$AAI?$AAL?$AAU?$AAR?$AAE?$AA?3?$AA?5?$AA?$DN?$AA?$DN?$AA?$DN?$AA?$DO?$AAN?$AAU?$AAL?$AAL?$AA?5?$AA?$CB?$AA?$DN?$AA?5?$AAl@ 0015fd38     secur.obj
 0002:0001ed98       ??_C@_1FO@FLAGFODA@?$AAA?$AAS?$AAS?$AAE?$AAR?$AAT?$AAI?$AAO?$AAN?$AA?5?$AAF?$AAA?$AAI?$AAL?$AAU?$AAR?$AAE?$AA?3?$AA?5?$AA?$DN?$AA?$DN?$AA?$DN?$AA?$DO?$AAN?$AAU?$AAL?$AAL?$AA?5?$AA?$CB?$AA?$DN?$AA?5?$AAl@ 0015fd98     secur.obj
 0002:0001edf8       ??_C@_1IK@DKNNDIIO@?$AAA?$AAS?$AAS?$AAE?$AAR?$AAT?$AAI?$AAO?$AAN?$AA?5?$AAF?$AAA?$AAI?$AAL?$AAU?$AAR?$AAE?$AA?3?$AA?5?$AA?$DN?$AA?$DN?$AA?$DN?$AA?$DO?$AAd?$AAw?$AAF?$AAa?$AAc?$AAi?$AAl?$AAi?$AAt@ 0015fdf8     secur.obj
 0002:0001ee88       ??_C@_1HE@MOEBJCH@?$AAS?$AAw?$AAi?$AAS?$AAe?$AAt?$AAS?$AAi?$AAm?$AAP?$AAa?$AAs?$AAs?$AAw?$AAo?$AAr?$AAd?$AAG?$AAo?$AAb?$AAi?$AA?5?$AAr?$AAe?$AAt?$AAu?$AAr?$AAn?$AAe?$AAd?$AA?5?$AAe@ 0015fe88     secur.obj
 0002:0001ef00       ??_C@_1GM@JGOLOLKI@?$AAS?$AAw?$AAi?$AAS?$AAe?$AAt?$AAS?$AAi?$AAm?$AAL?$AAo?$AAc?$AAk?$AAG?$AAo?$AAb?$AAi?$AA?5?$AAr?$AAe?$AAt?$AAu?$AAr?$AAn?$AAe?$AAd?$AA?5?$AAe?$AAr?$AAr?$AAo?$AAr@ 0015ff00     secur.obj
 0002:0001ef70       ??_C@_1EM@NMNGJAHL@?$AAS?$AAw?$AAi?$AAG?$AAe?$AAt?$AAS?$AAi?$AAm?$AAL?$AAo?$AAc?$AAk?$AAG?$AAo?$AAb?$AAi?$AA?5?$AAr?$AAe?$AAt?$AAu?$AAr?$AAn?$AAe?$AAd?$AA?5?$AAe?$AAr?$AAr?$AAo?$AAr@ 0015ff70     secur.obj
 0002:0001efc0       ??_C@_1EG@BIPCONJJ@?$AAm?$AAp?$AAF?$AAn?$AAS?$AAw?$AAi?$AAG?$AAe?$AAt?$AAG?$AAs?$AAm?$AAI?$AAM?$AAS?$AAI?$AA?5?$AAi?$AAs?$AA?5?$AAn?$AAo?$AAt?$AA?5?$AAs?$AAu?$AAp?$AAp?$AAo?$AAr?$AAt@ 0015ffc0     secur.obj
 0002:0001f008       ??_C@_06OLICBFOI@?$CFd?$CFd?$CFs?$AA@ 00160008     secur.obj
 0002:0001f010       ??_C@_1EO@INKOBDDP@?$AAS?$AAw?$AAi?$AAG?$AAe?$AAt?$AAE?$AAS?$AAN?$AAG?$AAo?$AAb?$AAi?$AA?$CI?$AA?$CJ?$AA?4?$AA?5?$AAE?$AAS?$AAN?$AA?5?$AA?$DN?$AA?5?$AA?$CF?$AAs?$AA?5?$AA?5?$AAs?$AAt?$AAr?$AAl?$AAe@ 00160010     secur.obj
 0002:0001f060       ??_C@_02DKCKIIND@?$CFs?$AA@ 00160060     secur.obj
 0002:0001f068       ??_C@_1HG@NNPBJGOB@?$AAA?$AAS?$AAS?$AAE?$AAR?$AAT?$AAI?$AAO?$AAN?$AA?5?$AAF?$AAA?$AAI?$AAL?$AAU?$AAR?$AAE?$AA?3?$AA?5?$AA?$DN?$AA?$DN?$AA?$DN?$AA?$DO?$AAd?$AAw?$AAT?$AAy?$AAp?$AAe?$AA?5?$AA?$CG?$AA?$CG@ 00160068     secur.obj
 0002:0001f0e0       ??_C@_1HC@FFOPKGLN@?$AAR?$AAI?$AAL?$AAD?$AAr?$AAv?$AA_?$AAS?$AAe?$AAt?$AAC?$AAa?$AAl?$AAl?$AAB?$AAa?$AAr?$AAr?$AAi?$AAn?$AAg?$AAS?$AAt?$AAa?$AAt?$AAu?$AAs?$AA?5?$AAt?$AAy?$AAp?$AAe@ 001600e0     secur.obj
 0002:0001f158       ??_C@_1MO@NHPKGFJF@?$AAA?$AAS?$AAS?$AAE?$AAR?$AAT?$AAI?$AAO?$AAN?$AA?5?$AAF?$AAA?$AAI?$AAL?$AAU?$AAR?$AAE?$AA?3?$AA?5?$AA?$DN?$AA?$DN?$AA?$DN?$AA?$DO?$AAR?$AAI?$AAL?$AA_?$AAB?$AAA?$AAR?$AAR?$AAI@ 00160158     secur.obj
 0002:0001f228       ??_C@_1CI@FEKDHFMO@?$AAQ?$AAM?$AAI?$AA?5?$AAr?$AAe?$AAt?$AAu?$AAr?$AAn?$AA?5?$AAe?$AAr?$AAr?$AAo?$AAr?$AA?5?$AA?$CF?$AAd?$AA?$AA@ 00160228     secur.obj
 0002:0001f250       ??_C@_1HI@EINFMDIC@?$AAG?$AAe?$AAt?$AAC?$AAa?$AAl?$AAl?$AAB?$AAa?$AAr?$AAr?$AAi?$AAn?$AAg?$AAS?$AAt?$AAa?$AAt?$AAu?$AAs?$AA?3?$AA?5?$AAB?$AAa?$AAr?$AAr?$AAi?$AAn?$AAg?$AA?5?$AAt?$AAy@ 00160250     secur.obj
 0002:0001f2c8       ??_C@_1DK@BJDKPNDI@?$AAC?$AAR?$AAa?$AAd?$AAi?$AAo?$AA?3?$AA?3?$AAS?$AAe?$AAt?$AAC?$AAa?$AAl?$AAl?$AAB?$AAa?$AAr?$AAr?$AAi?$AAn?$AAg?$AAS?$AAt?$AAa?$AAt?$AAu?$AAs?$AA?$AA@ 001602c8     secur.obj
 0002:0001f308       ??_C@_1HI@OFAPDAD@?$AAC?$AAR?$AAa?$AAd?$AAi?$AAo?$AA?3?$AA?3?$AAS?$AAe?$AAt?$AAC?$AAa?$AAl?$AAl?$AAB?$AAa?$AAr?$AAr?$AAi?$AAn?$AAg?$AAS?$AAt?$AAa?$AAt?$AAu?$AAs?$AA?5?$AAr?$AAe?$AAa@ 00160308     secur.obj
 0002:0001f380       ??_C@_1CC@JJFHMJLO@?$AA?5?$AAQ?$AAM?$AAI?$AA?5?$AAf?$AAa?$AAi?$AAl?$AAe?$AAd?$AA?5?$AA?$CF?$AAd?$AA?$CB?$AA?$CB?$AA?$AA@ 00160380     secur.obj
 0002:0001f3a8       ??_C@_1FI@EBGFICMJ@?$AAC?$AAR?$AAa?$AAd?$AAi?$AAo?$AA?3?$AA?3?$AAC?$AAh?$AAa?$AAn?$AAg?$AAe?$AAC?$AAa?$AAl?$AAl?$AAB?$AAa?$AAr?$AAr?$AAi?$AAn?$AAg?$AAP?$AAa?$AAs?$AAs?$AAw?$AAo?$AAr@ 001603a8     secur.obj
 0002:0001f400       ??_C@_0LB@CPGKIIJP@000000000111E180604028180E888462@ 00160400     smscb.obj
 0002:0001f520       ??_C@_1EC@BDIEMBDJ@?$AAP?$AAa?$AAr?$AAs?$AAe?$AAC?$AAe?$AAl?$AAl?$AAB?$AAr?$AAo?$AAa?$AAd?$AAc?$AAa?$AAs?$AAt?$AAM?$AAe?$AAs?$AAs?$AAa?$AAg?$AAe?$AA?5?$AAm?$AAe?$AAm?$AAs?$AAe?$AAt@ 00160520     smscb.obj
 0002:0001f564       ??_C@_1BI@JPBOAOGM@?$AA?4?$AA?2?$AAs?$AAm?$AAs?$AAc?$AAb?$AA?4?$AAc?$AAp?$AAp?$AA?$AA@ 00160564     smscb.obj
 0002:0001f57c       ??_C@_1BK@MNMIPOFN@?$AAa?$AAf?$AAt?$AAe?$AAr?$AA?5?$AAm?$AAe?$AAm?$AAs?$AAe?$AAt?$AA?$AA@ 0016057c     smscb.obj
 0002:0001f614       ??_C@_1BK@HMNBBHPE@?$AA?4?$AA?2?$AAs?$AAu?$AAp?$AAs?$AAv?$AAc?$AA?4?$AAc?$AAp?$AAp?$AA?$AA@ 00160614     supsvc.obj
 0002:0001f630       ??_C@_1DG@OHLCIDDE@?$AAR?$AAI?$AAL?$AAD?$AAr?$AAv?$AA_?$AAG?$AAe?$AAt?$AAC?$AAa?$AAl?$AAl?$AAe?$AAr?$AAI?$AAd?$AAS?$AAe?$AAt?$AAt?$AAi?$AAn?$AAg?$AAs?$AA?$AA@ 00160630     supsvc.obj
 0002:0001f668       ??_C@_1DG@MBOKFMKG@?$AAR?$AAI?$AAL?$AAD?$AAr?$AAv?$AA_?$AAG?$AAe?$AAt?$AAD?$AAi?$AAa?$AAl?$AAe?$AAd?$AAI?$AAd?$AAS?$AAe?$AAt?$AAt?$AAi?$AAn?$AAg?$AAs?$AA?$AA@ 00160668     supsvc.obj
 0002:0001f6a0       ??_C@_1DC@BNOMLNLB@?$AAR?$AAI?$AAL?$AAD?$AAr?$AAv?$AA_?$AAS?$AAe?$AAt?$AAD?$AAi?$AAa?$AAl?$AAe?$AAd?$AAI?$AAd?$AAS?$AAt?$AAa?$AAt?$AAu?$AAs?$AA?$AA@ 001606a0     supsvc.obj
 0002:0001f6d8       ??_C@_1GM@CNNAFOGE@?$AAR?$AAI?$AAL?$AAD?$AAr?$AAv?$AA_?$AAG?$AAe?$AAt?$AAC?$AAa?$AAl?$AAl?$AAF?$AAo?$AAr?$AAw?$AAa?$AAr?$AAd?$AAi?$AAn?$AAg?$AAS?$AAe?$AAt?$AAt?$AAi?$AAn?$AAg?$AAs@ 001606d8     supsvc.obj
 0002:0001f748       ??_C@_1FM@PDDHEPKG@?$AAR?$AAI?$AAL?$AAD?$AAr?$AAv?$AA_?$AAA?$AAd?$AAd?$AAC?$AAa?$AAl?$AAl?$AAF?$AAo?$AAr?$AAw?$AAa?$AAr?$AAd?$AAi?$AAn?$AAg?$AA?3?$AA?5?$AAr?$AAe?$AAa?$AAs?$AAo?$AAn@ 00160748     supsvc.obj
 0002:0001f7a8       ??_C@_1GC@LDIBELGO@?$AAR?$AAI?$AAL?$AAD?$AAr?$AAv?$AA_?$AAR?$AAe?$AAm?$AAo?$AAv?$AAe?$AAC?$AAa?$AAl?$AAl?$AAF?$AAo?$AAr?$AAw?$AAa?$AAr?$AAd?$AAi?$AAn?$AAg?$AA?3?$AA?5?$AAr?$AAe?$AAa@ 001607a8     supsvc.obj
 0002:0001f810       ??_C@_1HO@MPIIMJAB@?$AAR?$AAI?$AAL?$AAD?$AAr?$AAv?$AA_?$AAS?$AAe?$AAt?$AAC?$AAa?$AAl?$AAl?$AAF?$AAo?$AAr?$AAw?$AAa?$AAr?$AAd?$AAi?$AAn?$AAg?$AAS?$AAt?$AAa?$AAt?$AAu?$AAs?$AA?3?$AA?5@ 00160810     supsvc.obj
 0002:0001f890       ??_C@_1DO@NBCBADJ@?$AAR?$AAI?$AAL?$AAD?$AAr?$AAv?$AA_?$AAS?$AAe?$AAt?$AAC?$AAa?$AAl?$AAl?$AAF?$AAo?$AAr?$AAw?$AAa?$AAr?$AAd?$AAi?$AAn?$AAg?$AAS?$AAt?$AAa?$AAt?$AAu?$AAs?$AA?$AA@ 00160890     supsvc.obj
 0002:0001f8d0       ??_C@_1FA@DBGDGNAM@?$AAR?$AAI?$AAL?$AAD?$AAr?$AAv?$AA_?$AAG?$AAe?$AAt?$AAC?$AAa?$AAl?$AAl?$AAW?$AAa?$AAi?$AAt?$AAi?$AAn?$AAg?$AAS?$AAe?$AAt?$AAt?$AAi?$AAn?$AAg?$AAs?$AA?3?$AA?5?$AAc@ 001608d0     supsvc.obj
 0002:0001f920       ??_C@_1DM@MNPFKHCH@?$AAR?$AAI?$AAL?$AAD?$AAr?$AAv?$AA_?$AAG?$AAe?$AAt?$AAC?$AAa?$AAl?$AAl?$AAW?$AAa?$AAi?$AAt?$AAi?$AAn?$AAg?$AAS?$AAe?$AAt?$AAt?$AAi?$AAn?$AAg?$AAs?$AA?$AA@ 00160920     supsvc.obj
 0002:0001f960       ??_C@_1GO@KKFBHMHH@?$AAR?$AAI?$AAL?$AAD?$AAr?$AAv?$AA_?$AAS?$AAe?$AAt?$AAC?$AAa?$AAl?$AAl?$AAW?$AAa?$AAi?$AAt?$AAi?$AAn?$AAg?$AAS?$AAt?$AAa?$AAt?$AAu?$AAs?$AA?3?$AA?5?$AAs?$AAe?$AAt@ 00160960     supsvc.obj
 0002:0001f9d0       ??_C@_1HA@BGCPCPNE@?$AAR?$AAI?$AAL?$AAD?$AAr?$AAv?$AA_?$AAS?$AAe?$AAt?$AAC?$AAa?$AAl?$AAl?$AAW?$AAa?$AAi?$AAt?$AAi?$AAn?$AAg?$AAS?$AAt?$AAa?$AAt?$AAu?$AAs?$AA?3?$AA?5?$AAE?$AAr?$AAr@ 001609d0     supsvc.obj
 0002:0001fa40       ??_C@_1LC@MLCKOMKD@?$AAR?$AAI?$AAL?$AAD?$AAr?$AAv?$AA_?$AAS?$AAe?$AAt?$AAC?$AAa?$AAl?$AAl?$AAW?$AAa?$AAi?$AAt?$AAi?$AAn?$AAg?$AAS?$AAt?$AAa?$AAt?$AAu?$AAs?$AA?3?$AA?5?$AAn?$AAo?$AAO@ 00160a40     supsvc.obj
 0002:0001faf8       ??_C@_1FM@DLABNOGL@?$AAR?$AAI?$AAL?$AAD?$AAr?$AAv?$AA_?$AAS?$AAe?$AAt?$AAC?$AAa?$AAl?$AAl?$AAW?$AAa?$AAi?$AAt?$AAi?$AAn?$AAg?$AAS?$AAt?$AAa?$AAt?$AAu?$AAs?$AA?3?$AA?5?$AAp?$AAR?$AAi@ 00160af8     supsvc.obj
 0002:0001fb58       ??_C@_1FE@PPINNLOE@?$AAR?$AAI?$AAL?$AAD?$AAr?$AAv?$AA_?$AAS?$AAe?$AAt?$AAC?$AAa?$AAl?$AAl?$AAW?$AAa?$AAi?$AAt?$AAi?$AAn?$AAg?$AAS?$AAt?$AAa?$AAt?$AAu?$AAs?$AA?3?$AA?5?$AAp?$AAR?$AAa@ 00160b58     supsvc.obj
 0002:0001fbb0       ??_C@_1GC@EGGOHAMN@?$AAR?$AAI?$AAL?$AAD?$AAr?$AAv?$AA_?$AAS?$AAe?$AAt?$AAC?$AAa?$AAl?$AAl?$AAW?$AAa?$AAi?$AAt?$AAi?$AAn?$AAg?$AAS?$AAt?$AAa?$AAt?$AAu?$AAs?$AA?3?$AA?5?$AAc?$AAl?$AAa@ 00160bb0     supsvc.obj
 0002:0001fc14       ??_C@_1DI@BNJCCBAJ@?$AAR?$AAI?$AAL?$AAD?$AAr?$AAv?$AA_?$AAS?$AAe?$AAt?$AAC?$AAa?$AAl?$AAl?$AAW?$AAa?$AAi?$AAt?$AAi?$AAn?$AAg?$AAS?$AAt?$AAa?$AAt?$AAu?$AAs?$AA?$AA@ 00160c14     supsvc.obj
 0002:0001fc4c       ??_C@_1DE@DGFBFCFA@?$AAR?$AAI?$AAL?$AAD?$AAr?$AAv?$AA_?$AAS?$AAe?$AAn?$AAd?$AAS?$AAu?$AAp?$AAS?$AAe?$AAr?$AAv?$AAi?$AAc?$AAe?$AAD?$AAa?$AAt?$AAa?$AA?$AA@ 00160c4c     supsvc.obj
 0002:0001fc80       ??_C@_1EG@PMJNBJJG@?$AAA?$AAS?$AAS?$AAE?$AAR?$AAT?$AAI?$AAO?$AAN?$AA?5?$AAF?$AAA?$AAI?$AAL?$AAU?$AAR?$AAE?$AA?3?$AA?5?$AA?$DN?$AA?$DN?$AA?$DN?$AA?$DO?$AA0?$AA?5?$AA?$CB?$AA?$DN?$AA?5?$AAd?$AAw?$AAS?$AAi@ 00160c80     supsvc.obj
 0002:0001fcc8       ??_C@_1EO@FIBAKOGM@?$AAA?$AAS?$AAS?$AAE?$AAR?$AAT?$AAI?$AAO?$AAN?$AA?5?$AAF?$AAA?$AAI?$AAL?$AAU?$AAR?$AAE?$AA?3?$AA?5?$AA?$DN?$AA?$DN?$AA?$DN?$AA?$DO?$AAN?$AAU?$AAL?$AAL?$AA?5?$AA?$CB?$AA?$DN?$AA?5?$AAl@ 00160cc8     supsvc.obj
 0002:0001fd18       ??_C@_1DK@HFJPDDO@?$AAR?$AAI?$AAL?$AAD?$AAr?$AAv?$AA_?$AAS?$AAe?$AAn?$AAd?$AAS?$AAu?$AAp?$AAS?$AAe?$AAr?$AAv?$AAi?$AAc?$AAe?$AAD?$AAa?$AAt?$AAa?$AA?5?$AA?$CF?$AAd?$AA?$AA@ 00160d18     supsvc.obj
 0002:0001fd58       ??_C@_1EG@NGCBEONB@?$AAR?$AAI?$AAL?$AAD?$AAr?$AAv?$AA_?$AAC?$AAa?$AAn?$AAc?$AAe?$AAl?$AAS?$AAu?$AAp?$AAS?$AAe?$AAr?$AAv?$AAi?$AAc?$AAe?$AAD?$AAa?$AAt?$AAa?$AAS?$AAe?$AAs?$AAs?$AAi@ 00160d58     supsvc.obj
 0002:0001fda0       ??_C@_1DA@LBMENBGF@?$AAm?$AAp?$AAF?$AAn?$AAS?$AAw?$AAi?$AAA?$AAT?$AAG?$AAe?$AAt?$AAC?$AAL?$AAI?$AAP?$AA?5?$AAf?$AAa?$AAi?$AAl?$AAe?$AAd?$AA?$AA@ 00160da0     supsvc.obj
 0002:0001fdd0       ??_C@_1DI@LLELBFG@?$AAC?$AAR?$AAa?$AAd?$AAi?$AAo?$AA?3?$AA?3?$AAG?$AAe?$AAt?$AAC?$AAa?$AAl?$AAl?$AAe?$AAr?$AAI?$AAd?$AAS?$AAe?$AAt?$AAt?$AAi?$AAn?$AAg?$AAs?$AA?$AA@ 00160dd0     supsvc.obj
 0002:0001fe08       ??_C@_1DK@GBMCOBHH@?$AAC?$AAR?$AAa?$AAd?$AAi?$AAo?$AA?3?$AA?3?$AAS?$AAe?$AAt?$AAC?$AAa?$AAl?$AAl?$AAe?$AAr?$AAI?$AAd?$AAS?$AAt?$AAa?$AAt?$AAu?$AAs?$AA?5?$AA?$CF?$AAd?$AA?$AA@ 00160e08     supsvc.obj
 0002:0001fe48       ??_C@_1GE@FLBEKFPC@?$AAC?$AAR?$AAa?$AAd?$AAi?$AAo?$AA?3?$AA?3?$AAG?$AAe?$AAt?$AAH?$AAi?$AAd?$AAe?$AAI?$AAd?$AAS?$AAe?$AAt?$AAt?$AAi?$AAn?$AAg?$AAs?$AA?5?$AAS?$AAe?$AAt?$AAR?$AAe?$AAg@ 00160e48     supsvc.obj
 0002:0001feb0       ??_C@_1HA@GHIPONMM@?$AAG?$AAe?$AAt?$AAH?$AAi?$AAd?$AAe?$AAI?$AAd?$AAS?$AAe?$AAt?$AAt?$AAi?$AAn?$AAg?$AAs?$AA?3?$AA?5?$AAs?$AAt?$AAa?$AAt?$AAu?$AAs?$AA?5?$AA?$CF?$AAd?$AA?0?$AA?5?$AAp?$AAr@ 00160eb0     supsvc.obj
 0002:0001ff20       ??_C@_1DA@LEBALKOG@?$AAm?$AAp?$AAF?$AAn?$AAS?$AAw?$AAi?$AAA?$AAT?$AAG?$AAe?$AAt?$AAC?$AAL?$AAI?$AAR?$AA?5?$AAf?$AAa?$AAi?$AAl?$AAe?$AAd?$AA?$AA@ 00160f20     supsvc.obj
 0002:0001ff50       ??_C@_1DE@OFABBHEF@?$AAC?$AAR?$AAa?$AAd?$AAi?$AAo?$AA?3?$AA?3?$AAG?$AAe?$AAt?$AAH?$AAi?$AAd?$AAe?$AAI?$AAd?$AAS?$AAe?$AAt?$AAt?$AAi?$AAn?$AAg?$AAs?$AA?$AA@ 00160f50     supsvc.obj
 0002:0001ff88       ??_C@_1GA@BLNFEHEO@?$AAC?$AAR?$AAa?$AAd?$AAi?$AAo?$AA?3?$AA?3?$AAS?$AAe?$AAt?$AAH?$AAi?$AAd?$AAe?$AAI?$AAd?$AAS?$AAt?$AAa?$AAt?$AAu?$AAs?$AA?5?$AAS?$AAe?$AAt?$AAR?$AAe?$AAg?$AAi?$AAs@ 00160f88     supsvc.obj
 0002:0001ffe8       ??_C@_1DA@LKJEOPHL@?$AAC?$AAR?$AAa?$AAd?$AAi?$AAo?$AA?3?$AA?3?$AAS?$AAe?$AAt?$AAH?$AAi?$AAd?$AAe?$AAI?$AAd?$AAS?$AAt?$AAa?$AAt?$AAu?$AAs?$AA?$AA@ 00160fe8     supsvc.obj
 0002:00020018       ??_C@_1DG@CLNJDGLO@?$AAC?$AAR?$AAa?$AAd?$AAi?$AAo?$AA?3?$AA?3?$AAS?$AAe?$AAt?$AAH?$AAi?$AAd?$AAe?$AAI?$AAd?$AAS?$AAt?$AAa?$AAt?$AAu?$AAs?$AA?5?$AA?$CF?$AAd?$AA?$AA@ 00161018     supsvc.obj
 0002:00020050       ??_C@_1DA@KDDGKMDK@?$AAm?$AAp?$AAF?$AAn?$AAS?$AAw?$AAi?$AAA?$AAT?$AAG?$AAe?$AAt?$AAC?$AAO?$AAL?$AAP?$AA?5?$AAf?$AAa?$AAi?$AAl?$AAe?$AAd?$AA?$AA@ 00161050     supsvc.obj
 0002:00020080       ??_C@_1DI@CNOMGOME@?$AAC?$AAR?$AAa?$AAd?$AAi?$AAo?$AA?3?$AA?3?$AAG?$AAe?$AAt?$AAD?$AAi?$AAa?$AAl?$AAe?$AAd?$AAI?$AAd?$AAS?$AAe?$AAt?$AAt?$AAi?$AAn?$AAg?$AAs?$AA?$AA@ 00161080     supsvc.obj
 0002:000200b8       ??_C@_1HK@MCACFCKB@?$AAm?$AA_?$AAp?$AAS?$AAD?$AAK?$AAR?$AAI?$AAL?$AA?4?$AAG?$AAe?$AAt?$AAC?$AAa?$AAl?$AAl?$AAF?$AAo?$AAr?$AAw?$AAa?$AAr?$AAd?$AAi?$AAn?$AAg?$AA?5?$AAg?$AAi?$AAv?$AAi@ 001610b8     supsvc.obj
 0002:00020138       ??_C@_1IM@MOIMFPPP@?$AAm?$AA_?$AAp?$AAS?$AAD?$AAK?$AAR?$AAI?$AAL?$AA?4?$AAG?$AAe?$AAt?$AAC?$AAa?$AAl?$AAl?$AAF?$AAo?$AAr?$AAw?$AAa?$AAr?$AAd?$AAi?$AAn?$AAg?$AA?5?$AAr?$AAe?$AAa?$AAs@ 00161138     supsvc.obj
 0002:000201c8       ??_C@_1HC@DJCBLJKO@?$AAm?$AA_?$AAp?$AAS?$AAD?$AAK?$AAR?$AAI?$AAL?$AA?4?$AAG?$AAe?$AAt?$AAC?$AAa?$AAl?$AAl?$AAF?$AAo?$AAr?$AAw?$AAa?$AAr?$AAd?$AAi?$AAn?$AAg?$AA?5?$AAr?$AAe?$AAt?$AAr@ 001611c8     supsvc.obj
 0002:00020240       ??_C@_1FM@PGJNFKNN@?$AAG?$AAe?$AAt?$AAR?$AAe?$AAg?$AAi?$AAs?$AAt?$AAr?$AAy?$AAD?$AAW?$AAO?$AAR?$AAD?$AA?5?$AAS?$AAU?$AAP?$AAS?$AAV?$AAC?$AA_?$AAC?$AAA?$AAL?$AAL?$AA_?$AAF?$AAW?$AAD@ 00161240     supsvc.obj
 0002:000202a0       ??_C@_1EE@LIACLLCF@?$AAC?$AAR?$AAa?$AAd?$AAi?$AAo?$AA?3?$AA?3?$AAG?$AAe?$AAt?$AAC?$AAa?$AAl?$AAl?$AAF?$AAo?$AAr?$AAw?$AAa?$AAr?$AAd?$AAi?$AAn?$AAg?$AAS?$AAe?$AAt?$AAt?$AAi?$AAn?$AAg@ 001612a0     supsvc.obj
 0002:000202e8       ??_C@_1IE@MJFDKKHF@?$AAC?$AAR?$AAa?$AAd?$AAi?$AAo?$AA?3?$AA?3?$AAG?$AAe?$AAt?$AAC?$AAa?$AAl?$AAl?$AAF?$AAo?$AAr?$AAw?$AAa?$AAr?$AAd?$AAi?$AAn?$AAg?$AAS?$AAe?$AAt?$AAt?$AAi?$AAn?$AAg@ 001612e8     supsvc.obj
 0002:0002036c       ??_C@_1BK@PIOGDDKG@?$AAC?$AAa?$AAl?$AAl?$AAF?$AAw?$AAd?$AAR?$AAe?$AAt?$AAr?$AAy?$AA?$AA@ 0016136c     supsvc.obj
 0002:00020388       ??_C@_1GC@CODCKICN@?$AAC?$AAR?$AAa?$AAd?$AAi?$AAo?$AA?3?$AA?3?$AAA?$AAd?$AAd?$AAC?$AAa?$AAl?$AAl?$AAF?$AAo?$AAr?$AAw?$AAa?$AAr?$AAd?$AAi?$AAn?$AAg?$AA?3?$AA?5?$AAr?$AAe?$AAq?$AA?5?$AA?9@ 00161388     supsvc.obj
 0002:000203f0       ??_C@_1LO@FHJCNDFC@?$AAC?$AAR?$AAa?$AAd?$AAi?$AAo?$AA?3?$AA?3?$AAA?$AAd?$AAd?$AAC?$AAa?$AAl?$AAl?$AAF?$AAo?$AAr?$AAw?$AAa?$AAr?$AAd?$AAi?$AAn?$AAg?$AA?3?$AA?5?$AAr?$AAe?$AAq?$AA?5?$AA?9@ 001613f0     supsvc.obj
 0002:000204b0       ??_C@_1KG@PJCMKBBJ@?$AAC?$AAR?$AAa?$AAd?$AAi?$AAo?$AA?3?$AA?3?$AAA?$AAd?$AAd?$AAC?$AAa?$AAl?$AAl?$AAF?$AAo?$AAr?$AAw?$AAa?$AAr?$AAd?$AAi?$AAn?$AAg?$AA?3?$AA?5?$AAr?$AAe?$AAq?$AA?5?$AA?9@ 001614b0     supsvc.obj
 0002:00020558       ??_C@_1EE@POBEGNPJ@?$AAC?$AAR?$AAa?$AAd?$AAi?$AAo?$AA?3?$AA?3?$AAA?$AAd?$AAd?$AAC?$AAa?$AAl?$AAl?$AAF?$AAo?$AAr?$AAw?$AAa?$AAr?$AAd?$AAi?$AAn?$AAg?$AAS?$AAe?$AAt?$AAt?$AAi?$AAn?$AAg@ 00161558     supsvc.obj
 0002:000205a0       ??_C@_1HE@NJNHEGM@?$AAC?$AAR?$AAa?$AAd?$AAi?$AAo?$AA?3?$AA?3?$AAA?$AAd?$AAd?$AAC?$AAa?$AAl?$AAl?$AAF?$AAo?$AAr?$AAw?$AAa?$AAr?$AAd?$AAi?$AAn?$AAg?$AA?3?$AA?5?$AAr?$AAe?$AAa?$AAs?$AAo@ 001615a0     supsvc.obj
 0002:00020618       ??_C@_1LO@MAHIOJDL@?$AAC?$AAR?$AAa?$AAd?$AAi?$AAo?$AA?3?$AA?3?$AAS?$AAe?$AAt?$AAC?$AAa?$AAl?$AAl?$AAF?$AAo?$AAr?$AAw?$AAa?$AAr?$AAd?$AAi?$AAn?$AAg?$AA?3?$AA?5?$AAr?$AAe?$AAq?$AA?5?$AA?9@ 00161618     supsvc.obj
 0002:000206d8       ??_C@_1KG@PADLPMFK@?$AAC?$AAR?$AAa?$AAd?$AAi?$AAo?$AA?3?$AA?3?$AAS?$AAe?$AAt?$AAC?$AAa?$AAl?$AAl?$AAF?$AAo?$AAr?$AAw?$AAa?$AAr?$AAd?$AAi?$AAn?$AAg?$AA?3?$AA?5?$AAr?$AAe?$AAq?$AA?5?$AA?9@ 001616d8     supsvc.obj
 0002:00020780       ??_C@_1JC@MPNFMNGN@?$AAC?$AAR?$AAa?$AAd?$AAi?$AAo?$AA?3?$AA?3?$AAS?$AAe?$AAt?$AAC?$AAa?$AAl?$AAl?$AAF?$AAo?$AAr?$AAw?$AAa?$AAr?$AAd?$AAi?$AAn?$AAg?$AA?3?$AA?5?$AAI?$AAn?$AAv?$AAa?$AAl@ 00161780     supsvc.obj
 0002:00020814       ??_C@_1DE@HMHBPIAG@?$AAC?$AAR?$AAa?$AAd?$AAi?$AAo?$AA?3?$AA?3?$AAS?$AAe?$AAt?$AAC?$AAa?$AAl?$AAl?$AAF?$AAo?$AAr?$AAw?$AAa?$AAr?$AAd?$AAi?$AAn?$AAg?$AA?$AA@ 00161814     supsvc.obj
 0002:00020848       ??_C@_1JI@LHPCEFKH@?$AAC?$AAR?$AAa?$AAd?$AAi?$AAo?$AA?3?$AA?3?$AAS?$AAe?$AAt?$AAC?$AAa?$AAl?$AAl?$AAF?$AAo?$AAr?$AAw?$AAa?$AAr?$AAd?$AAi?$AAn?$AAg?$AA?3?$AA?5?$AAp?$AAS?$AAu?$AAp?$AAs@ 00161848     supsvc.obj
 0002:000208e0       ??_C@_1DK@EMFFGLMA@?$AAC?$AAR?$AAa?$AAd?$AAi?$AAo?$AA?3?$AA?3?$AAR?$AAe?$AAm?$AAo?$AAv?$AAe?$AAC?$AAa?$AAl?$AAl?$AAF?$AAo?$AAr?$AAw?$AAa?$AAr?$AAd?$AAi?$AAn?$AAg?$AA?$AA@ 001618e0     supsvc.obj
 0002:00020920       ??_C@_1HK@GKNEGBFG@?$AAC?$AAR?$AAa?$AAd?$AAi?$AAo?$AA?3?$AA?3?$AAR?$AAe?$AAm?$AAo?$AAv?$AAe?$AAC?$AAa?$AAl?$AAl?$AAF?$AAo?$AAr?$AAw?$AAa?$AAr?$AAd?$AAi?$AAn?$AAg?$AA?3?$AA?5?$AAr?$AAe@ 00161920     supsvc.obj
 0002:000209a0       ??_C@_1JA@DEPOJBII@?$AAG?$AAe?$AAt?$AAC?$AAa?$AAl?$AAl?$AAW?$AAa?$AAi?$AAt?$AAi?$AAn?$AAg?$AA?5?$AAs?$AAt?$AAi?$AAl?$AAl?$AA?5?$AAf?$AAa?$AAi?$AAl?$AAe?$AAd?$AA?5?$AAw?$AAi?$AAt?$AAh@ 001619a0     supsvc.obj
 0002:00020a30       ??_C@_1FO@BJPGJCIF@?$AAR?$AAe?$AAt?$AAr?$AAy?$AAi?$AAn?$AAg?$AA?5?$AAG?$AAe?$AAt?$AAC?$AAa?$AAl?$AAl?$AAW?$AAa?$AAi?$AAt?$AAi?$AAn?$AAg?$AA?5?$AAw?$AAi?$AAt?$AAh?$AA?5?$AAc?$AAl?$AAa@ 00161a30     supsvc.obj
 0002:00020a90       ??_C@_1II@GNBBMNPP@?$AAG?$AAe?$AAt?$AAC?$AAa?$AAl?$AAl?$AAW?$AAa?$AAi?$AAt?$AAi?$AAn?$AAg?$AA?5?$AAf?$AAa?$AAi?$AAl?$AAe?$AAd?$AA?5?$AAG?$AAe?$AAt?$AAC?$AAa?$AAl?$AAl?$AAW?$AAa?$AAi@ 00161a90     supsvc.obj
 0002:00020b18       ??_C@_1DO@NGLLJEII@?$AAC?$AAR?$AAa?$AAd?$AAi?$AAo?$AA?3?$AA?3?$AAG?$AAe?$AAt?$AAC?$AAa?$AAl?$AAl?$AAW?$AAa?$AAi?$AAt?$AAi?$AAn?$AAg?$AAS?$AAe?$AAt?$AAt?$AAi?$AAn?$AAg?$AAs?$AA?$AA@ 00161b18     supsvc.obj
 0002:00020b58       ??_C@_1EE@IPEBABPL@?$AAC?$AAR?$AAa?$AAd?$AAi?$AAo?$AA?3?$AA?3?$AAG?$AAe?$AAt?$AAC?$AAa?$AAl?$AAl?$AAW?$AAa?$AAi?$AAt?$AAi?$AAn?$AAg?$AAS?$AAe?$AAt?$AAt?$AAi?$AAn?$AAg?$AAs?$AA?5?$AA?$CF@ 00161b58     supsvc.obj
 0002:00020b9c       ??_C@_1CK@FHIKHMKH@?$AAQ?$AAM?$AAI?$AA?5?$AAr?$AAe?$AAt?$AAu?$AAr?$AAn?$AA?5?$AAe?$AAr?$AAr?$AAo?$AAr?$AA?0?$AA?5?$AA?$CF?$AAd?$AA?$AA@ 00161b9c     supsvc.obj
 0002:00020bc8       ??_C@_1EM@GPOIOJEK@?$AAS?$AAe?$AAt?$AAC?$AAa?$AAl?$AAl?$AAW?$AAa?$AAi?$AAt?$AAi?$AAn?$AAg?$AAS?$AAt?$AAa?$AAt?$AAu?$AAs?$AA?5?$AA0?$AAx?$AA?$CF?$AAx?$AA?0?$AA?5?$AA0?$AAx?$AA?$CF?$AAx?$AA?0@ 00161bc8     supsvc.obj
 0002:00020c18       ??_C@_1HK@LHJDJDIM@?$AAC?$AAR?$AAa?$AAd?$AAi?$AAo?$AA?3?$AA?3?$AAS?$AAe?$AAt?$AAC?$AAa?$AAl?$AAl?$AAW?$AAa?$AAi?$AAt?$AAi?$AAn?$AAg?$AAS?$AAt?$AAa?$AAt?$AAu?$AAs?$AA?3?$AA?5?$AAr?$AAe@ 00161c18     supsvc.obj
 0002:00020c98       ??_C@_1EK@BBCAJMAO@?$AAO?$AAr?$AAi?$AAg?$AAU?$AAS?$AAS?$AAD?$AA?5?$AAs?$AAe?$AAn?$AAd?$AA?5?$AAf?$AAa?$AAi?$AAl?$AAe?$AAd?$AA?5?$AA?$CB?$AA?5?$AAe?$AAr?$AAr?$AAo?$AAC?$AAo?$AAd?$AAe?$AA?5@ 00161c98     supsvc.obj
 0002:00020ce4       ??_C@_1CG@FPBOPME@?$AAC?$AAR?$AAa?$AAd?$AAi?$AAo?$AA?3?$AA?3?$AAA?$AAn?$AAs?$AAw?$AAe?$AAr?$AAU?$AAS?$AAS?$AAD?$AA?$AA@ 00161ce4     supsvc.obj
 0002:00020d0c       ??_C@_1DC@OANHHBPN@?$AAA?$AAn?$AAs?$AAw?$AAe?$AAr?$AAU?$AAS?$AAS?$AAD?$AA?5?$AAs?$AAe?$AAn?$AAd?$AA?5?$AAf?$AAa?$AAi?$AAl?$AAe?$AAd?$AA?5?$AA?$CB?$AA?$AA@ 00161d0c     supsvc.obj
 0002:00020d40       ??_C@_1CC@BPGNLMGI@?$AAC?$AAR?$AAa?$AAd?$AAi?$AAo?$AA?3?$AA?3?$AAS?$AAe?$AAn?$AAd?$AAU?$AAS?$AAS?$AAD?$AA?$AA@ 00161d40     supsvc.obj
 0002:00020d68       ??_C@_1EI@MAAAPLHB@?$AAC?$AAR?$AAa?$AAd?$AAi?$AAo?$AA?3?$AA?3?$AAC?$AAa?$AAn?$AAc?$AAe?$AAl?$AAS?$AAu?$AAp?$AAS?$AAe?$AAr?$AAv?$AAi?$AAc?$AAe?$AAD?$AAa?$AAt?$AAa?$AAS?$AAe?$AAs?$AAs@ 00161d68     supsvc.obj
 0002:00020db0       ??_C@_1EG@DHMNNHOP@?$AAC?$AAR?$AAa?$AAd?$AAi?$AAo?$AA?3?$AA?3?$AAG?$AAe?$AAt?$AAH?$AAi?$AAd?$AAe?$AAC?$AAo?$AAn?$AAn?$AAe?$AAc?$AAt?$AAe?$AAd?$AAI?$AAd?$AAS?$AAe?$AAt?$AAt?$AAi?$AAn@ 00161db0     supsvc.obj
 0002:00020df8       ??_C@_1EI@GHONJBBM@?$AAm?$AAp?$AAF?$AAn?$AAS?$AAw?$AAi?$AAA?$AAT?$AAS?$AAe?$AAt?$AAE?$AAn?$AAu?$AAm?$AA?5?$AAf?$AAa?$AAi?$AAl?$AAe?$AAd?$AA?0?$AA?5?$AAr?$AAc?$AAo?$AAd?$AAe?$AA?5?$AA?$DN@ 00161df8     supsvc.obj
 0002:00020e40       ??_C@_1DG@OAEBPANH@?$AAm?$AAp?$AAF?$AAn?$AAS?$AAw?$AAi?$AAA?$AAT?$AAS?$AAe?$AAt?$AAE?$AAn?$AAu?$AAm?$AA?5?$AAu?$AAn?$AAd?$AAe?$AAf?$AAi?$AAn?$AAe?$AAd?$AA?$AA@ 00161e40     supsvc.obj
 0002:00020e78       ??_C@_06MBABPIGL@1?0?$CC?$CFs?$CC?$AA@ 00161e78     supsvc.obj
 0002:00020e80       ??_C@_01GBGANLPD@0?$AA@    00161e80     supsvc.obj
 0002:00020e84       ??_C@_1CM@HHKBPOJP@?$AAS?$AAe?$AAn?$AAd?$AAS?$AAu?$AAp?$AAS?$AAv?$AAc?$AAs?$AAT?$AAh?$AAr?$AAe?$AAa?$AAd?$AAP?$AAr?$AAo?$AAc?$AA?$AA@ 00161e84     supsvc.obj
 0002:00020eb0       ??_C@_1DE@KNNDIIDC@?$AAp?$AAS?$AAS?$AAU?$AAS?$AAS?$AAD?$AAD?$AAa?$AAt?$AAa?$AA?5?$AAo?$AAu?$AAt?$AA?5?$AAo?$AAf?$AA?5?$AAM?$AAe?$AAm?$AAo?$AAr?$AAy?$AA?$AA@ 00161eb0     supsvc.obj
 0002:00020ee4       ??_C@_1DG@EGMMFFAI@?$AAC?$AAR?$AAa?$AAd?$AAi?$AAo?$AA?3?$AA?3?$AAS?$AAe?$AAn?$AAd?$AAS?$AAu?$AAp?$AAS?$AAe?$AAr?$AAv?$AAi?$AAc?$AAe?$AAD?$AAa?$AAt?$AAa?$AA?$AA@ 00161ee4     supsvc.obj
 0002:00020f1c       ??_C@_19GGMAHBDP@?$AA?$DM?$AAc?$AAr?$AA?$DO?$AA?$AA@ 00161f1c     toolbox.obj
 0002:00020f28       ??_C@_19CHKHCDBO@?$AA?$DM?$AAl?$AAf?$AA?$DO?$AA?$AA@ 00161f28     toolbox.obj
 0002:00020f34       ??_C@_1BG@FEAIPEDD@?$AA?4?$AA?2?$AAu?$AAt?$AAi?$AAl?$AA?4?$AAc?$AAp?$AAp?$AA?$AA@ 00161f34     util.obj
 0002:00020f50       ??_C@_1FA@IKMFKKLE@?$AAI?$AAn?$AAi?$AAt?$AAi?$AAa?$AAl?$AAi?$AAz?$AAe?$AAC?$AAa?$AAr?$AAr?$AAi?$AAe?$AAr?$AAI?$AAn?$AAd?$AAe?$AAx?$AA?3?$AAu?$AAn?$AAk?$AAn?$AAo?$AAw?$AAn?$AA?5?$AAc@ 00161f50     util.obj
 0002:00020fa0       ??_C@_15JCPNBDBO@?$AAS?$AAW?$AA?$AA@ 00161fa0     util.obj
 0002:00020fa8       ??_C@_19PNHLOHBK@?$AAR?$AAU?$AAI?$AAM?$AA?$AA@ 00161fa8     util.obj
 0002:00020fb4       ??_C@_17PCFLMGFN@?$AAV?$AAZ?$AAW?$AA?$AA@ 00161fb4     util.obj
 0002:00020fbc       ??_C@_17JPIPALNO@?$AAP?$AAC?$AAS?$AA?$AA@ 00161fbc     util.obj
 0002:00020fc4       ??_C@_1DC@GNGFOBBC@?$AAC?$AAa?$AAr?$AAr?$AAi?$AAe?$AAr?$AA?$DP?$AA?0?$AA?5?$AAl?$AAR?$AAe?$AAs?$AAu?$AAl?$AAt?$AA?5?$AA?$DN?$AA?5?$AA0?$AAx?$AA?$CF?$AAx?$AA?$AA@ 00161fc4     util.obj
 0002:00020ff8       ??_C@_1GI@JAFHCGK@?$AAF?$AAa?$AAi?$AAl?$AA?5?$AAt?$AAo?$AA?5?$AAr?$AAe?$AAa?$AAd?$AA?5?$AAm?$AAo?$AAS?$AAM?$AAS?$AAM?$AAa?$AAx?$AAL?$AAe?$AAn?$AA?5?$AAf?$AAr?$AAo?$AAm?$AA?5?$AAt?$AAh@ 00161ff8     util.obj
 0002:00021060       ??_C@_1EG@KNGEILEG@?$AAF?$AAa?$AAi?$AAl?$AAe?$AAd?$AA?5?$AAt?$AAo?$AA?5?$AAw?$AAr?$AAi?$AAt?$AAe?$AA?5?$AA?$CF?$AAs?$AA?5?$AAt?$AAo?$AA?5?$AAt?$AAh?$AAe?$AA?5?$AAr?$AAe?$AAg?$AAi?$AAs?$AAt@ 00162060     util.obj
 0002:000210a8       ??_C@_1DA@BDGFJIMP@?$AAI?$AAS?$AA6?$AA3?$AA7?$AAM?$AAa?$AAx?$AAA?$AAs?$AAc?$AAi?$AAi?$AAC?$AAh?$AAa?$AAr?$AAa?$AAc?$AAt?$AAe?$AAr?$AAs?$AA?$AA@ 001620a8     util.obj
 0002:000210d8       ??_C@_1EE@GHMKNJNF@?$AAS?$AAo?$AAf?$AAt?$AAw?$AAa?$AAr?$AAe?$AA?2?$AAM?$AAi?$AAc?$AAr?$AAo?$AAs?$AAo?$AAf?$AAt?$AA?2?$AAS?$AAM?$AAS?$AA?2?$AAT?$AAe?$AAx?$AAt?$AAS?$AAh?$AAa?$AAr?$AAe@ 001620d8     util.obj
 0002:00021120       ??_C@_1FO@ENPOKCCK@?$AAC?$AAa?$AAr?$AAr?$AAi?$AAe?$AAr?$AAS?$AAu?$AAf?$AAf?$AAi?$AAx?$AA?5?$AAn?$AAo?$AAt?$AA?5?$AAd?$AAe?$AAf?$AAi?$AAn?$AAe?$AAd?$AA?0?$AA?5?$AAf?$AAo?$AAr?$AAc?$AAe@ 00162120     util.obj
 0002:00021180       ??_C@_1GE@POENCNBC@?$AAE?$AAr?$AAr?$AAo?$AAr?$AA?5?$AAC?$AAo?$AAp?$AAy?$AAi?$AAn?$AAg?$AA?5?$AAF?$AAi?$AAl?$AAe?$AA?5?$AA?$CF?$AAs?$AA?5?$AAt?$AAo?$AA?5?$AAc?$AAa?$AAr?$AAr?$AAi?$AAe?$AAr@ 00162180     util.obj
 0002:000211e4       ??_C@_1CO@NLFOCNIF@?$AAW?$AAi?$AAn?$AAd?$AAo?$AAw?$AAs?$AA?2?$AAS?$AAW?$AAC?$AAa?$AAr?$AAr?$AAi?$AAe?$AAr?$AA1?$AA?4?$AAg?$AAi?$AAf?$AA?$AA@ 001621e4     util.obj
 0002:00021214       ??_C@_1CO@KMMAPPHF@?$AAW?$AAi?$AAn?$AAd?$AAo?$AAw?$AAs?$AA?2?$AAS?$AAW?$AAC?$AAa?$AAr?$AAr?$AAi?$AAe?$AAr?$AA2?$AA?4?$AAg?$AAi?$AAf?$AA?$AA@ 00162214     util.obj
 0002:00021244       ??_C@_1CO@NDOBFELI@?$AAE?$AAr?$AAr?$AAo?$AAr?$AA?5?$AAi?$AAn?$AA?5?$AAD?$AAe?$AAl?$AAe?$AAt?$AAe?$AAF?$AAi?$AAl?$AAe?$AA?5?$AA?$CF?$AAd?$AA?$AA@ 00162244     util.obj
 0002:00021274       ??_C@_1DM@IPENMKMD@?$AAE?$AAr?$AAr?$AAo?$AAr?$AA?5?$AAi?$AAn?$AA?5?$AAS?$AAe?$AAt?$AAF?$AAi?$AAl?$AAe?$AAA?$AAt?$AAt?$AAr?$AAi?$AAb?$AAu?$AAt?$AAe?$AAs?$AA?5?$AA?$CF?$AAd?$AA?$AA@ 00162274     util.obj
 0002:000212b0       ??_C@_1CM@BODKIHIL@?$AAE?$AAr?$AAr?$AAo?$AAr?$AA?5?$AAi?$AAn?$AA?5?$AAM?$AAo?$AAv?$AAe?$AAF?$AAi?$AAl?$AAe?$AAr?$AA?5?$AA?$CF?$AAd?$AA?$AA@ 001622b0     util.obj
 0002:000212dc       ??_C@_1DG@GEMLICON@?$AAW?$AAi?$AAn?$AAd?$AAo?$AAw?$AAs?$AA?2?$AAc?$AAa?$AAr?$AAr?$AAi?$AAe?$AAr?$AAl?$AAo?$AAg?$AAo?$AAo?$AAl?$AAd?$AA?4?$AAg?$AAi?$AAf?$AA?$AA@ 001622dc     util.obj
 0002:00021314       ??_C@_1DA@FIFLPKPO@?$AAW?$AAi?$AAn?$AAd?$AAo?$AAw?$AAs?$AA?2?$AAc?$AAa?$AAr?$AAr?$AAi?$AAe?$AAr?$AAl?$AAo?$AAg?$AAo?$AA?4?$AAg?$AAi?$AAf?$AA?$AA@ 00162314     util.obj
 0002:00021348       ??_C@_1FA@LNGGNDJA@?$AAc?$AAa?$AAr?$AAr?$AAi?$AAe?$AAr?$AAI?$AAD?$AA?5?$AA?$DN?$AA?5?$AA?$CF?$AAd?$AA?0?$AA?5?$AAd?$AAw?$AAC?$AAa?$AAr?$AAr?$AAi?$AAe?$AAr?$AAF?$AAr?$AAo?$AAm?$AAM?$AAo?$AAd@ 00162348     util.obj
 0002:00021398       ??_C@_1DA@EKFLLKJC@?$AAD?$AAy?$AAn?$AAa?$AAm?$AAi?$AAc?$AAC?$AAa?$AAr?$AAr?$AAi?$AAe?$AAr?$AAS?$AAu?$AAp?$AAp?$AAo?$AAr?$AAt?$AAe?$AAd?$AA?$AA@ 00162398     util.obj
 0002:000213c8       ??_C@_1BI@NHEMNIMN@?$AA?4?$AA?2?$AAv?$AAo?$AAi?$AAc?$AAe?$AA?4?$AAc?$AAp?$AAp?$AA?$AA@ 001623c8     voice.obj
 0002:000213e0       ??_C@_1CE@ILECDGGF@?$AAr?$AAi?$AAl?$AAA?$AAu?$AAd?$AAi?$AAo?$AAM?$AAo?$AAd?$AAe?$AA?5?$AA?$DN?$AA?5?$AA?$CF?$AAd?$AA?$AA@ 001623e0     voice.obj
 0002:00021408       ??_C@_1EO@GBDDINAC@?$AAS?$AAw?$AAi?$AAM?$AA2?$AAM?$AAA?$AAV?$AA_?$AAA?$AAu?$AAd?$AAi?$AAo?$AAG?$AAe?$AAt?$AAP?$AAr?$AAo?$AAf?$AAi?$AAl?$AAe?$AA?5?$AAf?$AAa?$AAi?$AAl?$AAe?$AAd?$AA?5@ 00162408     voice.obj
 0002:00021458       ??_C@_1JG@HEAINCJE@?$AAE?$AAx?$AAe?$AAc?$AAu?$AAt?$AAi?$AAn?$AAg?$AA?5?$AAS?$AAe?$AAt?$AAA?$AAu?$AAd?$AAi?$AAo?$AAG?$AAa?$AAi?$AAn?$AA?5?$AA?$CI?$AAS?$AAw?$AAi?$AAM?$AA2?$AAM?$AAA?$AAV@ 00162458     voice.obj
 0002:000214f0       ??_C@_1JI@EHOEPFLF@?$AAE?$AAx?$AAe?$AAc?$AAu?$AAt?$AAi?$AAn?$AAg?$AA?5?$AAS?$AAe?$AAt?$AAA?$AAu?$AAd?$AAi?$AAo?$AAG?$AAa?$AAi?$AAn?$AA?5?$AA?$CI?$AAS?$AAw?$AAi?$AA9?$AA0?$AA9?$AA0?$AAA@ 001624f0     voice.obj
 0002:00021588       ??_C@_1DM@OBHONIEE@?$AAp?$AAA?$AAu?$AAd?$AAi?$AAo?$AAG?$AAa?$AAi?$AAn?$AAD?$AAa?$AAt?$AAa?$AA?9?$AA?$DO?$AAd?$AAw?$AAR?$AAx?$AAG?$AAa?$AAi?$AAn?$AA?5?$AA0?$AAx?$AA?$CF?$AAx?$AA?$AA@ 00162588     voice.obj
 0002:000215c4       ??_C@_1DM@FBEDIKBE@?$AAp?$AAA?$AAu?$AAd?$AAi?$AAo?$AAG?$AAa?$AAi?$AAn?$AAD?$AAa?$AAt?$AAa?$AA?9?$AA?$DO?$AAd?$AAw?$AAT?$AAx?$AAG?$AAa?$AAi?$AAn?$AA?5?$AA0?$AAx?$AA?$CF?$AAx?$AA?$AA@ 001625c4     voice.obj
 0002:00021648       ??_C@_1LC@CLFIGADE@?$AAS?$AAw?$AAi?$AAS?$AAe?$AAt?$AAA?$AAu?$AAd?$AAi?$AAo?$AAM?$AAo?$AAd?$AAe?$AA?5?$AAw?$AAi?$AAt?$AAh?$AA?5?$AAm?$AAo?$AAd?$AAe?$AAm?$AAA?$AAu?$AAd?$AAi?$AAo?$AAP@ 00162648     voice.obj
 0002:00021700       ??_C@_1FI@LJOBPGFA@?$AAS?$AAw?$AAi?$AAS?$AAe?$AAt?$AAM?$AAI?$AAC?$AAM?$AAu?$AAt?$AAe?$AAS?$AAt?$AAa?$AAt?$AAu?$AAs?$AA?5?$AAw?$AAo?$AAr?$AAk?$AAs?$AA?5?$AAa?$AAr?$AAo?$AAu?$AAn?$AAd@ 00162700     voice.obj
 0002:00021758       ??_C@_1PI@FLAINBCE@?$AAS?$AAw?$AAi?$AAM?$AA2?$AAM?$AAA?$AAV?$AA_?$AAA?$AAu?$AAd?$AAi?$AAo?$AAS?$AAe?$AAt?$AAP?$AAr?$AAo?$AAf?$AAi?$AAl?$AAe?$AA?5?$AAf?$AAa?$AAi?$AAl?$AAe?$AAd?$AA?5@ 00162758     voice.obj
 0002:00021850       ??_C@_1FE@DNBFNEGG@?$AAS?$AAw?$AAi?$AAM?$AA2?$AAM?$AAA?$AAV?$AA_?$AAA?$AAu?$AAd?$AAi?$AAo?$AAG?$AAe?$AAt?$AAP?$AAr?$AAo?$AAf?$AAi?$AAl?$AAe?$AA?5?$AAf?$AAa?$AAi?$AAl?$AAe?$AAd?$AA?5@ 00162850     voice.obj
 0002:000218a8       ??_C@_1JK@IICNGNFE@?$AAC?$AAa?$AAc?$AAh?$AAe?$AA?1?$AAR?$AAe?$AAs?$AAt?$AAo?$AAr?$AAe?$AA?5?$AAa?$AAu?$AAd?$AAi?$AAo?$AA?5?$AAm?$AAo?$AAd?$AAe?$AA?5?$AA?$DN?$AA?5?$AA?$CF?$AAd?$AA?$CB?$AA?0?$AA?5@ 001628a8     voice.obj
 0002:00021944       ??_C@_1DM@PNBKAMBF@?$AAA?$AAu?$AAd?$AAi?$AAo?$AA?5?$AAR?$AAe?$AAg?$AA?5?$AAk?$AAe?$AAy?$AA?$CB?$AA?5?$AAl?$AAR?$AAe?$AAs?$AAu?$AAl?$AAt?$AA?5?$AA?$DN?$AA?5?$AA0?$AAx?$AA?$CF?$AAx?$AA?$AA@ 00162944     voice.obj
 0002:00021980       ??_C@_1GG@MIOADPDM@?$AAE?$AAn?$AAu?$AAm?$AA?5?$AAk?$AAe?$AAy?$AA?5?$AAa?$AAu?$AAd?$AAi?$AAo?$AA?$CB?$AA?5?$AAl?$AAS?$AAu?$AAb?$AAK?$AAe?$AAy?$AAR?$AAe?$AAs?$AAu?$AAl?$AAt?$AA?5?$AA?$DN?$AA?5@ 00162980     voice.obj
 0002:000219e8       ??_C@_1GC@LLKLNPOA@?$AAA?$AAu?$AAd?$AAi?$AAo?$AA?5?$AAS?$AAu?$AAb?$AA?5?$AAr?$AAe?$AAg?$AA?5?$AAk?$AAe?$AAy?$AA?$CB?$AA?5?$AAs?$AAz?$AAT?$AAe?$AAm?$AAp?$AA?5?$AA?$DN?$AA?5?$AA?$CF?$AAs?$AA?5?$AAl@ 001629e8     voice.obj
 0002:00021a4c       ??_C@_1CE@HLJLGBJD@?$AAR?$AAe?$AAg?$AAA?$AAu?$AAd?$AAi?$AAo?$AAM?$AAo?$AAd?$AAe?$AA?$CB?$AA?5?$AA?$DN?$AA?$CF?$AAd?$AA?$AA@ 00162a4c     voice.obj
 0002:00021a70       ??_C@_1CM@JLCJLJAL@?$AAr?$AAe?$AAg?$AAR?$AAx?$AAG?$AAa?$AAi?$AAn?$AAL?$AAe?$AAv?$AAe?$AAl?$AA?$CF?$AAd?$AA?$CB?$AA?5?$AAN?$AA?1?$AAA?$AA?$AA@ 00162a70     voice.obj
 0002:00021aa0       ??_C@_1KE@IPNNLGCC@?$AAS?$AAe?$AAt?$AAR?$AAX?$AAG?$AAa?$AAi?$AAn?$AAL?$AAe?$AAv?$AAe?$AAl?$AA?$CF?$AAd?$AA?$CB?$AA?0?$AA?5?$AAr?$AAe?$AAt?$AA?5?$AA?$DN?$AA?5?$AA?$CF?$AAd?$AA?5?$AAf?$AAo?$AAr?$AA?5@ 00162aa0     voice.obj
 0002:00021b44       ??_C@_1BI@LANPPLNJ@?$AAR?$AAx?$AAG?$AAa?$AAi?$AAn?$AAL?$AAe?$AAv?$AAe?$AAl?$AA?$AA@ 00162b44     voice.obj
 0002:00021b5c       ??_C@_1DI@BIOKNKJF@?$AAr?$AAe?$AAg?$AAR?$AAx?$AAP?$AAc?$AAm?$AAF?$AAi?$AAl?$AAt?$AAe?$AAr?$AAS?$AAt?$AAa?$AAg?$AAe?$AAN?$AAu?$AAm?$AA?$CB?$AA?5?$AAN?$AA?1?$AAA?$AA?$AA@ 00162b5c     voice.obj
 0002:00021b98       ??_C@_1KA@MMOKKDCL@?$AAS?$AAe?$AAt?$AAR?$AAX?$AAP?$AAC?$AAM?$AAF?$AAi?$AAl?$AAt?$AAe?$AAr?$AA?$CB?$AA?0?$AA?5?$AAr?$AAe?$AAt?$AA?5?$AA?$DN?$AA?5?$AA?$CF?$AAd?$AA?5?$AAf?$AAo?$AAr?$AA?5?$AAs?$AAw@ 00162b98     voice.obj
 0002:00021c38       ??_C@_1DG@IDCHKPJH@?$AAr?$AAe?$AAg?$AAR?$AAx?$AAP?$AAc?$AAm?$AAF?$AAi?$AAl?$AAt?$AAe?$AAr?$AAS?$AAt?$AAa?$AAg?$AAe?$AA?$CF?$AAd?$AA?$CB?$AA?5?$AAN?$AA?1?$AAA?$AA?$AA@ 00162c38     voice.obj
 0002:00021c70       ??_C@_1JC@HPEBMGEK@?$AAR?$AAx?$AAP?$AAc?$AAm?$AAF?$AAi?$AAl?$AAt?$AAe?$AAr?$AAS?$AAt?$AAa?$AAg?$AAe?$AA?$CF?$AAd?$AA?0?$AA?5?$AAf?$AAo?$AAr?$AA?5?$AAs?$AAw?$AAi?$AAA?$AAu?$AAd?$AAi?$AAo@ 00162c70     voice.obj
 0002:00021d04       ??_C@_1CC@KKFNFGLO@?$AAR?$AAx?$AAP?$AAc?$AAm?$AAF?$AAi?$AAl?$AAt?$AAe?$AAr?$AAS?$AAt?$AAa?$AAg?$AAe?$AA?$AA@ 00162d04     voice.obj
 0002:00021d28       ??_C@_1CI@NEKPCENE@?$AAR?$AAx?$AAP?$AAc?$AAm?$AAF?$AAi?$AAl?$AAt?$AAe?$AAr?$AAS?$AAt?$AAa?$AAg?$AAe?$AAN?$AAu?$AAm?$AA?$AA@ 00162d28     voice.obj
 0002:00021d50       ??_C@_1DI@LGKOICDB@?$AAr?$AAe?$AAg?$AAT?$AAx?$AAP?$AAc?$AAm?$AAF?$AAi?$AAl?$AAt?$AAe?$AAr?$AAS?$AAt?$AAa?$AAg?$AAe?$AAN?$AAu?$AAm?$AA?$CB?$AA?5?$AAN?$AA?1?$AAA?$AA?$AA@ 00162d50     voice.obj
 0002:00021d88       ??_C@_1KA@PHLIFGDD@?$AAS?$AAe?$AAt?$AAT?$AAX?$AAP?$AAC?$AAM?$AAF?$AAi?$AAl?$AAt?$AAe?$AAr?$AA?$CB?$AA?0?$AA?5?$AAr?$AAe?$AAt?$AA?5?$AA?$DN?$AA?5?$AA?$CF?$AAd?$AA?5?$AAf?$AAo?$AAr?$AA?5?$AAs?$AAw@ 00162d88     voice.obj
 0002:00021e28       ??_C@_1DG@OIDMFFP@?$AAr?$AAe?$AAg?$AAT?$AAx?$AAP?$AAc?$AAm?$AAF?$AAi?$AAl?$AAt?$AAe?$AAr?$AAS?$AAt?$AAa?$AAg?$AAe?$AA?$CF?$AAd?$AA?$CB?$AA?5?$AAN?$AA?1?$AAA?$AA?$AA@ 00162e28     voice.obj
 0002:00021e60       ??_C@_1JC@OPPEAMMH@?$AAT?$AAx?$AAP?$AAc?$AAm?$AAF?$AAi?$AAl?$AAt?$AAe?$AAr?$AAS?$AAt?$AAa?$AAg?$AAe?$AA?$CF?$AAd?$AA?0?$AA?5?$AAf?$AAo?$AAr?$AA?5?$AAs?$AAw?$AAi?$AAA?$AAu?$AAd?$AAi?$AAo@ 00162e60     voice.obj
 0002:00021ef4       ??_C@_1CC@HBFALAAK@?$AAT?$AAx?$AAP?$AAc?$AAm?$AAF?$AAi?$AAl?$AAt?$AAe?$AAr?$AAS?$AAt?$AAa?$AAg?$AAe?$AA?$AA@ 00162ef4     voice.obj
 0002:00021f18       ??_C@_1CI@IBNGEFME@?$AAT?$AAx?$AAP?$AAc?$AAm?$AAF?$AAi?$AAl?$AAt?$AAe?$AAr?$AAS?$AAt?$AAa?$AAg?$AAe?$AAN?$AAu?$AAm?$AA?$AA@ 00162f18     voice.obj
 0002:00021f40       ??_C@_1CI@PFEFJPKG@?$AAA?$AAu?$AAt?$AAo?$AAO?$AAu?$AAt?$AAp?$AAu?$AAt?$AAG?$AAa?$AAi?$AAn?$AA?$CB?$AA?5?$AAN?$AA?1?$AAA?$AA?$AA@ 00162f40     voice.obj
 0002:00021f68       ??_C@_1KG@BDGHCGEN@?$AAS?$AAe?$AAt?$AAA?$AAu?$AAt?$AAo?$AAO?$AAu?$AAt?$AAp?$AAu?$AAt?$AAG?$AAa?$AAi?$AAn?$AA?$CB?$AA?0?$AA?5?$AAr?$AAe?$AAt?$AA?5?$AA?$DN?$AA?5?$AA?$CF?$AAd?$AA?5?$AAf?$AAo?$AAr@ 00162f68     voice.obj
 0002:00022010       ??_C@_1BO@FOOOLIGK@?$AAA?$AAu?$AAt?$AAo?$AAO?$AAu?$AAt?$AAp?$AAu?$AAt?$AAG?$AAa?$AAi?$AAn?$AA?$AA@ 00163010     voice.obj
 0002:00022030       ??_C@_1CG@EFLHDPEO@?$AAA?$AAu?$AAt?$AAo?$AAI?$AAn?$AAp?$AAu?$AAt?$AAG?$AAa?$AAi?$AAn?$AA?$CB?$AA?5?$AAN?$AA?1?$AAA?$AA?$AA@ 00163030     voice.obj
 0002:00022058       ??_C@_1KE@ILNOCPJM@?$AAS?$AAe?$AAt?$AAA?$AAu?$AAt?$AAo?$AAI?$AAn?$AAp?$AAu?$AAt?$AAG?$AAa?$AAi?$AAn?$AA?$CB?$AA?0?$AA?5?$AAr?$AAe?$AAt?$AA?5?$AA?$DN?$AA?5?$AA?$CF?$AAd?$AA?5?$AAf?$AAo?$AAr?$AA?5@ 00163058     voice.obj
 0002:000220fc       ??_C@_1BM@FONMODNO@?$AAA?$AAu?$AAt?$AAo?$AAI?$AAn?$AAp?$AAu?$AAt?$AAG?$AAa?$AAi?$AAn?$AA?$AA@ 001630fc     voice.obj
 0002:00022118       ??_C@_1CM@LNPBGFOB@?$AAN?$AAo?$AAi?$AAs?$AAe?$AAS?$AAu?$AAp?$AAp?$AAr?$AAe?$AAs?$AAs?$AAi?$AAo?$AAn?$AA?$CB?$AA?5?$AAN?$AA?1?$AAA?$AA?$AA@ 00163118     voice.obj
 0002:00022148       ??_C@_1KK@CAIDPKOA@?$AAS?$AAe?$AAt?$AAN?$AAo?$AAi?$AAs?$AAe?$AAS?$AAu?$AAp?$AAp?$AAr?$AAe?$AAs?$AAs?$AAi?$AAo?$AAn?$AA?$CB?$AA?0?$AA?5?$AAr?$AAe?$AAt?$AA?5?$AA?$DN?$AA?5?$AA?$CF?$AAd?$AA?5?$AAf@ 00163148     voice.obj
 0002:000221f4       ??_C@_1CC@HFOHAJPI@?$AAN?$AAo?$AAi?$AAs?$AAe?$AAS?$AAu?$AAp?$AAp?$AAr?$AAe?$AAs?$AAs?$AAi?$AAo?$AAn?$AA?$AA@ 001631f4     voice.obj
 0002:00022218       ??_C@_1JM@JNHOJHOH@?$AAS?$AAe?$AAt?$AAM?$AAi?$AAc?$AAV?$AAo?$AAl?$AAu?$AAm?$AAe?$AA?$CB?$AA?0?$AA?5?$AAr?$AAe?$AAt?$AA?5?$AA?$DN?$AA?5?$AA?$CF?$AAd?$AA?5?$AAf?$AAo?$AAr?$AA?5?$AAs?$AAw?$AAi?$AAA@ 00163218     voice.obj
 0002:000222b4       ??_C@_1BM@GEEJFIPL@?$AAT?$AAx?$AAV?$AAo?$AAl?$AAu?$AAm?$AAe?$AAL?$AAe?$AAv?$AAe?$AAl?$AA?$AA@ 001632b4     voice.obj
 0002:000222d0       ??_C@_1CM@PALFEHBD@?$AAV?$AAo?$AAi?$AAc?$AAe?$AAV?$AAo?$AAl?$AAu?$AAm?$AAe?$AAL?$AAe?$AAv?$AAe?$AAl?$AA?$CB?$AA?5?$AAN?$AA?1?$AAA?$AA?$AA@ 001632d0     voice.obj
 0002:00022300       ??_C@_1KG@LNKDICFE@?$AAS?$AAe?$AAt?$AAR?$AAe?$AAc?$AAe?$AAi?$AAv?$AAe?$AAr?$AAV?$AAo?$AAl?$AAu?$AAm?$AAe?$AA?$CB?$AA?0?$AA?5?$AAr?$AAe?$AAt?$AA?5?$AA?$DN?$AA?5?$AA?$CF?$AAd?$AA?5?$AAf?$AAo?$AAr@ 00163300     voice.obj
 0002:000223a8       ??_C@_1CC@DPGJCOPO@?$AAV?$AAo?$AAi?$AAc?$AAe?$AAV?$AAo?$AAl?$AAu?$AAm?$AAe?$AAL?$AAe?$AAv?$AAe?$AAl?$AA?$AA@ 001633a8     voice.obj
 0002:000223cc       ??_C@_1CC@EHNIKHJM@?$AAo?$AAu?$AAt?$AAp?$AAu?$AAt?$AAL?$AAe?$AAv?$AAe?$AAl?$AA?$CB?$AA?5?$AAN?$AA?1?$AAA?$AA?$AA@ 001633cc     voice.obj
 0002:000223f0       ??_C@_1KI@MGMMIFOG@?$AAS?$AAw?$AAi?$AAS?$AAe?$AAt?$AAS?$AAp?$AAe?$AAa?$AAk?$AAe?$AAr?$AAL?$AAe?$AAv?$AAe?$AAl?$AA?$CB?$AA?0?$AA?5?$AAr?$AAe?$AAt?$AA?5?$AA?$DN?$AA?5?$AA?$CF?$AAd?$AA?5?$AAf?$AAo@ 001633f0     voice.obj
 0002:00022498       ??_C@_1BI@GGLCMFFO@?$AAO?$AAu?$AAt?$AAp?$AAu?$AAt?$AAL?$AAe?$AAv?$AAe?$AAl?$AA?$AA@ 00163498     voice.obj
 0002:000224b0       ??_C@_1CA@HNGHFHCG@?$AAi?$AAn?$AAp?$AAu?$AAt?$AAL?$AAe?$AAv?$AAe?$AAl?$AA?$CB?$AA?5?$AAN?$AA?1?$AAA?$AA?$AA@ 001634b0     voice.obj
 0002:000224d0       ??_C@_1KA@DKGKMM@?$AAS?$AAw?$AAi?$AAS?$AAe?$AAt?$AAM?$AAI?$AAC?$AAL?$AAe?$AAv?$AAe?$AAl?$AA?$CB?$AA?0?$AA?5?$AAr?$AAe?$AAt?$AA?5?$AA?$DN?$AA?5?$AA?$CF?$AAd?$AA?5?$AAf?$AAo?$AAr?$AA?5?$AAs?$AAw@ 001634d0     voice.obj
 0002:00022570       ??_C@_1BG@NLMKCJHL@?$AAI?$AAn?$AAp?$AAu?$AAt?$AAL?$AAe?$AAv?$AAe?$AAl?$AA?$AA@ 00163570     voice.obj
 0002:00022588       ??_C@_1CG@CNHNIHFI@?$AAs?$AAi?$AAd?$AAe?$AAT?$AAo?$AAn?$AAe?$AAL?$AAe?$AAv?$AAe?$AAl?$AA?$CB?$AA?5?$AAN?$AA?1?$AAA?$AA?$AA@ 00163588     voice.obj
 0002:000225b0       ??_C@_1LC@EHAANKBI@?$AAS?$AAw?$AAi?$AAS?$AAe?$AAt?$AAS?$AAi?$AAd?$AAe?$AAt?$AAo?$AAn?$AAe?$AAG?$AAa?$AAi?$AAn?$AAL?$AAe?$AAv?$AAe?$AAl?$AA?$CB?$AA?0?$AA?5?$AAr?$AAe?$AAt?$AA?5?$AA?$DN?$AA?5@ 001635b0     voice.obj
 0002:00022664       ??_C@_1BM@JAJFPEHG@?$AAS?$AAi?$AAd?$AAe?$AAT?$AAo?$AAn?$AAe?$AAL?$AAe?$AAv?$AAe?$AAl?$AA?$AA@ 00163664     voice.obj
 0002:00022680       ??_C@_1CG@LEKGEMNP@?$AAr?$AAe?$AAg?$AAE?$AAc?$AAh?$AAo?$AAC?$AAa?$AAn?$AAc?$AAe?$AAl?$AA?$CB?$AA?5?$AAN?$AA?1?$AAA?$AA?$AA@ 00163680     voice.obj
 0002:000226a8       ??_C@_1LC@DAODHGMA@?$AAS?$AAw?$AAi?$AAS?$AAe?$AAt?$AAE?$AAc?$AAh?$AAo?$AAC?$AAa?$AAn?$AAc?$AAe?$AAl?$AAP?$AAr?$AAo?$AAf?$AAi?$AAl?$AAe?$AA?$CB?$AA?0?$AA?5?$AAr?$AAe?$AAt?$AA?5?$AA?$DN?$AA?5@ 001636a8     voice.obj
 0002:00022760       ??_C@_1KM@IHCMNCDB@?$AAr?$AAe?$AAg?$AAE?$AAc?$AAh?$AAo?$AAC?$AAa?$AAn?$AAc?$AAe?$AAl?$AA?5?$AAt?$AAo?$AAo?$AA?5?$AAl?$AAa?$AAr?$AAg?$AAe?$AA?5?$AA?$CI?$AA?$DO?$AA2?$AA5?$AA5?$AA?$CJ?$AA?$CB?$AA?5@ 00163760     voice.obj
 0002:0002280c       ??_C@_1CA@GKOCMNAN@?$AAE?$AAc?$AAh?$AAo?$AAC?$AAa?$AAn?$AAc?$AAe?$AAl?$AAa?$AAt?$AAi?$AAo?$AAn?$AA?$AA@ 0016380c     voice.obj
 0002:00022830       ??_C@_1GA@JJIAEGBE@?$AAF?$AAo?$AAr?$AAg?$AAe?$AAt?$AA?5?$AAi?$AAt?$AA?4?$AA?5?$AAL?$AAe?$AAt?$AA?8?$AAs?$AA?5?$AAp?$AAr?$AAo?$AAg?$AAr?$AAa?$AAm?$AA?5?$AAt?$AAh?$AAe?$AA?5?$AAn?$AAe?$AAx@ 00163830     voice.obj
 0002:00022890       ??_C@_1LC@GEEDAGBO@?$AAS?$AAw?$AAi?$AAS?$AAe?$AAt?$AAA?$AAu?$AAd?$AAi?$AAo?$AAM?$AAo?$AAd?$AAe?$AA?$CB?$AA?0?$AA?5?$AAr?$AAe?$AAt?$AA?5?$AA?$DN?$AA?5?$AA?$CF?$AAd?$AA?0?$AA?5?$AAi?$AAt?$AAe?$AAr@ 00163890     voice.obj
 0002:00022948       ??_C@_1EA@GFHIKMNE@?$AAP?$AAr?$AAo?$AAg?$AAr?$AAa?$AAm?$AA?5?$AAf?$AAo?$AAr?$AA?5?$AAR?$AAI?$AAL?$AA?5?$AAa?$AAu?$AAd?$AAi?$AAo?$AA?5?$AAm?$AAo?$AAd?$AAe?$AA?5?$AA?$DN?$AA?5?$AA?$CF?$AAs?$AA?$AA@ 00163948     voice.obj
 0002:00022988       ??_C@_1CA@BHGNNNPK@?$AA?$CF?$AAs?$AA?2?$AAR?$AAI?$AAL?$AA?2?$AAA?$AAu?$AAd?$AAi?$AAo?$AA?2?$AA?$CF?$AAs?$AA?$AA@ 00163988     voice.obj
 0002:000229a8       ??_C@_1BK@BBAOAHBM@?$AA?$CF?$AAs?$AA?2?$AAR?$AAI?$AAL?$AA?2?$AAA?$AAu?$AAd?$AAi?$AAo?$AA?$AA@ 001639a8     voice.obj
 0002:000229c8       ??_C@_1FE@CLLDBKCP@?$AAS?$AAw?$AAi?$AAM?$AA2?$AAM?$AAA?$AAV?$AA_?$AAA?$AAu?$AAd?$AAi?$AAo?$AAG?$AAe?$AAt?$AAP?$AAr?$AAo?$AAf?$AAi?$AAl?$AAe?$AA?5?$AAf?$AAa?$AAi?$AAl?$AAe?$AAd?$AA?0@ 001639c8     voice.obj
 0002:00022a20       ??_C@_1FC@IDJHANDD@?$AAS?$AAw?$AAi?$AAM?$AA2?$AAM?$AAA?$AAV?$AA_?$AAA?$AAu?$AAd?$AAi?$AAo?$AAS?$AAe?$AAt?$AAA?$AAV?$AAM?$AAu?$AAt?$AAe?$AA?5?$AAf?$AAa?$AAi?$AAl?$AAe?$AAd?$AA?0?$AA?5@ 00163a20     voice.obj
 0002:00022a78       ??_C@_1GI@DEEFONNJ@?$AAS?$AAw?$AAi?$AAM?$AA2?$AAM?$AAA?$AAV?$AA_?$AAA?$AAu?$AAd?$AAi?$AAo?$AAS?$AAe?$AAt?$AAA?$AAV?$AAM?$AAu?$AAt?$AAe?$AA?5?$AAp?$AAr?$AAe?$AAv?$AAM?$AAi?$AAc?$AAM@ 00163a78     voice.obj
 0002:00022ae0       ??_C@_1HA@GAFALCAH@?$AAS?$AAw?$AAi?$AAM?$AA2?$AAM?$AAA?$AAV?$AA_?$AAA?$AAu?$AAd?$AAi?$AAo?$AAS?$AAe?$AAt?$AAA?$AAV?$AAM?$AAu?$AAt?$AAe?$AA?5?$AAp?$AAr?$AAe?$AAv?$AAE?$AAa?$AAr?$AAM@ 00163ae0     voice.obj
 0002:00022b50       ??_C@_1FA@HHMLNDGI@?$AAS?$AAw?$AAi?$AAM?$AA2?$AAM?$AAA?$AAV?$AA_?$AAA?$AAu?$AAd?$AAi?$AAo?$AAP?$AAl?$AAa?$AAy?$AAT?$AAo?$AAn?$AAe?$AA?5?$AAf?$AAa?$AAi?$AAl?$AAe?$AAd?$AA?0?$AA?5?$AAr@ 00163b50     voice.obj
 0002:00022ba0       ??_C@_1DO@EBCANLKN@?$AAP?$AAl?$AAa?$AAy?$AAA?$AAu?$AAd?$AAi?$AAo?$AAT?$AAo?$AAn?$AAe?$AA?5?$AAf?$AAa?$AAi?$AAl?$AAe?$AAd?$AA?0?$AA?5?$AAr?$AAe?$AAt?$AA?5?$AA?$DN?$AA?5?$AA?$CF?$AAd?$AA?$AA@ 00163ba0     voice.obj
 0002:00022be0       ??_C@_1FI@BGPNOJHC@?$AAS?$AAw?$AAi?$AAM?$AA2?$AAM?$AAA?$AAV?$AA_?$AAA?$AAu?$AAd?$AAi?$AAo?$AAG?$AAe?$AAt?$AAP?$AAr?$AAo?$AAf?$AAi?$AAl?$AAe?$AA?5?$AAf?$AAa?$AAi?$AAl?$AAe?$AAd?$AA?0@ 00163be0     voice.obj
 0002:00022c38       ??_C@_1IE@HJMBICOM@?$AAS?$AAw?$AAi?$AAM?$AA2?$AAM?$AAA?$AAV?$AA_?$AAA?$AAu?$AAd?$AAi?$AAo?$AAS?$AAe?$AAt?$AAP?$AAr?$AAo?$AAf?$AAi?$AAl?$AAe?$AA?5?$AAf?$AAa?$AAi?$AAl?$AAe?$AAd?$AA?4@ 00163c38     voice.obj
 0002:00022cc0       ??_C@_1LM@FBBHHPLE@?$AAS?$AAw?$AAi?$AAM?$AA2?$AAM?$AAA?$AAV?$AA_?$AAA?$AAu?$AAd?$AAi?$AAo?$AAS?$AAe?$AAt?$AAV?$AAo?$AAl?$AAD?$AAB?$AA?5?$AAf?$AAa?$AAi?$AAl?$AAe?$AAd?$AA?4?$AA?5?$AAr@ 00163cc0     voice.obj
 0002:00022d80       ??_C@_1LO@OBAKHGCK@?$AAS?$AAw?$AAi?$AAM?$AA2?$AAM?$AAA?$AAV?$AA_?$AAA?$AAu?$AAd?$AAi?$AAo?$AAS?$AAe?$AAt?$AAV?$AAo?$AAl?$AAu?$AAm?$AAe?$AA?5?$AAf?$AAa?$AAi?$AAl?$AAe?$AAd?$AA?4?$AA?5@ 00163d80     voice.obj
 0002:00022e40       ??_C@_1MC@MCEMEEBJ@?$AAS?$AAw?$AAi?$AAM?$AA2?$AAM?$AAA?$AAV?$AA_?$AAA?$AAu?$AAd?$AAi?$AAo?$AAS?$AAe?$AAt?$AAT?$AAx?$AAV?$AAo?$AAl?$AAu?$AAm?$AAe?$AA?5?$AAf?$AAa?$AAi?$AAl?$AAe?$AAd@ 00163e40     voice.obj
 0002:00022f08       ??_C@_1LI@PMDDBJCF@?$AAS?$AAw?$AAi?$AAM?$AA2?$AAM?$AAA?$AAV?$AA_?$AAA?$AAu?$AAd?$AAi?$AAo?$AAS?$AAe?$AAt?$AAS?$AAT?$AAG?$AA?5?$AAf?$AAa?$AAi?$AAl?$AAe?$AAd?$AA?4?$AA?5?$AAr?$AAe?$AAt@ 00163f08     voice.obj
 0002:00022fc0       ??_C@_1LI@NCHCPKCJ@?$AAS?$AAw?$AAi?$AAM?$AA2?$AAM?$AAA?$AAV?$AA_?$AAA?$AAu?$AAd?$AAi?$AAo?$AAS?$AAe?$AAt?$AAA?$AAV?$AAE?$AAC?$AA?5?$AAf?$AAa?$AAi?$AAl?$AAe?$AAd?$AA?5?$AAr?$AAe?$AAt@ 00163fc0     voice.obj
 0002:00023078       ??_C@_1NA@DPLKGNPI@?$AAS?$AAw?$AAi?$AAM?$AA2?$AAM?$AAA?$AAV?$AA_?$AAA?$AAu?$AAd?$AAi?$AAo?$AAG?$AAe?$AAt?$AAP?$AAr?$AAo?$AAf?$AAi?$AAl?$AAe?$AA?5?$AAf?$AAa?$AAi?$AAl?$AAe?$AAd?$AA?4@ 00164078     voice.obj
 0002:00023148       ??_C@_1NA@HFOCJGHM@?$AAS?$AAw?$AAi?$AAM?$AA2?$AAM?$AAA?$AAV?$AA_?$AAA?$AAu?$AAd?$AAi?$AAo?$AAS?$AAe?$AAt?$AAP?$AAr?$AAo?$AAf?$AAi?$AAl?$AAe?$AA?5?$AAf?$AAa?$AAi?$AAl?$AAe?$AAd?$AA?4@ 00164148     voice.obj
 0002:00023218       ??_C@_1JC@DFPGJFIC@?$AAg?$AAe?$AAn?$AAe?$AAr?$AAa?$AAt?$AAo?$AAr?$AA?5?$AA?$CF?$AAd?$AA?0?$AA?5?$AAp?$AAr?$AAo?$AAf?$AAi?$AAl?$AAe?$AA?5?$AA?$CF?$AAd?$AA?0?$AA?5?$AAe?$AAa?$AAr?$AAM?$AAu?$AAt@ 00164218     voice.obj
 0002:000232b0       ??_C@_1EM@PPDIAHIJ@?$AAP?$AAr?$AAo?$AAg?$AAr?$AAa?$AAm?$AAA?$AAu?$AAd?$AAi?$AAo?$AAP?$AAa?$AAr?$AAa?$AAm?$AAe?$AAt?$AAe?$AAr?$AA?5?$AAu?$AAn?$AAk?$AAn?$AAo?$AAw?$AAn?$AA?5?$AAm?$AAo@ 001642b0     voice.obj
 0002:00023300       ??_7bad_alloc@std@@6B@     00164300     libcpmt:string.obj
 0002:0002330c       ??_7logic_error@std@@6B@   0016430c     libcpmt:string.obj
 0002:00023318       ??_7length_error@std@@6B@  00164318     libcpmt:string.obj
 0002:00023324       ??_7out_of_range@std@@6B@  00164324     libcpmt:string.obj
 0002:00023378       ??_C@_0BA@JFNIOLAK@string?5too?5long?$AA@ 00164378     libcpmt:string.obj
 0002:000233d4       ??_C@_0BI@CFPLBAOH@invalid?5string?5position?$AA@ 001643d4     libcpmt:string.obj
 0002:000233ec       ??_R4bad_alloc@std@@6B@    001643ec     libcpmt:string.obj
 0002:00023400       ??_R3bad_alloc@std@@8      00164400     libcpmt:string.obj
 0002:00023410       ??_R2bad_alloc@std@@8      00164410     libcpmt:string.obj
 0002:0002341c       ??_R1A@?0A@EA@bad_alloc@std@@8 0016441c     libcpmt:string.obj
 0002:00023438       ??_R1A@?0A@EA@exception@std@@8 00164438     libcpmt:string.obj
 0002:00023454       ??_R3exception@std@@8      00164454     libcpmt:string.obj
 0002:00023464       ??_R2exception@std@@8      00164464     libcpmt:string.obj
 0002:0002346c       ??_R4logic_error@std@@6B@  0016446c     libcpmt:string.obj
 0002:00023480       ??_R3logic_error@std@@8    00164480     libcpmt:string.obj
 0002:00023490       ??_R2logic_error@std@@8    00164490     libcpmt:string.obj
 0002:0002349c       ??_R1A@?0A@EA@logic_error@std@@8 0016449c     libcpmt:string.obj
 0002:000234b8       ??_R4length_error@std@@6B@ 001644b8     libcpmt:string.obj
 0002:000234cc       ??_R3length_error@std@@8   001644cc     libcpmt:string.obj
 0002:000234dc       ??_R2length_error@std@@8   001644dc     libcpmt:string.obj
 0002:000234ec       ??_R1A@?0A@EA@length_error@std@@8 001644ec     libcpmt:string.obj
 0002:00023508       ??_R4out_of_range@std@@6B@ 00164508     libcpmt:string.obj
 0002:0002351c       ??_R3out_of_range@std@@8   0016451c     libcpmt:string.obj
 0002:0002352c       ??_R2out_of_range@std@@8   0016452c     libcpmt:string.obj
 0002:0002353c       ??_R1A@?0A@EA@out_of_range@std@@8 0016453c     libcpmt:string.obj
 0002:000236e4       _TI2?AVbad_alloc@std@@     001646e4     atcmd.obj
 0002:000236f4       _CTA2?AVbad_alloc@std@@    001646f4     atcmd.obj
 0002:00023700       _CT??_R0?AVbad_alloc@std@@@8??0bad_alloc@std@@QAA@ABV01@@Z12 00164700     atcmd.obj
 0002:0002371c       _CT??_R0?AVexception@std@@@8??0exception@std@@QAA@ABV01@@Z12 0016471c     atcmd.obj
 0002:00023738       _TI3?AVlength_error@std@@  00164738     atcmd.obj
 0002:00023748       _CTA3?AVlength_error@std@@ 00164748     atcmd.obj
 0002:00023758       _CT??_R0?AVlength_error@std@@@8??0length_error@std@@QAA@ABV01@@Z40 00164758     atcmd.obj
 0002:00023774       _CT??_R0?AVlogic_error@std@@@8??0logic_error@std@@QAA@ABV01@@Z40 00164774     atcmd.obj
 0002:00023790       _TI3?AVout_of_range@std@@  00164790     DatERI.obj
 0002:000237a0       _CTA3?AVout_of_range@std@@ 001647a0     DatERI.obj
 0002:000237b0       _CT??_R0?AVout_of_range@std@@@8??0out_of_range@std@@QAA@ABV01@@Z40 001647b0     DatERI.obj
 0002:000237cc       __IMPORT_DESCRIPTOR_sw_utilityG 001647cc     sw_utilityG:sw_utilityG.dll
 0002:000237e0       __IMPORT_DESCRIPTOR_ossvcs 001647e0     ossvcs:ossvcs.dll
 0002:000237f4       __IMPORT_DESCRIPTOR_ccoreutl 001647f4     ccoreutl:ccoreutl.dll
 0002:00023808       __IMPORT_DESCRIPTOR_WINSOCK 00164808     winsock:WINSOCK.dll
 0002:0002381c       __IMPORT_DESCRIPTOR_SDKRIL 0016481c     sdkril:SDKRIL.dll
 0002:00023830       __IMPORT_DESCRIPTOR_COREDLL 00164830     coredll:COREDLL.dll
 0002:00023844       __NULL_IMPORT_DESCRIPTOR   00164844     sw_utilityG:sw_utilityG.dll
 0003:00000000       __imp_EscapeCommFunction   00166000     coredll:COREDLL.dll
 0003:00000004       __imp_TlsGetValue          00166004     coredll:COREDLL.dll
 0003:00000008       __imp_TlsSetValue          00166008     coredll:COREDLL.dll
 0003:0000000c       __imp_TlsCall              0016600c     coredll:COREDLL.dll
 0003:00000010       __imp_?terminate@std@@YAXXZ 00166010     coredll:COREDLL.dll
 0003:00000014       __imp_RaiseException       00166014     coredll:COREDLL.dll
 0003:00000018       __imp___security_gen_cookie 00166018     coredll:COREDLL.dll
 0003:0000001c       __imp_LocalSize            0016601c     coredll:COREDLL.dll
 0003:00000020       __imp___report_gsfailure   00166020     coredll:COREDLL.dll
 0003:00000024       __imp_RegEnumKeyExW        00166024     coredll:COREDLL.dll
 0003:00000028       __imp_strtok               00166028     coredll:COREDLL.dll
 0003:0000002c       __imp_strtoul              0016602c     coredll:COREDLL.dll
 0003:00000030       __imp_MoveFileW            00166030     coredll:COREDLL.dll
 0003:00000034       __imp_SetFileAttributesW   00166034     coredll:COREDLL.dll
 0003:00000038       __imp_DeleteFileW          00166038     coredll:COREDLL.dll
 0003:0000003c       __imp_CopyFileW            0016603c     coredll:COREDLL.dll
 0003:00000040       __imp_strcmp               00166040     coredll:COREDLL.dll
 0003:00000044       __imp_LocalReAlloc         00166044     coredll:COREDLL.dll
 0003:00000048       __imp__vsnprintf           00166048     coredll:COREDLL.dll
 0003:0000004c       __imp__vsnwprintf          0016604c     coredll:COREDLL.dll
 0003:00000050       __imp_OutputDebugStringW   00166050     coredll:COREDLL.dll
 0003:00000054       __imp_SystemIdleTimerReset 00166054     coredll:COREDLL.dll
 0003:00000058       __imp_wcstombs             00166058     coredll:COREDLL.dll
 0003:0000005c       __imp_wcstoul              0016605c     coredll:COREDLL.dll
 0003:00000060       __imp_malloc               00166060     coredll:COREDLL.dll
 0003:00000064       __imp_free                 00166064     coredll:COREDLL.dll
 0003:00000068       __imp_CeSafeCopyMemory     00166068     coredll:COREDLL.dll
 0003:0000006c       __imp_swscanf              0016606c     coredll:COREDLL.dll
 0003:00000070       __imp_LocalAlloc           00166070     coredll:COREDLL.dll
 0003:00000074       __imp_memmove              00166074     coredll:COREDLL.dll
 0003:00000078       __imp_PowerPolicyNotify    00166078     coredll:COREDLL.dll
 0003:0000007c       __imp_TryEnterCriticalSection 0016607c     coredll:COREDLL.dll
 0003:00000080       __imp_LocalFree            00166080     coredll:COREDLL.dll
 0003:00000084       __imp_SetSystemTime        00166084     coredll:COREDLL.dll
 0003:00000088       __imp_CeSetThreadPriority  00166088     coredll:COREDLL.dll
 0003:0000008c       __imp__wcsupr              0016608c     coredll:COREDLL.dll
 0003:00000090       __imp_LoadLibraryW         00166090     coredll:COREDLL.dll
 0003:00000094       __imp_GetProcAddressW      00166094     coredll:COREDLL.dll
 0003:00000098       __imp__itow                00166098     coredll:COREDLL.dll
 0003:0000009c       __imp_CreateEventW         0016609c     coredll:COREDLL.dll
 0003:000000a0       __imp_RegQueryValueExW     001660a0     coredll:COREDLL.dll
 0003:000000a4       __imp_wcstok               001660a4     coredll:COREDLL.dll
 0003:000000a8       __imp_strstr               001660a8     coredll:COREDLL.dll
 0003:000000ac       __imp_StringCchPrintfW     001660ac     coredll:COREDLL.dll
 0003:000000b0       __imp_RegOpenKeyExW        001660b0     coredll:COREDLL.dll
 0003:000000b4       __imp_RegSetValueExW       001660b4     coredll:COREDLL.dll
 0003:000000b8       __imp_RegCloseKey          001660b8     coredll:COREDLL.dll
 0003:000000bc       __imp_RegCreateKeyExW      001660bc     coredll:COREDLL.dll
 0003:000000c0       __imp_wcsncmp              001660c0     coredll:COREDLL.dll
 0003:000000c4       __imp___dtou               001660c4     coredll:COREDLL.dll
 0003:000000c8       __imp___addd               001660c8     coredll:COREDLL.dll
 0003:000000cc       __imp___utod               001660cc     coredll:COREDLL.dll
 0003:000000d0       __imp___muld               001660d0     coredll:COREDLL.dll
 0003:000000d4       __imp_pow                  001660d4     coredll:COREDLL.dll
 0003:000000d8       __imp_FreeLibrary          001660d8     coredll:COREDLL.dll
 0003:000000dc       __imp_atoi                 001660dc     coredll:COREDLL.dll
 0003:000000e0       __imp__itoa                001660e0     coredll:COREDLL.dll
 0003:000000e4       __imp_sprintf              001660e4     coredll:COREDLL.dll
 0003:000000e8       __imp_SystemTimeToFileTime 001660e8     coredll:COREDLL.dll
 0003:000000ec       __imp_LocalFileTimeToFileTime 001660ec     coredll:COREDLL.dll
 0003:000000f0       __imp_FileTimeToSystemTime 001660f0     coredll:COREDLL.dll
 0003:000000f4       __imp_iswctype             001660f4     coredll:COREDLL.dll
 0003:000000f8       __imp_DeleteCriticalSection 001660f8     coredll:COREDLL.dll
 0003:000000fc       __imp_InitializeCriticalSection 001660fc     coredll:COREDLL.dll
 0003:00000100       __imp_KernelIoControl      00166100     coredll:COREDLL.dll
 0003:00000104       __imp_??_L@YAXPAXIHP6AX0@Z1@Z 00166104     coredll:COREDLL.dll
 0003:00000108       __imp_??_M@YAXPAXIHP6AX0@Z@Z 00166108     coredll:COREDLL.dll
 0003:0000010c       __imp_strncpy              0016610c     coredll:COREDLL.dll
 0003:00000110       __imp__wtol                00166110     coredll:COREDLL.dll
 0003:00000114       __imp_wcsncat              00166114     coredll:COREDLL.dll
 0003:00000118       __imp__snprintf            00166118     coredll:COREDLL.dll
 0003:0000011c       __imp_strncat              0016611c     coredll:COREDLL.dll
 0003:00000120       __imp_wsprintfW            00166120     coredll:COREDLL.dll
 0003:00000124       __imp_WideCharToMultiByte  00166124     coredll:COREDLL.dll
 0003:00000128       __imp__snwprintf           00166128     coredll:COREDLL.dll
 0003:0000012c       __imp_wcschr               0016612c     coredll:COREDLL.dll
 0003:00000130       __imp_wcsncpy              00166130     coredll:COREDLL.dll
 0003:00000134       __imp_WaitForMultipleObjects 00166134     coredll:COREDLL.dll
 0003:00000138       __imp___C_specific_handler 00166138     coredll:COREDLL.dll
 0003:0000013c       __imp_WaitCommEvent        0016613c     coredll:COREDLL.dll
 0003:00000140       __imp_ReadFile             00166140     coredll:COREDLL.dll
 0003:00000144       __imp_EventModify          00166144     coredll:COREDLL.dll
 0003:00000148       __imp_EnterCriticalSection 00166148     coredll:COREDLL.dll
 0003:0000014c       __imp_LeaveCriticalSection 0016614c     coredll:COREDLL.dll
 0003:00000150       __imp_strlen               00166150     coredll:COREDLL.dll
 0003:00000154       __imp_??0exception@std@@QAA@PBD@Z 00166154     coredll:COREDLL.dll
 0003:00000158       __imp_?what@exception@std@@UBAPBDXZ 00166158     coredll:COREDLL.dll
 0003:0000015c       __imp_??1exception@std@@UAA@XZ 0016615c     coredll:COREDLL.dll
 0003:00000160       __imp_??3@YAXPAX@Z         00166160     coredll:COREDLL.dll
 0003:00000164       __imp_SetThreadPriority    00166164     coredll:COREDLL.dll
 0003:00000168       __imp_??2@YAPAXI@Z         00166168     coredll:COREDLL.dll
 0003:0000016c       __imp___rt_udiv            0016616c     coredll:COREDLL.dll
 0003:00000170       __imp___CxxThrowException  00166170     coredll:COREDLL.dll
 0003:00000174       __imp_??_7type_info@@6B@   00166174     coredll:COREDLL.dll
 0003:00000178       __imp_??0exception@std@@QAA@ABV01@@Z 00166178     coredll:COREDLL.dll
 0003:0000017c       __imp_??0exception@std@@QAA@XZ 0016617c     coredll:COREDLL.dll
 0003:00000180       __imp_GetTickCount         00166180     coredll:COREDLL.dll
 0003:00000184       __imp_wcsstr               00166184     coredll:COREDLL.dll
 0003:00000188       __imp_??_V@YAXPAX@Z        00166188     coredll:COREDLL.dll
 0003:0000018c       __imp_??_U@YAPAXI@Z        0016618c     coredll:COREDLL.dll
 0003:00000190       __imp_memset               00166190     coredll:COREDLL.dll
 0003:00000194       __imp_Sleep                00166194     coredll:COREDLL.dll
 0003:00000198       __imp__isctype             00166198     coredll:COREDLL.dll
 0003:0000019c       __imp_wcscpy               0016619c     coredll:COREDLL.dll
 0003:000001a0       __imp_wcslen               001661a0     coredll:COREDLL.dll
 0003:000001a4       __imp_memcpy               001661a4     coredll:COREDLL.dll
 0003:000001a8       __imp__wcsicmp             001661a8     coredll:COREDLL.dll
 0003:000001ac       __imp_NKDbgPrintfW         001661ac     coredll:COREDLL.dll
 0003:000001b0       __imp_CloseHandle          001661b0     coredll:COREDLL.dll
 0003:000001b4       __imp_InterlockedCompareExchange 001661b4     coredll:COREDLL.dll
 0003:000001b8       __imp_MultiByteToWideChar  001661b8     coredll:COREDLL.dll
 0003:000001bc       __imp_swprintf             001661bc     coredll:COREDLL.dll
 0003:000001c0       __imp_strchr               001661c0     coredll:COREDLL.dll
 0003:000001c4       __imp_CreateThread         001661c4     coredll:COREDLL.dll
 0003:000001c8       __imp_WriteFile            001661c8     coredll:COREDLL.dll
 0003:000001cc       __imp_PurgeComm            001661cc     coredll:COREDLL.dll
 0003:000001d0       __imp_SetCommMask          001661d0     coredll:COREDLL.dll
 0003:000001d4       __imp_SetCommTimeouts      001661d4     coredll:COREDLL.dll
 0003:000001d8       __imp_GetCommModemStatus   001661d8     coredll:COREDLL.dll
 0003:000001dc       __imp_SetCommState         001661dc     coredll:COREDLL.dll
 0003:000001e0       __imp_CreateFileW          001661e0     coredll:COREDLL.dll
 0003:000001e4       __imp_MessageBoxW          001661e4     coredll:COREDLL.dll
 0003:000001e8       __imp_ShowWindow           001661e8     coredll:COREDLL.dll
 0003:000001ec       __imp_FindWindowW          001661ec     coredll:COREDLL.dll
 0003:000001f0       __imp_strcat               001661f0     coredll:COREDLL.dll
 0003:000001f4       __imp_SetSystemPowerState  001661f4     coredll:COREDLL.dll
 0003:000001f8       __imp_wcscmp               001661f8     coredll:COREDLL.dll
 0003:000001fc       __imp_CreateProcessW       001661fc     coredll:COREDLL.dll
 0003:00000200       __imp_strcpy               00166200     coredll:COREDLL.dll
 0003:00000204       __imp_CreateMutexW         00166204     coredll:COREDLL.dll
 0003:00000208       __imp_wcscat               00166208     coredll:COREDLL.dll
 0003:0000020c       __imp_GetLastError         0016620c     coredll:COREDLL.dll
 0003:00000210       __imp_TerminateThread      00166210     coredll:COREDLL.dll
 0003:00000214       __imp_WaitForSingleObject  00166214     coredll:COREDLL.dll
 0003:00000218       __imp_DeviceIoControl      00166218     coredll:COREDLL.dll
 0003:0000021c       \177COREDLL_NULL_THUNK_DATA 0016621c     coredll:COREDLL.dll
 0003:00000220       __imp_?SwiM2MAV_AudioSetAVEC@CSwiGobiDll@@QAAKPAE0@Z 00166220     sdkril:SDKRIL.dll
 0003:00000224       __imp_?SwiM2MAV_AudioSetSTG@CSwiGobiDll@@QAAKPAEPAG@Z 00166224     sdkril:SDKRIL.dll
 0003:00000228       __imp_?SwiM2MAV_AudioSetVolume@CSwiGobiDll@@QAAKPAE00@Z 00166228     sdkril:SDKRIL.dll
 0003:0000022c       __imp_?SwiM2MAV_AudioSetAVNS@CSwiGobiDll@@QAAKPAE0@Z 0016622c     sdkril:SDKRIL.dll
 0003:00000230       __imp_?SwiM2MAV_AudioSetVolDB@CSwiGobiDll@@QAAKPAE00PAG@Z 00166230     sdkril:SDKRIL.dll
 0003:00000234       __imp_?PlayAudioTone@CSwiGobiDll@@QAAKPAEPAG@Z 00166234     sdkril:SDKRIL.dll
 0003:00000238       __imp_?SwiM2MAV_AudioPlayTone@CSwiGobiDll@@QAAKPAE0PAG@Z 00166238     sdkril:SDKRIL.dll
 0003:0000023c       __imp_?GetAudioProfile@CSwiGobiDll@@QAAKPAE@Z 0016623c     sdkril:SDKRIL.dll
 0003:00000240       __imp_?SetEchoCancelMode@CSwiGobiDll@@QAAKPAE@Z 00166240     sdkril:SDKRIL.dll
 0003:00000244       __imp_?SetNoiseSuppression@CSwiGobiDll@@QAAKPAE@Z 00166244     sdkril:SDKRIL.dll
 0003:00000248       __imp_?SetAutoInputGain@CSwiGobiDll@@QAAKPAE@Z 00166248     sdkril:SDKRIL.dll
 0003:0000024c       __imp_?SetAutoOutputGain@CSwiGobiDll@@QAAKPAE@Z 0016624c     sdkril:SDKRIL.dll
 0003:00000250       __imp_?SetTXPCMFilter@CSwiGobiDll@@QAAKPAG0PAK0@Z 00166250     sdkril:SDKRIL.dll
 0003:00000254       __imp_?SetRXPCMFilter@CSwiGobiDll@@QAAKPAG0PAK0@Z 00166254     sdkril:SDKRIL.dll
 0003:00000258       __imp_?SetRXGainLevel@CSwiGobiDll@@QAAKPAEPAG1@Z 00166258     sdkril:SDKRIL.dll
 0003:0000025c       __imp_?SetAudioProfile@CSwiGobiDll@@QAAKPAE@Z 0016625c     sdkril:SDKRIL.dll
 0003:00000260       __imp_?SetMICMuteStatus@CSwiGobiDll@@QAAKPAE@Z 00166260     sdkril:SDKRIL.dll
 0003:00000264       __imp_?SetSpeakerMuteStatus@CSwiGobiDll@@QAAKPAE@Z 00166264     sdkril:SDKRIL.dll
 0003:00000268       __imp_?SetMicVolume@CSwiGobiDll@@QAAKPAG@Z 00166268     sdkril:SDKRIL.dll
 0003:0000026c       __imp_?SetReceiverVolume@CSwiGobiDll@@QAAKPAE@Z 0016626c     sdkril:SDKRIL.dll
 0003:00000270       __imp_?SwiM2MAV_AudioGetProfile@CSwiGobiDll@@QAAKPAE000000@Z 00166270     sdkril:SDKRIL.dll
 0003:00000274       __imp_?SwiM2MAV_AudioSetTxVolume@CSwiGobiDll@@QAAKPAEPAG@Z 00166274     sdkril:SDKRIL.dll
 0003:00000278       __imp_?SwiM2MAV_AudioSetProfile@CSwiGobiDll@@QAAKPAE00000@Z 00166278     sdkril:SDKRIL.dll
 0003:0000027c       __imp_?CancelUSSD@CSwiGobiDll@@QAAKXZ 0016627c     sdkril:SDKRIL.dll
 0003:00000280       __imp_?AnswerUSSD@CSwiGobiDll@@QAAKPAUUSSInfo@@@Z 00166280     sdkril:SDKRIL.dll
 0003:00000284       __imp_?OrigUSSD@CSwiGobiDll@@QAAKPAUUSSInfo@@PAGPAUalphaIDInfo@@0PAE3PAUccSUPSType@@@Z 00166284     sdkril:SDKRIL.dll
 0003:00000288       __imp_?GetCallWaiting@CSwiGobiDll@@QAAKPAE0PAGPAUalphaIDInfo@@00PAUccSUPSType@@@Z 00166288     sdkril:SDKRIL.dll
 0003:0000028c       __imp_?GetCallForwarding@CSwiGobiDll@@QAAKPAE0PAUgetCallFWInfo@@0PAUalphaIDInfo@@00PAUccSUPSType@@PAUgetExtCallFWInfo@@@Z 0016628c     sdkril:SDKRIL.dll
 0003:00000290       __imp_?ChangeBarringPwd@CSwiGobiDll@@QAAKPAUcallBarringPwd@@PAGPAUalphaIDInfo@@PAE3PAUccSUPSType@@@Z 00166290     sdkril:SDKRIL.dll
 0003:00000294       __imp_?SetSUPS@CSwiGobiDll@@QAAKPAUvoiceSetSUPSServiceReq@@PAGPAUalphaIDInfo@@PAE3PAUccSUPSType@@@Z 00166294     sdkril:SDKRIL.dll
 0003:00000298       __imp_?GetCallBarring@CSwiGobiDll@@QAAKPAE00PAGPAUalphaIDInfo@@00PAUccSUPSType@@@Z 00166298     sdkril:SDKRIL.dll
 0003:0000029c       __imp_SwiGetGsmProfileBasic 0016629c     sdkril:SDKRIL.dll
 0003:000002a0       __imp_SwiSetGsmProfileBasic 001662a0     sdkril:SDKRIL.dll
 0003:000002a4       __imp_?GetWaitingMessage@CSwiGobiDll@@QAAKPAUwaitingMsgInfo@@@Z 001662a4     sdkril:SDKRIL.dll
 0003:000002a8       __imp_??0CSwiGobiDll@@QAA@XZ 001662a8     sdkril:SDKRIL.dll
 0003:000002ac       __imp_?Initialize@CSwiGobiDll@@QAA_NXZ 001662ac     sdkril:SDKRIL.dll
 0003:000002b0       __imp_??1CSwiGobiDll@@QAA@XZ 001662b0     sdkril:SDKRIL.dll
 0003:000002b4       __imp_?GetDormancyState@CSwiGobiDll@@QAAKPAK@Z 001662b4     sdkril:SDKRIL.dll
 0003:000002b8       __imp_?GetDunCallInfo@CSwiGobiDll@@QAAKPAKPAE101111PA_KPAG221100002221@Z 001662b8     sdkril:SDKRIL.dll
 0003:000002bc       __imp_?UIMGetCardStatus@CSwiGobiDll@@QAAKPAHPAUQMI_UIM_GET_CARD_STATUS_RESP@@@Z 001662bc     sdkril:SDKRIL.dll
 0003:000002c0       __imp_?GetRTREConfig@CSwiGobiDll@@QAAKPAE0@Z 001662c0     sdkril:SDKRIL.dll
 0003:000002c4       __imp_SwiSetPower          001662c4     sdkril:SDKRIL.dll
 0003:000002c8       __imp_?DeletePhonebookRecord@CSwiGobiDll@@QAAKPAEPAG1@Z 001662c8     sdkril:SDKRIL.dll
 0003:000002cc       __imp_?WritePhonebookRecord@CSwiGobiDll@@QAAKPAEPAG1000000@Z 001662cc     sdkril:SDKRIL.dll
 0003:000002d0       __imp_?ReadPhonebookRecords@CSwiGobiDll@@QAAKPAEPAG111@Z 001662d0     sdkril:SDKRIL.dll
 0003:000002d4       __imp_?GetPhonebookCapabilities@CSwiGobiDll@@QAAKPAEPAG1100@Z 001662d4     sdkril:SDKRIL.dll
 0003:000002d8       __imp_?SetNMEAConfig@CSwiGobiDll@@QAAKEEEPAG@Z 001662d8     sdkril:SDKRIL.dll
 0003:000002dc       __imp_?SetPDSDefaults@CSwiGobiDll@@QAAKKEKK@Z 001662dc     sdkril:SDKRIL.dll
 0003:000002e0       __imp_?SetXTRAEmbeddedClient@CSwiGobiDll@@QAAKEE@Z 001662e0     sdkril:SDKRIL.dll
 0003:000002e4       __imp_?GetCellLocationInfo@CSwiGobiDll@@QAAKPAUgeranCellInfo@@PAUumtsCellInfo@@PAUcdmaCellInfo@@PAK@Z 001662e4     sdkril:SDKRIL.dll
 0003:000002e8       __imp_SwiPstGetDsMipActiveProf 001662e8     sdkril:SDKRIL.dll
 0003:000002ec       __imp_?DialCall@CSwiGobiDll@@QAAKPAUtDialReqParam@@PAEPAUalphaIDInfo@@1PAUccSUPSType@@@Z 001662ec     sdkril:SDKRIL.dll
 0003:000002f0       __imp_?SendFlash@CSwiGobiDll@@QAAKPAEPAD00@Z 001662f0     sdkril:SDKRIL.dll
 0003:000002f4       __imp_?EndCall@CSwiGobiDll@@QAAKPAE0@Z 001662f4     sdkril:SDKRIL.dll
 0003:000002f8       __imp_?StartDTMF@CSwiGobiDll@@QAAKPAE00@Z 001662f8     sdkril:SDKRIL.dll
 0003:000002fc       __imp_?StopDTMF@CSwiGobiDll@@QAAKPAE0@Z 001662fc     sdkril:SDKRIL.dll
 0003:00000300       __imp_?ManageCalls@CSwiGobiDll@@QAAKPAE0PAG@Z 00166300     sdkril:SDKRIL.dll
 0003:00000304       __imp_?AnserCall@CSwiGobiDll@@QAAKPAE0@Z 00166304     sdkril:SDKRIL.dll
 0003:00000308       \177SDKRIL_NULL_THUNK_DATA 00166308     sdkril:SDKRIL.dll
 0003:0000030c       __imp_htonl                0016630c     winsock:WINSOCK.dll
 0003:00000310       \177WINSOCK_NULL_THUNK_DATA 00166310     winsock:WINSOCK.dll
 0003:00000314       __imp_PHGetFeatureLevel    00166314     ccoreutl:ccoreutl.dll
 0003:00000318       \177ccoreutl_NULL_THUNK_DATA 00166318     ccoreutl:ccoreutl.dll
 0003:0000031c       __imp_GetStatStore         0016631c     ossvcs:ossvcs.dll
 0003:00000320       __imp_ValidateAPIPermission 00166320     ossvcs:ossvcs.dll
 0003:00000324       \177ossvcs_NULL_THUNK_DATA 00166324     ossvcs:ossvcs.dll
 0003:00000328       __imp_?ChangeCarrierIndex@@YAJKK@Z 00166328     sw_utilityG:sw_utilityG.dll
 0003:0000032c       __imp_?LogV@@YAXPBGZZ      0016632c     sw_utilityG:sw_utilityG.dll
 0003:00000330       __imp_?GetVerInfo@@YAPAGPAUHINSTANCE__@@@Z 00166330     sw_utilityG:sw_utilityG.dll
 0003:00000334       __imp_?InitLog@@YAXPAUHINSTANCE__@@@Z 00166334     sw_utilityG:sw_utilityG.dll
 0003:00000338       __imp_?GetRegValue@@YAJPAUHKEY__@@PBG1AAK@Z 00166338     sw_utilityG:sw_utilityG.dll
 0003:0000033c       __imp_?SetRegValue@@YAJPAUHKEY__@@PBG11@Z 0016633c     sw_utilityG:sw_utilityG.dll
 0003:00000340       __imp_?GetProductFeatures@@YAHAAK@Z 00166340     sw_utilityG:sw_utilityG.dll
 0003:00000344       __imp_?SWAI_GetRegValue@@YAJPAUHKEY__@@PBG1PAGPAK@Z 00166344     sw_utilityG:sw_utilityG.dll
 0003:00000348       __imp_?SWAI_SetRegValue@@YAJPAUHKEY__@@PBG1K@Z 00166348     sw_utilityG:sw_utilityG.dll
 0003:0000034c       __imp_?SWAI_GetRegValue@@YAJPAUHKEY__@@PBG1AAK@Z 0016634c     sw_utilityG:sw_utilityG.dll
 0003:00000350       __imp_?SetRegValue@@YAJPAUHKEY__@@PBG1K@Z 00166350     sw_utilityG:sw_utilityG.dll
 0003:00000354       __imp_?DisplayRawData@@YAXIPAEHPBG@Z 00166354     sw_utilityG:sw_utilityG.dll
 0003:00000358       __imp_?ConvertPrefMode@@YAH_NH@Z 00166358     sw_utilityG:sw_utilityG.dll
 0003:0000035c       __imp_?GetProductVersionStr@CVerInfo@@QAAPAGXZ 0016635c     sw_utilityG:sw_utilityG.dll
 0003:00000360       __imp_??0CVerInfo@@QAA@PAG@Z 00166360     sw_utilityG:sw_utilityG.dll
 0003:00000364       __imp_?GetRegValue@@YAJPAUHKEY__@@PBG1PAGPAK@Z 00166364     sw_utilityG:sw_utilityG.dll
 0003:00000368       __imp_??1CVerInfo@@QAA@XZ  00166368     sw_utilityG:sw_utilityG.dll
 0003:0000036c       __imp_?SW_TtoA@@YAPADPADPAGK@Z 0016636c     sw_utilityG:sw_utilityG.dll
 0003:00000370       __imp_?LocalToUTCTime@@YAHPAU_SYSTEMTIME@@0@Z 00166370     sw_utilityG:sw_utilityG.dll
 0003:00000374       __imp_?IP2DWORD@@YAKPBG@Z  00166374     sw_utilityG:sw_utilityG.dll
 0003:00000378       __imp_?DWORD2IP@@YAPBGK@Z  00166378     sw_utilityG:sw_utilityG.dll
 0003:0000037c       __imp_?GetCarrierIndex@@YAKXZ 0016637c     sw_utilityG:sw_utilityG.dll
 0003:00000380       __imp_?GetDataPortDetails@@YAHPAGAAK@Z 00166380     sw_utilityG:sw_utilityG.dll
 0003:00000384       __imp_?SW_AtoT@@YAPAGPAGPADK@Z 00166384     sw_utilityG:sw_utilityG.dll
 0003:00000388       __imp_?TBD_Output@@YAXW4TBD_CLASS_TYPE@@W4TBD_OUTPUT_LEVEL@@QBGZZ 00166388     sw_utilityG:sw_utilityG.dll
 0003:0000038c       __imp_?TBD_Assert@@YA_N_NQBG1H@Z 0016638c     sw_utilityG:sw_utilityG.dll
 0003:00000390       __imp_?LogC@@YAXPBGZZ      00166390     sw_utilityG:sw_utilityG.dll
 0003:00000394       __imp_?LogStoreFileLine@@YAXPAGH@Z 00166394     sw_utilityG:sw_utilityG.dll
 0003:00000398       \177sw_utilityG_NULL_THUNK_DATA 00166398     sw_utilityG:sw_utilityG.dll
 0003:0000039c       __xc_a                     0016639c     corelibc:crt0init.obj
 0003:000003b0       __xc_z                     001663b0     corelibc:crt0init.obj
 0003:000003b4       __xi_a                     001663b4     corelibc:crt0init.obj
 0003:000003b8       __xi_z                     001663b8     corelibc:crt0init.obj
 0003:000003bc       __xp_a                     001663bc     corelibc:crt0init.obj
 0003:000003c0       __xp_z                     001663c0     corelibc:crt0init.obj
 0003:000003c4       __xt_a                     001663c4     corelibc:crt0init.obj
 0003:000003c8       __xt_z                     001663c8     corelibc:crt0init.obj
 0003:00000a70       ??_R0?AVbad_alloc@std@@@8  00166a70     atcmd.obj
 0003:00000a8c       ??_R0?AVexception@std@@@8  00166a8c     atcmd.obj
 0003:00000aa8       ??_R0?AVlength_error@std@@@8 00166aa8     atcmd.obj
 0003:00000ac8       ??_R0?AVlogic_error@std@@@8 00166ac8     atcmd.obj
 0003:0000256c       ??_R0?AVout_of_range@std@@@8 0016856c     DatERI.obj
 0003:00002c2c       ?g_bRadioOff@@3HA          00168c2c     FakeResponse.obj
 0003:00002c30       ?bSingleInitThreadProc@@3_NA 00168c30     FakeResponse.obj
 0003:000046b8       ?csReceiveSms@@3VCriticalSection@@A 0016a6b8     msg.obj
 0003:00004d70       ?Convert2CDMANetworkPref@@3PAW4CDMA_NETWORK_PREF@@A 0016ad70     network.obj
 0003:00004d7c       ?Convert2UMTSNetworkPref@@3PAW4UMTS_NETWORK_PREF@@A 0016ad7c     network.obj
 0003:00005428       ?g_IsOSExpectNITZ@@3HA     0016b428     Radio.obj
 0003:0000542c       ?RIL_CALLSTAT_STR@@3PAPAGA 0016b42c     Radio.obj
 0003:00005448       ?theSWINotifCR@@3VCriticalSection@@A 0016b448     Radio.obj
 0003:00006ee0       ?g_IsFirstSend@@3HA        0016cee0     rilhandndis.obj
 0003:00006ee8       ?dhcpIpFrameReq@@3PAEA     0016cee8     rilhandndis.obj
 0003:000076d0       ?gIsPowerManagedSupported@@3HA 0016d6d0     rilmain.obj
 0003:000086f8       ?smscbsample@@3PADA        0016e6f8     smscb.obj
 0003:00009ae0       __security_cookie_complement 0016fae0     corelibc:seccook.obj
 0003:00009ae4       __security_cookie          0016fae4     corelibc:seccook.obj
 0003:00009af0       ?g_pCmdQ@@3PAV?$CThreadSafeQueue@PAVCCommand@@@@A 0016faf0     atcmd.obj
 0003:00009af4       ?m_pChannelLinker@ChannelLinker@@2PAV1@A 0016faf4     channel.obj
 0003:00009af8       ?g_IsCriticalPowerCondition@@3HA 0016faf8     misc.obj
 0003:00009afc       ?g_nMsgID@@3KA             0016fafc     msg.obj
 0003:00009b00       ?g_dwDelayNITZ@@3KA        0016fb00     Radio.obj
 0003:00009b04       ?g_TimeoutAPIDefault@@3KA  0016fb04     rilhand.obj
 0003:00009b08       ?g_TimeoutCmdInit@@3KA     0016fb08     rilhand.obj
 0003:00009b0c       ?g_dwPhoneFeatureLevel@@3KA 0016fb0c     rilhand.obj
 0003:00009b10       ?g_dwNetworkType@@3KA      0016fb10     rilhand.obj
 0003:00009b14       ?g_TimeoutWaitForInit@@3KA 0016fb14     rilhand.obj
 0003:00009b18       ?g_TimeoutCmdOnline@@3KA   0016fb18     rilhand.obj
 0003:00009b1c       ?g_TimeoutCmdNoOp@@3KA     0016fb1c     rilhand.obj
 0003:00009b20       ?g_TimeoutDTRDrop@@3KA     0016fb20     rilhand.obj
 0003:00009b24       ?g_pNotifQ@@3PAV?$CThreadSafeQueue@PAUSwiNotifyVariant@@@@A 0016fb24     rilhand.obj
 0003:00009b28       ?g_GlobalRILHandle@@3PAVCRilHandle@@A 0016fb28     rilhand.obj
 0003:00009b2c       ?g_arrWaitingCommands@@3V?$list@PAVCCommand@@V?$allocator@PAVCCommand@@@std@@@std@@A 0016fb2c     rilhand.obj
 0003:00009b38       ?g_tszUserDNS2@@3PAGA      0016fb38     rilhandndis.obj
 0003:00009bb8       ?g_tszUserDNS1@@3PAGA      0016fbb8     rilhandndis.obj
 0003:00009c38       ?g_pIPChannel@@3PAVCChannel@@A 0016fc38     rilhandndis.obj
 0003:00009c3c       ?g_NDISGetFnPtr@@3URILNDISGETFNPTR@@A 0016fc3c     rilhandndis.obj
 0003:00009c44       ?g_hSWUSBNDISEvent@@3PAXA  0016fc44     rilhandndis.obj
 0003:00009c48       ?g_csClosing@@3UCRITICAL_SECTION@@A 0016fc48     rilmain.obj
 0003:00009c5c       ?g_hCriticalErrorEvent@@3PAXA 0016fc5c     rilmain.obj
 0003:00009c60       ?g_hDriverPresentEvent@@3PAXA 0016fc60     rilmain.obj
 0003:00009c64       ?g_dwReadyState@@3KA       0016fc64     rilmain.obj
 0003:00009c68       ?g_dwLastError@@3KA        0016fc68     rilmain.obj
 0003:00009c6c       ?g_hinstDll@@3PAXA         0016fc6c     rilmain.obj
 0003:00009c70       ?g_SignalCriticalErrorEventId@@3KA 0016fc70     rilmain.obj
 0003:00009c74       ?g_hDeviceJustResumedEvent@@3PAXA 0016fc74     rilmain.obj
 0003:00009c78       ?g_CriticalLogging@@3HA    0016fc78     rilmain.obj
 0003:00009c7c       ?gLastDeviceDx@@3W4_CEDEVICE_POWER_STATE@@A 0016fc7c     rilmain.obj
 0003:00009c80       __onexitend                0016fc80     <common>
 0003:00009c84       __onexitbegin              0016fc84     <common>
 0003:00009c88       _exitflag                  0016fc88     <common>
 0003:00009c8c       _pRawDllMain               0016fc8c     <common>

 entry point at        0001:0003d1e8

 Static symbols

 0001:00000758       __catch$85883              00101758 f i atcmd.obj
 0001:00000784       __catch$85881              00101784 f i atcmd.obj
 0001:00000ad0       __unwind$86798             00101ad0 f i atcmd.obj
 0001:00000c78       __unwind$87069             00101c78 f i atcmd.obj
 0001:00000cf8       __unwind$87134             00101cf8 f i atcmd.obj
 0001:0000154c       __unwind$88163             0010254c f   atcmd.obj
 0001:00001564       __unwind$88164             00102564 f   atcmd.obj
 0001:00001950       __unwind$86034             00102950 f   callctrl.obj
 0001:00001eac       __unwind$86194             00102eac f   callctrl.obj
 0001:000020ec       __unwind$86295             001030ec f   callctrl.obj
 0001:00002278       __unwind$86378             00103278 f   callctrl.obj
 0001:00002430       __unwind$86421             00103430 f   callctrl.obj
 0001:000024ec       __unwind$86475             001034ec f   callctrl.obj
 0001:000029e8       __unwind$86777             001039e8 f   callctrl.obj
 0001:00002b54       __unwind$86806             00103b54 f   callctrl.obj
 0001:00003138       __unwind$86997             00104138 f   callctrl.obj
 0001:0000340c       __unwind$87138             0010440c f   callctrl.obj
 0001:00003660       __unwind$87220             00104660 f   callctrl.obj
 0001:00003d48       __unwind$87270             00104d48 f   callctrl.obj
 0001:00004184       __unwind$87347             00105184 f   callctrl.obj
 0001:00004300       __unwind$87444             00105300 f   callctrl.obj
 0001:0000459c       __unwind$87485             0010559c f   callctrl.obj
 0001:000046bc       __unwind$87543             001056bc f   callctrl.obj
 0001:00005600       __unwind$87793             00106600 f   callctrl.obj
 0001:00005970       __unwind$87917             00106970 f   callctrl.obj
 0001:00005c8c       __unwind$87990             00106c8c f   callctrl.obj
 0001:00005ec4       __unwind$88104             00106ec4 f   callctrl.obj
 0001:0000754c       __unwind$88438             0010854c f   callctrl.obj
 0001:0000755c       __unwind$88439             0010855c f   callctrl.obj
 0001:00008f7c       __unwind$83617             00109f7c f   command.obj
 0001:0000b514       __unwind$43483             0010c514 f i DatERI.obj
 0001:0000b9a8       __unwind$44074             0010c9a8 f i DatERI.obj
 0001:0000bd08       __unwind$44836             0010cd08 f i DatERI.obj
 0001:0000c068       __unwind$45452             0010d068 f i DatERI.obj
 0001:0000c8bc       __unwind$48192             0010d8bc f   DatERI.obj
 0001:0000c8d8       __unwind$48193             0010d8d8 f   DatERI.obj
 0001:0000cb04       __unwind$48757             0010db04 f   DatERI.obj
 0001:0000cb20       __unwind$48758             0010db20 f   DatERI.obj
 0001:0000dcc0       __unwind$87652             0010ecc0 f   FakeResponse.obj
 0001:0000e144       __unwind$89818             0010f144 f i FakeResponse.obj
 0001:0000e274       __unwind$90828             0010f274 f   FakeResponse.obj
 0001:0000e6e8       __unwind$91183             0010f6e8 f   FakeResponse.obj
 0001:0000f390       __unwind$84495             00110390 f   gprs.obj
 0001:0000f3a0       __unwind$84496             001103a0 f   gprs.obj
 0001:000115c8       __unwind$87483             001125c8 f   misc.obj
 0001:00013590       __unwind$88131             00114590 f   misc.obj
 0001:000176f0       __unwind$89463             001186f0 f   misc.obj
 0001:0001771c       __unwind$89464             0011871c f   misc.obj
 0001:00017740       __unwind$89465             00118740 f   misc.obj
 0001:0001776c       __unwind$89466             0011876c f   misc.obj
 0001:00017798       __unwind$89467             00118798 f   misc.obj
 0001:000177c4       __unwind$89468             001187c4 f   misc.obj
 0001:000177f0       __unwind$89469             001187f0 f   misc.obj
 0001:0001781c       __unwind$89470             0011881c f   misc.obj
 0001:00017bfc       __unwind$91760             00118bfc f i misc.obj
 0001:000180d4       __unwind$93002             001190d4 f i misc.obj
 0001:000180ec       __unwind$93003             001190ec f i misc.obj
 0001:00018300       __unwind$93840             00119300 f   misc.obj
 0001:00018318       __unwind$93841             00119318 f   misc.obj
 0001:00018664       __unwind$83214             00119664 f   monitor.obj
 0001:00019034       __unwind$85523             0011a034 f   msg.obj
 0001:0001a0b0       __unwind$85979             0011b0b0 f   msg.obj
 0001:0001a8e4       __unwind$86073             0011b8e4 f   msg.obj
 0001:0001b36c       __unwind$86268             0011c36c f   msg.obj
 0001:0001c44c       __unwind$86443             0011d44c f   msg.obj
 0001:0001cd90       __unwind$84732             0011dd90 f   network.obj
 0001:0001d8c8       __unwind$84956             0011e8c8 f   network.obj
 0001:0001e338       __unwind$85244             0011f338 f   network.obj
 0001:0001eab4       __unwind$85342             0011fab4 f   network.obj
 0001:0001eb10       ?BSCompareOperatorNames@@YAHPBX0@Z 0011fb10 f   Radio.obj
 0001:0001f608       __unwind$89336             00120608 f   Radio.obj
 0001:0002048c       __unwind$89682             0012148c f   Radio.obj
 0001:0002221c       __unwind$95524             0012321c f   Radio.obj
 0001:00022234       __unwind$95525             00123234 f   Radio.obj
 0001:0002224c       __unwind$95526             0012324c f   Radio.obj
 0001:00022264       __unwind$95527             00123264 f   Radio.obj
 0001:0002227c       __unwind$95530             0012327c f   Radio.obj
 0001:00022294       __unwind$95528             00123294 f   Radio.obj
 0001:000222ac       __unwind$95529             001232ac f   Radio.obj
 0001:000222c4       __unwind$95531             001232c4 f   Radio.obj
 0001:000222dc       __unwind$95532             001232dc f   Radio.obj
 0001:000227c0       __unwind$96418             001237c0 f i Radio.obj
 0001:00022c34       __unwind$97006             00123c34 f i Radio.obj
 0001:00022cb4       __unwind$97528             00123cb4 f i Radio.obj
 0001:00023114       __unwind$98177             00124114 f i Radio.obj
 0001:00023888       __unwind$100812            00124888 f   Radio.obj
 0001:000238a0       __unwind$100813            001248a0 f   Radio.obj
 0001:000238c8       __unwind$100814            001248c8 f   Radio.obj
 0001:000238e8       __unwind$100815            001248e8 f   Radio.obj
 0001:00023904       __unwind$100816            00124904 f   Radio.obj
 0001:00023924       __unwind$100817            00124924 f   Radio.obj
 0001:00023d48       __unwind$100956            00124d48 f   Radio.obj
 0001:00024170       __unwind$101672            00125170 f   Radio.obj
 0001:00024180       __unwind$101673            00125180 f   Radio.obj
 0001:00026870       __unwind$101869            00127870 f   Radio.obj
 0001:00026888       __unwind$101875            00127888 f   Radio.obj
 0001:000268a0       __unwind$101882            001278a0 f   Radio.obj
 0001:000268b8       __unwind$101883            001278b8 f   Radio.obj
 0001:000268d0       __unwind$101881            001278d0 f   Radio.obj
 0001:000268e8       __unwind$101876            001278e8 f   Radio.obj
 0001:00026900       __unwind$101868            00127900 f   Radio.obj
 0001:00026918       __unwind$101867            00127918 f   Radio.obj
 0001:00026930       __unwind$101880            00127930 f   Radio.obj
 0001:00026948       __unwind$101884            00127948 f   Radio.obj
 0001:00026960       __unwind$101878            00127960 f   Radio.obj
 0001:00026978       __unwind$101879            00127978 f   Radio.obj
 0001:00026990       __unwind$101885            00127990 f   Radio.obj
 0001:000269a8       __unwind$101877            001279a8 f   Radio.obj
 0001:000269c0       __unwind$101886            001279c0 f   Radio.obj
 0001:000269d8       __unwind$101870            001279d8 f   Radio.obj
 0001:000269f0       __unwind$101872            001279f0 f   Radio.obj
 0001:00026a08       __unwind$101871            00127a08 f   Radio.obj
 0001:00026a20       __unwind$101874            00127a20 f   Radio.obj
 0001:00026cc4       __unwind$102327            00127cc4 f   Radio.obj
 0001:00026cdc       __unwind$102328            00127cdc f   Radio.obj
 0001:00026d04       __unwind$102329            00127d04 f   Radio.obj
 0001:00026d24       __unwind$102330            00127d24 f   Radio.obj
 0001:00026d40       __unwind$102331            00127d40 f   Radio.obj
 0001:00026d60       __unwind$102332            00127d60 f   Radio.obj
 0001:00027900       __unwind$88237             00128900 f   rilhand.obj
 0001:00027928       __unwind$88238             00128928 f   rilhand.obj
 0001:00027948       __unwind$88239             00128948 f   rilhand.obj
 0001:00027a58       __unwind$88367             00128a58 f   rilhand.obj
 0001:00027c64       __unwind$88406             00128c64 f   rilhand.obj
 0001:00028544       __unwind$88894             00129544 f i rilhand.obj
 0001:00028668       __unwind$88955             00129668 f i rilhand.obj
 0001:000287dc       __unwind$89027             001297dc f i rilhand.obj
 0001:00029088       __unwind$89828             0012a088 f i rilhand.obj
 0001:00029d78       __unwind$90993             0012ad78 f   rilhand.obj
 0001:00029d90       __unwind$90995             0012ad90 f   rilhand.obj
 0001:00029da8       __unwind$90996             0012ada8 f   rilhand.obj
 0001:00029dc0       __unwind$90997             0012adc0 f   rilhand.obj
 0001:00029dd8       __unwind$90994             0012add8 f   rilhand.obj
 0001:00029df0       __unwind$90998             0012adf0 f   rilhand.obj
 0001:0002a110       __unwind$91441             0012b110 f   rilhand.obj
 0001:0002a378       __unwind$91871             0012b378 f   rilhand.obj
 0001:0002a43c       __unwind$91920             0012b43c f   rilhand.obj
 0001:0002c674       __unwind$92825             0012d674 f   rilhand.obj
 0001:0002c918       __unwind$92902             0012d918 f   rilhand.obj
 0001:0002c940       __unwind$92903             0012d940 f   rilhand.obj
 0001:0002c960       __unwind$92904             0012d960 f   rilhand.obj
 0001:0002c980       __unwind$92905             0012d980 f   rilhand.obj
 0001:0002cda4       __unwind$93016             0012dda4 f   rilhand.obj
 0001:0002cdbc       __unwind$93017             0012ddbc f   rilhand.obj
 0001:0002ea68       __unwind$86776             0012fa68 f   rilhandndis.obj
 0001:0002ee84       __unwind$88042             0012fe84 f i rilhandndis.obj
 0001:00030560       __unwind$86342             00131560 f i rilmain.obj
 0001:00030754       __unwind$86393             00131754 f   rilmain.obj
 0001:000308a4       __unwind$86449             001318a4 f   rilmain.obj
 0001:000308b4       __unwind$86450             001318b4 f   rilmain.obj
 0001:00033168       __unwind$87184             00134168 f   rilmain.obj
 0001:00035d90       ?ParseCellBroadcastDCS@@YAHEAAUrilmsgdcs_tag@@AAI@Z 00136d90 f   smscb.obj
 0001:0003afb0       __unwind$84208             0013bfb0 f   voice.obj
 0001:0003d410       doexit                     0013e410 f   corelibc:crt0dat.obj
 0001:0003ddac       __unwind$17778             0013edac f   libcpmt:string.obj
 0001:0003de3c       __unwind$17968             0013ee3c f   libcpmt:string.obj
 0001:0003e268       ?CanThisExceptionObjectBeDestructed@@YAEPAUEHExceptionRecord@@E@Z 0013f268 f   LIBCMT:frame_ce.obj
 0001:0003e5b4       ?CallCatchBlock@@YAPAXPAUEHExceptionRecord@@PAKPAU_CONTEXT@@PBU_s_FuncInfo@@PAXHK@Z 0013f5b4 f   LIBCMT:frame_ce.obj
 0001:0003e94c       ?BuildCatchObject@@YAXPAUEHExceptionRecord@@PAKPBU_s_HandlerType@@PBU_s_CatchableType@@@Z 0013f94c f   LIBCMT:frame_ce.obj
 0001:0003eb20       ?FindHandler@@YAEPAUEHExceptionRecord@@PAKPAU_CONTEXT@@PAU_DISPATCHER_CONTEXT@@PBU_s_FuncInfo@@H@Z 0013fb20 f   LIBCMT:frame_ce.obj
 0001:0003f49c       ??__EcsReceiveSms@@YAXXZ   0014049c f   msg.obj
 0001:0003f4c0       ??__EtheSWINotifCR@@YAXXZ  001404c0 f   Radio.obj
 0001:0003f4e4       ??__Eg_arrWaitingCommands@@YAXXZ 001404e4 f   rilhand.obj
 0001:0003f518       ??__FcsReceiveSms@@YAXXZ   00140518 f   msg.obj
 0001:0003f534       ??__FtheSWINotifCR@@YAXXZ  00140534 f   Radio.obj
 0001:0003f550       ??__Fg_arrWaitingCommands@@YAXXZ 00140550 f   rilhand.obj
